 MFC42u_original

 Timestamp is 35889ac7 (Wed Jun 17 21:42:47 1998)

 Preferred load address is 5f800000

 Start         Length     Name                   Class
 0001:00000000 0009738dH .text                   CODE
 0002:00000000 000357f8H .rdata                  DATA
 0003:00000000 00008674H .data                   DATA
 0004:00000000 0000a300H .rsrc                   DATA
 0005:00000000 0000edb4H .reloc                  DATA

  Address         Publics by Value              Rva+Base   Lib:Object

 0001:00000000       __EH_prolog                5f801000 f
 0001:00000006       ?GetData@CThreadLocalObject@@QAEPAVCNoTrackObject@@P6GPAV2@XZ@Z 5f801006 f
 0001:00000083       ?AfxGetModuleState@@YGPAVAFX_MODULE_STATE@@XZ 5f801083 f
 0001:000000ab       ?GetData@CProcessLocalObject@@QAEPAVCNoTrackObject@@P6GPAV2@XZ@Z 5f8010ab f
 0001:000000f8       ?AfxGetThread@@YGPAVCWinThread@@XZ 5f8010f8 f
 0001:00000109       ?AfxGetModuleThreadState@@YGPAVAFX_MODULE_THREAD_STATE@@XZ 5f801109 f
 0001:00000120       ?AfxGetMainWnd@@YGPAVCWnd@@XZ 5f801120 f
 0001:00000135       ?GetMainWnd@CWinThread@@UAEPAVCWnd@@XZ 5f801135 f
 0001:00000152       ?FromHandle@CWnd@@SGPAV1@PAUHWND__@@@Z 5f801152 f
 0001:00000179       ?afxMapHWND@@YGPAVCHandleMap@@H@Z 5f801179 f
 0001:000001ed       ?FromHandle@CHandleMap@@QAEPAVCObject@@PAX@Z 5f8011ed f
 0001:0000029d       ?AttachControlSite@CWnd@@IAEXPAVCHandleMap@@@Z 5f80129d f
 0001:000002d2       ?GetValueAt@CMapPtrToPtr@@QBEPAXPAX@Z 5f8012d2 f
 0001:00000305       ?FromHandlePermanent@CWnd@@SGPAV1@PAUHWND__@@@Z 5f801305 f
 0001:00000320       ?GetTopLevelParent@CWnd@@QBEPAV1@XZ 5f801320 f
 0001:00000348       ?AfxGetParentOwner@@YGPAUHWND__@@PAU1@@Z 5f801348 f
 0001:0000038f       ?GetOwner@CWnd@@QBEPAV1@XZ 5f80138f f
 0001:000003a6       ?PumpMessage@CWinThread@@UAEHXZ 5f8013a6 f
 0001:000003e6       ?PreTranslateMessage@CWinThread@@UAEHPAUtagMSG@@@Z 5f8013e6 f
 0001:0000043d       ?WalkPreTranslateTree@CWnd@@SGHPAUHWND__@@PAUtagMSG@@@Z 5f80143d f
 0001:0000047f       ?IsIdleMessage@CWinThread@@UAEHPAUtagMSG@@@Z 5f80147f f
 0001:000004ef       ?PreTranslateMessage@CWnd@@UAEHPAUtagMSG@@@Z 5f8014ef f
 0001:00000508       ?PreTranslateMessage@CFrameWnd@@UAEHPAUtagMSG@@@Z 5f801508 f
 0001:0000057a       ?_FilterToolTipMessage@CWnd@@SGXPAUtagMSG@@PAV1@@Z 5f80157a f
 0001:0000058a       ?FilterToolTipMessage@CWnd@@QAEXPAUtagMSG@@@Z 5f80158a f
 0001:00000667       ?AfxLockGlobals@@YGXH@Z    5f801667 f
 0001:000006d8       ?AfxUnlockGlobals@@YGXH@Z  5f8016d8 f
 0001:000006f9       ??0AFX_MAINTAIN_STATE2@@QAE@PAVAFX_MODULE_STATE@@@Z 5f8016f9 f
 0001:00000720       ?AfxWndProcBase@@YGJPAUHWND__@@IIJ@Z 5f801720 f
 0001:00000770       ?AfxWndProc@@YGJPAUHWND__@@IIJ@Z 5f801770 f
 0001:0000079e       ?AfxCallWndProc@@YGJPAVCWnd@@PAUHWND__@@IIJ@Z 5f80179e f
 0001:00000867       ?WindowProc@CWnd@@MAEJIIJ@Z 5f801867 f
 0001:000008ab       ?OnWndMsg@CWnd@@MAEHIIJPAJ@Z 5f8018ab f
 0001:00000c27       ?DefWindowProcW@CWnd@@MAEJIIJ@Z 5f801c27 f
 0001:00000c50       ?Default@CWnd@@IAEJXZ      5f801c50 f
 0001:00000c50       ?OnPaint@CCtrlView@@IAEXXZ 5f801c50 f
 0001:00000c77       ?GetTopLevelFrame@CWnd@@QBEPAVCFrameWnd@@XZ 5f801c77 f
 0001:00000cbe       ?GetParentFrame@CWnd@@QBEPAVCFrameWnd@@XZ 5f801cbe f
 0001:00000dc0       ?OnCreateAggregates@CCmdTarget@@UAEHXZ 5f801dc0 f
 0001:00000dc4       ?_AfxHandleSetCursor@@YGHPAVCWnd@@II@Z 5f801dc4 f
 0001:00000dfe       ?OnSetCursor@CFrameWnd@@IAEHPAVCWnd@@II@Z 5f801dfe f
 0001:00000e1b       ?AfxGetThreadState@@YGPAV_AFX_THREAD_STATE@@XZ 5f801e1b f
 0001:00000e2b       _memset                    5f801e2b f
 0001:00000e31       ??0CCmdTarget@@QAE@XZ      5f801e31 f
 0001:00000e7b       ??0CWnd@@QAE@XZ            5f801e7b f
 0001:00000e9d       ?_GetBaseInterfaceMap@CCmdTarget@@KGPBUAFX_INTERFACEMAP@@XZ 5f801e9d f
 0001:00000ea0       ?Alloc@CFixedAlloc@@QAEPAXXZ 5f801ea0 f
 0001:00000f19       ?Free@CFixedAlloc@@QAEXPAX@Z 5f801f19 f
 0001:00000f45       ?AfxFindMessageEntry@@YGPBUAFX_MSGMAP_ENTRY@@PBU1@III@Z 5f801f45 f
 0001:00000f85       ?_GetBaseMessageMap@CWnd@@KGPBUAFX_MSGMAP@@XZ 5f801f85 f
 0001:00000f8b       ?OnCmdMsg@CCmdTarget@@UAEHIHPAXPAUAFX_CMDHANDLERINFO@@@Z 5f801f8b f
 0001:00001008       ?_AfxDispatchCmdMsg@@YGHPAVCCmdTarget@@IHP81@AEXXZPAXIPAUAFX_CMDHANDLERINFO@@@Z 5f802008 f
 0001:000010a0       ??0CCmdUI@@QAE@XZ          5f8020a0 f
 0001:000010c6       ??0CString@@QAE@XZ         5f8020c6 f
 0001:000010d6       ?AfxGetEmptyString@@YGABVCString@@XZ 5f8020d6 f
 0001:000010dc       ?AllocBuffer@CString@@IAEXH@Z 5f8020dc f
 0001:0000115b       _memcpy                    5f80215b f
 0001:00001161       ?GetBuffer@CString@@QAEPAGH@Z 5f802161 f
 0001:000011b3       ??1CString@@QAE@XZ         5f8021b3 f
 0001:000011dd       ?Release@CString@@KGXPAUCStringData@@@Z 5f8021dd f
 0001:00001202       ?ReleaseBuffer@CString@@QAEXH@Z 5f802202 f
 0001:0000122b       ?CopyBeforeWrite@CString@@IAEXXZ 5f80222b f
 0001:0000123e       ?FreeData@CString@@KIXPAUCStringData@@@Z 5f80223e f
 0001:00001286       ?AfxDynamicDownCast@@YAPAVCObject@@PAUCRuntimeClass@@PAV1@@Z 5f802286 f
 0001:000012ab       ?IsKindOf@CObject@@QBEHPBUCRuntimeClass@@@Z 5f8022ab f
 0001:000012bd       ?IsDerivedFrom@CRuntimeClass@@QBEHPBU1@@Z 5f8022bd f
 0001:000012d8       ?_GetBaseMessageMap@CCheckListBox@@KGPBUAFX_MSGMAP@@XZ 5f8022d8 f
 0001:000012de       ?WindowProc@CControlBar@@UAEJIIJ@Z 5f8022de f
 0001:0000133d       ?GetMessageMap@CStatusBar@@MBEPBUAFX_MSGMAP@@XZ 5f80233d f
 0001:00001343       ?OnCmdMsg@CFrameWnd@@UAEHIHPAXPAUAFX_CMDHANDLERINFO@@@Z 5f802343 f
 0001:000013eb       ?GetActiveView@CFrameWnd@@QBEPAVCView@@XZ 5f8023eb f
 0001:000013f2       ?_GetBaseMessageMap@CCtrlView@@KGPBUAFX_MSGMAP@@XZ 5f8023f2 f
 0001:000013f8       ?_GetBaseMessageMap@CView@@KGPBUAFX_MSGMAP@@XZ 5f8023f8 f
 0001:000013fe       ?_GetBaseClass@COleObjectFactory@@KGPAUCRuntimeClass@@XZ 5f8023fe f
 0001:00001404       ?OnCmdMsg@CView@@UAEHIHPAXPAUAFX_CMDHANDLERINFO@@@Z 5f802404 f
 0001:00001481       ?OnCmdMsg@COleDocument@@UAEHIHPAXPAUAFX_CMDHANDLERINFO@@@Z 5f802481 f
 0001:000014c8       ?OnCmdMsg@CDocument@@UAEHIHPAXPAUAFX_CMDHANDLERINFO@@@Z 5f8024c8 f
 0001:0000150b       ?_GetBaseMessageMap@COleServerDoc@@KGPBUAFX_MSGMAP@@XZ 5f80250b f
 0001:00001511       ?_GetBaseMessageMap@CDocument@@KGPBUAFX_MSGMAP@@XZ 5f802511 f
 0001:00001517       ?OnCmdMsg@CDocTemplate@@UAEHIHPAXPAUAFX_CMDHANDLERINFO@@@Z 5f802517 f
 0001:0000154e       ?GetRuntimeClass@COleObjectFactory@@UBEPAUCRuntimeClass@@XZ 5f80254e f
 0001:00001554       ?GetActiveDocument@CFrameWnd@@UAEPAVCDocument@@XZ 5f802554 f
 0001:00001564       ?DoUpdate@CCmdUI@@QAEHPAVCCmdTarget@@H@Z 5f802564 f
 0001:000015c7       ?GetMessageMap@CToolBar@@MBEPBUAFX_MSGMAP@@XZ 5f8025c7 f
 0001:000015cd       ?_GetBaseMessageMap@CStatusBar@@KGPBUAFX_MSGMAP@@XZ 5f8025cd f
 0001:000015d3       ?_GetBaseMessageMap@CControlBar@@KGPBUAFX_MSGMAP@@XZ 5f8025d3 f
 0001:000015d9       ?GetMessageMap@CDockBar@@MBEPBUAFX_MSGMAP@@XZ 5f8025d9 f
 0001:000015df       ?GetFirstViewPosition@CDocument@@UBEPAU__POSITION@@XZ 5f8025df f
 0001:000015e3       ?GetNextView@CDocument@@UBEPAVCView@@AAPAU__POSITION@@@Z 5f8025e3 f
 0001:000015f7       ?_GetBaseMessageMap@CRichEditView@@KGPBUAFX_MSGMAP@@XZ 5f8025f7 f
 0001:000015fd       ?GetDefaultAccelerator@CFrameWnd@@UAEPAUHACCEL__@@XZ 5f8025fd f
 0001:00001623       ?GetDefaultAccelerator@COleServerDoc@@MAEPAUHACCEL__@@XZ 5f802623 f
 0001:00001647       ?GetStyle@CWnd@@QBEKXZ     5f802647 f
 0001:00001677       ??1CWnd@@UAE@XZ            5f802677 f
 0001:000016eb       ??1CCmdTarget@@UAE@XZ      5f8026eb f
 0001:0000172c       ?SendChildNotifyLastMsg@CWnd@@QAEHPAJ@Z 5f80272c f
 0001:00001759       ?OnChildNotify@CWnd@@MAEHIIJPAJ@Z 5f802759 f
 0001:0000177d       ?ReflectChildNotify@CWnd@@IAEHIIJPAJ@Z 5f80277d f
 0001:00001861       ?ReflectLastMsg@CWnd@@KGHPAUHWND__@@PAJ@Z 5f802861 f
 0001:000018c9       ?SendMessageToDescendants@CWnd@@SGXPAUHWND__@@IIJHH@Z 5f8028c9 f
 0001:00001948       ?GetBufferSetLength@CString@@QAEPAGH@Z 5f802948 f
 0001:00001969       ?GetWindowTextW@CWnd@@QBEXAAVCString@@@Z 5f802969 f
 0001:000019a7       ?GetFirstDocPosition@CSingleDocTemplate@@UBEPAU__POSITION@@XZ 5f8029a7 f
 0001:000019af       ?GetNextDoc@CSingleDocTemplate@@UBEPAVCDocument@@AAPAU__POSITION@@@Z 5f8029af f
 0001:000019c3       ?OnIdle@CWinApp@@UAEHJ@Z   5f8029c3 f
 0001:00001a2d       ?OnIdle@CWinThread@@UAEHJ@Z 5f802a2d f
 0001:00001b30       ?FreeDataChain@CPlex@@QAEXXZ 5f802b30 f
 0001:00001b48       ?RemoveAll@CMapWordToOb@@QAEXXZ 5f802b48 f
 0001:00001b75       ?AfxOleTermOrFreeLib@@YGXHH@Z 5f802b75 f
 0001:00001bbd       ?DeleteTemp@CHandleMap@@QAEXXZ 5f802bbd f
 0001:00001c26       ?OnCommand@CWnd@@MAEHIJ@Z  5f802c26 f
 0001:00001cbf       ?OnCommand@CFrameWnd@@MAEHIJ@Z 5f802cbf f
 0001:00001cee       ?AfxLockTempMaps@@YGXXZ    5f802cee f
 0001:00001cf7       ?AfxUnlockTempMaps@@YGHH@Z 5f802cf7 f
 0001:00001dde       ?OnKeyDown@CRichEditView@@IAEXIII@Z 5f802dde f
 0001:00001dfd       ?GetParaFormat@CRichEditCtrl@@QBEKAAU_paraformat@@@Z 5f802dfd f
 0001:00001e1b       ?OnSelChange@CRichEditView@@IAEXPAUtagNMHDR@@PAJ@Z 5f802e1b f
 0001:00001e34       ?GetSelectionCharFormat@CRichEditCtrl@@QBEKAAU_charformat@@@Z 5f802e34 f
 0001:00001e52       ?GetStartPosition@COleDocument@@UBEPAU__POSITION@@XZ 5f802e52 f
 0001:00001e56       ?GetNextItemOfKind@COleDocument@@IBEPAVCDocItem@@AAPAU__POSITION@@PAUCRuntimeClass@@@Z 5f802e56 f
 0001:00001e70       ?GetNextServerItem@COleDocument@@QBEPAVCOleServerItem@@AAPAU__POSITION@@@Z 5f802e70 f
 0001:00001e81       ?GetStartPosition@CRichEditDoc@@UBEPAU__POSITION@@XZ 5f802e81 f
 0001:00001e9a       ?UpdateAllItems@COleServerDoc@@QAEXPAVCOleServerItem@@JPAVCObject@@W4tagDVASPECT@@@Z 5f802e9a f
 0001:00001ec4       ?OnIdleUpdateCmdUI@CControlBar@@QAEJIJ@Z 5f802ec4 f
 0001:00001f57       ?OnUpdateCmdUI@CStatusBar@@UAEXPAVCFrameWnd@@H@Z 5f802f57 f
 0001:00001fcb       ?OnUpdateKeyIndicator@CFrameWnd@@IAEXPAVCCmdUI@@@Z 5f802fcb f
 0001:00002013       ?Enable@CStatusCmdUI@@UAEXH@Z 5f803013 f
 0001:0000204c       ?GetPaneStyle@CStatusBar@@QBEIH@Z 5f80304c f
 0001:0000205d       ?SetPaneStyle@CStatusBar@@QAEXHI@Z 5f80305d f
 0001:000020a9       ?UpdateDialogControls@CWnd@@QAEXPAVCCmdTarget@@H@Z 5f8030a9 f
 0001:00002194       ?OnUpdateCmdUI@CDockBar@@MAEXPAVCFrameWnd@@H@Z 5f803194 f
 0001:00002197       ?OnUpdateCmdUI@CToolBar@@UAEXPAVCFrameWnd@@H@Z 5f803197 f
 0001:00002243       ?_GetButton@CToolBar@@IBEXHPAU_TBBUTTON@@@Z 5f803243 f
 0001:00002262       ?Enable@CToolCmdUI@@UAEXH@Z 5f803262 f
 0001:000022a2       ?GetButtonStyle@CToolBar@@QBEIH@Z 5f8032a2 f
 0001:000022c5       ?SetButtonStyle@CToolBar@@QAEXHI@Z 5f8032c5 f
 0001:00002314       ?SetCheck@CToolCmdUI@@UAEXH@Z 5f803314 f
 0001:00002355       ?OnIdleUpdateCmdUI@CFrameWnd@@IAEXXZ 5f803355 f
 0001:0000239b       ?GetFirstDocTemplatePosition@CDocManager@@UBEPAU__POSITION@@XZ 5f80339b f
 0001:0000239f       ?GetNextDocTemplate@CDocManager@@UBEPAVCDocTemplate@@AAPAU__POSITION@@@Z 5f80339f f
 0001:000023af       ?OnIdle@CDocTemplate@@UAEXXZ 5f8033af f
 0001:000023e0       ?OnIdle@COleDocument@@UAEXXZ 5f8033e0 f
 0001:00002436       ?GetScrollBarCtrl@CView@@UBEPAVCScrollBar@@H@Z 5f803436 f
 0001:0000246d       ?GetParentSplitter@CView@@SGPAVCSplitterWnd@@PBVCWnd@@H@Z 5f80346d f
 0001:000024a6       ?_GetBaseClass@CStatic@@KGPAUCRuntimeClass@@XZ 5f8034a6 f
 0001:000024ac       ?_GetBaseClass@CPtrList@@KGPAUCRuntimeClass@@XZ 5f8034ac f
 0001:000024b2       ?GetScrollPos@CWnd@@QBEHH@Z 5f8034b2 f
 0001:000024d7       ?OnNotify@CWnd@@MAEHIJPAJ@Z 5f8034d7 f
 0001:00002551       ?OnUpdateCharBold@CRichEditView@@IAEXPAVCCmdUI@@@Z 5f803551 f
 0001:00002561       ?OnUpdateCharEffect@CRichEditView@@QAEXPAVCCmdUI@@KK@Z 5f803561 f
 0001:00002597       ?GetCharFormatSelection@CRichEditView@@QAEAAU_charformat@@XZ 5f803597 f
 0001:000025c4       ?OnUpdateCharItalic@CRichEditView@@IAEXPAVCCmdUI@@@Z 5f8035c4 f
 0001:000025d4       ?OnUpdateCharUnderline@CRichEditView@@IAEXPAVCCmdUI@@@Z 5f8035d4 f
 0001:000025e4       ?OnUpdateParaLeft@CRichEditView@@IAEXPAVCCmdUI@@@Z 5f8035e4 f
 0001:000025f2       ?OnUpdateParaAlign@CRichEditView@@QAEXPAVCCmdUI@@G@Z 5f8035f2 f
 0001:00002639       ?GetParaFormatSelection@CRichEditView@@QAEAAU_paraformat@@XZ 5f803639 f
 0001:00002666       ?OnUpdateParaCenter@CRichEditView@@IAEXPAVCCmdUI@@@Z 5f803666 f
 0001:00002674       ?OnUpdateParaRight@CRichEditView@@IAEXPAVCCmdUI@@@Z 5f803674 f
 0001:00002682       ?OnUpdateBullet@CRichEditView@@IAEXPAVCCmdUI@@@Z 5f803682 f
 0001:000026ae       ?GetDlgCtrlID@CWnd@@QBEHXZ 5f8036ae f
 0001:000026c3       ?AfxA2WHelper@@YGPAGPAGPBDH@Z 5f8036c3 f
 0001:000026ec       ?OnUpdateNeedText@CRichEditView@@IAEXPAVCCmdUI@@@Z 5f8036ec f
 0001:00002710       ?OnUpdateNeedSel@CRichEditView@@IAEXPAVCCmdUI@@@Z 5f803710 f
 0001:0000273b       ?GetSel@CRichEditCtrl@@QBEXAAJ0@Z 5f80373b f
 0001:00002768       ?OnUpdateNeedClip@CRichEditView@@IAEXPAVCCmdUI@@@Z 5f803768 f
 0001:0000277f       ?CanPaste@CRichEditView@@QBEHXZ 5f80377f f
 0001:000027a9       ?OnUpdateEditUndo@CEditView@@IAEXPAVCCmdUI@@@Z 5f8037a9 f
 0001:000027c7       ??2@YAPAXI@Z               5f8037c7 f
 0001:000027f0       ?AfxSetNewHandler@@YGP6AHI@ZP6AHI@Z@Z 5f8037f0 f
 0001:00002804       ??ACMapPtrToPtr@@QAEAAPAXPAX@Z 5f803804 f
 0001:00002856       ?GetAssocAt@CMapPtrToWord@@IBEPAUCAssoc@1@PAXAAI@Z 5f803856 f
 0001:00002888       ?NewAssoc@CMapPtrToPtr@@IAEPAUCAssoc@1@XZ 5f803888 f
 0001:000028d5       ?Create@CPlex@@SGPAU1@AAPAU1@II@Z 5f8038d5 f
 0001:000028f5       ?_AfxCbtFilterHook@@YGJHIJ@Z 5f8038f5 f
 0001:00002a44       ?CreateObject@CRuntimeClass@@QAEPAVCObject@@XZ 5f803a44 f
 0001:00002a7c       ?InitHashTable@CMapWordToOb@@QAEXIH@Z 5f803a7c f
 0001:00002aba       ?CreateObject@CTempWnd@@SGPAVCObject@@XZ 5f803aba f
 0001:00002afa       ?AfxLoadString@@YGHIPAGI@Z 5f803afa f
 0001:00002c3a       ??4CString@@QAEABV0@PBG@Z  5f803c3a f
 0001:00002c61       ?AssignCopy@CString@@IAEXHPBG@Z 5f803c61 f
 0001:00002c94       ?AllocBeforeWrite@CString@@IAEXH@Z 5f803c94 f
 0001:00002cbd       ?SetWindowTextW@CWnd@@QAEXPBG@Z 5f803cbd f
 0001:00002d05       ?Release@CString@@IAEXXZ   5f803d05 f
 0001:00002d17       ?Empty@CString@@QAEXXZ     5f803d17 f
 0001:00002d20       ?SetMessageText@CFrameWnd@@QAEXI@Z 5f803d20 f
 0001:00002d37       ??0CString@@QAE@PBG@Z      5f803d37 f
 0001:00002d87       ?_AfxMsgFilterHook@@YGJHIJ@Z 5f803d87 f
 0001:00002dc0       ?ProcessMessageFilter@CWinThread@@UAEHHPAUtagMSG@@@Z 5f803dc0 f
 0001:00002e43       ?FromHandle@CMenu@@SGPAV1@PAUHMENU__@@@Z 5f803e43 f
 0001:00002e58       ?afxMapHMENU@@YGPAVCHandleMap@@H@Z 5f803e58 f
 0001:00002ecc       ?CreateObject@CTempMenu@@SGPAVCObject@@XZ 5f803ecc f
 0001:00002ee9       ?OnEnterIdle@CWnd@@IAEXIPAV1@@Z 5f803ee9 f
 0001:00002f21       ??1CDC@@UAE@XZ             5f803f21 f
 0001:00002f63       ?afxMapHGDIOBJ@@YGPAVCHandleMap@@H@Z 5f803f63 f
 0001:00002fd7       ??0CDC@@QAE@XZ             5f803fd7 f
 0001:00002feb       ?_GetBaseMessageMap@CDialog@@KGPBUAFX_MSGMAP@@XZ 5f803feb f
 0001:00002ff1       ?GetSuperWndProcAddr@CWnd@@MAEPAP6GJPAUHWND__@@IIJ@ZXZ 5f803ff1 f
 0001:00002ff5       ?_AfxHandleActivate@@YGXPAVCWnd@@I0@Z 5f803ff5 f
 0001:00003056       ?PostNcDestroy@CWnd@@MAEXXZ 5f804056 f
 0001:00003057       ?SetWindowPos@CWnd@@QAEHPBV1@HHHHI@Z 5f804057 f
 0001:0000308e       ??0CString@@QAE@ABV0@@Z    5f80408e f
 0001:000030b5       ?ConcatCopy@CString@@IAEXHPBGH0@Z 5f8040b5 f
 0001:000030f6       ?AfxGetFileName@@YGIPBGPAGI@Z 5f8040f6 f
 0001:00003149       ?UpdateAllPanes@CStatusBar@@IAEXHH@Z 5f804149 f
 0001:00003291       ?SetPaneText@CStatusBar@@QAEHHPBGH@Z 5f804291 f
 0001:00003347       ?OnSetMessageString@CFrameWnd@@IAEJIJ@Z 5f804347 f
 0001:0000340a       ?GetMessageBar@CFrameWnd@@UAEPAVCWnd@@XZ 5f80440a f
 0001:0000341a       ?GetDescendantWindow@CWnd@@SGPAV1@PAUHWND__@@HH@Z 5f80441a f
 0001:00003494       ?OnPaint@CStatusBar@@IAEXXZ 5f804494 f
 0001:000034a9       ?GetMessageString@CFrameWnd@@UBEXIAAVCString@@@Z 5f8044a9 f
 0001:000034f1       ?OnSetText@CStatusBar@@IAEJIJ@Z 5f8044f1 f
 0001:0000351c       ?CommandToIndex@CStatusBar@@QBEHI@Z 5f80451c f
 0001:00003545       ?IsTracking@CFrameWnd@@QBEHXZ 5f804545 f
 0001:00003564       ?OnMenuSelect@CFrameWnd@@IAEXIIPAUHMENU__@@@Z 5f804564 f
 0001:0000365f       ?OnSysCommand@CFrameWnd@@IAEXIJ@Z 5f80465f f
 0001:00003688       ?OnInitMenu@CFrameWnd@@IAEXPAVCMenu@@@Z 5f804688 f
 0001:000036a1       ?OnInitMenuPopup@CFrameWnd@@IAEXPAVCMenu@@IH@Z 5f8046a1 f
 0001:000037c5       ?AfxCancelModes@@YGXPAUHWND__@@@Z 5f8047c5 f
 0001:00003813       ?_AfxIsComboBoxControl@@YGHPAUHWND__@@I@Z 5f804813 f
 0001:0000383c       ?OnEnterIdle@CFrameWnd@@IAEXIPAVCWnd@@@Z 5f80483c f
 0001:0000386d       ?AfxGetFileTitle@@YGIPBGPAGI@Z 5f80486d f
 0001:000038aa       _GetFileTitleW@12          5f8048aa f
 0001:000038b0       ?OnActivateFrame@CView@@MAEXIPAVCFrameWnd@@@Z 5f8048b0 f
 0001:000038b3       ?OnNcActivate@CFrameWnd@@IAEHH@Z 5f8048b3 f
 0001:000038ec       ?IsWindowEnabled@CWnd@@QBEHXZ 5f8048ec f
 0001:00003901       ?OnActivate@CFrameWnd@@IAEXIPAVCWnd@@H@Z 5f804901 f
 0001:000039db       ?NotifyFloatingWindows@CFrameWnd@@QAEXK@Z 5f8049db f
 0001:00003a73       ?AfxIsDescendant@@YGHPAUHWND__@@0@Z 5f804a73 f
 0001:00003a91       ?OnActivateView@CView@@MAEXHPAV1@0@Z 5f804a91 f
 0001:00003ab1       ?OnParentNotify@CWnd@@IAEXIJ@Z 5f804ab1 f
 0001:00003ae0       ?AfxGlobalFree@@YGXPAX@Z   5f804ae0 f
 0001:00003b18       ?OnDeleteItem@CWnd@@IAEXHPAUtagDELETEITEMSTRUCT@@@Z 5f804b18 f
 0001:00003b38       ?OnChangedRect@CRectTracker@@UAEXABVCRect@@@Z 5f804b38 f
 0001:00003b3b       ?SetSize@CDWordArray@@QAEXHH@Z 5f804b3b f
 0001:00003c55       ?SetAtGrow@CDWordArray@@QAEXHK@Z 5f804c55 f
 0001:00003c7c       ?OnChildNotify@CComboBox@@MAEHIIJPAJ@Z 5f804c7c f
 0001:00003ccc       ?OnUpdateFileExit@COleServerDoc@@IAEXPAVCCmdUI@@@Z 5f804ccc f
 0001:00003cdd       ?UpdateUsingHostObj@COleServerDoc@@IAEXIPAVCCmdUI@@@Z 5f804cdd f
 0001:00003d07       ??0CTestCmdUI@@QAE@XZ      5f804d07 f
 0001:00003d20       ?Enable@CCmdUI@@UAEXH@Z    5f804d20 f
 0001:00003d5d       ?OnUpdateRecentFileMenu@CWinApp@@IAEXPAVCCmdUI@@@Z 5f804d5d f
 0001:00003d77       ?UpdateMenu@CRecentFileList@@UAEXPAVCCmdUI@@@Z 5f804d77 f
 0001:00003fbe       ?GetDisplayName@CRecentFileList@@QBEHAAVCString@@HPBGHH@Z 5f804fbe f
 0001:000040cb       ??H@YG?AVCString@@ABV0@0@Z 5f8050cb f
 0001:00004131       ?_AfxAbbreviateName@@YGXPAGHH@Z 5f805131 f
 0001:00004165       ?OnUpdateFileSendMail@CDocument@@IAEXPAVCCmdUI@@@Z 5f805165 f
 0001:000041d9       ?OnCancelEditCntr@CRichEditView@@IAEXXZ 5f8051d9 f
 0001:000041e3       ??3@YAXPAX@Z               5f8051e3 f
 0001:000041ef       ?ShowWindow@CWnd@@QAEHH@Z  5f8051ef f
 0001:0000420a       ?DeleteObject@CGdiObject@@QAEHXZ 5f80520a f
 0001:00004220       ?RemoveKey@CMapPtrToWord@@QAEHPAX@Z 5f805220 f
 0001:00004262       ?FreeAssoc@CMapWordToOb@@IAEXPAUCAssoc@1@@Z 5f805262 f
 0001:0000427d       ?DestroyWindow@CWnd@@UAEHXZ 5f80527d f
 0001:000042c3       ?Detach@CWnd@@QAEPAUHWND__@@XZ 5f8052c3 f
 0001:000042f0       ?GetNextAssoc@CMapPtrToPtr@@QBEXAAPAU__POSITION@@AAPAX1@Z 5f8052f0 f
 0001:00004364       ??_GCTempWnd@@UAEPAXI@Z    5f805364 f
 0001:00004364       ??_ECTempWnd@@UAEPAXI@Z    5f805364 f
 0001:00004384       ??_GCTempMenu@@UAEPAXI@Z   5f805384 f
 0001:00004384       ??_ECTempMenu@@UAEPAXI@Z   5f805384 f
 0001:000043a4       ??1CTempMenu@@UAE@XZ       5f8053a4 f
 0001:000043d7       ?DestroyMenu@CMenu@@QAEHXZ 5f8053d7 f
 0001:000043e4       ?RemoveAll@CObList@@QAEXXZ 5f8053e4 f
 0001:00004404       ??1CPtrList@@UAE@XZ        5f805404 f
 0001:00004437       ?afxMapHDC@@YGPAVCHandleMap@@H@Z 5f805437 f
 0001:000044ab       ?Detach@CDC@@QAEPAUHDC__@@XZ 5f8054ab f
 0001:000044db       ?ReleaseAttribDC@CDC@@UAEXXZ 5f8054db f
 0001:000044e0       _RawDllMain@12             5f8054e0 f
 0001:0000459f       ?OnDestroy@CWnd@@IAEXXZ    5f80559f f
 0001:000045ba       ?OnNcDestroy@CWnd@@IAEXXZ  5f8055ba f
 0001:000046af       ?AfxUnhookWindowCreate@@YGHXZ 5f8056af f
 0001:000046cf       ?SetFocus@CWnd@@QAEPAV1@XZ 5f8056cf f
 0001:000046ea       ?_mbstowcsz@@YAHPAGPBDI@Z  5f8056ea f
 0001:0000471b       ??YCString@@QAEABV0@ABV0@@Z 5f80571b f
 0001:00004733       ?ConcatInPlace@CString@@IAEXHPBG@Z 5f805733 f
 0001:00004797       ?IsTopParentActive@CWnd@@QBEHXZ 5f805797 f
 0001:000047cb       ?OnSetFocus@CFrameWnd@@IAEXPAVCWnd@@@Z 5f8057cb f
 0001:000047e6       __DllMainCRTStartup@12     5f8057e6 f
 0001:00004888       ?CreateObject@?$CThreadLocal@V_AFX_THREAD_STATE@@@@SGPAVCNoTrackObject@@XZ 5f805888 f
 0001:000048bc       ??2CNoTrackObject@@SGPAXI@Z 5f8058bc f
 0001:000048d9       ??0_AFX_THREAD_STATE@@QAE@XZ 5f8058d9 f
 0001:000048f0       ?SetValue@CThreadSlotData@@QAEXHPAX@Z 5f8058f0 f
 0001:000049d8       ?AddHead@CSimpleList@@QAEXPAX@Z 5f8059d8 f
 0001:000049eb       __CRT_INIT@12              5f8059eb f
 0001:00004aa1       ??0CMapPtrToPtr@@QAE@H@Z   5f805aa1 f
 0001:00004ac8       ?CreateObject@?$CThreadLocal@VAFX_MODULE_THREAD_STATE@@@@SGPAVCNoTrackObject@@XZ 5f805ac8 f
 0001:00004afc       ??0AFX_MODULE_THREAD_STATE@@QAE@XZ 5f805afc f
 0001:00004b61       ??0CPtrList@@QAE@H@Z       5f805b61 f
 0001:00004b84       _DllMain@12                5f805b84 f
 0001:00004d0b       __imp_load__OleInitialize@4 5f805d0b f
 0001:00004d12       __tailMerge_ole32          5f805d12 f
 0001:00004d20       ___delayLoadHelper@8       5f805d20 f
 0001:00004e31       ?ExternalAddRef@CCmdTarget@@QAEKXZ 5f805e31 f
 0001:00004e47       ?InternalQueryInterface@CCmdTarget@@QAEKPBXPAPAX@Z 5f805e47 f
 0001:00004e89       ?GetInterface@CCmdTarget@@QAEPAUIUnknown@@PBX@Z 5f805e89 f
 0001:00004f3d       ?SetOccDialogInfo@CWnd@@MAEHPAU_AFX_OCC_DIALOG_INFO@@@Z 5f805f3d f
 0001:00004f62       ?ExternalRelease@CCmdTarget@@QAEKXZ 5f805f62 f
 0001:00004f6d       ?InternalRelease@CCmdTarget@@QAEKXZ 5f805f6d f
 0001:00004fa7       ?QueryAggregates@CCmdTarget@@QAEPAUIUnknown@@PBX@Z 5f805fa7 f
 0001:00004fe1       ?_GetBaseInterfaceMap@COleLinkingDoc@@KGPBUAFX_INTERFACEMAP@@XZ 5f805fe1 f
 0001:00004fe7       ?ExternalQueryInterface@CCmdTarget@@QAEKPBXPAPAX@Z 5f805fe7 f
 0001:00005002       ?_AfxGetOleModuleState@@YGPAVAFX_MODULE_STATE@@XZ 5f806002 f
 0001:00005008       ?AfxSetModuleState@@YGPAVAFX_MODULE_STATE@@PAV1@@Z 5f806008 f
 0001:00005026       ?OnActivateTopLevel@CWnd@@IAEJIJ@Z 5f806026 f
 0001:0000504a       ?AfxDeleteObject@@YGXPAPAX@Z 5f80604a f
 0001:00005065       ?CancelToolTips@CWnd@@SGXH@Z 5f806065 f
 0001:00005094       ?AfxOleGetUserCtrl@@YGHXZ  5f806094 f
 0001:0000509d       __imp_load__CoTaskMemFree@4 5f80609d f
 0001:000050a9       __imp_load__RegCloseKey@4  5f8060a9 f
 0001:000050b0       __tailMerge_ADVAPI32       5f8060b0 f
 0001:000050be       ??0CPtrArray@@QAE@XZ       5f8060be f
 0001:000050d5       ?ScreenToClient@CWnd@@QBEXPAUtagRECT@@@Z 5f8060d5 f
 0001:0000510d       ?UpdateFrameCounts@CDocument@@UAEXXZ 5f80610d f
 0001:000051fa       ?Revoke@COleLinkingDoc@@QAEXXZ 5f8061fa f
 0001:0000525e       ?_AfxRelease@@YGKPAPAUIUnknown@@@Z 5f80625e f
 0001:0000527a       ?GetNextClientItem@COleDocument@@QBEPAVCOleClientItem@@AAPAU__POSITION@@@Z 5f80627a f
 0001:0000528b       ?DeleteContents@COleServerDoc@@UAEXXZ 5f80628b f
 0001:000052fa       ?DeleteContents@COleDocument@@UAEXXZ 5f8062fa f
 0001:00005326       ?Detach@CGdiObject@@QAEPAXXZ 5f806326 f
 0001:0000534f       ?IsVisible@CControlBar@@UBEHXZ 5f80634f f
 0001:00005372       ?UpdateVisibleLock@COleLinkingDoc@@IAEXHH@Z 5f806372 f
 0001:000053ae       ?LockExternal@COleLinkingDoc@@IAEXHH@Z 5f8063ae f
 0001:000053f4       ?GetInterfaceHook@COleServerDoc@@MAEPAUIUnknown@@PBX@Z 5f8063f4 f
 0001:00005417       ?GetInterfaceMap@COleServerDoc@@MBEPBUAFX_INTERFACEMAP@@XZ 5f806417 f
 0001:0000541d       ?QueryInterface@XPersistStorage@COleServerDoc@@UAGJABU_GUID@@PAPAX@Z 5f80641d f
 0001:00005437       ?_GetBaseInterfaceMap@COleServerDoc@@KGPBUAFX_INTERFACEMAP@@XZ 5f806437 f
 0001:0000543d       ?Release@XPersistStorage@COleServerDoc@@UAGKXZ 5f80643d f
 0001:0000544f       ?AddTail@CPtrList@@QAEPAU__POSITION@@PAX@Z 5f80644f f
 0001:00005478       ?NewNode@CObList@@IAEPAUCNode@1@PAU21@0@Z 5f806478 f
 0001:000054d0       ?GetExStyle@CWnd@@QBEKXZ   5f8064d0 f
 0001:000054e7       ?OnShowWindow@CWnd@@IAEXHI@Z 5f8064e7 f
 0001:000054ef       ?AllocElements@CStatusBar@@QAEHHH@Z 5f8064ef f
 0001:00005554       ?AllocElements@CControlBar@@QAEHHH@Z 5f806554 f
 0001:0000558f       ?OnChangedViewList@CDocument@@UAEXXZ 5f80658f f
 0001:000055a7       ?GetDockedControlBar@CDockBar@@IBEPAVCControlBar@@H@Z 5f8065a7 f
 0001:000055c3       ?SetActiveView@CFrameWnd@@QAEXPAVCView@@H@Z 5f8065c3 f
 0001:00005613       ?OnActivateTopLevel@CFrameWnd@@IAEJIJ@Z 5f806613 f
 0001:0000568d       ?ExitHelpMode@CFrameWnd@@UAEXXZ 5f80668d f
 0001:000056a5       ?IsDockBar@CControlBar@@UBEHXZ 5f8066a5 f
 0001:000056a8       ?IsDockBar@CDockBar@@UBEHXZ 5f8066a8 f
 0001:000056ac       ?Remove@CSimpleList@@QAEHPAX@Z 5f8066ac f
 0001:000056d4       ?DeleteValues@CThreadSlotData@@QAEXPAUCThreadData@@PAUHINSTANCE__@@@Z 5f8066d4 f
 0001:00005771       ??_E_AFX_THREAD_STATE@@UAEPAXI@Z 5f806771 f
 0001:00005771       ??_G_AFX_THREAD_STATE@@UAEPAXI@Z 5f806771 f
 0001:0000578c       ??1_AFX_THREAD_STATE@@UAE@XZ 5f80678c f
 0001:000057f6       ??3CNoTrackObject@@SGXPAX@Z 5f8067f6 f
 0001:0000580a       ??_EAFX_MODULE_THREAD_STATE@@UAEPAXI@Z 5f80680a f
 0001:0000580a       ??_GAFX_MODULE_THREAD_STATE@@UAEPAXI@Z 5f80680a f
 0001:00005825       ??1AFX_MODULE_THREAD_STATE@@UAE@XZ 5f806825 f
 0001:000058f7       ??1CMapPtrToPtr@@UAE@XZ    5f8068f7 f
 0001:0000592a       ??_G_AFX_DB_STATE@@UAEPAXI@Z 5f80692a f
 0001:0000592a       ??_E_AFX_DB_STATE@@UAEPAXI@Z 5f80692a f
 0001:00005945       ??1_AFX_DB_STATE@@UAE@XZ   5f806945 f
 0001:00005946       ?GetDataNA@CThreadLocalObject@@QAEPAVCNoTrackObject@@XZ 5f806946 f
 0001:00005973       ??1CWinThread@@UAE@XZ      5f806973 f
 0001:000059c4       ?DeleteValues@CThreadSlotData@@QAEXPAUHINSTANCE__@@H@Z 5f8069c4 f
 0001:00005a1d       ??1CHandleMap@@QAE@XZ      5f806a1d f
 0001:00005a5e       ??_G_AFX_CTL3D_THREAD@@UAEPAXI@Z 5f806a5e f
 0001:00005a5e       ??_E_AFX_CTL3D_THREAD@@UAEPAXI@Z 5f806a5e f
 0001:00005a79       ??1_AFX_CTL3D_THREAD@@UAE@XZ 5f806a79 f
 0001:00005ab1       ?SaveModified@COleServerDoc@@MAEHXZ 5f806ab1 f
 0001:00005aca       ?SaveModified@COleDocument@@UAEHXZ 5f806aca f
 0001:00005b06       ?SaveModified@CDocument@@UAEHXZ 5f806b06 f
 0001:00005b32       ??0CFile@@QAE@XZ           5f806b32 f
 0001:00005b72       ??0CArchive@@QAE@PAVCFile@@IHPAX@Z 5f806b72 f
 0001:00005c4a       ?GetFilePath@CFile@@UBE?AVCString@@XZ 5f806c4a f
 0001:00005c8a       ??0CFileStatus@@QAE@XZ     5f806c8a f
 0001:00005ca6       ??0CTimeSpan@@QAE@XZ       5f806ca6 f
 0001:00005ca9       ?GetStatus@CFile@@QBEHAAUCFileStatus@@@Z 5f806ca9 f
 0001:00005d8a       ?Close@CArchive@@QAEXXZ    5f806d8a f
 0001:00005d98       ?Flush@CArchive@@QAEXXZ    5f806d98 f
 0001:00005dfd       ??1CArchive@@QAE@XZ        5f806dfd f
 0001:00005e3c       ?Abort@CArchive@@QAEXXZ    5f806e3c f
 0001:00005e7a       ??1CFile@@UAE@XZ           5f806e7a f
 0001:00005eca       ?BeginWaitCursor@CCmdTarget@@QAEXXZ 5f806eca f
 0001:00005edf       ?DoWaitCursor@CWinApp@@UAEXH@Z 5f806edf f
 0001:00005f3e       ?EndWaitCursor@CCmdTarget@@QAEXXZ 5f806f3e f
 0001:00005f53       ?GetView@CRichEditDoc@@UBEPAVCRichEditView@@XZ 5f806f53 f
 0001:00005f92       ?IsModified@CRichEditDoc@@UAEHXZ 5f806f92 f
 0001:00005fad       ?DeleteContents@CRichEditDoc@@UAEXXZ 5f806fad f
 0001:0000601a       ?UpdateModifiedFlag@CRichEditDoc@@UAEXXZ 5f80701a f
 0001:0000601b       ?GetLength@CFile@@UBEKXZ   5f80701b f
 0001:00006048       ?GetSectionKey@CWinApp@@QAEPAUHKEY__@@PBG@Z 5f807048 f
 0001:0000608e       ?GetAppRegistryKey@CWinApp@@QAEPAUHKEY__@@XZ 5f80708e f
 0001:00006125       ??0CMemFile@@QAE@I@Z       5f807125 f
 0001:00006155       ?GrowFile@CMemFile@@MAEXK@Z 5f807155 f
 0001:000061ac       ?Alloc@CMemFile@@MAEPAEK@Z 5f8071ac f
 0001:000061ba       ?Memcpy@CMemFile@@MAEPAEPAEPBEI@Z 5f8071ba f
 0001:000061df       ?Seek@CMemFile@@UAEJJI@Z   5f8071df f
 0001:0000621d       ?GetBufferPtr@CMemFile@@UAEIIIPAPAX0@Z 5f80721d f
 0001:000062c1       ?Serialize@CDockState@@UAEXAAVCArchive@@@Z 5f8072c1 f
 0001:000063e3       ?Clear@CDockState@@QAEXXZ  5f8073e3 f
 0001:0000641f       ??1CMemFile@@UAE@XZ        5f80741f f
 0001:0000646b       ?Close@CMemFile@@UAEXXZ    5f80746b f
 0001:00006495       ?Free@CMemFile@@MAEXPAE@Z  5f807495 f
 0001:000064a3       ??0CControlBarInfo@@QAE@XZ 5f8074a3 f
 0001:000064f1       ?Serialize@CControlBarInfo@@QAEXAAVCArchive@@PAVCDockState@@@Z 5f8074f1 f
 0001:000066e8       ?GetVersion@CDockState@@QAEKXZ 5f8076e8 f
 0001:000066ec       ?AfxSetWindowText@@YGXPAUHWND__@@PBG@Z 5f8076ec f
 0001:00006746       ?UpdateFrameTitleForDocument@CFrameWnd@@QAEXPBG@Z 5f807746 f
 0001:00006803       ??0AFX_EXCEPTION_LINK@@QAE@XZ 5f807803 f
 0001:00006819       ?AfxGetExceptionContext@@YAPAUAFX_EXCEPTION_CONTEXT@@XZ 5f807819 f
 0001:00006841       ?AfxTryCleanup@@YGXXZ      5f807841 f
 0001:0000685e       ?CommonConstruct@CWinThread@@QAEXXZ 5f80785e f
 0001:00006890       ?AfxInitThread@@YGXXZ      5f807890 f
 0001:000068e8       ?CreateObject@?$CThreadLocal@V_AFX_CTL3D_THREAD@@@@SGPAVCNoTrackObject@@XZ 5f8078e8 f
 0001:000068fe       ??0CHandleMap@@QAE@PAUCRuntimeClass@@IH@Z 5f8078fe f
 0001:0000695a       ?AfxOleSetUserCtrl@@YGXH@Z 5f80795a f
 0001:00006969       ??0CException@@QAE@XZ      5f807969 f
 0001:00006979       ?_AfxActivationWndProc@@YGJPAUHWND__@@IIJ@Z 5f807979 f
 0001:000069fd       ?Run@CWinApp@@UAEHXZ       5f8079fd f
 0001:00006a1d       ?Run@CWinThread@@UAEHXZ    5f807a1d f
 0001:00006aa0       ?AfxExtractSubString@@YGHAAVCString@@PBGHG@Z 5f807aa0 f
 0001:00006b16       ?CalcInsideRect@CControlBar@@QBEXAAVCRect@@H@Z 5f807b16 f
 0001:00006bbe       ?SelectObject@CDC@@QAEPAVCPen@@PAV2@@Z 5f807bbe f
 0001:00006bfd       ?OnInitialUpdate@CControlBar@@QAEXXZ 5f807bfd f
 0001:00006c07       ?_SetButton@CToolBar@@IAEXHPAU_TBBUTTON@@@Z 5f807c07 f
 0001:00006cfb       ?ModifyStyle@CWnd@@QAEHKKI@Z 5f807cfb f
 0001:00006d1e       ?ModifyStyle@CWnd@@SGHPAUHWND__@@KKI@Z 5f807d1e f
 0001:00006d38       ?_AfxModifyStyle@@YGHPAUHWND__@@HKKI@Z 5f807d38 f
 0001:00006d89       ?DragAcceptFiles@CWnd@@QAEXH@Z 5f807d89 f
 0001:00006d99       ?GetDocString@CDocTemplate@@UBEHAAVCString@@W4DocStringIndex@1@@Z 5f807d99 f
 0001:00006daf       ?CalcFixedLayout@CControlBar@@UAE?AVCSize@@HH@Z 5f807daf f
 0001:00006de3       ?CalcDynamicLayout@CToolBar@@UAE?AVCSize@@HK@Z 5f807de3 f
 0001:00006e44       ?CalcLayout@CToolBar@@IAE?AVCSize@@KH@Z 5f807e44 f
 0001:00007157       ?SizeToolBar@CToolBar@@IAEXPAU_TBBUTTON@@HHH@Z 5f808157 f
 0001:0000720b       ?WrapToolBar@CToolBar@@IAEHPAU_TBBUTTON@@HH@Z 5f80820b f
 0001:000072de       ?CalcSize@CToolBar@@IAE?AVCSize@@PAU_TBBUTTON@@H@Z 5f8082de f
 0001:000073f7       ?Layout@CToolBar@@IAEXXZ   5f8083f7 f
 0001:00007436       ?SetTextColor@CDC@@UAEKK@Z 5f808436 f
 0001:00007462       ?SetTitle@CDocument@@UAEXPBG@Z 5f808462 f
 0001:0000747f       ?RegisterIfServerAttached@COleLinkingDoc@@MAEHPBGH@Z 5f80847f f
 0001:000074ab       ?Register@COleLinkingDoc@@QAEHPAVCOleObjectFactory@@PBG@Z 5f8084ab f
 0001:0000758d       ?InitialUpdateFrame@CDocTemplate@@UAEXPAVCFrameWnd@@PAVCDocument@@H@Z 5f80858d f
 0001:000075a1       ?InitialUpdateFrame@CFrameWnd@@QAEXPAVCDocument@@H@Z 5f8085a1 f
 0001:00007667       ??_9@$BOI@AE               5f808667 f
 0001:0000766f       ?OnInitialUpdate@CView@@UAEXXZ 5f80866f f
 0001:0000767d       ?OnUpdate@CView@@MAEXPAV1@JPAVCObject@@@Z 5f80867d f
 0001:0000768d       ?ActivateFrame@CFrameWnd@@UAEXH@Z 5f80868d f
 0001:000076d2       ?BringToTop@CFrameWnd@@IAEXH@Z 5f8086d2 f
 0001:00007701       ??0CPaintDC@@QAE@PAVCWnd@@@Z 5f808701 f
 0001:00007756       ?ExtTextOutW@CDC@@UAEHHHIPBUtagRECT@@PBGIPAH@Z 5f808756 f
 0001:0000777b       ??1CPaintDC@@UAE@XZ        5f80877b f
 0001:000077c2       ?DrawBorders@CControlBar@@QAEXPAVCDC@@AAVCRect@@@Z 5f8087c2 f
 0001:000079c9       ?OnEraseBkgnd@CWnd@@IAEHPAVCDC@@@Z 5f8089c9 f
 0001:000079d1       ?DrawGripper@CControlBar@@QAEXPAVCDC@@ABVCRect@@@Z 5f8089d1 f
 0001:000079ef       ?FillSolidRect@CDC@@QAEXHHHHK@Z 5f8089ef f
 0001:00007a3b       ?OnPaint@CToolBar@@IAEXXZ  5f808a3b f
 0001:00007a55       ?OnEraseBkgnd@CToolBar@@IAEHPAVCDC@@@Z 5f808a55 f
 0001:00007a5d       __imp_load__CoLockObjectExternal@12 5f808a5d f
 0001:00007a69       ?OnShowViews@COleLinkingDoc@@MAEXH@Z 5f808a69 f
 0001:00007a7e       ?AddRef@XPersistStorage@COleServerDoc@@UAGKXZ 5f808a7e f
 0001:00007a90       __imp_load__GetFileTitleW@12 5f808a90 f
 0001:00007a97       __tailMerge_comdlg32       5f808a97 f
 0001:00007aa5       ?Open@CFile@@UAEHPBGIPAVCFileException@@@Z 5f808aa5 f
 0001:00007b76       ?AfxFullPath@@YGHPAGPBG@Z  5f808b76 f
 0001:00007c0d       ?AfxGetRoot@@YGXPBGAAVCString@@@Z 5f808c0d f
 0001:00007cae       ??0CTime@@QAE@ABU_FILETIME@@H@Z 5f808cae f
 0001:00007cfd       ??0CTime@@QAE@ABU_SYSTEMTIME@@H@Z 5f808cfd f
 0001:00007d48       ??0CTime@@QAE@HHHHHHH@Z    5f808d48 f
 0001:00007d95       ?Seek@CFile@@UAEJJI@Z      5f808d95 f
 0001:00007dba       ?Read@CFile@@UAEIPAXI@Z    5f808dba f
 0001:00007deb       ?Close@CFile@@UAEXXZ       5f808deb f
 0001:00007e22       ?OpenDocumentFile@CSingleDocTemplate@@UAEPAVCDocument@@PBGH@Z 5f808e22 f
 0001:00007f59       ?SetTitle@CRichEditDoc@@UAEXPBG@Z 5f808f59 f
 0001:00008016       ?DeleteContents@CRichEditView@@UAEXXZ 5f809016 f
 0001:00008046       ?SetSel@CRichEditCtrl@@QAEXJJ@Z 5f809046 f
 0001:0000806f       ?SetDefaultCharFormat@CRichEditCtrl@@QAEHAAU_charformat@@@Z 5f80906f f
 0001:0000808d       ?SetSelectionCharFormat@CRichEditCtrl@@QAEHAAU_charformat@@@Z 5f80908d f
 0001:000080ab       ?SetParaFormat@CRichEditCtrl@@QAEHAAU_paraformat@@@Z 5f8090ab f
 0001:000080c9       ?SetModifiedFlag@CRichEditDoc@@UAEXH@Z 5f8090c9 f
 0001:000080e8       ?OnInitialUpdate@CRichEditView@@MAEXXZ 5f8090e8 f
 0001:00008101       ?OnPaint@CControlBar@@QAEXXZ 5f809101 f
 0001:00008153       ?DoPaint@CControlBar@@UAEXPAVCDC@@@Z 5f809153 f
 0001:0000818a       ?MoveTo@CDC@@QAE?AVCPoint@@HH@Z 5f80918a f
 0001:000081cd       ?LineTo@CDC@@QAEHHH@Z      5f8091cd f
 0001:000081f5       ?SetBkMode@CDC@@QAEHH@Z    5f8091f5 f
 0001:00008220       ?OnUpdateFrameTitle@CFrameWnd@@UAEXH@Z 5f809220 f
 0001:00008263       ?MatchDocType@CDocTemplate@@UAE?AW4Confidence@1@PBGAAPAVCDocument@@@Z 5f809263 f
 0001:00008316       ?AfxComparePath@@YGHPBG0@Z 5f809316 f
 0001:00008351       ?OnOpenDocument@COleLinkingDoc@@UAEHPBG@Z 5f809351 f
 0001:000083a0       __imp_load__CreateFileMoniker@8 5f8093a0 f
 0001:000083ac       __imp_load__GetRunningObjectTable@8 5f8093ac f
 0001:000083b8       ?OnOpenDocument@COleDocument@@UAEHPBG@Z 5f8093b8 f
 0001:000083fd       ?OnOpenDocument@CDocument@@UAEHPBG@Z 5f8093fd f
 0001:0000852f       ?GetBufferPtr@CFile@@UAEIIIPAPAX0@Z 5f80952f f
 0001:00008534       ?Serialize@CRichEditDoc@@UAEXAAVCArchive@@@Z 5f809534 f
 0001:0000854e       ?Serialize@CRichEditView@@UAEXAAVCArchive@@@Z 5f80954e f
 0001:0000855c       ?Stream@CRichEditView@@QAEXAAVCArchive@@H@Z 5f80955c f
 0001:000085d6       ?EditStreamCallBack@CRichEditView@@SGKKPAEJPAJ@Z 5f8095d6 f
 0001:00008635       ?GetPosition@CFile@@UBEKXZ 5f809635 f
 0001:00008654       ?SetMessageText@CFrameWnd@@QAEXPBG@Z 5f809654 f
 0001:0000866b       ?ReleaseFile@CDocument@@UAEXPAVCFile@@H@Z 5f80966b f
 0001:00008693       ?SetPathName@CRichEditDoc@@UAEXPBGH@Z 5f809693 f
 0001:000086a3       ?SetPathName@CDocument@@UAEXPBGH@Z 5f8096a3 f
 0001:0000871f       ?AddToRecentFileList@CWinApp@@UAEXPBG@Z 5f80971f f
 0001:00008735       ?Add@CRecentFileList@@UAEXPBG@Z 5f809735 f
 0001:00008793       ?AfxBeginThread@@YGPAVCWinThread@@P6AIPAX@Z0HIKPAU_SECURITY_ATTRIBUTES@@@Z 5f809793 f
 0001:0000880d       ??0CWinThread@@QAE@P6AIPAX@Z0@Z 5f80980d f
 0001:00008851       ?CreateThread@CWinThread@@QAEHKIPAU_SECURITY_ATTRIBUTES@@@Z 5f809851 f
 0001:0000891c       ?_AfxThreadEntry@@YGIPAX@Z 5f80991c f
 0001:000089ec       ??1CButton@@UAE@XZ         5f8099ec f
 0001:00008a24       ?AfxEndThread@@YGXIH@Z     5f809a24 f
 0001:00008a6a       ?Delete@CWinThread@@UAEXXZ 5f809a6a f
 0001:00008a7c       ??_GCWinThread@@UAEPAXI@Z  5f809a7c f
 0001:00008a7c       ??_ECWinThread@@UAEPAXI@Z  5f809a7c f
 0001:00008a98       ?AfxTermThread@@YGXPAUHINSTANCE__@@@Z 5f809a98 f
 0001:00008ae3       ?AfxTlsAddRef@@YGXXZ       5f809ae3 f
 0001:00008aea       ?AfxCriticalInit@@YGHXZ    5f809aea f
 0001:00008b24       ??0CThreadSlotData@@QAE@XZ 5f809b24 f
 0001:00008b65       ?AllocSlot@CThreadSlotData@@QAEHXZ 5f809b65 f
 0001:00008c2a       __initterm                 5f809c2a f
 0001:00008c53       ??0CFixedAlloc@@QAE@II@Z   5f809c53 f
 0001:00008c7b       _atexit                    5f809c7b f
 0001:00008c8d       __onexit                   5f809c8d f
 0001:00008cb1       ___dllonexit               5f809cb1 f
 0001:00008dfa       ??0CSessionMapPtrToPtr@@QAE@XZ 5f809dfa f
 0001:00008e49       ??0CSyncObject@@QAE@PBG@Z  5f809e49 f
 0001:00008f48       ??0AFX_MODULE_STATE@@QAE@HP6GJPAUHWND__@@IIJ@ZKH@Z 5f809f48 f
 0001:00008ffe       ??0CMemoryException@@QAE@HI@Z 5f809ffe f
 0001:00009028       ??0CException@@QAE@H@Z     5f80a028 f
 0001:0000905d       ??0CNotSupportedException@@QAE@HI@Z 5f80a05d f
 0001:00009092       ?AfxClassInit@@YGXPAUCRuntimeClass@@@Z 5f80a092 f
 0001:0000914a       ??0CWnd@@AAE@PAUHWND__@@@Z 5f80a14a f
 0001:00009283       ??0CResourceException@@QAE@HI@Z 5f80a283 f
 0001:000092d0       ??0CUserException@@QAE@HI@Z 5f80a2d0 f
 0001:00009321       ??0AUX_DATA@@QAE@XZ        5f80a321 f
 0001:000093bc       ?UpdateSysMetrics@AUX_DATA@@QAEXXZ 5f80a3bc f
 0001:00009411       ?AfxEnableWin40Compatibility@@YGXXZ 5f80a411 f
 0001:00009441       ?UpdateSysColors@AUX_DATA@@QAEXXZ 5f80a441 f
 0001:000094ac       ??0OLE_DATA@@QAE@XZ        5f80a4ac f
 0001:000095aa       ??0CColorPropPageFactory@CColorPropPage@@QAE@ABU_GUID@@PAUCRuntimeClass@@HPBG@Z 5f80a5aa f
 0001:000095ce       ??0COleObjectFactory@@QAE@ABU_GUID@@PAUCRuntimeClass@@HPBG@Z 5f80a5ce f
 0001:00009680       ??0CFontPropPageFactory@CFontPropPage@@QAE@ABU_GUID@@PAUCRuntimeClass@@HPBG@Z 5f80a680 f
 0001:000096d1       ??0CPicturePropPageFactory@CPicturePropPage@@QAE@ABU_GUID@@PAUCRuntimeClass@@HPBG@Z 5f80a6d1 f
 0001:00009713       ??0CWinApp@@QAE@PBG@Z      5f80a713 f
 0001:000097f2       ??0CWinThread@@QAE@XZ      5f80a7f2 f
 0001:0000982f       ?AfxInitExtensionModule@@YGHAAUAFX_EXTENSION_MODULE@@PAUHINSTANCE__@@@Z 5f80a82f f
 0001:00009871       ?AfxWinInit@@YGHPAUHINSTANCE__@@0PAGH@Z 5f80a871 f
 0001:000098d4       ?SetCurrentHandles@CWinApp@@QAEXXZ 5f80a8d4 f
 0001:000099ed       ?RegisterAll@COleObjectFactory@@SGHXZ 5f80a9ed f
 0001:00009a7d       ?IsRegistered@COleObjectFactory@@UBEHXZ 5f80aa7d f
 0001:00009aad       ?Register@COleObjectFactory@@UAEHXZ 5f80aaad f
 0001:00009aad       ?Register@COleTemplateServer@@UAEHXZ 5f80aaad f
 0001:00009ac3       ??0CDynLinkLibrary@@QAE@AAUAFX_EXTENSION_MODULE@@H@Z 5f80aac3 f
 0001:00009b4d       ?CreateObject@?$CProcessLocal@V_AFX_BASE_MODULE_STATE@@@@SGPAVCNoTrackObject@@XZ 5f80ab4d f
 0001:00009b7f       ??0AFX_MODULE_STATE@@QAE@HP6GJPAUHWND__@@IIJ@ZK@Z 5f80ab7f f
 0001:00009be0       ?AfxWinMain@@YGHPAUHINSTANCE__@@0PAGH@Z 5f80abe0 f
 0001:00009c55       ?CreateObject@?$CProcessLocal@V_AFX_CTL3D_STATE@@@@SGPAVCNoTrackObject@@XZ 5f80ac55 f
 0001:00009c6b       ?InitApplication@CWinApp@@UAEHXZ 5f80ac6b f
 0001:00009cab       ?Enable3dControls@CWinApp@@IAEHXZ 5f80acab f
 0001:00009cc1       ?AfxOleInit@@YGHXZ         5f80acc1 f
 0001:00009d53       ??0COleMessageFilter@@QAE@XZ 5f80ad53 f
 0001:00009d95       ?Register@COleMessageFilter@@QAEHXZ 5f80ad95 f
 0001:00009db4       __imp_load__CoRegisterMessageFilter@8 5f80adb4 f
 0001:00009dc0       ?AddRef@XMessageFilter@COleMessageFilter@@UAGKXZ 5f80adc0 f
 0001:00009dcf       __imp_load__InitCommonControlsEx@4 5f80adcf f
 0001:00009dd6       __tailMerge_COMCTL32       5f80add6 f
 0001:00009de4       ?CreateObject@?$CProcessLocal@V_AFX_WIN_STATE@@@@SGPAVCNoTrackObject@@XZ 5f80ade4 f
 0001:00009e15       ??0_AFX_WIN_STATE@@QAE@XZ  5f80ae15 f
 0001:00009e1e       ?SubclassWindow@CWnd@@QAEHPAUHWND__@@@Z 5f80ae1e f
 0001:00009e61       ??0COleTemplateServer@@QAE@XZ 5f80ae61 f
 0001:00009e82       ??0CCommandLineInfo@@QAE@XZ 5f80ae82 f
 0001:00009ef1       ?LoadStdProfileSettings@CWinApp@@IAEXI@Z 5f80aef1 f
 0001:00009f6d       ??0CRecentFileList@@QAE@IPBG0HH@Z 5f80af6d f
 0001:0000a029       ??0CDocTemplate@@IAE@IPAUCRuntimeClass@@00@Z 5f80b029 f
 0001:0000a130       ??0CDocManager@@QAE@XZ     5f80b130 f
 0001:0000a16a       ??_L@YGXPAXIHP6EX0@Z1@Z    5f80b16a f
 0001:0000a1df       ?AddDocTemplate@CDocManager@@UAEXPAVCDocTemplate@@@Z 5f80b1df f
 0001:0000a244       ?LoadTemplate@CDocTemplate@@UAEXXZ 5f80b244 f
 0001:0000a307       ?ReadList@CRecentFileList@@UAEXXZ 5f80b307 f
 0001:0000a3a6       ?GetProfileStringW@CWinApp@@QAE?AVCString@@PBG00@Z 5f80b3a6 f
 0001:0000a4b7       ?GetProfileIntW@CWinApp@@QAEIPBG0H@Z 5f80b4b7 f
 0001:0000a526       ?SetServerInfo@CDocTemplate@@QAEXIIPAUCRuntimeClass@@0@Z 5f80b526 f
 0001:0000a553       ?ParseCommandLine@CWinApp@@QAEXAAVCCommandLineInfo@@@Z 5f80b553 f
 0001:0000a5ad       ??0CFrameWnd@@QAE@XZ       5f80b5ad f
 0001:0000a673       ?AddFrameWnd@CFrameWnd@@IAEXXZ 5f80b673 f
 0001:0000a694       ??0CStatusBar@@QAE@XZ      5f80b694 f
 0001:0000a6c6       ??0CControlBar@@IAE@XZ     5f80b6c6 f
 0001:0000a718       ??0CToolBar@@QAE@XZ        5f80b718 f
 0001:0000a77c       ?LoadFrame@CFrameWnd@@UAEHIKPAVCWnd@@PAUCCreateContext@@@Z 5f80b77c f
 0001:0000a848       ?_AfxRegisterWithIcon@@YGHPAUtagWNDCLASSW@@PBGI@Z 5f80b848 f
 0001:0000a889       ?AfxRegisterClass@@YGHPAUtagWNDCLASSW@@@Z 5f80b889 f
 0001:0000a8e7       ?GetIconWndClass@CFrameWnd@@IAEPBGKI@Z 5f80b8e7 f
 0001:0000a96a       ?AfxRegisterWndClass@@YGPBGIPAUHICON__@@PAUHBRUSH__@@0@Z 5f80b96a f
 0001:0000aa02       ?Create@CFrameWnd@@QAEHPBG0KABUtagRECT@@PAVCWnd@@0KPAUCCreateContext@@@Z 5f80ba02 f
 0001:0000aa8a       ?CreateEx@CWnd@@QAEHKPBG0KHHHHPAUHWND__@@PAUHMENU__@@PAX@Z 5f80ba8a f
 0001:0000ab40       ?OnCreate@CFrameWnd@@IAEHPAUtagCREATESTRUCTW@@@Z 5f80bb40 f
 0001:0000ab4f       ?OnCreateHelper@CFrameWnd@@IAEHPAUtagCREATESTRUCTW@@PAUCCreateContext@@@Z 5f80bb4f f
 0001:0000aba1       ?RecalcLayout@CFrameWnd@@UAEXH@Z 5f80bba1 f
 0001:0000ac1f       ?RepositionBars@CWnd@@QAEXIIIIPAUtagRECT@@PBU2@H@Z 5f80bc1f f
 0001:0000ad2c       ?CalcWindowRect@CWnd@@UAEXPAUtagRECT@@I@Z 5f80bd2c f
 0001:0000ad57       ?AfxRepositionWindow@@YGXPAUAFX_SIZEPARENTPARAMS@@PAUHWND__@@PBUtagRECT@@@Z 5f80bd57 f
 0001:0000addf       ?Create@CToolBar@@QAEHPAVCWnd@@KI@Z 5f80bddf f
 0001:0000ae21       ?CreateEx@CToolBar@@QAEHPAVCWnd@@KKVCRect@@I@Z 5f80be21 f
 0001:0000aec5       ?SetBorders@CControlBar@@QAEXHHHH@Z 5f80bec5 f
 0001:0000aee4       ?_AfxGetComCtlVersion@@YGKXZ 5f80bee4 f
 0001:0000af52       ?_AfxGetDropDownWidth@@YGHXZ 5f80bf52 f
 0001:0000afd3       ?Create@CWnd@@UAEHPBG0KABUtagRECT@@PAV1@IPAUCCreateContext@@@Z 5f80bfd3 f
 0001:0000b01f       ?PreCreateWindow@CControlBar@@UAEHAAUtagCREATESTRUCTW@@@Z 5f80c01f f
 0001:0000b092       ?PreCreateWindow@CWnd@@UAEHAAUtagCREATESTRUCTW@@@Z 5f80c092 f
 0001:0000b0a8       ?OnNcCreate@CToolBar@@IAEHPAUtagCREATESTRUCTW@@@Z 5f80c0a8 f
 0001:0000b0d9       ?OnNcCalcSize@CToolBar@@IAEXHPAUtagNCCALCSIZE_PARAMS@@@Z 5f80c0d9 f
 0001:0000b13a       ?OnCreate@CControlBar@@QAEHPAUtagCREATESTRUCTW@@@Z 5f80c13a f
 0001:0000b18f       ?SetSizes@CToolBar@@QAEXUtagSIZE@@0@Z 5f80c18f f
 0001:0000b1f4       ?OnSetBitmapSize@CToolBar@@IAEJIJ@Z 5f80c1f4 f
 0001:0000b207       ?OnSetSizeHelper@CToolBar@@IAEJAAVCSize@@J@Z 5f80c207 f
 0001:0000b258       ?OnSetButtonSize@CToolBar@@IAEJIJ@Z 5f80c258 f
 0001:0000b26b       ?LoadBitmapW@CToolBar@@QAEHPBG@Z 5f80c26b f
 0001:0000b2bf       ?AfxLoadSysColorBitmap@@YGPAUHBITMAP__@@PAUHINSTANCE__@@PAUHRSRC__@@H@Z 5f80c2bf f
 0001:0000b42b       ?AddReplaceBitmap@CToolBar@@QAEHPAUHBITMAP__@@@Z 5f80c42b f
 0001:0000b4a2       ?SetButtons@CToolBar@@QAEHPBIH@Z 5f80c4a2 f
 0001:0000b587       ?Create@CStatusBar@@QAEHPAVCWnd@@KI@Z 5f80c587 f
 0001:0000b59d       ?CreateEx@CStatusBar@@QAEHPAVCWnd@@KKI@Z 5f80c59d f
 0001:0000b60d       ?PreCreateWindow@CStatusBar@@UAEHAAUtagCREATESTRUCTW@@@Z 5f80c60d f
 0001:0000b63c       ?OnNcCalcSize@CStatusBar@@IAEXHPAUtagNCCALCSIZE_PARAMS@@@Z 5f80c63c f
 0001:0000b67e       ?OnSize@CStatusBar@@IAEXIHH@Z 5f80c67e f
 0001:0000b695       ?CalcInsideRect@CStatusBar@@QBEXAAVCRect@@H@Z 5f80c695 f
 0001:0000b705       ?OnChildNotify@CStatusBar@@MAEHIIJPAJ@Z 5f80c705 f
 0001:0000b727       ?SetIndicators@CStatusBar@@QAEHPBIH@Z 5f80c727 f
 0001:0000b864       ?Attach@CGdiObject@@QAEHPAX@Z 5f80c864 f
 0001:0000b890       ??0CClientDC@@QAE@PAVCWnd@@@Z 5f80c890 f
 0001:0000b8e7       ??1CClientDC@@UAE@XZ       5f80c8e7 f
 0001:0000b929       ?EnableDocking@CFrameWnd@@QAEXK@Z 5f80c929 f
 0001:0000b9bd       ?GetControlBar@CFrameWnd@@QAEPAVCControlBar@@I@Z 5f80c9bd f
 0001:0000b9f1       ??0CDockBar@@QAE@H@Z       5f80c9f1 f
 0001:0000ba6f       ?Create@CDockBar@@QAEHPAVCWnd@@KI@Z 5f80ca6f f
 0001:0000bab6       ?OnNcCalcSize@CDockBar@@IAEXHPAUtagNCCALCSIZE_PARAMS@@@Z 5f80cab6 f
 0001:0000bafc       ?EnableDocking@CControlBar@@QAEXK@Z 5f80cafc f
 0001:0000bb5b       ??0CDockContext@@QAE@PAVCControlBar@@@Z 5f80cb5b f
 0001:0000bbbc       ?SetBarStyle@CControlBar@@QAEXK@Z 5f80cbbc f
 0001:0000bbea       ?EnableToolTips@CWnd@@QAEHH@Z 5f80cbea f
 0001:0000bbf8       ?_EnableToolTips@CWnd@@QAEHHI@Z 5f80cbf8 f
 0001:0000bc46       ?OnBarStyleChange@CToolBar@@UAEXKK@Z 5f80cc46 f
 0001:0000bc79       ?DockControlBar@CFrameWnd@@QAEXPAVCControlBar@@IPBUtagRECT@@@Z 5f80cc79 f
 0001:0000bc9c       ?DockControlBar@CFrameWnd@@QAEXPAVCControlBar@@PAVCDockBar@@PBUtagRECT@@@Z 5f80cc9c f
 0001:0000bce8       ?DockControlBar@CDockBar@@QAEXPAVCControlBar@@PBUtagRECT@@@Z 5f80cce8 f
 0001:0000be45       ?GetWindowTextW@CWnd@@QBEHPAGH@Z 5f80ce45 f
 0001:0000be64       ?OnWindowPosChanging@CToolBar@@IAEXPAUtagWINDOWPOS@@@Z 5f80ce64 f
 0001:0000bea1       ?OnWindowPosChanging@CControlBar@@QAEXPAUtagWINDOWPOS@@@Z 5f80cea1 f
 0001:0000bf10       ?RemovePlaceHolder@CDockBar@@QAEXPAVCControlBar@@@Z 5f80cf10 f
 0001:0000bf49       ?FindBar@CDockBar@@QAEHPAVCControlBar@@H@Z 5f80cf49 f
 0001:0000bf77       ?GetDockingFrame@CControlBar@@QBEPAVCFrameWnd@@XZ 5f80cf77 f
 0001:0000bf89       ?LoadAccelTable@CFrameWnd@@QAEHPBG@Z 5f80cf89 f
 0001:0000bfb2       ?ConnectTemplate@COleTemplateServer@@QAEXABU_GUID@@PAVCDocTemplate@@H@Z 5f80cfb2 f
 0001:0000bfd5       __imp_load__DragAcceptFiles@8 5f80cfd5 f
 0001:0000bfdc       __tailMerge_SHELL32        5f80cfdc f
 0001:0000bfea       ?CreateNewDocument@CDocTemplate@@UAEPAVCDocument@@XZ 5f80cfea f
 0001:0000c015       ??0COleServerDoc@@QAE@XZ   5f80d015 f
 0001:0000c0ba       ??0COleLinkingDoc@@QAE@XZ  5f80d0ba f
 0001:0000c12f       ??0COleDocument@@QAE@XZ    5f80d12f f
 0001:0000c194       ??0CDocument@@QAE@XZ       5f80d194 f
 0001:0000c1f8       ??0CObList@@QAE@H@Z        5f80d1f8 f
 0001:0000c21b       ?AfxOleLockApp@@YGXXZ      5f80d21b f
 0001:0000c22b       ?AddDocument@CDocTemplate@@UAEXPAVCDocument@@@Z 5f80d22b f
 0001:0000c235       ?CreateNewFrame@CDocTemplate@@UAEPAVCFrameWnd@@PAVCDocument@@PAV2@@Z 5f80d235 f
 0001:0000c2a2       ?PreCreateWindow@CFrameWnd@@MAEHAAUtagCREATESTRUCTW@@@Z 5f80d2a2 f
 0001:0000c2e6       ?OnCreateClient@CFrameWnd@@MAEHPAUtagCREATESTRUCTW@@PAUCCreateContext@@@Z 5f80d2e6 f
 0001:0000c308       ?CreateView@CFrameWnd@@QAEPAVCWnd@@PAUCCreateContext@@I@Z 5f80d308 f
 0001:0000c384       ??0CView@@IAE@XZ           5f80d384 f
 0001:0000c39a       ?PreCreateWindow@CView@@MAEHAAUtagCREATESTRUCTW@@@Z 5f80d39a f
 0001:0000c3db       ?OnCreate@CView@@IAEHPAUtagCREATESTRUCTW@@@Z 5f80d3db f
 0001:0000c40b       ?AddView@CDocument@@QAEXPAVCView@@@Z 5f80d40b f
 0001:0000c42b       ?ProcessShellCommand@CWinApp@@QAEHAAVCCommandLineInfo@@@Z 5f80d42b f
 0001:0000c4a3       ?ModifyStyleEx@CWnd@@QAEHKKI@Z 5f80d4a3 f
 0001:0000c4c6       ?ModifyStyleEx@CWnd@@SGHPAUHWND__@@KKI@Z 5f80d4c6 f
 0001:0000c4e0       ?OnSizeParent@CControlBar@@QAEJIJ@Z 5f80d4e0 f
 0001:0000c629       ?RecalcDelayShow@CControlBar@@UAEKPAUAFX_SIZEPARENTPARAMS@@@Z 5f80d629 f
 0001:0000c659       ?CalcDynamicLayout@CControlBar@@UAE?AVCSize@@HK@Z 5f80d659 f
 0001:0000c68c       ?CalcFixedLayout@CStatusBar@@UAE?AVCSize@@HH@Z 5f80d68c f
 0001:0000c751       ?OnSize@CFrameWnd@@IAEXIHH@Z 5f80d751 f
 0001:0000c770       ?OnSizeParent@CDockBar@@IAEJIJ@Z 5f80d770 f
 0001:0000c7d6       ?CalcFixedLayout@CDockBar@@UAE?AVCSize@@HH@Z 5f80d7d6 f
 0001:0000ca8e       ?CalcFixedLayout@CToolBar@@UAE?AVCSize@@HH@Z 5f80da8e f
 0001:0000cac6       ?OnWindowPosChanging@CDockBar@@IAEXPAUtagWINDOWPOS@@@Z 5f80dac6 f
 0001:0000cae6       ??0CWindowDC@@QAE@PAVCWnd@@@Z 5f80dae6 f
 0001:0000cb3b       ??1CWindowDC@@UAE@XZ       5f80db3b f
 0001:0000cb7d       ?OnNewDocument@COleLinkingDoc@@UAEHXZ 5f80db7d f
 0001:0000cbae       ?OnNewDocument@COleDocument@@UAEHXZ 5f80dbae f
 0001:0000cbd2       ?OnNewDocument@CDocument@@UAEHXZ 5f80dbd2 f
 0001:0000cbf7       ?GetRuntimeClass@CView@@UBEPAUCRuntimeClass@@XZ 5f80dbf7 f
 0001:0000cbfd       ?EraseNonClient@CControlBar@@QAEXXZ 5f80dbfd f
 0001:0000cbfd       ?OnNcPaint@CStatusBar@@IAEXXZ 5f80dbfd f
 0001:0000ccca       ?ExcludeClipRect@CDC@@QAEHPBUtagRECT@@@Z 5f80dcca f
 0001:0000cd02       ?IntersectClipRect@CDC@@QAEHPBUtagRECT@@@Z 5f80dd02 f
 0001:0000cd3a       ?OnPaint@CDockBar@@IAEXXZ  5f80dd3a f
 0001:0000cd9a       ?GetDockedVisibleCount@CDockBar@@UBEHXZ 5f80dd9a f
 0001:0000cdd7       ?SetText@CToolCmdUI@@UAEXPBG@Z 5f80ddd7 f
 0001:0000cdda       ??0CDockState@@QAE@XZ      5f80ddda f
 0001:0000ce57       ??0CSingleDocTemplate@@QAE@IPAUCRuntimeClass@@00@Z 5f80de57 f
 0001:0000ce7f       ??_ECPtrList@@UAEPAXI@Z    5f80de7f f
 0001:0000ceaa       ?ParseParam@CCommandLineInfo@@UAEXPBGHH@Z 5f80deaa f
 0001:0000cedf       ?ParseParamNotFlag@CCommandLineInfo@@IAEXPBG@Z 5f80dedf f
 0001:0000ceff       ?ParseLast@CCommandLineInfo@@IAEXH@Z 5f80deff f
 0001:0000cf2e       ?SetRegistryKey@CWinApp@@IAEXPBG@Z 5f80df2e f
 0001:0000cf75       __imp_load__RegOpenKeyExW@20 5f80df75 f
 0001:0000cf81       __imp_load__RegCreateKeyExW@36 5f80df81 f
 0001:0000cf8d       __imp_load__RegQueryValueExW@24 5f80df8d f
 0001:0000cf99       ?GetProfileBinary@CWinApp@@QAEHPBG0PAPAEPAI@Z 5f80df99 f
 0001:0000d03b       ?Write@CMemFile@@UAEXPBXI@Z 5f80e03b f
 0001:0000d07d       ??5CArchive@@QAEAAV0@AAJ@Z 5f80e07d f
 0001:0000d0b1       ?FillBuffer@CArchive@@QAEXI@Z 5f80e0b1 f
 0001:0000d10d       ?Read@CArchive@@QAEIPAXI@Z 5f80e10d f
 0001:0000d157       ?SetScreenSize@CDockState@@QAEXAAVCSize@@@Z 5f80e157 f
 0001:0000d18d       ??5CArchive@@QAEAAV0@AAG@Z 5f80e18d f
 0001:0000d1b8       ?ScalePoint@CDockState@@QAEXAAVCPoint@@@Z 5f80e1b8 f
 0001:0000d1e6       ?ScaleRectPos@CDockState@@QAEXAAVCRect@@@Z 5f80e1e6 f
 0001:0000d232       ?SubclassDlgItem@CWnd@@QAEHIPAV1@@Z 5f80e232 f
 0001:0000d25e       ?OnChildNotify@CButton@@MAEHIIJPAJ@Z 5f80e25e f
 0001:0000d28c       ?OnDrawItem@CWnd@@IAEXHPAUtagDRAWITEMSTRUCT@@@Z 5f80e28c f
 0001:0000d2b4       ?SelectGdiObject@CDC@@KGPAVCGdiObject@@PAUHDC__@@PAX@Z 5f80e2b4 f
 0001:0000d2cb       __imp_load__PrintDlgW@4    5f80e2cb f
 0001:0000d2d7       ?SetContainerInfo@CDocTemplate@@QAEXI@Z 5f80e2d7 f
 0001:0000d2ef       ??0CRichEditDoc@@IAE@XZ    5f80e2ef f
 0001:0000d312       ?AddDocument@CSingleDocTemplate@@UAEXPAVCDocument@@@Z 5f80e312 f
 0001:0000d328       ??0CRichEditView@@QAE@XZ   5f80e328 f
 0001:0000d3e8       ??0CCtrlView@@QAE@PBGK@Z   5f80e3e8 f
 0001:0000d439       ??0CDWordArray@@QAE@XZ     5f80e439 f
 0001:0000d450       ?PreCreateWindow@CRichEditView@@MAEHAAUtagCREATESTRUCTW@@@Z 5f80e450 f
 0001:0000d485       ?AfxInitRichEdit@@YGHXZ    5f80e485 f
 0001:0000d4b5       ?CreateObject@?$CProcessLocal@V_AFX_RICHEDIT_STATE@@@@SGPAVCNoTrackObject@@XZ 5f80e4b5 f
 0001:0000d4f2       ??0_AFX_EDIT_STATE@@QAE@XZ 5f80e4f2 f
 0001:0000d537       ?PreCreateWindow@CCtrlView@@MAEHAAUtagCREATESTRUCTW@@@Z 5f80e537 f
 0001:0000d581       ?OnCreate@CRichEditView@@IAEHPAUtagCREATESTRUCTW@@@Z 5f80e581 f
 0001:0000d604       ?AddRef@XRichEditOleCallback@CRichEditView@@UAGKXZ 5f80e604 f
 0001:0000d617       ?GetIRichEditOle@CRichEditCtrl@@QBEPAUIRichEditOle@@XZ 5f80e617 f
 0001:0000d638       ?WrapChanged@CRichEditView@@MAEXXZ 5f80e638 f
 0001:0000d69b       ?AfxW2AHelper@@YGPADPADPBGH@Z 5f80e69b f
 0001:0000d6c5       ?GetWindowPlacement@CWnd@@QBEHPAUtagWINDOWPLACEMENT@@@Z 5f80e6c5 f
 0001:0000d6dc       ?CalcWindowRect@CView@@UAEXPAUtagRECT@@I@Z 5f80e6dc f
 0001:0000d6fd       ?Create@CComboBox@@QAEHKABUtagRECT@@PAVCWnd@@I@Z 5f80e6fd f
 0001:0000d71e       ?OnMeasureItem@CWnd@@IAEXHPAUtagMEASUREITEMSTRUCT@@@Z 5f80e71e f
 0001:0000d75c       ?SetButtonInfo@CToolBar@@QAEXHIIH@Z 5f80e75c f
 0001:0000d7cb       ?GetItemRect@CToolBar@@UBEXHPAUtagRECT@@@Z 5f80e7cb f
 0001:0000d801       ?ClientToScreen@CWnd@@QBEXPAUtagRECT@@@Z 5f80e801 f
 0001:0000d839       ?SetDefaultTitle@CSingleDocTemplate@@UAEXPAVCDocument@@@Z 5f80e839 f
 0001:0000d89b       ?SetDockState@CFrameWnd@@QAEXABVCDockState@@@Z 5f80e89b f
 0001:0000d936       ?SetBarInfo@CControlBar@@QAEXPAVCControlBarInfo@@PAVCFrameWnd@@@Z 5f80e936 f
 0001:0000da04       ?SetBarInfo@CDockBar@@QAEXPAVCControlBarInfo@@PAVCFrameWnd@@@Z 5f80ea04 f
 0001:0000db87       ?RemoveControlBar@CDockBar@@QAEHPAVCControlBar@@HH@Z 5f80eb87 f
 0001:0000dc0b       ?RemoveAt@CObArray@@QAEXHH@Z 5f80ec0b f
 0001:0000dc43       ?InsertAt@CPtrArray@@QAEXHPAXH@Z 5f80ec43 f
 0001:0000dcd6       ?_GetBaseClass@CRichEditView@@KGPAUCRuntimeClass@@XZ 5f80ecd6 f
 0001:0000dcdc       ?OpenDocumentFile@CWinApp@@UAEPAVCDocument@@PBG@Z 5f80ecdc f
 0001:0000dcee       ?OpenDocumentFile@CDocManager@@UAEPAVCDocument@@PBG@Z 5f80ecee f
 0001:0000ddcd       ?AfxResolveShortcut@@YGHPAVCWnd@@PBGPAGH@Z 5f80edcd f
 0001:0000de14       __imp_load__SHGetFileInfoW@20 5f80ee14 f
 0001:0000de20       ?OnNTCtlColor@CWnd@@IAEJIJ@Z 5f80ee20 f
 0001:0000de66       ?GrayCtlColor@CWnd@@SGHPAUHDC__@@PAUHWND__@@IPAUHBRUSH__@@K@Z 5f80ee66 f
 0001:0000de8c       ??1CDialog@@UAE@XZ         5f80ee8c f
 0001:0000dec9       ?OnCtlColor@CDialog@@IAEPAUHBRUSH__@@PAVCDC@@PAVCWnd@@I@Z 5f80eec9 f
 0001:0000dedd       ?OnGrayCtlColor@CWnd@@QAEPAUHBRUSH__@@PAVCDC@@PAV1@I@Z 5f80eedd f
 0001:0000df3e       ??_ECTempGdiObject@@UAEPAXI@Z 5f80ef3e f
 0001:0000df3e       ??_GCTempGdiObject@@UAEPAXI@Z 5f80ef3e f
 0001:0000df5e       ??1CTempGdiObject@@UAE@XZ  5f80ef5e f
 0001:0000df91       ?Attach@CDC@@QAEHPAUHDC__@@@Z 5f80ef91 f
 0001:0000dfc7       ?SetAttribDC@CDC@@UAEXPAUHDC__@@@Z 5f80efc7 f
 0001:0000dfd1       ?OnCtlColor@CControlBar@@QAEPAUHBRUSH__@@PAVCDC@@PAVCWnd@@I@Z 5f80efd1 f
 0001:0000e025       ?OnCtlColor@CWnd@@IAEPAUHBRUSH__@@PAVCDC@@PAV1@I@Z 5f80f025 f
 0001:0000e04b       ?Attach@CWnd@@QAEHPAUHWND__@@@Z 5f80f04b f
 0001:0000e083       ?FromHandle@CGdiObject@@SGPAV1@PAX@Z 5f80f083 f
 0001:0000e098       ?LoadStringW@CString@@QAEHI@Z 5f80f098 f
 0001:0000e0e6       _memcmp                    5f80f0e6 f
 0001:0000e0ec       ?AfxHookWindowCreate@@YGXPAVCWnd@@@Z 5f80f0ec f
 0001:0000e139       ?AfxGetAfxWndProc@@YGP6GJPAUHWND__@@IIJ@ZXZ 5f80f139 f
 0001:0000e145       ?CreateObject@CTempGdiObject@@SGPAVCObject@@XZ 5f80f145 f
 0001:0000e162       ?FromHandle@CDC@@SGPAV1@PAUHDC__@@@Z 5f80f162 f
 0001:0000e177       ?SetViewportOrg@CDC@@UAE?AVCPoint@@HH@Z 5f80f177 f
 0001:0000e1ba       ?OnEraseBkgnd@CFrameWnd@@IAEHPAVCDC@@@Z 5f80f1ba f
 0001:0000e1d0       ??_ECTempDC@@UAEPAXI@Z     5f80f1d0 f
 0001:0000e1d0       ??_GCTempDC@@UAEPAXI@Z     5f80f1d0 f
 0001:0000e1f0       ?SaveDC@CDC@@UAEHXZ        5f80f1f0 f
 0001:0000e21b       ?RestoreDC@CDC@@UAEHH@Z    5f80f21b f
 0001:0000e25a       ??0CMapStringToPtr@@QAE@H@Z 5f80f25a f
 0001:0000e281       ?Lookup@CMapStringToPtr@@QBEHPBGAAPAX@Z 5f80f281 f
 0001:0000e2a3       ?GetAssocAt@CMapStringToPtr@@IBEPAUCAssoc@1@PBGAAI@Z 5f80f2a3 f
 0001:0000e2fc       ??ACMapStringToPtr@@QAEAAPAXPBG@Z 5f80f2fc f
 0001:0000e360       ?NewAssoc@CMapStringToPtr@@IAEPAUCAssoc@1@XZ 5f80f360 f
 0001:0000e3c5       ?RemoveKey@CMapStringToPtr@@QAEHPBG@Z 5f80f3c5 f
 0001:0000e42e       ?FreeAssoc@CMapStringToOb@@IAEXPAUCAssoc@1@@Z 5f80f42e f
 0001:0000e454       ??0CString@@QAE@PBD@Z      5f80f454 f
 0001:0000e4a1       ??1CMapStringToPtr@@UAE@XZ 5f80f4a1 f
 0001:0000e4d4       ?RemoveAll@CMapStringToOb@@QAEXXZ 5f80f4d4 f
 0001:0000e528       ?HandleSetFont@CDialog@@IAEJIJ@Z 5f80f528 f
 0001:0000e54c       ?MeasureItem@CMenu@@UAEXPAUtagMEASUREITEMSTRUCT@@@Z 5f80f54c f
 0001:0000e54f       ?_AfxPreInitDialog@@YGXPAVCWnd@@PAUtagRECT@@PAK@Z 5f80f54f f
 0001:0000e572       ?HandleInitDialog@CDialog@@IAEJIJ@Z 5f80f572 f
 0001:0000e5af       ?_AfxPostInitDialog@@YGXPAVCWnd@@ABUtagRECT@@K@Z 5f80f5af f
 0001:0000e62a       ??0CDialog@@QAE@IPAVCWnd@@@Z 5f80f62a f
 0001:0000e663       ?CenterWindow@CWnd@@QAEXPAV1@@Z 5f80f663 f
 0001:0000e7f8       _xMonitorFromWindow@8      5f80f7f8 f
 0001:0000e81e       _InitMultipleMonitorStubs  5f80f81e f
 0001:0000e8a9       _xGetMonitorInfo@8         5f80f8a9 f
 0001:0000e933       ?UpdatePrinterSelection@CWinApp@@IAEXH@Z 5f80f933 f
 0001:0000eae2       ??0CPrintDialog@@QAE@HKPAVCWnd@@@Z 5f80fae2 f
 0001:0000eb74       ?GetDefaults@CPrintDialog@@QAEHXZ 5f80fb74 f
 0001:0000eb84       _PrintDlgW@4               5f80fb84 f
 0001:0000eb8a       ?AfxFindResourceHandle@@YGPAUHINSTANCE__@@PBG0@Z 5f80fb8a f
 0001:0000ec52       ?AfxEndDeferRegisterClass@@YGHJ@Z 5f80fc52 f
 0001:0000eecb       ?_AfxInitCommonControls@@YGJPAUtagINITCOMMONCONTROLSEX@@J@Z 5f80fecb f
 0001:0000ef14       ??4CString@@QAEABV0@ABV0@@Z 5f80ff14 f
 0001:0000ef5f       ?CreateObject@CTempDC@@SGPAVCObject@@XZ 5f80ff5f f
 0001:0000ef85       ?UpdateData@CWnd@@QAEHH@Z  5f80ff85 f
 0001:0000effe       ??0CDataExchange@@QAE@PAVCWnd@@H@Z 5f80fffe f
 0001:0000f014       ?AfxDlgProc@@YGHPAUHWND__@@IIJ@Z 5f810014 f
 0001:0000f04d       ?CreateDlgIndirect@CWnd@@IAEHPBUDLGTEMPLATE@@PAV1@PAUHINSTANCE__@@@Z 5f81004d f
 0001:0000f17b       ?GetFont@CDialogTemplate@@SAHPBUDLGTEMPLATE@@AAVCString@@AAG@Z 5f81017b f
 0001:0000f1c9       ?GetFontSizeField@CDialogTemplate@@KAPAEPBUDLGTEMPLATE@@@Z 5f8101c9 f
 0001:0000f21c       ?Create@CDialog@@QAEHPBGPAVCWnd@@@Z 5f81021c f
 0001:0000f26d       ?CreateIndirect@CDialog@@IAEHPAXPAVCWnd@@PAUHINSTANCE__@@@Z 5f81026d f
 0001:0000f290       ?CreateIndirect@CDialog@@IAEHPBUDLGTEMPLATE@@PAVCWnd@@PAXPAUHINSTANCE__@@@Z 5f810290 f
 0001:0000f2bb       ?OnInitDialog@CDialog@@UAEHXZ 5f8102bb f
 0001:0000f307       ?ExecuteDlgInit@CWnd@@QAEHPBG@Z 5f810307 f
 0001:0000f34b       ?ExecuteDlgInit@CWnd@@QAEHPAX@Z 5f81034b f
 0001:0000f38b       ?GetDlgItem@CWnd@@QBEPAV1@H@Z 5f81038b f
 0001:0000f3ac       ?_GetBaseClass@COleDialog@@KGPAUCRuntimeClass@@XZ 5f8103ac f
 0001:0000f3b2       ??0CDialog@@QAE@XZ         5f8103b2 f
 0001:0000f3d4       ?GetMessageMap@CDialog@@MBEPBUAFX_MSGMAP@@XZ 5f8103d4 f
 0001:0000f3da       ?EnableModeless@CWinApp@@QAEXH@Z 5f8103da f
 0001:0000f403       ?OnCmdMsg@CDialog@@UAEHIHPAXPAUAFX_CMDHANDLERINFO@@@Z 5f810403 f
 0001:0000f444       ?OnEnable@CFrameWnd@@IAEXH@Z 5f810444 f
 0001:0000f4dc       ?GetMessageMap@CPrintDialog@@MBEPBUAFX_MSGMAP@@XZ 5f8104dc f
 0001:0000f4e2       ?GetMessageMap@CCommonDialog@@MBEPBUAFX_MSGMAP@@XZ 5f8104e2 f
 0001:0000f4e8       ?_GetBaseMessageMap@CCommonDialog@@KGPBUAFX_MSGMAP@@XZ 5f8104e8 f
 0001:0000f4ee       ?PostModal@CDialog@@IAEXXZ 5f8104ee f
 0001:0000f529       ??_9@$BNA@AE               5f810529 f
 0001:0000f531       ?OnCancel@CCommonDialog@@MAEXXZ 5f810531 f
 0001:0000f536       ??_9@$BMM@AE               5f810536 f
 0001:0000f53e       ?OnOK@CCommonDialog@@MAEXXZ 5f81053e f
 0001:0000f555       ?GetDeviceName@CPrintDialog@@QBE?AVCString@@XZ 5f810555 f
 0001:0000f589       ?GetPortName@CPrintDialog@@QBE?AVCString@@XZ 5f810589 f
 0001:0000f5bd       ?BeginModalState@CFrameWnd@@UAEXXZ 5f8105bd f
 0001:0000f631       ?Serialize@CObject@@UAEXAAVCArchive@@@Z 5f810631 f
 0001:0000f634       ?CheckAutoCenter@CDialog@@UAEHXZ 5f810634 f
 0001:0000f6aa       ?PreModal@CDialog@@IAEPAUHWND__@@XZ 5f8106aa f
 0001:0000f6e5       ?GetSafeOwner_@CWnd@@SGPAUHWND__@@PAU2@PAPAU2@@Z 5f8106e5 f
 0001:0000f779       ?GetRoutingFrame_@CCmdTarget@@KGPAVCFrameWnd@@XZ 5f810779 f
 0001:0000f785       ?EndModalState@CFrameWnd@@UAEXXZ 5f810785 f
 0001:0000f7af       ??1CPrintInfo@@QAE@XZ      5f8107af f
 0001:0000f80a       ??_GCFindReplaceDialog@@UAEPAXI@Z 5f81080a f
 0001:0000f80a       ??_ECFindReplaceDialog@@UAEPAXI@Z 5f81080a f
 0001:0000f826       ?CreatePrinterDC@CWinApp@@QAEHAAVCDC@@@Z 5f810826 f
 0001:0000f85c       ?AfxCreateDC@@YGPAUHDC__@@PAX0@Z 5f81085c f
 0001:0000f8ca       ?DeleteDC@CDC@@QAEHXZ      5f8108ca f
 0001:0000f8d7       ?OnPrinterChanged@CRichEditView@@MAEXABVCDC@@@Z 5f8108d7 f
 0001:0000f962       ?GetLBText@CComboBox@@QBEXHAAVCString@@@Z 5f810962 f
 0001:0000f9a5       ?AfxFormatStrings@@YGXAAVCString@@PBGPBQBGH@Z 5f8109a5 f
 0001:0000fa8c       ?SetMapMode@CDC@@UAEHH@Z   5f810a8c f
 0001:0000fab7       ?Enable@CTestCmdUI@@UAEXH@Z 5f810ab7 f
 0001:0000fac8       ?OnFilePrint@CView@@IAEXXZ 5f810ac8 f
 0001:0000ff02       ??0CPrintInfo@@QAE@XZ      5f810f02 f
 0001:0000ff8a       ?GetCurrentMessage@CWnd@@KGPBUtagMSG@@XZ 5f810f8a f
 0001:0000ffbf       ?DoPreparePrinting@CView@@QAEHPAUCPrintInfo@@@Z 5f810fbf f
 0001:00010053       ?DoPrintDialog@CWinApp@@QAEHPAVCPrintDialog@@@Z 5f811053 f
 0001:000100b8       ?GetDriverName@CPrintDialog@@QBE?AVCString@@XZ 5f8110b8 f
 0001:000100eb       ?DoModal@CPrintDialog@@UAEHXZ 5f8110eb f
 0001:00010119       ?OnBeginPrinting@CRichEditView@@MAEXPAVCDC@@PAUCPrintInfo@@@Z 5f811119 f
 0001:00010145       ?EnableWindow@CWnd@@QAEHH@Z 5f811145 f
 0001:00010160       ??0CPrintingDialog@@QAE@PAVCWnd@@@Z 5f811160 f
 0001:000101b3       ?OnInitDialog@CPrintingDialog@@UAEHXZ 5f8111b3 f
 0001:000101d7       ?SetDlgItemTextW@CWnd@@QAEXHPBG@Z 5f8111d7 f
 0001:000101f6       ?AfxFormatString1@@YGXAAVCString@@IPBG@Z 5f8111f6 f
 0001:0001020d       ?AfxFormatStrings@@YGXAAVCString@@IPBQBGH@Z 5f81120d f
 0001:00010247       ?_AfxAbortProc@@YGHPAUHDC__@@H@Z 5f811247 f
 0001:0001028b       ?OnPrepareDC@CRichEditView@@UAEXPAVCDC@@PAUCPrintInfo@@@Z 5f81128b f
 0001:000102c4       ?OnPrint@CRichEditView@@MAEXPAVCDC@@PAUCPrintInfo@@@Z 5f8112c4 f
 0001:0001032f       ?PrintPage@CRichEditView@@QAEJPAVCDC@@JJ@Z 5f81132f f
 0001:000103ff       ?GetPageRect@CRichEditView@@QBE?AVCRect@@XZ 5f8113ff f
 0001:00010433       ?GetPrintRect@CRichEditView@@QBE?AVCRect@@XZ 5f811433 f
 0001:00010474       ?PaginateTo@CRichEditView@@IAEHPAVCDC@@PAUCPrintInfo@@@Z 5f811474 f
 0001:0001054e       ?IntersectClipRect@CDC@@QAEHHHHH@Z 5f81154e f
 0001:00010585       ?OnEndPrinting@CRichEditView@@MAEXPAVCDC@@PAUCPrintInfo@@@Z 5f811585 f
 0001:000105ad       ?_GetBaseMessageMap@CMDIChildWnd@@KGPBUAFX_MSGMAP@@XZ 5f8115ad f
 0001:000105b3       ?DefWindowProcW@CMDIFrameWnd@@MAEJIIJ@Z 5f8115b3 f
 0001:000105d1       ?OnCmdMsg@CMDIFrameWnd@@UAEHIHPAXPAUAFX_CMDHANDLERINFO@@@Z 5f8115d1 f
 0001:00010662       ?MDIGetActive@CMDIFrameWnd@@QBEPAVCMDIChildWnd@@PAH@Z 5f811662 f
 0001:000106a5       ?GetMessageMap@CMDIChildWnd@@MBEPBUAFX_MSGMAP@@XZ 5f8116a5 f
 0001:000106ab       ?PreTranslateMessage@CMDIFrameWnd@@UAEHPAUtagMSG@@@Z 5f8116ab f
 0001:0001076d       ?PreTranslateMessage@CMDIChildWnd@@UAEHPAUtagMSG@@@Z 5f81176d f
 0001:000107c8       ?SetText@CCmdUI@@UAEXPBG@Z 5f8117c8 f
 0001:00010812       ?PreTranslateInput@CWnd@@QAEHPAUtagMSG@@@Z 5f811812 f
 0001:00010842       ??0CPoint@@QAE@UtagPOINT@@@Z 5f811842 f
 0001:00010854       ?QueryInterface@XClassFactory@COleObjectFactory@@UAGJABU_GUID@@PAPAX@Z 5f811854 f
 0001:0001086b       ?GetInterfaceMap@COleObjectFactory@@MBEPBUAFX_INTERFACEMAP@@XZ 5f81186b f
 0001:00010871       ?Release@XClassFactory@COleObjectFactory@@UAGKXZ 5f811871 f
 0001:00010880       __imp_load__CoRevokeClassObject@4 5f811880 f
 0001:0001088c       ?Release@COleDispatchImpl@@UAGKXZ 5f81188c f
 0001:0001089b       ?PreTranslateMessage@CDialog@@UAEHPAUtagMSG@@@Z 5f81189b f
 0001:000108ec       ?IsDialogMessageW@CWnd@@QAEHPAUtagMSG@@@Z 5f8118ec f
 0001:0001090a       ?GetInterfaceMap@CCmdTarget@@MBEPBUAFX_INTERFACEMAP@@XZ 5f81190a f
 0001:00010910       ?QueryInterface@COleDispatchImpl@@UAGJABU_GUID@@PAPAX@Z 5f811910 f
 0001:00010927       ?RunEmbedded@CWinApp@@QAEHXZ 5f811927 f
 0001:00010946       ?_AfxParseOption@@YGHPAGPBG@Z 5f811946 f
 0001:000109b5       ?EnableAutomation@CCmdTarget@@QAEXXZ 5f8119b5 f
 0001:000109bd       ?AddRef@COleDispatchImpl@@UAGKXZ 5f8119bd f
 0001:000109cc       ?RunAutomated@CWinApp@@QAEHXZ 5f8119cc f
 0001:000109e4       ?AfxOleRegisterServerClass@@YGHABU_GUID@@PBG11W4OLE_APPTYPE@@PAPBG3H1@Z 5f8119e4 f
 0001:00010a0d       ?Find@CString@@QBEHG@Z     5f811a0d f
 0001:00010a1b       ?Find@CString@@QBEHGH@Z    5f811a1b f
 0001:00010a34       ?OnUpdateContextHelp@CFrameWnd@@IAEXPAVCCmdUI@@@Z 5f811a34 f
 0001:00010a63       ??4CString@@QAEABV0@PBD@Z  5f811a63 f
 0001:00010aa3       ?DefWindowProcW@CMDIChildWnd@@MAEJIIJ@Z 5f811aa3 f
 0001:00010abb       ?GetInterfaceMap@COleDropTarget@@MBEPBUAFX_INTERFACEMAP@@XZ 5f811abb f
 0001:00010ac1       ?QueryInterface@XDropTarget@COleDropTarget@@UAGJABU_GUID@@PAPAX@Z 5f811ac1 f
 0001:00010ad8       ?_GetBaseInterfaceMap@COleServerItem@@KGPBUAFX_INTERFACEMAP@@XZ 5f811ad8 f
 0001:00010ade       ?Release@XDropTarget@COleDropTarget@@UAGKXZ 5f811ade f
 0001:00010aed       ?GetMDIFrame@CMDIChildWnd@@QAEPAVCMDIFrameWnd@@XZ 5f811aed f
 0001:00010b04       ?OnUpdateFrameTitle@CMDIFrameWnd@@UAEXH@Z 5f811b04 f
 0001:00010bbe       ?OnMDIActivate@CMDIChildWnd@@IAEXHPAVCWnd@@0@Z 5f811bbe f
 0001:00010c74       ?UpdateClientEdge@CMDIChildWnd@@IAEHPAUtagRECT@@@Z 5f811c74 f
 0001:00010cf2       ?OnUpdateFrameTitle@CMDIChildWnd@@MAEXH@Z 5f811cf2 f
 0001:00010d63       ?OnUpdateFrameMenu@CMDIChildWnd@@UAEXHPAVCWnd@@PAUHMENU__@@@Z 5f811d63 f
 0001:00010def       ?OnNcActivate@CMDIChildWnd@@IAEHH@Z 5f811def f
 0001:00010df7       ?GetActiveFrame@CMDIFrameWnd@@UAEPAVCFrameWnd@@XZ 5f811df7 f
 0001:00010e0b       ?OnIdleUpdateCmdUI@CMDIFrameWnd@@IAEXXZ 5f811e0b f
 0001:00010e2c       ??0COleDataObject@@QAE@XZ  5f811e2c f
 0001:00010e40       ?AttachClipboard@COleDataObject@@QAEHXZ 5f811e40 f
 0001:00010e47       ?IsDataAvailable@COleDataObject@@QAEHGPAUtagFORMATETC@@@Z 5f811e47 f
 0001:00010e6a       ?Release@COleDataObject@@QAEXXZ 5f811e6a f
 0001:00010e86       ?GetFirstDocPosition@CMultiDocTemplate@@UBEPAU__POSITION@@XZ 5f811e86 f
 0001:00010e8a       ?GetNextDoc@CMultiDocTemplate@@UBEPAVCDocument@@AAPAU__POSITION@@@Z 5f811e8a f
 0001:00010e9a       ?OnCommand@CMDIFrameWnd@@MAEHIJ@Z 5f811e9a f
 0001:00010ed7       ?SaveAllModified@CWinApp@@UAEHXZ 5f811ed7 f
 0001:00010eea       ?SaveAllModified@CDocManager@@UAEHXZ 5f811eea f
 0001:00010f0f       ?SaveAllModified@CDocTemplate@@UAEHXZ 5f811f0f f
 0001:00010f4b       ?UpdateModifiedFlag@COleDocument@@UAEXXZ 5f811f4b f
 0001:00010f73       ?PreCloseFrame@COleDocument@@UAEXPAVCFrameWnd@@@Z 5f811f73 f
 0001:00010fca       ?GetInPlaceActiveItem@COleDocument@@UAEPAVCOleClientItem@@PAVCWnd@@@Z 5f811fca f
 0001:00011012       ?DestroyWindow@CMDIChildWnd@@UAEHXZ 5f812012 f
 0001:0001107b       ?MDIDestroy@CMDIChildWnd@@QAEXXZ 5f81207b f
 0001:000110a2       ?OnDestroy@CMDIChildWnd@@IAEXXZ 5f8120a2 f
 0001:000110b5       ?Revoke@COleDropTarget@@UAEXXZ 5f8120b5 f
 0001:000110ef       __imp_load__RevokeDragDrop@4 5f8120ef f
 0001:000110fb       ??1COleDropTarget@@UAE@XZ  5f8120fb f
 0001:00011138       ??_GCMDIFrameWnd@@UAEPAXI@Z 5f812138 f
 0001:00011138       ??_ECMDIFrameWnd@@UAEPAXI@Z 5f812138 f
 0001:00011154       ?RemoveDocument@CMultiDocTemplate@@UAEXPAVCDocument@@@Z 5f812154 f
 0001:0001117c       ?OnDestroy@CMDIFrameWnd@@IAEXXZ 5f81217c f
 0001:000111a2       ??1CMultiDocTemplate@@UAE@XZ 5f8121a2 f
 0001:000111eb       ?Format@CString@@QAAXPBGZZ 5f8121eb f
 0001:000111fe       ?FormatV@CString@@QAEXPBGPAD@Z 5f8121fe f
 0001:0001146c       __imp_load__CoRegisterClassObject@20 5f81246c f
 0001:00011478       ?AddRef@XClassFactory@COleObjectFactory@@UAGKXZ 5f812478 f
 0001:00011489       ?UpdateRegistryAll@COleObjectFactory@@SGHH@Z 5f812489 f
 0001:000114f1       ?UpdateRegistry@COleObjectFactory@@MAEHH@Z 5f8124f1 f
 0001:00011505       ?UpdateRegistry@COleObjectFactory@@QAEXPBG@Z 5f812505 f
 0001:0001152d       ?AfxOleRegisterServerClass@@YGHABU_GUID@@PBG11W4OLE_APPTYPE@@PAPBG3H11@Z 5f81252d f
 0001:000115e5       ??0CAfxOleSymbolTable@@QAE@H@Z 5f8125e5 f
 0001:00011612       ?_AfxOleMakeSymbolTable@@YGHAAVCAfxOleSymbolTable@@ABU_GUID@@PBG22H22@Z 5f812612 f
 0001:00011799       __imp_load__StringFromCLSID@8 5f812799 f
 0001:000117a5       ?SetAt@CAfxOleSymbolTable@@QAEXHPBG@Z 5f8127a5 f
 0001:000117db       ?AfxGetModuleShortFileName@@YGXPAUHINSTANCE__@@AAVCString@@@Z 5f8127db f
 0001:0001182a       ?AfxOleRegisterHelper@@YGHPBQBG0HHPAUHKEY__@@@Z 5f81282a f
 0001:0001196a       __imp_load__RegOpenKeyW@12 5f81296a f
 0001:00011976       __imp_load__RegQueryValueW@16 5f812976 f
 0001:00011982       __imp_load__RegSetValueW@20 5f812982 f
 0001:0001198e       ??1CAfxOleSymbolTable@@QAE@XZ 5f81298e f
 0001:000119b6       ??0CMultiDocTemplate@@QAE@IPAUCRuntimeClass@@00@Z 5f8129b6 f
 0001:00011a1f       ?LoadTemplate@CMultiDocTemplate@@UAEXXZ 5f812a1f f
 0001:00011a65       ?AddDocTemplate@CWinApp@@QAEXPAVCDocTemplate@@@Z 5f812a65 f
 0001:00011ac1       ??0CMDIFrameWnd@@QAE@XZ    5f812ac1 f
 0001:00011ada       ?LoadFrame@CMDIFrameWnd@@UAEHIKPAVCWnd@@PAUCCreateContext@@@Z 5f812ada f
 0001:00011b09       ?PreCreateWindow@CMDIFrameWnd@@UAEHAAUtagCREATESTRUCTW@@@Z 5f812b09 f
 0001:00011b29       ?OnCreateClient@CMDIFrameWnd@@UAEHPAUtagCREATESTRUCTW@@PAUCCreateContext@@@Z 5f812b29 f
 0001:00011b75       ?CreateClient@CMDIFrameWnd@@UAEHPAUtagCREATESTRUCTW@@PAVCMenu@@@Z 5f812b75 f
 0001:00011c11       ?EnableShellOpen@CWinApp@@IAEXXZ 5f812c11 f
 0001:00011c3b       ?UpdateRegistry@COleTemplateServer@@QAEXW4OLE_APPTYPE@@PAPBG1@Z 5f812c3b f
 0001:00011dad       ?GetFirstDocTemplatePosition@CWinApp@@QBEPAU__POSITION@@XZ 5f812dad f
 0001:00011dc0       ?GetNextDocTemplate@CWinApp@@QBEPAVCDocTemplate@@AAPAU__POSITION@@@Z 5f812dc0 f
 0001:00011dd2       __imp_load__ExtractIconW@12 5f812dd2 f
 0001:00011dde       ?RegisterShellFileTypes@CWinApp@@IAEXH@Z 5f812dde f
 0001:00011df0       ?RegisterShellFileTypes@CDocManager@@UAEXH@Z 5f812df0 f
 0001:000121fd       ?_AfxSetRegKey@@YGHPBG00@Z 5f8131fd f
 0001:0001228b       ??YCString@@QAEABV0@PBG@Z  5f81328b f
 0001:000122b2       __imp_load__RegCreateKeyW@12 5f8132b2 f
 0001:000122be       ?OnFileNew@CWinApp@@IAEXXZ 5f8132be f
 0001:000122d1       ?OnFileNew@CDocManager@@UAEXXZ 5f8132d1 f
 0001:0001231a       ?OpenDocumentFile@CMultiDocTemplate@@UAEPAVCDocument@@PBGH@Z 5f81331a f
 0001:000123ad       ?AddDocument@CMultiDocTemplate@@UAEXPAVCDocument@@@Z 5f8133ad f
 0001:000123c9       ?CreateObject@CMDIChildWnd@@SGPAVCObject@@XZ 5f8133c9 f
 0001:000123fe       ??0CMDIChildWnd@@QAE@XZ    5f8133fe f
 0001:0001241e       ?LoadFrame@CMDIChildWnd@@UAEHIKPAVCWnd@@PAUCCreateContext@@@Z 5f81341e f
 0001:000124ed       ?PreCreateWindow@CMDIChildWnd@@UAEHAAUtagCREATESTRUCTW@@@Z 5f8134ed f
 0001:000124f9       ?Create@CMDIChildWnd@@UAEHPBG0KABUtagRECT@@PAVCMDIFrameWnd@@PAUCCreateContext@@@Z 5f8134f9 f
 0001:00012609       ?OnNcCreate@CMDIChildWnd@@IAEHPAUtagCREATESTRUCTW@@@Z 5f813609 f
 0001:00012638       ?OnCreate@CMDIChildWnd@@IAEHPAUtagCREATESTRUCTW@@@Z 5f813638 f
 0001:0001264a       ??0CScrollView@@IAE@XZ     5f81364a f
 0001:00012671       ??0COleDropTarget@@QAE@XZ  5f813671 f
 0001:00012711       ?Register@COleDropTarget@@QAEHPAVCWnd@@@Z 5f813711 f
 0001:0001276d       ?AddRef@XDropTarget@COleDropTarget@@UAGKXZ 5f81376d f
 0001:0001277c       __imp_load__RegisterDragDrop@8 5f81377c f
 0001:00012788       ?SetScrollSizes@CScrollView@@QAEXHUtagSIZE@@ABU2@1@Z 5f813788 f
 0001:000128bd       ?UpdateBars@CScrollView@@IAEXXZ 5f8138bd f
 0001:000129a8       ?GetTrueClientSize@CScrollView@@IAEHAAVCSize@@0@Z 5f8139a8 f
 0001:00012a20       ?GetScrollBarSizes@CScrollView@@IAEXAAVCSize@@@Z 5f813a20 f
 0001:00012a7d       ?GetRuntimeClass@CMDIChildWnd@@UBEPAUCRuntimeClass@@XZ 5f813a7d f
 0001:00012a83       ?_GetBaseClass@COleIPFrameWnd@@KGPAUCRuntimeClass@@XZ 5f813a83 f
 0001:00012a89       ?OnPrepareDC@CScrollView@@UAEXPAVCDC@@PAUCPrintInfo@@@Z 5f813a89 f
 0001:00012af9       ?GetDeviceScrollPosition@CScrollView@@QBE?AVCPoint@@XZ 5f813af9 f
 0001:00012b31       ?OnPrepareDC@CView@@UAEXPAVCDC@@PAUCPrintInfo@@@Z 5f813b31 f
 0001:00012b40       ?SetViewportExt@CDC@@UAE?AVCSize@@HH@Z 5f813b40 f
 0001:00012b83       ?SetWindowExt@CDC@@UAE?AVCSize@@HH@Z 5f813b83 f
 0001:00012bc6       ?LPtoDP@CDC@@QBEXPAUtagSIZE@@@Z 5f813bc6 f
 0001:00012c2f       _abs                       5f813c2f f
 0001:00012c35       ?OnSize@CScrollView@@QAEXIHH@Z 5f813c35 f
 0001:00012c52       ?OnWindowPosChanging@CMDIChildWnd@@IAEXPAUtagWINDOWPOS@@@Z 5f813c52 f
 0001:00012c7f       ?OnSize@CMDIChildWnd@@IAEXIHH@Z 5f813c7f f
 0001:00012caa       ?CalcWindowRect@CScrollView@@UAEXPAUtagRECT@@I@Z 5f813caa f
 0001:00012ce2       ?GetScrollBarState@CScrollView@@IAEXVCSize@@AAV2@1AAVCPoint@@H@Z 5f813ce2 f
 0001:00012d7f       ?ScrollToDevicePosition@CScrollView@@IAEXUtagPOINT@@@Z 5f813d7f f
 0001:00012dd1       ?SetScrollPos@CWnd@@QAEHHHH@Z 5f813dd1 f
 0001:00012dfe       ?ScrollWindow@CWnd@@QAEXHHPBUtagRECT@@0@Z 5f813dfe f
 0001:00012e55       ?EnableScrollBarCtrl@CWnd@@QAEXHH@Z 5f813e55 f
 0001:00012e89       ?SetDefaultTitle@CMultiDocTemplate@@UAEXPAVCDocument@@@Z 5f813e89 f
 0001:00012f13       ?ActivateFrame@CMDIChildWnd@@UAEXH@Z 5f813f13 f
 0001:00012fc0       ?GetDefaultMenu@COleServerDoc@@MAEPAUHMENU__@@XZ 5f813fc0 f
 0001:00012fe4       ?GetWindowMenuPopup@CMDIFrameWnd@@UAEPAUHMENU__@@PAU2@@Z 5f813fe4 f
 0001:00013052       ?OnQueryNewPalette@CFrameWnd@@IAEHXZ 5f814052 f
 0001:00013069       ?OnSize@CMDIFrameWnd@@IAEXIHH@Z 5f814069 f
 0001:0001307d       ?OnPaint@CView@@IAEXXZ     5f81407d f
 0001:000130d1       ?RectVisible@CDC@@UBEHPBUtagRECT@@@Z 5f8140d1 f
 0001:000130e1       ?GetMessageBar@CMDIChildWnd@@MAEPAVCWnd@@XZ 5f8140e1 f
 0001:000130f0       ?PreTranslateMessage@CControlBar@@UAEHPAUtagMSG@@@Z 5f8140f0 f
 0001:0001318e       ?DDX_Control@@YGXPAVCDataExchange@@HAAVCWnd@@@Z 5f81418e f
 0001:000131d3       ?HandleInComingCall@XMessageFilter@COleMessageFilter@@UAGKKPAUHTASK__@@KPAUtagINTERFACEINFO@@@Z 5f8141d3 f
 0001:00013222       ?InvokeHelperV@COleDispatchDriver@@QAEXJGGPAXPBEPAD@Z 5f814222 f
 0001:0001346d       ?AfxVariantInit@@YGXPAUtagVARIANT@@@Z 5f81446d f
 0001:00013480       ?Invoke@COleDispatchImpl@@UAGJJABU_GUID@@KGPAUtagDISPPARAMS@@PAUtagVARIANT@@PAUtagEXCEPINFO@@PAI@Z 5f814480 f
 0001:0001367b       ?IsInvokeAllowed@CCmdTarget@@UAEHJ@Z 5f81467b f
 0001:00013681       ?GetDispEntry@CCmdTarget@@IAGPBUAFX_DISPMAP_ENTRY@@J@Z 5f814681 f
 0001:000136f7       ?GetEntryCount@CCmdTarget@@KGIPBUAFX_DISPMAP@@@Z 5f8146f7 f
 0001:00013726       ?CallMemberFunc@CCmdTarget@@IAEJPBUAFX_DISPMAP_ENTRY@@GPAUtagVARIANT@@PAUtagDISPPARAMS@@PAI@Z 5f814726 f
 0001:0001390b       ?GetStackSize@CCmdTarget@@KGIPBEG@Z 5f81490b f
 0001:0001394e       ?PushStackArgs@CCmdTarget@@IAEJPAEPBEPAXGPAUtagDISPPARAMS@@PAIPAUtagVARIANT@@@Z 5f81494e f
 0001:00013a58       __AfxDispatchCall@12       5f814a58 f
 0001:00013a69       ?InvokeHelper@COleDispatchDriver@@QAAXJGGPAXPBEZZ 5f814a69 f
 0001:00013a89       ?ContinueModal@CWnd@@UAEHXZ 5f814a89 f
 0001:00013b74       ?OnOK@CDialog@@MAEXXZ      5f814b74 f
 0001:00013b8d       ?EndDialog@CDialog@@QAEXH@Z 5f814b8d f
 0001:00013bb0       ?EndModalLoop@CWnd@@UAEXH@Z 5f814bb0 f
 0001:00013bd4       ?OnFinalRelease@CWnd@@UAEXXZ 5f814bd4 f
 0001:00013be6       ?ReleaseDispatch@COleDispatchDriver@@QAEXXZ 5f814be6 f
 0001:00013c00       ??1CEdit@@UAE@XZ           5f814c00 f
 0001:00013c38       ??1CStatic@@UAE@XZ         5f814c38 f
 0001:00013c70       ??0COleDispatchDriver@@QAE@XZ 5f814c70 f
 0001:00013c7d       ?DoModal@CDialog@@UAEHXZ   5f814c7d f
 0001:00013d90       ?PrepareCtrl@CDataExchange@@QAEPAUHWND__@@H@Z 5f814d90 f
 0001:00013dbe       ?GetDlgItem@CWnd@@QBEXHPAPAUHWND__@@@Z 5f814dbe f
 0001:00013ddf       ?CreateDispatch@COleDispatchDriver@@QAEHABU_GUID@@PAVCOleException@@@Z 5f814ddf f
 0001:00013e63       __imp_load__CoCreateInstance@20 5f814e63 f
 0001:00013e6f       __imp_load__OleRun@4       5f814e6f f
 0001:00013e7b       ?CreateInstance@XClassFactory@COleObjectFactory@@UAGJPAUIUnknown@@ABU_GUID@@PAPAX@Z 5f814e7b f
 0001:00013e98       ?CreateInstanceLic@XClassFactory@COleObjectFactory@@UAGJPAUIUnknown@@0ABU_GUID@@PAGPAPAX@Z 5f814e98 f
 0001:00013f7c       ?IsLicenseValid@COleObjectFactory@@QAEHXZ 5f814f7c f
 0001:00013f97       ?VerifyUserLicense@COleObjectFactory@@MAEHXZ 5f814f97 f
 0001:00013f9b       ?OnCreateObject@COleObjectFactory@@MAEPAVCCmdTarget@@XZ 5f814f9b f
 0001:00013fb2       ?_AfxQueryInterface@@YGPAUIUnknown@@PAU1@ABU_GUID@@@Z 5f814fb2 f
 0001:00013fd6       ?SetProperty@COleDispatchDriver@@QAAXJGZZ 5f814fd6 f
 0001:00014014       __imp_load__VariantClear@4 5f815014 f
 0001:0001401b       __tailMerge_OLEAUT32       5f81501b f
 0001:00014029       ?GetProperty@COleDispatchDriver@@QBEXJGPAX@Z 5f815029 f
 0001:00014045       __imp_load__VariantChangeType@16 5f815045 f
 0001:0001404e       ?RunModalLoop@CWnd@@QAEHK@Z 5f81504e f
 0001:00014161       __imp_load__SysAllocString@4 5f815161 f
 0001:0001416d       ?MessagePending@XMessageFilter@COleMessageFilter@@UAGKPAUHTASK__@@KK@Z 5f81516d f
 0001:000141e1       ?OnMessagePending@COleMessageFilter@@UAEHPBUtagMSG@@@Z 5f8151e1 f
 0001:0001422e       ??1CThreadLocalObject@@QAE@XZ 5f81522e f
 0001:00014251       ??1CProcessLocalObject@@QAE@XZ 5f815251 f
 0001:0001427d       ??1AFX_MODULE_STATE@@UAE@XZ 5f81527d f
 0001:000142db       ?FreeSlot@CThreadSlotData@@QAEXH@Z 5f8152db f
 0001:00014338       __imp_load__RegSetValueExW@24 5f815338 f
 0001:00014344       ??1CCommandLineInfo@@UAE@XZ 5f815344 f
 0001:000143c1       ??1CFixedAlloc@@QAE@XZ     5f8153c1 f
 0001:000143d5       ?FreeAll@CFixedAlloc@@QAEXXZ 5f8153d5 f
 0001:00014479       ??_G_AFX_BASE_MODULE_STATE@@UAEPAXI@Z 5f815479 f
 0001:00014479       ??_E_AFX_BASE_MODULE_STATE@@UAEPAXI@Z 5f815479 f
 0001:000144bc       ?AfxCriticalTerm@@YGXXZ    5f8154bc f
 0001:0001450c       ?AfxTlsRelease@@YGXXZ      5f81550c f
 0001:00014534       ??1CThreadSlotData@@QAE@XZ 5f815534 f
 0001:0001458b       ?AfxOleCanExitApp@@YGHXZ   5f81558b f
 0001:0001459b       ?AfxPostQuitMessage@@YGXH@Z 5f81559b f
 0001:000145be       ?AfxOleTerm@@YGXH@Z        5f8155be f
 0001:00014619       ?FlushClipboard@COleDataSource@@SGXXZ 5f815619 f
 0001:00014627       ?GetClipboardOwner@COleDataSource@@SGPAV1@XZ 5f815627 f
 0001:00014648       ?CreateObject@?$CProcessLocal@V_AFX_OLE_STATE@@@@SGPAVCNoTrackObject@@XZ 5f815648 f
 0001:00014679       ??0_AFX_OLE_STATE@@QAE@XZ  5f815679 f
 0001:00014682       ?RevokeAll@COleObjectFactory@@SGXXZ 5f815682 f
 0001:000146d7       ?Revoke@COleObjectFactory@@QAEXXZ 5f8156d7 f
 0001:000146fa       ?AfxOleUnlockAllControls@@YGXXZ 5f8156fa f
 0001:00014724       ?Disconnect@COleDispatchImpl@@UAEXXZ 5f815724 f
 0001:00014727       ?ExternalDisconnect@CCmdTarget@@QAEXXZ 5f815727 f
 0001:00014754       ?ExitInstance@CWinApp@@UAEHXZ 5f815754 f
 0001:0001478a       ?SaveStdProfileSettings@CWinApp@@IAEXXZ 5f81578a f
 0001:000147ac       ?AfxWinTerm@@YGXXZ         5f8157ac f
 0001:0001483b       ??_GCOleMessageFilter@@UAEPAXI@Z 5f81583b f
 0001:0001483b       ??_ECOleMessageFilter@@UAEPAXI@Z 5f81583b f
 0001:00014857       ??1COleMessageFilter@@UAE@XZ 5f815857 f
 0001:0001488f       ?Revoke@COleMessageFilter@@QAEXXZ 5f81588f f
 0001:000148a8       ?Release@XMessageFilter@COleMessageFilter@@UAGKXZ 5f8158a8 f
 0001:000148b7       __imp_load__CoFreeUnusedLibraries@0 5f8158b7 f
 0001:000148c3       __imp_load__OleUninitialize@0 5f8158c3 f
 0001:0001490c       ??1CWinApp@@UAE@XZ         5f81590c f
 0001:00014a2e       ??1COleObjectFactory@@UAE@XZ 5f815a2e f
 0001:00014a95       ??_ECDynLinkLibrary@@UAEPAXI@Z 5f815a95 f
 0001:00014a95       ??_GCDynLinkLibrary@@UAEPAXI@Z 5f815a95 f
 0001:00014ab1       ??1CDynLinkLibrary@@UAE@XZ 5f815ab1 f
 0001:00014b01       ?AfxTermExtensionModule@@YGXAAUAFX_EXTENSION_MODULE@@H@Z 5f815b01 f
 0001:00014b43       ?AfxTermLocalData@@YGXPAUHINSTANCE__@@H@Z 5f815b43 f
 0001:00014b5d       ?AfxResetMsgCache@@YGXXZ   5f815b5d f
 0001:00014bae       ?AfxEditviewTerm@@YAXXZ    5f815bae f
 0001:00014bbe       ??1AUX_DATA@@QAE@XZ        5f815bbe f
 0001:00014bc8       ?AfxWingdixTerm@@YAXXZ     5f815bc8 f
 0001:00014bd8       ??1CUserException@@UAE@XZ  5f815bd8 f
 0001:00014be5       ??1CMemoryException@@UAE@XZ 5f815be5 f
 0001:00014beb       ??1CSimpleException@@UAE@XZ 5f815beb f
 0001:00014bf7       ??1CResourceException@@UAE@XZ 5f815bf7 f
 0001:00014c09       ?AfxTrackerTerm@@YAXXZ     5f815c09 f
 0001:00014c1e       ?_AfxWinminiTerm@@YAXXZ    5f815c1e f
 0001:00014c92       ??1CNotSupportedException@@UAE@XZ 5f815c92 f
 0001:00014cb1       ??_E_AFX_OLE_STATE@@UAEPAXI@Z 5f815cb1 f
 0001:00014cb1       ??_G_AFX_OLE_STATE@@UAEPAXI@Z 5f815cb1 f
 0001:00014ccc       ??1_AFX_OLE_STATE@@UAE@XZ  5f815ccc f
 0001:00014ce7       ??_G_AFX_CTL3D_STATE@@UAEPAXI@Z 5f815ce7 f
 0001:00014ce7       ??_E_AFX_CTL3D_STATE@@UAEPAXI@Z 5f815ce7 f
 0001:00014d02       ??1_AFX_CTL3D_STATE@@UAE@XZ 5f815d02 f
 0001:00014d8b       ??1CSessionMapPtrToPtr@@UAE@XZ 5f815d8b f
 0001:00014dda       ??1CSyncObject@@UAE@XZ     5f815dda f
 0001:00014df6       __imp_load__CoDisconnectObject@8 5f815df6 f
 0001:00014e02       ??_G_AFX_WIN_STATE@@UAEPAXI@Z 5f815e02 f
 0001:00014e02       ??_E_AFX_WIN_STATE@@UAEPAXI@Z 5f815e02 f
 0001:00014e1d       ??1_AFX_WIN_STATE@@UAE@XZ  5f815e1d f
 0001:00014e4a       ?OnAppExit@CWinApp@@IAEXXZ 5f815e4a f
 0001:00014e5d       ?OnClose@CFrameWnd@@IAEXXZ 5f815e5d f
 0001:00014f03       ?HideApplication@CWinApp@@QAEXXZ 5f815f03 f
 0001:00014f35       ?CloseAllDocuments@CWinApp@@QAEXH@Z 5f815f35 f
 0001:00014f4b       ?CloseAllDocuments@CDocManager@@UAEXH@Z 5f815f4b f
 0001:00014f6c       ?CloseAllDocuments@CDocTemplate@@UAEXH@Z 5f815f6c f
 0001:00014f9f       ?OnCloseDocument@COleServerDoc@@UAEXXZ 5f815f9f f
 0001:00015031       ?NotifyAllItems@COleServerDoc@@IAEXW4OLE_NOTIFICATION@@K@Z 5f816031 f
 0001:0001505b       ?OnCloseDocument@COleLinkingDoc@@UAEXXZ 5f81605b f
 0001:000150b0       ?OnCloseDocument@COleDocument@@UAEXXZ 5f8160b0 f
 0001:000150d4       ?OnCloseDocument@CDocument@@UAEXXZ 5f8160d4 f
 0001:00015123       ?OnDestroy@CFrameWnd@@IAEXXZ 5f816123 f
 0001:00015170       ?DestroyDockBars@CFrameWnd@@QAEXXZ 5f816170 f
 0001:000151f5       ?OnDestroy@CView@@IAEXXZ   5f8161f5 f
 0001:00015224       ?PostNcDestroy@CView@@MAEXXZ 5f816224 f
 0001:00015230       ??1CScrollView@@UAE@XZ     5f816230 f
 0001:00015236       ??1CView@@UAE@XZ           5f816236 f
 0001:00015276       ?RemoveView@CDocument@@QAEXPAVCView@@@Z 5f816276 f
 0001:000152a5       ?Find@CObList@@QBEPAU__POSITION@@PAVCObject@@PAU2@@Z 5f8162a5 f
 0001:000152c8       ?RemoveAt@CObList@@QAEXPAU__POSITION@@@Z 5f8162c8 f
 0001:000152ff       ?FreeNode@CObList@@IAEXPAUCNode@1@@Z 5f8162ff f
 0001:0001531a       ?PostNcDestroy@CFrameWnd@@MAEXXZ 5f81631a f
 0001:00015326       ??1CFrameWnd@@UAE@XZ       5f816326 f
 0001:0001538a       ?RemoveFrameWnd@CFrameWnd@@IAEXXZ 5f81638a f
 0001:000153ab       ??1CObList@@UAE@XZ         5f8163ab f
 0001:000153de       ??1COleServerDoc@@UAE@XZ   5f8163de f
 0001:00015485       ??1COleLinkingDoc@@UAE@XZ  5f816485 f
 0001:000154dd       ?DisconnectViews@CDocument@@QAEXXZ 5f8164dd f
 0001:000154ec       ?GetInterfaceMap@COleLinkingDoc@@MBEPBUAFX_INTERFACEMAP@@XZ 5f8164ec f
 0001:000154f2       ?QueryInterface@XPersistFile@COleLinkingDoc@@UAGJABU_GUID@@PAPAX@Z 5f8164f2 f
 0001:0001550c       ?Release@XPersistFile@COleLinkingDoc@@UAGKXZ 5f81650c f
 0001:0001551e       ??1COleDocument@@UAE@XZ    5f81651e f
 0001:0001558b       ?AfxOleUnlockApp@@YGXXZ    5f81658b f
 0001:000155a2       ?AfxOleOnReleaseAllObjects@@YGXXZ 5f8165a2 f
 0001:000155b2       ??1CDocument@@UAE@XZ       5f8165b2 f
 0001:0001561e       ?RemoveDocument@CDocTemplate@@UAEXPAVCDocument@@@Z 5f81661e f
 0001:00015629       ?DestroyWindow@CControlBar@@UAEHXZ 5f816629 f
 0001:00015649       ?IsFloating@CControlBar@@QBEHXZ 5f816649 f
 0001:00015661       ?OnDestroy@CControlBar@@QAEXXZ 5f816661 f
 0001:0001568f       ?RemoveControlBar@CFrameWnd@@QAEXPAVCControlBar@@@Z 5f81668f f
 0001:000156b0       ?PostNcDestroy@CControlBar@@UAEXXZ 5f8166b0 f
 0001:000156c2       ??_GCDockBar@@UAEPAXI@Z    5f8166c2 f
 0001:000156c2       ??_ECDockBar@@UAEPAXI@Z    5f8166c2 f
 0001:000156de       ??1CDockBar@@UAE@XZ        5f8166de f
 0001:0001574f       ??1CControlBarInfo@@QAE@XZ 5f81674f f
 0001:00015752       ??1CPtrArray@@UAE@XZ       5f816752 f
 0001:00015789       ??1CControlBar@@UAE@XZ     5f816789 f
 0001:0001580b       ??1CToolBar@@UAE@XZ        5f81680b f
 0001:0001585c       ??1CDockContext@@QAE@XZ    5f81685c f
 0001:00015871       ??1CStatusBar@@UAE@XZ      5f816871 f
 0001:000158ac       ?WriteList@CRecentFileList@@UAEXXZ 5f8168ac f
 0001:0001592d       ?WriteProfileStringW@CWinApp@@QAEHPBG00@Z 5f81692d f
 0001:000159c4       ??_ECDocManager@@UAEPAXI@Z 5f8169c4 f
 0001:000159ef       ??1CDocManager@@UAE@XZ     5f8169ef f
 0001:00015a62       ??1CSingleDocTemplate@@UAE@XZ 5f816a62 f
 0001:00015a68       ??1CDocTemplate@@UAE@XZ    5f816a68 f
 0001:00015ac9       ??_ECRecentFileList@@UAEPAXI@Z 5f816ac9 f
 0001:00015ac9       ??_GCRecentFileList@@UAEPAXI@Z 5f816ac9 f
 0001:00015ae5       ??1CRecentFileList@@UAE@XZ 5f816ae5 f
 0001:00015b42       ??_ECString@@QAEPAXI@Z     5f816b42 f
 0001:00015b7a       ??_M@YGXPAXIHP6EX0@Z@Z     5f816b7a f
 0001:00015bed       ?CanCloseFrame@COleServerDoc@@UAEHPAVCFrameWnd@@@Z 5f816bed f
 0001:00015c12       ?CanCloseFrame@CDocument@@UAEHPAVCFrameWnd@@@Z 5f816c12 f
 0001:00015c5a       ?GetDockState@CFrameWnd@@QBEXAAVCDockState@@@Z 5f816c5a f
 0001:00015cd5       ?GetBarInfo@CControlBar@@QAEXPAVCControlBarInfo@@@Z 5f816cd5 f
 0001:00015d9d       ?GetBarInfo@CDockBar@@QAEXPAVCControlBarInfo@@@Z 5f816d9d f
 0001:00015e24       ?PreCloseFrame@CRichEditDoc@@UAEXPAVCFrameWnd@@@Z 5f816e24 f
 0001:00015e85       ?OnDestroy@CRichEditView@@IAEXXZ 5f816e85 f
 0001:00015e9e       ?Release@XRichEditOleCallback@CRichEditView@@UAGKXZ 5f816e9e f
 0001:00015eb0       ??1CDWordArray@@UAE@XZ     5f816eb0 f
 0001:00015ee7       ??1CComboBox@@UAE@XZ       5f816ee7 f
 0001:00015f1f       ?RemoveDocument@CSingleDocTemplate@@UAEXPAVCDocument@@@Z 5f816f1f f
 0001:00015f33       ?WriteProfileInt@CWinApp@@QAEHPBG0H@Z 5f816f33 f
 0001:00015f82       ?WriteProfileBinary@CWinApp@@QAEHPBG0PAEI@Z 5f816f82 f
 0001:00015fd0       ??6CArchive@@QAEAAV0@M@Z   5f816fd0 f
 0001:00015ff8       ?GetScreenSize@CDockState@@QAE?AVCSize@@XZ 5f816ff8 f
 0001:00016012       ?Write@CArchive@@QAEXPBXI@Z 5f817012 f
 0001:00016051       ??6CArchive@@QAEAAV0@G@Z   5f817051 f
 0001:00016077       ?Realloc@CMemFile@@MAEPAEPAEK@Z 5f817077 f
 0001:0001608a       ?Read@CMemFile@@UAEIPAXI@Z 5f81708a f
 0001:000160cf       __imp_load__RegDeleteKeyW@8 5f8170cf f
 0001:000160db       ??1CDockState@@UAE@XZ      5f8170db f
 0001:00016144       ??_G_AFX_RICHEDIT_STATE@@UAEPAXI@Z 5f817144 f
 0001:00016144       ??_E_AFX_RICHEDIT_STATE@@UAEPAXI@Z 5f817144 f
 0001:0001615f       ??1_AFX_RICHEDIT_STATE@@UAE@XZ 5f81715f f
 0001:0001617f       ??1_AFX_EDIT_STATE@@UAE@XZ 5f81717f f
 0001:000161be       __alloca_probe             5f8171be  
 0001:000161be       __chkstk                   5f8171be  
 0001:000161ef       ??_ECObject@@UAEPAXI@Z     5f8171ef f
 0001:000161ef       ??_GCObject@@UAEPAXI@Z     5f8171ef f
 0001:0001620c       ??_ECMemoryException@@UAEPAXI@Z 5f81720c f
 0001:0001620c       ??_GCMemoryException@@UAEPAXI@Z 5f81720c f
 0001:00016228       ??_GCNotSupportedException@@UAEPAXI@Z 5f817228 f
 0001:00016228       ??_ECNotSupportedException@@UAEPAXI@Z 5f817228 f
 0001:00016244       ??6CArchive@@QAEAAV0@E@Z   5f817244 f
 0001:00016271       ??5CArchive@@QAEAAV0@AAE@Z 5f817271 f
 0001:000162b1       ??3CObject@@SGXPAX@Z       5f8172b1 f
 0001:000162be       ??_ECArchiveException@@UAEPAXI@Z 5f8172be f
 0001:000162be       ??_GCArchiveException@@UAEPAXI@Z 5f8172be f
 0001:000162da       ??1CArchiveException@@UAE@XZ 5f8172da f
 0001:00016310       ??_ECFileException@@UAEPAXI@Z 5f817310 f
 0001:00016310       ??_GCFileException@@UAEPAXI@Z 5f817310 f
 0001:0001632c       ?SetFilePath@CFile@@UAEXPBG@Z 5f81732c f
 0001:0001633b       ?GetAt@CStringArray@@QBE?AVCString@@H@Z 5f81733b f
 0001:00016377       ??_ECSyncObject@@UAEPAXI@Z 5f817377 f
 0001:00016377       ??_GCSyncObject@@UAEPAXI@Z 5f817377 f
 0001:000163a3       ?Lock@CSyncObject@@UAEHK@Z 5f8173a3 f
 0001:000163b8       ?Unlock@CSyncObject@@UAEHJPAJ@Z 5f8173b8 f
 0001:000163be       ??0CSemaphore@@QAE@JJPBGPAU_SECURITY_ATTRIBUTES@@@Z 5f8173be f
 0001:00016410       ??1CSemaphore@@UAE@XZ      5f817410 f
 0001:0001641b       ?Unlock@CSemaphore@@UAEHJPAJ@Z 5f81741b f
 0001:0001642f       ??0CMutex@@QAE@HPBGPAU_SECURITY_ATTRIBUTES@@@Z 5f81742f f
 0001:0001647e       ??1CMutex@@UAE@XZ          5f81747e f
 0001:00016489       ?Unlock@CMutex@@UAEHXZ     5f817489 f
 0001:00016493       ??0CEvent@@QAE@HHPBGPAU_SECURITY_ATTRIBUTES@@@Z 5f817493 f
 0001:000164e5       ??1CEvent@@UAE@XZ          5f8174e5 f
 0001:000164f0       ??0CSingleLock@@QAE@PAVCSyncObject@@H@Z 5f8174f0 f
 0001:00016517       ?Lock@CSingleLock@@QAEHK@Z 5f817517 f
 0001:0001652c       ?Unlock@CSingleLock@@QAEHXZ 5f81752c f
 0001:0001654e       ?Unlock@CSingleLock@@QAEHJPAJ@Z 5f81754e f
 0001:0001657a       ??0CMultiLock@@QAE@QAPAVCSyncObject@@KH@Z 5f81757a f
 0001:000165f2       ??1CMultiLock@@QAE@XZ      5f8175f2 f
 0001:00016613       ?Lock@CMultiLock@@QAEKKHK@Z 5f817613 f
 0001:0001667c       ?Unlock@CMultiLock@@QAEHXZ 5f81767c f
 0001:000166b2       ?Unlock@CMultiLock@@QAEHJPAJ@Z 5f8176b2 f
 0001:000166fc       ?Unlock@CSemaphore@@UAEHXZ 5f8176fc f
 0001:00016767       _xMonitorFromRect@8        5f817767 f
 0001:0001683f       ?BeginModalState@CWnd@@UAEXXZ 5f81783f f
 0001:0001684b       ?EndModalState@CWnd@@UAEXXZ 5f81784b f
 0001:0001685a       ?GetTitle@CFrameWnd@@QBE?AVCString@@XZ 5f81785a f
 0001:00016878       ?MDIActivate@CMDIChildWnd@@QAEXXZ 5f817878 f
 0001:0001689f       ??0CPoint@@QAE@K@Z         5f81789f f
 0001:000168b6       ?OnCancelMode@CWnd@@IAEXXZ 5f8178b6 f
 0001:000168bb       ?PtVisible@CDC@@UBEHHH@Z   5f8178bb f
 0001:000168cf       ?GrayStringW@CDC@@UAEHPAVCBrush@@P6GHPAUHDC__@@JH@ZJHHHHH@Z 5f8178cf f
 0001:000168ff       ?GetCurSel@CListBox@@QBEHXZ 5f8178ff f
 0001:00016912       ?LoadBitmapW@CBitmap@@QAEHI@Z 5f817912 f
 0001:00016936       ?GetFont@CWnd@@QBEPAVCFont@@XZ 5f817936 f
 0001:0001694c       ?GetTabControl@CPropertySheet@@QBEPAVCTabCtrl@@XZ 5f81794c f
 0001:00016965       ??H@YG?AVCString@@ABV0@D@Z 5f817965 f
 0001:00016985       ??_ECCommonDialog@@UAEPAXI@Z 5f817985 f
 0001:00016985       ??_GCCommonDialog@@UAEPAXI@Z 5f817985 f
 0001:000169a1       ??1CCommonDialog@@UAE@XZ   5f8179a1 f
 0001:000169a6       ?GetFaceName@CFontDialog@@QBE?AVCString@@XZ 5f8179a6 f
 0001:000169c4       ??_GCComboBoxEx@@UAEPAXI@Z 5f8179c4 f
 0001:000169c4       ??_ECComboBoxEx@@UAEPAXI@Z 5f8179c4 f
 0001:000169e0       ??_GCIPAddressCtrl@@UAEPAXI@Z 5f8179e0 f
 0001:000169e0       ??_ECIPAddressCtrl@@UAEPAXI@Z 5f8179e0 f
 0001:000169fc       ??_GCResourceException@@UAEPAXI@Z 5f8179fc f
 0001:000169fc       ??_ECResourceException@@UAEPAXI@Z 5f8179fc f
 0001:00016a18       ??_GCUserException@@UAEPAXI@Z 5f817a18 f
 0001:00016a18       ??_ECUserException@@UAEPAXI@Z 5f817a18 f
 0001:00016a34       ?TextOutW@CDC@@UAEHHHPBGH@Z 5f817a34 f
 0001:00016a50       ?TabbedTextOutW@CDC@@UAE?AVCSize@@HHPBGHHPAHH@Z 5f817a50 f
 0001:00016a88       ?DrawTextW@CDC@@UAEHPBGHPAUtagRECT@@I@Z 5f817a88 f
 0001:00016aa4       ?Escape@CDC@@UAEHHHPBDPAX@Z 5f817aa4 f
 0001:00016ac0       ??0CGdiObject@@QAE@XZ      5f817ac0 f
 0001:00016acd       ??1CMenu@@UAE@XZ           5f817acd f
 0001:00016b00       ?IsModified@CDocument@@UAEHXZ 5f817b00 f
 0001:00016b04       ?SetModifiedFlag@CDocument@@UAEXH@Z 5f817b04 f
 0001:00016b0e       ?GetReplaceString@CFindReplaceDialog@@QBE?AVCString@@XZ 5f817b0e f
 0001:00016b28       ?GetFindString@CFindReplaceDialog@@QBE?AVCString@@XZ 5f817b28 f
 0001:00016b42       ??1CListView@@UAE@XZ       5f817b42 f
 0001:00016b77       ??1CTreeView@@UAE@XZ       5f817b77 f
 0001:00016bac       ??1CCriticalSection@@UAE@XZ 5f817bac f
 0001:00016bc8       ?Lock@CCriticalSection@@UAEHK@Z 5f817bc8 f
 0001:00016bd8       ?Unlock@CCriticalSection@@UAEHXZ 5f817bd8 f
 0001:00016be6       ?GetServerName@CInternetConnection@@QBE?AVCString@@XZ 5f817be6 f
 0001:00016c01       ??0CGopherLocator@@QAE@ABV0@@Z 5f817c01 f
 0001:00016c59       ??_ECGopherLocator@@UAEPAXI@Z 5f817c59 f
 0001:00016c59       ??_GCGopherLocator@@UAEPAXI@Z 5f817c59 f
 0001:00016c75       ??0CFileFind@@QAE@XZ       5f817c75 f
 0001:00016cbf       ?Close@CFileFind@@QAEXXZ   5f817cbf f
 0001:00016cff       ?CloseContext@CFileFind@@MAEXXZ 5f817cff f
 0001:00016d09       ?FindFile@CFileFind@@UAEHPBGK@Z 5f817d09 f
 0001:00016dec       ?MatchesMask@CFileFind@@UBEHK@Z 5f817dec f
 0001:00016e06       ?GetLastAccessTime@CFileFind@@UBEHPAU_FILETIME@@@Z 5f817e06 f
 0001:00016e2a       ?GetLastWriteTime@CFileFind@@UBEHPAU_FILETIME@@@Z 5f817e2a f
 0001:00016e4e       ?GetCreationTime@CFileFind@@UBEHPAU_FILETIME@@@Z 5f817e4e f
 0001:00016e72       ?GetLastAccessTime@CFileFind@@UBEHAAVCTime@@@Z 5f817e72 f
 0001:00016e9d       ?GetLastWriteTime@CFileFind@@UBEHAAVCTime@@@Z 5f817e9d f
 0001:00016ec8       ?GetCreationTime@CFileFind@@UBEHAAVCTime@@@Z 5f817ec8 f
 0001:00016ef3       ?IsDots@CFileFind@@UBEHXZ  5f817ef3 f
 0001:00016f30       ?FindNextFileW@CFileFind@@UAEHXZ 5f817f30 f
 0001:00016f6b       ?GetFileURL@CFileFind@@UBE?AVCString@@XZ 5f817f6b f
 0001:00016fe4       ?GetRoot@CFileFind@@UBE?AVCString@@XZ 5f817fe4 f
 0001:00016fff       ?GetFilePath@CFileFind@@UBE?AVCString@@XZ 5f817fff f
 0001:0001709a       ?GetFileTitle@CFileFind@@UBE?AVCString@@XZ 5f81809a f
 0001:0001712c       ?GetFileName@CFileFind@@UBE?AVCString@@XZ 5f81812c f
 0001:0001718f       ?GetLength@CFileFind@@QBEKXZ 5f81818f f
 0001:0001719d       ?GetLength64@CFileFind@@QBE_JXZ 5f81819d f
 0001:000171ae       ??1COleDataObject@@QAE@XZ  5f8181ae f
 0001:000171b3       ?AfxCheckError@@YGXJ@Z     5f8181b3 f
 0001:000171d2       ?_AfxCompareSafeArrays@@YGHPAUtagSAFEARRAY@@0@Z 5f8181d2 f
 0001:00017441       ?_AfxCreateOneDimArray@@YGXAAUtagVARIANT@@K@Z 5f818441 f
 0001:000174ed       ?_AfxCopyBinaryData@@YGXPAUtagSAFEARRAY@@PBXK@Z 5f8184ed f
 0001:00017528       ??0COleVariant@@QAE@ABV0@@Z 5f818528 f
 0001:00017548       ??0COleVariant@@QAE@PBGG@Z 5f818548 f
 0001:00017577       ?SetString@COleVariant@@QAEXPBGG@Z 5f818577 f
 0001:000175ab       ??0COleVariant@@QAE@FG@Z   5f8185ab f
 0001:000175e1       ??0COleVariant@@QAE@JG@Z   5f8185e1 f
 0001:00017623       ?_ClearCompat@COleVariant@@QAEXXZ 5f818623 f
 0001:0001762b       ?ChangeType@COleVariant@@QAEXGPAUtagVARIANT@@@Z 5f81862b f
 0001:00017656       ?Attach@COleVariant@@QAEXAAUtagVARIANT@@@Z 5f818656 f
 0001:0001767a       ?Detach@COleVariant@@QAE?AUtagVARIANT@@XZ 5f81867a f
 0001:000176a1       ??8COleVariant@@QBEHABUtagVARIANT@@@Z 5f8186a1 f
 0001:000177c4       ??4COleVariant@@QAEABV0@ABV0@@Z 5f8187c4 f
 0001:000177de       ??4COleVariant@@QAEABV0@QBG@Z 5f8187de f
 0001:00017816       ??4COleVariant@@QAEABV0@ABVCString@@@Z 5f818816 f
 0001:00017843       ??4COleVariant@@QAEABV0@E@Z 5f818843 f
 0001:00017865       ??4COleVariant@@QAEABV0@F@Z 5f818865 f
 0001:000178a8       ??4COleVariant@@QAEABV0@J@Z 5f8188a8 f
 0001:000178ee       ??4COleVariant@@QAEABV0@ABVCOleCurrency@@@Z 5f8188ee f
 0001:00017918       ??4COleVariant@@QAEABV0@M@Z 5f818918 f
 0001:0001793a       ??4COleVariant@@QAEABV0@N@Z 5f81893a f
 0001:0001795c       ??4COleVariant@@QAEABV0@ABVCOleDateTime@@@Z 5f81895c f
 0001:00017980       ??4COleVariant@@QAEABV0@ABVCByteArray@@@Z 5f818980 f
 0001:000179a7       ??4COleVariant@@QAEABV0@ABVCLongBinary@@@Z 5f8189a7 f
 0001:000179dd       ??6@YGAAVCArchive@@AAV0@VCOleVariant@@@Z 5f8189dd f
 0001:00017ba8       ??5@YGAAVCArchive@@AAV0@AAVCOleVariant@@@Z 5f818ba8 f
 0001:00017ddc       ?ConstructElements@@YGXPAVCOleVariant@@H@Z 5f818ddc f
 0001:00017e07       ?DestructElements@@YGXPAVCOleVariant@@H@Z 5f818e07 f
 0001:00017e2c       ?CopyElements@@YGXPAVCOleVariant@@PBV1@H@Z 5f818e2c f
 0001:00017e58       ?SerializeElements@@YGXAAVCArchive@@PAVCOleVariant@@H@Z 5f818e58 f
 0001:00017eb3       ?HashKey@@YGIABUtagVARIANT@@@Z 5f818eb3 f
 0001:00017f3b       ??0COleCurrency@@QAE@JJ@Z  5f818f3b f
 0001:00017f55       ??4COleCurrency@@QAEABV0@TtagCY@@@Z 5f818f55 f
 0001:00017f6b       ??4COleCurrency@@QAEABV0@ABV0@@Z 5f818f6b f
 0001:00017f84       ??4COleCurrency@@QAEABV0@ABUtagVARIANT@@@Z 5f818f84 f
 0001:00018022       ??MCOleCurrency@@QBEHABV0@@Z 5f819022 f
 0001:00018048       ??OCOleCurrency@@QBEHABV0@@Z 5f819048 f
 0001:0001806e       ??NCOleCurrency@@QBEHABV0@@Z 5f81906e f
 0001:00018093       ??PCOleCurrency@@QBEHABV0@@Z 5f819093 f
 0001:000180b8       ??HCOleCurrency@@QBE?AV0@ABV0@@Z 5f8190b8 f
 0001:00018144       ??GCOleCurrency@@QBE?AV0@ABV0@@Z 5f819144 f
 0001:000181cf       ??GCOleCurrency@@QBE?AV0@XZ 5f8191cf f
 0001:00018219       ??DCOleCurrency@@QBE?AV0@J@Z 5f819219 f
 0001:000183f3       ??KCOleCurrency@@QBE?AV0@J@Z 5f8193f3 f
 0001:0001865c       ?SetCurrency@COleCurrency@@QAEXJJ@Z 5f81965c f
 0001:00018702       ?ParseCurrency@COleCurrency@@QAEHPBGKK@Z 5f819702 f
 0001:00018791       ?Format@COleCurrency@@QBE?AVCString@@KK@Z 5f819791 f
 0001:00018857       ??6@YGAAVCArchive@@AAV0@VCOleCurrency@@@Z 5f819857 f
 0001:0001887f       ??5@YGAAVCArchive@@AAV0@AAVCOleCurrency@@@Z 5f81987f f
 0001:000188ac       ?_AfxOleDateFromTm@@YGHGGGGGGAAN@Z 5f8198ac f
 0001:000189fb       ?_AfxTmFromOleDate@@YGHNAAUtm@@@Z 5f8199fb f
 0001:00018bfa       ?_AfxTmConvertToStandardFormat@@YGXAAUtm@@@Z 5f819bfa f
 0001:00018c11       ?_AfxDoubleFromDate@@YGNN@Z 5f819c11 f
 0001:00018c38       ?_AfxDateFromDouble@@YGNN@Z 5f819c38 f
 0001:00018c5f       ?GetTickCount@COleDateTime@@SG?AV1@XZ 5f819c5f f
 0001:00018c8f       ??6CArchive@@QAEAAV0@N@Z   5f819c8f f
 0001:00018cbc       ?GetAsSystemTime@COleDateTime@@QBEHAAU_SYSTEMTIME@@@Z 5f819cbc f
 0001:00018d26       ?GetYear@COleDateTime@@QBEHXZ 5f819d26 f
 0001:00018d50       ?GetMonth@COleDateTime@@QBEHXZ 5f819d50 f
 0001:00018d7a       ?GetDay@COleDateTime@@QBEHXZ 5f819d7a f
 0001:00018da4       ?GetHour@COleDateTime@@QBEHXZ 5f819da4 f
 0001:00018dce       ?GetMinute@COleDateTime@@QBEHXZ 5f819dce f
 0001:00018df8       ??5CArchive@@QAEAAV0@AAN@Z 5f819df8 f
 0001:00018e30       ?GetSecond@COleDateTime@@QBEHXZ 5f819e30 f
 0001:00018e5a       ?GetDayOfWeek@COleDateTime@@QBEHXZ 5f819e5a f
 0001:00018e84       ?GetDayOfYear@COleDateTime@@QBEHXZ 5f819e84 f
 0001:00018eae       ??4COleDateTime@@QAEABV0@ABUtagVARIANT@@@Z 5f819eae f
 0001:00018f3d       ??4COleDateTime@@QAEABV0@ABJ@Z 5f819f3d f
 0001:00018f8f       ??4COleDateTime@@QAEABV0@ABU_SYSTEMTIME@@@Z 5f819f8f f
 0001:00018fc7       ??4COleDateTime@@QAEABV0@ABU_FILETIME@@@Z 5f819fc7 f
 0001:00019029       ??MCOleDateTime@@QBEHABV0@@Z 5f81a029 f
 0001:0001905f       ??OCOleDateTime@@QBEHABV0@@Z 5f81a05f f
 0001:00019095       ??NCOleDateTime@@QBEHABV0@@Z 5f81a095 f
 0001:000190cb       ??PCOleDateTime@@QBEHABV0@@Z 5f81a0cb f
 0001:00019101       ??HCOleDateTime@@QBE?AV0@ABVCOleDateTimeSpan@@@Z 5f81a101 f
 0001:0001917e       ??GCOleDateTime@@QBE?AV0@ABVCOleDateTimeSpan@@@Z 5f81a17e f
 0001:000191fb       ??GCOleDateTime@@QBE?AVCOleDateTimeSpan@@ABV0@@Z 5f81a1fb f
 0001:0001925a       ?SetDateTime@COleDateTime@@QAEHHHHHHH@Z 5f81a25a f
 0001:00019285       ?ParseDateTime@COleDateTime@@QAEHPBGKK@Z 5f81a285 f
 0001:00019312       ?Format@COleDateTime@@QBE?AVCString@@KK@Z 5f81a312 f
 0001:000193da       ?Format@COleDateTime@@QBE?AVCString@@PBG@Z 5f81a3da f
 0001:000194a3       ?Format@COleDateTime@@QBE?AVCString@@I@Z 5f81a4a3 f
 0001:000194ff       ?CheckRange@COleDateTime@@IAEXXZ 5f81a4ff f
 0001:00019521       ??6@YGAAVCArchive@@AAV0@VCOleDateTime@@@Z 5f81a521 f
 0001:00019543       ??5@YGAAVCArchive@@AAV0@AAVCOleDateTime@@@Z 5f81a543 f
 0001:00019563       ?GetHours@COleDateTimeSpan@@QBEJXZ 5f81a563 f
 0001:00019596       ?GetMinutes@COleDateTimeSpan@@QBEJXZ 5f81a596 f
 0001:000195cf       ?GetSeconds@COleDateTimeSpan@@QBEJXZ 5f81a5cf f
 0001:00019608       ??4COleDateTimeSpan@@QAEABV0@N@Z 5f81a608 f
 0001:00019617       ??4COleDateTimeSpan@@QAEABV0@ABV0@@Z 5f81a617 f
 0001:0001962a       ??HCOleDateTimeSpan@@QBE?AV0@ABV0@@Z 5f81a62a f
 0001:00019689       ??GCOleDateTimeSpan@@QBE?AV0@ABV0@@Z 5f81a689 f
 0001:000196e8       ?SetDateTimeSpan@COleDateTimeSpan@@QAEXJHHH@Z 5f81a6e8 f
 0001:00019717       ?Format@COleDateTimeSpan@@QBE?AVCString@@PBG@Z 5f81a717 f
 0001:000198c0       ?Format@COleDateTimeSpan@@QBE?AVCString@@I@Z 5f81a8c0 f
 0001:0001991c       ?CheckRange@COleDateTimeSpan@@QAEXXZ 5f81a91c f
 0001:0001993e       ??0COleSafeArray@@QAE@PBUtagSAFEARRAY@@G@Z 5f81a93e f
 0001:00019983       ??0COleSafeArray@@QAE@PBUtagVARIANT@@@Z 5f81a983 f
 0001:000199b5       ??8COleSafeArray@@QBEHPBUtagSAFEARRAY@@@Z 5f81a9b5 f
 0001:000199c4       ??8COleSafeArray@@QBEHABV0@@Z 5f81a9c4 f
 0001:000199e2       ?CreateOneDim@COleSafeArray@@QAEXGKPBXJ@Z 5f81a9e2 f
 0001:00019a3e       ?GetOneDimSize@COleSafeArray@@QAEKXZ 5f81aa3e f
 0001:00019a68       ?ResizeOneDim@COleSafeArray@@QAEXK@Z 5f81aa68 f
 0001:00019a84       ?Create@COleSafeArray@@QAEXGKPAK@Z 5f81aa84 f
 0001:00019b07       ?Create@COleSafeArray@@QAEXGKPAUtagSAFEARRAYBOUND@@@Z 5f81ab07 f
 0001:00019b51       ?AccessData@COleSafeArray@@QAEXPAPAX@Z 5f81ab51 f
 0001:00019b67       ?UnaccessData@COleSafeArray@@QAEXXZ 5f81ab67 f
 0001:00019b77       ?AllocData@COleSafeArray@@QAEXXZ 5f81ab77 f
 0001:00019b87       ?AllocDescriptor@COleSafeArray@@QAEXK@Z 5f81ab87 f
 0001:00019b9e       ?Copy@COleSafeArray@@QAEXPAPAUtagSAFEARRAY@@@Z 5f81ab9e f
 0001:00019bb4       ?GetLBound@COleSafeArray@@QAEXKPAJ@Z 5f81abb4 f
 0001:00019bce       ?GetUBound@COleSafeArray@@QAEXKPAJ@Z 5f81abce f
 0001:00019be8       ?GetElement@COleSafeArray@@QAEXPAJPAX@Z 5f81abe8 f
 0001:00019c02       ?PtrOfIndex@COleSafeArray@@QAEXPAJPAPAX@Z 5f81ac02 f
 0001:00019c1c       ?PutElement@COleSafeArray@@QAEXPAJPAX@Z 5f81ac1c f
 0001:00019c36       ?Redim@COleSafeArray@@QAEXPAUtagSAFEARRAYBOUND@@@Z 5f81ac36 f
 0001:00019c4c       ?Lock@COleSafeArray@@QAEXXZ 5f81ac4c f
 0001:00019c5c       ?Unlock@COleSafeArray@@QAEXXZ 5f81ac5c f
 0001:00019c6c       ?Destroy@COleSafeArray@@QAEXXZ 5f81ac6c f
 0001:00019c7c       ?DestroyData@COleSafeArray@@QAEXXZ 5f81ac7c f
 0001:00019c8c       ?DestroyDescriptor@COleSafeArray@@QAEXXZ 5f81ac8c f
 0001:00019c9c       ?AfxSafeArrayInit@@YGXPAVCOleSafeArray@@@Z 5f81ac9c f
 0001:00019caf       ?DDX_Text@@YGXPAVCDataExchange@@HAAVCOleDateTime@@@Z 5f81acaf f
 0001:00019d76       ?DDX_Text@@YGXPAVCDataExchange@@HAAVCOleCurrency@@@Z 5f81ad76 f
 0001:00019e3d       ??0COleVariant@@QAE@PBU_ITEMIDLIST@@@Z 5f81ae3d f
 0001:00019ea2       ??_9@$BBAI@AE              5f81aea2 f
 0001:00019eaa       ?GetInterfaceMap@CEnumOleVerb@@MBEPBUAFX_INTERFACEMAP@@XZ 5f81aeaa f
 0001:00019eb0       ??1CEnumOleVerb@@UAE@XZ    5f81aeb0 f
 0001:00019ee9       ??_GCEnumOleVerb@@UAEPAXI@Z 5f81aee9 f
 0001:00019ee9       ??_ECEnumOleVerb@@UAEPAXI@Z 5f81aee9 f
 0001:00019f05       ?OnNext@CEnumOleVerb@@MAEHPAX@Z 5f81af05 f
 0001:00019f34       ?EnumOleVerbs@CCmdTarget@@QAEHPAPAUIEnumOLEVERB@@@Z 5f81af34 f
 0001:0001a0a2       ?DoOleVerb@CCmdTarget@@QAEHJPAUtagMSG@@PAUHWND__@@PBUtagRECT@@@Z 5f81b0a2 f
 0001:0001a17c       ?OnSize@CWnd@@IAEXIHH@Z    5f81b17c f
 0001:0001a184       ?EnableTypeLib@CCmdTarget@@QAEXXZ 5f81b184 f
 0001:0001a1a9       ?GetTypeInfoOfGuid@CCmdTarget@@QAEJKABU_GUID@@PAPAUITypeInfo@@@Z 5f81b1a9 f
 0001:0001a2c3       ?AfxGetTypeLibCache@@YGPAVCTypeLibCache@@PBU_GUID@@@Z 5f81b2c3 f
 0001:0001a39d       ??_GCTypeLibCacheMap@@UAEPAXI@Z 5f81b39d f
 0001:0001a39d       ??_ECTypeLibCacheMap@@UAEPAXI@Z 5f81b39d f
 0001:0001a3b9       ??1CTypeLibCacheMap@@UAE@XZ 5f81b3b9 f
 0001:0001a3be       ?Lock@CTypeLibCache@@QAEXXZ 5f81b3be f
 0001:0001a3d3       ?Lookup@CTypeLibCache@@QAEHKPAPAUITypeLib@@@Z 5f81b3d3 f
 0001:0001a404       ?Cache@CTypeLibCache@@QAEXKPAUITypeLib@@@Z 5f81b404 f
 0001:0001a447       ?LookupTypeInfo@CTypeLibCache@@QAEHKABU_GUID@@PAPAUITypeInfo@@@Z 5f81b447 f
 0001:0001a498       ?CacheTypeInfo@CTypeLibCache@@QAEXKABU_GUID@@PAUITypeInfo@@@Z 5f81b498 f
 0001:0001a4ce       ??8@YAHABU_GUID@@0@Z       5f81b4ce f
 0001:0001a4e6       ?T2OLE@@YAPAGPAG@Z         5f81b4e6 f
 0001:0001a4eb       ?Create@CDateTimeCtrl@@QAEHKABUtagRECT@@PAVCWnd@@I@Z 5f81b4eb f
 0001:0001a51c       ?GetRange@CDateTimeCtrl@@QBEKPAVCTime@@0@Z 5f81b51c f
 0001:0001a590       ?GetRange@CDateTimeCtrl@@QBEKPAVCOleDateTime@@0@Z 5f81b590 f
 0001:0001a61c       ?SetRange@CDateTimeCtrl@@QAEHPBVCTime@@0@Z 5f81b61c f
 0001:0001a66f       ?SetRange@CDateTimeCtrl@@QAEHPBVCOleDateTime@@0@Z 5f81b66f f
 0001:0001a6ce       ?SetTime@CDateTimeCtrl@@QAEHPAU_SYSTEMTIME@@@Z 5f81b6ce f
 0001:0001a6ed       ?SetTime@CDateTimeCtrl@@QAEHABVCOleDateTime@@@Z 5f81b6ed f
 0001:0001a72b       ?SetTime@CDateTimeCtrl@@QAEHPBVCTime@@@Z 5f81b72b f
 0001:0001a767       ?GetTime@CDateTimeCtrl@@QBEHAAVCOleDateTime@@@Z 5f81b767 f
 0001:0001a7c0       ?GetTime@CDateTimeCtrl@@QBEKAAVCTime@@@Z 5f81b7c0 f
 0001:0001a7fd       ??1CDateTimeCtrl@@UAE@XZ   5f81b7fd f
 0001:0001a835       ?Create@CMonthCalCtrl@@QAEHKABUtagRECT@@PAVCWnd@@I@Z 5f81b835 f
 0001:0001a866       ?Create@CMonthCalCtrl@@QAEHKABUtagPOINT@@PAVCWnd@@I@Z 5f81b866 f
 0001:0001a8d4       ?SizeMinReq@CMonthCalCtrl@@QAEHH@Z 5f81b8d4 f
 0001:0001a928       ?SetToday@CMonthCalCtrl@@QAEXABVCOleDateTime@@@Z 5f81b928 f
 0001:0001a971       ?SetToday@CMonthCalCtrl@@QAEXPBVCTime@@@Z 5f81b971 f
 0001:0001a9be       ?SetCurSel@CMonthCalCtrl@@QAEHABVCOleDateTime@@@Z 5f81b9be f
 0001:0001aa00       ?SetCurSel@CMonthCalCtrl@@QAEHABVCTime@@@Z 5f81ba00 f
 0001:0001aa39       ?GetCurSel@CMonthCalCtrl@@QBEHAAVCOleDateTime@@@Z 5f81ba39 f
 0001:0001aa7b       ?GetToday@CMonthCalCtrl@@QBEHAAVCOleDateTime@@@Z 5f81ba7b f
 0001:0001aabd       ?GetCurSel@CMonthCalCtrl@@QBEHAAVCTime@@@Z 5f81babd f
 0001:0001aafa       ?GetToday@CMonthCalCtrl@@QBEHAAVCTime@@@Z 5f81bafa f
 0001:0001ab37       ??1CMonthCalCtrl@@UAE@XZ   5f81bb37 f
 0001:0001ab6f       ?GetFirstDayOfWeek@CMonthCalCtrl@@QBEHPAH@Z 5f81bb6f f
 0001:0001ab96       ?SetFirstDayOfWeek@CMonthCalCtrl@@QAEHHPAH@Z 5f81bb96 f
 0001:0001abbd       ?SetDayState@CMonthCalCtrl@@QAEHHPAK@Z 5f81bbbd f
 0001:0001abd6       ?SetRange@CMonthCalCtrl@@QAEHPBVCOleDateTime@@0@Z 5f81bbd6 f
 0001:0001ac35       ?SetRange@CMonthCalCtrl@@QAEHQAU_SYSTEMTIME@@0@Z 5f81bc35 f
 0001:0001ac8d       ?GetRange@CMonthCalCtrl@@QBEKPAVCOleDateTime@@0@Z 5f81bc8d f
 0001:0001ad0b       ?GetRange@CMonthCalCtrl@@QBEKPAU_SYSTEMTIME@@0@Z 5f81bd0b f
 0001:0001ad7b       ?SetRange@CMonthCalCtrl@@QAEHPBVCTime@@0@Z 5f81bd7b f
 0001:0001adce       ?GetRange@CMonthCalCtrl@@QBEKPAVCTime@@0@Z 5f81bdce f
 0001:0001ae42       ?GetMonthRange@CMonthCalCtrl@@QBEHAAVCOleDateTime@@0K@Z 5f81be42 f
 0001:0001aead       ?GetMonthRange@CMonthCalCtrl@@QBEHPAU_SYSTEMTIME@@0K@Z 5f81bead f
 0001:0001aef1       ?GetMonthRange@CMonthCalCtrl@@QBEHAAVCTime@@0K@Z 5f81bef1 f
 0001:0001af52       ?GetSelRange@CMonthCalCtrl@@QBEHPAU_SYSTEMTIME@@0@Z 5f81bf52 f
 0001:0001af99       ?SetSelRange@CMonthCalCtrl@@QAEHQAU_SYSTEMTIME@@0@Z 5f81bf99 f
 0001:0001afda       ?SetSelRange@CMonthCalCtrl@@QAEHABVCOleDateTime@@0@Z 5f81bfda f
 0001:0001b028       ?GetSelRange@CMonthCalCtrl@@QBEHAAVCOleDateTime@@0@Z 5f81c028 f
 0001:0001b096       ?SetSelRange@CMonthCalCtrl@@QAEHABVCTime@@0@Z 5f81c096 f
 0001:0001b0df       ?GetSelRange@CMonthCalCtrl@@QBEHAAVCTime@@0@Z 5f81c0df f
 0001:0001b143       ?DDX_DateTimeCtrl@@YGXPAVCDataExchange@@HAAVCOleDateTime@@@Z 5f81c143 f
 0001:0001b174       ?DDX_DateTimeCtrl@@YGXPAVCDataExchange@@HAAVCTime@@@Z 5f81c174 f
 0001:0001b1a5       ?DDX_MonthCalCtrl@@YGXPAVCDataExchange@@HAAVCOleDateTime@@@Z 5f81c1a5 f
 0001:0001b1d6       ?DDX_MonthCalCtrl@@YGXPAVCDataExchange@@HAAVCTime@@@Z 5f81c1d6 f
 0001:0001b207       ?DDV_MinMaxDateTime@@YGXPAVCDataExchange@@AAVCTime@@PBV2@2@Z 5f81c207 f
 0001:0001b26b       ?DDV_MinMaxDateTime@@YGXPAVCDataExchange@@AAVCOleDateTime@@PBV2@2@Z 5f81c26b f
 0001:0001b2cc       ?DDV_MinMaxMonth@@YGXPAVCDataExchange@@AAVCTime@@PBV2@2@Z 5f81c2cc f
 0001:0001b330       ?DDV_MinMaxMonth@@YGXPAVCDataExchange@@AAVCOleDateTime@@PBV2@2@Z 5f81c330 f
 0001:0001b384       ??MCTime@@QBEHV0@@Z        5f81c384 f
 0001:0001b392       ??OCTime@@QBEHV0@@Z        5f81c392 f
 0001:0001b3a0       ??_GCDateTimeCtrl@@UAEPAXI@Z 5f81c3a0 f
 0001:0001b3a0       ??_ECDateTimeCtrl@@UAEPAXI@Z 5f81c3a0 f
 0001:0001b3bc       ??_GCMonthCalCtrl@@UAEPAXI@Z 5f81c3bc f
 0001:0001b3bc       ??_ECMonthCalCtrl@@UAEPAXI@Z 5f81c3bc f
 0001:0001b3d8       ?GetMessageMap@CHtmlView@@MBEPBUAFX_MSGMAP@@XZ 5f81c3d8 f
 0001:0001b3de       ?_GetBaseEventSinkMap@CHtmlView@@KGPBUAFX_EVENTSINKMAP@@XZ 5f81c3de f
 0001:0001b3e4       ?GetEventSinkMap@CHtmlView@@MBEPBUAFX_EVENTSINKMAP@@XZ 5f81c3e4 f
 0001:0001b3ea       ??0CHtmlView@@IAE@XZ       5f81c3ea f
 0001:0001b42d       ??_ECHtmlView@@UAEPAXI@Z   5f81c42d f
 0001:0001b42d       ??_GCHtmlView@@UAEPAXI@Z   5f81c42d f
 0001:0001b449       ??1CHtmlView@@UAE@XZ       5f81c449 f
 0001:0001b49e       ?OnFilePrint@CHtmlView@@QAEXXZ 5f81c49e f
 0001:0001b4f0       ?OnDestroy@CHtmlView@@IAEXXZ 5f81c4f0 f
 0001:0001b4fd       ?OnSize@CHtmlView@@IAEXIHH@Z 5f81c4fd f
 0001:0001b574       ?OnPaint@CHtmlView@@IAEXXZ 5f81c574 f
 0001:0001b579       ?Create@CHtmlView@@UAEHPBG0KABUtagRECT@@PAVCWnd@@IPAUCCreateContext@@@Z 5f81c579 f
 0001:0001b622       ?GetType@CHtmlView@@QBE?AVCString@@XZ 5f81c622 f
 0001:0001b682       ?GetLeft@CHtmlView@@QBEJXZ 5f81c682 f
 0001:0001b69b       ?GetTop@CHtmlView@@QBEJXZ  5f81c69b f
 0001:0001b6b4       ?GetToolBar@CHtmlView@@QBEHXZ 5f81c6b4 f
 0001:0001b6d0       ?GetHeight@CHtmlView@@QBEJXZ 5f81c6d0 f
 0001:0001b6e9       ?GetVisible@CHtmlView@@QBEHXZ 5f81c6e9 f
 0001:0001b706       ?GetLocationName@CHtmlView@@QBE?AVCString@@XZ 5f81c706 f
 0001:0001b766       ?GetLocationURL@CHtmlView@@QBE?AVCString@@XZ 5f81c766 f
 0001:0001b7c6       ?GetBusy@CHtmlView@@QBEHXZ 5f81c7c6 f
 0001:0001b7e0       ?GetReadyState@CHtmlView@@QBE?AW4tagREADYSTATE@@XZ 5f81c7e0 f
 0001:0001b7fc       ?GetOffline@CHtmlView@@QBEHXZ 5f81c7fc f
 0001:0001b819       ?GetSilent@CHtmlView@@QBEHXZ 5f81c819 f
 0001:0001b836       ?GetApplication@CHtmlView@@QBEPAUIDispatch@@XZ 5f81c836 f
 0001:0001b84f       ?GetParentBrowser@CHtmlView@@QBEPAUIDispatch@@XZ 5f81c84f f
 0001:0001b868       ?GetContainer@CHtmlView@@QBEPAUIDispatch@@XZ 5f81c868 f
 0001:0001b881       ?GetHtmlDocument@CHtmlView@@QBEPAUIDispatch@@XZ 5f81c881 f
 0001:0001b89a       ?GetTopLevelContainer@CHtmlView@@QBEHXZ 5f81c89a f
 0001:0001b8b4       ?GetMenuBar@CHtmlView@@QBEHXZ 5f81c8b4 f
 0001:0001b8d1       ?GetFullScreen@CHtmlView@@QBEHXZ 5f81c8d1 f
 0001:0001b8ee       ?GetStatusBar@CHtmlView@@QBEHXZ 5f81c8ee f
 0001:0001b90b       ?QueryStatusWB@CHtmlView@@QBE?AW4OLECMDF@@W4OLECMDID@@@Z 5f81c90b f
 0001:0001b92b       ?ExecWB@CHtmlView@@QAEXW4OLECMDID@@W4OLECMDEXECOPT@@PAUtagVARIANT@@2@Z 5f81c92b f
 0001:0001b94d       ?GetRegisterAsBrowser@CHtmlView@@QBEHXZ 5f81c94d f
 0001:0001b96a       ?GetRegisterAsDropTarget@CHtmlView@@QBEHXZ 5f81c96a f
 0001:0001b987       ?GetTheaterMode@CHtmlView@@QBEHXZ 5f81c987 f
 0001:0001b9a4       ?GetAddressBar@CHtmlView@@QBEHXZ 5f81c9a4 f
 0001:0001b9c1       ?LoadFromResource@CHtmlView@@QAEHPBG@Z 5f81c9c1 f
 0001:0001ba60       ?LoadFromResource@CHtmlView@@QAEHI@Z 5f81ca60 f
 0001:0001baff       ?Navigate@CHtmlView@@QAEXPBGK00PAXK@Z 5f81caff f
 0001:0001bbe9       ?Navigate2@CHtmlView@@QAEXPAU_ITEMIDLIST@@KPBG@Z 5f81cbe9 f
 0001:0001bc85       ?Navigate2@CHtmlView@@QAEXPBGK00PAXK@Z 5f81cc85 f
 0001:0001bd67       ?Navigate2@CHtmlView@@QAEXPBGKAAVCByteArray@@00@Z 5f81cd67 f
 0001:0001be25       ?PutProperty@CHtmlView@@QAEXPBGABUtagVARIANT@@@Z 5f81ce25 f
 0001:0001be8d       ?GetProperty@CHtmlView@@QAEHPBGAAVCString@@@Z 5f81ce8d f
 0001:0001bf26       ?GetProperty@CHtmlView@@QAE?AVCOleVariant@@PBG@Z 5f81cf26 f
 0001:0001bf93       ?GetFullName@CHtmlView@@QBE?AVCString@@XZ 5f81cf93 f
 0001:0001bff6       ?NavigateComplete2@CHtmlView@@MAEXPAUIDispatch@@PAUtagVARIANT@@@Z 5f81cff6 f
 0001:0001c03d       ?BeforeNavigate2@CHtmlView@@MAEXPAUIDispatch@@PAUtagVARIANT@@1111PAH@Z 5f81d03d f
 0001:0001c157       ?DocumentComplete@CHtmlView@@MAEXPAUIDispatch@@PAUtagVARIANT@@@Z 5f81d157 f
 0001:0001c19e       ?OnFullScreen@CHtmlView@@UAEXH@Z 5f81d19e f
 0001:0001c1a1       ?OnBeforeNavigate2@CHtmlView@@UAEXPBGK0AAVCByteArray@@0PAH@Z 5f81d1a1 f
 0001:0001c1a4       ?OnStatusTextChange@CHtmlView@@UAEXPBG@Z 5f81d1a4 f
 0001:0001c1bb       ??_9@$BBDM@AE              5f81d1bb f
 0001:0001c1c3       ??_9@$BBFM@AE              5f81d1c3 f
 0001:0001c1cb       ??_9@$BBBM@AE              5f81d1cb f
 0001:0001c1d3       ??_9@$BBEA@AE              5f81d1d3 f
 0001:0001c1db       ??_9@$BBGA@AE              5f81d1db f
 0001:0001c1e3       ??_9@$BBCA@AE              5f81d1e3 f
 0001:0001c1eb       ??_9@$BBEE@AE              5f81d1eb f
 0001:0001c1f3       ??_9@$BBCE@AE              5f81d1f3 f
 0001:0001c1fb       ??_9@$BBEI@AE              5f81d1fb f
 0001:0001c203       ??_9@$BBCI@AE              5f81d203 f
 0001:0001c20b       ??_9@$BBEM@AE              5f81d20b f
 0001:0001c213       ??_9@$BBCM@AE              5f81d213 f
 0001:0001c21b       ??_9@$BBFA@AE              5f81d21b f
 0001:0001c223       ??_9@$BBDA@AE              5f81d223 f
 0001:0001c22b       ??_9@$BBFE@AE              5f81d22b f
 0001:0001c233       ??_9@$BBDE@AE              5f81d233 f
 0001:0001c23b       ??_9@$BBFI@AE              5f81d23b f
 0001:0001c243       ??_9@$BBBI@AE              5f81d243 f
 0001:0001c24b       ?AfxEnableControlContainer@@YAXPAVCOccManager@@@Z 5f81d24b f
 0001:0001c272       ?_AfxFindFirstDlgItem@@YGPAUDLGITEMTEMPLATE@@PBUDLGTEMPLATE@@@Z 5f81d272 f
 0001:0001c2f6       ?_AfxFindNextDlgItem@@YGPAUDLGITEMTEMPLATE@@PAU1@H@Z 5f81d2f6 f
 0001:0001c34a       ?OnEvent@COccManager@@UAEHPAVCCmdTarget@@IPAUAFX_EVENT@@PAUAFX_CMDHANDLERINFO@@@Z 5f81d34a f
 0001:0001c362       ?CreateContainer@COccManager@@UAEPAVCOleControlContainer@@PAVCWnd@@@Z 5f81d362 f
 0001:0001c399       ?CreateSite@COccManager@@UAEPAVCOleControlSite@@PAVCOleControlContainer@@@Z 5f81d399 f
 0001:0001c3d3       ?PreCreateDialog@COccManager@@UAEPBUDLGTEMPLATE@@PAU_AFX_OCC_DIALOG_INFO@@PBU2@@Z 5f81d3d3 f
 0001:0001c41e       ?PostCreateDialog@COccManager@@UAEXPAU_AFX_OCC_DIALOG_INFO@@@Z 5f81d41e f
 0001:0001c443       ?SplitDialogTemplate@COccManager@@UAEPAUDLGTEMPLATE@@PBU2@PAPAUDLGITEMTEMPLATE@@@Z 5f81d443 f
 0001:0001c582       ?CreateDlgControls@COccManager@@UAEHPAVCWnd@@PBGPAU_AFX_OCC_DIALOG_INFO@@@Z 5f81d582 f
 0001:0001c5e4       ?CreateDlgControls@COccManager@@UAEHPAVCWnd@@PAXPAU_AFX_OCC_DIALOG_INFO@@@Z 5f81d5e4 f
 0001:0001c754       ?BindControls@COccManager@@IAEXPAVCWnd@@@Z 5f81d754 f
 0001:0001c86f       ?CreateDlgControl@COccManager@@IAEPAUHWND__@@PAVCWnd@@PAU2@HPAUDLGITEMTEMPLATE@@GPAEK@Z 5f81d86f f
 0001:0001cb40       ?PrepareOleCtrl@CDataExchange@@QAEPAVCWnd@@H@Z 5f81db40 f
 0001:0001cb72       ?CreateObject@?$CProcessLocal@VCOccManager@@@@SGPAVCNoTrackObject@@XZ 5f81db72 f
 0001:0001cb87       ??_GCOccManager@@UAEPAXI@Z 5f81db87 f
 0001:0001cb87       ??_ECOccManager@@UAEPAXI@Z 5f81db87 f
 0001:0001cba2       ?OnEvent@CCmdTarget@@QAEHIPAUAFX_EVENT@@PAUAFX_CMDHANDLERINFO@@@Z 5f81dba2 f
 0001:0001cdb5       ?GetEventSinkEntry@CCmdTarget@@IAGPBUAFX_EVENTSINKMAP_ENTRY@@IPAUAFX_EVENT@@@Z 5f81ddb5 f
 0001:0001ce2c       ?CreateControl@CWnd@@QAEHPBG0KABUtagRECT@@PAV1@IPAVCFile@@HPAG@Z 5f81de2c f
 0001:0001ce71       ?CreateControl@CWnd@@QAEHABU_GUID@@PBGKABUtagRECT@@PAV1@IPAVCFile@@HPAG@Z 5f81de71 f
 0001:0001cecf       ?CreateControl@CWnd@@QAEHABU_GUID@@PBGKPBUtagPOINT@@PBUtagSIZE@@PAV1@IPAVCFile@@HPAG@Z 5f81decf f
 0001:0001cf18       ?InitControlContainer@CWnd@@IAEHXZ 5f81df18 f
 0001:0001cfc1       ?GetInterfaceMap@COleControlContainer@@MBEPBUAFX_INTERFACEMAP@@XZ 5f81dfc1 f
 0001:0001cfc7       ?_GetBaseDispatchMap@COleControlContainer@@KGPBUAFX_DISPMAP@@XZ 5f81dfc7 f
 0001:0001cfcd       ?GetDispatchMap@COleControlContainer@@MBEPBUAFX_DISPMAP@@XZ 5f81dfcd f
 0001:0001cfd3       ??0COleControlContainer@@QAE@PAVCWnd@@@Z 5f81dfd3 f
 0001:0001d032       ??_GCOleControlContainer@@UAEPAXI@Z 5f81e032 f
 0001:0001d032       ??_ECOleControlContainer@@UAEPAXI@Z 5f81e032 f
 0001:0001d04e       ??1COleControlContainer@@UAE@XZ 5f81e04e f
 0001:0001d12c       ?CreateControl@COleControlContainer@@QAEHPAVCWnd@@ABU_GUID@@PBGKABUtagRECT@@IPAVCFile@@HPAGPAPAVCOleControlSite@@@Z 5f81e12c f
 0001:0001d18d       ?CreateControl@COleControlContainer@@QAEHPAVCWnd@@ABU_GUID@@PBGKPBUtagPOINT@@PBUtagSIZE@@IPAVCFile@@HPAGPAPAVCOleControlSite@@@Z 5f81e18d f
 0001:0001d248       ?FindItem@COleControlContainer@@UBEPAVCOleControlSite@@I@Z 5f81e248 f
 0001:0001d292       ?GetAmbientProp@COleControlContainer@@UAEHPAVCOleControlSite@@JPAUtagVARIANT@@@Z 5f81e292 f
 0001:0001d49a       ?CreateOleFont@COleControlContainer@@QAEXPAVCFont@@@Z 5f81e49a f
 0001:0001d5e4       ?FreezeAllEvents@COleControlContainer@@QAEXH@Z 5f81e5e4 f
 0001:0001d625       ?ScrollChildren@COleControlContainer@@UAEXHH@Z 5f81e625 f
 0001:0001d67f       ?OnUIActivate@COleControlContainer@@UAEXPAVCOleControlSite@@@Z 5f81e67f f
 0001:0001d69d       ?OnUIDeactivate@COleControlContainer@@UAEXPAVCOleControlSite@@@Z 5f81e69d f
 0001:0001d6ad       ?CheckDlgButton@COleControlContainer@@UAEXHI@Z 5f81e6ad f
 0001:0001d6ea       ?CheckRadioButton@COleControlContainer@@UAEXHHH@Z 5f81e6ea f
 0001:0001d712       ?GetDlgItem@COleControlContainer@@UBEPAVCWnd@@H@Z 5f81e712 f
 0001:0001d72d       ?GetDlgItem@COleControlContainer@@UBEXHPAPAUHWND__@@@Z 5f81e72d f
 0001:0001d769       ?GetDlgItemInt@COleControlContainer@@UBEIHPAHH@Z 5f81e769 f
 0001:0001d825       ?GetDlgItemTextW@COleControlContainer@@UBEHHPAGH@Z 5f81e825 f
 0001:0001d844       ?SendDlgItemMessageW@COleControlContainer@@UAEJHIIJ@Z 5f81e844 f
 0001:0001d869       ?SetDlgItemInt@COleControlContainer@@UAEXHIH@Z 5f81e869 f
 0001:0001d8a8       ?SetDlgItemTextW@COleControlContainer@@UAEXHPBG@Z 5f81e8a8 f
 0001:0001d8c3       ?IsDlgButtonChecked@COleControlContainer@@UBEIH@Z 5f81e8c3 f
 0001:0001d93f       ?QueryInterface@XOleIPFrame@COleControlContainer@@UAGJABU_GUID@@PAPAX@Z 5f81e93f f
 0001:0001d956       ?AddRef@XOleIPFrame@COleControlContainer@@UAGKXZ 5f81e956 f
 0001:0001d967       ?Release@XOleIPFrame@COleControlContainer@@UAGKXZ 5f81e967 f
 0001:0001d976       ?GetWindow@XOleIPFrame@COleControlContainer@@UAGJPAPAUHWND__@@@Z 5f81e976 f
 0001:0001d98b       ?RequestBorderSpace@XOleIPFrame@COleControlContainer@@UAGJPBUtagRECT@@@Z 5f81e98b f
 0001:0001d993       ?SetActiveObject@XOleIPFrame@COleControlContainer@@UAGJPAUIOleInPlaceActiveObject@@PBG@Z 5f81e993 f
 0001:0001d9ca       ?InsertMenus@XOleIPFrame@COleControlContainer@@UAGJPAUHMENU__@@PAUtagOleMenuGroupWidths@@@Z 5f81e9ca f
 0001:0001d9d2       ?EnableModeless@XOleIPFrame@COleControlContainer@@UAGJH@Z 5f81e9d2 f
 0001:0001d9d7       ?GetInterfaceMap@CEnumUnknown@@MBEPBUAFX_INTERFACEMAP@@XZ 5f81e9d7 f
 0001:0001d9dd       ??1CEnumUnknown@@UAE@XZ    5f81e9dd f
 0001:0001da33       ??_ECEnumUnknown@@UAEPAXI@Z 5f81ea33 f
 0001:0001da33       ??_GCEnumUnknown@@UAEPAXI@Z 5f81ea33 f
 0001:0001da4f       ?OnNext@CEnumUnknown@@MAEHPAX@Z 5f81ea4f f
 0001:0001da6d       ?QueryInterface@XOleContainer@COleControlContainer@@UAGJABU_GUID@@PAPAX@Z 5f81ea6d f
 0001:0001da84       ?Release@XOleContainer@COleControlContainer@@UAGKXZ 5f81ea84 f
 0001:0001da93       ?AddRef@XOleContainer@COleControlContainer@@UAGKXZ 5f81ea93 f
 0001:0001daa4       ?ParseDisplayName@XOleContainer@COleControlContainer@@UAGJPAUIBindCtx@@PAGPAKPAPAUIMoniker@@@Z 5f81eaa4 f
 0001:0001daac       ?EnumObjects@XOleContainer@COleControlContainer@@UAGJKPAPAUIEnumUnknown@@@Z 5f81eaac f
 0001:0001dbba       ?GetInterfaceMap@COleControlSite@@MBEPBUAFX_INTERFACEMAP@@XZ 5f81ebba f
 0001:0001dbc0       ??0COleControlSite@@QAE@PAVCOleControlContainer@@@Z 5f81ebc0 f
 0001:0001dccb       ??_ECOleControlSite@@UAEPAXI@Z 5f81eccb f
 0001:0001dccb       ??_GCOleControlSite@@UAEPAXI@Z 5f81eccb f
 0001:0001dce7       ??1COleControlSite@@UAE@XZ 5f81ece7 f
 0001:0001de13       ?SetExtent@COleControlSite@@IAEHXZ 5f81ee13 f
 0001:0001debb       ?CreateControl@COleControlSite@@QAEJPAVCWnd@@ABU_GUID@@PBGKABUtagRECT@@IPAVCFile@@HPAG@Z 5f81eebb f
 0001:0001df19       ?CreateControl@COleControlSite@@QAEJPAVCWnd@@ABU_GUID@@PBGKPBUtagPOINT@@PBUtagSIZE@@IPAVCFile@@HPAG@Z 5f81ef19 f
 0001:0001e1d6       ?DestroyControl@COleControlSite@@UAEHXZ 5f81f1d6 f
 0001:0001e205       ?_AfxCoCreateInstanceLic@@YGJABU_GUID@@PAUIUnknown@@K0PAPAXPAG@Z 5f81f205 f
 0001:0001e292       ?QuickActivate@COleControlSite@@UAEHXZ 5f81f292 f
 0001:0001e433       ?CreateOrLoad@COleControlSite@@IAEJABU_GUID@@PAVCFile@@HPAG@Z 5f81f433 f
 0001:0001e745       ?GetID@COleControlSite@@QAEIXZ 5f81f745 f
 0001:0001e749       ?DoVerb@COleControlSite@@UAEJJPAUtagMSG@@@Z 5f81f749 f
 0001:0001e775       ?IsDefaultButton@COleControlSite@@QAEHXZ 5f81f775 f
 0001:0001e789       ?SetDefaultButton@COleControlSite@@QAEXH@Z 5f81f789 f
 0001:0001e7d9       ?ConnectSink@COleControlSite@@IAEKABU_GUID@@PAUIUnknown@@@Z 5f81f7d9 f
 0001:0001e841       ?DisconnectSink@COleControlSite@@IAEXABU_GUID@@K@Z 5f81f841 f
 0001:0001e89f       ?GetEventIID@COleControlSite@@QAEHPAU_GUID@@@Z 5f81f89f f
 0001:0001ea0c       ?GetControlInfo@COleControlSite@@QAEXXZ 5f81fa0c f
 0001:0001ea5a       ?IsMatchingMnemonic@COleControlSite@@QAEHPAUtagMSG@@@Z 5f81fa5a f
 0001:0001eb07       ?SendMnemonic@COleControlSite@@QAEXPAUtagMSG@@@Z 5f81fb07 f
 0001:0001eb4f       ?FreezeEvents@COleControlSite@@QAEXH@Z 5f81fb4f f
 0001:0001eb85       ?AttachWindow@COleControlSite@@IAEXXZ 5f81fb85 f
 0001:0001ebc2       ?DetachWindow@COleControlSite@@IAEXXZ 5f81fbc2 f
 0001:0001ec10       ?OnEvent@COleControlSite@@IAEHPAUAFX_EVENT@@@Z 5f81fc10 f
 0001:0001ec4d       ?InvokeHelperV@COleControlSite@@UAEXJGGPAXPBEPAD@Z 5f81fc4d f
 0001:0001eca3       ?SetPropertyV@COleControlSite@@UAEXJGPAD@Z 5f81fca3 f
 0001:0001ecf6       ?InvokeHelper@COleControlSite@@UAAXJGGPAXPBEZZ 5f81fcf6 f
 0001:0001ed16       ?GetProperty@COleControlSite@@UBEXJGPAX@Z 5f81fd16 f
 0001:0001ed32       ?SetProperty@COleControlSite@@UAAXJGZZ 5f81fd32 f
 0001:0001ed49       ?SafeSetProperty@COleControlSite@@UAAHJGZZ 5f81fd49 f
 0001:0001ed9c       ?GetStyle@COleControlSite@@UBEKXZ 5f81fd9c f
 0001:0001ee52       ?GetExStyle@COleControlSite@@UBEKXZ 5f81fe52 f
 0001:0001eeba       ?ModifyStyle@COleControlSite@@UAEHKKI@Z 5f81feba f
 0001:0001ef4a       ?ModifyStyleEx@COleControlSite@@UAEHKKI@Z 5f81ff4a f
 0001:0001ef9a       ?SetWindowTextW@COleControlSite@@UAEXPBG@Z 5f81ff9a f
 0001:0001efcd       ?GetWindowTextW@COleControlSite@@UBEXAAVCString@@@Z 5f81ffcd f
 0001:0001f03c       ?GetWindowTextW@COleControlSite@@UBEHPAGH@Z 5f82003c f
 0001:0001f09b       ?GetWindowTextLengthW@COleControlSite@@UBEHXZ 5f82009b f
 0001:0001f0e4       ?SetDlgCtrlID@COleControlSite@@UAEHH@Z 5f8200e4 f
 0001:0001f0f1       ?MoveWindow@COleControlSite@@UAEXHHHHH@Z 5f8200f1 f
 0001:0001f16b       ?SetWindowPos@COleControlSite@@UAEHPBVCWnd@@HHHHI@Z 5f82016b f
 0001:0001f220       ?ShowWindow@COleControlSite@@UAEHH@Z 5f820220 f
 0001:0001f25f       ?IsWindowEnabled@COleControlSite@@UBEHXZ 5f82025f f
 0001:0001f2ad       ?EnableWindow@COleControlSite@@UAEHH@Z 5f8202ad f
 0001:0001f316       ?SetFocus@COleControlSite@@UAEPAVCWnd@@XZ 5f820316 f
 0001:0001f34f       ?EnableDSC@COleControlSite@@UAEXXZ 5f82034f f
 0001:0001f3a3       ?BindDefaultProperty@COleControlSite@@UAEXJGPBGPAVCWnd@@@Z 5f8203a3 f
 0001:0001f445       ?BindProperty@COleControlSite@@UAEXJPAVCWnd@@@Z 5f820445 f
 0001:0001f55f       ?AddRef@XOleClientSite@COleControlSite@@UAGKXZ 5f82055f f
 0001:0001f572       ?Release@XOleClientSite@COleControlSite@@UAGKXZ 5f820572 f
 0001:0001f584       ?QueryInterface@XOleClientSite@COleControlSite@@UAGJABU_GUID@@PAPAX@Z 5f820584 f
 0001:0001f59e       ?GetContainer@XOleClientSite@COleControlSite@@UAGJPAPAUIOleContainer@@@Z 5f82059e f
 0001:0001f5b9       ?ShowObject@XOleClientSite@COleControlSite@@UAGJXZ 5f8205b9 f
 0001:0001f602       ?RequestNewObjectLayout@XOleClientSite@COleControlSite@@UAGJXZ 5f820602 f
 0001:0001f60a       ?AddRef@XOleIPSite@COleControlSite@@UAGKXZ 5f82060a f
 0001:0001f61d       ?Release@XOleIPSite@COleControlSite@@UAGKXZ 5f82061d f
 0001:0001f62f       ?QueryInterface@XOleIPSite@COleControlSite@@UAGJABU_GUID@@PAPAX@Z 5f82062f f
 0001:0001f649       ?GetWindow@XOleIPSite@COleControlSite@@UAGJPAPAUHWND__@@@Z 5f820649 f
 0001:0001f674       ?CanInPlaceActivate@XOleIPSite@COleControlSite@@UAGJXZ 5f820674 f
 0001:0001f679       ?OnUIActivate@XOleIPSite@COleControlSite@@UAGJXZ 5f820679 f
 0001:0001f690       ?GetWindowContext@XOleIPSite@COleControlSite@@UAGJPAPAUIOleInPlaceFrame@@PAPAUIOleInPlaceUIWindow@@PAUtagRECT@@2PAUtagOIFI@@@Z 5f820690 f
 0001:0001f739       ?Scroll@XOleIPSite@COleControlSite@@UAGJUtagSIZE@@@Z 5f820739 f
 0001:0001f73f       ?OnUIDeactivate@XOleIPSite@COleControlSite@@UAGJH@Z 5f82073f f
 0001:0001f756       ?OnInPlaceDeactivate@XOleIPSite@COleControlSite@@UAGJXZ 5f820756 f
 0001:0001f79f       ?DeactivateAndUndo@XOleIPSite@COleControlSite@@UAGJXZ 5f82079f f
 0001:0001f7b1       ?OnPosRectChange@XOleIPSite@COleControlSite@@UAGJPBUtagRECT@@@Z 5f8207b1 f
 0001:0001f804       ?AddRef@XOleControlSite@COleControlSite@@UAGKXZ 5f820804 f
 0001:0001f817       ?Release@XOleControlSite@COleControlSite@@UAGKXZ 5f820817 f
 0001:0001f829       ?QueryInterface@XOleControlSite@COleControlSite@@UAGJABU_GUID@@PAPAX@Z 5f820829 f
 0001:0001f843       ?OnControlInfoChanged@XOleControlSite@COleControlSite@@UAGJXZ 5f820843 f
 0001:0001f857       ?TransformCoords@XOleControlSite@COleControlSite@@UAGJPAU_POINTL@@PAUtagPOINTF@@K@Z 5f820857 f
 0001:0001f95c       ?AddRef@XAmbientProps@COleControlSite@@UAGKXZ 5f82095c f
 0001:0001f96f       ?Release@XAmbientProps@COleControlSite@@UAGKXZ 5f82096f f
 0001:0001f981       ?QueryInterface@XAmbientProps@COleControlSite@@UAGJABU_GUID@@PAPAX@Z 5f820981 f
 0001:0001f99b       ?GetTypeInfo@XAmbientProps@COleControlSite@@UAGJIKPAPAUITypeInfo@@@Z 5f82099b f
 0001:0001f9a3       ?GetIDsOfNames@XAmbientProps@COleControlSite@@UAGJABU_GUID@@PAPAGIKPAJ@Z 5f8209a3 f
 0001:0001f9ab       ?Invoke@XAmbientProps@COleControlSite@@UAGJJABU_GUID@@KGPAUtagDISPPARAMS@@PAUtagVARIANT@@PAUtagEXCEPINFO@@PAI@Z 5f8209ab f
 0001:0001fa0e       ?QueryInterface@XPropertyNotifySink@COleControlSite@@UAGJABU_GUID@@PAPAX@Z 5f820a0e f
 0001:0001fa58       ?AddRef@XPropertyNotifySink@COleControlSite@@UAGKXZ 5f820a58 f
 0001:0001fa5e       ?OnChanged@XPropertyNotifySink@COleControlSite@@UAGJJ@Z 5f820a5e f
 0001:0001fba7       ?OnRequestEdit@XPropertyNotifySink@COleControlSite@@UAGJJ@Z 5f820ba7 f
 0001:0001fc2e       ?QueryInterface@XEventSink@COleControlSite@@UAGJABU_GUID@@PAPAX@Z 5f820c2e f
 0001:0001fc92       ?Invoke@XEventSink@COleControlSite@@UAGJJABU_GUID@@KGPAUtagDISPPARAMS@@PAUtagVARIANT@@PAUtagEXCEPINFO@@PAI@Z 5f820c92 f
 0001:0001fd16       ??0CDataSourceControl@@QAE@PAVCOleControlSite@@@Z 5f820d16 f
 0001:0001fd64       ??1CDataSourceControl@@QAE@XZ 5f820d64 f
 0001:0001ff44       ?ReleaseAccessors@CAccessorBase@ATL@@QAEJPAUIUnknown@@@Z 5f820f44 f
 0001:0001ffcb       ??1CRowset@ATL@@QAE@XZ     5f820fcb f
 0001:00020016       ?Close@CRowset@ATL@@QAEXXZ 5f821016 f
 0001:00020045       ?ReleaseRows@CRowset@ATL@@QAEJXZ 5f821045 f
 0001:00020065       ?Close@CDynamicAccessor@ATL@@QAEXXZ 5f821065 f
 0001:0002009f       ?Initialize@CDataSourceControl@@QAEJXZ 5f82109f f
 0001:0002023d       ?GetCursor@CDataSourceControl@@UAEPAUIUnknown@@XZ 5f82123d f
 0001:000202a4       ?GetMetaData@CDataSourceControl@@QAEJXZ 5f8212a4 f
 0001:000205e2       ??0CRowset@ATL@@QAE@PAUIRowset@@@Z 5f8215e2 f
 0001:00020633       ?MoveFirst@CRowset@ATL@@QAEJXZ 5f821633 f
 0001:00020656       ?MoveNext@CRowset@ATL@@QAEJJ_N@Z 5f821656 f
 0001:000206af       ?GetData@CRowset@ATL@@QAEJXZ 5f8216af f
 0001:000206e3       ?GetData@CRowset@ATL@@QAEJH@Z 5f8216e3 f
 0001:00020706       ?SetupOptionalRowsetInterfaces@CRowset@ATL@@QAEXXZ 5f821706 f
 0001:0002071b       ?BindColumns@CDynamicAccessor@ATL@@QAEJPAUIUnknown@@@Z 5f82171b f
 0001:000209d2       ?AllocateAccessorMemory@CAccessorBase@ATL@@QAEJH@Z 5f8219d2 f
 0001:00020a2e       ?BindEntries@CAccessorBase@ATL@@SAJPAUtagDBBINDING@@HPAKKPAUIAccessor@@@Z 5f821a2e f
 0001:00020a78       ?Bind@CAccessorBase@ATL@@SAXPAUtagDBBINDING@@KGKEEKKKKPAUtagDBOBJECT@@@Z 5f821a78 f
 0001:00020af7       ?CopyColumnID@CDataSourceControl@@QAEHPAUtagDBCOLUMNID@@PBU2@@Z 5f821af7 f
 0001:00020b65       ?BindProp@CDataSourceControl@@UAEXPAVCOleControlSite@@H@Z 5f821b65 f
 0001:00020caa       ?TranslateColumnNo@CDynamicAccessor@ATL@@QBE_NAAK@Z 5f821caa f
 0001:00020cfd       ?BindProp@CDataSourceControl@@UAEXPAVCDataBoundProperty@@H@Z 5f821cfd f
 0001:00020d45       ?BindColumns@CDataSourceControl@@UAEXXZ 5f821d45 f
 0001:00020eef       ?GetBoundClientRow@CDataSourceControl@@QAEJXZ 5f821eef f
 0001:00020f4c       ?ToVariant@CDataSourceControl@@QAE?AVCOleVariant@@H@Z 5f821f4c f
 0001:000216c5       ?GetStatus@CDynamicAccessor@ATL@@QBE_NKPAK@Z 5f8226c5 f
 0001:00021709       ?_GetDataPtr@CDynamicAccessor@ATL@@QBEPAXK@Z 5f822709 f
 0001:00021720       ?UpdateControls@CDataSourceControl@@UAEJXZ 5f822720 f
 0001:000218bb       ?UpdateCursor@CDataSourceControl@@UAEJXZ 5f8228bb f
 0001:00022210       ?SetData@CRowset@ATL@@QBEJXZ 5f823210 f
 0001:00022238       ?SetData@CRowset@ATL@@QBEJH@Z 5f823238 f
 0001:00022267       ?CreateAccessor@CManualAccessor@ATL@@QAEJHPAXK@Z 5f823267 f
 0001:000222de       ?AddBindEntry@CManualAccessor@ATL@@QAEXKGKPAX00@Z 5f8232de f
 0001:00022332       ?BindColumns@CManualAccessor@ATL@@QAEJPAUIUnknown@@@Z 5f823332 f
 0001:000223ca       ??0CDataBoundProperty@@QAE@PAV0@JG@Z 5f8233ca f
 0001:000223f0       ?SetDSCSite@CDataBoundProperty@@QAEXPAVCOleControlSite@@@Z 5f8233f0 f
 0001:00022404       ?GetNext@CDataBoundProperty@@QAEPAV1@XZ 5f823404 f
 0001:00022408       ?RemoveSource@CDataBoundProperty@@QAEXXZ 5f823408 f
 0001:0002240c       ?Notify@CDataBoundProperty@@QAEXXZ 5f82340c f
 0001:0002248f       ?GetCursor@CDataBoundProperty@@QAEPAUIUnknown@@XZ 5f82348f f
 0001:000224c5       ?GetCursor@COleControlSite@@IAEJJPAPAUIUnknown@@PAPAX@Z 5f8234c5 f
 0001:000224fc       ?AddRef@XBoundObjectSite@COleControlSite@@UAGKXZ 5f8234fc f
 0001:00022543       ?Release@XBoundObjectSite@COleControlSite@@UAGKXZ 5f823543 f
 0001:0002258a       ?QueryInterface@XBoundObjectSite@COleControlSite@@UAGJABU_GUID@@PAPAX@Z 5f82358a f
 0001:000225d7       ?GetCursor@XBoundObjectSite@COleControlSite@@UAGJJPAPAUICursor@@PAPAX@Z 5f8235d7 f
 0001:00022627       ?QueryInterface@XNotifyDBEvents@COleControlSite@@UAGJABU_GUID@@PAPAX@Z 5f823627 f
 0001:00022671       ?OKToDo@XNotifyDBEvents@COleControlSite@@UAGJKKQAUtagDBNOTIFYREASON@@@Z 5f823671 f
 0001:000226fb       ?Cancelled@XNotifyDBEvents@COleControlSite@@UAGJKKQAUtagDBNOTIFYREASON@@@Z 5f8236fb f
 0001:0002274d       ?SyncBefore@XNotifyDBEvents@COleControlSite@@UAGJKKQAUtagDBNOTIFYREASON@@@Z 5f82374d f
 0001:000227d2       ?AboutToDo@XNotifyDBEvents@COleControlSite@@UAGJKKQAUtagDBNOTIFYREASON@@@Z 5f8237d2 f
 0001:00022824       ?FailedToDo@XNotifyDBEvents@COleControlSite@@UAGJKKQAUtagDBNOTIFYREASON@@@Z 5f823824 f
 0001:00022876       ?SyncAfter@XNotifyDBEvents@COleControlSite@@UAGJKKQAUtagDBNOTIFYREASON@@@Z 5f823876 f
 0001:0002291a       ?DidEvent@XNotifyDBEvents@COleControlSite@@UAGJKKQAUtagDBNOTIFYREASON@@@Z 5f82391a f
 0001:000229a3       ?FireEvent@XNotifyDBEvents@COleControlSite@@QAEJKKQAUtagDBNOTIFYREASON@@W4DSCSTATE@@@Z 5f8239a3 f
 0001:00022a65       ?QueryInterface@XRowsetNotify@COleControlSite@@UAGJABU_GUID@@PAPAX@Z 5f823a65 f
 0001:00022aaf       ?OnFieldChange@XRowsetNotify@COleControlSite@@UAGJPAUIRowset@@KKQAKKKH@Z 5f823aaf f
 0001:00022b97       ?OnRowChange@XRowsetNotify@COleControlSite@@UAGJPAUIRowset@@KQBKKKH@Z 5f823b97 f
 0001:00022d3d       ?OnRowsetChange@XRowsetNotify@COleControlSite@@UAGJPAUIRowset@@KKH@Z 5f823d3d f
 0001:00022de7       ?AtlComPtrAssign@ATL@@YGPAUIUnknown@@PAPAU2@PAU2@@Z 5f823de7 f
 0001:00022e10       ??1COleDispatchDriver@@QAE@XZ 5f823e10 f
 0001:00022e15       ??0AFX_EVENT@@QAE@H@Z      5f823e15 f
 0001:00022e38       ??0COleControlLock@@QAE@ABU_GUID@@@Z 5f823e38 f
 0001:00022ea7       ??_GCOleControlLock@@UAEPAXI@Z 5f823ea7 f
 0001:00022ea7       ??_ECOleControlLock@@UAEPAXI@Z 5f823ea7 f
 0001:00022ec3       ??1COleControlLock@@UAE@XZ 5f823ec3 f
 0001:00022eea       ?AfxOleLockControl@@YGHABU_GUID@@@Z 5f823eea f
 0001:00022f89       ?AfxOleLockControl@@YGHPBG@Z 5f823f89 f
 0001:00022fb0       ?AfxOleUnlockControl@@YGHPBG@Z 5f823fb0 f
 0001:00022fd7       ?AfxOleUnlockControl@@YGHABU_GUID@@@Z 5f823fd7 f
 0001:0002305a       ?DDX_OCText@@YGXPAVCDataExchange@@HJAAVCString@@@Z 5f82405a f
 0001:00023099       ?DDX_OCTextRO@@YGXPAVCDataExchange@@HJAAVCString@@@Z 5f824099 f
 0001:000230db       ?DDX_OCBool@@YGXPAVCDataExchange@@HJAAH@Z 5f8240db f
 0001:0002311a       ?DDX_OCBoolRO@@YGXPAVCDataExchange@@HJAAH@Z 5f82411a f
 0001:00023137       ?DDX_OCIntRO@@YGXPAVCDataExchange@@HJAAH@Z 5f824137 f
 0001:00023154       ?DDX_OCIntRO@@YGXPAVCDataExchange@@HJAAJ@Z 5f824154 f
 0001:00023171       ?DDX_OCShort@@YGXPAVCDataExchange@@HJAAF@Z 5f824171 f
 0001:000231b2       ?DDX_OCShortRO@@YGXPAVCDataExchange@@HJAAF@Z 5f8241b2 f
 0001:000231cf       ?DDX_OCColor@@YGXPAVCDataExchange@@HJAAK@Z 5f8241cf f
 0001:0002320e       ?DDX_OCColorRO@@YGXPAVCDataExchange@@HJAAK@Z 5f82420e f
 0001:0002322b       ?DDX_OCFloat@@YGXPAVCDataExchange@@HJAAM@Z 5f82422b f
 0001:0002326f       ?DDX_OCFloatRO@@YGXPAVCDataExchange@@HJAAM@Z 5f82426f f
 0001:00023295       ?DDX_OCFloat@@YGXPAVCDataExchange@@HJAAN@Z 5f824295 f
 0001:000232d9       ?DDX_OCFloatRO@@YGXPAVCDataExchange@@HJAAN@Z 5f8242d9 f
 0001:000232ff       ?_AfxGetDlgCode@@YGKPAVCWnd@@PAUtagMSG@@@Z 5f8242ff f
 0001:0002332d       ?_AfxDlgSetFocus@@YGXPAVCWnd@@@Z 5f82432d f
 0001:0002335b       ?_AfxGetChildControl@@YGPAVCWnd@@PAV1@0@Z 5f82435b f
 0001:000233b4       ?_AfxNextControl@@YGPAVCWnd@@PAV1@0I@Z 5f8243b4 f
 0001:00023490       ?IsMatchingMnemonic@COccManager@@SAHPAVCWnd@@PAUtagMSG@@@Z 5f824490 f
 0001:000234af       ?_AfxFindNextMnem@@YGPAVCWnd@@PAV1@0PAUtagMSG@@@Z 5f8244af f
 0001:00023534       ?IsLabelControl@COccManager@@SAHPAVCWnd@@@Z 5f824534 f
 0001:0002355a       ?_AfxGetNextMnem@@YGPAVCWnd@@PAV1@0PAUtagMSG@@@Z 5f82455a f
 0001:000235cf       ?UIActivateControl@COccManager@@KAXPAVCWnd@@@Z 5f8245cf f
 0001:0002362c       ?UIDeactivateIfNecessary@COccManager@@KAXPAVCWnd@@0@Z 5f82462c f
 0001:0002369f       ?_AfxFindDlgItem@@YGPAVCWnd@@PAV1@K@Z 5f82469f f
 0001:000236f6       ?SetDefaultButton@COccManager@@SAXPAVCWnd@@H@Z 5f8246f6 f
 0001:00023743       ?GetDefBtnCode@COccManager@@SAKPAVCWnd@@@Z 5f824743 f
 0001:00023753       ?GetDefBtnCode@COleControlSite@@QAEKXZ 5f824753 f
 0001:00023778       ?_AfxRemoveDefaultButton@@YGXPAVCWnd@@0@Z 5f824778 f
 0001:000237da       ?_AfxOriginalDefButton@@YGHPAVCWnd@@@Z 5f8247da f
 0001:00023807       ?_AfxCheckDefPushButton@@YGXPAVCWnd@@00@Z 5f824807 f
 0001:000238ef       ?IsDialogMessageW@COccManager@@UAEHPAVCWnd@@PAUtagMSG@@@Z 5f8248ef f
 0001:00023ce8       ?OnActivateView@CDocObjectServer@@MAEJXZ 5f824ce8 f
 0001:0002402f       ?AddRef@XOleDocumentView@CDocObjectServer@@UAGKXZ 5f82502f f
 0001:0002406e       ?Release@XOleDocumentView@CDocObjectServer@@UAGKXZ 5f82506e f
 0001:000240ad       ?QueryInterface@XOleDocumentView@CDocObjectServer@@UAGJABU_GUID@@PAPAX@Z 5f8250ad f
 0001:000240f2       ?SetInPlaceSite@XOleDocumentView@CDocObjectServer@@UAGJPAUIOleInPlaceSite@@@Z 5f8250f2 f
 0001:00024163       ?GetInPlaceSite@XOleDocumentView@CDocObjectServer@@UAGJPAPAUIOleInPlaceSite@@@Z 5f825163 f
 0001:000241b1       ?GetDocument@XOleDocumentView@CDocObjectServer@@UAGJPAPAUIUnknown@@@Z 5f8251b1 f
 0001:000241f9       ?OnSetItemRects@CDocObjectServer@@IAEXPAUtagRECT@@0@Z 5f8251f9 f
 0001:0002420f       ?SetRect@XOleDocumentView@CDocObjectServer@@UAGJPAUtagRECT@@@Z 5f82520f f
 0001:0002427e       ?GetRect@XOleDocumentView@CDocObjectServer@@UAGJPAUtagRECT@@@Z 5f82527e f
 0001:000242c2       ?SetRectComplex@XOleDocumentView@CDocObjectServer@@UAGJPAUtagRECT@@000@Z 5f8252c2 f
 0001:000242e7       ?Show@XOleDocumentView@CDocObjectServer@@UAGJH@Z 5f8252e7 f
 0001:0002433c       ?UIActivate@XOleDocumentView@CDocObjectServer@@UAGJH@Z 5f82533c f
 0001:00024398       ?Open@XOleDocumentView@CDocObjectServer@@UAGJXZ 5f825398 f
 0001:000243ea       ?CloseView@XOleDocumentView@CDocObjectServer@@UAGJK@Z 5f8253ea f
 0001:00024431       ?SaveViewState@XOleDocumentView@CDocObjectServer@@UAGJPAUIStream@@@Z 5f825431 f
 0001:0002455b       ?ApplyViewState@XOleDocumentView@CDocObjectServer@@UAGJPAUIStream@@@Z 5f82555b f
 0001:00024685       ?Clone@XOleDocumentView@CDocObjectServer@@UAGJPAUIOleInPlaceSite@@PAPAUIOleDocumentView@@@Z 5f825685 f
 0001:000246aa       ?_GetBaseClass@CDocObjectServer@@KGPAUCRuntimeClass@@XZ 5f8256aa f
 0001:000246b0       ?GetRuntimeClass@CDocObjectServer@@UBEPAUCRuntimeClass@@XZ 5f8256b0 f
 0001:000246b6       ?_GetBaseMessageMap@CDocObjectServer@@KGPBUAFX_MSGMAP@@XZ 5f8256b6 f
 0001:000246bc       ?GetMessageMap@CDocObjectServer@@MBEPBUAFX_MSGMAP@@XZ 5f8256bc f
 0001:000246c2       ?_GetBaseInterfaceMap@CDocObjectServer@@KGPBUAFX_INTERFACEMAP@@XZ 5f8256c2 f
 0001:000246c8       ?GetInterfaceMap@CDocObjectServer@@MBEPBUAFX_INTERFACEMAP@@XZ 5f8256c8 f
 0001:000246ce       ??0CDocObjectServer@@QAE@PAVCOleServerDoc@@PAUIOleDocumentSite@@@Z 5f8256ce f
 0001:00024722       ??_ECDocObjectServer@@UAEPAXI@Z 5f825722 f
 0001:00024722       ??_GCDocObjectServer@@UAEPAXI@Z 5f825722 f
 0001:0002473e       ??1CDocObjectServer@@UAE@XZ 5f82573e f
 0001:00024776       ?ReleaseDocSite@CDocObjectServer@@QAEXXZ 5f825776 f
 0001:0002478c       ?SetDocSite@CDocObjectServer@@QAEXPAUIOleDocumentSite@@@Z 5f82578c f
 0001:0002479f       ?OnCloseDocument@CDocObjectServer@@UAEXXZ 5f82579f f
 0001:000247b4       ?OnExecOleCmd@CDocObjectServer@@IAGJPBU_GUID@@KKPAUtagVARIANT@@1@Z 5f8257b4 f
 0001:000247e3       ?GetControllingFrame@CDocObjectServer@@QBEPAVCOleDocIPFrameWnd@@XZ 5f8257e3 f
 0001:00024828       ?DoPreparePrinting@CDocObjectServer@@IAEHPAVCView@@PAUCPrintInfo@@@Z 5f825828 f
 0001:0002483b       ?DoPrepareDC@CDocObjectServer@@IAEXPAVCView@@PAVCDC@@PAUCPrintInfo@@@Z 5f82583b f
 0001:00024852       ?DoPrint@CDocObjectServer@@IAEXPAVCView@@PAVCDC@@PAUCPrintInfo@@@Z 5f825852 f
 0001:00024869       ?DoBeginPrinting@CDocObjectServer@@IAEXPAVCView@@PAVCDC@@PAUCPrintInfo@@@Z 5f825869 f
 0001:00024880       ?DoEndPrinting@CDocObjectServer@@IAEXPAVCView@@PAVCDC@@PAUCPrintInfo@@@Z 5f825880 f
 0001:00024897       ?AddRef@XPrint@CDocObjectServer@@UAGKXZ 5f825897 f
 0001:000248d6       ?Release@XPrint@CDocObjectServer@@UAGKXZ 5f8258d6 f
 0001:00024915       ?QueryInterface@XPrint@CDocObjectServer@@UAGJABU_GUID@@PAPAX@Z 5f825915 f
 0001:0002495c       ?SetInitialPageNum@XPrint@CDocObjectServer@@UAGJJ@Z 5f82595c f
 0001:00024986       ?GetPageInfo@XPrint@CDocObjectServer@@UAGJPAJ0@Z 5f825986 f
 0001:00024a74       ?Print@XPrint@CDocObjectServer@@UAGJKPAPAUtagDVTARGETDEVICE@@PAPAUtagPAGESET@@PAUtagSTGMEDIUM@@PAUIContinueCallback@@JPAJ4@Z 5f825a74 f
 0001:00025177       ?AddRef@XOleDocument@CDocObjectServer@@UAGKXZ 5f826177 f
 0001:000251b6       ?Release@XOleDocument@CDocObjectServer@@UAGKXZ 5f8261b6 f
 0001:000251f5       ?QueryInterface@XOleDocument@CDocObjectServer@@UAGJABU_GUID@@PAPAX@Z 5f8261f5 f
 0001:0002523c       ?CreateView@XOleDocument@CDocObjectServer@@UAGJPAUIOleInPlaceSite@@PAUIStream@@KPAPAUIOleDocumentView@@@Z 5f82623c f
 0001:000252d0       ?GetDocMiscStatus@XOleDocument@CDocObjectServer@@UAGJPAK@Z 5f8262d0 f
 0001:000252f8       ?EnumViews@XOleDocument@CDocObjectServer@@UAGJPAPAUIEnumOleDocumentViews@@PAPAUIOleDocumentView@@@Z 5f8262f8 f
 0001:00025342       ?AddRef@XOleObject@CDocObjectServer@@UAGKXZ 5f826342 f
 0001:00025381       ?Release@XOleObject@CDocObjectServer@@UAGKXZ 5f826381 f
 0001:000253c0       ?QueryInterface@XOleObject@CDocObjectServer@@UAGJABU_GUID@@PAPAX@Z 5f8263c0 f
 0001:00025405       ?SetClientSite@XOleObject@CDocObjectServer@@UAGJPAUIOleClientSite@@@Z 5f826405 f
 0001:00025478       ?GetClientSite@XOleObject@CDocObjectServer@@UAGJPAPAUIOleClientSite@@@Z 5f826478 f
 0001:000254c5       ?SetHostNames@XOleObject@CDocObjectServer@@UAGJPBG0@Z 5f8264c5 f
 0001:00025515       ?Close@XOleObject@CDocObjectServer@@UAGJK@Z 5f826515 f
 0001:00025562       ?SetMoniker@XOleObject@CDocObjectServer@@UAGJKPAUIMoniker@@@Z 5f826562 f
 0001:000255b2       ?GetMoniker@XOleObject@CDocObjectServer@@UAGJKKPAPAUIMoniker@@@Z 5f8265b2 f
 0001:00025605       ?InitFromData@XOleObject@CDocObjectServer@@UAGJPAUIDataObject@@HK@Z 5f826605 f
 0001:00025658       ?GetClipboardData@XOleObject@CDocObjectServer@@UAGJKPAPAUIDataObject@@@Z 5f826658 f
 0001:000256a8       ?DoVerb@XOleObject@CDocObjectServer@@UAGJJPAUtagMSG@@PAUIOleClientSite@@JPAUHWND__@@PBUtagRECT@@@Z 5f8266a8 f
 0001:00025704       ?EnumVerbs@XOleObject@CDocObjectServer@@UAGJPAPAUIEnumOLEVERB@@@Z 5f826704 f
 0001:00025751       ?Update@XOleObject@CDocObjectServer@@UAGJXZ 5f826751 f
 0001:0002579b       ?IsUpToDate@XOleObject@CDocObjectServer@@UAGJXZ 5f82679b f
 0001:000257e5       ?GetUserClassID@XOleObject@CDocObjectServer@@UAGJPAU_GUID@@@Z 5f8267e5 f
 0001:00025832       ?GetUserType@XOleObject@CDocObjectServer@@UAGJKPAPAG@Z 5f826832 f
 0001:00025882       ?SetExtent@XOleObject@CDocObjectServer@@UAGJKPAUtagSIZE@@@Z 5f826882 f
 0001:000258e1       ?GetExtent@XOleObject@CDocObjectServer@@UAGJKPAUtagSIZE@@@Z 5f8268e1 f
 0001:00025931       ?Advise@XOleObject@CDocObjectServer@@UAGJPAUIAdviseSink@@PAK@Z 5f826931 f
 0001:00025981       ?Unadvise@XOleObject@CDocObjectServer@@UAGJK@Z 5f826981 f
 0001:000259ce       ?EnumAdvise@XOleObject@CDocObjectServer@@UAGJPAPAUIEnumSTATDATA@@@Z 5f8269ce f
 0001:00025a1b       ?GetMiscStatus@XOleObject@CDocObjectServer@@UAGJKPAK@Z 5f826a1b f
 0001:00025a6b       ?SetColorScheme@XOleObject@CDocObjectServer@@UAGJPAUtagLOGPALETTE@@@Z 5f826a6b f
 0001:00025ab8       ?_GetBaseClass@CDocObjectServerItem@@KGPAUCRuntimeClass@@XZ 5f826ab8 f
 0001:00025abe       ?GetRuntimeClass@CDocObjectServerItem@@UBEPAUCRuntimeClass@@XZ 5f826abe f
 0001:00025ac4       ??0CDocObjectServerItem@@IAE@PAVCOleServerDoc@@H@Z 5f826ac4 f
 0001:00025ae0       ??_ECDocObjectServerItem@@UAEPAXI@Z 5f826ae0 f
 0001:00025ae0       ??_GCDocObjectServerItem@@UAEPAXI@Z 5f826ae0 f
 0001:00025afc       ??1CDocObjectServerItem@@UAE@XZ 5f826afc f
 0001:00025b02       ??1COleServerItem@@UAE@XZ  5f826b02 f
 0001:00025baa       ?OnDoVerb@CDocObjectServerItem@@MAEXJ@Z 5f826baa f
 0001:00025bd7       ?OnHide@CDocObjectServerItem@@MAEXXZ 5f826bd7 f
 0001:00025bf2       ?OnOpen@CDocObjectServerItem@@MAEXXZ 5f826bf2 f
 0001:00025c04       ?ActivateDocObject@COleServerDoc@@QAEXXZ 5f826c04 f
 0001:00025c12       ?ActivateDocObject@CDocObjectServer@@QAEXXZ 5f826c12 f
 0001:00025c2a       ?OnShow@CDocObjectServerItem@@MAEXXZ 5f826c2a f
 0001:00025c3e       ??0COleCmdUI@@QAE@PAU_tagOLECMD@@KPBU_GUID@@@Z 5f826c3e f
 0001:00025c6f       ?Enable@COleCmdUI@@UAEXH@Z 5f826c6f f
 0001:00025c96       ?SetCheck@COleCmdUI@@UAEXH@Z 5f826c96 f
 0001:00025cda       ?SetText@COleCmdUI@@UAEXPBG@Z 5f826cda f
 0001:00025ce9       ?DoUpdate@COleCmdUI@@UAEHPAVCCmdTarget@@H@Z 5f826ce9 f
 0001:00025da4       ?AddRef@XOleCommandTarget@CDocObjectServer@@UAGKXZ 5f826da4 f
 0001:00025de3       ?Release@XOleCommandTarget@CDocObjectServer@@UAGKXZ 5f826de3 f
 0001:00025e22       ?QueryInterface@XOleCommandTarget@CDocObjectServer@@UAGJABU_GUID@@PAPAX@Z 5f826e22 f
 0001:00025e67       ?_AfxQueryStatusOleCommandHelper@@YGJPAVCCmdTarget@@PBU_GUID@@KQAU_tagOLECMD@@PAU_tagOLECMDTEXT@@@Z 5f826e67 f
 0001:00025f62       ?QueryStatus@XOleCommandTarget@CDocObjectServer@@UAGJPBU_GUID@@KQAU_tagOLECMD@@PAU_tagOLECMDTEXT@@@Z 5f826f62 f
 0001:00025fb5       ?_AfxExecOleCommandHelper@@YGJPAVCCmdTarget@@PBU_GUID@@KKPAUtagVARIANT@@2@Z 5f826fb5 f
 0001:0002605b       ?Exec@XOleCommandTarget@CDocObjectServer@@UAGJPBU_GUID@@KKPAUtagVARIANT@@1@Z 5f82705b f
 0001:000260cd       ?CreateObject@COleDocIPFrameWnd@@SGPAVCObject@@XZ 5f8270cd f
 0001:00026102       ?_GetBaseClass@COleDocIPFrameWnd@@KGPAUCRuntimeClass@@XZ 5f827102 f
 0001:00026108       ?GetRuntimeClass@COleDocIPFrameWnd@@UBEPAUCRuntimeClass@@XZ 5f827108 f
 0001:0002610e       ?_GetBaseMessageMap@COleDocIPFrameWnd@@KGPBUAFX_MSGMAP@@XZ 5f82710e f
 0001:00026114       ?GetMessageMap@COleDocIPFrameWnd@@MBEPBUAFX_MSGMAP@@XZ 5f827114 f
 0001:0002611a       ??0COleDocIPFrameWnd@@QAE@XZ 5f82711a f
 0001:00026133       ??1COleDocIPFrameWnd@@UAE@XZ 5f827133 f
 0001:00026139       ??1COleIPFrameWnd@@UAE@XZ  5f827139 f
 0001:000261b7       ?OnRequestPositionChange@COleDocIPFrameWnd@@MAEXPBUtagRECT@@@Z 5f8271b7 f
 0001:000261d6       ?RecalcLayout@COleDocIPFrameWnd@@MAEXH@Z 5f8271d6 f
 0001:00026333       ?BuildSharedMenu@COleDocIPFrameWnd@@MAEHXZ 5f827333 f
 0001:000263d1       ?DestroySharedMenu@COleDocIPFrameWnd@@MAEXXZ 5f8273d1 f
 0001:00026445       ?_GetBaseClass@COleDocObjectItem@@KGPAUCRuntimeClass@@XZ 5f827445 f
 0001:0002644b       ?GetRuntimeClass@COleDocObjectItem@@UBEPAUCRuntimeClass@@XZ 5f82744b f
 0001:00026451       ?_GetBaseInterfaceMap@COleDocObjectItem@@KGPBUAFX_INTERFACEMAP@@XZ 5f827451 f
 0001:00026457       ?GetInterfaceMap@COleDocObjectItem@@MBEPBUAFX_INTERFACEMAP@@XZ 5f827457 f
 0001:0002645d       ??0COleDocObjectItem@@QAE@PAVCOleDocument@@@Z 5f82745d f
 0001:00026493       ??_ECOleDocObjectItem@@UAEPAXI@Z 5f827493 f
 0001:00026493       ??_GCOleDocObjectItem@@UAEPAXI@Z 5f827493 f
 0001:000264af       ??1COleDocObjectItem@@UAE@XZ 5f8274af f
 0001:00026507       ?AddRef@XOleDocumentSite@COleDocObjectItem@@UAGKXZ 5f827507 f
 0001:0002654b       ?Release@XOleDocumentSite@COleDocObjectItem@@UAGKXZ 5f82754b f
 0001:0002658f       ?QueryInterface@XOleDocumentSite@COleDocObjectItem@@UAGJABU_GUID@@PAPAX@Z 5f82758f f
 0001:000265d9       ?ActivateMe@XOleDocumentSite@COleDocObjectItem@@UAGJPAUIOleDocumentView@@@Z 5f8275d9 f
 0001:0002671d       ?ActivateAndShow@COleDocObjectItem@@IAEXXZ 5f82771d f
 0001:0002675c       ?OnGetItemPosition@COleDocObjectItem@@MAEXAAVCRect@@@Z 5f82775c f
 0001:0002676f       ?Release@COleDocObjectItem@@UAEXW4tagOLECLOSE@@@Z 5f82776f f
 0001:0002679f       ?ExecCommand@COleDocObjectItem@@QAEJKKPBU_GUID@@@Z 5f82779f f
 0001:000267e2       ?SupportsIPrint@COleDocObjectItem@@IAEHXZ 5f8277e2 f
 0001:00026845       ?GetPageCount@COleDocObjectItem@@QAEHPAJ0@Z 5f827845 f
 0001:00026890       ?GetHelpMenu@COleDocObjectItem@@MAEPAVCMenu@@AAI@Z 5f827890 f
 0001:000268bd       ?OnInsertMenus@COleDocObjectItem@@UAEXPAVCMenu@@PAUtagOleMenuGroupWidths@@@Z 5f8278bd f
 0001:00026a5e       ?OnRemoveMenus@COleDocObjectItem@@UAEXPAVCMenu@@@Z 5f827a5e f
 0001:00026acb       ?OnPreparePrinting@COleDocObjectItem@@SAHPAVCView@@PAUCPrintInfo@@H@Z 5f827acb f
 0001:00026bcb       ?OnPrint@COleDocObjectItem@@SAXPAVCView@@PAUCPrintInfo@@H@Z 5f827bcb f
 0001:00026d7b       ??0?$CIP@UIUnknown@@$1?IID_IUnknown@@3U_GUID@@B@@QAE@PAUIUnknown@@H@Z 5f827d7b f
 0001:00026d96       ??B?$CIP@UIUnknown@@$1?IID_IUnknown@@3U_GUID@@B@@QAEPAUIUnknown@@XZ 5f827d96 f
 0001:00026d99       ??0CMonikerFile@@QAE@XZ    5f827d99 f
 0001:00026dd2       ?GetMoniker@CMonikerFile@@QBEPAUIMoniker@@XZ 5f827dd2 f
 0001:00026dd6       ?SetBinding@CAsyncMonikerFile@@IAEXPAUIBinding@@@Z 5f827dd6 f
 0001:00026de5       ?SetFormatEtc@CAsyncMonikerFile@@IAEXPAUtagFORMATETC@@@Z 5f827de5 f
 0001:00026def       ?AddRef@XOleCache@COleControl@@UAGKXZ 5f827def f
 0001:00026e01       ?Release@XOleCache@COleControl@@UAGKXZ 5f827e01 f
 0001:00026e13       ?QueryInterface@XOleCache@COleControl@@UAGJABU_GUID@@PAPAX@Z 5f827e13 f
 0001:00026e2d       ?Cache@XOleCache@COleControl@@UAGJPAUtagFORMATETC@@KPAK@Z 5f827e2d f
 0001:00026e6b       ?Uncache@XOleCache@COleControl@@UAGJK@Z 5f827e6b f
 0001:00026ea1       ?EnumCache@XOleCache@COleControl@@UAGJPAPAUIEnumSTATDATA@@@Z 5f827ea1 f
 0001:00026ed7       ?InitCache@XOleCache@COleControl@@UAGJPAUIDataObject@@@Z 5f827ed7 f
 0001:00026f0d       ?SetData@XOleCache@COleControl@@UAGJPAUtagFORMATETC@@PAUtagSTGMEDIUM@@H@Z 5f827f0d f
 0001:00026f4b       ?_AfxGetParkingWindow@@YGPAUHWND__@@XZ 5f827f4b f
 0001:00026fe2       ?_AfxReleaseParkingWindow@@YGXXZ 5f827fe2 f
 0001:00027064       ?GetInterfaceMap@COleControl@@MBEPBUAFX_INTERFACEMAP@@XZ 5f828064 f
 0001:0002706a       ?_GetBaseMessageMap@COleControl@@KGPBUAFX_MSGMAP@@XZ 5f82806a f
 0001:00027070       ?GetMessageMap@COleControl@@MBEPBUAFX_MSGMAP@@XZ 5f828070 f
 0001:00027076       ??0COleControl@@QAE@XZ     5f828076 f
 0001:000272ad       ??_ECOleControl@@UAEPAXI@Z 5f8282ad f
 0001:000272ad       ??_GCOleControl@@UAEPAXI@Z 5f8282ad f
 0001:000272c9       ??1COleControl@@UAE@XZ     5f8282c9 f
 0001:000273ac       ?ReleaseCaches@COleControl@@IAEXXZ 5f8283ac f
 0001:000274b2       ?OnFinalRelease@COleControl@@MAEXXZ 5f8284b2 f
 0001:000274e6       ?GetInterfaceHook@COleControl@@MAEPAUIUnknown@@PBX@Z 5f8284e6 f
 0001:00027563       ?SetInitialSize@COleControl@@QAEXHH@Z 5f828563 f
 0001:0002759e       ?GetDispatchIID@COleControl@@MAEHPAU_GUID@@@Z 5f82859e f
 0001:000275bc       ?InitializeIIDs@COleControl@@QAEXPBU_GUID@@0@Z 5f8285bc f
 0001:000275e4       ?_AfxFillPSOnStack@@YGXXZ  5f8285e4 f
 0001:0002760b       ?DoSuperclassPaint@COleControl@@QAEXPAVCDC@@ABVCRect@@@Z 5f82860b f
 0001:000276f5       ?IsSubclassedControl@COleControl@@UAEHXZ 5f8286f5 f
 0001:0002771e       ?CreateControlWindow@COleControl@@MAEHPAUHWND__@@ABVCRect@@PBUtagRECT@@@Z 5f82871e f
 0001:0002794b       ?ReparentControlWindow@COleControl@@UAEXPAUHWND__@@0@Z 5f82894b f
 0001:0002795c       ?GetControlSize@COleControl@@QAEXPAH0@Z 5f82895c f
 0001:00027997       ?SetControlSize@COleControl@@QAEHHH@Z 5f828997 f
 0001:000279df       ?SetRectInContainer@COleControl@@QAEHPBUtagRECT@@@Z 5f8289df f
 0001:00027a27       ?OnResetState@COleControl@@UAEXXZ 5f828a27 f
 0001:00027a54       ?_AfxDrawBorders@@YGXPAVCDC@@AAVCRect@@HH@Z 5f828a54 f
 0001:00027aaf       ?DrawContent@COleControl@@IAEXPAVCDC@@AAVCRect@@@Z 5f828aaf f
 0001:00027b81       ?DrawMetafile@COleControl@@IAEXPAVCDC@@AAVCRect@@@Z 5f828b81 f
 0001:00027c02       ?OnDraw@COleControl@@UAEXPAVCDC@@ABVCRect@@1@Z 5f828c02 f
 0001:00027c05       ?OnDrawMetafile@COleControl@@UAEXPAVCDC@@ABVCRect@@@Z 5f828c05 f
 0001:00027c1c       ?GetMetafileData@COleControl@@IAEHPAUtagFORMATETC@@PAUtagSTGMEDIUM@@@Z 5f828c1c f
 0001:00027d96       ?QueryDefHandler@COleControl@@IAEPAXABU_GUID@@@Z 5f828d96 f
 0001:00027dfa       ?InvalidateControl@COleControl@@QAEXPBUtagRECT@@H@Z 5f828dfa f
 0001:00027ea7       ?GetOuterWindow@COleControl@@IBEPAVCWnd@@XZ 5f828ea7 f
 0001:00027eb4       ?OnReflectorDestroyed@COleControl@@MAEXXZ 5f828eb4 f
 0001:00027ebc       ?SaveState@COleControl@@IAEJPAUIStream@@@Z 5f828ebc f
 0001:00027f4a       ?LoadState@COleControl@@IAEJPAUIStream@@@Z 5f828f4a f
 0001:00028029       ?SendAdvise@COleControl@@IAEXI@Z 5f829029 f
 0001:0002813b       ?OnHide@COleControl@@MAEJXZ 5f82913b f
 0001:0002819a       ?OnOpen@COleControl@@MAEJHPAUtagMSG@@@Z 5f82919a f
 0001:00028286       ?CreateFrameWindow@COleControl@@MAEPAVCControlFrameWnd@@XZ 5f829286 f
 0001:000282f0       ?OnFrameClose@COleControl@@MAEXXZ 5f8292f0 f
 0001:00028356       ?ResizeOpenControl@COleControl@@IAEXHH@Z 5f829356 f
 0001:00028395       ?ResizeFrameWindow@COleControl@@MAEXHH@Z 5f829395 f
 0001:00028405       ?GetRectInContainer@COleControl@@QAEHPAUtagRECT@@@Z 5f829405 f
 0001:0002842f       ?GetPropPageIDs@COleControl@@MAEPAU_GUID@@AAK@Z 5f82942f f
 0001:0002843b       ?OnEdit@COleControl@@UAEHPAUtagMSG@@PAUHWND__@@PBUtagRECT@@@Z 5f82943b f
 0001:00028469       ?_AfxGetTopLevelWindow@@YGPAUHWND__@@PAU1@@Z 5f829469 f
 0001:00028481       ?OnProperties@COleControl@@UAEHPAUtagMSG@@PAUHWND__@@PBUtagRECT@@@Z 5f829481 f
 0001:0002854f       ?GetControlFlags@COleControl@@UAEKXZ 5f82954f f
 0001:00028553       ?OnPaint@COleControl@@IAEXPAVCDC@@@Z 5f829553 f
 0001:00028658       ?OnEraseBkgnd@COleControl@@IAEHPAVCDC@@@Z 5f829658 f
 0001:00028677       ?Serialize@COleControl@@MAEXAAVCArchive@@@Z 5f829677 f
 0001:000286bb       ?DoPropExchange@COleControl@@UAEXPAVCPropExchange@@@Z 5f8296bb f
 0001:000286d6       ?ControlInfoChanged@COleControl@@QAEXXZ 5f8296d6 f
 0001:000286e7       ?LockInPlaceActive@COleControl@@QAEHH@Z 5f8296e7 f
 0001:0002870b       ?GetExtendedControl@COleControl@@QAEPAUIDispatch@@XZ 5f82970b f
 0001:0002872c       ?TransformCoords@COleControl@@QAEXPAU_POINTL@@PAUtagPOINTF@@K@Z 5f82972c f
 0001:0002877c       ?AddRef@XOleControl@COleControl@@UAGKXZ 5f82977c f
 0001:0002878e       ?Release@XOleControl@COleControl@@UAGKXZ 5f82978e f
 0001:000287a0       ?QueryInterface@XOleControl@COleControl@@UAGJABU_GUID@@PAPAX@Z 5f8297a0 f
 0001:000287ba       ?GetControlInfo@XOleControl@COleControl@@UAGJPAUtagCONTROLINFO@@@Z 5f8297ba f
 0001:00028809       ?OnMnemonic@XOleControl@COleControl@@UAGJPAUtagMSG@@@Z 5f829809 f
 0001:00028858       ?OnAmbientPropertyChange@XOleControl@COleControl@@UAGJJ@Z 5f829858 f
 0001:000288d9       ?FreezeEvents@XOleControl@COleControl@@UAGJH@Z 5f8298d9 f
 0001:00028949       ?OnGetControlInfo@COleControl@@UAEXPAUtagCONTROLINFO@@@Z 5f829949 f
 0001:0002895c       ?OnSetClientSite@COleControl@@UAEXXZ 5f82995c f
 0001:00028997       ?GetClientSite@COleControl@@QAEPAUIOleClientSite@@XZ 5f829997 f
 0001:0002899e       ?TranslateColor@COleControl@@QAEKKPAUHPALETTE__@@@Z 5f82999e f
 0001:000289bd       ?Refresh@COleControl@@QAEXXZ 5f8299bd f
 0001:000289d9       ?DoClick@COleControl@@QAEXXZ 5f8299d9 f
 0001:000289e4       ?OnNcCreate@COleControl@@IAEHPAUtagCREATESTRUCTW@@@Z 5f8299e4 f
 0001:00028a02       ?RecreateControlWindow@COleControl@@QAEXXZ 5f829a02 f
 0001:00028abe       ?CreateWindowForSubclassedControl@COleControl@@IAEXXZ 5f829abe f
 0001:00028b2e       ?OnMouseActivate@COleControl@@IAEHPAVCWnd@@II@Z 5f829b2e f
 0001:00028b51       ?PreModalDialog@COleControl@@QAEXPAUHWND__@@@Z 5f829b51 f
 0001:00028b7e       ?PostModalDialog@COleControl@@QAEXPAUHWND__@@@Z 5f829b7e f
 0001:00028bab       ?SetModifiedFlag@COleControl@@QAEXH@Z 5f829bab f
 0001:00028bcb       ?IsModified@COleControl@@QAEHXZ 5f829bcb f
 0001:00028bd8       ?WillAmbientsBeValidDuringLoad@COleControl@@QAEHXZ 5f829bd8 f
 0001:00028be5       ?EnableSimpleFrame@COleControl@@QAEXXZ 5f829be5 f
 0001:00028bed       ?IgnoreWindowMessage@COleControl@@IAEHIIJPAJ@Z 5f829bed f
 0001:00028c48       ?WindowProc@COleControl@@UAEJIIJ@Z 5f829c48 f
 0001:00028d98       ?DefWindowProcW@COleControl@@MAEJIIJ@Z 5f829d98 f
 0001:00028db6       ?OnCreate@COleControl@@IAEHPAUtagCREATESTRUCTW@@@Z 5f829db6 f
 0001:00028dd4       ?OnSize@COleControl@@IAEXIHH@Z 5f829dd4 f
 0001:00028dee       ?OnMove@COleControl@@IAEXHH@Z 5f829dee f
 0001:00028e08       ?OnInitMenuPopup@COleControl@@IAEXPAVCMenu@@IH@Z 5f829e08 f
 0001:00028f49       ?OnMenuSelect@COleControl@@IAEXIIPAUHMENU__@@@Z 5f829f49 f
 0001:00028ff9       ?GetMessageString@COleControl@@UBEXIAAVCString@@@Z 5f829ff9 f
 0001:0002903f       ?OnSetMessageString@COleControl@@IAEJIJ@Z 5f82a03f f
 0001:000290c4       ?OnEnterIdle@COleControl@@IAEXIPAVCWnd@@@Z 5f82a0c4 f
 0001:000290ed       ?AddRef@XSpecifyPropertyPages@COleControl@@UAGKXZ 5f82a0ed f
 0001:000290ff       ?Release@XSpecifyPropertyPages@COleControl@@UAGKXZ 5f82a0ff f
 0001:00029111       ?QueryInterface@XSpecifyPropertyPages@COleControl@@UAGJABU_GUID@@PAPAX@Z 5f82a111 f
 0001:0002912b       ?GetPages@XSpecifyPropertyPages@COleControl@@UAGJPAUtagCAUUID@@@Z 5f82a12b f
 0001:000291d4       ?OnDestroy@COleControl@@IAEXXZ 5f82a1d4 f
 0001:00029214       ?OnKillFocus@COleControl@@IAEXPAVCWnd@@@Z 5f82a214 f
 0001:00029232       ?OnSetFocus@COleControl@@IAEXPAVCWnd@@@Z 5f82a232 f
 0001:00029250       ?OnOcmCtlColorBtn@COleControl@@IAEJIJ@Z 5f82a250 f
 0001:00029269       ?OnOcmCtlColorDlg@COleControl@@IAEJIJ@Z 5f82a269 f
 0001:00029282       ?OnOcmCtlColorEdit@COleControl@@IAEJIJ@Z 5f82a282 f
 0001:0002929b       ?OnOcmCtlColorListBox@COleControl@@IAEJIJ@Z 5f82a29b f
 0001:000292b4       ?OnOcmCtlColorMsgBox@COleControl@@IAEJIJ@Z 5f82a2b4 f
 0001:000292cd       ?OnOcmCtlColorScrollBar@COleControl@@IAEJIJ@Z 5f82a2cd f
 0001:000292e6       ?OnOcmCtlColorStatic@COleControl@@IAEJIJ@Z 5f82a2e6 f
 0001:000292ff       ?ThrowError@COleControl@@QAEXJII@Z 5f82a2ff f
 0001:00029341       ?ThrowError@COleControl@@QAEXJPBGI@Z 5f82a341 f
 0001:00029389       ?IsInvokeAllowed@COleControl@@MAEHJ@Z 5f82a389 f
 0001:00029398       ?GetIID@XPropConnPt@COleControl@@UAEABU_GUID@@XZ 5f82a398 f
 0001:0002939e       ??_EXEventConnPt@COleControl@@UAEPAXI@Z 5f82a39e f
 0001:0002939e       ??_GXEventConnPt@COleControl@@UAEPAXI@Z 5f82a39e f
 0001:000293ba       ??1CConnectionPoint@@UAE@XZ 5f82a3ba f
 0001:000293ba       ??1XPropConnPt@COleControl@@UAE@XZ 5f82a3ba f
 0001:0002941f       ??_GCReflectorWnd@@UAEPAXI@Z 5f82a41f f
 0001:0002941f       ??_ECReflectorWnd@@UAEPAXI@Z 5f82a41f f
 0001:0002943b       ??0CParkingWnd@@QAE@XZ     5f82a43b f
 0001:000294ad       ??_ECParkingWnd@@UAEPAXI@Z 5f82a4ad f
 0001:000294ad       ??_GCParkingWnd@@UAEPAXI@Z 5f82a4ad f
 0001:000294c9       ??1CParkingWnd@@UAE@XZ     5f82a4c9 f
 0001:000294fe       ?_GetBaseConnectionMap@COleControl@@KGPBUAFX_CONNECTIONMAP@@XZ 5f82a4fe f
 0001:00029504       ?GetConnectionMap@COleControl@@MBEPBUAFX_CONNECTIONMAP@@XZ 5f82a504 f
 0001:0002950a       ?GetConnectionHook@COleControl@@MAEPAUIConnectionPoint@@ABU_GUID@@@Z 5f82a50a f
 0001:00029535       ?GetExtraConnectionPoints@COleControl@@MAEHPAVCPtrArray@@@Z 5f82a535 f
 0001:0002954e       ?AddRef@XProvideClassInfo@COleControl@@UAGKXZ 5f82a54e f
 0001:00029560       ?Release@XProvideClassInfo@COleControl@@UAGKXZ 5f82a560 f
 0001:00029572       ?QueryInterface@XProvideClassInfo@COleControl@@UAGJABU_GUID@@PAPAX@Z 5f82a572 f
 0001:0002958c       ?GetClassInfoW@XProvideClassInfo@COleControl@@UAGJPAPAUITypeInfo@@@Z 5f82a58c f
 0001:000295f0       ?GetGUID@XProvideClassInfo@COleControl@@UAGJKPAU_GUID@@@Z 5f82a5f0 f
 0001:00029626       ?OnAdvise@XEventConnPt@COleControl@@UAEXH@Z 5f82a626 f
 0001:0002966d       ?GetIID@XEventConnPt@COleControl@@UAEABU_GUID@@XZ 5f82a66d f
 0001:0002967d       ?QuerySinkInterface@XEventConnPt@COleControl@@UAEPAUIUnknown@@PAU3@@Z 5f82a67d f
 0001:000296b2       ?AfxConnectionAdvise@@YGHPAUIUnknown@@ABU_GUID@@0HPAK@Z 5f82a6b2 f
 0001:00029724       ?AfxConnectionUnadvise@@YGHPAUIUnknown@@ABU_GUID@@0HK@Z 5f82a724 f
 0001:000297a1       ?_AfxRegisterClipFormat@@YGGABU_GUID@@@Z 5f82a7a1 f
 0001:000297fe       ?_AfxGetClipboardFormatConvertVBX@@YGGXZ 5f82a7fe f
 0001:0002981a       ?_AfxGetClipboardFormatPersistPropset@@YGGXZ 5f82a81a f
 0001:00029836       ?_AfxOleMatchPropsetClipFormat@@YGHGPAU_GUID@@@Z 5f82a836 f
 0001:00029870       ?AddRef@XDataObject@COleControl@@UAGKXZ 5f82a870 f
 0001:00029882       ?Release@XDataObject@COleControl@@UAGKXZ 5f82a882 f
 0001:00029894       ?QueryInterface@XDataObject@COleControl@@UAGJABU_GUID@@PAPAX@Z 5f82a894 f
 0001:000298ae       ?GetData@XDataObject@COleControl@@UAGJPAUtagFORMATETC@@PAUtagSTGMEDIUM@@@Z 5f82a8ae f
 0001:000298dd       ?GetDataHere@XDataObject@COleControl@@UAGJPAUtagFORMATETC@@PAUtagSTGMEDIUM@@@Z 5f82a8dd f
 0001:0002990c       ?QueryGetData@XDataObject@COleControl@@UAGJPAUtagFORMATETC@@@Z 5f82a90c f
 0001:00029937       ?GetCanonicalFormatEtc@XDataObject@COleControl@@UAGJPAUtagFORMATETC@@0@Z 5f82a937 f
 0001:00029966       ?SetData@XDataObject@COleControl@@UAGJPAUtagFORMATETC@@PAUtagSTGMEDIUM@@H@Z 5f82a966 f
 0001:00029999       ?EnumFormatEtc@XDataObject@COleControl@@UAGJKPAPAUIEnumFORMATETC@@@Z 5f82a999 f
 0001:000299c8       ?DAdvise@XDataObject@COleControl@@UAGJPAUtagFORMATETC@@KPAUIAdviseSink@@PAK@Z 5f82a9c8 f
 0001:00029a0c       ?DUnadvise@XDataObject@COleControl@@UAGJK@Z 5f82aa0c f
 0001:00029a2b       ?EnumDAdvise@XDataObject@COleControl@@UAGJPAPAUIEnumSTATDATA@@@Z 5f82aa2b f
 0001:00029a4e       ??0CControlDataSource@COleControl@@QAE@PAV1@@Z 5f82aa4e f
 0001:00029a70       ??_GCControlDataSource@COleControl@@UAEPAXI@Z 5f82aa70 f
 0001:00029a70       ??_ECControlDataSource@COleControl@@UAEPAXI@Z 5f82aa70 f
 0001:00029a8c       ??1COleDataSource@@UAE@XZ  5f82aa8c f
 0001:00029a8c       ??1CControlDataSource@COleControl@@UAE@XZ 5f82aa8c f
 0001:00029ade       ?OnRenderGlobalData@CControlDataSource@COleControl@@MAEHPAUtagFORMATETC@@PAPAX@Z 5f82aade f
 0001:00029af4       ?OnRenderFileData@CControlDataSource@COleControl@@MAEHPAUtagFORMATETC@@PAVCFile@@@Z 5f82aaf4 f
 0001:00029b0a       ?OnRenderData@CControlDataSource@COleControl@@MAEHPAUtagFORMATETC@@PAUtagSTGMEDIUM@@@Z 5f82ab0a f
 0001:00029b3c       ?OnSetData@CControlDataSource@COleControl@@MAEHPAUtagFORMATETC@@PAUtagSTGMEDIUM@@H@Z 5f82ab3c f
 0001:00029b56       ?OnRenderData@COleControl@@UAEHPAUtagFORMATETC@@PAUtagSTGMEDIUM@@@Z 5f82ab56 f
 0001:00029ba4       ?OnSetData@COleControl@@UAEHPAUtagFORMATETC@@PAUtagSTGMEDIUM@@H@Z 5f82aba4 f
 0001:00029bf2       ?GetDataSource@COleControl@@IAEPAVCControlDataSource@1@XZ 5f82abf2 f
 0001:00029c8a       ?SetInitialDataFormats@COleControl@@MAEXXZ 5f82ac8a f
 0001:00029d19       ?InitStockEventMask@COleControl@@IAEXXZ 5f82ad19 f
 0001:00029d8c       ?GetEventMap@COleControl@@MBEPBUAFX_EVENTMAP@@XZ 5f82ad8c f
 0001:00029d92       ?GetEventMapEntry@COleControl@@IBEPBUAFX_EVENTMAP_ENTRY@@PBGPAJ@Z 5f82ad92 f
 0001:00029df6       ?FireEventV@COleControl@@IAEXJPAEPAD@Z 5f82adf6 f
 0001:00029e99       ?FireEvent@COleControl@@QAAXJPAEZZ 5f82ae99 f
 0001:00029eb0       ?_AfxShiftState@@YGFXZ     5f82aeb0 f
 0001:00029ee9       ?OnSysKeyDown@COleControl@@IAEXIII@Z 5f82aee9 f
 0001:00029f36       ?OnSysKeyUp@COleControl@@IAEXIII@Z 5f82af36 f
 0001:00029f83       ?OnKeyDown@COleControl@@IAEXIII@Z 5f82af83 f
 0001:00029fd0       ?OnKeyUp@COleControl@@IAEXIII@Z 5f82afd0 f
 0001:0002a01d       ?KeyUp@COleControl@@IAEXPAG@Z 5f82b01d f
 0001:0002a06f       ?KeyDown@COleControl@@IAEXPAG@Z 5f82b06f f
 0001:0002a0c1       ?_AfxPostTrailByte@@YGXPAVCWnd@@E@Z 5f82b0c1 f
 0001:0002a12f       ?OnGetDlgCode@COleControl@@IAEIXZ 5f82b12f f
 0001:0002a166       ?OnChar@COleControl@@IAEXIII@Z 5f82b166 f
 0001:0002a2e3       ?OnKeyDownEvent@COleControl@@UAEXGG@Z 5f82b2e3 f
 0001:0002a2e6       ?ButtonDown@COleControl@@IAEXGIVCPoint@@@Z 5f82b2e6 f
 0001:0002a36f       ?ButtonUp@COleControl@@IAEXGIVCPoint@@@Z 5f82b36f f
 0001:0002a443       ?ButtonDblClk@COleControl@@IAEXGIVCPoint@@@Z 5f82b443 f
 0001:0002a497       ?OnMouseMove@COleControl@@IAEXIVCPoint@@@Z 5f82b497 f
 0001:0002a4f0       ?OnLButtonDown@COleControl@@IAEXIVCPoint@@@Z 5f82b4f0 f
 0001:0002a506       ?OnLButtonUp@COleControl@@IAEXIVCPoint@@@Z 5f82b506 f
 0001:0002a51c       ?OnLButtonDblClk@COleControl@@IAEXIVCPoint@@@Z 5f82b51c f
 0001:0002a532       ?OnMButtonDown@COleControl@@IAEXIVCPoint@@@Z 5f82b532 f
 0001:0002a548       ?OnMButtonUp@COleControl@@IAEXIVCPoint@@@Z 5f82b548 f
 0001:0002a55e       ?OnMButtonDblClk@COleControl@@IAEXIVCPoint@@@Z 5f82b55e f
 0001:0002a574       ?OnRButtonDown@COleControl@@IAEXIVCPoint@@@Z 5f82b574 f
 0001:0002a58a       ?OnRButtonUp@COleControl@@IAEXIVCPoint@@@Z 5f82b58a f
 0001:0002a5a0       ?OnRButtonDblClk@COleControl@@IAEXIVCPoint@@@Z 5f82b5a0 f
 0001:0002a5b6       ?OnButtonDown@COleControl@@IAEXGIVCPoint@@@Z 5f82b5b6 f
 0001:0002a5f1       ?OnButtonUp@COleControl@@IAEXGIVCPoint@@@Z 5f82b5f1 f
 0001:0002a665       ?OnButtonDblClk@COleControl@@IAEXGIVCPoint@@@Z 5f82b665 f
 0001:0002a692       ?OnCancelMode@COleControl@@IAEXXZ 5f82b692 f
 0001:0002a6c0       ?OnClick@COleControl@@UAEXG@Z 5f82b6c0 f
 0001:0002a6e7       ?FireError@COleControl@@QAEXJPBGI@Z 5f82b6e7 f
 0001:0002a790       ?DisplayError@COleControl@@UAEXJPBG00I@Z 5f82b790 f
 0001:0002a7a2       ?GetMessageMap@CControlFrameWnd@@MBEPBUAFX_MSGMAP@@XZ 5f82b7a2 f
 0001:0002a7a8       ??0CControlFrameWnd@@QAE@PAVCOleControl@@@Z 5f82b7a8 f
 0001:0002a7c3       ??1CControlFrameWnd@@UAE@XZ 5f82b7c3 f
 0001:0002a7c8       ?PreCreateWindow@CControlFrameWnd@@UAEHAAUtagCREATESTRUCTW@@@Z 5f82b7c8 f
 0001:0002a7e6       ?Create@CControlFrameWnd@@UAEHPBG@Z 5f82b7e6 f
 0001:0002a80d       ?OnClose@CControlFrameWnd@@IAEXXZ 5f82b80d f
 0001:0002a824       ?PostNcDestroy@CControlFrameWnd@@MAEXXZ 5f82b824 f
 0001:0002a830       ?OnActivate@CControlFrameWnd@@IAEXIPAVCWnd@@H@Z 5f82b830 f
 0001:0002a844       ??0CFontHolder@@QAE@PAUIPropertyNotifySink@@@Z 5f82b844 f
 0001:0002a857       ?SetFontNotifySink@CFontHolder@@QAEXPAUIPropertyNotifySink@@@Z 5f82b857 f
 0001:0002a861       ?ReleaseFont@CFontHolder@@QAEXXZ 5f82b861 f
 0001:0002a861       ??1CFontHolder@@QAE@XZ     5f82b861 f
 0001:0002a88a       ?InitializeFont@CFontHolder@@QAEXPBUtagFONTDESC@@PAUIDispatch@@@Z 5f82b88a f
 0001:0002a907       ?_AfxIsSameFont@@YGHAAVCFontHolder@@PBUtagFONTDESC@@PAUIFontDisp@@@Z 5f82b907 f
 0001:0002aa99       ?GetFontHandle@CFontHolder@@QAEPAUHFONT__@@XZ 5f82ba99 f
 0001:0002aaaa       ?GetFontHandle@CFontHolder@@QAEPAUHFONT__@@JJ@Z 5f82baaa f
 0001:0002aadf       ?Select@CFontHolder@@QAEPAVCFont@@PAVCDC@@JJ@Z 5f82badf f
 0001:0002ab2a       ?QueryTextMetrics@CFontHolder@@QAEXPAUtagTEXTMETRICW@@@Z 5f82bb2a f
 0001:0002ab4f       ?SetFont@CFontHolder@@QAEXPAUIFont@@@Z 5f82bb4f f
 0001:0002ab7f       ?GetDisplayString@CFontHolder@@QAEHAAVCString@@@Z 5f82bb7f f
 0001:0002ab90       ??0_AFXCTL_UIACTIVE_INFO@@QAE@PAUHMENU__@@PAUIOleInPlaceFrame@@@Z 5f82bb90 f
 0001:0002abfd       ??1_AFXCTL_UIACTIVE_INFO@@QAE@XZ 5f82bbfd f
 0001:0002ac1e       ?_GetClippingCoordinates@@YGXPBUtagRECT@@0PAU1@PAUtagPOINT@@@Z 5f82bc1e f
 0001:0002ac85       ?OnActivateInPlace@COleControl@@MAEJHPAUtagMSG@@@Z 5f82bc85 f
 0001:0002b050       ?ForwardActivationMsg@COleControl@@IAEXPAUtagMSG@@@Z 5f82c050 f
 0001:0002b11c       ?BuildSharedMenu@COleControl@@MAEHXZ 5f82c11c f
 0001:0002b1bb       ?DestroySharedMenu@COleControl@@MAEXXZ 5f82c1bb f
 0001:0002b223       ?AddFrameLevelUI@COleControl@@MAEXXZ 5f82c223 f
 0001:0002b251       ?RemoveFrameLevelUI@COleControl@@MAEXXZ 5f82c251 f
 0001:0002b285       ?OnShowToolBars@COleControl@@UAEXXZ 5f82c285 f
 0001:0002b294       ?OnHideToolBars@COleControl@@UAEXXZ 5f82c294 f
 0001:0002b295       ?AddRef@XOleInPlaceObject@COleControl@@UAGKXZ 5f82c295 f
 0001:0002b2a7       ?Release@XOleInPlaceObject@COleControl@@UAGKXZ 5f82c2a7 f
 0001:0002b2b9       ?QueryInterface@XOleInPlaceObject@COleControl@@UAGJABU_GUID@@PAPAX@Z 5f82c2b9 f
 0001:0002b2d3       ?GetWindow@XOleInPlaceObject@COleControl@@UAGJPAPAUHWND__@@@Z 5f82c2d3 f
 0001:0002b309       ?InPlaceDeactivate@XOleInPlaceObject@COleControl@@UAGJXZ 5f82c309 f
 0001:0002b3c5       ?UIDeactivate@XOleInPlaceObject@COleControl@@UAGJXZ 5f82c3c5 f
 0001:0002b469       ?SetObjectRects@XOleInPlaceObject@COleControl@@UAGJPBUtagRECT@@0@Z 5f82c469 f
 0001:0002b4c7       ?OnSetObjectRects@COleControl@@UAEHPBUtagRECT@@0@Z 5f82c4c7 f
 0001:0002b5b9       ?AddRef@XOleInPlaceActiveObject@COleControl@@UAGKXZ 5f82c5b9 f
 0001:0002b5cb       ?Release@XOleInPlaceActiveObject@COleControl@@UAGKXZ 5f82c5cb f
 0001:0002b5dd       ?QueryInterface@XOleInPlaceActiveObject@COleControl@@UAGJABU_GUID@@PAPAX@Z 5f82c5dd f
 0001:0002b5f7       ?GetWindow@XOleInPlaceActiveObject@COleControl@@UAGJPAPAUHWND__@@@Z 5f82c5f7 f
 0001:0002b60b       ?TranslateAcceleratorW@XOleInPlaceActiveObject@COleControl@@UAGJPAUtagMSG@@@Z 5f82c60b f
 0001:0002b688       ?OnDocWindowActivate@XOleInPlaceActiveObject@COleControl@@UAGJH@Z 5f82c688 f
 0001:0002b6ef       ?ResizeBorder@XOleInPlaceActiveObject@COleControl@@UAGJPBUtagRECT@@PAUIOleInPlaceUIWindow@@H@Z 5f82c6ef f
 0001:0002b6f4       ?AfxVerifyLicFile@@YGHPAUHINSTANCE__@@PBG1I@Z 5f82c6f4 f
 0001:0002b7f2       ??0CConnectionPoint@@QAE@XZ 5f82c7f2 f
 0001:0002b813       ??_ECConnectionPoint@@UAEPAXI@Z 5f82c813 f
 0001:0002b813       ??_GCConnectionPoint@@UAEPAXI@Z 5f82c813 f
 0001:0002b82f       ?GetStartPosition@CConnectionPoint@@QBEPAU__POSITION@@XZ 5f82c82f f
 0001:0002b84d       ?GetNextConnection@CConnectionPoint@@QBEPAUIUnknown@@AAPAU__POSITION@@@Z 5f82c84d f
 0001:0002b881       ?GetConnections@CConnectionPoint@@QAEPBVCPtrArray@@XZ 5f82c881 f
 0001:0002b894       ?GetMaxConnections@CConnectionPoint@@UAEHXZ 5f82c894 f
 0001:0002b898       ?GetContainer@CConnectionPoint@@UAEPAUIConnectionPointContainer@@XZ 5f82c898 f
 0001:0002b8b6       ?CreateConnectionArray@CConnectionPoint@@QAEXXZ 5f82c8b6 f
 0001:0002b90c       ?GetConnectionCount@CConnectionPoint@@QAEHXZ 5f82c90c f
 0001:0002b924       ?QuerySinkInterface@CConnectionPoint@@UAEPAUIUnknown@@PAU2@@Z 5f82c924 f
 0001:0002b949       ?Release@XConnPt@CConnectionPoint@@UAGKXZ 5f82c949 f
 0001:0002b958       ?AddRef@XConnPt@CConnectionPoint@@UAGKXZ 5f82c958 f
 0001:0002b969       ?QueryInterface@XConnPt@CConnectionPoint@@UAGJABU_GUID@@PAPAX@Z 5f82c969 f
 0001:0002b9b3       ?GetConnectionInterface@XConnPt@CConnectionPoint@@UAGJPAU_GUID@@@Z 5f82c9b3 f
 0001:0002b9d3       ?GetConnectionPointContainer@XConnPt@CConnectionPoint@@UAGJPAPAUIConnectionPointContainer@@@Z 5f82c9d3 f
 0001:0002b9f7       ?Advise@XConnPt@CConnectionPoint@@UAGJPAUIUnknown@@PAK@Z 5f82c9f7 f
 0001:0002ba89       ?Unadvise@XConnPt@CConnectionPoint@@UAGJK@Z 5f82ca89 f
 0001:0002baf6       ?GetInterfaceMap@CEnumConnections@@MBEPBUAFX_INTERFACEMAP@@XZ 5f82caf6 f
 0001:0002bafc       ??0CEnumConnections@@QAE@PBXI@Z 5f82cafc f
 0001:0002bb20       ??_GCEnumConnections@@UAEPAXI@Z 5f82cb20 f
 0001:0002bb20       ??_ECEnumConnections@@UAEPAXI@Z 5f82cb20 f
 0001:0002bb3c       ??1CEnumConnections@@UAE@XZ 5f82cb3c f
 0001:0002bb92       ?OnClone@CEnumConnections@@MAEPAVCEnumArray@@XZ 5f82cb92 f
 0001:0002bbdb       ?AddConnection@CEnumConnections@@QAEXPAUtagCONNECTDATA@@@Z 5f82cbdb f
 0001:0002bc44       ?EnumConnections@XConnPt@CConnectionPoint@@UAGJPAPAUIEnumConnections@@@Z 5f82cc44 f
 0001:0002bd33       ?GetInterfaceMap@CEnumConnPoints@@MBEPBUAFX_INTERFACEMAP@@XZ 5f82cd33 f
 0001:0002bd39       ??0CEnumConnPoints@@QAE@PBXI@Z 5f82cd39 f
 0001:0002bd5d       ??_GCEnumConnPoints@@UAEPAXI@Z 5f82cd5d f
 0001:0002bd5d       ??_ECEnumConnPoints@@UAEPAXI@Z 5f82cd5d f
 0001:0002bd79       ??1CEnumConnPoints@@UAE@XZ 5f82cd79 f
 0001:0002bdcf       ?AddConnPoint@CEnumConnPoints@@QAEXPAUIConnectionPoint@@@Z 5f82cdcf f
 0001:0002be2d       ?AddRef@COleConnPtContainer@@UAGKXZ 5f82ce2d f
 0001:0002be3c       ?Release@COleConnPtContainer@@UAGKXZ 5f82ce3c f
 0001:0002be4b       ?QueryInterface@COleConnPtContainer@@UAGJABU_GUID@@PAPAX@Z 5f82ce4b f
 0001:0002be62       ?EnumConnectionPoints@COleConnPtContainer@@UAGJPAPAUIEnumConnectionPoints@@@Z 5f82ce62 f
 0001:0002bf63       ?FindConnectionPoint@COleConnPtContainer@@UAGJABU_GUID@@PAPAUIConnectionPoint@@@Z 5f82cf63 f
 0001:0002bfd5       ?EnableConnections@CCmdTarget@@QAEXXZ 5f82cfd5 f
 0001:0002bfdd       ?AddRef@XOleObject@COleControl@@UAGKXZ 5f82cfdd f
 0001:0002bfef       ?Release@XOleObject@COleControl@@UAGKXZ 5f82cfef f
 0001:0002c001       ?QueryInterface@XOleObject@COleControl@@UAGJABU_GUID@@PAPAX@Z 5f82d001 f
 0001:0002c01b       ?SetClientSite@XOleObject@COleControl@@UAGJPAUIOleClientSite@@@Z 5f82d01b f
 0001:0002c18f       ?GetClientSite@XOleObject@COleControl@@UAGJPAPAUIOleClientSite@@@Z 5f82d18f f
 0001:0002c1bb       ?SetHostNames@XOleObject@COleControl@@UAGJPBG0@Z 5f82d1bb f
 0001:0002c1c0       ?Close@XOleObject@COleControl@@UAGJK@Z 5f82d1c0 f
 0001:0002c20f       ?OnClose@COleControl@@UAEXK@Z 5f82d20f f
 0001:0002c258       ?DoVerb@XOleObject@COleControl@@UAGJJPAUtagMSG@@PAUIOleClientSite@@JPAUHWND__@@PBUtagRECT@@@Z 5f82d258 f
 0001:0002c3e2       ?OnDoVerb@COleControl@@UAEHJPAUtagMSG@@PAUHWND__@@PBUtagRECT@@@Z 5f82d3e2 f
 0001:0002c3fa       ?EnumVerbs@XOleObject@COleControl@@UAGJPAPAUIEnumOLEVERB@@@Z 5f82d3fa f
 0001:0002c455       ?OnEnumVerbs@COleControl@@UAEHPAPAUIEnumOLEVERB@@@Z 5f82d455 f
 0001:0002c461       ?GetUserClassID@XOleObject@COleControl@@UAGJPAU_GUID@@@Z 5f82d461 f
 0001:0002c47e       ?GetUserType@XOleObject@COleControl@@UAGJKPAPAG@Z 5f82d47e f
 0001:0002c4e3       ?GetUserType@COleControl@@IAEXPAG@Z 5f82d4e3 f
 0001:0002c532       ?SetExtent@XOleObject@COleControl@@UAGJKPAUtagSIZE@@@Z 5f82d532 f
 0001:0002c567       ?OnSetExtent@COleControl@@UAEHPAUtagSIZE@@@Z 5f82d567 f
 0001:0002c650       ?GetExtent@XOleObject@COleControl@@UAGJKPAUtagSIZE@@@Z 5f82d650 f
 0001:0002c67c       ?Advise@XOleObject@COleControl@@UAGJPAUIAdviseSink@@PAK@Z 5f82d67c f
 0001:0002c6a9       ?Unadvise@XOleObject@COleControl@@UAGJK@Z 5f82d6a9 f
 0001:0002c6c8       ?EnumAdvise@XOleObject@COleControl@@UAGJPAPAUIEnumSTATDATA@@@Z 5f82d6c8 f
 0001:0002c6e7       ?GetMiscStatus@XOleObject@COleControl@@UAGJKPAK@Z 5f82d6e7 f
 0001:0002c714       ??0CPictureHolder@@QAE@XZ  5f82d714 f
 0001:0002c71a       ??1CPictureHolder@@QAE@XZ  5f82d71a f
 0001:0002c721       ?CreateEmpty@CPictureHolder@@QAEHXZ 5f82d721 f
 0001:0002c759       ?CreateFromBitmap@CPictureHolder@@QAEHI@Z 5f82d759 f
 0001:0002c7c0       ?CreateFromBitmap@CPictureHolder@@QAEHPAVCBitmap@@PAVCPalette@@H@Z 5f82d7c0 f
 0001:0002c814       ?CreateFromBitmap@CPictureHolder@@QAEHPAUHBITMAP__@@PAUHPALETTE__@@H@Z 5f82d814 f
 0001:0002c85e       ?CreateFromMetafile@CPictureHolder@@QAEHPAUHMETAFILE__@@HHH@Z 5f82d85e f
 0001:0002c8ae       ?CreateFromIcon@CPictureHolder@@QAEHI@Z 5f82d8ae f
 0001:0002c8d9       ?CreateFromIcon@CPictureHolder@@QAEHPAUHICON__@@H@Z 5f82d8d9 f
 0001:0002c91d       ?GetPictureDispatch@CPictureHolder@@QAEPAUIPictureDisp@@XZ 5f82d91d f
 0001:0002c93e       ?SetPictureDispatch@CPictureHolder@@QAEXPAUIPictureDisp@@@Z 5f82d93e f
 0001:0002c97d       ?Render@CPictureHolder@@QAEXPAVCDC@@ABVCRect@@1@Z 5f82d97d f
 0001:0002c9e1       ?GetType@CPictureHolder@@QAEFXZ 5f82d9e1 f
 0001:0002c9ff       ?GetDisplayString@CPictureHolder@@QAEHAAVCString@@@Z 5f82d9ff f
 0001:0002caab       ?_AfxGetArchiveStream@@YGPAUIStream@@AAVCArchive@@AAVCArchiveStream@@@Z 5f82daab f
 0001:0002cadc       ?_AfxInitBlob@@YGHPAPAXPAX@Z 5f82dadc f
 0001:0002cb30       ?_AfxCopyBlob@@YGHPAPAXPAX@Z 5f82db30 f
 0001:0002cb5d       ?_AfxCopyPropValue@@YGHGPAXPBX@Z 5f82db5d f
 0001:0002cbe4       ?ExchangeExtent@COleControl@@QAEHPAVCPropExchange@@@Z 5f82dbe4 f
 0001:0002cc6d       ?SerializeVersion@COleControl@@QAEKAAVCArchive@@KH@Z 5f82dc6d f
 0001:0002cca1       ?ResetVersion@COleControl@@QAEXK@Z 5f82dca1 f
 0001:0002ccab       ?SerializeExtent@COleControl@@QAEXAAVCArchive@@@Z 5f82dcab f
 0001:0002cd21       ?ExchangeVersion@CPropExchange@@UAEHAAKKH@Z 5f82dd21 f
 0001:0002cd72       ??0CArchivePropExchange@@QAE@AAVCArchive@@@Z 5f82dd72 f
 0001:0002cd95       ?ExchangeProp@CArchivePropExchange@@UAEHPBGGPAXPBX@Z 5f82dd95 f
 0001:0002cefa       ?ExchangeBlobProp@CArchivePropExchange@@UAEHPBGPAPAXPAX@Z 5f82defa f
 0001:0002cfa0       ?_AfxPeekAtClassIDInStream@@YGHPAUIStream@@PAU_GUID@@@Z 5f82dfa0 f
 0001:0002cfd9       ?_AfxIsSameUnknownObject@@YGHABU_GUID@@PAUIUnknown@@1@Z 5f82dfd9 f
 0001:0002d045       ?ExchangePersistentProp@CArchivePropExchange@@UAEHPBGPAPAUIUnknown@@ABU_GUID@@PAU2@@Z 5f82e045 f
 0001:0002d2a6       ?ExchangeFontProp@CArchivePropExchange@@UAEHPBGAAVCFontHolder@@PBUtagFONTDESC@@PAUIFontDisp@@@Z 5f82e2a6 f
 0001:0002d38b       ??0CResetPropExchange@@QAE@XZ 5f82e38b f
 0001:0002d3a3       ?ExchangeProp@CResetPropExchange@@UAEHPBGGPAXPBX@Z 5f82e3a3 f
 0001:0002d3b7       ?ExchangeBlobProp@CResetPropExchange@@UAEHPBGPAPAXPAX@Z 5f82e3b7 f
 0001:0002d3e4       ?ExchangePersistentProp@CResetPropExchange@@UAEHPBGPAPAUIUnknown@@ABU_GUID@@PAU2@@Z 5f82e3e4 f
 0001:0002d411       ?ExchangeFontProp@CResetPropExchange@@UAEHPBGAAVCFontHolder@@PBUtagFONTDESC@@PAUIFontDisp@@@Z 5f82e411 f
 0001:0002d428       ??0CAsyncPropExchange@@QAE@K@Z 5f82e428 f
 0001:0002d443       ?ExchangeVersion@CAsyncPropExchange@@UAEHAAKKH@Z 5f82e443 f
 0001:0002d477       ?PX_Short@@YAHPAVCPropExchange@@PBGAAF@Z 5f82e477 f
 0001:0002d497       ?PX_Short@@YAHPAVCPropExchange@@PBGAAFF@Z 5f82e497 f
 0001:0002d4ba       ?PX_ULong@@YAHPAVCPropExchange@@PBGAAKK@Z 5f82e4ba f
 0001:0002d4dd       ?PX_Color@@YAHPAVCPropExchange@@PBGAAK@Z 5f82e4dd f
 0001:0002d4fd       ?PX_Bool@@YAHPAVCPropExchange@@PBGAAH@Z 5f82e4fd f
 0001:0002d51d       ?PX_Bool@@YAHPAVCPropExchange@@PBGAAHH@Z 5f82e51d f
 0001:0002d540       ?PX_String@@YAHPAVCPropExchange@@PBGAAVCString@@@Z 5f82e540 f
 0001:0002d560       ?PX_String@@YAHPAVCPropExchange@@PBGAAVCString@@ABV2@@Z 5f82e560 f
 0001:0002d582       ?PX_String@@YAHPAVCPropExchange@@PBGAAVCString@@1@Z 5f82e582 f
 0001:0002d5a4       ?PX_Currency@@YAHPAVCPropExchange@@PBGAATtagCY@@@Z 5f82e5a4 f
 0001:0002d5c4       ?PX_Currency@@YAHPAVCPropExchange@@PBGAATtagCY@@T2@@Z 5f82e5c4 f
 0001:0002d5e7       ?PX_Float@@YAHPAVCPropExchange@@PBGAAM@Z 5f82e5e7 f
 0001:0002d607       ?PX_Float@@YAHPAVCPropExchange@@PBGAAMM@Z 5f82e607 f
 0001:0002d62a       ?PX_Double@@YAHPAVCPropExchange@@PBGAAN@Z 5f82e62a f
 0001:0002d64a       ?PX_Double@@YAHPAVCPropExchange@@PBGAANN@Z 5f82e64a f
 0001:0002d66d       ?PX_Blob@@YAHPAVCPropExchange@@PBGAAPAXPAX@Z 5f82e66d f
 0001:0002d68d       ?PX_Font@@YAHPAVCPropExchange@@PBGAAVCFontHolder@@PBUtagFONTDESC@@PAUIFontDisp@@@Z 5f82e68d f
 0001:0002d6b1       ?PX_IUnknown@@YAHPAVCPropExchange@@PBGAAPAUIUnknown@@ABU_GUID@@PAU2@@Z 5f82e6b1 f
 0001:0002d6d5       ?PX_Picture@@YAHPAVCPropExchange@@PBGAAVCPictureHolder@@@Z 5f82e6d5 f
 0001:0002d6fc       ?PX_Picture@@YAHPAVCPropExchange@@PBGAAVCPictureHolder@@2@Z 5f82e6fc f
 0001:0002d727       ?PX_VBXFontConvert@@YAHPAVCPropExchange@@AAVCFontHolder@@@Z 5f82e727 f
 0001:0002d857       ?_Afx_PX_DataPath@@YGHPAVCPropExchange@@PBGAAVCDataPathProperty@@GPBX@Z 5f82e857 f
 0001:0002d97b       ?PX_DataPath@@YAHPAVCPropExchange@@PBGAAVCDataPathProperty@@1@Z 5f82e97b f
 0001:0002d993       ?PX_DataPath@@YAHPAVCPropExchange@@PBGAAVCDataPathProperty@@ABVCString@@@Z 5f82e993 f
 0001:0002d9ab       ?GetPath@CDataPathProperty@@QBE?AVCString@@XZ 5f82e9ab f
 0001:0002d9c6       ?GetInterfaceMap@COlePropertyPage@@MBEPBUAFX_INTERFACEMAP@@XZ 5f82e9c6 f
 0001:0002d9cc       ?_GetBaseMessageMap@COlePropertyPage@@KGPBUAFX_MSGMAP@@XZ 5f82e9cc f
 0001:0002d9d2       ??0AFX_DDPDATA@@QAE@PAXHH0IPBG@Z 5f82e9d2 f
 0001:0002da05       ??_EAFX_DDPDATA@@UAEPAXI@Z 5f82ea05 f
 0001:0002da05       ??_GAFX_DDPDATA@@UAEPAXI@Z 5f82ea05 f
 0001:0002da21       ?_AfxCleanupDDPs@@YGXAAVCPtrArray@@@Z 5f82ea21 f
 0001:0002da58       ??0COlePropertyPage@@QAE@II@Z 5f82ea58 f
 0001:0002db43       ??_ECOlePropertyPage@@UAEPAXI@Z 5f82eb43 f
 0001:0002db43       ??_GCOlePropertyPage@@UAEPAXI@Z 5f82eb43 f
 0001:0002db5f       ?OnSetPageSite@COlePropertyPage@@UAEXXZ 5f82eb5f f
 0001:0002dcd7       ?OnInitDialog@COlePropertyPage@@UAEHXZ 5f82ecd7 f
 0001:0002dcdf       ?PreTranslateMessage@COlePropertyPage@@MAEHPAUtagMSG@@@Z 5f82ecdf f
 0001:0002ddcf       ?CleanupObjectArray@COlePropertyPage@@IAEXXZ 5f82edcf f
 0001:0002de67       ?OnFinalRelease@COlePropertyPage@@MAEXXZ 5f82ee67 f
 0001:0002de84       ?WindowProc@COlePropertyPage@@MAEJIIJ@Z 5f82ee84 f
 0001:0002df07       ?OnCtlColor@COlePropertyPage@@IAEPAUHBRUSH__@@PAVCDC@@PAVCWnd@@I@Z 5f82ef07 f
 0001:0002df54       ?GetObjectArray@COlePropertyPage@@QAEPAPAUIDispatch@@PAK@Z 5f82ef54 f
 0001:0002df6d       ?SetModifiedFlag@COlePropertyPage@@QAEXH@Z 5f82ef6d f
 0001:0002dfae       ?SetPageName@COlePropertyPage@@QAEXPBG@Z 5f82efae f
 0001:0002dfc0       ?SetDialogResource@COlePropertyPage@@QAEXPAX@Z 5f82efc0 f
 0001:0002e02f       ?SetHelpInfo@COlePropertyPage@@QAEXPBG0K@Z 5f82f02f f
 0001:0002e05e       ?GetPageSite@COlePropertyPage@@QAEPAUIPropertyPageSite@@XZ 5f82f05e f
 0001:0002e065       ?MessageBoxW@COlePropertyPage@@QAEHPBG0I@Z 5f82f065 f
 0001:0002e090       ?AddRef@XPropertyPage@COlePropertyPage@@UAGKXZ 5f82f090 f
 0001:0002e0a2       ?Release@XPropertyPage@COlePropertyPage@@UAGKXZ 5f82f0a2 f
 0001:0002e0b4       ?QueryInterface@XPropertyPage@COlePropertyPage@@UAGJABU_GUID@@PAPAX@Z 5f82f0b4 f
 0001:0002e0ce       ?SetPageSite@XPropertyPage@COlePropertyPage@@UAGJPAUIPropertyPageSite@@@Z 5f82f0ce f
 0001:0002e137       ?Activate@XPropertyPage@COlePropertyPage@@UAGJPAUHWND__@@PBUtagRECT@@H@Z 5f82f137 f
 0001:0002e280       ?EnumChildProc@COlePropertyPage@@KGHPAUHWND__@@J@Z 5f82f280 f
 0001:0002e290       ?EnumControls@COlePropertyPage@@KGHPAUHWND__@@J@Z 5f82f290 f
 0001:0002e2c6       ?Deactivate@XPropertyPage@COlePropertyPage@@UAGJXZ 5f82f2c6 f
 0001:0002e30f       ?GetPageInfo@XPropertyPage@COlePropertyPage@@UAGJPAUtagPROPPAGEINFO@@@Z 5f82f30f f
 0001:0002e353       ?SetObjects@XPropertyPage@COlePropertyPage@@UAGJKPAPAUIUnknown@@@Z 5f82f353 f
 0001:0002e483       ?Show@XPropertyPage@COlePropertyPage@@UAGJI@Z 5f82f483 f
 0001:0002e4ad       ?Move@XPropertyPage@COlePropertyPage@@UAGJPBUtagRECT@@@Z 5f82f4ad f
 0001:0002e4dc       ?IsPageDirty@XPropertyPage@COlePropertyPage@@UAGJXZ 5f82f4dc f
 0001:0002e4eb       ?Apply@XPropertyPage@COlePropertyPage@@UAGJXZ 5f82f4eb f
 0001:0002e5a4       ?Help@XPropertyPage@COlePropertyPage@@UAGJPBG@Z 5f82f5a4 f
 0001:0002e5fc       ?_AfxAtEndOfTabList@@YGHPAVCDialog@@I@Z 5f82f5fc f
 0001:0002e69c       ?TranslateAcceleratorW@XPropertyPage@COlePropertyPage@@UAGJPAUtagMSG@@@Z 5f82f69c f
 0001:0002e85a       ?EditProperty@XPropertyPage@COlePropertyPage@@UAGJJ@Z 5f82f85a f
 0001:0002e8b5       ?QueryInterface@XPropNotifySink@COlePropertyPage@@UAGJABU_GUID@@PAPAX@Z 5f82f8b5 f
 0001:0002e8ff       ?OnChanged@XPropNotifySink@COlePropertyPage@@UAGJJ@Z 5f82f8ff f
 0001:0002e96a       ?_AfxIsRadioButton@@YGHPAUHWND__@@@Z 5f82f96a f
 0001:0002e98d       ?OnCommand@COlePropertyPage@@MAEHIJ@Z 5f82f98d f
 0001:0002eb0e       ?IgnoreApply@COlePropertyPage@@QAEXI@Z 5f82fb0e f
 0001:0002eb23       ?GetControlStatus@COlePropertyPage@@QAEHI@Z 5f82fb23 f
 0001:0002eb57       ?SetControlStatus@COlePropertyPage@@QAEHIH@Z 5f82fb57 f
 0001:0002eb91       ?SetPropText@COlePropertyPage@@QAEHPBGAAE@Z 5f82fb91 f
 0001:0002ec48       ?GetPropText@COlePropertyPage@@QAEHPBGPAE@Z 5f82fc48 f
 0001:0002ed0f       ?SetPropText@COlePropertyPage@@QAEHPBGAAF@Z 5f82fd0f f
 0001:0002edc6       ?GetPropText@COlePropertyPage@@QAEHPBGPAF@Z 5f82fdc6 f
 0001:0002ee96       ?SetPropText@COlePropertyPage@@QAEHPBGAAH@Z 5f82fe96 f
 0001:0002ef4b       ?GetPropText@COlePropertyPage@@QAEHPBGPAH@Z 5f82ff4b f
 0001:0002f012       ?SetPropText@COlePropertyPage@@QAEHPBGAAI@Z 5f830012 f
 0001:0002f0c7       ?GetPropText@COlePropertyPage@@QAEHPBGPAI@Z 5f8300c7 f
 0001:0002f18e       ?SetPropText@COlePropertyPage@@QAEHPBGAAJ@Z 5f83018e f
 0001:0002f243       ?GetPropText@COlePropertyPage@@QAEHPBGPAJ@Z 5f830243 f
 0001:0002f30a       ?SetPropText@COlePropertyPage@@QAEHPBGAAK@Z 5f83030a f
 0001:0002f3bf       ?GetPropText@COlePropertyPage@@QAEHPBGPAK@Z 5f8303bf f
 0001:0002f486       ?SetPropText@COlePropertyPage@@QAEHPBGAAM@Z 5f830486 f
 0001:0002f540       ?GetPropText@COlePropertyPage@@QAEHPBGPAM@Z 5f830540 f
 0001:0002f61a       ?SetPropText@COlePropertyPage@@QAEHPBGAAN@Z 5f83061a f
 0001:0002f6d4       ?GetPropText@COlePropertyPage@@QAEHPBGPAN@Z 5f8306d4 f
 0001:0002f7af       ?SetPropText@COlePropertyPage@@QAEHPBGAAVCString@@@Z 5f8307af f
 0001:0002f864       ?GetPropText@COlePropertyPage@@QAEHPBGPAVCString@@@Z 5f830864 f
 0001:0002f997       ?SetPropCheck@COlePropertyPage@@QAEHPBGH@Z 5f830997 f
 0001:0002fa56       ?GetPropCheck@COlePropertyPage@@QAEHPBGPAH@Z 5f830a56 f
 0001:0002fb2d       ?SetPropRadio@COlePropertyPage@@QAEHPBGH@Z 5f830b2d f
 0001:0002fbe2       ?GetPropRadio@COlePropertyPage@@QAEHPBGPAH@Z 5f830be2 f
 0001:0002fcaf       ?SetPropIndex@COlePropertyPage@@QAEHPBGH@Z 5f830caf f
 0001:0002fcbf       ?GetPropIndex@COlePropertyPage@@QAEHPBGPAH@Z 5f830cbf f
 0001:0002fccf       ?DDP_EndText@@YGXPAVCDataExchange@@HPAEPBG@Z 5f830ccf f
 0001:0002fceb       ?DDP_Text@@YGXPAVCDataExchange@@HAAEPBG@Z 5f830ceb f
 0001:0002fd5d       ?DDP_EndText@@YGXPAVCDataExchange@@HPAFPBG@Z 5f830d5d f
 0001:0002fd79       ?DDP_Text@@YGXPAVCDataExchange@@HAAFPBG@Z 5f830d79 f
 0001:0002fdeb       ?DDP_EndText@@YGXPAVCDataExchange@@HPAHPBG@Z 5f830deb f
 0001:0002fe07       ?DDP_Text@@YGXPAVCDataExchange@@HAAHPBG@Z 5f830e07 f
 0001:0002fe79       ?DDP_EndText@@YGXPAVCDataExchange@@HPAIPBG@Z 5f830e79 f
 0001:0002fe95       ?DDP_Text@@YGXPAVCDataExchange@@HAAIPBG@Z 5f830e95 f
 0001:0002ff07       ?DDP_EndText@@YGXPAVCDataExchange@@HPAJPBG@Z 5f830f07 f
 0001:0002ff23       ?DDP_Text@@YGXPAVCDataExchange@@HAAJPBG@Z 5f830f23 f
 0001:0002ff95       ?DDP_EndText@@YGXPAVCDataExchange@@HPAKPBG@Z 5f830f95 f
 0001:0002ffb1       ?DDP_Text@@YGXPAVCDataExchange@@HAAKPBG@Z 5f830fb1 f
 0001:00030023       ?DDP_EndText@@YGXPAVCDataExchange@@HPAMPBG@Z 5f831023 f
 0001:0003003f       ?DDP_Text@@YGXPAVCDataExchange@@HAAMPBG@Z 5f83103f f
 0001:000300b1       ?DDP_EndText@@YGXPAVCDataExchange@@HPANPBG@Z 5f8310b1 f
 0001:000300cd       ?DDP_Text@@YGXPAVCDataExchange@@HAANPBG@Z 5f8310cd f
 0001:0003013f       ?DDP_EndText@@YGXPAVCDataExchange@@HPAVCString@@PBG@Z 5f83113f f
 0001:0003015b       ?DDP_Text@@YGXPAVCDataExchange@@HAAVCString@@PBG@Z 5f83115b f
 0001:000301cd       ?DDP_EndCheck@@YGXPAVCDataExchange@@HPAHPBG@Z 5f8311cd f
 0001:000301eb       ?DDP_Check@@YGXPAVCDataExchange@@HAAHPBG@Z 5f8311eb f
 0001:0003025d       ?DDP_EndRadio@@YGXPAVCDataExchange@@HPAHPBG@Z 5f83125d f
 0001:0003027b       ?DDP_Radio@@YGXPAVCDataExchange@@HAAHPBG@Z 5f83127b f
 0001:000302ed       ?DDP_PostProcessing@@YGXPAVCDataExchange@@@Z 5f8312ed f
 0001:000303dd       ?InitStockPropMask@COleControl@@IAEXXZ 5f8313dd f
 0001:00030448       ?_AfxToggleBorderStyle@@YGXPAVCWnd@@@Z 5f831448 f
 0001:00030482       ?_AfxToggleAppearance@@YGXPAVCWnd@@@Z 5f831482 f
 0001:000304bc       ?ExchangeStockProps@COleControl@@QAEXPAVCPropExchange@@@Z 5f8314bc f
 0001:000307aa       ?SerializeStockProps@COleControl@@QAEXAAVCArchive@@@Z 5f8317aa f
 0001:00030b7e       ?ResetStockProps@COleControl@@QAEXXZ 5f831b7e f
 0001:00030c67       ?GetAppearance@COleControl@@QAEFXZ 5f831c67 f
 0001:00030c6f       ?SetAppearance@COleControl@@QAEXF@Z 5f831c6f f
 0001:00030ce2       ?GetBackColor@COleControl@@QAEKXZ 5f831ce2 f
 0001:00030ce9       ?SetBackColor@COleControl@@QAEXK@Z 5f831ce9 f
 0001:00030d59       ?OnBackColorChanged@COleControl@@UAEXXZ 5f831d59 f
 0001:00030d63       ?GetBorderStyle@COleControl@@QAEFXZ 5f831d63 f
 0001:00030d6b       ?SetBorderStyle@COleControl@@QAEXF@Z 5f831d6b f
 0001:00030dde       ?InternalGetText@COleControl@@QAEABVCString@@XZ 5f831dde f
 0001:00030e55       ?GetText@COleControl@@QAEPAGXZ 5f831e55 f
 0001:00030e5c       ?AllocSysString@CString@@QBEPAGXZ 5f831e5c f
 0001:00030e78       ?SetText@COleControl@@QAEXPBG@Z 5f831e78 f
 0001:00030eaa       ?OnSetText@COleControl@@IAEJIJ@Z 5f831eaa f
 0001:00030fb4       ?GetEnabled@COleControl@@QAEHXZ 5f831fb4 f
 0001:00030fbb       ?SetEnabled@COleControl@@QAEXH@Z 5f831fbb f
 0001:00031038       ?InternalGetFont@COleControl@@QAEAAVCFontHolder@@XZ 5f832038 f
 0001:0003103f       ?GetFont@COleControl@@QAEPAUIFontDisp@@XZ 5f83203f f
 0001:00031045       ?GetFontDispatch@CFontHolder@@QAEPAUIFontDisp@@XZ 5f832045 f
 0001:00031066       ?SetFont@COleControl@@QAEXPAUIFontDisp@@@Z 5f832066 f
 0001:0003109b       ?OnFontChanged@COleControl@@UAEXXZ 5f83209b f
 0001:00031140       ?GetForeColor@COleControl@@QAEKXZ 5f832140 f
 0001:00031147       ?SetForeColor@COleControl@@QAEXK@Z 5f832147 f
 0001:000311b7       ?GetHwnd@COleControl@@QAEIXZ 5f8321b7 f
 0001:000311c7       ?GetReadyState@COleControl@@QAEJXZ 5f8321c7 f
 0001:000311ce       ?QueryInterface@XFontNotification@COleControl@@UAGJABU_GUID@@PAPAX@Z 5f8321ce f
 0001:00031212       ?OnChanged@XFontNotification@COleControl@@UAGJJ@Z 5f832212 f
 0001:00031271       ?SelectStockFont@COleControl@@QAEPAVCFont@@PAVCDC@@@Z 5f832271 f
 0001:00031284       ?SelectFontObject@COleControl@@QAEPAVCFont@@PAVCDC@@AAVCFontHolder@@@Z 5f832284 f
 0001:000312a1       ?GetStockTextMetrics@COleControl@@QAEXPAUtagTEXTMETRICW@@@Z 5f8322a1 f
 0001:000312b3       ?GetFontTextMetrics@COleControl@@QAEXPAUtagTEXTMETRICW@@AAVCFontHolder@@@Z 5f8322b3 f
 0001:000312c3       ?_GetI4Property@@YGHPAUIDispatch@@JPAK@Z 5f8322c3 f
 0001:0003137e       ?GetAmbientDispatchDriver@COleControl@@IAEPAVCOleDispatchDriver@@XZ 5f83237e f
 0001:000313bd       ?GetAmbientProperty@COleControl@@QAEHJGPAX@Z 5f8323bd f
 0001:000314fd       ?AmbientAppearance@COleControl@@QAEFXZ 5f8324fd f
 0001:0003151e       ?AmbientBackColor@COleControl@@QAEKXZ 5f83251e f
 0001:00031546       ?AmbientDisplayName@COleControl@@QAE?AVCString@@XZ 5f832546 f
 0001:000315a8       ?AmbientFont@COleControl@@QAEPAUIFontDisp@@XZ 5f8325a8 f
 0001:000315c8       ?AmbientForeColor@COleControl@@QAEKXZ 5f8325c8 f
 0001:000315f0       ?AmbientLocaleID@COleControl@@QAEKXZ 5f8325f0 f
 0001:00031610       ?AmbientScaleUnits@COleControl@@QAE?AVCString@@XZ 5f832610 f
 0001:00031672       ?AmbientTextAlign@COleControl@@QAEFXZ 5f832672 f
 0001:00031693       ?AmbientUserMode@COleControl@@QAEHXZ 5f832693 f
 0001:000316b7       ?AmbientUIDead@COleControl@@QAEHXZ 5f8326b7 f
 0001:000316d7       ?AmbientShowGrabHandles@COleControl@@QAEHXZ 5f8326d7 f
 0001:000316fb       ?AmbientShowHatching@COleControl@@QAEHXZ 5f8326fb f
 0001:0003171f       ?BoundPropertyChanged@COleControl@@QAEXJ@Z 5f83271f f
 0001:00031757       ?BoundPropertyRequestEdit@COleControl@@QAEHJ@Z 5f832757 f
 0001:00031799       ?SetNotPermitted@COleControl@@QAEXXZ 5f832799 f
 0001:000317ab       ?SetNotSupported@COleControl@@QAEXXZ 5f8327ab f
 0001:000317bd       ?GetNotSupported@COleControl@@QAEXXZ 5f8327bd f
 0001:000317cf       ?AddRef@XPerPropertyBrowsing@COleControl@@UAGKXZ 5f8327cf f
 0001:000317e1       ?Release@XPerPropertyBrowsing@COleControl@@UAGKXZ 5f8327e1 f
 0001:000317f3       ?QueryInterface@XPerPropertyBrowsing@COleControl@@UAGJABU_GUID@@PAPAX@Z 5f8327f3 f
 0001:0003180d       ?GetDisplayString@XPerPropertyBrowsing@COleControl@@UAGJJPAPAG@Z 5f83280d f
 0001:0003189e       ?OnGetDisplayString@COleControl@@UAEHJAAVCString@@@Z 5f83289e f
 0001:00031913       ?MapPropertyToPage@XPerPropertyBrowsing@COleControl@@UAGJJPAU_GUID@@@Z 5f832913 f
 0001:000319a7       ?OnMapPropertyToPage@COleControl@@UAEHJPAU_GUID@@PAH@Z 5f8329a7 f
 0001:000319ec       ?GetPredefinedStrings@XPerPropertyBrowsing@COleControl@@UAGJJPAUtagCALPOLESTR@@PAUtagCADWORD@@@Z 5f8329ec f
 0001:00031b7b       ?_AfxCopyString@@YGPAGPBG@Z 5f832b7b f
 0001:00031bb1       ?OnGetPredefinedStrings@COleControl@@UAEHJPAVCStringArray@@PAVCDWordArray@@@Z 5f832bb1 f
 0001:00031c7d       ?GetPredefinedValue@XPerPropertyBrowsing@COleControl@@UAGJJKPAUtagVARIANT@@@Z 5f832c7d f
 0001:00031cde       ?OnGetPredefinedValue@COleControl@@UAEHJKPAUtagVARIANT@@@Z 5f832cde f
 0001:00031d16       ?Load@COleControl@@QAEXPBGAAVCDataPathProperty@@@Z 5f832d16 f
 0001:00031d2d       ?Open@CDataPathProperty@@UAEHPAVCFileException@@@Z 5f832d2d f
 0001:00031d54       ?Open@CDataPathProperty@@UAEHPBGPAVCFileException@@@Z 5f832d54 f
 0001:00031d75       ?Open@CDataPathProperty@@UAEHPAVCOleControl@@PAVCFileException@@@Z 5f832d75 f
 0001:00031d8b       ?Open@CDataPathProperty@@UAEHPBGPAVCOleControl@@PAVCFileException@@@Z 5f832d8b f
 0001:00031db3       ?_AfxTransferFileContent@@YAKPAVCFile@@0@Z 5f832db3 f
 0001:00031dfc       ?OnDataAvailable@CCachedDataPathProperty@@UAEXKK@Z 5f832dfc f
 0001:00031e73       ?Close@CCachedDataPathProperty@@UAEXXZ 5f832e73 f
 0001:00031e8a       ?ResetData@CCachedDataPathProperty@@UAEXXZ 5f832e8a f
 0001:00031e96       ?_AfxCreateMemoryStream@@YGPAUIStream@@XZ 5f832e96 f
 0001:00031ed4       ?GetPropsetData@COleControl@@IAEHPAUtagFORMATETC@@PAUtagSTGMEDIUM@@ABU_GUID@@@Z 5f832ed4 f
 0001:00032100       ?SetPropsetData@COleControl@@IAEHPAUtagFORMATETC@@PAUtagSTGMEDIUM@@ABU_GUID@@@Z 5f833100 f
 0001:00032273       ??0CPropsetPropExchange@@QAE@AAVCPropertySection@@PAUIStorage@@H@Z 5f833273 f
 0001:000322a2       ?_AfxGetSizeOfVarType@@YGIG@Z 5f8332a2 f
 0001:000322d9       ?_AfxCoerceNumber@@YGHPAXG0G@Z 5f8332d9 f
 0001:00032354       ?_AfxIsSamePropValue@@YGHGPBX0@Z 5f833354 f
 0001:000323c2       ?ExchangeProp@CPropsetPropExchange@@UAEHPBGGPAXPBX@Z 5f8333c2 f
 0001:000325c2       ?ExchangeBlobProp@CPropsetPropExchange@@UAEHPBGPAPAXPAX@Z 5f8335c2 f
 0001:000326a2       ?_AfxSaveStreamDataAsBlobProp@@YGHPAUIStream@@AAVCPropertySection@@KK@Z 5f8336a2 f
 0001:0003276b       ?_AfxInitStreamDataFromBlobProp@@YGHPAUIStream@@PAVCProperty@@@Z 5f83376b f
 0001:000327c5       ?_AfxCreateFontFromStream@@YGPAUIFont@@PAUIStream@@@Z 5f8337c5 f
 0001:00032896       ?_AfxLoadObjectFromStreamedPropset@@YGHPAUIUnknown@@PAUIStream@@@Z 5f833896 f
 0001:0003290b       ?_AfxGetClassIDFromStreamedPropset@@YGHPAU_GUID@@PAUIStream@@@Z 5f83390b f
 0001:0003297b       ?_AfxCreateObjectFromStreamedPropset@@YGPAUIUnknown@@PAUIStream@@ABU_GUID@@@Z 5f83397b f
 0001:00032a6b       ?_AfxLoadStreamFromPropset@@YGPAUIStream@@AAVCPropertySection@@PBGAAK@Z 5f833a6b f
 0001:00032ad6       ?_AfxSaveObjectInPropset@@YGHPAUIUnknown@@AAVCPropertySection@@K@Z 5f833ad6 f
 0001:00032bfb       ?ExchangePersistentProp@CPropsetPropExchange@@UAEHPBGPAPAUIUnknown@@ABU_GUID@@PAU2@@Z 5f833bfb f
 0001:00032d3f       ?ExchangeFontProp@CPropsetPropExchange@@UAEHPBGAAVCFontHolder@@PBUtagFONTDESC@@PAUIFontDisp@@@Z 5f833d3f f
 0001:00032df9       ?AddRef@XPersistStorage@COleControl@@UAGKXZ 5f833df9 f
 0001:00032e0b       ?Release@XPersistStorage@COleControl@@UAGKXZ 5f833e0b f
 0001:00032e1d       ?QueryInterface@XPersistStorage@COleControl@@UAGJABU_GUID@@PAPAX@Z 5f833e1d f
 0001:00032e37       ?GetClassID@XPersistStorage@COleControl@@UAGJPAU_GUID@@@Z 5f833e37 f
 0001:00032e54       ?IsDirty@XPersistStorage@COleControl@@UAGJXZ 5f833e54 f
 0001:00032e9e       ?InitNew@XPersistStorage@COleControl@@UAGJPAUIStorage@@@Z 5f833e9e f
 0001:00032f36       ?Load@XPersistStorage@COleControl@@UAGJPAUIStorage@@@Z 5f833f36 f
 0001:0003304f       ?Save@XPersistStorage@COleControl@@UAGJPAUIStorage@@H@Z 5f83404f f
 0001:0003311e       ?SaveCompleted@XPersistStorage@COleControl@@UAGJPAUIStorage@@@Z 5f83411e f
 0001:00033163       ?HandsOffStorage@XPersistStorage@COleControl@@UAGJXZ 5f834163 f
 0001:00033195       ?AddRef@XPersistStreamInit@COleControl@@UAGKXZ 5f834195 f
 0001:000331a7       ?Release@XPersistStreamInit@COleControl@@UAGKXZ 5f8341a7 f
 0001:000331b9       ?QueryInterface@XPersistStreamInit@COleControl@@UAGJABU_GUID@@PAPAX@Z 5f8341b9 f
 0001:000331d3       ?GetClassID@XPersistStreamInit@COleControl@@UAGJPAU_GUID@@@Z 5f8341d3 f
 0001:000331f0       ?IsDirty@XPersistStreamInit@COleControl@@UAGJXZ 5f8341f0 f
 0001:00033205       ?Load@XPersistStreamInit@COleControl@@UAGJPAUIStream@@@Z 5f834205 f
 0001:0003324f       ?Save@XPersistStreamInit@COleControl@@UAGJPAUIStream@@H@Z 5f83424f f
 0001:000332a6       ?InitNew@XPersistStreamInit@COleControl@@UAGJXZ 5f8342a6 f
 0001:00033314       ?AddRef@XPersistMemory@COleControl@@UAGKXZ 5f834314 f
 0001:00033326       ?Release@XPersistMemory@COleControl@@UAGKXZ 5f834326 f
 0001:00033338       ?QueryInterface@XPersistMemory@COleControl@@UAGJABU_GUID@@PAPAX@Z 5f834338 f
 0001:00033352       ?GetClassID@XPersistMemory@COleControl@@UAGJPAU_GUID@@@Z 5f834352 f
 0001:0003336f       ?IsDirty@XPersistMemory@COleControl@@UAGJXZ 5f83436f f
 0001:00033384       ?Load@XPersistMemory@COleControl@@UAGJPAXK@Z 5f834384 f
 0001:00033492       ?InitNew@XPersistMemory@COleControl@@UAGJXZ 5f834492 f
 0001:00033500       ?Create@CReflectorWnd@@QAEHABVCRect@@PAUHWND__@@@Z 5f834500 f
 0001:00033544       ?PostNcDestroy@CReflectorWnd@@MAEXXZ 5f834544 f
 0001:00033565       ?WindowProc@CReflectorWnd@@MAEJIIJ@Z 5f834565 f
 0001:000335f8       ?SetControl@CReflectorWnd@@QAEXPAVCOleControl@@@Z 5f8345f8 f
 0001:00033602       ?WindowProc@CParkingWnd@@UAEJIIJ@Z 5f834602 f
 0001:0003370f       ?_AfxRecursiveRegDeleteKey@@YGJPAUHKEY__@@PAG@Z 5f83470f f
 0001:00033754       ?_AfxUnregisterInterfaces@@YAXPAUITypeLib@@@Z 5f834754 f
 0001:00033814       ?AfxOleRegisterTypeLib@@YGHPAUHINSTANCE__@@ABU_GUID@@PBG2@Z 5f834814 f
 0001:00033933       ?AfxOleUnregisterTypeLib@@YGHABU_GUID@@GGK@Z 5f834933 f
 0001:00033bc0       ?AfxOleRegisterControlClass@@YGHPAUHINSTANCE__@@ABU_GUID@@PBGIIHK1GG@Z 5f834bc0 f
 0001:00033e3d       ?AfxOleUnregisterClass@@YGHABU_GUID@@PBG@Z 5f834e3d f
 0001:00033f8c       ?AfxOleRegisterPropertyPageClass@@YGHPAUHINSTANCE__@@ABU_GUID@@I@Z 5f834f8c f
 0001:00033fa2       ?AfxOleRegisterPropertyPageClass@@YGHPAUHINSTANCE__@@ABU_GUID@@IH@Z 5f834fa2 f
 0001:000340f9       ?_AfxOffsetTrackerRect@@YGXAAVCRect@@PAVCWnd@@@Z 5f8350f9 f
 0001:00034168       ?CreateTracker@COleControl@@IAEXHH@Z 5f835168 f
 0001:0003417a       ?CreateTracker@COleControl@@IAEXHHPBUtagRECT@@@Z 5f83517a f
 0001:0003424b       ?DestroyTracker@COleControl@@IAEXXZ 5f83524b f
 0001:00034289       ?OnNcPaint@COleControl@@IAEXXZ 5f835289 f
 0001:000343f1       ?OnNcCalcSize@COleControl@@IAEXHPAUtagNCCALCSIZE_PARAMS@@@Z 5f8353f1 f
 0001:0003443d       ?OnNcHitTest@COleControl@@IAEIVCPoint@@@Z 5f83543d f
 0001:0003451c       ?OnNcLButtonDown@COleControl@@IAEXIVCPoint@@@Z 5f83551c f
 0001:000346de       ?OnSetCursor@COleControl@@IAEHPAVCWnd@@II@Z 5f8356de f
 0001:00034744       ??_ECControlRectTracker@@UAEPAXI@Z 5f835744 f
 0001:00034744       ??_GCControlRectTracker@@UAEPAXI@Z 5f835744 f
 0001:00034760       ??1CRectTracker@@UAE@XZ    5f835760 f
 0001:00034760       ??1CControlRectTracker@@UAE@XZ 5f835760 f
 0001:00034767       ?OnGetViewExtent@COleControl@@UAEHKJPAUtagDVTARGETDEVICE@@PAUtagSIZE@@@Z 5f835767 f
 0001:00034799       ?OnGetViewRect@COleControl@@UAEHKPAU_RECTL@@@Z 5f835799 f
 0001:000347d0       ?OnGetViewStatus@COleControl@@UAEKXZ 5f8357d0 f
 0001:000347d4       ?OnQueryHitPoint@COleControl@@UAEHKPBUtagRECT@@UtagPOINT@@JPAK@Z 5f8357d4 f
 0001:000347ee       ?OnQueryHitRect@COleControl@@UAEHKPBUtagRECT@@0JPAK@Z 5f8357ee f
 0001:00034808       ?OnGetNaturalExtent@COleControl@@UAEHKJPAUtagDVTARGETDEVICE@@PAUHDC__@@PAUtagExtentInfo@@PAUtagSIZE@@@Z 5f835808 f
 0001:0003480d       ?AddRef@XViewObject@COleControl@@UAGKXZ 5f83580d f
 0001:0003481f       ?Release@XViewObject@COleControl@@UAGKXZ 5f83581f f
 0001:00034831       ?QueryInterface@XViewObject@COleControl@@UAGJABU_GUID@@PAPAX@Z 5f835831 f
 0001:0003484b       ?Draw@XViewObject@COleControl@@UAGJKJPAXPAUtagDVTARGETDEVICE@@PAUHDC__@@2PBU_RECTL@@3P6GHK@ZK@Z 5f83584b f
 0001:00034a14       ?GetColorSet@XViewObject@COleControl@@UAGJKJPAXPAUtagDVTARGETDEVICE@@PAUHDC__@@PAPAUtagLOGPALETTE@@@Z 5f835a14 f
 0001:00034a82       ?SetAdvise@XViewObject@COleControl@@UAGJKKPAUIAdviseSink@@@Z 5f835a82 f
 0001:00034b20       ?GetAdvise@XViewObject@COleControl@@UAGJPAK0PAPAUIAdviseSink@@@Z 5f835b20 f
 0001:00034b86       ?GetExtent@XViewObject@COleControl@@UAGJKJPAUtagDVTARGETDEVICE@@PAUtagSIZE@@@Z 5f835b86 f
 0001:00034bb8       ?GetRect@XViewObject@COleControl@@UAGJKPAU_RECTL@@@Z 5f835bb8 f
 0001:00034be7       ?GetViewStatus@XViewObject@COleControl@@UAGJPAK@Z 5f835be7 f
 0001:00034c08       ?QueryHitPoint@XViewObject@COleControl@@UAGJKPBUtagRECT@@UtagPOINT@@JPAK@Z 5f835c08 f
 0001:00034c40       ?QueryHitRect@XViewObject@COleControl@@UAGJKPBUtagRECT@@0JPAK@Z 5f835c40 f
 0001:00034c75       ?GetNaturalExtent@XViewObject@COleControl@@UAGJKJPAUtagDVTARGETDEVICE@@PAUHDC__@@PAUtagExtentInfo@@PAUtagSIZE@@@Z 5f835c75 f
 0001:00034cad       ?_AfxCountPrefixedStringA@@YGPAXPBD@Z 5f835cad f
 0001:00034ce4       ?_AfxCountPrefixedStringW@@YGPAXPBG@Z 5f835ce4 f
 0001:00034d1f       ?_AfxConvertStringProp@@YGPAEPAEKKI@Z 5f835d1f f
 0001:00034e25       ??0CProperty@@QAE@XZ       5f835e25 f
 0001:00034e32       ??0CProperty@@QAE@KQAXK@Z  5f835e32 f
 0001:00034e59       ?FreeValue@CProperty@@AAEXXZ 5f835e59 f
 0001:00034e59       ??1CProperty@@QAE@XZ       5f835e59 f
 0001:00034e71       ?Set@CProperty@@QAEHKQAXK@Z 5f835e71 f
 0001:00034e8a       ?Set@CProperty@@QAEHQAXK@Z 5f835e8a f
 0001:00034e9d       ?Set@CProperty@@QAEHQAX@Z  5f835e9d f
 0001:00035055       ?Get@CProperty@@QAEPAXXZ   5f836055 f
 0001:0003505d       ?Get@CProperty@@QAEPAXPAK@Z 5f83605d f
 0001:00035109       ?SetType@CProperty@@QAEXK@Z 5f836109 f
 0001:00035113       ?GetID@CProperty@@QAEKXZ   5f836113 f
 0001:00035116       ?SetID@CProperty@@QAEXK@Z  5f836116 f
 0001:0003511f       ?GetRawValue@CProperty@@QAEPAXXZ 5f83611f f
 0001:00035123       ?WriteToStream@CProperty@@QAEHPAUIStream@@@Z 5f836123 f
 0001:000352c5       ?ReadFromStream@CProperty@@QAEHPAUIStream@@@Z 5f8362c5 f
 0001:000354da       ?AllocValue@CProperty@@AAEPAXK@Z 5f8364da f
 0001:000354ef       ??0CPropertySection@@QAE@XZ 5f8364ef f
 0001:0003554a       ??0CPropertySection@@QAE@U_GUID@@@Z 5f83654a f
 0001:000355a5       ??1CPropertySection@@QAE@XZ 5f8365a5 f
 0001:000355f3       ?GetFormatID@CPropertySection@@QAE?AU_GUID@@XZ 5f8365f3 f
 0001:00035606       ?SetFormatID@CPropertySection@@QAEXU_GUID@@@Z 5f836606 f
 0001:00035617       ?Set@CPropertySection@@QAEHKPAXK@Z 5f836617 f
 0001:00035697       ?Set@CPropertySection@@QAEHKPAX@Z 5f836697 f
 0001:000356c5       ?Get@CPropertySection@@QAEPAXK@Z 5f8366c5 f
 0001:000356d3       ?Get@CPropertySection@@QAEPAXKPAK@Z 5f8366d3 f
 0001:000356f2       ?Remove@CPropertySection@@QAEXK@Z 5f8366f2 f
 0001:00035731       ?RemoveAll@CPropertySection@@QAEXXZ 5f836731 f
 0001:0003576a       ?GetProperty@CPropertySection@@QAEPAVCProperty@@K@Z 5f83676a f
 0001:00035787       ?AddProperty@CPropertySection@@QAEXPAVCProperty@@@Z 5f836787 f
 0001:0003579d       ?GetSize@CPropertySection@@QAEKXZ 5f83679d f
 0001:000357a1       ?GetCount@CPropertySection@@QAEKXZ 5f8367a1 f
 0001:000357a5       ?GetList@CPropertySection@@QAEPAVCPtrList@@XZ 5f8367a5 f
 0001:000357a9       ?WriteToStream@CPropertySection@@QAEHPAUIStream@@@Z 5f8367a9 f
 0001:000358fe       ?ReadFromStream@CPropertySection@@QAEHPAUIStream@@T_LARGE_INTEGER@@@Z 5f8368fe f
 0001:00035a2b       ?GetID@CPropertySection@@QAEHPBGPAK@Z 5f836a2b f
 0001:00035a8f       ?SetName@CPropertySection@@QAEHKPBG@Z 5f836a8f f
 0001:00035b1a       ?ReadNameDictFromStream@CPropertySection@@QAEHPAUIStream@@@Z 5f836b1a f
 0001:00035c0b       ?_AfxWriteNameDictEntry@@YGHPAUIStream@@KAAVCString@@@Z 5f836c0b f
 0001:00035c88       ?WriteNameDictToStream@CPropertySection@@QAEHPAUIStream@@@Z 5f836c88 f
 0001:00035d39       ?SetSectionName@CPropertySection@@QAEHPBG@Z 5f836d39 f
 0001:00035d4b       ?GetSectionName@CPropertySection@@QAEPBGXZ 5f836d4b f
 0001:00035d4f       ??0CPropertySet@@QAE@XZ    5f836d4f f
 0001:00035d8f       ??0CPropertySet@@QAE@U_GUID@@@Z 5f836d8f f
 0001:00035dd0       ?Set@CPropertySet@@QAEHU_GUID@@KPAXK@Z 5f836dd0 f
 0001:00035e56       ?Set@CPropertySet@@QAEHU_GUID@@KPAX@Z 5f836e56 f
 0001:00035e86       ?Get@CPropertySet@@QAEPAXU_GUID@@KPAK@Z 5f836e86 f
 0001:00035eb6       ?Get@CPropertySet@@QAEPAXU_GUID@@K@Z 5f836eb6 f
 0001:00035ed5       ?Remove@CPropertySet@@QAEXU_GUID@@K@Z 5f836ed5 f
 0001:00035efd       ?Remove@CPropertySet@@QAEXU_GUID@@@Z 5f836efd f
 0001:00035f54       ?RemoveAll@CPropertySet@@QAEXXZ 5f836f54 f
 0001:00035f8d       ?GetSection@CPropertySet@@QAEPAVCPropertySection@@U_GUID@@@Z 5f836f8d f
 0001:00035fbc       ?AddSection@CPropertySet@@QAEPAVCPropertySection@@U_GUID@@@Z 5f836fbc f
 0001:0003602d       ?AddSection@CPropertySet@@QAEXPAVCPropertySection@@@Z 5f83702d f
 0001:00036043       ?GetProperty@CPropertySet@@QAEPAVCProperty@@U_GUID@@K@Z 5f837043 f
 0001:0003606f       ?AddProperty@CPropertySet@@QAEXU_GUID@@PAVCProperty@@@Z 5f83706f f
 0001:00036097       ?GetByteOrder@CPropertySet@@QAEGXZ 5f837097 f
 0001:0003609b       ?GetFormatVersion@CPropertySet@@QAEGXZ 5f83709b f
 0001:000360a0       ?SetFormatVersion@CPropertySet@@QAEXG@Z 5f8370a0 f
 0001:000360ac       ?GetOSVersion@CPropertySet@@QAEKXZ 5f8370ac f
 0001:000360b0       ?GetClassID@CPropertySet@@QAE?AU_GUID@@XZ 5f8370b0 f
 0001:000360c4       ?SetClassID@CPropertySet@@QAEXU_GUID@@@Z 5f8370c4 f
 0001:000360d6       ?GetCount@CPropertySet@@QAEKXZ 5f8370d6 f
 0001:000360da       ?GetList@CPropertySet@@QAEPAVCPtrList@@XZ 5f8370da f
 0001:000360de       ?WriteToStream@CPropertySet@@QAEHPAUIStream@@@Z 5f8370de f
 0001:000361b3       ?ReadFromStream@CPropertySet@@QAEHPAUIStream@@@Z 5f8371b3 f
 0001:000362e2       ??0CBlobProperty@@QAE@PAX@Z 5f8372e2 f
 0001:000362fb       ?AddRef@CBlobProperty@@UAGKXZ 5f8372fb f
 0001:0003630c       ?Release@CBlobProperty@@UAGKXZ 5f83730c f
 0001:00036332       ?QueryInterface@CBlobProperty@@UAGJABU_GUID@@PAPAX@Z 5f837332 f
 0001:0003639a       ?GetClassID@CBlobProperty@@UAGJPAU_GUID@@@Z 5f83739a f
 0001:000363b0       ?Load@CBlobProperty@@UAGJPAUIStream@@@Z 5f8373b0 f
 0001:0003644f       ?Save@CBlobProperty@@UAGJPAUIStream@@H@Z 5f83744f f
 0001:000364a8       ?GetSizeMax@CBlobProperty@@UAGJPAT_ULARGE_INTEGER@@@Z 5f8374a8 f
 0001:000364df       ??0CPropbagPropExchange@@QAE@PAUIPropertyBag@@PAUIErrorLog@@HH@Z 5f8374df f
 0001:00036528       ?ExchangeProp@CPropbagPropExchange@@UAEHPBGGPAXPBX@Z 5f837528 f
 0001:000366dc       ?ExchangeBlobProp@CPropbagPropExchange@@UAEHPBGPAPAXPAX@Z 5f8376dc f
 0001:000367b6       ?ExchangeFontProp@CPropbagPropExchange@@UAEHPBGAAVCFontHolder@@PBUtagFONTDESC@@PAUIFontDisp@@@Z 5f8377b6 f
 0001:0003687a       ?ExchangePersistentProp@CPropbagPropExchange@@UAEHPBGPAPAUIUnknown@@ABU_GUID@@PAU2@@Z 5f83787a f
 0001:0003693d       ?AddRef@XPersistPropertyBag@COleControl@@UAGKXZ 5f83793d f
 0001:0003694f       ?Release@XPersistPropertyBag@COleControl@@UAGKXZ 5f83794f f
 0001:00036961       ?QueryInterface@XPersistPropertyBag@COleControl@@UAGJABU_GUID@@PAPAX@Z 5f837961 f
 0001:0003697b       ?GetClassID@XPersistPropertyBag@COleControl@@UAGJPAU_GUID@@@Z 5f83797b f
 0001:00036998       ?InitNew@XPersistPropertyBag@COleControl@@UAGJXZ 5f837998 f
 0001:00036a06       ?Load@XPersistPropertyBag@COleControl@@UAGJPAUIPropertyBag@@PAUIErrorLog@@@Z 5f837a06 f
 0001:00036ae8       ?Save@XPersistPropertyBag@COleControl@@UAGJPAUIPropertyBag@@HH@Z 5f837ae8 f
 0001:00036b91       ??0_AFXCTL_AMBIENT_CACHE@@QAE@XZ 5f837b91 f
 0001:00036b9a       ?Cache@_AFXCTL_AMBIENT_CACHE@@QAEXPAUtagQACONTAINER@@@Z 5f837b9a f
 0001:00036bf1       ?AddRef@XQuickActivate@COleControl@@UAGKXZ 5f837bf1 f
 0001:00036c03       ?Release@XQuickActivate@COleControl@@UAGKXZ 5f837c03 f
 0001:00036c15       ?QueryInterface@XQuickActivate@COleControl@@UAGJABU_GUID@@PAPAX@Z 5f837c15 f
 0001:00036c2f       ?QuickActivate@XQuickActivate@COleControl@@UAGJPAUtagQACONTAINER@@PAUtagQACONTROL@@@Z 5f837c2f f
 0001:00036d3a       ?SetContentExtent@XQuickActivate@COleControl@@UAGJPAUtagSIZE@@@Z 5f837d3a f
 0001:00036d50       ?GetContentExtent@XQuickActivate@COleControl@@UAGJPAUtagSIZE@@@Z 5f837d50 f
 0001:00036d66       ?_GetBaseClass@CWindowlessDC@@KGPAUCRuntimeClass@@XZ 5f837d66 f
 0001:00036d6c       ?GetRuntimeClass@CWindowlessDC@@UBEPAUCRuntimeClass@@XZ 5f837d6c f
 0001:00036d72       ??0CWindowlessDC@@QAE@PAUHDC__@@AAVCPoint@@@Z 5f837d72 f
 0001:00036df2       ??_GCWindowlessDC@@UAEPAXI@Z 5f837df2 f
 0001:00036df2       ??_ECWindowlessDC@@UAEPAXI@Z 5f837df2 f
 0001:00036e0e       ??1CWindowlessDC@@UAE@XZ   5f837e0e f
 0001:00036e13       ?Detach@CWindowlessDC@@QAEPAUHDC__@@XZ 5f837e13 f
 0001:00036e3b       ?GetClientOffset@COleControl@@UBEXPAJ0@Z 5f837e3b f
 0001:00036e93       ?ParentToClient@COleControl@@UBEIPBUtagRECT@@PAUtagPOINT@@H@Z 5f837e93 f
 0001:00036f2a       ?ClientToParent@COleControl@@UBEXPBUtagRECT@@PAUtagPOINT@@@Z 5f837f2a f
 0001:00036f59       ?GetActivationPolicy@COleControl@@UAEKXZ 5f837f59 f
 0001:00036f5c       ?OnInactiveSetCursor@COleControl@@UAEHPBUtagRECT@@JJKH@Z 5f837f5c f
 0001:00036fcc       ?OnInactiveMouseMove@COleControl@@UAEXPBUtagRECT@@JJK@Z 5f837fcc f
 0001:0003701a       ?AddRef@XPointerInactive@COleControl@@UAGKXZ 5f83801a f
 0001:0003702c       ?Release@XPointerInactive@COleControl@@UAGKXZ 5f83802c f
 0001:0003703e       ?QueryInterface@XPointerInactive@COleControl@@UAGJABU_GUID@@PAPAX@Z 5f83803e f
 0001:00037058       ?GetActivationPolicy@XPointerInactive@COleControl@@UAGJPAK@Z 5f838058 f
 0001:00037079       ?OnInactiveSetCursor@XPointerInactive@COleControl@@UAGJPBUtagRECT@@JJKH@Z 5f838079 f
 0001:000370a5       ?OnInactiveMouseMove@XPointerInactive@COleControl@@UAGJPBUtagRECT@@JJK@Z 5f8380a5 f
 0001:000370cb       ?OnWindowlessMessage@COleControl@@UAEHIIJPAJ@Z 5f8380cb f
 0001:00037139       ?OnWindowMessage@XOleInPlaceObject@COleControl@@UAGJIIJPAJ@Z 5f838139 f
 0001:00037162       ?GetDropTarget@XOleInPlaceObject@COleControl@@UAGJPAPAUIDropTarget@@@Z 5f838162 f
 0001:0003718f       ?SetCapture@COleControl@@QAEPAVCWnd@@XZ 5f83818f f
 0001:000371d0       ?ReleaseCapture@COleControl@@QAEHXZ 5f8381d0 f
 0001:000371fc       ?GetCapture@COleControl@@QAEPAVCWnd@@XZ 5f8381fc f
 0001:00037235       ?SetFocus@COleControl@@QAEPAVCWnd@@XZ 5f838235 f
 0001:0003726e       ?GetFocus@COleControl@@QAEPAVCWnd@@XZ 5f83826e f
 0001:000372a7       ?GetDC@COleControl@@QAEPAVCDC@@PBUtagRECT@@K@Z 5f8382a7 f
 0001:0003739f       ?ReleaseDC@COleControl@@QAEHPAVCDC@@@Z 5f83839f f
 0001:00037403       ?InvalidateRgn@COleControl@@QAEXPAVCRgn@@H@Z 5f838403 f
 0001:000374d6       ?ScrollWindow@COleControl@@QAEXHHPBUtagRECT@@0@Z 5f8384d6 f
 0001:000375a0       ?ClipCaretRect@COleControl@@QAEHPAUtagRECT@@@Z 5f8385a0 f
 0001:00037628       ?GetClientRect@COleControl@@UBEXPAUtagRECT@@@Z 5f838628 f
 0001:000376a7       ??0CColorButton@@QAE@XZ    5f8386a7 f
 0001:000376bd       ??_GCColorButton@@UAEPAXI@Z 5f8386bd f
 0001:000376bd       ??_ECColorButton@@UAEPAXI@Z 5f8386bd f
 0001:000376d9       ??1CColorButton@@UAE@XZ    5f8386d9 f
 0001:000376de       ?SetFaceColor@CColorButton@@QAEXK@Z 5f8386de f
 0001:000376e8       ?colGetFaceColor@CColorButton@@QAEKXZ 5f8386e8 f
 0001:000376ec       ?DrawItem@CColorButton@@MAEXPAUtagDRAWITEMSTRUCT@@@Z 5f8386ec f
 0001:000378a2       ?GetMessageMap@CColorPropPage@@MBEPBUAFX_MSGMAP@@XZ 5f8388a2 f
 0001:000378a8       ??0CColorPropPage@@QAE@XZ  5f8388a8 f
 0001:00037938       ??_ECColorPropPage@@UAEPAXI@Z 5f838938 f
 0001:00037938       ??_GCColorPropPage@@UAEPAXI@Z 5f838938 f
 0001:00037954       ??1CColorPropPage@@UAE@XZ  5f838954 f
 0001:000379c9       ?OnInitDialog@CColorPropPage@@MAEHXZ 5f8389c9 f
 0001:00037a30       ?FillSysColors@CColorPropPage@@IAEXXZ 5f838a30 f
 0001:00037ac6       ?DoDataExchange@CColorPropPage@@MAEXPAVCDataExchange@@@Z 5f838ac6 f
 0001:00037c58       ?SetColorProp@CColorPropPage@@IAEHPAVCDataExchange@@KPBG@Z 5f838c58 f
 0001:00037d4a       ?GetColorProp@CColorPropPage@@IAEHPAVCDataExchange@@PAKPBG@Z 5f838d4a f
 0001:00037e3d       ?OnSelect@CColorPropPage@@AAEXXZ 5f838e3d f
 0001:00037e55       ?SetButton@CColorPropPage@@AAEXPAVCColorButton@@@Z 5f838e55 f
 0001:00037eb9       ?OnSelchangeColorprop@CColorPropPage@@AAEXXZ 5f838eb9 f
 0001:00037ec6       ?_AfxDraw3DFrame@@YAXPAVCDC@@VCRect@@KK@Z 5f838ec6 f
 0001:00037fe8       ?_AfxDraw3DButtonFrame@@YAXPAVCDC@@VCRect@@H@Z 5f838fe8 f
 0001:000381b6       ?_AfxInitPalette@@YAPAUHPALETTE__@@XZ 5f8391b6 f
 0001:000382bd       ?OnSelchangeSystemcolors@CColorPropPage@@AAEXXZ 5f8392bd f
 0001:000382ed       ?OnEditProperty@CColorPropPage@@MAEHJ@Z 5f8392ed f
 0001:00038300       ?OnObjectsChanged@CColorPropPage@@MAEXXZ 5f839300 f
 0001:0003837d       ?GetClassID@CColorPropPage@@UAEJPAU_GUID@@@Z 5f83937d f
 0001:00038393       ?UpdateRegistry@CColorPropPageFactory@CColorPropPage@@UAEHH@Z 5f839393 f
 0001:000383c5       ??_GCColorPropPageFactory@CColorPropPage@@UAEPAXI@Z 5f8393c5 f
 0001:000383c5       ??_ECColorPropPageFactory@CColorPropPage@@UAEPAXI@Z 5f8393c5 f
 0001:000383e1       ?GetMessageMap@CFontPropPage@@MBEPBUAFX_MSGMAP@@XZ 5f8393e1 f
 0001:000383e7       ??0CFontPropPage@@QAE@XZ   5f8393e7 f
 0001:000384aa       ??_ECFontPropPage@@UAEPAXI@Z 5f8394aa f
 0001:000384aa       ??_GCFontPropPage@@UAEPAXI@Z 5f8394aa f
 0001:000384c6       ??1CSizeComboBox@@UAE@XZ   5f8394c6 f
 0001:000384cb       ??1CFontPropPage@@UAE@XZ   5f8394cb f
 0001:00038586       ??_GCSizeComboBox@@UAEPAXI@Z 5f839586 f
 0001:00038586       ??_ECSizeComboBox@@UAEPAXI@Z 5f839586 f
 0001:000385a2       ?_AfxStringFromCy@@YAHAAVCString@@AATtagCY@@@Z 5f8395a2 f
 0001:0003860d       ?_AfxCyFromString@@YAHAATtagCY@@PBG@Z 5f83960d f
 0001:00038679       ?_AfxDrawMaskedBitmap@@YAXPAVCDC@@PAVCBitmap@@1HHHH@Z 5f839679 f
 0001:000387ce       ?_AfxInitMaskFromBitmap@@YAXPAVCBitmap@@0@Z 5f8397ce f
 0001:00038912       ?DoDataExchange@CFontPropPage@@MAEXPAVCDataExchange@@@Z 5f839912 f
 0001:00038b2b       ??0tagFONTOBJECT@@QAE@ABU0@@Z 5f839b2b f
 0001:00038b6c       ?SetFontProps@CFontPropPage@@IAEHPAVCDataExchange@@UtagFONTOBJECT@@PBG@Z 5f839b6c f
 0001:00038d5e       ?GetFontProps@CFontPropPage@@IAEHPAVCDataExchange@@PAUtagFONTOBJECT@@PBGPAUtagMERGEOBJECT@@@Z 5f839d5e f
 0001:00038f71       ?OnInitDialog@CFontPropPage@@MAEHXZ 5f839f71 f
 0001:00038f94       ?FillFacenameList@CFontPropPage@@IAEXXZ 5f839f94 f
 0001:00039065       ?EnumFontFamiliesCallBack@CFontPropPage@@KGHPAUtagENUMLOGFONTW@@PAUtagNEWTEXTMETRICW@@HJ@Z 5f83a065 f
 0001:0003913e       ?EnumFontFamiliesCallBack2@CFontPropPage@@KGHPAUtagENUMLOGFONTW@@PAUtagNEWTEXTMETRICW@@HJ@Z 5f83a13e f
 0001:000391ed       ??0CFontComboBox@@QAE@XZ   5f83a1ed f
 0001:0003924f       ??_ECFontComboBox@@UAEPAXI@Z 5f83a24f f
 0001:0003924f       ??_GCFontComboBox@@UAEPAXI@Z 5f83a24f f
 0001:0003926b       ?AddFont@CFontComboBox@@QAEHPAUtagLOGFONTW@@K@Z 5f83a26b f
 0001:00039314       ?GetFontItem@CFontComboBox@@QAEPAUFONTITEM_PPG@@H@Z 5f83a314 f
 0001:0003939e       ?GetLogFont@CFontComboBox@@QAEPAUtagLOGFONTW@@H@Z 5f83a39e f
 0001:000393ad       ?GetFontType@CFontComboBox@@QAEKH@Z 5f83a3ad f
 0001:000393bb       ?GetCurrentName@CFontComboBox@@QAE?AVCString@@XZ 5f83a3bb f
 0001:00039416       ?DrawItem@CFontComboBox@@UAEXPAUtagDRAWITEMSTRUCT@@@Z 5f83a416 f
 0001:00039542       ?DeleteItem@CFontComboBox@@UAEXPAUtagDELETEITEMSTRUCT@@@Z 5f83a542 f
 0001:0003955e       ?AddSize@CSizeComboBox@@QAEHHJ@Z 5f83a55e f
 0001:00039661       ?GetPointSize@CSizeComboBox@@QAEXAATtagCY@@@Z 5f83a661 f
 0001:0003968c       ?GetHeight@CSizeComboBox@@QAEJH@Z 5f83a68c f
 0001:0003972d       ?UpdateLogFont@CSizeComboBox@@QAEXPAUtagLOGFONTW@@H@Z 5f83a72d f
 0001:00039743       ?OnEditupdateFontnames@CFontPropPage@@IAEXXZ 5f83a743 f
 0001:000397cc       ?OnEditupdateFontsizes@CFontPropPage@@IAEXXZ 5f83a7cc f
 0001:00039829       ?OnSelchangeFontnames@CFontPropPage@@IAEXXZ 5f83a829 f
 0001:00039829       ?FillSizeList@CFontPropPage@@IAEXXZ 5f83a829 f
 0001:00039a81       ?UpdateSampleFont@CFontPropPage@@IAEXXZ 5f83aa81 f
 0001:00039b40       ?OnPaint@CFontPropPage@@MAEXXZ 5f83ab40 f
 0001:00039ce7       ?OnSelchangeFontsizes@CFontPropPage@@IAEXXZ 5f83ace7 f
 0001:00039d20       ?OnSelchangeFontstyles@CFontPropPage@@IAEXXZ 5f83ad20 f
 0001:00039d61       ?OnEditchangeFontstyles@CFontPropPage@@IAEXXZ 5f83ad61 f
 0001:00039e0c       ?SelectFontFromList@CFontPropPage@@IAEXVCString@@PAUtagMERGEOBJECT@@@Z 5f83ae0c f
 0001:00039f7f       ?OnStrikeout@CFontPropPage@@IAEXXZ 5f83af7f f
 0001:00039fbd       ?OnUnderline@CFontPropPage@@IAEXXZ 5f83afbd f
 0001:00039ffb       ?OnSelchangeFontprop@CFontPropPage@@IAEXXZ 5f83affb f
 0001:0003a008       ?OnObjectsChanged@CFontPropPage@@MAEXXZ 5f83b008 f
 0001:0003a0b4       ?GetClassID@CFontPropPage@@UAEJPAU_GUID@@@Z 5f83b0b4 f
 0001:0003a0ca       ?UpdateRegistry@CFontPropPageFactory@CFontPropPage@@UAEHH@Z 5f83b0ca f
 0001:0003a0fc       ??_9@$BOM@AE               5f83b0fc f
 0001:0003a104       ??1CFontPropPageFactory@CFontPropPage@@UAE@XZ 5f83b104 f
 0001:0003a109       ?GetMessageMap@CPicturePropPage@@MBEPBUAFX_MSGMAP@@XZ 5f83b109 f
 0001:0003a10f       ??0CPicturePropPage@@QAE@XZ 5f83b10f f
 0001:0003a17b       ??_GCPicturePropPage@@UAEPAXI@Z 5f83b17b f
 0001:0003a17b       ??_ECPicturePropPage@@UAEPAXI@Z 5f83b17b f
 0001:0003a197       ??1CPicturePropPage@@UAE@XZ 5f83b197 f
 0001:0003a218       ?OnInitDialog@CPicturePropPage@@MAEHXZ 5f83b218 f
 0001:0003a25e       ?DoDataExchange@CPicturePropPage@@MAEXPAVCDataExchange@@@Z 5f83b25e f
 0001:0003a2f0       ?SetPictureProp@CPicturePropPage@@IAEHPAVCDataExchange@@PAUIPictureDisp@@PBG@Z 5f83b2f0 f
 0001:0003a3f8       ?GetPictureProp@CPicturePropPage@@IAEHPAVCDataExchange@@PAPAUIPictureDisp@@PBG@Z 5f83b3f8 f
 0001:0003a524       ?OnPaint@CPicturePropPage@@IAEXXZ 5f83b524 f
 0001:0003a69c       ?_AfxCreateStreamOnFile@@YAJPBGPAPAUIStream@@PAJ@Z 5f83b69c f
 0001:0003a7ae       ?OnBrowse@CPicturePropPage@@IAEXXZ 5f83b7ae f
 0001:0003a9ea       ?OnClear@CPicturePropPage@@IAEXXZ 5f83b9ea f
 0001:0003aa18       ?ChangePicture@CPicturePropPage@@IAEXPAUIPicture@@@Z 5f83ba18 f
 0001:0003aa8b       ?OnSelchangePictProp@CPicturePropPage@@IAEXXZ 5f83ba8b f
 0001:0003ab2f       ?OnEditProperty@CPicturePropPage@@MAEHJ@Z 5f83bb2f f
 0001:0003ab42       ?OnObjectsChanged@CPicturePropPage@@MAEXXZ 5f83bb42 f
 0001:0003ab80       ?GetClassID@CPicturePropPage@@UAEJPAU_GUID@@@Z 5f83bb80 f
 0001:0003ab96       ?UpdateRegistry@CPicturePropPageFactory@CPicturePropPage@@UAEHH@Z 5f83bb96 f
 0001:0003abc8       ?_GetBaseMessageMap@CStockPropPage@@KGPBUAFX_MSGMAP@@XZ 5f83bbc8 f
 0001:0003abce       ?GetMessageMap@CStockPropPage@@MBEPBUAFX_MSGMAP@@XZ 5f83bbce f
 0001:0003abd4       ?_AfxSizeComboToContent@@YAXPAVCComboBox@@@Z 5f83bbd4 f
 0001:0003ac54       ??0CStockPropPage@@QAE@II@Z 5f83bc54 f
 0001:0003ac9d       ??_ECStockPropPage@@UAEPAXI@Z 5f83bc9d f
 0001:0003ac9d       ??_GCStockPropPage@@UAEPAXI@Z 5f83bc9d f
 0001:0003acb9       ?FillPropnameList@CStockPropPage@@IAEXABU_GUID@@HAAVCComboBox@@@Z 5f83bcb9 f
 0001:0003aec5       ?OnSelchangePropname@CStockPropPage@@IAEXAAVCComboBox@@@Z 5f83bec5 f
 0001:0003af37       ?OnEditProperty@CStockPropPage@@IAEHJAAVCComboBox@@@Z 5f83bf37 f
 0001:0003af9b       ?AfxOleTypeMatchGuid@@YGHPAUITypeInfo@@PAUtagTYPEDESC@@ABU_GUID@@K@Z 5f83bf9b f
 0001:0003b050       ?AfxThrowDBException@@YGXFPAVCDatabase@@PAX@Z 5f83c050 f
 0001:0003b0b3       ??0CDBException@@QAE@F@Z   5f83c0b3 f
 0001:0003b12b       ??_ECDBException@@UAEPAXI@Z 5f83c12b f
 0001:0003b12b       ??_GCDBException@@UAEPAXI@Z 5f83c12b f
 0001:0003b147       ?BuildErrorString@CDBException@@UAEXPAVCDatabase@@PAXH@Z 5f83c147 f
 0001:0003b36e       ?GetErrorMessage@CDBException@@UAEHPAGIPAI@Z 5f83c36e f
 0001:0003b39f       ?Empty@CDBException@@QAEXXZ 5f83c39f f
 0001:0003b3b4       ?AfxGetHENV@@YGPAXXZ       5f83c3b4 f
 0001:0003b3c7       ??0CDatabase@@QAE@XZ       5f83c3c7 f
 0001:0003b42e       ??1CDatabase@@UAE@XZ       5f83c42e f
 0001:0003b47c       ?Open@CDatabase@@UAEHPBGHH0H@Z 5f83c47c f
 0001:0003b571       ?OpenEx@CDatabase@@UAEHPBGK@Z 5f83c571 f
 0001:0003b5f2       ?ExecuteSQL@CDatabase@@QAEXPBG@Z 5f83c5f2 f
 0001:0003b751       ?Cancel@CDatabase@@QAEXXZ  5f83c751 f
 0001:0003b75a       ?Close@CDatabase@@UAEXXZ   5f83c75a f
 0001:0003b7f5       ?Free@CDatabase@@IAEXXZ    5f83c7f5 f
 0001:0003b867       ?OnSetOptions@CDatabase@@UAEXPAX@Z 5f83c867 f
 0001:0003b892       ?GetDatabaseName@CDatabase@@QBE?AVCString@@XZ 5f83c892 f
 0001:0003b8d6       ?BeginTrans@CDatabase@@QAEHXZ 5f83c8d6 f
 0001:0003b8f9       ?CommitTrans@CDatabase@@QAEHXZ 5f83c8f9 f
 0001:0003b93e       ?Rollback@CDatabase@@QAEHXZ 5f83c93e f
 0001:0003b983       ?Check@CDatabase@@UBEHF@Z  5f83c983 f
 0001:0003b992       ?CheckHstmt@CDatabase@@QBGHFPAX@Z 5f83c992 f
 0001:0003b9af       ?ReplaceBrackets@CDatabase@@QAEXPAG@Z 5f83c9af f
 0001:0003ba3b       ?AllocConnect@CDatabase@@IAEXK@Z 5f83ca3b f
 0001:0003baf7       ?Connect@CDatabase@@IAEHK@Z 5f83caf7 f
 0001:0003bc3c       ?VerifyConnect@CDatabase@@IAEXXZ 5f83cc3c f
 0001:0003bcc3       ?GetConnectInfo@CDatabase@@IAEXXZ 5f83ccc3 f
 0001:0003be85       ??0CRecordset@@QAE@PAVCDatabase@@@Z 5f83ce85 f
 0001:0003c09a       ??_ECRecordset@@UAEPAXI@Z  5f83d09a f
 0001:0003c09a       ??_GCRecordset@@UAEPAXI@Z  5f83d09a f
 0001:0003c0b6       ??1CRecordset@@UAE@XZ      5f83d0b6 f
 0001:0003c1c8       ?Open@CRecordset@@UAEHIPBGK@Z 5f83d1c8 f
 0001:0003c29c       ?Close@CRecordset@@UAEXXZ  5f83d29c f
 0001:0003c466       ??_ECODBCFieldInfo@@QAEPAXI@Z 5f83d466 f
 0001:0003c4b1       ??1CODBCFieldInfo@@QAE@XZ  5f83d4b1 f
 0001:0003c4b6       ?IsOpen@CRecordset@@QBEHXZ 5f83d4b6 f
 0001:0003c571       ?IsFieldDirty@CRecordset@@QAEHPAX@Z 5f83d571 f
 0001:0003c5de       ?IsFieldNull@CRecordset@@QAEHPAX@Z 5f83d5de f
 0001:0003c62f       ?IsFieldNullable@CRecordset@@QAEHPAX@Z 5f83d62f f
 0001:0003c669       ?CanBookmark@CRecordset@@QBEHXZ 5f83d669 f
 0001:0003c68c       ?Move@CRecordset@@UAEXJG@Z 5f83d68c f
 0001:0003c767       ?CheckRowsetError@CRecordset@@UAEXF@Z 5f83d767 f
 0001:0003c820       ?GetBookmark@CRecordset@@QAEXAAVCDBVariant@@@Z 5f83d820 f
 0001:0003c8ac       ?SetBookmark@CRecordset@@QAEXABVCDBVariant@@@Z 5f83d8ac f
 0001:0003c8ed       ?SetRowsetSize@CRecordset@@UAEXK@Z 5f83d8ed f
 0001:0003c99f       ?AddNew@CRecordset@@UAEXXZ 5f83d99f f
 0001:0003c9fe       ?Edit@CRecordset@@UAEXXZ   5f83d9fe f
 0001:0003cab7       ?Update@CRecordset@@UAEHXZ 5f83dab7 f
 0001:0003caeb       ?Delete@CRecordset@@UAEXXZ 5f83daeb f
 0001:0003cb12       ?CancelUpdate@CRecordset@@QAEXXZ 5f83db12 f
 0001:0003cb2a       ?LoadFields@CRecordset@@QAEXXZ 5f83db2a f
 0001:0003cb54       ?FlushResultSet@CRecordset@@QBEHXZ 5f83db54 f
 0001:0003cb93       ?GetODBCFieldInfo@CRecordset@@QAEXPBGAAUCODBCFieldInfo@@@Z 5f83db93 f
 0001:0003cbb6       ?GetODBCFieldInfo@CRecordset@@QAEXFAAUCODBCFieldInfo@@@Z 5f83dbb6 f
 0001:0003cbf9       ?GetFieldValue@CRecordset@@QAEXPBGAAVCDBVariant@@F@Z 5f83dbf9 f
 0001:0003cc2d       ?GetFieldValue@CRecordset@@QAEXFAAVCDBVariant@@F@Z 5f83dc2d f
 0001:0003cd99       ?GetFieldValue@CRecordset@@QAEXPBGAAVCString@@@Z 5f83dd99 f
 0001:0003cdbc       ?GetFieldValue@CRecordset@@QAEXFAAVCString@@@Z 5f83ddbc f
 0001:0003cea6       ?SetFieldDirty@CRecordset@@QAEXPAXH@Z 5f83dea6 f
 0001:0003ceec       ?SetFieldNull@CRecordset@@QAEXPAXH@Z 5f83deec f
 0001:0003cf4b       ?SetParamNull@CRecordset@@QAEXHH@Z 5f83df4b f
 0001:0003cf7b       ?SetLockingMode@CRecordset@@QAEXI@Z 5f83df7b f
 0001:0003cfce       ?Requery@CRecordset@@UAEHXZ 5f83dfce f
 0001:0003d107       ?Cancel@CRecordset@@QAEXXZ 5f83e107 f
 0001:0003d124       ?GetDefaultConnect@CRecordset@@UAE?AVCString@@XZ 5f83e124 f
 0001:0003d140       ?GetDefaultSQL@CRecordset@@UAE?AVCString@@XZ 5f83e140 f
 0001:0003d15c       ?OnSetOptions@CRecordset@@UAEXPAX@Z 5f83e15c f
 0001:0003d1b5       ?Check@CRecordset@@UBEHF@Z 5f83e1b5 f
 0001:0003d1d7       ?SetState@CRecordset@@IAEXHPBGK@Z 5f83e1d7 f
 0001:0003d287       ?AllocHstmt@CRecordset@@IAEHXZ 5f83e287 f
 0001:0003d463       ?BuildSQL@CRecordset@@IAEXPBG@Z 5f83e463 f
 0001:0003d54a       ?PrepareAndExecute@CRecordset@@IAEXXZ 5f83e54a f
 0001:0003d777       ?VerifyDriverBehavior@CRecordset@@IAEXXZ 5f83e777 f
 0001:0003d80d       ?VerifyCursorSupport@CRecordset@@IAEKXZ 5f83e80d f
 0001:0003d89f       ?AllocAndCacheFieldInfo@CRecordset@@IAEXXZ 5f83e89f f
 0001:0003d9cd       ??0CODBCFieldInfo@@QAE@XZ  5f83e9cd f
 0001:0003d9d9       ?AllocRowset@CRecordset@@IAEXXZ 5f83e9d9 f
 0001:0003da09       ?FreeRowset@CRecordset@@IAEXXZ 5f83ea09 f
 0001:0003da61       ?EnableBookmarks@CRecordset@@IAEXXZ 5f83ea61 f
 0001:0003da9b       ?SetUpdateMethod@CRecordset@@IAEXXZ 5f83ea9b f
 0001:0003dabd       ?SetConcurrencyAndCursorType@CRecordset@@IAEXPAXK@Z 5f83eabd f
 0001:0003dbb1       ?IsSQLUpdatable@CRecordset@@QAEHPBG@Z 5f83ebb1 f
 0001:0003dc0a       ?IsSelectQueryUpdatable@CRecordset@@QAEHPBG@Z 5f83ec0a f
 0001:0003dd3a       ?IsJoin@CRecordset@@SGHPBG@Z 5f83ed3a f
 0001:0003dd68       ?FindSQLToken@CRecordset@@SGPBGPBG0@Z 5f83ed68 f
 0001:0003de8e       ?InitRecord@CRecordset@@QAEXXZ 5f83ee8e f
 0001:0003dec0       ?ResetCursor@CRecordset@@QAEXXZ 5f83eec0 f
 0001:0003dee8       ?CheckRowsetCurrencyStatus@CRecordset@@QAEXGJ@Z 5f83eee8 f
 0001:0003df79       ?FetchData@CRecordset@@QAEFGJPAK@Z 5f83ef79 f
 0001:0003dff6       ?SkipDeletedRecords@CRecordset@@QAEXGJPAKPAF@Z 5f83eff6 f
 0001:0003e0d3       ?SetRowsetCurrencyStatus@CRecordset@@UAEXFGJK@Z 5f83f0d3 f
 0001:0003e2e6       ?RefreshRowset@CRecordset@@QAEXGG@Z 5f83f2e6 f
 0001:0003e329       ?SetRowsetCursorPosition@CRecordset@@QAEXGG@Z 5f83f329 f
 0001:0003e348       ?BuildSelectSQL@CRecordset@@IAEXXZ 5f83f348 f
 0001:0003e469       ?AppendFilterAndSortSQL@CRecordset@@IAEXXZ 5f83f469 f
 0001:0003e4be       ?IsRecordsetUpdatable@CRecordset@@IAEHXZ 5f83f4be f
 0001:0003e4f8       ?ExecuteSetPosUpdate@CRecordset@@IAEXXZ 5f83f4f8 f
 0001:0003e58d       ?PrepareUpdateHstmt@CRecordset@@IAEXXZ 5f83f58d f
 0001:0003e606       ?BuildUpdateSQL@CRecordset@@IAEXXZ 5f83f606 f
 0001:0003e82a       ?ExecuteUpdateSQL@CRecordset@@IAEXXZ 5f83f82a f
 0001:0003e942       ?SendLongBinaryData@CRecordset@@IAEXPAX@Z 5f83f942 f
 0001:0003ea9f       ?AllocStatusArrays@CRecordset@@QAEXXZ 5f83fa9f f
 0001:0003eb85       ?GetBoundFieldIndex@CRecordset@@QAEHPAX@Z 5f83fb85 f
 0001:0003eba7       ?GetBoundParamIndex@CRecordset@@QAEHPAX@Z 5f83fba7 f
 0001:0003ebc9       ?GetFieldIndexByName@CRecordset@@QAEFPBG@Z 5f83fbc9 f
 0001:0003ec13       ?GetFieldLengthBuffer@CRecordset@@QAEPAJKH@Z 5f83fc13 f
 0001:0003ec3a       ?GetFieldStatus@CRecordset@@QAEEK@Z 5f83fc3a f
 0001:0003ec4a       ?SetFieldStatus@CRecordset@@QAEXKE@Z 5f83fc4a f
 0001:0003ec5f       ?ClearFieldStatus@CRecordset@@QAEXXZ 5f83fc5f f
 0001:0003ec73       ?IsFieldStatusDirty@CRecordset@@QBEHK@Z 5f83fc73 f
 0001:0003ec86       ?SetDirtyFieldStatus@CRecordset@@QAEXK@Z 5f83fc86 f
 0001:0003ec98       ?ClearDirtyFieldStatus@CRecordset@@QAEXK@Z 5f83fc98 f
 0001:0003ecaa       ?IsFieldStatusNull@CRecordset@@QBEHK@Z 5f83fcaa f
 0001:0003ecbd       ?SetNullFieldStatus@CRecordset@@QAEXK@Z 5f83fcbd f
 0001:0003eccf       ?ClearNullFieldStatus@CRecordset@@QAEXK@Z 5f83fccf f
 0001:0003ece1       ?IsParamStatusNull@CRecordset@@QBEHK@Z 5f83fce1 f
 0001:0003ecf4       ?SetNullParamStatus@CRecordset@@QAEXK@Z 5f83fcf4 f
 0001:0003ed06       ?ClearNullParamStatus@CRecordset@@QAEXK@Z 5f83fd06 f
 0001:0003ed18       ?IsFieldNullable@CRecordset@@QBEHK@Z 5f83fd18 f
 0001:0003ed31       ?BindParams@CRecordset@@QAEIPAX@Z 5f83fd31 f
 0001:0003ed60       ?RebindParams@CRecordset@@QAEXPAX@Z 5f83fd60 f
 0001:0003ed92       ?BindFieldsToColumns@CRecordset@@QAEIXZ 5f83fd92 f
 0001:0003edca       ?BindFieldsForUpdate@CRecordset@@QAEXXZ 5f83fdca f
 0001:0003ee04       ?UnbindFieldsForUpdate@CRecordset@@QAEXXZ 5f83fe04 f
 0001:0003ee3e       ?Fixups@CRecordset@@QAEXXZ 5f83fe3e f
 0001:0003ee68       ?AppendNames@CRecordset@@QAEIPAVCString@@PBG@Z 5f83fe68 f
 0001:0003eea8       ?AppendNamesValues@CRecordset@@QAEIPAXPAVCString@@PBG@Z 5f83fea8 f
 0001:0003eee3       ?AppendValues@CRecordset@@QAEIPAXPAVCString@@PBG@Z 5f83fee3 f
 0001:0003ef1e       ?StoreFields@CRecordset@@QAEXXZ 5f83ff1e f
 0001:0003ef42       ?MarkForUpdate@CRecordset@@QAEXXZ 5f83ff42 f
 0001:0003ef66       ?MarkForAddNew@CRecordset@@QAEXXZ 5f83ff66 f
 0001:0003ef8a       ?AllocDataCache@CRecordset@@QAEXXZ 5f83ff8a f
 0001:0003efae       ?FreeDataCache@CRecordset@@QAEXXZ 5f83ffae f
 0001:0003f040       ?UpdateInsertDelete@CRecordset@@IAEHXZ 5f840040 f
 0001:0003f235       ?GetLBReallocSize@CRecordset@@MAEJJ@Z 5f840235 f
 0001:0003f23e       ?GetDefaultFieldType@CRecordset@@SGFF@Z 5f84023e f
 0001:0003f2ca       ?GetDataBuffer@CRecordset@@SGPAXAAVCDBVariant@@FPAHFK@Z 5f8402ca f
 0001:0003f47c       ?GetTextLen@CRecordset@@SGHFK@Z 5f84047c f
 0001:0003f4a8       ?GetData@CRecordset@@SGJPAVCDatabase@@PAXFF1HF@Z 5f8404a8 f
 0001:0003f4f8       ?GetLongCharDataAndCleanup@CRecordset@@SGXPAVCDatabase@@PAXFJPAPAXHAAVCString@@F@Z 5f8404f8 f
 0001:0003f586       ?GetLongBinaryDataAndCleanup@CRecordset@@SGXPAVCDatabase@@PAXFJPAPAXHAAVCDBVariant@@F@Z 5f840586 f
 0001:0003f640       ?AfxSetCurrentRecord@@YGXPAJJF@Z 5f840640 f
 0001:0003f65e       ?AfxSetRecordCount@@YGXPAJJJHF@Z 5f84065e f
 0001:0003f676       ?AfxSetRecordCount@@YGXPAJJHF@Z 5f840676 f
 0001:0003f6a0       ?ThrowDBException@CDatabase@@MAEXF@Z 5f8406a0 f
 0001:0003f6b0       ?ThrowDBException@CRecordset@@UAEXFPAX@Z 5f8406b0 f
 0001:0003f6cb       ??0CFieldExchange@@QAE@IPAVCRecordset@@PAX@Z 5f8406cb f
 0001:0003f707       ?IsFieldType@CFieldExchange@@QAEHPAI@Z 5f840707 f
 0001:0003f744       ?Default@CFieldExchange@@QAEXPBGPAXPAJHII@Z 5f840744 f
 0001:0003fa32       ?RFX_Text@@YGXPAVCFieldExchange@@PBGPAGHHF@Z 5f840a32 f
 0001:0004012a       ?RFX_Text@@YGXPAVCFieldExchange@@PBGAAVCString@@HHF@Z 5f84112a f
 0001:000408e6       ?RFX_Int@@YGXPAVCFieldExchange@@PBGAAH@Z 5f8418e6 f
 0001:00040a0d       ?RFX_Long@@YGXPAVCFieldExchange@@PBGAAJ@Z 5f841a0d f
 0001:00040b35       ?RFX_Byte@@YGXPAVCFieldExchange@@PBGAAE@Z 5f841b35 f
 0001:00040c52       ?RFX_Bool@@YGXPAVCFieldExchange@@PBGAAH@Z 5f841c52 f
 0001:00040d7a       ?RFX_Binary@@YGXPAVCFieldExchange@@PBGAAVCByteArray@@H@Z 5f841d7a f
 0001:00040fc7       ?RFX_Date@@YGXPAVCFieldExchange@@PBGAAVCTime@@@Z 5f841fc7 f
 0001:00041685       ?RFX_Date@@YGXPAVCFieldExchange@@PBGAAUtagTIMESTAMP_STRUCT@@@Z 5f842685 f
 0001:0004183f       ?RFX_Date@@YGXPAVCFieldExchange@@PBGAAVCOleDateTime@@@Z 5f84283f f
 0001:00041e68       ??9CTime@@QBEHV0@@Z        5f842e68 f
 0001:00041e76       ?RFX_LongBinary@@YGXPAVCFieldExchange@@PBGAAVCLongBinary@@@Z 5f842e76 f
 0001:0004214b       ?GetLongBinarySize@CFieldExchange@@QAEJH@Z 5f84314b f
 0001:00042191       ?GetLongBinaryData@CFieldExchange@@QAEXHAAVCLongBinary@@PAJ@Z 5f843191 f
 0001:000422ff       ?ReallocLongBinary@CFieldExchange@@QAEPAEAAVCLongBinary@@JJ@Z 5f8432ff f
 0001:00042381       ?AfxStoreField@@YGXAAVCRecordset@@IPAX@Z 5f843381 f
 0001:000423ed       ?AfxLoadField@@YGXAAVCRecordset@@IPAXPAJ@Z 5f8433ed f
 0001:00042464       ?AfxCompareValueByRef@@YGHPAX0H@Z 5f843464 f
 0001:000425b7       ??8CTime@@QBEHV0@@Z        5f8435b7 f
 0001:000425c5       ?AfxCopyValueByRef@@YGXPAX0PAJH@Z 5f8435c5 f
 0001:000426f2       ?RFX_Text_Bulk@@YGXPAVCFieldExchange@@PBGPAPADPAPAJH@Z 5f8436f2 f
 0001:0004277b       ?RFX_Bool_Bulk@@YGXPAVCFieldExchange@@PBGPAPAHPAPAJ@Z 5f84377b f
 0001:000427fd       ?RFX_Date_Bulk@@YGXPAVCFieldExchange@@PBGPAPAUtagTIMESTAMP_STRUCT@@PAPAJ@Z 5f8437fd f
 0001:00042884       ?RFX_Byte_Bulk@@YGXPAVCFieldExchange@@PBGPAPAEPAPAJ@Z 5f843884 f
 0001:00042906       ?RFX_Binary_Bulk@@YGXPAVCFieldExchange@@PBGPAPAEPAPAJH@Z 5f843906 f
 0001:0004298f       ?AfxRFXBulkDefault@@YGXPAVCFieldExchange@@PBGPAXPAJHI@Z 5f84398f f
 0001:000429f6       ?GetMessageMap@CRecordView@@MBEPBUAFX_MSGMAP@@XZ 5f8439f6 f
 0001:000429fc       ??0CRecordView@@IAE@PBG@Z  5f8439fc f
 0001:00042a14       ??_ECRecordView@@UAEPAXI@Z 5f843a14 f
 0001:00042a14       ??_GCRecordView@@UAEPAXI@Z 5f843a14 f
 0001:00042a30       ??0CRecordView@@IAE@I@Z    5f843a30 f
 0001:00042a48       ??1CRecordView@@UAE@XZ     5f843a48 f
 0001:00042a53       ?OnInitialUpdate@CRecordView@@UAEXXZ 5f843a53 f
 0001:00042ab9       ?IsOnFirstRecord@CRecordView@@QAEHXZ 5f843ab9 f
 0001:00042ad1       ?IsOnLastRecord@CRecordView@@QAEHXZ 5f843ad1 f
 0001:00042afa       ?OnMove@CRecordView@@UAEHI@Z 5f843afa f
 0001:00042ba9       ?OnUpdateRecordFirst@CRecordView@@IAEXPAVCCmdUI@@@Z 5f843ba9 f
 0001:00042bfd       ?OnUpdateRecordPrev@CRecordView@@IAEXPAVCCmdUI@@@Z 5f843bfd f
 0001:00042c09       ?OnUpdateRecordNext@CRecordView@@IAEXPAVCCmdUI@@@Z 5f843c09 f
 0001:00042c54       ?OnUpdateRecordLast@CRecordView@@IAEXPAVCCmdUI@@@Z 5f843c54 f
 0001:00042ca8       ?AfxFieldText@@YGHPAVCDataExchange@@HPAXPAVCRecordset@@@Z 5f843ca8 f
 0001:00042d78       ?DDX_FieldText@@YGXPAVCDataExchange@@HAAHPAVCRecordset@@@Z 5f843d78 f
 0001:00042da2       ?DDX_FieldText@@YGXPAVCDataExchange@@HAAEPAVCRecordset@@@Z 5f843da2 f
 0001:00042dcc       ?DDX_FieldText@@YGXPAVCDataExchange@@HAAIPAVCRecordset@@@Z 5f843dcc f
 0001:00042df6       ?DDX_FieldText@@YGXPAVCDataExchange@@HAAJPAVCRecordset@@@Z 5f843df6 f
 0001:00042e20       ?DDX_FieldText@@YGXPAVCDataExchange@@HAAKPAVCRecordset@@@Z 5f843e20 f
 0001:00042e4a       ?DDX_FieldText@@YGXPAVCDataExchange@@HAAVCString@@PAVCRecordset@@@Z 5f843e4a f
 0001:00042f74       ?DDX_FieldText@@YGXPAVCDataExchange@@HPAGHPAVCRecordset@@@Z 5f843f74 f
 0001:00043011       ?DDX_FieldLBString@@YGXPAVCDataExchange@@HAAVCString@@PAVCRecordset@@@Z 5f844011 f
 0001:0004311b       ?DDX_FieldLBStringExact@@YGXPAVCDataExchange@@HAAVCString@@PAVCRecordset@@@Z 5f84411b f
 0001:0004319a       ?DDX_FieldLBIndex@@YGXPAVCDataExchange@@HAAHPAVCRecordset@@@Z 5f84419a f
 0001:000431dc       ?DDX_FieldCBString@@YGXPAVCDataExchange@@HAAVCString@@PAVCRecordset@@@Z 5f8441dc f
 0001:00043322       ?DDX_FieldCBStringExact@@YGXPAVCDataExchange@@HAAVCString@@PAVCRecordset@@@Z 5f844322 f
 0001:000433a1       ?DDX_FieldCBIndex@@YGXPAVCDataExchange@@HAAHPAVCRecordset@@@Z 5f8443a1 f
 0001:000433e3       ?DDX_FieldScroll@@YGXPAVCDataExchange@@HAAHPAVCRecordset@@@Z 5f8443e3 f
 0001:00043425       ?DDX_FieldCheck@@YGXPAVCDataExchange@@HAAHPAVCRecordset@@@Z 5f844425 f
 0001:000434d8       ?DDX_FieldRadio@@YGXPAVCDataExchange@@HAAHPAVCRecordset@@@Z 5f8444d8 f
 0001:00043546       ??_9@$BBBE@AE              5f844546 f
 0001:0004354e       ?RFX_Single@@YGXPAVCFieldExchange@@PBGAAM@Z 5f84454e f
 0001:00043689       ?RFX_Double@@YGXPAVCFieldExchange@@PBGAAN@Z 5f844689 f
 0001:000437d6       ?RFX_Single_Bulk@@YGXPAVCFieldExchange@@PBGPAPAMPAPAJ@Z 5f8447d6 f
 0001:00043858       ?RFX_Double_Bulk@@YGXPAVCFieldExchange@@PBGPAPANPAPAJ@Z 5f844858 f
 0001:000438df       ?DDX_FieldText@@YGXPAVCDataExchange@@HAAMPAVCRecordset@@@Z 5f8448df f
 0001:00043913       ?DDX_FieldText@@YGXPAVCDataExchange@@HAANPAVCRecordset@@@Z 5f844913 f
 0001:00043947       ??0CLongBinary@@QAE@XZ     5f844947 f
 0001:00043954       ??1CLongBinary@@UAE@XZ     5f844954 f
 0001:00043977       ??0CDBVariant@@QAE@XZ      5f844977 f
 0001:00043984       ??_GCDBVariant@@UAEPAXI@Z  5f844984 f
 0001:00043984       ??_ECDBVariant@@UAEPAXI@Z  5f844984 f
 0001:000439c4       ??1CDBVariant@@UAE@XZ      5f8449c4 f
 0001:000439ca       ?Clear@CDBVariant@@QAEXXZ  5f8449ca f
 0001:000439ed       ??0_AFX_DAO_STATE@@QAE@XZ  5f8449ed f
 0001:00043a29       ??_G_AFX_DAO_STATE@@UAEPAXI@Z 5f844a29 f
 0001:00043a29       ??_E_AFX_DAO_STATE@@UAEPAXI@Z 5f844a29 f
 0001:00043a44       ??1_AFX_DAO_STATE@@UAE@XZ  5f844a44 f
 0001:00043a70       ?AfxDaoCheck@@YGXJPBD0HHH@Z 5f844a70 f
 0001:00043a9e       ??0CDaoIndexInfo@@QAE@XZ   5f844a9e f
 0001:00043abf       ??_ECDaoIndexInfo@@UAEPAXI@Z 5f844abf f
 0001:00043abf       ??_GCDaoIndexInfo@@UAEPAXI@Z 5f844abf f
 0001:00043adb       ??_ECDaoIndexFieldInfo@@QAEPAXI@Z 5f844adb f
 0001:00043b26       ??0CDaoRelationInfo@@QAE@XZ 5f844b26 f
 0001:00043b79       ??_GCDaoRelationInfo@@UAEPAXI@Z 5f844b79 f
 0001:00043b79       ??_ECDaoRelationInfo@@UAEPAXI@Z 5f844b79 f
 0001:00043b95       ??_ECDaoRelationFieldInfo@@QAEPAXI@Z 5f844b95 f
 0001:00043be0       ?_GetBaseClass@CDaoException@@KGPAUCRuntimeClass@@XZ 5f844be0 f
 0001:00043be6       ?GetRuntimeClass@CDaoException@@UBEPAUCRuntimeClass@@XZ 5f844be6 f
 0001:00043bec       ??0CDaoException@@QAE@XZ   5f844bec f
 0001:00043c09       ??1CDaoException@@UAE@XZ   5f844c09 f
 0001:00043c74       ??1CDaoErrorInfo@@QAE@XZ   5f844c74 f
 0001:00043cb9       ?GetErrorCount@CDaoException@@QAEFXZ 5f844cb9 f
 0001:00043cfe       ?GetErrorInfo@CDaoException@@QAEXH@Z 5f844cfe f
 0001:00043d8e       ?GetErrorMessage@CDaoException@@UAEHPAGIPAI@Z 5f844d8e f
 0001:00043e26       ?InitErrorsCollection@CDaoException@@IAEXXZ 5f844e26 f
 0001:00043e58       ?FillErrorInfo@CDaoException@@IAEXXZ 5f844e58 f
 0001:00043f91       ??0CDaoErrorInfo@@QAE@XZ   5f844f91 f
 0001:00043fd1       ?AfxThrowDaoException@@YGXHJ@Z 5f844fd1 f
 0001:0004405e       ?_GetBaseClass@CDaoWorkspace@@KGPAUCRuntimeClass@@XZ 5f84505e f
 0001:00044069       ?GetRuntimeClass@CDaoWorkspace@@UBEPAUCRuntimeClass@@XZ 5f845069 f
 0001:0004406f       ??0CDaoWorkspace@@QAE@XZ   5f84506f f
 0001:000440be       ??1CDaoWorkspace@@UAE@XZ   5f8450be f
 0001:00044121       ?Create@CDaoWorkspace@@UAEXPBG00@Z 5f845121 f
 0001:000441d4       ?Append@CDaoWorkspace@@UAEXXZ 5f8451d4 f
 0001:00044266       ?Open@CDaoWorkspace@@UAEXPBG@Z 5f845266 f
 0001:00044333       ?Close@CDaoWorkspace@@UAEXXZ 5f845333 f
 0001:000443d5       ?GetVersion@CDaoWorkspace@@SG?AVCString@@XZ 5f8453d5 f
 0001:0004444c       ?GetIniPath@CDaoWorkspace@@SG?AVCString@@XZ 5f84544c f
 0001:000444c3       ?SetIniPath@CDaoWorkspace@@SGXPBG@Z 5f8454c3 f
 0001:00044526       ?SetDefaultUser@CDaoWorkspace@@SGXPBG@Z 5f845526 f
 0001:00044589       ?SetDefaultPassword@CDaoWorkspace@@SGXPBG@Z 5f845589 f
 0001:000445ec       ?GetLoginTimeout@CDaoWorkspace@@SGFXZ 5f8455ec f
 0001:00044625       ?SetLoginTimeout@CDaoWorkspace@@SGXF@Z 5f845625 f
 0001:00044657       ?GetName@CDaoWorkspace@@QAE?AVCString@@XZ 5f845657 f
 0001:000446bf       ?GetUserNameW@CDaoWorkspace@@QAE?AVCString@@XZ 5f8456bf f
 0001:00044727       ?SetIsolateODBCTrans@CDaoWorkspace@@QAEXH@Z 5f845727 f
 0001:00044749       ?GetIsolateODBCTrans@CDaoWorkspace@@QAEHXZ 5f845749 f
 0001:00044773       ?CompactDatabase@CDaoWorkspace@@SGXPBG00H0@Z 5f845773 f
 0001:0004489e       ?CompactDatabase@CDaoWorkspace@@SGXPBG00H@Z 5f84589e f
 0001:000448b8       ?RepairDatabase@CDaoWorkspace@@SGXPBG@Z 5f8458b8 f
 0001:0004491b       ?Idle@CDaoWorkspace@@SGXH@Z 5f84591b f
 0001:00044988       ?GetWorkspaceCount@CDaoWorkspace@@QAEFXZ 5f845988 f
 0001:000449bc       ?GetWorkspaceInfo@CDaoWorkspace@@QAEXHAAUCDaoWorkspaceInfo@@K@Z 5f8459bc f
 0001:00044a45       ?GetWorkspaceInfo@CDaoWorkspace@@QAEXPBGAAUCDaoWorkspaceInfo@@K@Z 5f845a45 f
 0001:00044ace       ?GetDatabaseCount@CDaoWorkspace@@QAEFXZ 5f845ace f
 0001:00044b02       ?GetDatabaseInfo@CDaoWorkspace@@QAEXHAAUCDaoDatabaseInfo@@K@Z 5f845b02 f
 0001:00044b8b       ?GetDatabaseInfo@CDaoWorkspace@@QAEXPBGAAUCDaoDatabaseInfo@@K@Z 5f845b8b f
 0001:00044c14       ?BeginTrans@CDaoWorkspace@@QAEXXZ 5f845c14 f
 0001:00044c2b       ?CommitTrans@CDaoWorkspace@@QAEXXZ 5f845c2b f
 0001:00044c8c       ?Rollback@CDaoWorkspace@@QAEXXZ 5f845c8c f
 0001:00044ca3       ?InitializeEngine@CDaoWorkspace@@KAXXZ 5f845ca3 f
 0001:00044ca3       ?AfxDaoInit@@YGXXZ         5f845ca3 f
 0001:00044dba       ?InitWorkspacesCollection@CDaoWorkspace@@IAEXXZ 5f845dba f
 0001:00044dee       ?FillWorkspaceInfo@CDaoWorkspace@@IAEXPAUDAOWorkspace@@AAUCDaoWorkspaceInfo@@K@Z 5f845dee f
 0001:00044ebe       ?InitDatabasesCollection@CDaoWorkspace@@IAEXXZ 5f845ebe f
 0001:00044ed9       ?FillDatabaseInfo@CDaoWorkspace@@IAEXPAUDAODatabase@@AAUCDaoDatabaseInfo@@K@Z 5f845ed9 f
 0001:00045027       ?GetRuntimeClass@CDaoDatabase@@UBEPAUCRuntimeClass@@XZ 5f846027 f
 0001:0004502d       ??0CDaoDatabase@@QAE@PAVCDaoWorkspace@@@Z 5f84602d f
 0001:000450a3       ??1CDaoDatabase@@UAE@XZ    5f8460a3 f
 0001:00045128       ?Create@CDaoDatabase@@UAEXPBG0H@Z 5f846128 f
 0001:000451e1       ?Open@CDaoDatabase@@UAEXPBGHH0@Z 5f8461e1 f
 0001:000452e4       ?Close@CDaoDatabase@@UAEXXZ 5f8462e4 f
 0001:0004540f       ?CanUpdate@CDaoDatabase@@QAEHXZ 5f84640f f
 0001:00045439       ?GetName@CDaoDatabase@@QAE?AVCString@@XZ 5f846439 f
 0001:000454a1       ?GetConnect@CDaoDatabase@@QAE?AVCString@@XZ 5f8464a1 f
 0001:00045509       ?GetVersion@CDaoDatabase@@QAE?AVCString@@XZ 5f846509 f
 0001:00045571       ?GetQueryTimeout@CDaoDatabase@@QAEFXZ 5f846571 f
 0001:00045595       ?SetQueryTimeout@CDaoDatabase@@QAEXF@Z 5f846595 f
 0001:000455b2       ?GetRecordsAffected@CDaoDatabase@@QAEJXZ 5f8465b2 f
 0001:000455d5       ?DeleteTableDef@CDaoDatabase@@QAEXPBG@Z 5f8465d5 f
 0001:00045633       ?DeleteQueryDef@CDaoDatabase@@QAEXPBG@Z 5f846633 f
 0001:00045691       ?CreateRelation@CDaoDatabase@@QAEXPBG00J00@Z 5f846691 f
 0001:0004574f       ?CreateRelation@CDaoDatabase@@QAEXAAUCDaoRelationInfo@@@Z 5f84674f f
 0001:000459ce       ?DeleteRelation@CDaoDatabase@@QAEXPBG@Z 5f8469ce f
 0001:00045a2c       ?Execute@CDaoDatabase@@QAEXPBGH@Z 5f846a2c f
 0001:00045aa6       ?GetTableDefCount@CDaoDatabase@@QAEFXZ 5f846aa6 f
 0001:00045ada       ?GetTableDefInfo@CDaoDatabase@@QAEXHAAUCDaoTableDefInfo@@K@Z 5f846ada f
 0001:00045b63       ?GetTableDefInfo@CDaoDatabase@@QAEXPBGAAUCDaoTableDefInfo@@K@Z 5f846b63 f
 0001:00045bec       ?GetRelationCount@CDaoDatabase@@QAEFXZ 5f846bec f
 0001:00045c20       ?GetRelationInfo@CDaoDatabase@@QAEXHAAUCDaoRelationInfo@@K@Z 5f846c20 f
 0001:00045ca9       ?GetRelationInfo@CDaoDatabase@@QAEXPBGAAUCDaoRelationInfo@@K@Z 5f846ca9 f
 0001:00045d32       ?GetQueryDefCount@CDaoDatabase@@QAEFXZ 5f846d32 f
 0001:00045d66       ?GetQueryDefInfo@CDaoDatabase@@QAEXHAAUCDaoQueryDefInfo@@K@Z 5f846d66 f
 0001:00045def       ?GetQueryDefInfo@CDaoDatabase@@QAEXPBGAAUCDaoQueryDefInfo@@K@Z 5f846def f
 0001:00045e78       ?InitWorkspace@CDaoDatabase@@IAEXXZ 5f846e78 f
 0001:00045edb       ?InitTableDefsCollection@CDaoDatabase@@IAEXXZ 5f846edb f
 0001:00045ef6       ?FillTableDefInfo@CDaoDatabase@@IAEXPAU_DAOTableDef@@AAUCDaoTableDefInfo@@K@Z 5f846ef6 f
 0001:000460c8       ?InitRelationsCollection@CDaoDatabase@@IAEXXZ 5f8470c8 f
 0001:000460e3       ?FillRelationInfo@CDaoDatabase@@IAEXPAU_DAORelation@@AAUCDaoRelationInfo@@K@Z 5f8470e3 f
 0001:000463a7       ??0CDaoRelationFieldInfo@@QAE@XZ 5f8473a7 f
 0001:000463d8       ?InitQueryDefsCollection@CDaoDatabase@@IAEXXZ 5f8473d8 f
 0001:000463f3       ?FillQueryDefInfo@CDaoDatabase@@IAEXPAU_DAOQueryDef@@AAUCDaoQueryDefInfo@@K@Z 5f8473f3 f
 0001:00046577       ?GetRuntimeClass@CDaoTableDef@@UBEPAUCRuntimeClass@@XZ 5f847577 f
 0001:0004657d       ??0CDaoTableDef@@QAE@PAVCDaoDatabase@@@Z 5f84757d f
 0001:000465a0       ??_ECDaoTableDef@@UAEPAXI@Z 5f8475a0 f
 0001:000465a0       ??_GCDaoTableDef@@UAEPAXI@Z 5f8475a0 f
 0001:000465bc       ??1CDaoTableDef@@UAE@XZ    5f8475bc f
 0001:00046608       ?Create@CDaoTableDef@@UAEXPBGJ00@Z 5f847608 f
 0001:0004670d       ?Append@CDaoTableDef@@UAEXXZ 5f84770d f
 0001:00046791       ?Open@CDaoTableDef@@UAEXPBG@Z 5f847791 f
 0001:0004685d       ?Close@CDaoTableDef@@UAEXXZ 5f84785d f
 0001:000468a8       ?CanUpdate@CDaoTableDef@@QAEHXZ 5f8478a8 f
 0001:000468d2       ?SetName@CDaoTableDef@@QAEXPBG@Z 5f8478d2 f
 0001:00046924       ?GetName@CDaoTableDef@@QAE?AVCString@@XZ 5f847924 f
 0001:0004698c       ?SetSourceTableName@CDaoTableDef@@QAEXPBG@Z 5f84798c f
 0001:000469de       ?GetSourceTableName@CDaoTableDef@@QAE?AVCString@@XZ 5f8479de f
 0001:00046a46       ?SetConnect@CDaoTableDef@@QAEXPBG@Z 5f847a46 f
 0001:00046a98       ?GetConnect@CDaoTableDef@@QAE?AVCString@@XZ 5f847a98 f
 0001:00046b00       ?SetAttributes@CDaoTableDef@@QAEXJ@Z 5f847b00 f
 0001:00046b1d       ?GetAttributes@CDaoTableDef@@QAEJXZ 5f847b1d f
 0001:00046b40       ?GetDateCreated@CDaoTableDef@@QAE?AVCOleDateTime@@XZ 5f847b40 f
 0001:00046b9e       ?GetDateLastUpdated@CDaoTableDef@@QAE?AVCOleDateTime@@XZ 5f847b9e f
 0001:00046bfc       ?SetValidationRule@CDaoTableDef@@QAEXPBG@Z 5f847bfc f
 0001:00046c4e       ?GetValidationRule@CDaoTableDef@@QAE?AVCString@@XZ 5f847c4e f
 0001:00046cb6       ?SetValidationText@CDaoTableDef@@QAEXPBG@Z 5f847cb6 f
 0001:00046d08       ?GetValidationText@CDaoTableDef@@QAE?AVCString@@XZ 5f847d08 f
 0001:00046d70       ?GetRecordCount@CDaoTableDef@@QAEJXZ 5f847d70 f
 0001:00046d93       ?CreateField@CDaoTableDef@@QAEXPBGFJJ@Z 5f847d93 f
 0001:00046e04       ??0CDaoFieldInfo@@QAE@XZ   5f847e04 f
 0001:00046e71       ?CreateField@CDaoTableDef@@QAEXAAUCDaoFieldInfo@@@Z 5f847e71 f
 0001:00046f93       ?DeleteField@CDaoTableDef@@QAEXPBG@Z 5f847f93 f
 0001:00046ff1       ?DeleteField@CDaoTableDef@@QAEXH@Z 5f847ff1 f
 0001:00047042       ?CreateIndex@CDaoTableDef@@QAEXAAUCDaoIndexInfo@@@Z 5f848042 f
 0001:00047107       ?DeleteIndex@CDaoTableDef@@QAEXPBG@Z 5f848107 f
 0001:00047165       ?DeleteIndex@CDaoTableDef@@QAEXH@Z 5f848165 f
 0001:000471b6       ?GetFieldCount@CDaoTableDef@@QAEFXZ 5f8481b6 f
 0001:000471ea       ?GetFieldInfo@CDaoTableDef@@QAEXHAAUCDaoFieldInfo@@K@Z 5f8481ea f
 0001:00047274       ?GetFieldInfo@CDaoTableDef@@QAEXPBGAAUCDaoFieldInfo@@K@Z 5f848274 f
 0001:000472fe       ?GetIndexCount@CDaoTableDef@@QAEFXZ 5f8482fe f
 0001:00047332       ?GetIndexInfo@CDaoTableDef@@QAEXHAAUCDaoIndexInfo@@K@Z 5f848332 f
 0001:000473bc       ?GetIndexInfo@CDaoTableDef@@QAEXPBGAAUCDaoIndexInfo@@K@Z 5f8483bc f
 0001:00047446       ?RefreshLink@CDaoTableDef@@QAEXXZ 5f848446 f
 0001:0004745d       ?InitFieldsCollection@CDaoTableDef@@IAEXXZ 5f84845d f
 0001:00047478       ?InitIndexesCollection@CDaoTableDef@@IAEXXZ 5f848478 f
 0001:00047493       ?GetRuntimeClass@CDaoQueryDef@@UBEPAUCRuntimeClass@@XZ 5f848493 f
 0001:00047499       ??0CDaoQueryDef@@QAE@PAVCDaoDatabase@@@Z 5f848499 f
 0001:000474bc       ??_ECDaoQueryDef@@UAEPAXI@Z 5f8484bc f
 0001:000474bc       ??_GCDaoQueryDef@@UAEPAXI@Z 5f8484bc f
 0001:000474d8       ??1CDaoQueryDef@@UAE@XZ    5f8484d8 f
 0001:00047524       ?Create@CDaoQueryDef@@UAEXPBG0@Z 5f848524 f
 0001:00047642       ?Append@CDaoQueryDef@@UAEXXZ 5f848642 f
 0001:000476c6       ?Open@CDaoQueryDef@@UAEXPBG@Z 5f8486c6 f
 0001:0004779f       ?Close@CDaoQueryDef@@UAEXXZ 5f84879f f
 0001:000477f3       ?CanUpdate@CDaoQueryDef@@QAEHXZ 5f8487f3 f
 0001:0004781d       ?GetName@CDaoQueryDef@@QAE?AVCString@@XZ 5f84881d f
 0001:00047885       ?SetName@CDaoQueryDef@@QAEXPBG@Z 5f848885 f
 0001:000478d7       ?GetSQL@CDaoQueryDef@@QAE?AVCString@@XZ 5f8488d7 f
 0001:0004793f       ?SetSQL@CDaoQueryDef@@QAEXPBG@Z 5f84893f f
 0001:00047991       ?GetType@CDaoQueryDef@@QAEFXZ 5f848991 f
 0001:000479b5       ?GetDateCreated@CDaoQueryDef@@QAE?AVCOleDateTime@@XZ 5f8489b5 f
 0001:00047a13       ?GetDateLastUpdated@CDaoQueryDef@@QAE?AVCOleDateTime@@XZ 5f848a13 f
 0001:00047a71       ?GetConnect@CDaoQueryDef@@QAE?AVCString@@XZ 5f848a71 f
 0001:00047ad9       ?SetConnect@CDaoQueryDef@@QAEXPBG@Z 5f848ad9 f
 0001:00047b2b       ?GetODBCTimeout@CDaoQueryDef@@QAEFXZ 5f848b2b f
 0001:00047b4f       ?SetODBCTimeout@CDaoQueryDef@@QAEXF@Z 5f848b4f f
 0001:00047b6c       ?GetRecordsAffected@CDaoQueryDef@@QAEJXZ 5f848b6c f
 0001:00047b8f       ?Execute@CDaoQueryDef@@UAEXH@Z 5f848b8f f
 0001:00047beb       ?GetParamValue@CDaoQueryDef@@UAE?AVCOleVariant@@PBG@Z 5f848beb f
 0001:00047cc6       ?GetParamValue@CDaoQueryDef@@UAE?AVCOleVariant@@H@Z 5f848cc6 f
 0001:00047da1       ?SetParamValue@CDaoQueryDef@@UAEXPBGABVCOleVariant@@@Z 5f848da1 f
 0001:00047e5d       ?SetParamValue@CDaoQueryDef@@UAEXHABVCOleVariant@@@Z 5f848e5d f
 0001:00047f19       ?SetParamValueNull@CDaoQueryDef@@QAEXPBG@Z 5f848f19 f
 0001:00047f61       ?SetParamValueNull@CDaoQueryDef@@QAEXH@Z 5f848f61 f
 0001:00047fa9       ?GetFieldCount@CDaoQueryDef@@QAEFXZ 5f848fa9 f
 0001:00047fdd       ?GetFieldInfo@CDaoQueryDef@@QAEXHAAUCDaoFieldInfo@@K@Z 5f848fdd f
 0001:00048067       ?GetFieldInfo@CDaoQueryDef@@QAEXPBGAAUCDaoFieldInfo@@K@Z 5f849067 f
 0001:000480f1       ?GetParameterCount@CDaoQueryDef@@QAEFXZ 5f8490f1 f
 0001:00048125       ?GetParameterInfo@CDaoQueryDef@@QAEXHAAUCDaoParameterInfo@@K@Z 5f849125 f
 0001:000481ae       ?GetParameterInfo@CDaoQueryDef@@QAEXPBGAAUCDaoParameterInfo@@K@Z 5f8491ae f
 0001:00048237       ?InitFieldsCollection@CDaoQueryDef@@IAEXXZ 5f849237 f
 0001:00048252       ?InitParametersCollection@CDaoQueryDef@@IAEXXZ 5f849252 f
 0001:0004826d       ?FillParameterInfo@CDaoQueryDef@@IAEXPAUDAOParameter@@AAUCDaoParameterInfo@@K@Z 5f84926d f
 0001:0004834f       ?GetRuntimeClass@CDaoRecordset@@UBEPAUCRuntimeClass@@XZ 5f84934f f
 0001:00048355       ??0CDaoRecordset@@QAE@PAVCDaoDatabase@@@Z 5f849355 f
 0001:0004841e       ??1CDaoRecordset@@UAE@XZ   5f84941e f
 0001:000484d0       ?Open@CDaoRecordset@@UAEXHPBGH@Z 5f8494d0 f
 0001:0004889d       ?Open@CDaoRecordset@@UAEXPAVCDaoQueryDef@@HH@Z 5f84989d f
 0001:000489d9       ?Open@CDaoRecordset@@UAEXPAVCDaoTableDef@@HH@Z 5f8499d9 f
 0001:00048b01       ?Close@CDaoRecordset@@UAEXXZ 5f849b01 f
 0001:00048c23       ?Requery@CDaoRecordset@@UAEXXZ 5f849c23 f
 0001:00048d3b       ?IsBOF@CDaoRecordset@@QBEHXZ 5f849d3b f
 0001:00048d65       ?IsEOF@CDaoRecordset@@QBEHXZ 5f849d65 f
 0001:00048d8f       ?IsDeleted@CDaoRecordset@@QBEHXZ 5f849d8f f
 0001:00048d93       ?CanScroll@CDaoRecordset@@QBEHXZ 5f849d93 f
 0001:00048d97       ?CanUpdate@CDaoRecordset@@QBEHXZ 5f849d97 f
 0001:00048dc1       ?CanAppend@CDaoRecordset@@QBEHXZ 5f849dc1 f
 0001:00048dc5       ?CanRestart@CDaoRecordset@@QAEHXZ 5f849dc5 f
 0001:00048def       ?CanTransact@CDaoRecordset@@QAEHXZ 5f849def f
 0001:00048e19       ?CanBookmark@CDaoRecordset@@QAEHXZ 5f849e19 f
 0001:00048e43       ?GetName@CDaoRecordset@@QAE?AVCString@@XZ 5f849e43 f
 0001:00048eab       ?GetType@CDaoRecordset@@QAEFXZ 5f849eab f
 0001:00048ecf       ?GetEditMode@CDaoRecordset@@QAEFXZ 5f849ecf f
 0001:00048ef6       ?GetSQL@CDaoRecordset@@QBE?AVCString@@XZ 5f849ef6 f
 0001:00048f11       ?GetDateCreated@CDaoRecordset@@QAE?AVCOleDateTime@@XZ 5f849f11 f
 0001:00048f6f       ?GetDateLastUpdated@CDaoRecordset@@QAE?AVCOleDateTime@@XZ 5f849f6f f
 0001:00048fcd       ?GetLastModifiedBookmark@CDaoRecordset@@QAE?AVCOleVariant@@XZ 5f849fcd f
 0001:00049036       ?GetValidationRule@CDaoRecordset@@QAE?AVCString@@XZ 5f84a036 f
 0001:000490a1       ?GetValidationText@CDaoRecordset@@QAE?AVCString@@XZ 5f84a0a1 f
 0001:00049109       ?GetCurrentIndex@CDaoRecordset@@QAE?AVCString@@XZ 5f84a109 f
 0001:00049171       ?SetCurrentIndex@CDaoRecordset@@QAEXPBG@Z 5f84a171 f
 0001:000491ca       ?GetRecordCount@CDaoRecordset@@QAEJXZ 5f84a1ca f
 0001:000491ed       ?SetFieldDirty@CDaoRecordset@@QAEXPAXH@Z 5f84a1ed f
 0001:00049238       ?IsFieldDirty@CDaoRecordset@@QAEHPAX@Z 5f84a238 f
 0001:000492a5       ?SetFieldNull@CDaoRecordset@@QAEXPAXH@Z 5f84a2a5 f
 0001:00049308       ?IsFieldNull@CDaoRecordset@@QAEHPAX@Z 5f84a308 f
 0001:00049351       ?IsFieldNullable@CDaoRecordset@@QAEHPAX@Z 5f84a351 f
 0001:00049405       ?GetFieldCount@CDaoRecordset@@QAEFXZ 5f84a405 f
 0001:00049439       ?GetFieldInfo@CDaoRecordset@@QAEXHAAUCDaoFieldInfo@@K@Z 5f84a439 f
 0001:000494c3       ?GetFieldInfo@CDaoRecordset@@QAEXPBGAAUCDaoFieldInfo@@K@Z 5f84a4c3 f
 0001:0004954d       ?GetIndexCount@CDaoRecordset@@QAEFXZ 5f84a54d f
 0001:00049581       ?GetIndexInfo@CDaoRecordset@@QAEXHAAUCDaoIndexInfo@@K@Z 5f84a581 f
 0001:0004960b       ?GetIndexInfo@CDaoRecordset@@QAEXPBGAAUCDaoIndexInfo@@K@Z 5f84a60b f
 0001:00049695       ?GetBookmark@CDaoRecordset@@QAE?AVCOleVariant@@XZ 5f84a695 f
 0001:000496fe       ?SetBookmark@CDaoRecordset@@QAEXVCOleVariant@@@Z 5f84a6fe f
 0001:00049748       ?GetAbsolutePosition@CDaoRecordset@@QAEJXZ 5f84a748 f
 0001:0004976e       ?SetAbsolutePosition@CDaoRecordset@@QAEXJ@Z 5f84a76e f
 0001:00049799       ?GetPercentPosition@CDaoRecordset@@QAEMXZ 5f84a799 f
 0001:000497bf       ?SetPercentPosition@CDaoRecordset@@QAEXM@Z 5f84a7bf f
 0001:000497ee       ?MoveNext@CDaoRecordset@@QAEXXZ 5f84a7ee f
 0001:000497f6       ?MovePrev@CDaoRecordset@@QAEXXZ 5f84a7f6 f
 0001:000497fe       ?MoveFirst@CDaoRecordset@@QAEXXZ 5f84a7fe f
 0001:00049809       ?MoveLast@CDaoRecordset@@QAEXXZ 5f84a809 f
 0001:00049814       ?Move@CDaoRecordset@@UAEXJ@Z 5f84a814 f
 0001:000498fd       ?FindNext@CDaoRecordset@@QAEHPBG@Z 5f84a8fd f
 0001:0004990b       ?FindPrev@CDaoRecordset@@QAEHPBG@Z 5f84a90b f
 0001:00049919       ?FindFirst@CDaoRecordset@@QAEHPBG@Z 5f84a919 f
 0001:0004992a       ?FindLast@CDaoRecordset@@QAEHPBG@Z 5f84a92a f
 0001:0004993b       ?Find@CDaoRecordset@@UAEHJPBG@Z 5f84a93b f
 0001:00049a0b       ?Seek@CDaoRecordset@@QAEHPBGPAVCOleVariant@@11@Z 5f84aa0b f
 0001:00049b77       ?Seek@CDaoRecordset@@QAEHPBGPAVCOleVariant@@G@Z 5f84ab77 f
 0001:00049cc0       ?CancelUpdate@CDaoRecordset@@UAEXXZ 5f84acc0 f
 0001:00049cf1       ?SetLockingMode@CDaoRecordset@@QAEXH@Z 5f84acf1 f
 0001:00049d13       ?GetLockingMode@CDaoRecordset@@QAEHXZ 5f84ad13 f
 0001:00049d3d       ?SetCacheStart@CDaoRecordset@@QAEXVCOleVariant@@@Z 5f84ad3d f
 0001:00049d7f       ?GetCacheStart@CDaoRecordset@@QAE?AVCOleVariant@@XZ 5f84ad7f f
 0001:00049deb       ?SetCacheSize@CDaoRecordset@@QAEXJ@Z 5f84adeb f
 0001:00049e0b       ?GetCacheSize@CDaoRecordset@@QAEJXZ 5f84ae0b f
 0001:00049e31       ?FillCache@CDaoRecordset@@QAEXPAJPAVCOleVariant@@@Z 5f84ae31 f
 0001:00049ee6       ?AddNew@CDaoRecordset@@UAEXXZ 5f84aee6 f
 0001:00049f42       ?Edit@CDaoRecordset@@UAEXXZ 5f84af42 f
 0001:00049f9a       ?Update@CDaoRecordset@@UAEXXZ 5f84af9a f
 0001:00049ff5       ?Delete@CDaoRecordset@@UAEXXZ 5f84aff5 f
 0001:0004a039       ?GetFieldValue@CDaoRecordset@@UAE?AVCOleVariant@@PBG@Z 5f84b039 f
 0001:0004a090       ?GetFieldValue@CDaoRecordset@@UAE?AVCOleVariant@@H@Z 5f84b090 f
 0001:0004a0e7       ?GetFieldValue@CDaoRecordset@@UAEXPBGAAVCOleVariant@@@Z 5f84b0e7 f
 0001:0004a152       ?GetFieldValue@CDaoRecordset@@UAEXHAAVCOleVariant@@@Z 5f84b152 f
 0001:0004a1bd       ?SetFieldValue@CDaoRecordset@@UAEXPBGABVCOleVariant@@@Z 5f84b1bd f
 0001:0004a234       ?SetFieldValue@CDaoRecordset@@UAEXHABVCOleVariant@@@Z 5f84b234 f
 0001:0004a2ab       ?SetFieldValue@CDaoRecordset@@QAEXHPBG@Z 5f84b2ab f
 0001:0004a2f3       ?SetFieldValue@CDaoRecordset@@QAEXPBG0@Z 5f84b2f3 f
 0001:0004a33b       ?SetFieldValueNull@CDaoRecordset@@QAEXPBG@Z 5f84b33b f
 0001:0004a383       ?SetFieldValueNull@CDaoRecordset@@QAEXH@Z 5f84b383 f
 0001:0004a3cb       ?GetParamValue@CDaoRecordset@@UAE?AVCOleVariant@@PBG@Z 5f84b3cb f
 0001:0004a3e8       ?GetParamValue@CDaoRecordset@@UAE?AVCOleVariant@@H@Z 5f84b3e8 f
 0001:0004a405       ?SetParamValue@CDaoRecordset@@UAEXPBGABVCOleVariant@@@Z 5f84b405 f
 0001:0004a418       ?SetParamValue@CDaoRecordset@@UAEXHABVCOleVariant@@@Z 5f84b418 f
 0001:0004a42b       ?SetParamValueNull@CDaoRecordset@@QAEXPBG@Z 5f84b42b f
 0001:0004a473       ?SetParamValueNull@CDaoRecordset@@QAEXH@Z 5f84b473 f
 0001:0004a4bb       ?GetFieldLength@CDaoRecordset@@QAEKH@Z 5f84b4bb f
 0001:0004a4c8       ?InitFieldsCollection@CDaoRecordset@@IAEXXZ 5f84b4c8 f
 0001:0004a4e6       ?InitIndexesCollection@CDaoRecordset@@IAEXXZ 5f84b4e6 f
 0001:0004a504       ?BuildSQL@CDaoRecordset@@IAEXXZ 5f84b504 f
 0001:0004a5c5       ?AllocDatabase@CDaoRecordset@@IAEXXZ 5f84b5c5 f
 0001:0004a64a       ?BuildSelectList@CDaoRecordset@@IAEXXZ 5f84b64a f
 0001:0004a67b       ?BuildParameterList@CDaoRecordset@@IAEXXZ 5f84b67b f
 0001:0004a6cb       ?BindFields@CDaoRecordset@@IAEXXZ 5f84b6cb f
 0001:0004a793       ?BindParameters@CDaoRecordset@@IAEXXZ 5f84b793 f
 0001:0004a7bd       ?Fixup@CDaoRecordset@@IAEXXZ 5f84b7bd f
 0001:0004a7e1       ?AllocCache@CDaoRecordset@@IAEXXZ 5f84b7e1 f
 0001:0004a84e       ?StoreFields@CDaoRecordset@@IAEXXZ 5f84b84e f
 0001:0004a87d       ?LoadFields@CDaoRecordset@@IAEXXZ 5f84b87d f
 0001:0004a8b7       ?FreeCache@CDaoRecordset@@IAEXXZ 5f84b8b7 f
 0001:0004a933       ?MarkForAddNew@CDaoRecordset@@IAEXXZ 5f84b933 f
 0001:0004a957       ?MarkForEdit@CDaoRecordset@@IAEXXZ 5f84b957 f
 0001:0004a97b       ?GetFieldIndex@CDaoRecordset@@IAEHPAX@Z 5f84b97b f
 0001:0004a99e       ?SetDirtyFields@CDaoRecordset@@MAEXXZ 5f84b99e f
 0001:0004a9cd       ?SetCursorAttributes@CDaoRecordset@@QAEXXZ 5f84b9cd f
 0001:0004aa04       ?GetDataAndFixupNulls@CDaoRecordset@@QAEXXZ 5f84ba04 f
 0001:0004aa99       ?IsFieldStatusDirty@CDaoRecordset@@QAEHI@Z 5f84ba99 f
 0001:0004aaaf       ?SetDirtyFieldStatus@CDaoRecordset@@QAEXI@Z 5f84baaf f
 0001:0004aabe       ?ClearDirtyFieldStatus@CDaoRecordset@@QAEXI@Z 5f84babe f
 0001:0004aacd       ?IsFieldStatusNull@CDaoRecordset@@QAEHI@Z 5f84bacd f
 0001:0004aae3       ?SetNullFieldStatus@CDaoRecordset@@QAEXI@Z 5f84bae3 f
 0001:0004aaf2       ?ClearNullFieldStatus@CDaoRecordset@@QAEXI@Z 5f84baf2 f
 0001:0004ab01       ?IsFieldStatusNullable@CDaoRecordset@@QAEHI@Z 5f84bb01 f
 0001:0004ab17       ?SetNullableFieldStatus@CDaoRecordset@@QAEXI@Z 5f84bb17 f
 0001:0004ab26       ?IsFieldStatusNullableKnown@CDaoRecordset@@QAEHI@Z 5f84bb26 f
 0001:0004ab3c       ?SetNullableKnownFieldStatus@CDaoRecordset@@QAEXI@Z 5f84bb3c f
 0001:0004ab4b       ?ClearFieldStatusFlags@CDaoRecordset@@QAEXXZ 5f84bb4b f
 0001:0004ab5c       ?IsMatch@CDaoRecordset@@QAEHXZ 5f84bb5c f
 0001:0004ab87       ?StripBrackets@CDaoRecordset@@SAXPBGPAG@Z 5f84bb87 f
 0001:0004abc2       ?ThrowDaoException@CDaoRecordset@@MAEXH@Z 5f84bbc2 f
 0001:0004abd0       ?AfxGetFieldInfo@@YAXPAU_DAOField@@AAUCDaoFieldInfo@@K@Z 5f84bbd0 f
 0001:0004ae54       ?AfxSetFieldInfo@@YAXPAU_DAOField@@AAUCDaoFieldInfo@@@Z 5f84be54 f
 0001:0004afae       ?AfxGetDefaultValue@@YAXPAU_DAOField@@AAVCString@@@Z 5f84bfae f
 0001:0004b038       ?AfxSetDefaultValue@@YAXPAU_DAOField@@AAVCString@@@Z 5f84c038 f
 0001:0004b0b3       ?AfxGetIndexInfo@@YAXPAU_DAOIndex@@AAUCDaoIndexInfo@@K@Z 5f84c0b3 f
 0001:0004b220       ?AfxSetIndexInfo@@YAXPAU_DAOIndex@@AAUCDaoIndexInfo@@@Z 5f84c220 f
 0001:0004b2b2       ?AfxGetIndexFields@@YAXPAU_DAOIndex@@PAPAUDAOIndexFields@@@Z 5f84c2b2 f
 0001:0004b339       ?AfxGetIndexFieldInfo@@YAXPAU_DAOIndex@@AAUCDaoIndexInfo@@@Z 5f84c339 f
 0001:0004b555       ?AfxSetIndexFieldInfo@@YAXPAU_DAOIndex@@AAUCDaoIndexInfo@@@Z 5f84c555 f
 0001:0004b68e       ?ThrowGetRowsDaoException@@YAXJ@Z 5f84c68e f
 0001:0004b755       ?AfxGetDaoState@@YAPAV_AFX_DAO_STATE@@XZ 5f84c755 f
 0001:0004b800       ?AfxDaoGetEngine@@YGPAU_DAODBEngine@@XZ 5f84c800 f
 0001:0004b809       ?AfxDaoTerm@@YGXXZ         5f84c809 f
 0001:0004b889       ??_9@$BEM@AG               5f84c889 f
 0001:0004b892       ??_9@$BHE@AG               5f84c892 f
 0001:0004b89b       ??_9@$BHI@AG               5f84c89b f
 0001:0004b8a4       ??0CDaoFieldExchange@@QAE@IPAVCDaoRecordset@@PAX@Z 5f84c8a4 f
 0001:0004b8c8       ?IsValidOperation@CDaoFieldExchange@@QAEHXZ 5f84c8c8 f
 0001:0004b8ed       ?AppendParamType@CDaoFieldExchange@@SGXAAVCString@@K@Z 5f84c8ed f
 0001:0004bb27       ?GetCacheValue@CDaoFieldExchange@@SGPAUCDaoFieldCache@@PAVCDaoRecordset@@PAX@Z 5f84cb27 f
 0001:0004bb52       ?SetNullValue@CDaoFieldExchange@@SGXPAXK@Z 5f84cb52 f
 0001:0004bc0a       ?IsNullValue@CDaoFieldExchange@@SGHPAXK@Z 5f84cc0a f
 0001:0004bcb9       ?AllocCacheValue@CDaoFieldExchange@@SGXAAPAUCDaoFieldCache@@K@Z 5f84ccb9 f
 0001:0004be3f       ?DeleteCacheValue@CDaoFieldExchange@@SGXPAUCDaoFieldCache@@K@Z 5f84ce3f f
 0001:0004be91       ?CopyValue@CDaoFieldExchange@@SGXPAX0K@Z 5f84ce91 f
 0001:0004bfb1       ?CompareValue@CDaoFieldExchange@@SGHPAX0K@Z 5f84cfb1 f
 0001:0004c118       ?FillVariant@CDaoFieldExchange@@SGXPAXKPAPAVCOleVariant@@@Z 5f84d118 f
 0001:0004c273       ?Default@CDaoFieldExchange@@QAEXPBGPAXKK@Z 5f84d273 f
 0001:0004c73c       ?DFX_Text@@YGXPAVCDaoFieldExchange@@PBGAAVCString@@HK@Z 5f84d73c f
 0001:0004c7f8       ?DFX_Binary@@YGXPAVCDaoFieldExchange@@PBGAAVCByteArray@@HK@Z 5f84d7f8 f
 0001:0004c875       ?DFX_LongBinary@@YGXPAVCDaoFieldExchange@@PBGAAVCLongBinary@@KK@Z 5f84d875 f
 0001:0004c902       ?DFX_Bool@@YGXPAVCDaoFieldExchange@@PBGAAHK@Z 5f84d902 f
 0001:0004c98c       ?DFX_Byte@@YGXPAVCDaoFieldExchange@@PBGAAEK@Z 5f84d98c f
 0001:0004c9fe       ?DFX_Short@@YGXPAVCDaoFieldExchange@@PBGAAFK@Z 5f84d9fe f
 0001:0004ca72       ?DFX_Long@@YGXPAVCDaoFieldExchange@@PBGAAJK@Z 5f84da72 f
 0001:0004cae4       ?DFX_Currency@@YGXPAVCDaoFieldExchange@@PBGAAVCOleCurrency@@K@Z 5f84dae4 f
 0001:0004cb82       ?DFX_Single@@YGXPAVCDaoFieldExchange@@PBGAAMK@Z 5f84db82 f
 0001:0004cbf8       ?DFX_Double@@YGXPAVCDaoFieldExchange@@PBGAANK@Z 5f84dbf8 f
 0001:0004cc69       ?DFX_DateTime@@YGXPAVCDaoFieldExchange@@PBGAAVCOleDateTime@@K@Z 5f84dc69 f
 0001:0004cd06       _DaoStringAllocCallback@12 5f84dd06 f
 0001:0004cd60       _DaoBinaryAllocCallback@12 5f84dd60 f
 0001:0004cdbf       _DaoLongBinaryAllocCallback@12 5f84ddbf f
 0001:0004ce36       ?AllocLongBinary@@YAXAAVCLongBinary@@K@Z 5f84de36 f
 0001:0004ce90       ?_GetBaseClass@CDaoRecordView@@KGPAUCRuntimeClass@@XZ 5f84de90 f
 0001:0004ce96       ?GetRuntimeClass@CDaoRecordView@@UBEPAUCRuntimeClass@@XZ 5f84de96 f
 0001:0004ce9c       ?_GetBaseMessageMap@CDaoRecordView@@KGPBUAFX_MSGMAP@@XZ 5f84de9c f
 0001:0004cea2       ?GetMessageMap@CDaoRecordView@@MBEPBUAFX_MSGMAP@@XZ 5f84dea2 f
 0001:0004cea8       ??0CDaoRecordView@@IAE@PBG@Z 5f84dea8 f
 0001:0004cf35       ??_GCDaoRecordView@@UAEPAXI@Z 5f84df35 f
 0001:0004cf35       ??_ECDaoRecordView@@UAEPAXI@Z 5f84df35 f
 0001:0004cf51       ??0CDaoRecordView@@IAE@I@Z 5f84df51 f
 0001:0004cfde       ??1CDaoRecordView@@UAE@XZ  5f84dfde f
 0001:0004d013       ?OnInitialUpdate@CDaoRecordView@@UAEXXZ 5f84e013 f
 0001:0004d0f3       ?OnMove@CDaoRecordView@@UAEHI@Z 5f84e0f3 f
 0001:0004d390       ?IsOnFirstRecord@CDaoRecordView@@QAEHXZ 5f84e390 f
 0001:0004d3a3       ?IsOnLastRecord@CDaoRecordView@@QAEHXZ 5f84e3a3 f
 0001:0004d3b6       ?AfxFieldText@@YGHPAVCDataExchange@@HPAXPAVCDaoRecordset@@@Z 5f84e3b6 f
 0001:0004d461       ?DDX_FieldText@@YGXPAVCDataExchange@@HAAHPAVCDaoRecordset@@@Z 5f84e461 f
 0001:0004d48b       ?DDX_FieldText@@YGXPAVCDataExchange@@HAAEPAVCDaoRecordset@@@Z 5f84e48b f
 0001:0004d4b5       ?DDX_FieldText@@YGXPAVCDataExchange@@HAAFPAVCDaoRecordset@@@Z 5f84e4b5 f
 0001:0004d4df       ?DDX_FieldText@@YGXPAVCDataExchange@@HAAJPAVCDaoRecordset@@@Z 5f84e4df f
 0001:0004d509       ?DDX_FieldText@@YGXPAVCDataExchange@@HAAKPAVCDaoRecordset@@@Z 5f84e509 f
 0001:0004d533       ?DDX_FieldText@@YGXPAVCDataExchange@@HAAVCOleCurrency@@PAVCDaoRecordset@@@Z 5f84e533 f
 0001:0004d55d       ?DDX_FieldText@@YGXPAVCDataExchange@@HAAMPAVCDaoRecordset@@@Z 5f84e55d f
 0001:0004d587       ?DDX_FieldText@@YGXPAVCDataExchange@@HAANPAVCDaoRecordset@@@Z 5f84e587 f
 0001:0004d5b1       ?DDX_FieldText@@YGXPAVCDataExchange@@HAAVCOleDateTime@@PAVCDaoRecordset@@@Z 5f84e5b1 f
 0001:0004d5db       ?DDX_FieldText@@YGXPAVCDataExchange@@HAAVCString@@PAVCDaoRecordset@@@Z 5f84e5db f
 0001:0004d605       ?DDX_FieldText@@YGXPAVCDataExchange@@HPAGHPAVCDaoRecordset@@@Z 5f84e605 f
 0001:0004d633       ?DDX_FieldLBString@@YGXPAVCDataExchange@@HAAVCString@@PAVCDaoRecordset@@@Z 5f84e633 f
 0001:0004d723       ?DDX_FieldLBStringExact@@YGXPAVCDataExchange@@HAAVCString@@PAVCDaoRecordset@@@Z 5f84e723 f
 0001:0004d79c       ?DDX_FieldCBString@@YGXPAVCDataExchange@@HAAVCString@@PAVCDaoRecordset@@@Z 5f84e79c f
 0001:0004d869       ?DDX_FieldCBStringExact@@YGXPAVCDataExchange@@HAAVCString@@PAVCDaoRecordset@@@Z 5f84e869 f
 0001:0004d8e2       ?DDX_FieldLBIndex@@YGXPAVCDataExchange@@HAAHPAVCDaoRecordset@@@Z 5f84e8e2 f
 0001:0004d91e       ?DDX_FieldCBIndex@@YGXPAVCDataExchange@@HAAHPAVCDaoRecordset@@@Z 5f84e91e f
 0001:0004d95a       ?DDX_FieldScroll@@YGXPAVCDataExchange@@HAAHPAVCDaoRecordset@@@Z 5f84e95a f
 0001:0004d996       ?DDX_FieldSlider@@YGXPAVCDataExchange@@HAAHPAVCDaoRecordset@@@Z 5f84e996 f
 0001:0004d9d2       ?DDX_FieldCheck@@YGXPAVCDataExchange@@HAAHPAVCDaoRecordset@@@Z 5f84e9d2 f
 0001:0004da7e       ?DDX_FieldRadio@@YGXPAVCDataExchange@@HAAHPAVCDaoRecordset@@@Z 5f84ea7e f
 0001:0004dae7       ?OnUpdateRecordNext@CDaoRecordView@@IAEXPAVCCmdUI@@@Z 5f84eae7 f
 0001:0004dafe       ?OnUpdateRecordPrev@CDaoRecordView@@IAEXPAVCCmdUI@@@Z 5f84eafe f
 0001:0004db15       ?OnUpdateRecordLast@CDaoRecordView@@IAEXPAVCCmdUI@@@Z 5f84eb15 f
 0001:0004db2c       ?MoveLast@CRowset@ATL@@QAEJXZ 5f84eb2c f
 0001:0004db7e       ??0CPen@@QAE@XZ            5f84eb7e f
 0001:0004db8b       ??0CBrush@@QAE@XZ          5f84eb8b f
 0001:0004db98       ??0CFont@@QAE@XZ           5f84eb98 f
 0001:0004dba5       ??0CBitmap@@QAE@XZ         5f84eba5 f
 0001:0004dbb2       ??0CPalette@@QAE@XZ        5f84ebb2 f
 0001:0004dbbf       ??1CPalette@@UAE@XZ        5f84ebbf f
 0001:0004dbf2       ??0CRgn@@QAE@XZ            5f84ebf2 f
 0001:0004dbff       ??0CMenu@@QAE@XZ           5f84ebff f
 0001:0004dc0c       ??0CStatic@@QAE@XZ         5f84ec0c f
 0001:0004dc1e       ??0CButton@@QAE@XZ         5f84ec1e f
 0001:0004dc30       ??0CListBox@@QAE@XZ        5f84ec30 f
 0001:0004dc42       ??0CCheckListBox@@QAE@XZ   5f84ec42 f
 0001:0004dc5c       ??1CCheckListBox@@UAE@XZ   5f84ec5c f
 0001:0004dc5c       ??1CListBox@@UAE@XZ        5f84ec5c f
 0001:0004dc94       ??0CComboBox@@QAE@XZ       5f84ec94 f
 0001:0004dca6       ??0CEdit@@QAE@XZ           5f84eca6 f
 0001:0004dcb8       ??0CScrollBar@@QAE@XZ      5f84ecb8 f
 0001:0004dcca       ??0CRectTracker@@QAE@XZ    5f84ecca f
 0001:0004dcdc       ??0CBitmapButton@@QAE@XZ   5f84ecdc f
 0001:0004dd0d       ??1CBitmapButton@@UAE@XZ   5f84ed0d f
 0001:0004dda1       ??0COleVariant@@QAE@XZ     5f84eda1 f
 0001:0004ddae       ??0CDataPathProperty@@QAE@PAVCOleControl@@@Z 5f84edae f
 0001:0004dded       ??0CCachedDataPathProperty@@QAE@PAVCOleControl@@@Z 5f84eded f
 0001:0004de46       ??1CCachedDataPathProperty@@UAE@XZ 5f84ee46 f
 0001:0004de8a       ??0CCriticalSection@@QAE@XZ 5f84ee8a f
 0001:0004dea8       ??0CDragListBox@@QAE@XZ    5f84eea8 f
 0001:0004debe       ??0CToolBarCtrl@@QAE@XZ    5f84eebe f
 0001:0004ded0       ??0CStatusBarCtrl@@QAE@XZ  5f84eed0 f
 0001:0004dee2       ??0CListCtrl@@QAE@XZ       5f84eee2 f
 0001:0004def4       ??0CTreeCtrl@@QAE@XZ       5f84eef4 f
 0001:0004df06       ??0CHotKeyCtrl@@QAE@XZ     5f84ef06 f
 0001:0004df18       ??0CSpinButtonCtrl@@QAE@XZ 5f84ef18 f
 0001:0004df2a       ??0CSliderCtrl@@QAE@XZ     5f84ef2a f
 0001:0004df3c       ??0CProgressCtrl@@QAE@XZ   5f84ef3c f
 0001:0004df4e       ??0CHeaderCtrl@@QAE@XZ     5f84ef4e f
 0001:0004df60       ??0CTabCtrl@@QAE@XZ        5f84ef60 f
 0001:0004df72       ??0CAnimateCtrl@@QAE@XZ    5f84ef72 f
 0001:0004df84       ??0CRichEditCtrl@@QAE@XZ   5f84ef84 f
 0001:0004df96       ??0CListView@@QAE@XZ       5f84ef96 f
 0001:0004dfb2       ??0CTreeView@@QAE@XZ       5f84efb2 f
 0001:0004dfce       ??_Gtype_info@@UAEPAXI@Z   5f84efce f
 0001:0004dfce       ??_Etype_info@@UAEPAXI@Z   5f84efce f
 0001:0004dff6       __CxxThrowException@8      5f84eff6 f
 0001:0004dffc       __purecall                 5f84effc f
 0001:0004e002       __alldiv                   5f84f002 f
 0001:0004e0ac       __allmul                   5f84f0ac f
 0001:0004e0e0       __allshr                   5f84f0e0 f
 0001:0004e12d       ?__ArrayUnwind@@YGXPAXIHP6EX0@Z@Z 5f84f12d f
 0001:0004e19c       __ftol                     5f84f19c f
 0001:0004e1a2       _labs                      5f84f1a2 f
 0001:0004e1a8       _fabs                      5f84f1a8 f
 0001:0004e1d1       ??1type_info@@UAE@XZ       5f84f1d1 f
 0001:0004e1d7       __except_handler3          5f84f1d7 f
 0001:0004e1dd       ?terminate@@YAXXZ          5f84f1dd f
 0001:0004e1e3       _ReuseDDElParam@20         5f84f1e3 f
 0001:0004e1e9       _UnpackDDElParam@16        5f84f1e9 f
 0001:0004e1ef       __imp_load__OleCreateFontIndirect@12 5f84f1ef f
 0001:0004e1f6       __tailMerge_OLEPRO32       5f84f1f6 f
 0001:0004e204       __imp_load__OleCreatePropertyFrame@44 5f84f204 f
 0001:0004e20d       __imp_load__OleTranslateColor@12 5f84f20d f
 0001:0004e216       __imp_load__OleCreatePictureIndirect@16 5f84f216 f
 0001:0004e21f       __imp_load__OleLoadPicture@20 5f84f21f f
 0001:0004e228       __imp_load__SetFileSecurityW@12 5f84f228 f
 0001:0004e234       __imp_load__GetFileSecurityW@20 5f84f234 f
 0001:0004e240       __imp_load__RegEnumKeyW@16 5f84f240 f
 0001:0004e24c       __imp_load__RegDeleteValueW@8 5f84f24c f
 0001:0004e258       __imp_load__OleLockRunning@12 5f84f258 f
 0001:0004e264       __imp_load__OleSetContainedObject@8 5f84f264 f
 0001:0004e270       __imp_load__OleCreateFromData@28 5f84f270 f
 0001:0004e27c       __imp_load__OleCreateLinkFromData@28 5f84f27c f
 0001:0004e288       __imp_load__OleCreateStaticFromData@28 5f84f288 f
 0001:0004e294       __imp_load__OleCreateFromFile@32 5f84f294 f
 0001:0004e2a0       __imp_load__OleCreateLinkToFile@28 5f84f2a0 f
 0001:0004e2ac       __imp_load__OleCreate@28   5f84f2ac f
 0001:0004e2b8       __imp_load__OleLoad@16     5f84f2b8 f
 0001:0004e2c4       __imp_load__OleSave@12     5f84f2c4 f
 0001:0004e2d0       __imp_load__StgCreateDocfileOnILockBytes@16 5f84f2d0 f
 0001:0004e2dc       __imp_load__CreateILockBytesOnHGlobal@12 5f84f2dc f
 0001:0004e2e8       __imp_load__StgOpenStorageOnILockBytes@24 5f84f2e8 f
 0001:0004e2f4       __imp_load__GetHGlobalFromILockBytes@8 5f84f2f4 f
 0001:0004e300       __imp_load__ReleaseStgMedium@4 5f84f300 f
 0001:0004e30c       __imp_load__OleGetIconOfClass@12 5f84f30c f
 0001:0004e318       __imp_load__WriteClassStm@8 5f84f318 f
 0001:0004e324       __imp_load__OleSaveToStream@8 5f84f324 f
 0001:0004e330       __imp_load__CreateStreamOnHGlobal@12 5f84f330 f
 0001:0004e33c       __imp_load__CreateItemMoniker@12 5f84f33c f
 0001:0004e348       __imp_load__CreateGenericComposite@12 5f84f348 f
 0001:0004e354       __imp_load__OleSetMenuDescriptor@20 5f84f354 f
 0001:0004e360       __imp_load__OleQueryCreateFromData@4 5f84f360 f
 0001:0004e36c       __imp_load__OleQueryLinkFromData@4 5f84f36c f
 0001:0004e378       __imp_load__OleIsRunning@4 5f84f378 f
 0001:0004e384       __imp_load__CoTaskMemAlloc@4 5f84f384 f
 0001:0004e390       __imp_load__OleGetClipboard@4 5f84f390 f
 0001:0004e39c       __imp_load__OleSetClipboard@4 5f84f39c f
 0001:0004e3a8       __imp_load__OleFlushClipboard@0 5f84f3a8 f
 0001:0004e3b4       __imp_load__OleIsCurrentClipboard@4 5f84f3b4 f
 0001:0004e3c0       __imp_load__CLSIDFromProgID@8 5f84f3c0 f
 0001:0004e3cc       __imp_load__CLSIDFromString@8 5f84f3cc f
 0001:0004e3d8       __imp_load__CreateBindCtx@8 5f84f3d8 f
 0001:0004e3e4       __imp_load__GetClassFile@8 5f84f3e4 f
 0001:0004e3f0       __imp_load__OleRegGetUserType@12 5f84f3f0 f
 0001:0004e3fc       __imp_load__ReadFmtUserTypeStg@12 5f84f3fc f
 0001:0004e408       __imp_load__ReadClassStg@8 5f84f408 f
 0001:0004e414       __imp_load__StgCreateDocfile@16 5f84f414 f
 0001:0004e420       __imp_load__StgOpenStorage@24 5f84f420 f
 0001:0004e42c       __imp_load__StgIsStorageFile@4 5f84f42c f
 0001:0004e438       __imp_load__DoDragDrop@16  5f84f438 f
 0001:0004e444       __imp_load__OleTranslateAccelerator@12 5f84f444 f
 0001:0004e450       __imp_load__IsAccelerator@16 5f84f450 f
 0001:0004e45c       __imp_load__OleCreateMenuDescriptor@8 5f84f45c f
 0001:0004e468       __imp_load__OleDestroyMenuDescriptor@4 5f84f468 f
 0001:0004e474       __imp_load__WriteClassStg@8 5f84f474 f
 0001:0004e480       __imp_load__OleDuplicateData@12 5f84f480 f
 0001:0004e48c       __imp_load__SetConvertStg@8 5f84f48c f
 0001:0004e498       __imp_load__WriteFmtUserTypeStg@12 5f84f498 f
 0001:0004e4a4       __imp_load__CoTreatAsClass@8 5f84f4a4 f
 0001:0004e4b0       __imp_load__OleRegEnumVerbs@8 5f84f4b0 f
 0001:0004e4bc       __imp_load__OleRegGetMiscStatus@12 5f84f4bc f
 0001:0004e4c8       __imp_load__CreateOleAdviseHolder@4 5f84f4c8 f
 0001:0004e4d4       __imp_load__CreateDataAdviseHolder@4 5f84f4d4 f
 0001:0004e4e0       __imp_load__CoGetClassObject@20 5f84f4e0 f
 0001:0004e4ec       __imp_load__CoGetMalloc@8  5f84f4ec f
 0001:0004e4f8       __imp_load__CreateDataCache@16 5f84f4f8 f
 0001:0004e504       __imp_load__ReadClassStm@8 5f84f504 f
 0001:0004e510       __imp_load__OleLoadFromStream@12 5f84f510 f
 0001:0004e51c       __imp_load__StringFromGUID2@12 5f84f51c f
 0001:0004e528       __imp_load__CoInitialize@4 5f84f528 f
 0001:0004e534       __imp_load__CoUninitialize@0 5f84f534 f
 0001:0004e540       __imp_load__SysStringLen@4 5f84f540 f
 0001:0004e54c       __imp_load__VariantCopy@8  5f84f54c f
 0001:0004e558       __imp_load__SysAllocStringLen@8 5f84f558 f
 0001:0004e564       __imp_load__SysReAllocStringLen@12 5f84f564 f
 0001:0004e570       __imp_load__SysFreeString@4 5f84f570 f
 0001:0004e57c       __imp_load__SafeArrayUnaccessData@4 5f84f57c f
 0001:0004e588       __imp_load__SafeArrayAccessData@8 5f84f588 f
 0001:0004e594       __imp_load__SafeArrayGetUBound@12 5f84f594 f
 0001:0004e5a0       __imp_load__SafeArrayGetLBound@12 5f84f5a0 f
 0001:0004e5ac       __imp_load__SafeArrayGetElemsize@4 5f84f5ac f
 0001:0004e5b8       __imp_load__SafeArrayGetDim@4 5f84f5b8 f
 0001:0004e5c4       __imp_load__SafeArrayCreate@12 5f84f5c4 f
 0001:0004e5d0       __imp_load__SafeArrayRedim@8 5f84f5d0 f
 0001:0004e5dc       __imp_load__SysStringByteLen@4 5f84f5dc f
 0001:0004e5e8       __imp_load__SysAllocStringByteLen@8 5f84f5e8 f
 0001:0004e5f4       __imp_load__VarCyFromStr@16 5f84f5f4 f
 0001:0004e600       __imp_load__VarBstrFromCy@20 5f84f600 f
 0001:0004e60c       __imp_load__VarDateFromStr@16 5f84f60c f
 0001:0004e618       __imp_load__VarBstrFromDate@20 5f84f618 f
 0001:0004e624       __imp_load__SafeArrayCopy@8 5f84f624 f
 0001:0004e630       __imp_load__SafeArrayAllocData@4 5f84f630 f
 0001:0004e63c       __imp_load__SafeArrayAllocDescriptor@8 5f84f63c f
 0001:0004e648       __imp_load__SafeArrayGetElement@12 5f84f648 f
 0001:0004e654       __imp_load__SafeArrayPtrOfIndex@12 5f84f654 f
 0001:0004e660       __imp_load__SafeArrayPutElement@12 5f84f660 f
 0001:0004e66c       __imp_load__SafeArrayLock@4 5f84f66c f
 0001:0004e678       __imp_load__SafeArrayUnlock@4 5f84f678 f
 0001:0004e684       __imp_load__SafeArrayDestroy@4 5f84f684 f
 0001:0004e690       __imp_load__SafeArrayDestroyData@4 5f84f690 f
 0001:0004e69c       __imp_load__SafeArrayDestroyDescriptor@4 5f84f69c f
 0001:0004e6a8       __imp_load__SafeArrayCreateVector@12 5f84f6a8 f
 0001:0004e6b4       __imp_load__LoadTypeLib@8  5f84f6b4 f
 0001:0004e6c0       __imp_load__VariantTimeToSystemTime@12 5f84f6c0 f
 0001:0004e6cc       __imp_load__RegisterTypeLib@12 5f84f6cc f
 0001:0004e6d8       __imp_load__LoadRegTypeLib@20 5f84f6d8 f
 0001:0004e6e4       __imp_load__InitCommonControls@0 5f84f6e4 f
 0001:0004e6f0       __imp_load__MakeDragList@4 5f84f6f0 f
 0001:0004e6fc       __imp_load__LBItemFromPt@16 5f84f6fc f
 0001:0004e708       __imp_load__ImageList_Destroy@4 5f84f708 f
 0001:0004e714       __imp_load__ImageList_Create@20 5f84f714 f
 0001:0004e720       __imp_load__ImageList_LoadImageW@28 5f84f720 f
 0001:0004e72c       __imp_load__ImageList_Merge@24 5f84f72c f
 0001:0004e738       __imp_load__ImageList_Read@4 5f84f738 f
 0001:0004e744       _ImageList_Read@4          5f84f744 f
 0001:0004e74a       __imp_load__ImageList_Write@8 5f84f74a f
 0001:0004e756       _ImageList_Write@8         5f84f756 f
 0001:0004e75c       __imp_load__PropertySheetW@4 5f84f75c f
 0001:0004e768       __imp_load__DestroyPropertySheetPage@4 5f84f768 f
 0001:0004e774       __imp_load__CreatePropertySheetPageW@4 5f84f774 f
 0001:0004e780       __imp_load__ImageList_DrawIndirect@4 5f84f780 f
 0001:0004e78c       __imp_load__ImageList_Duplicate@4 5f84f78c f
 0001:0004e798       __imp_load__DragFinish@4   5f84f798 f
 0001:0004e7a4       __imp_load__DragQueryFileW@16 5f84f7a4 f
 0001:0004e7b0       __imp_load__GetSaveFileNameW@4 5f84f7b0 f
 0001:0004e7bc       _GetSaveFileNameW@4        5f84f7bc f
 0001:0004e7c2       __imp_load__GetOpenFileNameW@4 5f84f7c2 f
 0001:0004e7ce       _GetOpenFileNameW@4        5f84f7ce f
 0001:0004e7d4       __imp_load__PageSetupDlgW@4 5f84f7d4 f
 0001:0004e7e0       _PageSetupDlgW@4           5f84f7e0 f
 0001:0004e7e6       __imp_load__ChooseColorW@4 5f84f7e6 f
 0001:0004e7f2       _ChooseColorW@4            5f84f7f2 f
 0001:0004e7f8       __imp_load__ChooseFontW@4  5f84f7f8 f
 0001:0004e804       _ChooseFontW@4             5f84f804 f
 0001:0004e80a       __imp_load__ReplaceTextW@4 5f84f80a f
 0001:0004e816       _ReplaceTextW@4            5f84f816 f
 0001:0004e81c       __imp_load__FindTextW@4    5f84f81c f
 0001:0004e828       _FindTextW@4               5f84f828 f
 0001:0004e82e       __imp_load__CommDlgExtendedError@0 5f84f82e f
 0001:0004e83a       _CommDlgExtendedError@0    5f84f83a f
 0001:0004e840       __imp_load__ClosePrinter@4 5f84f840 f
 0001:0004e847       __tailMerge_WINSPOOL       5f84f847 f
 0001:0004e855       _ClosePrinter@4            5f84f855 f
 0001:0004e85b       __imp_load__DocumentPropertiesW@24 5f84f85b f
 0001:0004e864       _DocumentPropertiesW@24    5f84f864 f
 0001:0004e86a       __imp_load__OpenPrinterW@12 5f84f86a f
 0001:0004e873       _OpenPrinterW@12           5f84f873 f
 0001:0004e879       __imp_load__InternetCrackUrlW@16 5f84f879 f
 0001:0004e880       __tailMerge_WININET        5f84f880 f
 0001:0004e88e       __imp_load__InternetCanonicalizeUrlW@16 5f84f88e f
 0001:0004e897       __imp_load__InternetQueryOptionW@16 5f84f897 f
 0001:0004e8a0       __imp_load__InternetOpenW@20 5f84f8a0 f
 0001:0004e8a9       __imp_load__InternetCloseHandle@4 5f84f8a9 f
 0001:0004e8b2       __imp_load__InternetOpenUrlW@24 5f84f8b2 f
 0001:0004e8bb       __imp_load__InternetSetOptionExW@20 5f84f8bb f
 0001:0004e8c4       __imp_load__InternetSetStatusCallback@8 5f84f8c4 f
 0001:0004e8cd       __imp_load__InternetSetCookieW@12 5f84f8cd f
 0001:0004e8d6       __imp_load__InternetGetCookieW@16 5f84f8d6 f
 0001:0004e8df       __imp_load__InternetSetFilePointer@20 5f84f8df f
 0001:0004e8e8       __imp_load__InternetWriteFile@16 5f84f8e8 f
 0001:0004e8f1       __imp_load__InternetReadFile@16 5f84f8f1 f
 0001:0004e8fa       __imp_load__InternetQueryDataAvailable@16 5f84f8fa f
 0001:0004e906       __imp_load__InternetConnectW@32 5f84f906 f
 0001:0004e912       __imp_load__FtpDeleteFileW@8 5f84f912 f
 0001:0004e91e       __imp_load__FtpRenameFileW@12 5f84f91e f
 0001:0004e92a       __imp_load__FtpCreateDirectoryW@8 5f84f92a f
 0001:0004e936       __imp_load__FtpRemoveDirectoryW@8 5f84f936 f
 0001:0004e942       __imp_load__FtpSetCurrentDirectoryW@8 5f84f942 f
 0001:0004e94e       __imp_load__FtpGetCurrentDirectoryW@12 5f84f94e f
 0001:0004e95a       __imp_load__FtpOpenFileW@20 5f84f95a f
 0001:0004e966       __imp_load__FtpPutFileW@20 5f84f966 f
 0001:0004e972       __imp_load__FtpGetFileW@28 5f84f972 f
 0001:0004e97e       __imp_load__GopherCreateLocatorW@28 5f84f97e f
 0001:0004e98a       __imp_load__GopherGetAttributeW@32 5f84f98a f
 0001:0004e996       __imp_load__GopherOpenFileW@20 5f84f996 f
 0001:0004e9a2       __imp_load__HttpOpenRequestW@32 5f84f9a2 f
 0001:0004e9ae       __imp_load__InternetErrorDlg@20 5f84f9ae f
 0001:0004e9ba       __imp_load__HttpAddRequestHeadersW@16 5f84f9ba f
 0001:0004e9c6       __imp_load__HttpSendRequestW@20 5f84f9c6 f
 0001:0004e9d2       __imp_load__HttpEndRequestW@16 5f84f9d2 f
 0001:0004e9de       __imp_load__HttpSendRequestExW@20 5f84f9de f
 0001:0004e9ea       __imp_load__HttpQueryInfoW@20 5f84f9ea f
 0001:0004e9f6       __imp_load__FtpFindFirstFileW@20 5f84f9f6 f
 0001:0004ea02       __imp_load__InternetFindNextFileW@8 5f84fa02 f
 0001:0004ea0e       __imp_load__GopherFindFirstFileW@24 5f84fa0e f
 0001:0004ea1a       __imp_load__InternetGetLastResponseInfoW@12 5f84fa1a f
 0001:0004ea26       __imp_load__WSACleanup@0   5f84fa26 f
 0001:0004ea2d       __tailMerge_WSOCK32        5f84fa2d f
 0001:0004ea3b       _WSACleanup@0              5f84fa3b f
 0001:0004ea41       __imp_load__WSAStartup@8   5f84fa41 f
 0001:0004ea4a       _WSAStartup@8              5f84fa4a f
 0001:0004ea50       __imp_load__WSASetLastError@4 5f84fa50 f
 0001:0004ea59       _WSASetLastError@4         5f84fa59 f
 0001:0004ea5f       __imp_load__WSAGetLastError@0 5f84fa5f f
 0001:0004ea68       _WSAGetLastError@0         5f84fa68 f
 0001:0004ea6e       __imp_load__inet_ntoa@4    5f84fa6e f
 0001:0004ea77       _inet_ntoa@4               5f84fa77 f
 0001:0004ea7d       __imp_load__ntohs@4        5f84fa7d f
 0001:0004ea86       _ntohs@4                   5f84fa86 f
 0001:0004ea8c       __imp_load__getpeername@12 5f84fa8c f
 0001:0004ea95       _getpeername@12            5f84fa95 f
 0001:0004ea9b       __imp_load__getsockname@12 5f84fa9b f
 0001:0004eaa4       _getsockname@12            5f84faa4 f
 0001:0004eaaa       __imp_load__accept@12      5f84faaa f
 0001:0004eab6       _accept@12                 5f84fab6 f
 0001:0004eabc       __imp_load__inet_addr@4    5f84fabc f
 0001:0004eac8       _inet_addr@4               5f84fac8 f
 0001:0004eace       __imp_load__bind@12        5f84face f
 0001:0004eada       _bind@12                   5f84fada f
 0001:0004eae0       __imp_load__htons@4        5f84fae0 f
 0001:0004eaec       _htons@4                   5f84faec f
 0001:0004eaf2       __imp_load__htonl@4        5f84faf2 f
 0001:0004eafe       _htonl@4                   5f84fafe f
 0001:0004eb04       __imp_load__closesocket@4  5f84fb04 f
 0001:0004eb10       _closesocket@4             5f84fb10 f
 0001:0004eb16       __imp_load__gethostbyname@4 5f84fb16 f
 0001:0004eb22       _gethostbyname@4           5f84fb22 f
 0001:0004eb28       __imp_load__recv@16        5f84fb28 f
 0001:0004eb34       _recv@16                   5f84fb34 f
 0001:0004eb3a       __imp_load__send@16        5f84fb3a f
 0001:0004eb46       _send@16                   5f84fb46 f
 0001:0004eb4c       __imp_load__WSAAsyncSelect@16 5f84fb4c f
 0001:0004eb58       _WSAAsyncSelect@16         5f84fb58 f
 0001:0004eb5e       __imp_load__ioctlsocket@12 5f84fb5e f
 0001:0004eb6a       _ioctlsocket@12            5f84fb6a f
 0001:0004eb70       __imp_load__socket@12      5f84fb70 f
 0001:0004eb7c       _socket@12                 5f84fb7c f
 0001:0004eb82       __imp_load__recvfrom@24    5f84fb82 f
 0001:0004eb8e       _recvfrom@24               5f84fb8e f
 0001:0004eb94       __imp_load__sendto@24      5f84fb94 f
 0001:0004eba0       _sendto@24                 5f84fba0 f
 0001:0004eba6       __imp_load__connect@12     5f84fba6 f
 0001:0004ebb2       _connect@12                5f84fbb2 f
 0001:0004ebb8       __imp_load__OleUIInsertObjectW@4 5f84fbb8 f
 0001:0004ebbf       __tailMerge_oledlg         5f84fbbf f
 0001:0004ebcd       _OleUIInsertObjectW@4      5f84fbcd f
 0001:0004ebd3       __imp_load__OleUIConvertW@4 5f84fbd3 f
 0001:0004ebdc       _OleUIConvertW@4           5f84fbdc f
 0001:0004ebe2       __imp_load__OleUIChangeIconW@4 5f84fbe2 f
 0001:0004ebeb       _OleUIChangeIconW@4        5f84fbeb f
 0001:0004ebf1       __imp_load__OleUIEditLinksW@4 5f84fbf1 f
 0001:0004ebfa       _OleUIEditLinksW@4         5f84fbfa f
 0001:0004ec00       __imp_load__OleUIUpdateLinksW@16 5f84fc00 f
 0001:0004ec09       _OleUIUpdateLinksW@16      5f84fc09 f
 0001:0004ec0f       __imp_load__OleUIPasteSpecialW@4 5f84fc0f f
 0001:0004ec18       _OleUIPasteSpecialW@4      5f84fc18 f
 0001:0004ec1e       __imp_load__OleUIBusyW@4   5f84fc1e f
 0001:0004ec27       _OleUIBusyW@4              5f84fc27 f
 0001:0004ec2d       __imp_load__OleUIObjectPropertiesW@4 5f84fc2d f
 0001:0004ec36       _OleUIObjectPropertiesW@4  5f84fc36 f
 0001:0004ec3c       __imp_load__OleUIChangeSourceW@4 5f84fc3c f
 0001:0004ec48       _OleUIChangeSourceW@4      5f84fc48 f
 0001:0004ec4e       __imp_load__OleUIAddVerbMenuW@36 5f84fc4e f
 0001:0004ec5a       _OleUIAddVerbMenuW@36      5f84fc5a f
 0001:0004ec60       __imp_load__CreateURLMoniker@12 5f84fc60 f
 0001:0004ec67       __tailMerge_urlmon         5f84fc67 f
 0001:0004ec75       _CreateURLMoniker@12       5f84fc75 f
 0001:0004ec7b       __imp_load__CreateAsyncBindCtx@16 5f84fc7b f
 0001:0004ec84       _CreateAsyncBindCtx@16     5f84fc84 f
 0001:0004ec8a       __imp_load__RegisterBindStatusCallback@16 5f84fc8a f
 0001:0004ec93       _RegisterBindStatusCallback@16 5f84fc93 f
 0001:0004ec99       __imp_load__IsAsyncMoniker@4 5f84fc99 f
 0001:0004eca2       _IsAsyncMoniker@4          5f84fca2 f
 0001:0004eca8       __imp_load__SQLError@32    5f84fca8 f
 0001:0004ecaf       __tailMerge_ODBC32         5f84fcaf f
 0001:0004ecbd       _SQLError@32               5f84fcbd f
 0001:0004ecc3       __imp_load__SQLCancel@4    5f84fcc3 f
 0001:0004eccc       _SQLCancel@4               5f84fccc f
 0001:0004ecd2       __imp_load__SQLFreeStmt@8  5f84fcd2 f
 0001:0004ecdb       _SQLFreeStmt@8             5f84fcdb f
 0001:0004ece1       __imp_load__SQLMoreResults@4 5f84fce1 f
 0001:0004ecea       _SQLMoreResults@4          5f84fcea f
 0001:0004ecf0       __imp_load__SQLFetch@4     5f84fcf0 f
 0001:0004ecf9       _SQLFetch@4                5f84fcf9 f
 0001:0004ecff       __imp_load__SQLNumResultCols@8 5f84fcff f
 0001:0004ed08       _SQLNumResultCols@8        5f84fd08 f
 0001:0004ed0e       __imp_load__SQLExecDirect@12 5f84fd0e f
 0001:0004ed17       _SQLExecDirect@12          5f84fd17 f
 0001:0004ed1d       __imp_load__SQLAllocStmt@8 5f84fd1d f
 0001:0004ed26       _SQLAllocStmt@8            5f84fd26 f
 0001:0004ed2c       __imp_load__SQLFreeConnect@4 5f84fd2c f
 0001:0004ed38       _SQLFreeConnect@4          5f84fd38 f
 0001:0004ed3e       __imp_load__SQLDisconnect@4 5f84fd3e f
 0001:0004ed4a       _SQLDisconnect@4           5f84fd4a f
 0001:0004ed50       __imp_load__SQLFreeEnv@4   5f84fd50 f
 0001:0004ed5c       _SQLFreeEnv@4              5f84fd5c f
 0001:0004ed62       __imp_load__SQLSetStmtOption@12 5f84fd62 f
 0001:0004ed6e       _SQLSetStmtOption@12       5f84fd6e f
 0001:0004ed74       __imp_load__SQLGetInfo@20  5f84fd74 f
 0001:0004ed80       _SQLGetInfo@20             5f84fd80 f
 0001:0004ed86       __imp_load__SQLSetConnectOption@12 5f84fd86 f
 0001:0004ed92       _SQLSetConnectOption@12    5f84fd92 f
 0001:0004ed98       __imp_load__SQLTransact@12 5f84fd98 f
 0001:0004eda4       _SQLTransact@12            5f84fda4 f
 0001:0004edaa       __imp_load__SQLAllocConnect@8 5f84fdaa f
 0001:0004edb6       _SQLAllocConnect@8         5f84fdb6 f
 0001:0004edbc       __imp_load__SQLAllocEnv@4  5f84fdbc f
 0001:0004edc8       _SQLAllocEnv@4             5f84fdc8 f
 0001:0004edce       __imp_load__SQLDriverConnect@32 5f84fdce f
 0001:0004edda       _SQLDriverConnect@32       5f84fdda f
 0001:0004ede0       __imp_load__SQLGetData@24  5f84fde0 f
 0001:0004edec       _SQLGetData@24             5f84fdec f
 0001:0004edf2       __imp_load__SQLSetPos@16   5f84fdf2 f
 0001:0004edfe       _SQLSetPos@16              5f84fdfe f
 0001:0004ee04       __imp_load__SQLExecute@4   5f84fe04 f
 0001:0004ee10       _SQLExecute@4              5f84fe10 f
 0001:0004ee16       __imp_load__SQLGetStmtOption@12 5f84fe16 f
 0001:0004ee22       _SQLGetStmtOption@12       5f84fe22 f
 0001:0004ee28       __imp_load__SQLPrepare@12  5f84fe28 f
 0001:0004ee34       _SQLPrepare@12             5f84fe34 f
 0001:0004ee3a       __imp_load__SQLGetFunctions@12 5f84fe3a f
 0001:0004ee46       _SQLGetFunctions@12        5f84fe46 f
 0001:0004ee4c       __imp_load__SQLDescribeCol@36 5f84fe4c f
 0001:0004ee58       _SQLDescribeCol@36         5f84fe58 f
 0001:0004ee5e       __imp_load__SQLExtendedFetch@20 5f84fe5e f
 0001:0004ee6a       _SQLExtendedFetch@20       5f84fe6a f
 0001:0004ee70       __imp_load__SQLGetCursorName@16 5f84fe70 f
 0001:0004ee7c       _SQLGetCursorName@16       5f84fe7c f
 0001:0004ee82       __imp_load__SQLRowCount@8  5f84fe82 f
 0001:0004ee8e       _SQLRowCount@8             5f84fe8e f
 0001:0004ee94       __imp_load__SQLPutData@12  5f84fe94 f
 0001:0004eea0       _SQLPutData@12             5f84fea0 f
 0001:0004eea6       __imp_load__SQLParamData@8 5f84fea6 f
 0001:0004eeb2       _SQLParamData@8            5f84feb2 f
 0001:0004eeb8       __imp_load__SQLBindCol@24  5f84feb8 f
 0001:0004eec4       _SQLBindCol@24             5f84fec4 f
 0001:0004eeca       __imp_load__SQLBindParameter@40 5f84feca f
 0001:0004eed6       _SQLBindParameter@40       5f84fed6 f
 0001:0004f047       ?InitString@CSimpleException@@QAEXXZ 5f850047 f
 0001:0004f070       ?GetErrorMessage@CSimpleException@@UAEHPAGIPAI@Z 5f850070 f
 0001:0004f0b4       ?AfxThrowMemoryException@@YGXXZ 5f8500b4 f
 0001:0004f0cd       ?AfxThrowNotSupportedException@@YGXXZ 5f8500cd f
 0001:0004f0e6       ?AfxIsValidString@@YGHPBGH@Z 5f8500e6 f
 0001:0004f112       ?AfxIsValidString@@YGHPBDH@Z 5f850112 f
 0001:0004f133       ?AfxIsValidAddress@@YGHPBXIH@Z 5f850133 f
 0001:0004f16c       ?AfxAbort@@YGXXZ           5f85016c f
 0001:0004f177       ??0CString@@QAE@GH@Z       5f850177 f
 0001:0004f1b2       ??0CString@@QAE@PBGH@Z     5f8501b2 f
 0001:0004f1e8       ??0CString@@QAE@PBDH@Z     5f8501e8 f
 0001:0004f230       ??4CString@@QAEABV0@G@Z    5f850230 f
 0001:0004f245       ??H@YG?AVCString@@ABV0@G@Z 5f850245 f
 0001:0004f2a7       ??H@YG?AVCString@@GABV0@@Z 5f8502a7 f
 0001:0004f309       ?Delete@CString@@QAEHHH@Z  5f850309 f
 0001:0004f36c       ?Insert@CString@@QAEHHG@Z  5f85036c f
 0001:0004f404       ?Insert@CString@@QAEHHPBG@Z 5f850404 f
 0001:0004f4d3       ?Replace@CString@@QAEHGG@Z 5f8504d3 f
 0001:0004f517       ?Replace@CString@@QAEHPBG0@Z 5f850517 f
 0001:0004f6a0       ?Remove@CString@@QAEHG@Z   5f8506a0 f
 0001:0004f6dc       ?Mid@CString@@QBE?AV1@H@Z  5f8506dc f
 0001:0004f6ff       ?Mid@CString@@QBE?AV1@HH@Z 5f8506ff f
 0001:0004f7a0       ?Right@CString@@QBE?AV1@H@Z 5f8507a0 f
 0001:0004f825       ?Left@CString@@QBE?AV1@H@Z 5f850825 f
 0001:0004f8a5       ?SpanIncluding@CString@@QBE?AV1@PBG@Z 5f8508a5 f
 0001:0004f8d0       ?SpanExcluding@CString@@QBE?AV1@PBG@Z 5f8508d0 f
 0001:0004f8fb       ?ReverseFind@CString@@QBEHG@Z 5f8508fb f
 0001:0004f91e       ?Find@CString@@QBEHPBG@Z   5f85091e f
 0001:0004f92c       ?Find@CString@@QBEHPBGH@Z  5f85092c f
 0001:0004faac       ?Format@CString@@QAAXIZZ   5f850aac f
 0001:0004faf5       ?FormatMessageW@CString@@QAAXPBGZZ 5f850af5 f
 0001:0004fb41       ?FormatMessageW@CString@@QAAXIZZ 5f850b41 f
 0001:0004fbc4       ?TrimRight@CString@@QAEXPBG@Z 5f850bc4 f
 0001:0004fc15       ?TrimRight@CString@@QAEXG@Z 5f850c15 f
 0001:0004fc58       ?TrimRight@CString@@QAEXXZ 5f850c58 f
 0001:0004fca2       ?TrimLeft@CString@@QAEXPBG@Z 5f850ca2 f
 0001:0004fd09       ?TrimLeft@CString@@QAEXG@Z 5f850d09 f
 0001:0004fd4d       ?TrimLeft@CString@@QAEXXZ  5f850d4d f
 0001:0004fd9c       ?ConstructElements@@YGXPAVCString@@H@Z 5f850d9c f
 0001:0004fdcb       ?DestructElements@@YGXPAVCString@@H@Z 5f850dcb f
 0001:0004fdef       ?CopyElements@@YGXPAVCString@@PBV1@H@Z 5f850def f
 0001:0004fe1b       ?HashKey@@YGIPBG@Z         5f850e1b f
 0001:0004fe38       ?HashKey@@YGIPBD@Z         5f850e38 f
 0001:0004fe52       ??0CTime@@QAE@GGH@Z        5f850e52 f
 0001:0004fecc       ?GetTickCount@CTime@@SG?AV1@XZ 5f850ecc f
 0001:0004feef       ?GetGmtTm@CTime@@QBEPAUtm@@PAU2@@Z 5f850eef f
 0001:0004ff1d       ?GetLocalTm@CTime@@QBEPAUtm@@PAU2@@Z 5f850f1d f
 0001:0004ff4e       ?GetAsSystemTime@CTime@@QBEHAAU_SYSTEMTIME@@@Z 5f850f4e f
 0001:0004ffa5       ??6@YGAAVCArchive@@AAV0@VCTimeSpan@@@Z 5f850fa5 f
 0001:0004ffb5       ??5@YGAAVCArchive@@AAV0@AAVCTimeSpan@@@Z 5f850fb5 f
 0001:0004ffc5       ?Format@CTimeSpan@@QBE?AVCString@@PBG@Z 5f850fc5 f
 0001:000500fc       ?Format@CTimeSpan@@QBE?AVCString@@I@Z 5f8510fc f
 0001:00050158       ?Format@CTime@@QBE?AVCString@@PBG@Z 5f851158 f
 0001:000501ac       ?FormatGmt@CTime@@QBE?AVCString@@PBG@Z 5f8511ac f
 0001:00050200       ?Format@CTime@@QBE?AVCString@@I@Z 5f851200 f
 0001:0005025c       ?FormatGmt@CTime@@QBE?AVCString@@I@Z 5f85125c f
 0001:000502b8       ?Format@CTime@@QBE?AVCString@@PBD@Z 5f8512b8 f
 0001:0005030b       ?FormatGmt@CTime@@QBE?AVCString@@PBD@Z 5f85130b f
 0001:0005035e       ?Format@CTimeSpan@@QBE?AVCString@@PBD@Z 5f85135e f
 0001:000503b1       ??0CTime@@QAE@ABV0@@Z      5f8513b1 f
 0001:000503be       ?LoadBitmaps@CBitmapButton@@QAEHPBG000@Z 5f8513be f
 0001:0005048e       ?SizeToContent@CBitmapButton@@QAEXXZ 5f85148e f
 0001:000504be       ?AutoLoad@CBitmapButton@@QAEHIPAVCWnd@@@Z 5f8514be f
 0001:000505cd       ?DrawItem@CBitmapButton@@MAEXPAUtagDRAWITEMSTRUCT@@@Z 5f8515cd f
 0001:000506d2       ?_AfxCommDlgProc@@YGIPAUHWND__@@IIJ@Z 5f8516d2 f
 0001:00050865       ?OnHelpInfo@CCommonDialog@@IAEHPAUtagHELPINFO@@@Z 5f851865 f
 0001:0005086d       ??0CFileDialog@@QAE@HPBG0K0PAVCWnd@@@Z 5f85186d f
 0001:000509c5       ??_GCFileDialog@@UAEPAXI@Z 5f8519c5 f
 0001:000509c5       ??_ECFileDialog@@UAEPAXI@Z 5f8519c5 f
 0001:000509e1       ?DoModal@CFileDialog@@UAEHXZ 5f8519e1 f
 0001:00050acc       ?GetPathName@CFileDialog@@QBE?AVCString@@XZ 5f851acc f
 0001:00050bda       ?GetFileName@CFileDialog@@QBE?AVCString@@XZ 5f851bda f
 0001:00050c95       ?GetFileExt@CFileDialog@@QBE?AVCString@@XZ 5f851c95 f
 0001:00050da5       ?GetFileTitle@CFileDialog@@QBE?AVCString@@XZ 5f851da5 f
 0001:00050e11       ?GetNextPathName@CFileDialog@@QBE?AVCString@@AAPAU__POSITION@@@Z 5f851e11 f
 0001:00050ff4       ?SetTemplate@CFileDialog@@QAEXPBG0@Z 5f851ff4 f
 0001:0005101a       ?GetFolderPath@CFileDialog@@QBE?AVCString@@XZ 5f85201a f
 0001:000510b3       ?SetControlText@CFileDialog@@QAEXHPBD@Z 5f8520b3 f
 0001:000510db       ?HideControl@CFileDialog@@QAEXH@Z 5f8520db f
 0001:00051101       ?SetDefExt@CFileDialog@@QAEXPBD@Z 5f852101 f
 0001:00051127       ?OnShareViolation@CFileDialog@@MAEIPBG@Z 5f852127 f
 0001:0005112c       ?OnLBSelChangedNotify@CFileDialog@@MAEXIII@Z 5f85212c f
 0001:0005112f       ?OnInitDone@CFileDialog@@MAEXXZ 5f85212f f
 0001:00051148       ?OnTypeChange@CFileDialog@@MAEXXZ 5f852148 f
 0001:00051149       ?OnNotify@CFileDialog@@MAEHIJPAJ@Z 5f852149 f
 0001:00051223       ??0CPageSetupDialog@@QAE@KPAVCWnd@@@Z 5f852223 f
 0001:000512a6       ?DoModal@CPageSetupDialog@@UAEHXZ 5f8522a6 f
 0001:000512d2       ?GetDevMode@CPageSetupDialog@@QBEPAU_devicemodeW@@XZ 5f8522d2 f
 0001:000512e2       ?GetDriverName@CPageSetupDialog@@QBE?AVCString@@XZ 5f8522e2 f
 0001:0005131e       ?GetDeviceName@CPageSetupDialog@@QBE?AVCString@@XZ 5f85231e f
 0001:0005135b       ?GetPortName@CPageSetupDialog@@QBE?AVCString@@XZ 5f85235b f
 0001:00051398       ?CreatePrinterDC@CPageSetupDialog@@QAEPAUHDC__@@XZ 5f852398 f
 0001:000513a4       ?GetMargins@CPageSetupDialog@@QBEXPAUtagRECT@@0@Z 5f8523a4 f
 0001:000513e0       ?OnDrawPage@CPageSetupDialog@@UAEIPAVCDC@@IPAUtagRECT@@@Z 5f8523e0 f
 0001:000513e5       ?PaintHookProc@CPageSetupDialog@@KGIPAUHWND__@@IIJ@Z 5f8523e5 f
 0001:0005148c       ??0CPrintDialog@@IAE@AAUtagPDW@@@Z 5f85248c f
 0001:000514ab       ?AttachOnSetup@CPrintDialog@@MAEPAV1@XZ 5f8524ab f
 0001:000514fb       ?OnPrintSetup@CPrintDialog@@IAEXXZ 5f8524fb f
 0001:0005152b       ?CreatePrinterDC@CPrintDialog@@QAEPAUHDC__@@XZ 5f85252b f
 0001:0005154a       ?GetCopies@CPrintDialog@@QBEHXZ 5f85254a f
 0001:00051562       ?GetDevMode@CPrintDialog@@QBEPAU_devicemodeW@@XZ 5f852562 f
 0001:000515bc       ??0_AFX_COLOR_STATE@@QAE@XZ 5f8525bc f
 0001:000515d6       ??_E_AFX_COLOR_STATE@@UAEPAXI@Z 5f8525d6 f
 0001:000515d6       ??_G_AFX_COLOR_STATE@@UAEPAXI@Z 5f8525d6 f
 0001:000515f1       ??1_AFX_COLOR_STATE@@UAE@XZ 5f8525f1 f
 0001:000515f2       ?GetMessageMap@CColorDialog@@MBEPBUAFX_MSGMAP@@XZ 5f8525f2 f
 0001:000515f8       ??0CColorDialog@@QAE@KKPAVCWnd@@@Z 5f8525f8 f
 0001:00051688       ??1CColorDialog@@UAE@XZ    5f852688 f
 0001:0005168d       ?DoModal@CColorDialog@@UAEHXZ 5f85268d f
 0001:000516b9       ?OnColorOK@CColorDialog@@MAEHXZ 5f8526b9 f
 0001:000516bc       ?SetCurrentColor@CColorDialog@@QAEXK@Z 5f8526bc f
 0001:000516d4       ?GetSavedCustomColors@CColorDialog@@SGPAKXZ 5f8526d4 f
 0001:000516e7       ?OnCtlColor@CColorDialog@@IAEPAUHBRUSH__@@PAVCDC@@PAVCWnd@@I@Z 5f8526e7 f
 0001:000516ef       ??0CFontDialog@@QAE@PAUtagLOGFONTW@@KPAVCDC@@PAVCWnd@@@Z 5f8526ef f
 0001:000517d1       ??0CFontDialog@@QAE@ABU_charformat@@KPAVCDC@@PAVCWnd@@@Z 5f8527d1 f
 0001:000518ab       ?DoModal@CFontDialog@@UAEHXZ 5f8528ab f
 0001:000518f3       ?GetCurrentFont@CFontDialog@@QAEXPAUtagLOGFONTW@@@Z 5f8528f3 f
 0001:00051924       ?FillInLogFont@CFontDialog@@QAEKABU_charformat@@@Z 5f852924 f
 0001:00051af5       ?GetCharFormat@CFontDialog@@QBEXAAU_charformat@@@Z 5f852af5 f
 0001:00051c19       ??0CFindReplaceDialog@@QAE@XZ 5f852c19 f
 0001:00051c9e       ?PostNcDestroy@CFindReplaceDialog@@MAEXXZ 5f852c9e f
 0001:00051caa       ?Create@CFindReplaceDialog@@QAEHHPBG0KPAVCWnd@@@Z 5f852caa f
 0001:00051d5e       ?GetNotifier@CFindReplaceDialog@@SGPAV1@J@Z 5f852d5e f
 0001:00051d68       ??0CArchiveStream@@QAE@PAVCArchive@@@Z 5f852d68 f
 0001:00051d7a       ?AddRef@CArchiveStream@@UAGKXZ 5f852d7a f
 0001:00051d80       ?Release@CArchiveStream@@UAGKXZ 5f852d80 f
 0001:00051d85       ?QueryInterface@CArchiveStream@@UAGJABU_GUID@@PAPAX@Z 5f852d85 f
 0001:00051dc9       ?Read@CArchiveStream@@UAGJPAXKPAK@Z 5f852dc9 f
 0001:00051e21       ?Write@CArchiveStream@@UAGJPBXKPAK@Z 5f852e21 f
 0001:00051e7a       ?Seek@CArchiveStream@@UAGJT_LARGE_INTEGER@@KPAT_ULARGE_INTEGER@@@Z 5f852e7a f
 0001:00051efa       ?SetSize@CArchiveStream@@UAGJT_ULARGE_INTEGER@@@Z 5f852efa f
 0001:00051f02       ?CopyTo@CArchiveStream@@UAGJPAUIStream@@T_ULARGE_INTEGER@@PAT3@2@Z 5f852f02 f
 0001:00051f0a       ?Commit@CArchiveStream@@UAGJK@Z 5f852f0a f
 0001:00051f12       ?Revert@CArchiveStream@@UAGJXZ 5f852f12 f
 0001:00051f1a       ?GetMessageMap@CToolTipCtrl@@MBEPBUAFX_MSGMAP@@XZ 5f852f1a f
 0001:00051f20       ??0CToolTipCtrl@@QAE@XZ    5f852f20 f
 0001:00051f59       ?Create@CToolTipCtrl@@QAEHPAVCWnd@@K@Z 5f852f59 f
 0001:00051fae       ??1CToolTipCtrl@@UAE@XZ    5f852fae f
 0001:00051ff5       ?DestroyToolTipCtrl@CToolTipCtrl@@QAEHXZ 5f852ff5 f
 0001:00052023       ?OnAddTool@CToolTipCtrl@@IAEJIJ@Z 5f853023 f
 0001:00052097       ?OnDisableModal@CToolTipCtrl@@IAEJIJ@Z 5f853097 f
 0001:000520ae       ?OnEnable@CToolTipCtrl@@IAEXH@Z 5f8530ae f
 0001:000520c5       ?OnWindowFromPoint@CToolTipCtrl@@IAEJIJ@Z 5f8530c5 f
 0001:0005213d       ?AddTool@CToolTipCtrl@@QAEHPAVCWnd@@PBGPBUtagRECT@@I@Z 5f85313d f
 0001:0005218b       ?AddTool@CToolTipCtrl@@QAEHPAVCWnd@@IPBUtagRECT@@I@Z 5f85318b f
 0001:000521ef       ?DelTool@CToolTipCtrl@@QAEXPAVCWnd@@I@Z 5f8531ef f
 0001:00052220       ?GetText@CToolTipCtrl@@QBEXAAVCString@@PAVCWnd@@I@Z 5f853220 f
 0001:0005226b       ?GetToolInfo@CToolTipCtrl@@QBEHAAVCToolInfo@@PAVCWnd@@I@Z 5f85326b f
 0001:0005229d       ?HitTest@CToolTipCtrl@@QBEHPAVCWnd@@VCPoint@@PAUtagTOOLINFOW@@@Z 5f85329d f
 0001:00052310       ?SetToolRect@CToolTipCtrl@@QAEXPAVCWnd@@IPBUtagRECT@@@Z 5f853310 f
 0001:00052352       ?UpdateTipText@CToolTipCtrl@@QAEXPBGPAVCWnd@@I@Z 5f853352 f
 0001:00052389       ?UpdateTipText@CToolTipCtrl@@QAEXIPAVCWnd@@I@Z 5f853389 f
 0001:000523d9       ?FillInToolInfo@CToolTipCtrl@@QBEXAAUtagTOOLINFOW@@PAVCWnd@@I@Z 5f8533d9 f
 0001:0005248a       ?EnableTrackingToolTips@CWnd@@QAEHH@Z 5f85348a f
 0001:0005249b       ?_AfxRelayToolTipMessage@@YGXPAVCToolTipCtrl@@PAUtagMSG@@@Z 5f85349b f
 0001:000528c5       ??1CDragListBox@@UAE@XZ    5f8538c5 f
 0001:000528fd       ?PreSubclassWindow@CDragListBox@@UAEXXZ 5f8538fd f
 0001:00052907       ?BeginDrag@CDragListBox@@UAEHVCPoint@@@Z 5f853907 f
 0001:00052933       ?CancelDrag@CDragListBox@@UAEXVCPoint@@@Z 5f853933 f
 0001:00052940       ?Dragging@CDragListBox@@UAEIVCPoint@@@Z 5f853940 f
 0001:0005298a       ?Dropped@CDragListBox@@UAEXHVCPoint@@@Z 5f85398a f
 0001:00052a69       ?DrawInsert@CDragListBox@@UAEXH@Z 5f853a69 f
 0001:00052a8e       ?DrawSingle@CDragListBox@@QAEXH@Z 5f853a8e f
 0001:00052b85       ?OnChildNotify@CDragListBox@@MAEHIIJPAJ@Z 5f853b85 f
 0001:00052c3e       ?GetMessageMap@CToolBarCtrl@@MBEPBUAFX_MSGMAP@@XZ 5f853c3e f
 0001:00052c44       ?Create@CToolBarCtrl@@QAEHKABUtagRECT@@PAVCWnd@@I@Z 5f853c44 f
 0001:00052c75       ??1CToolBarCtrl@@UAE@XZ    5f853c75 f
 0001:00052cad       ?AddBitmap@CToolBarCtrl@@QAEHHPAVCBitmap@@@Z 5f853cad f
 0001:00052ce1       ?AddBitmap@CToolBarCtrl@@QAEHHI@Z 5f853ce1 f
 0001:00052d16       ?SaveState@CToolBarCtrl@@QAEXPAUHKEY__@@PBG1@Z 5f853d16 f
 0001:00052d46       ?RestoreState@CToolBarCtrl@@QAEXPAUHKEY__@@PBG1@Z 5f853d46 f
 0001:00052d76       ?AddString@CToolBarCtrl@@QAEHI@Z 5f853d76 f
 0001:00052da3       ?OnCreate@CToolBarCtrl@@IAEHPAUtagCREATESTRUCTW@@@Z 5f853da3 f
 0001:00052dcc       ?GetDropTarget@CToolBarCtrl@@QBEJPAPAUIDropTarget@@@Z 5f853dcc f
 0001:00052de6       ?Create@CStatusBarCtrl@@QAEHKABUtagRECT@@PAVCWnd@@I@Z 5f853de6 f
 0001:00052e17       ??1CStatusBarCtrl@@UAE@XZ  5f853e17 f
 0001:00052e4f       ?GetText@CStatusBarCtrl@@QBEHPBGHPAH@Z 5f853e4f f
 0001:00052e7a       ?GetText@CStatusBarCtrl@@QBE?AVCString@@HPAH@Z 5f853e7a f
 0001:00052f19       ?GetTextLength@CStatusBarCtrl@@QBEHHPAH@Z 5f853f19 f
 0001:00052f42       ?GetTipText@CStatusBarCtrl@@QBE?AVCString@@H@Z 5f853f42 f
 0001:00052f84       ?GetBorders@CStatusBarCtrl@@QBEHAAH00@Z 5f853f84 f
 0001:00052fbe       ?GetMessageMap@CListCtrl@@MBEPBUAFX_MSGMAP@@XZ 5f853fbe f
 0001:00052fc4       ?Create@CListCtrl@@QAEHKABUtagRECT@@PAVCWnd@@I@Z 5f853fc4 f
 0001:00052ff5       ??1CListCtrl@@UAE@XZ       5f853ff5 f
 0001:0005302d       ?GetItemRect@CListCtrl@@QBEHHPAUtagRECT@@I@Z 5f85402d f
 0001:0005304d       ?SetItemCountEx@CListCtrl@@QAEHHK@Z 5f85404d f
 0001:00053066       ?SetIconSpacing@CListCtrl@@QAE?AVCSize@@V2@@Z 5f854066 f
 0001:0005309b       ?GetSubItemRect@CListCtrl@@QAEHHHHAAVCRect@@@Z 5f85409b f
 0001:000530dd       ?InsertColumn@CListCtrl@@QAEHHPBGHHH@Z 5f8540dd f
 0001:00053130       ?InsertItem@CListCtrl@@QAEHIHPBGIIHJ@Z 5f854130 f
 0001:0005317c       ?HitTest@CListCtrl@@QBEHVCPoint@@PAI@Z 5f85417c f
 0001:000531b2       ?SetItem@CListCtrl@@QAEHHHIPBGHIIJ@Z 5f8541b2 f
 0001:00053200       ?SetItemState@CListCtrl@@QAEHHII@Z 5f854200 f
 0001:0005322b       ?SetItemText@CListCtrl@@QAEHHHPBG@Z 5f85422b f
 0001:00053256       ?GetItemText@CListCtrl@@QBE?AVCString@@HH@Z 5f854256 f
 0001:000532fb       ?GetItemText@CListCtrl@@QBEHHHPAGH@Z 5f8542fb f
 0001:00053340       ?GetItemData@CListCtrl@@QBEKH@Z 5f854340 f
 0001:00053382       ?DrawItem@CListCtrl@@UAEXPAUtagDRAWITEMSTRUCT@@@Z 5f854382 f
 0001:00053385       ?RemoveImageList@CListCtrl@@IAEXH@Z 5f854385 f
 0001:000533be       ?OnNcDestroy@CListCtrl@@IAEXXZ 5f8543be f
 0001:000533e3       ?CreateDragImage@CListCtrl@@QAEPAVCImageList@@HPAUtagPOINT@@@Z 5f8543e3 f
 0001:00053448       ?_GetBaseMessageMap@CTreeCtrl@@KGPBUAFX_MSGMAP@@XZ 5f854448 f
 0001:0005344e       ?GetMessageMap@CTreeCtrl@@MBEPBUAFX_MSGMAP@@XZ 5f85444e f
 0001:00053454       ?Create@CTreeCtrl@@QAEHKABUtagRECT@@PAVCWnd@@I@Z 5f854454 f
 0001:00053485       ??1CTreeCtrl@@UAE@XZ       5f854485 f
 0001:000534bd       ?GetItemRect@CTreeCtrl@@QBEHPAU_TREEITEM@@PAUtagRECT@@H@Z 5f8544bd f
 0001:000534dd       ?GetItemText@CTreeCtrl@@QBE?AVCString@@PAU_TREEITEM@@@Z 5f8544dd f
 0001:0005357d       ?GetItemImage@CTreeCtrl@@QBEHPAU_TREEITEM@@AAH1@Z 5f85457d f
 0001:000535bc       ?GetItemState@CTreeCtrl@@QBEIPAU_TREEITEM@@I@Z 5f8545bc f
 0001:000535f4       ?GetItemData@CTreeCtrl@@QBEKPAU_TREEITEM@@@Z 5f8545f4 f
 0001:00053622       ?ItemHasChildren@CTreeCtrl@@QBEHPAU_TREEITEM@@@Z 5f854622 f
 0001:00053650       ?SetItem@CTreeCtrl@@QAEHPAU_TREEITEM@@IPBGHHIIJ@Z 5f854650 f
 0001:0005369e       ?InsertItem@CTreeCtrl@@QAEPAU_TREEITEM@@IPBGHHIIJPAU2@1@Z 5f85469e f
 0001:000536f2       ?HitTest@CTreeCtrl@@QBEPAU_TREEITEM@@VCPoint@@PAI@Z 5f8546f2 f
 0001:00053728       ?RemoveImageList@CTreeCtrl@@IAEXH@Z 5f854728 f
 0001:00053761       ?OnDestroy@CTreeCtrl@@QAEXXZ 5f854761 f
 0001:0005377d       ?CreateDragImage@CTreeCtrl@@QAEPAVCImageList@@PAU_TREEITEM@@@Z 5f85477d f
 0001:000537e0       ?GetCheck@CTreeCtrl@@QBEHPAU_TREEITEM@@@Z 5f8547e0 f
 0001:00053819       ?SetCheck@CTreeCtrl@@QAEHPAU_TREEITEM@@H@Z 5f854819 f
 0001:0005385a       ?Create@CSpinButtonCtrl@@QAEHKABUtagRECT@@PAVCWnd@@I@Z 5f85485a f
 0001:00053888       ??1CSpinButtonCtrl@@UAE@XZ 5f854888 f
 0001:000538c0       ?GetRange@CSpinButtonCtrl@@QBEXAAH0@Z 5f8548c0 f
 0001:000538ec       ?Create@CSliderCtrl@@QAEHKABUtagRECT@@PAVCWnd@@I@Z 5f8548ec f
 0001:0005391d       ??1CSliderCtrl@@UAE@XZ     5f85491d f
 0001:00053955       ?GetRange@CSliderCtrl@@QBEXAAH0@Z 5f854955 f
 0001:0005398c       ?SetRange@CSliderCtrl@@QAEXHHH@Z 5f85498c f
 0001:000539bf       ?GetSelection@CSliderCtrl@@QBEXAAH0@Z 5f8549bf f
 0001:000539f6       ?SetSelection@CSliderCtrl@@QAEXHH@Z 5f8549f6 f
 0001:00053a25       ?Create@CProgressCtrl@@QAEHKABUtagRECT@@PAVCWnd@@I@Z 5f854a25 f
 0001:00053a56       ??1CProgressCtrl@@UAE@XZ   5f854a56 f
 0001:00053a8e       ?Create@CHeaderCtrl@@QAEHKABUtagRECT@@PAVCWnd@@I@Z 5f854a8e f
 0001:00053abf       ??1CHeaderCtrl@@UAE@XZ     5f854abf f
 0001:00053af7       ?OnChildNotify@CHeaderCtrl@@MAEHIIJPAJ@Z 5f854af7 f
 0001:00053b25       ?Create@CHotKeyCtrl@@QAEHKABUtagRECT@@PAVCWnd@@I@Z 5f854b25 f
 0001:00053b56       ??1CHotKeyCtrl@@UAE@XZ     5f854b56 f
 0001:00053b8e       ?GetHotKey@CHotKeyCtrl@@QBEXAAG0@Z 5f854b8e f
 0001:00053bbd       ?GetMessageMap@CTabCtrl@@MBEPBUAFX_MSGMAP@@XZ 5f854bbd f
 0001:00053bc3       ?Create@CTabCtrl@@QAEHKABUtagRECT@@PAVCWnd@@I@Z 5f854bc3 f
 0001:00053bf4       ??1CTabCtrl@@UAE@XZ        5f854bf4 f
 0001:00053c2c       ?OnDestroy@CTabCtrl@@IAEXXZ 5f854c2c f
 0001:00053c66       ?GetItemState@CTabCtrl@@QBEKHK@Z 5f854c66 f
 0001:00053c95       ?SetItemState@CTabCtrl@@QAEHHKK@Z 5f854c95 f
 0001:00053cc7       ?InsertItem@CTabCtrl@@QAEHIHPBGHJ@Z 5f854cc7 f
 0001:00053cfe       ?InsertItem@CTabCtrl@@QAEHIHPBGHJKK@Z 5f854cfe f
 0001:00053d41       ?Create@CAnimateCtrl@@QAEHKABUtagRECT@@PAVCWnd@@I@Z 5f854d41 f
 0001:00053d72       ??1CAnimateCtrl@@UAE@XZ    5f854d72 f
 0001:00053daa       ??1CRichEditCtrl@@UAE@XZ   5f854daa f
 0001:00053de2       ?afxMapHIMAGELIST@@YGPAVCHandleMap@@H@Z 5f854de2 f
 0001:00053e54       ??0CImageList@@QAE@XZ      5f854e54 f
 0001:00053e61       ?Detach@CImageList@@QAEPAU_IMAGELIST@@XZ 5f854e61 f
 0001:00053e8a       ?DeleteImageList@CImageList@@QAEHXZ 5f854e8a f
 0001:00053ea0       ?FromHandle@CImageList@@SGPAV1@PAU_IMAGELIST@@@Z 5f854ea0 f
 0001:00053eb5       ?FromHandlePermanent@CImageList@@SGPAV1@PAU_IMAGELIST@@@Z 5f854eb5 f
 0001:00053ed0       ?Create@CImageList@@QAEHHHIHH@Z 5f854ed0 f
 0001:00053ef8       ?Create@CImageList@@QAEHIHHK@Z 5f854ef8 f
 0001:00053f2c       ?Create@CImageList@@QAEHAAV1@H0HHH@Z 5f854f2c f
 0001:00053f5d       ?Attach@CImageList@@QAEHPAU_IMAGELIST@@@Z 5f854f5d f
 0001:00053f89       ?Read@CImageList@@QAEHPAVCArchive@@@Z 5f854f89 f
 0001:00053fb6       ?Write@CImageList@@QAEHPAVCArchive@@@Z 5f854fb6 f
 0001:00053fda       ?AfxGetRichEditState@@YAPAV_AFX_RICHEDIT_STATE@@XZ 5f854fda f
 0001:00053fea       ?Create@CRichEditCtrl@@QAEHKABUtagRECT@@PAVCWnd@@I@Z 5f854fea f
 0001:0005401a       ?GetLine@CRichEditCtrl@@QBEHHPAG@Z 5f85501a f
 0001:00054033       ?LineIndex@CRichEditCtrl@@QBEHH@Z 5f855033 f
 0001:0005404a       ?LineLength@CRichEditCtrl@@QBEHH@Z 5f85504a f
 0001:00054061       ?LineScroll@CRichEditCtrl@@QAEXHH@Z 5f855061 f
 0001:0005407a       ?CanPaste@CRichEditCtrl@@QBEHI@Z 5f85507a f
 0001:000540b9       ?PasteSpecial@CRichEditCtrl@@QAEXIKPAUHMETAFILE__@@@Z 5f8550b9 f
 0001:000540e3       ?GetLine@CRichEditCtrl@@QBEHHPAGH@Z 5f8550e3 f
 0001:00054103       ?GetSelText@CRichEditCtrl@@QBE?AVCString@@XZ 5f855103 f
 0001:00054169       ?SetWordCharFormat@CRichEditCtrl@@QAEHAAU_charformat@@@Z 5f855169 f
 0001:00054187       ?GetDefaultCharFormat@CRichEditCtrl@@QBEKAAU_charformat@@@Z 5f855187 f
 0001:000541a5       ?Create@CComboBoxEx@@QAEHKABUtagRECT@@PAVCWnd@@I@Z 5f8551a5 f
 0001:000541d6       ?DeleteItem@CComboBoxEx@@QAEHH@Z 5f8551d6 f
 0001:000541ed       ?GetItem@CComboBoxEx@@QAEHPAUtagCOMBOBOXEXITEMW@@@Z 5f8551ed f
 0001:00054204       ?InsertItem@CComboBoxEx@@QAEHPBUtagCOMBOBOXEXITEMW@@@Z 5f855204 f
 0001:0005421b       ?SetItem@CComboBoxEx@@QAEHPBUtagCOMBOBOXEXITEMW@@@Z 5f85521b f
 0001:00054232       ??1CComboBoxEx@@UAE@XZ     5f855232 f
 0001:0005426a       ?Create@CReBarCtrl@@QAEHKABUtagRECT@@PAVCWnd@@I@Z 5f85526a f
 0001:0005429b       ?GetImageList@CReBarCtrl@@QBEPAVCImageList@@XZ 5f85529b f
 0001:000542d5       ?SetImageList@CReBarCtrl@@QAEHPAVCImageList@@@Z 5f8552d5 f
 0001:00054313       ?GetColorScheme@CReBarCtrl@@QAEHPAUtagCOLORSCHEME@@@Z 5f855313 f
 0001:00054331       ?SetColorScheme@CReBarCtrl@@QAEXPBUtagCOLORSCHEME@@@Z 5f855331 f
 0001:0005434f       ?SetColumnOrderArray@CListCtrl@@QAEHHPAH@Z 5f85534f f
 0001:00054368       ?GetColumnOrderArray@CListCtrl@@QAEHPAHH@Z 5f855368 f
 0001:000543af       ?SetBkImage@CListCtrl@@QAEHPAUHBITMAP__@@HHH@Z 5f8553af f
 0001:000543f3       ?SetBkImage@CListCtrl@@QAEHPAGHHH@Z 5f8553f3 f
 0001:00054437       ?GetCheck@CListCtrl@@QBEHH@Z 5f855437 f
 0001:00054455       ?SetCheck@CListCtrl@@QAEHHH@Z 5f855455 f
 0001:0005448a       ?GetHeaderCtrl@CListCtrl@@QAEPAVCHeaderCtrl@@XZ 5f85548a f
 0001:000544a8       ?SetOrderArray@CHeaderCtrl@@QAEHHPAH@Z 5f8554a8 f
 0001:000544c1       ?GetOrderArray@CHeaderCtrl@@QAEHPAHH@Z 5f8554c1 f
 0001:00054500       ?GetRange@CProgressCtrl@@QAEXAAH0@Z 5f855500 f
 0001:0005452d       ?DrawIndirect@CImageList@@QAEHPAU_IMAGELISTDRAWPARAMS@@@Z 5f85552d f
 0001:00054547       ?DrawIndirect@CImageList@@QAEHPAVCDC@@HUtagPOINT@@UtagSIZE@@1IKKK@Z 5f855547 f
 0001:000545a5       ?Create@CImageList@@QAEHPAV1@@Z 5f8555a5 f
 0001:000545c1       ??0CByteArray@@QAE@XZ      5f8555c1 f
 0001:000545d8       ?SetSize@CByteArray@@QAEXHH@Z 5f8555d8 f
 0001:000546cc       ?Append@CByteArray@@QAEHABV1@@Z 5f8556cc f
 0001:00054701       ?Copy@CByteArray@@QAEXABV1@@Z 5f855701 f
 0001:00054729       ?FreeExtra@CByteArray@@QAEXXZ 5f855729 f
 0001:00054767       ?SetAtGrow@CByteArray@@QAEXHE@Z 5f855767 f
 0001:0005478e       ?InsertAt@CByteArray@@QAEXHEH@Z 5f85578e f
 0001:00054800       ?RemoveAt@CByteArray@@QAEXHH@Z 5f855800 f
 0001:00054831       ?InsertAt@CByteArray@@QAEXHPAV1@@Z 5f855831 f
 0001:00054873       ?Serialize@CByteArray@@UAEXAAVCArchive@@@Z 5f855873 f
 0001:000548d7       ?Append@CDWordArray@@QAEHABV1@@Z 5f8558d7 f
 0001:00054911       ?Copy@CDWordArray@@QAEXABV1@@Z 5f855911 f
 0001:0005493d       ?InsertAt@CDWordArray@@QAEXHPAV1@@Z 5f85593d f
 0001:00054984       ?Serialize@CDWordArray@@UAEXAAVCArchive@@@Z 5f855984 f
 0001:000549d9       ??0CObArray@@QAE@XZ        5f8559d9 f
 0001:000549f0       ??1CObArray@@UAE@XZ        5f8559f0 f
 0001:00054a27       ?FreeExtra@CObArray@@QAEXXZ 5f855a27 f
 0001:00054a6c       ?Serialize@CObArray@@UAEXAAVCArchive@@@Z 5f855a6c f
 0001:00054adc       ??0CStringArray@@QAE@XZ    5f855adc f
 0001:00054b15       ?SetSize@CStringArray@@QAEXHH@Z 5f855b15 f
 0001:00054c5c       ?Append@CStringArray@@QAEHABV1@@Z 5f855c5c f
 0001:00054cbc       ?Copy@CStringArray@@QAEXABV1@@Z 5f855cbc f
 0001:00054ce4       ?SetAtGrow@CStringArray@@QAEXHPBG@Z 5f855ce4 f
 0001:00054d10       ?SetAtGrow@CStringArray@@QAEXHABVCString@@@Z 5f855d10 f
 0001:00054d3c       ?InsertEmpty@CStringArray@@IAEXHH@Z 5f855d3c f
 0001:00054db3       ?InsertAt@CStringArray@@QAEXHPBGH@Z 5f855db3 f
 0001:00054e1a       ?InsertAt@CStringArray@@QAEXHABVCString@@H@Z 5f855e1a f
 0001:00054e53       ?RemoveAt@CStringArray@@QAEXHH@Z 5f855e53 f
 0001:00054eb0       ?InsertAt@CStringArray@@QAEXHPAV1@@Z 5f855eb0 f
 0001:00054f49       ?Serialize@CStringArray@@UAEXAAVCArchive@@@Z 5f855f49 f
 0001:00054fb2       ??0CUIntArray@@QAE@XZ      5f855fb2 f
 0001:00054fc9       ??0CWordArray@@QAE@XZ      5f855fc9 f
 0001:00054fe0       ??1CWordArray@@UAE@XZ      5f855fe0 f
 0001:00055017       ?SetSize@CWordArray@@QAEXHH@Z 5f856017 f
 0001:00055127       ?Append@CWordArray@@QAEHABV1@@Z 5f856127 f
 0001:00055160       ?Copy@CWordArray@@QAEXABV1@@Z 5f856160 f
 0001:0005518b       ?FreeExtra@CWordArray@@QAEXXZ 5f85618b f
 0001:000551ce       ?SetAtGrow@CWordArray@@QAEXHG@Z 5f8561ce f
 0001:000551f7       ?InsertAt@CWordArray@@QAEXHGH@Z 5f8561f7 f
 0001:00055284       ?RemoveAt@CWordArray@@QAEXHH@Z 5f856284 f
 0001:000552bb       ?InsertAt@CWordArray@@QAEXHPAV1@@Z 5f8562bb f
 0001:00055303       ?Serialize@CWordArray@@UAEXAAVCArchive@@@Z 5f856303 f
 0001:00055356       ?AddHead@CObList@@QAEPAU__POSITION@@PAVCObject@@@Z 5f856356 f
 0001:00055380       ?AddTail@CObList@@QAEXPAV1@@Z 5f856380 f
 0001:000553a4       ?RemoveHead@CObList@@QAEPAVCObject@@XZ 5f8563a4 f
 0001:000553c8       ?RemoveTail@CObList@@QAEPAVCObject@@XZ 5f8563c8 f
 0001:000553ec       ?InsertBefore@CObList@@QAEPAU__POSITION@@PAU2@PAVCObject@@@Z 5f8563ec f
 0001:0005542b       ?InsertAfter@CObList@@QAEPAU__POSITION@@PAU2@PAVCObject@@@Z 5f85642b f
 0001:0005546f       ?Serialize@CObList@@UAEXAAVCArchive@@@Z 5f85646f f
 0001:000554cb       ?AddHead@CPtrList@@QAEXPAV1@@Z 5f8564cb f
 0001:000554f0       ??0CStringList@@QAE@H@Z    5f8564f0 f
 0001:00055513       ?RemoveAll@CStringList@@QAEXXZ 5f856513 f
 0001:00055548       ??1CStringList@@UAE@XZ     5f856548 f
 0001:0005557b       ?NewNode@CStringList@@IAEPAUCNode@1@PAU21@0@Z 5f85657b f
 0001:000555e7       ?FreeNode@CStringList@@IAEXPAUCNode@1@@Z 5f8565e7 f
 0001:00055610       ?AddHead@CStringList@@QAEPAU__POSITION@@PBG@Z 5f856610 f
 0001:00055653       ?AddHead@CStringList@@QAEPAU__POSITION@@ABVCString@@@Z 5f856653 f
 0001:00055688       ?AddTail@CStringList@@QAEPAU__POSITION@@PBG@Z 5f856688 f
 0001:000556cb       ?AddTail@CStringList@@QAEPAU__POSITION@@ABVCString@@@Z 5f8566cb f
 0001:000556ff       ?AddHead@CStringList@@QAEXPAV1@@Z 5f8566ff f
 0001:00055725       ?AddTail@CStringList@@QAEXPAV1@@Z 5f856725 f
 0001:0005574a       ?RemoveHead@CStringList@@QAE?AVCString@@XZ 5f85674a f
 0001:000557be       ?RemoveTail@CStringList@@QAE?AVCString@@XZ 5f8567be f
 0001:00055832       ?InsertBefore@CStringList@@QAEPAU__POSITION@@PAU2@PBG@Z 5f856832 f
 0001:00055878       ?InsertBefore@CStringList@@QAEPAU__POSITION@@PAU2@ABVCString@@@Z 5f856878 f
 0001:000558c2       ?InsertAfter@CStringList@@QAEPAU__POSITION@@PAU2@PBG@Z 5f8568c2 f
 0001:00055908       ?InsertAfter@CStringList@@QAEPAU__POSITION@@PAU2@ABVCString@@@Z 5f856908 f
 0001:00055950       ?RemoveAt@CStringList@@QAEXPAU__POSITION@@@Z 5f856950 f
 0001:00055987       ?FindIndex@CStringList@@QBEPAU__POSITION@@H@Z 5f856987 f
 0001:000559ad       ?Find@CStringList@@QBEPAU__POSITION@@PBGPAU2@@Z 5f8569ad f
 0001:000559e2       ?Serialize@CStringList@@UAEXAAVCArchive@@@Z 5f8569e2 f
 0001:00055a6e       ?Lookup@CMapPtrToPtr@@QBEHPAXAAPAX@Z 5f856a6e f
 0001:00055a90       ??0CMapPtrToWord@@QAE@H@Z  5f856a90 f
 0001:00055ab7       ??1CMapPtrToWord@@UAE@XZ   5f856ab7 f
 0001:00055aea       ?NewAssoc@CMapPtrToWord@@IAEPAUCAssoc@1@XZ 5f856aea f
 0001:00055b38       ?Lookup@CMapPtrToWord@@QBEHPAXAAG@Z 5f856b38 f
 0001:00055b5c       ??ACMapPtrToWord@@QAEAAGPAX@Z 5f856b5c f
 0001:00055bac       ?GetNextAssoc@CMapPtrToWord@@QBEXAAPAU__POSITION@@AAPAXAAG@Z 5f856bac f
 0001:00055c20       ??0CMapStringToOb@@QAE@H@Z 5f856c20 f
 0001:00055c47       ??1CMapStringToOb@@UAE@XZ  5f856c47 f
 0001:00055c86       ?Serialize@CMapStringToOb@@UAEXAAVCArchive@@@Z 5f856c86 f
 0001:00055d48       ?LookupKey@CMapStringToPtr@@QBEHPBGAAPBG@Z 5f856d48 f
 0001:00055d7a       ?GetNextAssoc@CMapStringToPtr@@QBEXAAPAU__POSITION@@AAVCString@@AAPAX@Z 5f856d7a f
 0001:00055de5       ??0CMapStringToString@@QAE@H@Z 5f856de5 f
 0001:00055e0c       ?RemoveAll@CMapStringToString@@QAEXXZ 5f856e0c f
 0001:00055e66       ??1CMapStringToString@@UAE@XZ 5f856e66 f
 0001:00055e99       ?NewAssoc@CMapStringToString@@IAEPAUCAssoc@1@XZ 5f856e99 f
 0001:00055f0c       ?FreeAssoc@CMapStringToString@@IAEXPAUCAssoc@1@@Z 5f856f0c f
 0001:00055f3d       ?Lookup@CMapStringToString@@QBEHPBGAAVCString@@@Z 5f856f3d f
 0001:00055f63       ??ACMapStringToString@@QAEAAVCString@@PBG@Z 5f856f63 f
 0001:00055fc5       ?RemoveKey@CMapStringToString@@QAEHPBG@Z 5f856fc5 f
 0001:0005602c       ?GetNextAssoc@CMapStringToString@@QBEXAAPAU__POSITION@@AAVCString@@1@Z 5f85702c f
 0001:0005609b       ?Serialize@CMapStringToString@@UAEXAAVCArchive@@@Z 5f85709b f
 0001:00056178       ??0CMapWordToOb@@QAE@H@Z   5f857178 f
 0001:000561af       ??1CMapWordToOb@@UAE@XZ    5f8571af f
 0001:000561e2       ?NewAssoc@CMapWordToOb@@IAEPAUCAssoc@1@XZ 5f8571e2 f
 0001:00056230       ??ACMapWordToOb@@QAEAAPAVCObject@@G@Z 5f857230 f
 0001:00056281       ?Serialize@CMapWordToOb@@UAEXAAVCArchive@@@Z 5f857281 f
 0001:0005631a       ??0CMapWordToPtr@@QAE@H@Z  5f85731a f
 0001:00056341       ??1CMapWordToPtr@@UAE@XZ   5f857341 f
 0001:00056374       ?GetAssocAt@CMapWordToPtr@@IBEPAUCAssoc@1@GAAI@Z 5f857374 f
 0001:000563a9       ?Lookup@CMapWordToPtr@@QBEHGAAPAX@Z 5f8573a9 f
 0001:000563cb       ?RemoveKey@CMapWordToPtr@@QAEHG@Z 5f8573cb f
 0001:00056410       ?GetNextAssoc@CMapWordToPtr@@QBEXAAPAU__POSITION@@AAGAAPAX@Z 5f857410 f
 0001:00056485       ?GetRuntimeClass@CObject@@UBEPAUCRuntimeClass@@XZ 5f857485 f
 0001:0005649c       ?IsSerializable@CObject@@QBEHXZ 5f85749c f
 0001:000564af       ??0AFX_CLASSINIT_COMPAT@@QAE@PAUCRuntimeClass@@@Z 5f8574af f
 0001:000564db       ?Delete@CException@@QAEXXZ 5f8574db f
 0001:000564ed       ?GetErrorMessage@CException@@UAEHPAGIPAI@Z 5f8574ed f
 0001:0005650f       ?ReportError@CException@@UAEHII@Z 5f85750f f
 0001:0005656e       ?AfxThrowLastCleanup@@YGXXZ 5f85756e f
 0001:0005657e       ?AfxNewHandler@@YAHI@Z     5f85757e f
 0001:00056586       ?AfxGetNewHandler@@YGP6AHI@ZXZ 5f857586 f
 0001:000565b9       ?IsDirSep@@YAHG@Z          5f8575b9 f
 0001:000565d0       ??0CFile@@QAE@H@Z          5f8575d0 f
 0001:00056614       ??0CFile@@QAE@PBGI@Z       5f857614 f
 0001:000566be       ?Duplicate@CFile@@UBEPAV1@XZ 5f8576be f
 0001:000567e2       ?Write@CFile@@UAEXPBXI@Z   5f8577e2 f
 0001:00056853       ?Flush@CFile@@UAEXXZ       5f857853 f
 0001:00056887       ?Abort@CFile@@UAEXXZ       5f857887 f
 0001:000568a7       ?LockRange@CFile@@UAEXKK@Z 5f8578a7 f
 0001:000568d0       ?UnlockRange@CFile@@UAEXKK@Z 5f8578d0 f
 0001:000568f9       ?SetLength@CFile@@UAEXK@Z  5f8578f9 f
 0001:00056925       ?Rename@CFile@@SGXPBG0@Z   5f857925 f
 0001:00056947       ?Remove@CFile@@SGXPBG@Z    5f857947 f
 0001:00056965       ?CreateInstance@AFX_COM@@QAEJABU_GUID@@PAUIUnknown@@0PAPAX@Z 5f857965 f
 0001:000569a7       ?GetClassObject@AFX_COM@@QAEJABU_GUID@@0PAPAX@Z 5f8579a7 f
 0001:00056a44       ?AfxStringFromCLSID@@YG?AVCString@@ABU_GUID@@@Z 5f857a44 f
 0001:00056ab3       ?AfxGetInProcServer@@YGHPBGAAVCString@@@Z 5f857ab3 f
 0001:00056d71       ??0CStdioFile@@QAE@XZ      5f857d71 f
 0001:00056d87       ??0CStdioFile@@QAE@PAU_iobuf@@@Z 5f857d87 f
 0001:00056db1       ??0CStdioFile@@QAE@PBGI@Z  5f857db1 f
 0001:00056e4e       ?Open@CStdioFile@@UAEHPBGIPAVCFileException@@@Z 5f857e4e f
 0001:00056f40       ?Read@CStdioFile@@UAEIPAXI@Z 5f857f40 f
 0001:00056fb0       ?Write@CStdioFile@@UAEXPBXI@Z 5f857fb0 f
 0001:00056fe5       ?WriteString@CStdioFile@@UAEXPBG@Z 5f857fe5 f
 0001:00057014       ?ReadString@CStdioFile@@UAEPAGPAGI@Z 5f858014 f
 0001:0005705c       ?ReadString@CStdioFile@@UAEHAAVCString@@@Z 5f85805c f
 0001:00057128       ?Seek@CStdioFile@@UAEJJI@Z 5f858128 f
 0001:00057163       ?GetPosition@CStdioFile@@UBEKXZ 5f858163 f
 0001:0005718f       ?Flush@CStdioFile@@UAEXXZ  5f85818f f
 0001:000571b9       ?Close@CStdioFile@@UAEXXZ  5f8581b9 f
 0001:000571f1       ?Abort@CStdioFile@@UAEXXZ  5f8581f1 f
 0001:00057217       ?Duplicate@CStdioFile@@UBEPAVCFile@@XZ 5f858217 f
 0001:0005721f       ?UnlockRange@CStdioFile@@UAEXKK@Z 5f85821f f
 0001:00057227       ?ThrowOsError@CFileException@@SGXJPBG@Z 5f858227 f
 0001:00057248       ?ThrowErrno@CFileException@@SGXHPBG@Z 5f858248 f
 0001:0005726d       ?GetErrorMessage@CFileException@@UAEHPAGIPAI@Z 5f85826d f
 0001:0005730d       ?AfxThrowFileException@@YGXHJPBG@Z 5f85830d f
 0001:0005737c       ?ErrnoToException@CFileException@@SGHH@Z 5f85837c f
 0001:000573d4       ?OsErrorToException@CFileException@@SGHJ@Z 5f8583d4 f
 0001:0005764f       ?GetFileName@CFile@@UBE?AVCString@@XZ 5f85864f f
 0001:000576e0       ?GetFileTitle@CFile@@UBE?AVCString@@XZ 5f8586e0 f
 0001:00057793       ?GetStatus@CFile@@SGHPBGAAUCFileStatus@@@Z 5f858793 f
 0001:00057847       ?AfxTimeToFileTime@@YAXABVCTime@@PAU_FILETIME@@@Z 5f858847 f
 0001:000578fa       ?SetStatus@CFile@@SGXPBGABUCFileStatus@@@Z 5f8588fa f
 0001:00057a27       ?GetStatus@CMemFile@@QBEHAAUCFileStatus@@@Z 5f858a27 f
 0001:00057aa3       ?AllocCopy@CString@@IBEXAAV1@HHH@Z 5f858aa3 f
 0001:00057b1c       ??H@YG?AVCString@@ABV0@PBG@Z 5f858b1c f
 0001:00057b90       ??H@YG?AVCString@@PBGABV0@@Z 5f858b90 f
 0001:00057c0b       ??YCString@@QAEABV0@G@Z    5f858c0b f
 0001:00057c27       ?FreeExtra@CString@@QAEXXZ 5f858c27 f
 0001:00057c5d       ?LockBuffer@CString@@QAEPAGXZ 5f858c5d f
 0001:00057c6f       ?UnlockBuffer@CString@@QAEXXZ 5f858c6f f
 0001:00057ca5       ?FindOneOf@CString@@QBEHPBG@Z 5f858ca5 f
 0001:00057cc8       ?MakeUpper@CString@@QAEXXZ 5f858cc8 f
 0001:00057cdb       ?MakeLower@CString@@QAEXXZ 5f858cdb f
 0001:00057cee       ?MakeReverse@CString@@QAEXXZ 5f858cee f
 0001:00057d01       ?SetAt@CString@@QAEXHG@Z   5f858d01 f
 0001:00057d1c       ?_wcstombsz@@YAHPADPBGI@Z  5f858d1c f
 0001:00057f02       ?_AfxGrayBackgroundWndProc@@YGJPAUHWND__@@IIJ@Z 5f858f02 f
 0001:00057fff       ?CreateEx@CWnd@@QAEHKPBG0KABUtagRECT@@PAV1@IPAX@Z 5f858fff f
 0001:00058191       ?OnToolHitTest@CWnd@@UBEHVCPoint@@PAUtagTOOLINFOW@@@Z 5f859191 f
 0001:00058213       ?GetDlgItemTextW@CWnd@@QBEHHAAVCString@@@Z 5f859213 f
 0001:00058283       ?SetWindowPlacement@CWnd@@QAEHPBUtagWINDOWPLACEMENT@@@Z 5f859283 f
 0001:000582bf       ?OnCompareItem@CWnd@@IAEHHPAUtagCOMPAREITEMSTRUCT@@@Z 5f8592bf f
 0001:000582e9       ?OnVKeyToItem@CWnd@@IAEHIPAVCListBox@@I@Z 5f8592e9 f
 0001:00058314       ?TrackPopupMenu@CMenu@@QAEHIHHPAVCWnd@@PBUtagRECT@@@Z 5f859314 f
 0001:00058368       ?_AfxFindPopupMenuFromID@@YGPAVCMenu@@PAV1@I@Z 5f859368 f
 0001:0005849f       ?WinHelpW@CWnd@@UAEXKI@Z   5f85949f f
 0001:0005870f       ?GetTopLevelOwner@CWnd@@QBEPAV1@XZ 5f85970f f
 0001:0005873f       ?GetParentOwner@CWnd@@QBEPAV1@XZ 5f85973f f
 0001:00058783       ?ActivateTopParent@CWnd@@QAEXXZ 5f859783 f
 0001:000587c4       ?GetSafeOwner@CWnd@@SGPAV1@PAV1@PAPAUHWND__@@@Z 5f8597c4 f
 0001:000587e2       ?MessageBoxW@CWnd@@QAEHPBG0I@Z 5f8597e2 f
 0001:00058832       ?SetScrollRange@CWnd@@QAEXHHHH@Z 5f859832 f
 0001:00058865       ?GetScrollRange@CWnd@@QBEXHPAH0@Z 5f859865 f
 0001:000588b4       ?SetScrollInfo@CWnd@@QAEHHPAUtagSCROLLINFO@@H@Z 5f8598b4 f
 0001:00058901       ?GetScrollInfo@CWnd@@QAEHHPAUtagSCROLLINFO@@I@Z 5f859901 f
 0001:0005894e       ?GetScrollLimit@CWnd@@QAEHH@Z 5f85994e f
 0001:00058a67       ?HandleFloatingSysCommand@CWnd@@QAEHIJ@Z 5f859a67 f
 0001:00058bcb       ?OnSysColorChange@CWnd@@IAEXXZ 5f859bcb f
 0001:00058c48       ?OnSettingChange@CWnd@@IAEXIPBG@Z 5f859c48 f
 0001:00058c9b       ?OnWinIniChange@CWnd@@IAEXPBG@Z 5f859c9b f
 0001:00058ce7       ?OnDevModeChange@CWnd@@IAEXPAG@Z 5f859ce7 f
 0001:00058d32       ?OnHelpInfo@CWnd@@IAEHPAUtagHELPINFO@@@Z 5f859d32 f
 0001:00058d96       ?OnDisplayChange@CWnd@@IAEJIJ@Z 5f859d96 f
 0001:00058ddf       ?OnDragList@CWnd@@IAEJIJ@Z 5f859ddf f
 0001:00058e09       ?OnVScroll@CWnd@@IAEXIIPAVCScrollBar@@@Z 5f859e09 f
 0001:00058ebf       ?OnQuery3dControls@CWnd@@IAEJIJ@Z 5f859ebf f
 0001:00059244       ?SubclassCtl3d@CWnd@@QAEHH@Z 5f85a244 f
 0001:0005928e       ?SubclassDlg3d@CWnd@@QAEHK@Z 5f85a28e f
 0001:00059308       ?UnsubclassWindow@CWnd@@QAEPAUHWND__@@XZ 5f85a308 f
 0001:00059330       ??3CTempWnd@@SAXPAX@Z      5f85a330 f
 0001:0005938f       ?DeleteTempMap@CWnd@@SGXXZ 5f85a38f f
 0001:0005939c       ?DeleteTempMap@CImageList@@SGXXZ 5f85a39c f
 0001:000593a9       ?DeleteTempMap@CDC@@SGXXZ  5f85a3a9 f
 0001:000593b6       ?DeleteTempMap@CGdiObject@@SGXXZ 5f85a3b6 f
 0001:000593c3       ?DeleteTempMap@CMenu@@SGXXZ 5f85a3c3 f
 0001:000594ba       ?CreateIndirect@CDialog@@QAEHPAXPAVCWnd@@@Z 5f85a4ba f
 0001:000594cc       ?CreateIndirect@CDialog@@QAEHPBUDLGTEMPLATE@@PAVCWnd@@PAX@Z 5f85a4cc f
 0001:000594e2       ?CreateDlg@CWnd@@IAEHPBGPAV1@@Z 5f85a4e2 f
 0001:0005952b       ?CreateDlgIndirect@CWnd@@IAEHPBUDLGTEMPLATE@@PAV1@@Z 5f85a52b f
 0001:0005968e       ?SetOccDialogInfo@CDialog@@MAEHPAU_AFX_OCC_DIALOG_INFO@@@Z 5f85a68e f
 0001:0005969b       ??0CDialog@@QAE@PBGPAVCWnd@@@Z 5f85a69b f
 0001:000596dd       ?InitModalIndirect@CDialog@@QAEHPAXPAVCWnd@@@Z 5f85a6dd f
 0001:000596f7       ?InitModalIndirect@CDialog@@QAEHPBUDLGTEMPLATE@@PAVCWnd@@PAX@Z 5f85a6f7 f
 0001:0005981a       ?AfxHelpEnabled@@YGHXZ     5f85a81a f
 0001:000598a1       ?OnCancel@CDialog@@MAEXXZ  5f85a8a1 f
 0001:000598ca       ?OnCommandHelp@CDialog@@IAEJIJ@Z 5f85a8ca f
 0001:00059908       ?OnHelpHitTest@CDialog@@IAEJIJ@Z 5f85a908 f
 0001:0005991b       ?_AfxConvertDialogUnitsToPixels@@YGXPBGGHHPAUtagSIZE@@@Z 5f85a91b f
 0001:00059a2b       ?IsDialogEx@@YAHPBUDLGTEMPLATE@@@Z 5f85aa2b f
 0001:00059a3b       ?HasFont@@YAHPBUDLGTEMPLATE@@@Z 5f85aa3b f
 0001:00059a52       ?FontAttrSize@@YAHH@Z      5f85aa52 f
 0001:00059a61       ??0CDialogTemplate@@QAE@PBUDLGTEMPLATE@@@Z 5f85aa61 f
 0001:00059a90       ??0CDialogTemplate@@QAE@PAX@Z 5f85aa90 f
 0001:00059ad1       ?SetTemplate@CDialogTemplate@@IAEHPBUDLGTEMPLATE@@I@Z 5f85aad1 f
 0001:00059b31       ?Load@CDialogTemplate@@QAEHPBG@Z 5f85ab31 f
 0001:00059b8b       ?Detach@CDialogTemplate@@QAEPAXXZ 5f85ab8b f
 0001:00059b91       ?HasFont@CDialogTemplate@@QBEHXZ 5f85ab91 f
 0001:00059be4       ?GetTemplateSize@CDialogTemplate@@KAIPBUDLGTEMPLATE@@@Z 5f85abe4 f
 0001:00059ca7       ?GetFont@CDialogTemplate@@QBEHAAVCString@@AAG@Z 5f85aca7 f
 0001:00059cd5       ?SetFont@CDialogTemplate@@QAEHPBGG@Z 5f85acd5 f
 0001:00059df6       ?SetSystemFont@CDialogTemplate@@QAEHG@Z 5f85adf6 f
 0001:00059e87       ?GetSizeInDialogUnits@CDialogTemplate@@QBEXPAUtagSIZE@@@Z 5f85ae87 f
 0001:00059ec7       ?GetSizeInPixels@CDialogTemplate@@QBEXPAUtagSIZE@@@Z 5f85aec7 f
 0001:00059fba       ?FromHandlePermanent@CMenu@@SGPAV1@PAUHMENU__@@@Z 5f85afba f
 0001:00059fd5       ?Attach@CMenu@@QAEHPAUHMENU__@@@Z 5f85afd5 f
 0001:0005a001       ?Detach@CMenu@@QAEPAUHMENU__@@XZ 5f85b001 f
 0001:0005a041       ?OnAmbientProperty@CWnd@@UAEHPAVCOleControlSite@@JPAUtagVARIANT@@@Z 5f85b041 f
 0001:0005a058       ?GetControlUnknown@CWnd@@QAEPAUIUnknown@@XZ 5f85b058 f
 0001:0005a064       ?CheckDlgButton@CWnd@@QAEXHI@Z 5f85b064 f
 0001:0005a090       ?CheckRadioButton@CWnd@@QAEXHHH@Z 5f85b090 f
 0001:0005a0e6       ?GetDlgItemInt@CWnd@@QBEIHPAHH@Z 5f85b0e6 f
 0001:0005a118       ?GetDlgItemTextW@CWnd@@QBEHHPAGH@Z 5f85b118 f
 0001:0005a14d       ?SendDlgItemMessageW@CWnd@@QAEJHIIJ@Z 5f85b14d f
 0001:0005a188       ?SetDlgItemInt@CWnd@@QAEXHIH@Z 5f85b188 f
 0001:0005a1d4       ?IsDlgButtonChecked@CWnd@@QBEIH@Z 5f85b1d4 f
 0001:0005a1fb       ?ScrollWindowEx@CWnd@@QAEHHHPBUtagRECT@@0PAVCRgn@@PAU2@I@Z 5f85b1fb f
 0001:0005a2ce       ?GetWindowTextLengthW@CWnd@@QBEHXZ 5f85b2ce f
 0001:0005a2f3       ?SetDlgCtrlID@CWnd@@QAEHH@Z 5f85b2f3 f
 0001:0005a31c       ?MoveWindow@CWnd@@QAEXHHHHH@Z 5f85b31c f
 0001:0005a3b8       ?InvokeHelper@CWnd@@QAAXJGGPAXPBEZZ 5f85b3b8 f
 0001:0005a3df       ?GetProperty@CWnd@@QBEXJGPAX@Z 5f85b3df f
 0001:0005a401       ?SetProperty@CWnd@@QAAXJGZZ 5f85b401 f
 0001:0005a41f       ?GetDSCCursor@CWnd@@QAEPAUIUnknown@@XZ 5f85b41f f
 0001:0005a444       ?BindDefaultProperty@CWnd@@QAEXJGPBGPAV1@@Z 5f85b444 f
 0001:0005a462       ?BindProperty@CWnd@@QAEXJPAV1@@Z 5f85b462 f
 0001:0005a485       ?AttachControlSite@CWnd@@QAEXPAV1@@Z 5f85b485 f
 0001:0005a4a1       ?AttachControlSite@COleControlContainer@@QAEXPAVCWnd@@@Z 5f85b4a1 f
 0001:0005a5fc       ?GetTypeLib@CCmdTarget@@UAEJKPAPAUITypeLib@@@Z 5f85b5fc f
 0001:0005a604       ?RestoreWaitCursor@CCmdTarget@@QAEXXZ 5f85b604 f
 0001:0005a619       ?GetDispatchMap@CCmdTarget@@MBEPBUAFX_DISPMAP@@XZ 5f85b619 f
 0001:0005a61f       ?GetEventSinkMap@CCmdTarget@@MBEPBUAFX_EVENTSINKMAP@@XZ 5f85b61f f
 0001:0005a625       ?OnFinalRelease@CCmdTarget@@UAEXXZ 5f85b625 f
 0001:0005a657       ?GetConnectionMap@CCmdTarget@@MBEPBUAFX_CONNECTIONMAP@@XZ 5f85b657 f
 0001:0005a65d       ?GetCommandMap@CCmdTarget@@MBEPBUAFX_OLECMDMAP@@XZ 5f85b65d f
 0001:0005a663       ?GetRoutingView@CCmdTarget@@IAEPAVCView@@XZ 5f85b663 f
 0001:0005a663       ?GetRoutingView_@CCmdTarget@@KGPAVCView@@XZ 5f85b663 f
 0001:0005a66f       ?GetRoutingFrame@CCmdTarget@@IAEPAVCFrameWnd@@XZ 5f85b66f f
 0001:0005a6ce       ?SetCheck@CCmdUI@@UAEXH@Z  5f85b6ce f
 0001:0005a730       ?SetRadio@CCmdUI@@UAEXH@Z  5f85b730 f
 0001:0005a82b       ?AfxBeginThread@@YGPAVCWinThread@@PAUCRuntimeClass@@HIKPAU_SECURITY_ATTRIBUTES@@@Z 5f85b82b f
 0001:0005a8fb       ?ExitInstance@CWinThread@@UAEHXZ 5f85b8fb f
 0001:0005a92a       ?DispatchThreadMessage@CWinThread@@IAEXPAUtagMSG@@@Z 5f85b92a f
 0001:0005a936       ?DispatchThreadMessageEx@CWinThread@@IAEHPAUtagMSG@@@Z 5f85b936 f
 0001:0005a9c4       ?ProcessWndProcException@CWinThread@@UAEJPAVCException@@PBUtagMSG@@@Z 5f85b9c4 f
 0001:0005aa1b       ?IsHelpKey@@YGHPAUtagMSG@@@Z 5f85ba1b f
 0001:0005aa66       ?IsEnterKey@@YAHPAUtagMSG@@@Z 5f85ba66 f
 0001:0005aa80       ?IsButtonUp@@YAHPAUtagMSG@@@Z 5f85ba80 f
 0001:0005ab8a       ?GetMessageMap@CWinApp@@MBEPBUAFX_MSGMAP@@XZ 5f85bb8a f
 0001:0005ab9c       ?WinHelpW@CWinApp@@UAEXKI@Z 5f85bb9c f
 0001:0005abd3       ?ProcessWndProcException@CWinApp@@UAEJPAVCException@@PBUtagMSG@@@Z 5f85bbd3 f
 0001:0005ac4a       ?DevModeChange@CWinApp@@QAEXPAG@Z 5f85bc4a f
 0001:0005adcc       ?Remove@CRecentFileList@@UAEXH@Z 5f85bdcc f
 0001:0005ae11       ?_GetBaseClass@COleControlModule@@KGPAUCRuntimeClass@@XZ 5f85be11 f
 0001:0005ae17       ?GetRuntimeClass@COleControlModule@@UBEPAUCRuntimeClass@@XZ 5f85be17 f
 0001:0005ae1d       ?InitInstance@COleControlModule@@UAEHXZ 5f85be1d f
 0001:0005ae26       ?ExitInstance@COleControlModule@@UAEHXZ 5f85be26 f
 0001:0005ae37       ??6@YGAAVCArchive@@AAV0@ABVCString@@@Z 5f85be37 f
 0001:0005aec5       ?_AfxReadStringLength@@YGIAAVCArchive@@@Z 5f85bec5 f
 0001:0005af1c       ??5@YGAAVCArchive@@AAV0@AAVCString@@@Z 5f85bf1c f
 0001:0005afad       ?SerializeElements@@YGXAAVCArchive@@PAVCString@@H@Z 5f85bfad f
 0001:0005affb       ?Load@CRuntimeClass@@SGPAU1@AAVCArchive@@PAI@Z 5f85bffb f
 0001:0005b0c4       ?Store@CRuntimeClass@@QBEXAAVCArchive@@@Z 5f85c0c4 f
 0001:0005b30a       ?WriteCount@CArchive@@QAEXK@Z 5f85c30a f
 0001:0005b338       ?ReadCount@CArchive@@QAEKXZ 5f85c338 f
 0001:0005b368       ?WriteString@CArchive@@QAEXPBG@Z 5f85c368 f
 0001:0005b387       ?ReadString@CArchive@@QAEPAGPAGI@Z 5f85c387 f
 0001:0005b442       ?ReadString@CArchive@@QAEHAAVCString@@@Z 5f85c442 f
 0001:0005b4de       ?CheckCount@CArchive@@QAEXXZ 5f85c4de f
 0001:0005b4f2       ?WriteObject@CArchive@@QAEXPBVCObject@@@Z 5f85c4f2 f
 0001:0005b571       ?ReadObject@CArchive@@QAEPAVCObject@@PBUCRuntimeClass@@@Z 5f85c571 f
 0001:0005b620       ?GetObjectSchema@CArchive@@QAEIXZ 5f85c620 f
 0001:0005b628       ?MapObject@CArchive@@QAEXPBVCObject@@@Z 5f85c628 f
 0001:0005b720       ?WriteClass@CArchive@@QAEXPBUCRuntimeClass@@@Z 5f85c720 f
 0001:0005b7b1       ?ReadClass@CArchive@@QAEPAUCRuntimeClass@@PBU2@PAIPAK@Z 5f85c7b1 f
 0001:0005b98c       ?SerializeClass@CArchive@@QAEXPBUCRuntimeClass@@@Z 5f85c98c f
 0001:0005b9b0       ?GetErrorMessage@CArchiveException@@UAEHPAGIPAI@Z 5f85c9b0 f
 0001:0005ba50       ?AfxThrowArchiveException@@YGXHPBG@Z 5f85ca50 f
 0001:0005badd       ?SetOutputDC@CDC@@UAEXPAUHDC__@@@Z 5f85cadd f
 0001:0005bae7       ?ReleaseOutputDC@CDC@@UAEXXZ 5f85cae7 f
 0001:0005baec       ?StartDocW@CDC@@QAEHPBG@Z  5f85caec f
 0001:0005bb4a       ?SelectStockObject@CDC@@UAEPAVCGdiObject@@H@Z 5f85cb4a f
 0001:0005bb9d       ?SelectObject@CDC@@QAEHPAVCRgn@@@Z 5f85cb9d f
 0001:0005bbe2       ?SelectPalette@CDC@@QAEPAVCPalette@@PAV2@H@Z 5f85cbe2 f
 0001:0005bc04       ?SetBkColor@CDC@@UAEKK@Z   5f85cc04 f
 0001:0005bc3f       ?SetPolyFillMode@CDC@@QAEHH@Z 5f85cc3f f
 0001:0005bc6d       ?SetROP2@CDC@@QAEHH@Z      5f85cc6d f
 0001:0005bc9b       ?SetStretchBltMode@CDC@@QAEHH@Z 5f85cc9b f
 0001:0005bcf3       ?OffsetViewportOrg@CDC@@UAE?AVCPoint@@HH@Z 5f85ccf3 f
 0001:0005bd51       ?ScaleViewportExt@CDC@@UAE?AVCSize@@HHHH@Z 5f85cd51 f
 0001:0005bda9       ?SetWindowOrg@CDC@@QAE?AVCPoint@@HH@Z 5f85cda9 f
 0001:0005bdf5       ?OffsetWindowOrg@CDC@@QAE?AVCPoint@@HH@Z 5f85cdf5 f
 0001:0005be53       ?ScaleWindowExt@CDC@@UAE?AVCSize@@HHHH@Z 5f85ce53 f
 0001:0005beab       ?GetClipBox@CDC@@UBEHPAUtagRECT@@@Z 5f85ceab f
 0001:0005bebb       ?SelectClipRgn@CDC@@QAEHPAVCRgn@@@Z 5f85cebb f
 0001:0005befb       ?ExcludeClipRect@CDC@@QAEHHHHH@Z 5f85cefb f
 0001:0005bf77       ?OffsetClipRgn@CDC@@QAEHHH@Z 5f85cf77 f
 0001:0005bfd5       ?SetTextAlign@CDC@@QAEII@Z 5f85cfd5 f
 0001:0005c00a       ?SetTextJustification@CDC@@QAEHHH@Z 5f85d00a f
 0001:0005c040       ?SetTextCharacterExtra@CDC@@QAEHH@Z 5f85d040 f
 0001:0005c071       ?SetMapperFlags@CDC@@QAEKK@Z 5f85d071 f
 0001:0005c0a0       ?GetLayout@CDC@@QBEKXZ     5f85d0a0 f
 0001:0005c0d6       ?SetLayout@CDC@@QAEKK@Z    5f85d0d6 f
 0001:0005c136       ?ArcTo@CDC@@QAEHHHHHHHHH@Z 5f85d136 f
 0001:0005c18e       ?SetArcDirection@CDC@@QAEHH@Z 5f85d18e f
 0001:0005c1bc       ?PolyDraw@CDC@@QAEHPBUtagPOINT@@PBEH@Z 5f85d1bc f
 0001:0005c205       ?PolylineTo@CDC@@QAEHPBUtagPOINT@@H@Z 5f85d205 f
 0001:0005c24b       ?SetColorAdjustment@CDC@@QAEHPBUtagCOLORADJUSTMENT@@@Z 5f85d24b f
 0001:0005c279       ?PolyBezierTo@CDC@@QAEHPBUtagPOINT@@H@Z 5f85d279 f
 0001:0005c2bf       ?SelectClipPath@CDC@@QAEHH@Z 5f85d2bf f
 0001:0005c31d       ?SelectClipRgn@CDC@@QAEHPAVCRgn@@H@Z 5f85d31d f
 0001:0005c365       ?AfxEnumMetaFileProc@@YGHPAUHDC__@@PAUtagHANDLETABLE@@PAUtagMETARECORD@@HJ@Z 5f85d365 f
 0001:0005c5a5       ?PlayMetaFile@CDC@@QAEHPAUHMETAFILE__@@@Z 5f85d5a5 f
 0001:0005c5de       ?DPtoLP@CDC@@QBEXPAUtagSIZE@@@Z 5f85d5de f
 0001:0005c651       ??_GCClientDC@@UAEPAXI@Z   5f85d651 f
 0001:0005c651       ??_ECClientDC@@UAEPAXI@Z   5f85d651 f
 0001:0005c677       ??_GCWindowDC@@UAEPAXI@Z   5f85d677 f
 0001:0005c677       ??_ECWindowDC@@UAEPAXI@Z   5f85d677 f
 0001:0005c69d       ??_GCPaintDC@@UAEPAXI@Z    5f85d69d f
 0001:0005c69d       ??_ECPaintDC@@UAEPAXI@Z    5f85d69d f
 0001:0005c6c7       ??0CPen@@QAE@HHK@Z         5f85d6c7 f
 0001:0005c717       ??0CPen@@QAE@HHPBUtagLOGBRUSH@@HPBK@Z 5f85d717 f
 0001:0005c76d       ??0CBrush@@QAE@K@Z         5f85d76d f
 0001:0005c7b7       ??0CBrush@@QAE@HK@Z        5f85d7b7 f
 0001:0005c804       ??0CBrush@@QAE@PAVCBitmap@@@Z 5f85d804 f
 0001:0005c851       ?CreateDIBPatternBrush@CBrush@@QAEHPAXI@Z 5f85d851 f
 0001:0005c883       ?AfxThrowResourceException@@YGXXZ 5f85d883 f
 0001:0005c89c       ?AfxThrowUserException@@YGXXZ 5f85d89c f
 0001:0005c8b5       ?AfxCustomLogFont@@YGHIPAUtagLOGFONTW@@@Z 5f85d8b5 f
 0001:0005c958       ?_AfxCompareClassName@@YGHPAUHWND__@@PBG@Z 5f85d958 f
 0001:0005c983       ?_AfxChildWindowFromPoint@@YGPAUHWND__@@PAU1@UtagPOINT@@@Z 5f85d983 f
 0001:0005ca34       ?AfxCriticalNewHandler@@YAHI@Z 5f85da34 f
 0001:0005ca89       ?GetMessageMap@CDocument@@MBEPBUAFX_MSGMAP@@XZ 5f85da89 f
 0001:0005ca8f       ??_GCDocument@@UAEPAXI@Z   5f85da8f f
 0001:0005ca8f       ??_ECDocument@@UAEPAXI@Z   5f85da8f f
 0001:0005caab       ?OnFinalRelease@CDocument@@UAEXXZ 5f85daab f
 0001:0005cace       ?DeleteContents@CDocument@@UAEXXZ 5f85dace f
 0001:0005cadf       ?PreCloseFrame@CDocument@@UAEXPAVCFrameWnd@@@Z 5f85dadf f
 0001:0005cae2       ?OnFileClose@CDocument@@IAEXXZ 5f85dae2 f
 0001:0005cafd       ?OnFileSave@CDocument@@IAEXXZ 5f85dafd f
 0001:0005cb05       ?OnFileSaveAs@CDocument@@IAEXXZ 5f85db05 f
 0001:0005cb12       ?DoFileSave@CDocument@@UAEHXZ 5f85db12 f
 0001:0005cb4d       ?DoSave@CDocument@@UAEHPBGH@Z 5f85db4d f
 0001:0005cdb2       ?GetDefaultMenu@CDocument@@UAEPAUHMENU__@@XZ 5f85ddb2 f
 0001:0005cdb5       ?ReportSaveLoadException@CDocument@@UAEXPBGPAVCException@@HI@Z 5f85ddb5 f
 0001:0005cf1a       ?GetTempName@CMirrorFile@@SA?AVCString@@PBGH@Z 5f85df1a f
 0001:0005cfc1       ?Open@CMirrorFile@@UAEHPBGIPAVCFileException@@@Z 5f85dfc1 f
 0001:0005d173       ?Abort@CMirrorFile@@UAEXXZ 5f85e173 f
 0001:0005d18c       ?Close@CMirrorFile@@UAEXXZ 5f85e18c f
 0001:0005d29d       ?GetFile@CDocument@@UAEPAVCFile@@PBGIPAVCFileException@@@Z 5f85e29d f
 0001:0005d313       ??1CMirrorFile@@UAE@XZ     5f85e313 f
 0001:0005d3ef       ?OnSaveDocument@CDocument@@UAEHPBG@Z 5f85e3ef f
 0001:0005d5ae       ?UpdateAllViews@CDocument@@QAEXPAVCView@@JPAVCObject@@@Z 5f85e5ae f
 0001:0005d5ef       ?SendInitialUpdate@CDocument@@QAEXXZ 5f85e5ef f
 0001:0005d62e       ??_GCDocTemplate@@UAEPAXI@Z 5f85e62e f
 0001:0005d62e       ??_ECDocTemplate@@UAEPAXI@Z 5f85e62e f
 0001:0005d669       ?CreateOleFrame@CDocTemplate@@QAEPAVCFrameWnd@@PAVCWnd@@PAVCDocument@@H@Z 5f85e669 f
 0001:0005d703       ??_GCSingleDocTemplate@@UAEPAXI@Z 5f85e703 f
 0001:0005d703       ??_ECSingleDocTemplate@@UAEPAXI@Z 5f85e703 f
 0001:0005d7c1       ??_ECMultiDocTemplate@@UAEPAXI@Z 5f85e7c1 f
 0001:0005d7c1       ??_GCMultiDocTemplate@@UAEPAXI@Z 5f85e7c1 f
 0001:0005d91b       ?GetOpenDocumentCount@CDocManager@@UAEHXZ 5f85e91b f
 0001:0005d961       ??_ECView@@UAEPAXI@Z       5f85e961 f
 0001:0005d961       ??_GCView@@UAEPAXI@Z       5f85e961 f
 0001:0005d9dd       ?OnPrint@CView@@MAEXPAVCDC@@PAUCPrintInfo@@@Z 5f85e9dd f
 0001:0005d9ec       ?IsSelected@CView@@UBEHPBVCObject@@@Z 5f85e9ec f
 0001:0005d9f1       ?OnMouseActivate@CView@@IAEHPAVCWnd@@II@Z 5f85e9f1 f
 0001:0005da62       ?OnScroll@CView@@UAEHIIH@Z 5f85ea62 f
 0001:0005da67       ?OnDragScroll@CView@@UAEKKVCPoint@@@Z 5f85ea67 f
 0001:0005da6f       ?OnDragEnter@CView@@UAEKPAVCOleDataObject@@KVCPoint@@@Z 5f85ea6f f
 0001:0005da74       ?OnDropEx@CView@@UAEKPAVCOleDataObject@@KKVCPoint@@@Z 5f85ea74 f
 0001:0005daf9       ?OnUpdateSplitCmd@CView@@IAEXPAVCCmdUI@@@Z 5f85eaf9 f
 0001:0005db21       ?OnSplitCmd@CView@@IAEHI@Z 5f85eb21 f
 0001:0005db3d       ?OnUpdateNextPaneMenu@CView@@IAEXPAVCCmdUI@@@Z 5f85eb3d f
 0001:0005db7b       ?OnNextPaneCmd@CView@@IAEHI@Z 5f85eb7b f
 0001:0005dbc4       ?OnPreparePrinting@CView@@MAEHPAUCPrintInfo@@@Z 5f85ebc4 f
 0001:0005dbca       ?OnEndPrintPreview@CView@@MAEXPAVCDC@@PAUCPrintInfo@@UtagPOINT@@PAVCPreviewView@@@Z 5f85ebca f
 0001:0005dc6d       ?GetMessageMap@CCtrlView@@MBEPBUAFX_MSGMAP@@XZ 5f85ec6d f
 0001:0005dc73       ??_ECCtrlView@@UAEPAXI@Z   5f85ec73 f
 0001:0005dc73       ??_GCCtrlView@@UAEPAXI@Z   5f85ec73 f
 0001:0005dc8f       ?GetMessageMap@CScrollView@@MBEPBUAFX_MSGMAP@@XZ 5f85ec8f f
 0001:0005dc95       ?_AfxGetMouseScrollLines@@YGIXZ 5f85ec95 f
 0001:0005ddcf       ??_ECScrollView@@UAEPAXI@Z 5f85edcf f
 0001:0005ddcf       ??_GCScrollView@@UAEPAXI@Z 5f85edcf f
 0001:0005de6e       ?SetScaleToFitSize@CScrollView@@QAEXUtagSIZE@@@Z 5f85ee6e f
 0001:0005df17       ?GetScrollPosition@CScrollView@@QBE?AVCPoint@@XZ 5f85ef17 f
 0001:0005dfa8       ?ScrollToPosition@CScrollView@@QAEXUtagPOINT@@@Z 5f85efa8 f
 0001:0005e097       ?GetDeviceScrollSizes@CScrollView@@QBEXAAHAAUtagSIZE@@11@Z 5f85f097 f
 0001:0005e0d0       ?FillOutsideRect@CScrollView@@QAEXPAVCDC@@PAVCBrush@@@Z 5f85f0d0 f
 0001:0005e153       ?ResizeParentToFit@CScrollView@@QAEXH@Z 5f85f153 f
 0001:0005e280       ?CenterOnPoint@CScrollView@@IAEXVCPoint@@@Z 5f85f280 f
 0001:0005e4b0       ?OnHScroll@CScrollView@@QAEXIIPAVCScrollBar@@@Z 5f85f4b0 f
 0001:0005e4f4       ?OnVScroll@CScrollView@@QAEXIIPAVCScrollBar@@@Z 5f85f4f4 f
 0001:0005e53c       ?OnMouseWheel@CScrollView@@QAEHIFVCPoint@@@Z 5f85f53c f
 0001:0005e570       ?DoMouseWheel@CScrollView@@QAEHIFVCPoint@@@Z 5f85f570 f
 0001:0005e698       ?OnScroll@CScrollView@@UAEHIIH@Z 5f85f698 f
 0001:0005e77b       ?OnScrollBy@CScrollView@@UAEHVCSize@@H@Z 5f85f77b f
 0001:0005e877       ??0CFormView@@IAE@PBG@Z    5f85f877 f
 0001:0005e89a       ??_ECFormView@@UAEPAXI@Z   5f85f89a f
 0001:0005e89a       ??_GCFormView@@UAEPAXI@Z   5f85f89a f
 0001:0005e8b6       ??1CFormView@@UAE@XZ       5f85f8b6 f
 0001:0005e8bb       ??0CFormView@@IAE@I@Z      5f85f8bb f
 0001:0005e8df       ?Create@CFormView@@MAEHPBG0KABUtagRECT@@PAVCWnd@@IPAUCCreateContext@@@Z 5f85f8df f
 0001:0005e9f3       ?OnCreate@CFormView@@IAEHPAUtagCREATESTRUCTW@@@Z 5f85f9f3 f
 0001:0005ea05       ?OnActivateView@CFormView@@MAEXHPAVCView@@0@Z 5f85fa05 f
 0001:0005ea28       ?OnActivateFrame@CFormView@@MAEXIPAVCFrameWnd@@@Z 5f85fa28 f
 0001:0005ea37       ?SaveFocusControl@CFormView@@IAEHXZ 5f85fa37 f
 0001:0005ea62       ?OnSetFocus@CFormView@@IAEXPAVCWnd@@@Z 5f85fa62 f
 0001:0005ea9c       ?PreTranslateMessage@CFormView@@MAEHPAUtagMSG@@@Z 5f85fa9c f
 0001:0005eb06       ?HandleInitDialog@CFormView@@IAEJIJ@Z 5f85fb06 f
 0001:0005eb36       ?SetOccDialogInfo@CFormView@@MAEHPAU_AFX_OCC_DIALOG_INFO@@@Z 5f85fb36 f
 0001:0005eb43       ?GetOpenDocumentCount@CWinApp@@QAEHXZ 5f85fb43 f
 0001:0005eb4e       ?_GetBaseMessageMap@COleDBRecordView@@KGPBUAFX_MSGMAP@@XZ 5f85fb4e f
 0001:0005eb54       ?GetMessageMap@COleDBRecordView@@MBEPBUAFX_MSGMAP@@XZ 5f85fb54 f
 0001:0005eb5a       ?OnInitialUpdate@COleDBRecordView@@UAEXXZ 5f85fb5a f
 0001:0005eb5a       ?OnInitialUpdate@CFormView@@UAEXXZ 5f85fb5a f
 0001:0005eb6d       ?OnMove@COleDBRecordView@@UAEHI@Z 5f85fb6d f
 0001:0005ec24       ?OnUpdateRecordPrev@COleDBRecordView@@IAEXPAVCCmdUI@@@Z 5f85fc24 f
 0001:0005ec3f       ?OnUpdateRecordLast@COleDBRecordView@@IAEXPAVCCmdUI@@@Z 5f85fc3f f
 0001:0005ed25       ??0CMemFile@@QAE@PAEII@Z   5f85fd25 f
 0001:0005ed61       ?Attach@CMemFile@@QAEXPAEII@Z 5f85fd61 f
 0001:0005ed8c       ?Detach@CMemFile@@QAEPAEXZ 5f85fd8c f
 0001:0005ed9e       ?GetPosition@CMemFile@@UBEKXZ 5f85fd9e f
 0001:0005edb6       ?SetLength@CMemFile@@UAEXK@Z 5f85fdb6 f
 0001:0005ee01       ?Flush@CMemFile@@UAEXXZ    5f85fe01 f
 0001:0005ee02       ?Abort@CMemFile@@UAEXXZ    5f85fe02 f
 0001:0005ee07       ?UnlockRange@CMemFile@@UAEXKK@Z 5f85fe07 f
 0001:0005ee0f       ?Duplicate@CMemFile@@UBEPAVCFile@@XZ 5f85fe0f f
 0001:0005ee29       ?OnHelp@CWnd@@QAEXXZ       5f85fe29 f
 0001:0005eecb       ?OnHelp@CFrameWnd@@IAEXXZ  5f85fecb f
 0001:0005eefe       ?OnHelpIndex@CWnd@@QAEXXZ  5f85fefe f
 0001:0005ef15       ?OnHelpFinder@CWnd@@QAEXXZ 5f85ff15 f
 0001:0005ef2c       ?OnHelpUsing@CWnd@@QAEXXZ  5f85ff2c f
 0001:0005ef43       ?CanEnterHelpMode@CFrameWnd@@QAEHXZ 5f85ff43 f
 0001:0005efa0       ?OnContextHelp@CFrameWnd@@QAEXXZ 5f85ffa0 f
 0001:0005f142       ?SetHelpCapture@CFrameWnd@@IAEPAUHWND__@@UtagPOINT@@PAH@Z 5f860142 f
 0001:0005f263       ?_AfxMapClientArea@@YGKPAUHWND__@@UtagPOINT@@@Z 5f860263 f
 0001:0005f2fc       ?_AfxMapNonClientArea@@YGKH@Z 5f8602fc f
 0001:0005f316       ?ProcessHelpMsg@CFrameWnd@@IAEHAAUtagMSG@@PAK@Z 5f860316 f
 0001:0005f54b       ?ResetTimer@CControlBar@@QAEXII@Z 5f86054b f
 0001:0005f581       ?OnTimer@CControlBar@@QAEXI@Z 5f860581 f
 0001:0005f706       ?SetStatusText@CControlBar@@UAEHH@Z 5f860706 f
 0001:0005f99b       ?OnHelpHitTest@CControlBar@@QAEJIJ@Z 5f86099b f
 0001:0005faa8       ?OnMouseActivate@CControlBar@@QAEHPAVCWnd@@II@Z 5f860aa8 f
 0001:0005fadb       ?OnLButtonDown@CControlBar@@QAEXIVCPoint@@@Z 5f860adb f
 0001:0005fb21       ?OnLButtonDblClk@CControlBar@@QAEXIVCPoint@@@Z 5f860b21 f
 0001:0005fbf0       ?DelayShow@CControlBar@@UAEXH@Z 5f860bf0 f
 0001:0005fcc6       ?CommandToIndex@CToolBar@@QBEHI@Z 5f860cc6 f
 0001:0005fcdc       ?GetItemID@CToolBar@@QBEIH@Z 5f860cdc f
 0001:0005feb2       ?GetButtonInfo@CToolBar@@QBEXHAAI0AAH@Z 5f860eb2 f
 0001:0005feea       ?OnToolHitTest@CToolBar@@UBEHVCPoint@@PAUtagTOOLINFOW@@@Z 5f860eea f
 0001:0005ffb5       ?SetButtonText@CToolBar@@QAEHHPBG@Z 5f860fb5 f
 0001:000600b3       ?GetButtonText@CToolBar@@QBE?AVCString@@H@Z 5f8610b3 f
 0001:00060111       ?GetButtonText@CToolBar@@QBEXHAAVCString@@@Z 5f861111 f
 0001:000601b8       ?OnNcHitTest@CToolBar@@IAEIVCPoint@@@Z 5f8611b8 f
 0001:000601eb       ?OnPreserveZeroBorderHelper@CToolBar@@IAEJIJ@Z 5f8611eb f
 0001:0006023a       ?OnSysColorChange@CToolBar@@IAEXXZ 5f86123a f
 0001:00060273       ??0CDialogBar@@QAE@XZ      5f861273 f
 0001:00060293       ??1CDialogBar@@UAE@XZ      5f861293 f
 0001:000602cb       ?Create@CDialogBar@@QAEHPAVCWnd@@PBGII@Z 5f8612cb f
 0001:000603ce       ?CalcFixedLayout@CDialogBar@@UAE?AVCSize@@HH@Z 5f8613ce f
 0001:00060418       ?OnUpdateCmdUI@CDialogBar@@UAEXPAVCFrameWnd@@H@Z 5f861418 f
 0001:00060428       ?GetMessageMap@CDialogBar@@MBEPBUAFX_MSGMAP@@XZ 5f861428 f
 0001:0006042e       ?HandleInitDialog@CDialogBar@@IAEJIJ@Z 5f86142e f
 0001:00060469       ?SetOccDialogInfo@CDialogBar@@MAEHPAU_AFX_OCC_DIALOG_INFO@@@Z 5f861469 f
 0001:0006048d       ?GetItemID@CStatusBar@@QBEIH@Z 5f86148d f
 0001:0006049d       ?GetItemRect@CStatusBar@@QBEXHPAUtagRECT@@@Z 5f86149d f
 0001:000604d4       ?GetPaneInfo@CStatusBar@@QBEXHAAI0AAH@Z 5f8614d4 f
 0001:000604fe       ?SetPaneInfo@CStatusBar@@QAEXHIIH@Z 5f8614fe f
 0001:0006057a       ?GetPaneText@CStatusBar@@QBEXHAAVCString@@@Z 5f86157a f
 0001:00060595       ?GetPaneText@CStatusBar@@QBE?AVCString@@H@Z 5f861595 f
 0001:000605ce       ?OnNcHitTest@CStatusBar@@IAEIVCPoint@@@Z 5f8615ce f
 0001:000605e2       ?OnBarStyleChange@CStatusBar@@UAEXKK@Z 5f8615e2 f
 0001:00060620       ?OnGetText@CStatusBar@@IAEJIJ@Z 5f861620 f
 0001:00060678       ?OnGetTextLength@CStatusBar@@IAEJIJ@Z 5f861678 f
 0001:0006069c       ?OnSetMinHeight@CStatusBar@@IAEJIJ@Z 5f86169c f
 0001:000606af       ?SetCheck@CStatusCmdUI@@UAEXH@Z 5f8616af f
 0001:000606dd       ?SetText@CStatusCmdUI@@UAEXPBG@Z 5f8616dd f
 0001:000606f1       ?GetDockedCount@CDockBar@@QBEHXZ 5f8616f1 f
 0001:00060837       ?ReDockControlBar@CDockBar@@QAEXPAVCControlBar@@PBUtagRECT@@@Z 5f861837 f
 0001:00060d6a       ?ShowAll@CDockBar@@QAEXH@Z 5f861d6a f
 0001:00060dab       ?Insert@CDockBar@@IAEHPAVCControlBar@@VCRect@@VCPoint@@@Z 5f861dab f
 0001:00060f01       ?_GetBaseMessageMap@CMiniDockFrameWnd@@KGPBUAFX_MSGMAP@@XZ 5f861f01 f
 0001:00060f07       ?GetMessageMap@CMiniDockFrameWnd@@MBEPBUAFX_MSGMAP@@XZ 5f861f07 f
 0001:00060f0d       ?OnMouseActivate@CMiniDockFrameWnd@@QAEHPAVCWnd@@II@Z 5f861f0d f
 0001:00060f28       ??0CMiniDockFrameWnd@@QAE@XZ 5f861f28 f
 0001:00060f6b       ??_GCMiniDockFrameWnd@@UAEPAXI@Z 5f861f6b f
 0001:00060f6b       ??_ECMiniDockFrameWnd@@UAEPAXI@Z 5f861f6b f
 0001:00060f87       ??1CMiniDockFrameWnd@@UAE@XZ 5f861f87 f
 0001:00060fbf       ?Create@CMiniDockFrameWnd@@UAEHPAVCWnd@@K@Z 5f861fbf f
 0001:00061124       ?RecalcLayout@CMiniDockFrameWnd@@UAEXH@Z 5f862124 f
 0001:0006116c       ?OnClose@CMiniDockFrameWnd@@QAEXXZ 5f86216c f
 0001:0006117a       ?OnNcLButtonDown@CMiniDockFrameWnd@@QAEXIVCPoint@@@Z 5f86217a f
 0001:00061220       ?OnNcLButtonDblClk@CMiniDockFrameWnd@@QAEXIVCPoint@@@Z 5f862220 f
 0001:00061271       ?_AfxAdjustRectangle@@YGXAAVCRect@@VCPoint@@@Z 5f862271 f
 0001:000612cc       ?StartDrag@CDockContext@@UAEXVCPoint@@@Z 5f8622cc f
 0001:0006161f       ?Move@CDockContext@@QAEXVCPoint@@@Z 5f86261f f
 0001:0006169b       ?OnKey@CDockContext@@QAEXHH@Z 5f86269b f
 0001:000616cf       ?EndDrag@CDockContext@@QAEXXZ 5f8626cf f
 0001:000617da       ?StartResize@CDockContext@@UAEXHVCPoint@@@Z 5f8627da f
 0001:00061927       ?Stretch@CDockContext@@QAEXVCPoint@@@Z 5f862927 f
 0001:00061aac       ?EndResize@CDockContext@@QAEXXZ 5f862aac f
 0001:00061aef       ?ToggleDocking@CDockContext@@UAEXXZ 5f862aef f
 0001:00061bc4       ?InitLoop@CDockContext@@QAEXXZ 5f862bc4 f
 0001:00061c81       ?CancelLoop@CDockContext@@QAEXXZ 5f862c81 f
 0001:00061cca       ?DrawFocusRect@CDockContext@@QAEXH@Z 5f862cca f
 0001:00061dea       ?UpdateState@CDockContext@@QAEXPAHH@Z 5f862dea f
 0001:00061e3c       ?CanDock@CDockContext@@QAEKXZ 5f862e3c f
 0001:00061f62       ?GetDockBar@CDockContext@@QAEPAVCDockBar@@K@Z 5f862f62 f
 0001:00061faa       ?Track@CDockContext@@QAEHXZ 5f862faa f
 0001:000620c8       ?LoadState@CControlBarInfo@@QAEHPBGHPAVCDockState@@@Z 5f8630c8 f
 0001:00062335       ?SaveState@CControlBarInfo@@QAEHPBGH@Z 5f863335 f
 0001:00062587       ?LoadState@CDockState@@QAEXPBG@Z 5f863587 f
 0001:0006266e       ?SaveState@CDockState@@QAEXPBG@Z 5f86366e f
 0001:000627c1       ?LoadBarState@CFrameWnd@@QAEXPBG@Z 5f8637c1 f
 0001:0006280e       ?SaveBarState@CFrameWnd@@QBEXPBG@Z 5f86380e f
 0001:000629bb       ?GetMessageMap@CReBar@@MBEPBUAFX_MSGMAP@@XZ 5f8639bb f
 0001:000629c1       ??0CReBar@@QAE@XZ          5f8639c1 f
 0001:000629fc       ??_ECReBar@@UAEPAXI@Z      5f8639fc f
 0001:000629fc       ??_GCReBar@@UAEPAXI@Z      5f8639fc f
 0001:00062a18       ??1CReBar@@UAE@XZ          5f863a18 f
 0001:00062a1d       ?OnRecalcParent@CReBar@@IAEXXZ 5f863a1d f
 0001:00062a2f       ?OnHeightChange@CReBar@@IAEXPAUtagNMHDR@@PAJ@Z 5f863a2f f
 0001:00062a6f       ?OnShowBand@CReBar@@IAEJIJ@Z 5f863a6f f
 0001:00062b06       ?_AddBar@CReBar@@IAEHPAVCWnd@@PAUtagREBARBANDINFOW@@@Z 5f863b06 f
 0001:00062bc3       ?AddBar@CReBar@@QAEHPAVCWnd@@PBGPAVCBitmap@@K@Z 5f863bc3 f
 0001:00062c08       ?AddBar@CReBar@@QAEHPAVCWnd@@KKPBGK@Z 5f863c08 f
 0001:00062c48       ?CalcFixedLayout@CReBar@@UAE?AVCSize@@HH@Z 5f863c48 f
 0001:00062dd9       ?Create@CReBar@@QAEHPAVCWnd@@KKI@Z 5f863dd9 f
 0001:00062e4c       ?OnNcCreate@CReBar@@IAEHPAUtagCREATESTRUCTW@@@Z 5f863e4c f
 0001:00062e78       ?OnNcCalcSize@CReBar@@IAEXHPAUtagNCCALCSIZE_PARAMS@@@Z 5f863e78 f
 0001:00062ec4       ?OnPaint@CReBar@@IAEXXZ    5f863ec4 f
 0001:00062ec9       ?OnToolHitTest@CReBar@@UBEHVCPoint@@PAUtagTOOLINFOW@@@Z 5f863ec9 f
 0001:00062f0e       ?WindowProc@CReBar@@MAEJIIJ@Z 5f863f0e f
 0001:00062f4b       ?PrepareEditCtrl@CDataExchange@@QAEPAUHWND__@@H@Z 5f863f4b f
 0001:00062f6c       ?Fail@CDataExchange@@QAEXXZ 5f863f6c f
 0001:00062fa1       ?_AfxSimpleScanf@@YGHPBG0PAD@Z 5f863fa1 f
 0001:0006305a       ?_Afx_DDX_TextWithFormat@@YAXPAVCDataExchange@@HPBGIZZ 5f86405a f
 0001:000630ca       ?DDX_Text@@YGXPAVCDataExchange@@HAAE@Z 5f8640ca f
 0001:0006313b       ?DDX_Text@@YGXPAVCDataExchange@@HAAF@Z 5f86413b f
 0001:00063176       ?DDX_Text@@YGXPAVCDataExchange@@HAAH@Z 5f864176 f
 0001:000631a5       ?DDX_Text@@YGXPAVCDataExchange@@HAAI@Z 5f8641a5 f
 0001:000631d4       ?DDX_Text@@YGXPAVCDataExchange@@HAAJ@Z 5f8641d4 f
 0001:00063203       ?DDX_Text@@YGXPAVCDataExchange@@HAAK@Z 5f864203 f
 0001:00063232       ?DDX_Text@@YGXPAVCDataExchange@@HAAVCString@@@Z 5f864232 f
 0001:00063284       ?DDX_Text@@YGXPAVCDataExchange@@HPAGH@Z 5f864284 f
 0001:000632c2       ?DDX_Check@@YGXPAVCDataExchange@@HAAH@Z 5f8642c2 f
 0001:00063314       ?DDX_Radio@@YGXPAVCDataExchange@@HAAH@Z 5f864314 f
 0001:000633a5       ?DDX_LBString@@YGXPAVCDataExchange@@HAAVCString@@@Z 5f8643a5 f
 0001:00063425       ?DDX_LBStringExact@@YGXPAVCDataExchange@@HAAVCString@@@Z 5f864425 f
 0001:00063476       ?DDX_CBString@@YGXPAVCDataExchange@@HAAVCString@@@Z 5f864476 f
 0001:000634f5       ?DDX_CBStringExact@@YGXPAVCDataExchange@@HAAVCString@@@Z 5f8644f5 f
 0001:00063552       ?DDX_LBIndex@@YGXPAVCDataExchange@@HAAH@Z 5f864552 f
 0001:00063594       ?DDX_CBIndex@@YGXPAVCDataExchange@@HAAH@Z 5f864594 f
 0001:000635d6       ?DDX_Scroll@@YGXPAVCDataExchange@@HAAH@Z 5f8645d6 f
 0001:00063611       ?DDX_Slider@@YGXPAVCDataExchange@@HAAH@Z 5f864611 f
 0001:00063655       ?_AfxFailMinMaxWithFormat@@YGXPAVCDataExchange@@JJPBGI@Z 5f864655 f
 0001:000636ee       ?DDV_MinMaxByte@@YGXPAVCDataExchange@@EEE@Z 5f8646ee f
 0001:0006371e       ?DDV_MinMaxShort@@YGXPAVCDataExchange@@FFF@Z 5f86471e f
 0001:00063751       ?DDV_MinMaxInt@@YGXPAVCDataExchange@@HHH@Z 5f864751 f
 0001:0006377d       ?DDV_MinMaxUInt@@YGXPAVCDataExchange@@III@Z 5f86477d f
 0001:000637a9       ?DDV_MinMaxSlider@@YGXPAVCDataExchange@@KKK@Z 5f8647a9 f
 0001:000637ec       ?DDV_MaxChars@@YGXPAVCDataExchange@@ABVCString@@H@Z 5f8647ec f
 0001:000638af       ?AfxFailMaxChars@@YGXPAVCDataExchange@@H@Z 5f8648af f
 0001:00063927       ?AfxFailRadio@@YGXPAVCDataExchange@@@Z 5f864927 f
 0001:00063987       ?_AfxSimpleFloatParse@@YGHPBGAAN@Z 5f864987 f
 0001:000639f6       ?AfxTextFloatFormat@@YGXPAVCDataExchange@@HPAXNH@Z 5f8649f6 f
 0001:00063a8b       ?DDX_Text@@YGXPAVCDataExchange@@HAAM@Z 5f864a8b f
 0001:00063aa9       ?DDX_Text@@YGXPAVCDataExchange@@HAAN@Z 5f864aa9 f
 0001:00063ac7       ?_AfxFailMinMaxReal@@YGXPAVCDataExchange@@NNHI@Z 5f864ac7 f
 0001:00063b78       ?DDV_MinMaxFloat@@YGXPAVCDataExchange@@ABMMM@Z 5f864b78 f
 0001:00063bb5       ?DDV_MinMaxDouble@@YGXPAVCDataExchange@@ABNNN@Z 5f864bb5 f
 0001:00063bf2       ?_AfxAppendFilterSuffix@@YGXAAVCString@@AAUtagOFNW@@PAVCDocTemplate@@PAV1@@Z 5f864bf2 f
 0001:00063cd0       ?_GetBaseMessageMap@CNewTypeDlg@@KGPBUAFX_MSGMAP@@XZ 5f864cd0 f
 0001:00063cd6       ?GetMessageMap@CNewTypeDlg@@MBEPBUAFX_MSGMAP@@XZ 5f864cd6 f
 0001:00063cdc       ?OnInitDialog@CNewTypeDlg@@MAEHXZ 5f864cdc f
 0001:00063df1       ?OnOK@CNewTypeDlg@@MAEXXZ  5f864df1 f
 0001:00063e3b       ?DoPromptFileName@CDocManager@@UAEHAAVCString@@IKHPAVCDocTemplate@@@Z 5f864e3b f
 0001:00063fe6       ?GetDocumentCount@CDocManager@@IAEHXZ 5f864fe6 f
 0001:00064028       ?OnDDECommand@CDocManager@@UAEHPAG@Z 5f865028 f
 0001:0006468d       ??_ECNewTypeDlg@@UAEPAXI@Z 5f86568d f
 0001:0006468d       ??_GCNewTypeDlg@@UAEPAXI@Z 5f86568d f
 0001:000646a9       ?OnFileOpen@CDocManager@@UAEXXZ 5f8656a9 f
 0001:0006470e       ?GetMessageMap@CSplitterWnd@@MBEPBUAFX_MSGMAP@@XZ 5f86570e f
 0001:00064714       ??0CSplitterWnd@@QAE@XZ    5f865714 f
 0001:0006477f       ??1CSplitterWnd@@UAE@XZ    5f86577f f
 0001:000647c7       ?Create@CSplitterWnd@@QAEHPAVCWnd@@HHUtagSIZE@@PAUCCreateContext@@KI@Z 5f8657c7 f
 0001:00064840       ?CreateStatic@CSplitterWnd@@QAEHPAVCWnd@@HHKI@Z 5f865840 f
 0001:00064873       ?CreateCommon@CSplitterWnd@@IAEHPAVCWnd@@UtagSIZE@@KI@Z 5f865873 f
 0001:00064985       ?OnNcCreate@CSplitterWnd@@IAEHPAUtagCREATESTRUCTW@@@Z 5f865985 f
 0001:000649b7       ?CreateView@CSplitterWnd@@UAEHHHPAUCRuntimeClass@@UtagSIZE@@PAUCCreateContext@@@Z 5f8659b7 f
 0001:00064af4       ?CreateScrollBarCtrl@CSplitterWnd@@UAEHKI@Z 5f865af4 f
 0001:00064b31       ?IdFromRowCol@CSplitterWnd@@QBEHHH@Z 5f865b31 f
 0001:00064b44       ?GetPane@CSplitterWnd@@QBEPAVCWnd@@HH@Z 5f865b44 f
 0001:00064b60       ?IsChildPane@CSplitterWnd@@QAEHPAVCWnd@@PAH1@Z 5f865b60 f
 0001:00064bdc       ?GetRowInfo@CSplitterWnd@@QBEXHAAH0@Z 5f865bdc f
 0001:00064c0c       ?SetRowInfo@CSplitterWnd@@QAEXHHH@Z 5f865c0c f
 0001:00064c38       ?GetColumnInfo@CSplitterWnd@@QBEXHAAH0@Z 5f865c38 f
 0001:00064c60       ?SetColumnInfo@CSplitterWnd@@QAEXHHH@Z 5f865c60 f
 0001:00064c84       ?GetScrollStyle@CSplitterWnd@@QBEKXZ 5f865c84 f
 0001:00064c9c       ?SetScrollStyle@CSplitterWnd@@QAEXK@Z 5f865c9c f
 0001:00064dd5       ?DeleteView@CSplitterWnd@@UAEXHH@Z 5f865dd5 f
 0001:00064e12       ?OnDrawSplitter@CSplitterWnd@@MAEXPAVCDC@@W4ESplitType@1@ABVCRect@@@Z 5f865e12 f
 0001:00064f2d       ?_AfxCanSplitRowCol@@YGHPAUCRowColInfo@CSplitterWnd@@HH@Z 5f865f2d f
 0001:00064f4d       ?SplitRow@CSplitterWnd@@UAEHH@Z 5f865f4d f
 0001:00065055       ?SplitColumn@CSplitterWnd@@UAEHH@Z 5f866055 f
 0001:00065157       ?DeleteRow@CSplitterWnd@@UAEXH@Z 5f866157 f
 0001:00065270       ?DeleteColumn@CSplitterWnd@@UAEXH@Z 5f866270 f
 0001:00065389       ?GetInsideRect@CSplitterWnd@@MBEXAAVCRect@@@Z 5f866389 f
 0001:000653d7       ?StartTracking@CSplitterWnd@@MAEXH@Z 5f8663d7 f
 0001:000655a3       ?TrackRowSize@CSplitterWnd@@MAEXHH@Z 5f8665a3 f
 0001:00065638       ?TrackColumnSize@CSplitterWnd@@MAEXHH@Z 5f866638 f
 0001:000656c4       ?StopTracking@CSplitterWnd@@MAEXH@Z 5f8666c4 f
 0001:00065867       ?GetHitRect@CSplitterWnd@@MAEXHAAVCRect@@@Z 5f866867 f
 0001:00065a32       ?HitTest@CSplitterWnd@@MBEHVCPoint@@@Z 5f866a32 f
 0001:00065bec       ?OnInvertTracker@CSplitterWnd@@MAEXABVCRect@@@Z 5f866bec f
 0001:00065c62       ?DoKeyboardSplit@CSplitterWnd@@UAEHXZ 5f866c62 f
 0001:00065d62       ?OnDisplayChange@CSplitterWnd@@IAEXXZ 5f866d62 f
 0001:00065d8b       ?OnSize@CSplitterWnd@@IAEXIHH@Z 5f866d8b f
 0001:00065db6       ?_AfxLayoutRowCol@@YGXPAUCRowColInfo@CSplitterWnd@@HHH@Z 5f866db6 f
 0001:00065e76       ?_AfxDeferClientPos@@YGXPAUAFX_SIZEPARENTPARAMS@@PAVCWnd@@HHHHH@Z 5f866e76 f
 0001:00065f85       ?GetSizingParent@CSplitterWnd@@IAEPAVCWnd@@XZ 5f866f85 f
 0001:0006601b       ?RecalcLayout@CSplitterWnd@@UAEXXZ 5f86701b f
 0001:000662de       ?DrawAllSplitBars@CSplitterWnd@@MAEXPAVCDC@@HH@Z 5f8672de f
 0001:000664e1       ?OnPaint@CSplitterWnd@@IAEXXZ 5f8674e1 f
 0001:000666cc       ?OnSetCursor@CSplitterWnd@@IAEHPAVCWnd@@II@Z 5f8676cc f
 0001:000666ec       ?SetSplitCursor@CSplitterWnd@@MAEXH@Z 5f8676ec f
 0001:000667d9       ?OnMouseMove@CSplitterWnd@@IAEXIVCPoint@@@Z 5f8677d9 f
 0001:00066955       ?OnLButtonDown@CSplitterWnd@@IAEXIVCPoint@@@Z 5f867955 f
 0001:00066980       ?OnLButtonDblClk@CSplitterWnd@@IAEXIVCPoint@@@Z 5f867980 f
 0001:00066ac9       ?OnLButtonUp@CSplitterWnd@@IAEXIVCPoint@@@Z 5f867ac9 f
 0001:00066ad6       ?OnCancelMode@CSplitterWnd@@IAEXXZ 5f867ad6 f
 0001:00066ae1       ?OnKeyDown@CSplitterWnd@@IAEXIII@Z 5f867ae1 f
 0001:00066c16       ?OnSysCommand@CSplitterWnd@@IAEXIJ@Z 5f867c16 f
 0001:00066c55       ?OnCommand@CSplitterWnd@@MAEHIJ@Z 5f867c55 f
 0001:00066c8f       ?OnNotify@CSplitterWnd@@MAEHIJPAJ@Z 5f867c8f f
 0001:00066ccc       ?OnMouseWheel@CSplitterWnd@@IAEHIFVCPoint@@@Z 5f867ccc f
 0001:00066d92       ?OnHScroll@CSplitterWnd@@IAEXIIPAVCScrollBar@@@Z 5f867d92 f
 0001:00066e28       ?OnVScroll@CSplitterWnd@@IAEXIIPAVCScrollBar@@@Z 5f867e28 f
 0001:00066ebe       ?DoScroll@CSplitterWnd@@UAEHPAVCView@@IH@Z 5f867ebe f
 0001:00067015       ?DoScrollBy@CSplitterWnd@@UAEHPAVCView@@VCSize@@H@Z 5f868015 f
 0001:0006716c       ?CanActivateNext@CSplitterWnd@@UAEHH@Z 5f86816c f
 0001:00067192       ?ActivateNext@CSplitterWnd@@UAEXH@Z 5f868192 f
 0001:00067203       ?SetActivePane@CSplitterWnd@@UAEXHHPAVCWnd@@@Z 5f868203 f
 0001:0006724d       ?GetActivePane@CSplitterWnd@@UAEPAVCWnd@@PAH0@Z 5f86824d f
 0001:000672a5       ?OnDDECommand@CWinApp@@UAEHPAG@Z 5f8682a5 f
 0001:000672bf       ?OnOpenRecentFile@CWinApp@@IAEHI@Z 5f8682bf f
 0001:00067303       ?DoMessageBox@CWinApp@@UAEHPBGII@Z 5f868303 f
 0001:000673f9       ?AfxMessageBox@@YGHPBGII@Z 5f8683f9 f
 0001:00067431       ?AfxMessageBox@@YGHIII@Z   5f868431 f
 0001:00067574       ?OnFileOpen@CWinApp@@IAEXXZ 5f868574 f
 0001:0006757f       ?DoPromptFileName@CWinApp@@QAEHAAVCString@@IKHPAVCDocTemplate@@@Z 5f86857f f
 0001:000675fe       ?AfxFormatString2@@YGXAAVCString@@IPBG1@Z 5f8685fe f
 0001:00067624       ?OnHelp@CWinApp@@IAEXXZ    5f868624 f
 0001:00067668       ?OnHelpIndex@CWinApp@@IAEXXZ 5f868668 f
 0001:00067675       ?OnHelpFinder@CWinApp@@IAEXXZ 5f868675 f
 0001:00067682       ?OnHelpUsing@CWinApp@@IAEXXZ 5f868682 f
 0001:0006768f       ?OnContextHelp@CWinApp@@IAEXXZ 5f86868f f
 0001:000676c5       ??0CSharedFile@@QAE@II@Z   5f8686c5 f
 0001:000676ef       ?SetHandle@CSharedFile@@QAEXPAXH@Z 5f8686ef f
 0001:0006771d       ?Alloc@CSharedFile@@MAEPAEK@Z 5f86871d f
 0001:0006773f       ?Realloc@CSharedFile@@MAEPAEPAEK@Z 5f86873f f
 0001:00067777       ?Free@CSharedFile@@MAEXPAE@Z 5f868777 f
 0001:00067790       ?Detach@CSharedFile@@QAEPAXXZ 5f868790 f
 0001:000677f2       ?OnPaletteChanged@CFrameWnd@@IAEXPAVCWnd@@@Z 5f8687f2 f
 0001:00067890       ?OnCommandHelp@CFrameWnd@@IAEJIJ@Z 5f868890 f
 0001:000678e8       ?OnHelpHitTest@CFrameWnd@@IAEJIJ@Z 5f8688e8 f
 0001:00067a65       ?ShowOwnedWindows@CFrameWnd@@QAEXH@Z 5f868a65 f
 0001:00067b87       ?OnUpdateFrameMenu@CFrameWnd@@UAEXPAUHMENU__@@@Z 5f868b87 f
 0001:00067c3a       ?OnHScroll@CFrameWnd@@IAEXIIPAVCScrollBar@@@Z 5f868c3a f
 0001:00067c63       ?OnVScroll@CFrameWnd@@IAEXIIPAVCScrollBar@@@Z 5f868c63 f
 0001:00067d2d       ?OnDropFiles@CFrameWnd@@IAEXPAUHDROP__@@@Z 5f868d2d f
 0001:00067da2       ?OnQueryEndSession@CFrameWnd@@IAEHXZ 5f868da2 f
 0001:00067dc7       ?OnEndSession@CFrameWnd@@IAEXH@Z 5f868dc7 f
 0001:00067dff       ?OnDDEInitiate@CFrameWnd@@IAEJIJ@Z 5f868dff f
 0001:00067ec2       ?OnDDEExecute@CFrameWnd@@IAEJIJ@Z 5f868ec2 f
 0001:00067f5d       ?OnDDETerminate@CFrameWnd@@IAEJIJ@Z 5f868f5d f
 0001:00067f8b       ?ShowControlBar@CFrameWnd@@QAEXPAVCControlBar@@HH@Z 5f868f8b f
 0001:000681d9       ?OnPopMessageString@CFrameWnd@@IAEJIJ@Z 5f8691d9 f
 0001:00068213       ?OnHelpPromptAddr@CFrameWnd@@IAEJIJ@Z 5f869213 f
 0001:0006822a       ?OnUpdateControlBarMenu@CFrameWnd@@QAEXPAVCCmdUI@@@Z 5f86922a f
 0001:0006825f       ?OnBarCheck@CFrameWnd@@QAEHI@Z 5f86925f f
 0001:00068298       ?OnToolTipText@CFrameWnd@@IAEHIPAUtagNMHDR@@PAJ@Z 5f869298 f
 0001:00068401       ?OnSetPreviewMode@CFrameWnd@@UAEXHPAUCPrintPreviewState@@@Z 5f869401 f
 0001:00068618       ?DelayUpdateFrameMenu@CFrameWnd@@UAEXPAUHMENU__@@@Z 5f869618 f
 0001:00068679       ?GetActiveFrame@CFrameWnd@@UAEPAV1@XZ 5f869679 f
 0001:000686f9       ?NegotiateBorderSpace@CFrameWnd@@UAEHIPAUtagRECT@@@Z 5f8696f9 f
 0001:00068773       ?OnRegisteredMouseWheel@CFrameWnd@@IAEJIJ@Z 5f869773 f
 0001:0006884c       ?CreateFloatingFrame@CFrameWnd@@QAEPAVCMiniDockFrameWnd@@K@Z 5f86984c f
 0001:000688b8       ?ReDockControlBar@CFrameWnd@@QAEXPAVCControlBar@@PAVCDockBar@@PBUtagRECT@@@Z 5f8698b8 f
 0001:0006893d       ?FloatControlBar@CFrameWnd@@QAEXPAVCControlBar@@VCPoint@@K@Z 5f86993d f
 0001:00068a3a       ?CanDock@CFrameWnd@@QAEKVCRect@@KPAPAVCDockBar@@@Z 5f869a3a f
 0001:00068ae6       ?GetMessageMap@CMDIFrameWnd@@MBEPBUAFX_MSGMAP@@XZ 5f869ae6 f
 0001:00068b2c       ?OnCommandHelp@CMDIFrameWnd@@IAEJIJ@Z 5f869b2c f
 0001:00068bf4       ?DelayUpdateFrameMenu@CMDIFrameWnd@@UAEXPAUHMENU__@@@Z 5f869bf4 f
 0001:00068c3f       ?OnMenuChar@CMDIFrameWnd@@IAEJIIPAVCMenu@@@Z 5f869c3f f
 0001:00068c90       ?CreateNewChild@CMDIFrameWnd@@QAEPAVCMDIChildWnd@@PAUCRuntimeClass@@IPAUHMENU__@@PAUHACCEL__@@@Z 5f869c90 f
 0001:00068d74       ??1CMDIChildWnd@@UAE@XZ    5f869d74 f
 0001:00068ee6       ?OnMouseActivate@CMDIChildWnd@@IAEHPAVCWnd@@II@Z 5f869ee6 f
 0001:00068f1d       ?OnToolTipText@CMDIChildWnd@@IAEHIPAUtagNMHDR@@PAJ@Z 5f869f1d f
 0001:00068fbe       ?SetHandles@CMDIChildWnd@@QAEXPAUHMENU__@@PAUHACCEL__@@@Z 5f869fbe f
 0001:00068fd9       ?OnUpdateFrameMenu@CMDIFrameWnd@@UAEXPAUHMENU__@@@Z 5f869fd9 f
 0001:000690d3       ?OnUpdateMDIWindowCmd@CMDIFrameWnd@@IAEXPAVCCmdUI@@@Z 5f86a0d3 f
 0001:000690f2       ?OnMDIWindowCmd@CMDIFrameWnd@@IAEHI@Z 5f86a0f2 f
 0001:00069138       ?OnWindowNew@CMDIFrameWnd@@IAEXXZ 5f86a138 f
 0001:00069187       ?GetMessageMap@CMiniFrameWnd@@MBEPBUAFX_MSGMAP@@XZ 5f86a187 f
 0001:0006918d       ??0CMiniFrameWnd@@QAE@XZ   5f86a18d f
 0001:000691d7       ??_GCMiniFrameWnd@@UAEPAXI@Z 5f86a1d7 f
 0001:000691d7       ??_ECMiniFrameWnd@@UAEPAXI@Z 5f86a1d7 f
 0001:000691f3       ?Initialize@CMiniFrameWnd@@SAXXZ 5f86a1f3 f
 0001:0006937d       ?Create@CMiniFrameWnd@@QAEHPBG0KABUtagRECT@@PAVCWnd@@I@Z 5f86a37d f
 0001:0006939d       ?CreateEx@CMiniFrameWnd@@QAEHKPBG0KABUtagRECT@@PAVCWnd@@I@Z 5f86a39d f
 0001:00069410       ?OnNcCreate@CMiniFrameWnd@@QAEHPAUtagCREATESTRUCTW@@@Z 5f86a410 f
 0001:00069498       ?PreCreateWindow@CMiniFrameWnd@@MAEHAAUtagCREATESTRUCTW@@@Z 5f86a498 f
 0001:000694d1       ?OnGetMinMaxInfo@CMiniFrameWnd@@QAEXPAUtagMINMAXINFO@@@Z 5f86a4d1 f
 0001:00069519       ?OnNcActivate@CMiniFrameWnd@@QAEHH@Z 5f86a519 f
 0001:0006956a       ?OnNcCalcSize@CMiniFrameWnd@@QAEXHPAUtagNCCALCSIZE_PARAMS@@@Z 5f86a56a f
 0001:000695d0       ?OnNcHitTest@CMiniFrameWnd@@QAEIVCPoint@@@Z 5f86a5d0 f
 0001:000698df       ?OnNcLButtonDown@CMiniFrameWnd@@QAEXIVCPoint@@@Z 5f86a8df f
 0001:00069924       ?OnMouseMove@CMiniFrameWnd@@QAEXIVCPoint@@@Z 5f86a924 f
 0001:000699ab       ?OnLButtonUp@CMiniFrameWnd@@QAEXIVCPoint@@@Z 5f86a9ab f
 0001:00069a0b       ?InvertSysMenu@CMiniFrameWnd@@IAEXXZ 5f86aa0b f
 0001:00069aa3       ?_AfxDrawFrame@@YGXPAVCDC@@PBUtagRECT@@HHAAVCBrush@@@Z 5f86aaa3 f
 0001:00069b60       ?OnNcPaint@CMiniFrameWnd@@QAEXXZ 5f86ab60 f
 0001:0006a0dd       ?OnSysCommand@CMiniFrameWnd@@QAEXIJ@Z 5f86b0dd f
 0001:0006a145       ?CalcWindowRect@CMiniFrameWnd@@UAEXPAUtagRECT@@I@Z 5f86b145 f
 0001:0006a1ad       ?CalcBorders@CMiniFrameWnd@@SGXPAUtagRECT@@KK@Z 5f86b1ad f
 0001:0006a219       ?OnGetText@CMiniFrameWnd@@QAEJIJ@Z 5f86b219 f
 0001:0006a254       ?OnGetTextLength@CMiniFrameWnd@@QAEJIJ@Z 5f86b254 f
 0001:0006a270       ?OnSetText@CMiniFrameWnd@@QAEJIJ@Z 5f86b270 f
 0001:0006a2f7       ?OnFloatStatus@CMiniFrameWnd@@QAEJIJ@Z 5f86b2f7 f
 0001:0006a3a1       ?OnQueryCenterWnd@CMiniFrameWnd@@QAEJIJ@Z 5f86b3a1 f
 0001:0006a3c7       ??0CRectTracker@@QAE@PBUtagRECT@@I@Z 5f86b3c7 f
 0001:0006a3f0       ?Construct@CRectTracker@@IAEXXZ 5f86b3f0 f
 0001:0006a57e       ?Draw@CRectTracker@@QBEXPAVCDC@@@Z 5f86b57e f
 0001:0006a7eb       ?SetCursor@CRectTracker@@QBEHPAVCWnd@@I@Z 5f86b7eb f
 0001:0006a86b       ?HitTest@CRectTracker@@QBEHVCPoint@@@Z 5f86b86b f
 0001:0006a8b7       ?NormalizeHit@CRectTracker@@QBEHH@Z 5f86b8b7 f
 0001:0006a8f5       ?Track@CRectTracker@@QAEHPAVCWnd@@VCPoint@@H0@Z 5f86b8f5 f
 0001:0006a92d       ?TrackRubberBand@CRectTracker@@QAEHPAVCWnd@@VCPoint@@H@Z 5f86b92d f
 0001:0006a968       ?DrawTrackerRect@CRectTracker@@UAEXPBUtagRECT@@PAVCWnd@@PAVCDC@@1@Z 5f86b968 f
 0001:0006aa3b       ?AdjustRect@CRectTracker@@UAEXHPAUtagRECT@@@Z 5f86ba3b f
 0001:0006ab2e       ?GetTrueRect@CRectTracker@@QBEXPAUtagRECT@@@Z 5f86bb2e f
 0001:0006ab80       ?GetHandleRect@CRectTracker@@IBEXHPAVCRect@@@Z 5f86bb80 f
 0001:0006ac4c       ?GetHandleSize@CRectTracker@@MBEHPBUtagRECT@@@Z 5f86bc4c f
 0001:0006acac       ?HitTestHandles@CRectTracker@@IBEHVCPoint@@@Z 5f86bcac f
 0001:0006ad6b       ?TrackHandle@CRectTracker@@IAEHHPAVCWnd@@VCPoint@@0@Z 5f86bd6b f
 0001:0006aff5       ?GetModifyPointers@CRectTracker@@IAEXHPAPAH0PAH1@Z 5f86bff5 f
 0001:0006b09b       ?GetHandleMask@CRectTracker@@UBEIXZ 5f86c09b f
 0001:0006b0dd       ?Create@CStatic@@QAEHPBGKABUtagRECT@@PAVCWnd@@I@Z 5f86c0dd f
 0001:0006b0ff       ?Create@CButton@@QAEHPBGKABUtagRECT@@PAVCWnd@@I@Z 5f86c0ff f
 0001:0006b121       ?GetCheckedRadioButton@CWnd@@QAEHHH@Z 5f86c121 f
 0001:0006b149       ?Create@CListBox@@QAEHKABUtagRECT@@PAVCWnd@@I@Z 5f86c149 f
 0001:0006b16a       ?CharToItem@CListBox@@UAEHII@Z 5f86c16a f
 0001:0006b172       ?OnChildNotify@CListBox@@MAEHIIJPAJ@Z 5f86c172 f
 0001:0006b20f       ?GetText@CListBox@@QBEXHAAVCString@@@Z 5f86c20f f
 0001:0006b252       ?ItemFromPoint@CListBox@@QBEIVCPoint@@AAH@Z 5f86c252 f
 0001:0006b28a       ?CompareItem@CComboBox@@UAEHPAUtagCOMPAREITEMSTRUCT@@@Z 5f86c28a f
 0001:0006b2b4       ?Create@CEdit@@QAEHKABUtagRECT@@PAVCWnd@@I@Z 5f86c2b4 f
 0001:0006b2d5       ?Create@CScrollBar@@QAEHKABUtagRECT@@PAVCWnd@@I@Z 5f86c2d5 f
 0001:0006b2f6       ??1CScrollBar@@UAE@XZ      5f86c2f6 f
 0001:0006b32e       ??0_AFX_CHECKLIST_STATE@@QAE@XZ 5f86c32e f
 0001:0006b3d0       ??_G_AFX_CHECKLIST_STATE@@UAEPAXI@Z 5f86c3d0 f
 0001:0006b3d0       ??_E_AFX_CHECKLIST_STATE@@UAEPAXI@Z 5f86c3d0 f
 0001:0006b3eb       ??1_AFX_CHECKLIST_STATE@@UAE@XZ 5f86c3eb f
 0001:0006b400       ?GetMessageMap@CCheckListBox@@MBEPBUAFX_MSGMAP@@XZ 5f86c400 f
 0001:0006b406       ?Create@CCheckListBox@@QAEHKABUtagRECT@@PAVCWnd@@I@Z 5f86c406 f
 0001:0006b428       ?SetCheckStyle@CCheckListBox@@QAEXI@Z 5f86c428 f
 0001:0006b432       ?SetCheck@CCheckListBox@@QAEXHH@Z 5f86c432 f
 0001:0006b4ad       ?GetCheck@CCheckListBox@@QAEHH@Z 5f86c4ad f
 0001:0006b4d2       ?Enable@CCheckListBox@@QAEXHH@Z 5f86c4d2 f
 0001:0006b539       ?IsEnabled@CCheckListBox@@QAEHH@Z 5f86c539 f
 0001:0006b560       ?OnGetCheckPosition@CCheckListBox@@UAE?AVCRect@@V2@0@Z 5f86c560 f
 0001:0006b575       ?DrawItem@CCheckListBox@@UAEXPAUtagDRAWITEMSTRUCT@@@Z 5f86c575 f
 0001:0006b6ee       ?PreDrawItem@CCheckListBox@@IAEXPAUtagDRAWITEMSTRUCT@@@Z 5f86c6ee f
 0001:0006b983       ?PreMeasureItem@CCheckListBox@@IAEXPAUtagMEASUREITEMSTRUCT@@@Z 5f86c983 f
 0001:0006ba0e       ?PreCompareItem@CCheckListBox@@IAEHPAUtagCOMPAREITEMSTRUCT@@@Z 5f86ca0e f
 0001:0006ba5f       ?PreDeleteItem@CCheckListBox@@IAEXPAUtagDELETEITEMSTRUCT@@@Z 5f86ca5f f
 0001:0006bac8       ?OnChildNotify@CCheckListBox@@MAEHIIJPAJ@Z 5f86cac8 f
 0001:0006bb23       ?CalcMinimumItemHeight@CCheckListBox@@IAEHXZ 5f86cb23 f
 0001:0006bbbe       ?InvalidateCheck@CCheckListBox@@IAEXH@Z 5f86cbbe f
 0001:0006bc10       ?InvalidateItem@CCheckListBox@@IAEXH@Z 5f86cc10 f
 0001:0006bc42       ?CheckFromPoint@CCheckListBox@@IAEHVCPoint@@AAH@Z 5f86cc42 f
 0001:0006bd3e       ?SetSelectionCheck@CCheckListBox@@IAEXH@Z 5f86cd3e f
 0001:0006bdb6       ?OnLButtonDown@CCheckListBox@@IAEXIVCPoint@@@Z 5f86cdb6 f
 0001:0006beb3       ?OnLButtonDblClk@CCheckListBox@@IAEXIVCPoint@@@Z 5f86ceb3 f
 0001:0006beed       ?OnKeyDown@CCheckListBox@@IAEXIII@Z 5f86ceed f
 0001:0006c05d       ?OnCreate@CCheckListBox@@IAEHPAUtagCREATESTRUCTW@@@Z 5f86d05d f
 0001:0006c09d       ?OnSetFont@CCheckListBox@@IAEJIJ@Z 5f86d09d f
 0001:0006c0d4       ?OnLBAddString@CCheckListBox@@IAEJIJ@Z 5f86d0d4 f
 0001:0006c13c       ?OnLBFindString@CCheckListBox@@IAEJIJ@Z 5f86d13c f
 0001:0006c1bd       ?OnLBFindStringExact@CCheckListBox@@IAEJIJ@Z 5f86d1bd f
 0001:0006c23e       ?OnLBGetItemData@CCheckListBox@@IAEJIJ@Z 5f86d23e f
 0001:0006c262       ?OnLBGetText@CCheckListBox@@IAEJIJ@Z 5f86d262 f
 0001:0006c28b       ?OnLBInsertString@CCheckListBox@@IAEJIJ@Z 5f86d28b f
 0001:0006c2f3       ?OnLBSelectString@CCheckListBox@@IAEJIJ@Z 5f86d2f3 f
 0001:0006c383       ?OnLBSetItemData@CCheckListBox@@IAEJIJ@Z 5f86d383 f
 0001:0006c3f7       ?OnLBSetItemHeight@CCheckListBox@@IAEJIJ@Z 5f86d3f7 f
 0001:0006c430       ?AfxPropPageCallback@@YGIPAUHWND__@@IPAU_PROPSHEETPAGEW@@@Z 5f86d430 f
 0001:0006c47e       ?_GetBaseMessageMap@CPropertyPage@@KGPBUAFX_MSGMAP@@XZ 5f86d47e f
 0001:0006c484       ?GetMessageMap@CPropertyPage@@MBEPBUAFX_MSGMAP@@XZ 5f86d484 f
 0001:0006c48a       ??0CPropertyPage@@QAE@II@Z 5f86d48a f
 0001:0006c4d9       ??_GCPropertyPage@@UAEPAXI@Z 5f86d4d9 f
 0001:0006c4d9       ??_ECPropertyPage@@UAEPAXI@Z 5f86d4d9 f
 0001:0006c4f5       ??0CPropertyPage@@QAE@PBGI@Z 5f86d4f5 f
 0001:0006c542       ?Construct@CPropertyPage@@QAEXII@Z 5f86d542 f
 0001:0006c554       ?Construct@CPropertyPage@@QAEXPBGI@Z 5f86d554 f
 0001:0006c564       ??0CPropertyPage@@QAE@XZ   5f86d564 f
 0001:0006c5ad       ?CommonConstruct@CPropertyPage@@IAEXPBGI@Z 5f86d5ad f
 0001:0006c64b       ?Cleanup@CPropertyPage@@IAEXXZ 5f86d64b f
 0001:0006c67c       ?_AfxChangePropPageFont@@YGPAUDLGTEMPLATE@@PBU1@H@Z 5f86d67c f
 0001:0006c761       ?InitDialogInfo@CPropertyPage@@IAEPBUDLGTEMPLATE@@PBU2@@Z 5f86d761 f
 0001:0006c792       ?PreProcessPageTemplate@CPropertyPage@@IAEXAAU_PROPSHEETPAGEW@@H@Z 5f86d792 f
 0001:0006c819       ?CancelToClose@CPropertyPage@@QAEXXZ 5f86d819 f
 0001:0006c83b       ?SetModified@CPropertyPage@@QAEXH@Z 5f86d83b f
 0001:0006c877       ?QuerySiblings@CPropertyPage@@QAEJIJ@Z 5f86d877 f
 0001:0006c89f       ?OnApply@CPropertyPage@@UAEHXZ 5f86d89f f
 0001:0006c8ab       ?OnReset@CPropertyPage@@UAEXXZ 5f86d8ab f
 0001:0006c8b3       ?OnSetActive@CPropertyPage@@UAEHXZ 5f86d8b3 f
 0001:0006c8cd       ?OnKillActive@CPropertyPage@@UAEHXZ 5f86d8cd f
 0001:0006c8db       ?OnQueryCancel@CPropertyPage@@UAEHXZ 5f86d8db f
 0001:0006c8df       ?OnWizardNext@CPropertyPage@@UAEJXZ 5f86d8df f
 0001:0006c8e2       ?MapWizardResult@CPropertyPage@@IAEJJ@Z 5f86d8e2 f
 0001:0006c95c       ?IsButtonEnabled@CPropertyPage@@IAEHH@Z 5f86d95c f
 0001:0006c97e       ?OnNotify@CPropertyPage@@MAEHIJPAJ@Z 5f86d97e f
 0001:0006caf6       ?PreTranslateMessage@CPropertyPage@@MAEHPAUtagMSG@@@Z 5f86daf6 f
 0001:0006cb04       ?OnCtlColor@CPropertyPage@@IAEPAUHBRUSH__@@PAVCDC@@PAVCWnd@@I@Z 5f86db04 f
 0001:0006cb75       ?EndDialog@CPropertyPage@@QAEXH@Z 5f86db75 f
 0001:0006cba3       ?GetMessageMap@CPropertySheet@@MBEPBUAFX_MSGMAP@@XZ 5f86dba3 f
 0001:0006cba9       ?GetPropSheetHeader@CPropertySheet@@QAEPAU_AFX_OLDPROPSHEETHEADER@@XZ 5f86dba9 f
 0001:0006cbc9       ?OnSetDefID@CPropertySheet@@IAEJIJ@Z 5f86dbc9 f
 0001:0006cc97       ??0CPropertySheet@@QAE@XZ  5f86dc97 f
 0001:0006cce9       ??_ECPropertySheet@@UAEPAXI@Z 5f86dce9 f
 0001:0006cce9       ??_GCPropertySheet@@UAEPAXI@Z 5f86dce9 f
 0001:0006cd05       ??0CPropertySheet@@QAE@IPAVCWnd@@I@Z 5f86dd05 f
 0001:0006cd69       ??0CPropertySheet@@QAE@PBGPAVCWnd@@I@Z 5f86dd69 f
 0001:0006cdcd       ?Construct@CPropertySheet@@QAEXIPAVCWnd@@I@Z 5f86ddcd f
 0001:0006cdef       ?Construct@CPropertySheet@@QAEXPBGPAVCWnd@@I@Z 5f86ddef f
 0001:0006ce11       ?CommonConstruct@CPropertySheet@@QAEXPAVCWnd@@I@Z 5f86de11 f
 0001:0006ce6c       ?EnableStackedTabs@CPropertySheet@@QAEXH@Z 5f86de6c f
 0001:0006ce79       ?SetTitle@CPropertySheet@@QAEXPBGI@Z 5f86de79 f
 0001:0006cec5       ?PreTranslateMessage@CPropertySheet@@UAEHPAUtagMSG@@@Z 5f86dec5 f
 0001:0006cf26       ?OnCmdMsg@CPropertySheet@@UAEHIHPAXPAUAFX_CMDHANDLERINFO@@@Z 5f86df26 f
 0001:0006cfab       ?GetActivePage@CPropertySheet@@QBEPAVCPropertyPage@@XZ 5f86dfab f
 0001:0006cfdc       ?ContinueModal@CPropertySheet@@UAEHXZ 5f86dfdc f
 0001:0006cffe       ?DoModal@CPropertySheet@@UAEHXZ 5f86dffe f
 0001:0006d172       ?AfxPropSheetCallback@@YGHPAUHWND__@@IJ@Z 5f86e172 f
 0001:0006d1c9       ?Create@CPropertySheet@@QAEHPAVCWnd@@KK@Z 5f86e1c9 f
 0001:0006d288       ?BuildPropPageArray@CPropertySheet@@UAEXXZ 5f86e288 f
 0001:0006d2ff       ?GetPageCount@CPropertySheet@@QBEHXZ 5f86e2ff f
 0001:0006d321       ?GetActiveIndex@CPropertySheet@@QBEHXZ 5f86e321 f
 0001:0006d348       ?SetActivePage@CPropertySheet@@QAEHH@Z 5f86e348 f
 0001:0006d375       ?GetPageIndex@CPropertySheet@@QAEHPAVCPropertyPage@@@Z 5f86e375 f
 0001:0006d3a8       ?SetActivePage@CPropertySheet@@QAEHPAVCPropertyPage@@@Z 5f86e3a8 f
 0001:0006d3c0       ?AddPage@CPropertySheet@@QAEXPAVCPropertyPage@@@Z 5f86e3c0 f
 0001:0006d482       ?RemovePage@CPropertySheet@@QAEXPAVCPropertyPage@@@Z 5f86e482 f
 0001:0006d49a       ?RemovePage@CPropertySheet@@QAEXH@Z 5f86e49a f
 0001:0006d4c8       ?EndDialog@CPropertySheet@@QAEXH@Z 5f86e4c8 f
 0001:0006d4fc       ?OnClose@CPropertySheet@@IAEXXZ 5f86e4fc f
 0001:0006d515       ?OnSysCommand@CPropertySheet@@IAEXIJ@Z 5f86e515 f
 0001:0006d54d       ?OnInitDialog@CPropertySheet@@UAEHXZ 5f86e54d f
 0001:0006d728       ?OnNcCreate@CPropertySheet@@IAEHPAUtagCREATESTRUCTW@@@Z 5f86e728 f
 0001:0006d744       ?HandleInitDialog@CPropertySheet@@IAEJIJ@Z 5f86e744 f
 0001:0006d74f       ?OnCommand@CPropertySheet@@UAEHIJ@Z 5f86e74f f
 0001:0006d7c0       ?OnCommandHelp@CPropertySheet@@IAEJIJ@Z 5f86e7c0 f
 0001:0006d7de       ?OnCtlColor@CPropertySheet@@IAEPAUHBRUSH__@@PAVCDC@@PAVCWnd@@I@Z 5f86e7de f
 0001:0006d84f       ??0CPropertyPageEx@@QAE@IIII@Z 5f86e84f f
 0001:0006d8b3       ??_ECPropertyPageEx@@UAEPAXI@Z 5f86e8b3 f
 0001:0006d8b3       ??_GCPropertyPageEx@@UAEPAXI@Z 5f86e8b3 f
 0001:0006d8cf       ??1CPropertyPageEx@@UAE@XZ 5f86e8cf f
 0001:0006d919       ??0CPropertyPageEx@@QAE@PBGIII@Z 5f86e919 f
 0001:0006d97b       ?Construct@CPropertyPageEx@@QAEXIIII@Z 5f86e97b f
 0001:0006d995       ?Construct@CPropertyPageEx@@QAEXPBGIII@Z 5f86e995 f
 0001:0006d9ad       ??0CPropertyPageEx@@QAE@XZ 5f86e9ad f
 0001:0006da08       ?CommonConstruct@CPropertyPageEx@@IAEXPBGIII@Z 5f86ea08 f
 0001:0006dacf       ??0CPropertySheetEx@@QAE@XZ 5f86eacf f
 0001:0006db0b       ??_GCPropertySheetEx@@UAEPAXI@Z 5f86eb0b f
 0001:0006db0b       ??_ECPropertySheetEx@@UAEPAXI@Z 5f86eb0b f
 0001:0006db27       ??0CPropertySheetEx@@QAE@IPAVCWnd@@IPAUHBITMAP__@@PAUHPALETTE__@@1@Z 5f86eb27 f
 0001:0006db79       ??0CPropertySheetEx@@QAE@PBGPAVCWnd@@IPAUHBITMAP__@@PAUHPALETTE__@@2@Z 5f86eb79 f
 0001:0006dbcb       ?Construct@CPropertySheetEx@@QAEXIPAVCWnd@@IPAUHBITMAP__@@PAUHPALETTE__@@1@Z 5f86ebcb f
 0001:0006dbf7       ?Construct@CPropertySheetEx@@QAEXPBGPAVCWnd@@IPAUHBITMAP__@@PAUHPALETTE__@@2@Z 5f86ebf7 f
 0001:0006dc23       ?CommonConstruct@CPropertySheetEx@@QAEXPAVCWnd@@IPAUHBITMAP__@@PAUHPALETTE__@@1@Z 5f86ec23 f
 0001:0006dcce       ?BuildPropPageArray@CPropertySheetEx@@UAEXXZ 5f86ecce f
 0001:0006dd9e       ??1CPropertySheetEx@@UAE@XZ 5f86ed9e f
 0001:0006dddd       ?AddPage@CPropertySheetEx@@QAEXPAVCPropertyPageEx@@@Z 5f86eddd f
 0001:0006ded0       ?DPtoHIMETRIC@CDC@@QBEXPAUtagSIZE@@@Z 5f86eed0 f
 0001:0006df5e       ?HIMETRICtoDP@CDC@@QBEXPAUtagSIZE@@@Z 5f86ef5e f
 0001:0006dfec       ?LPtoHIMETRIC@CDC@@QBEXPAUtagSIZE@@@Z 5f86efec f
 0001:0006e007       ?HIMETRICtoLP@CDC@@QBEXPAUtagSIZE@@@Z 5f86f007 f
 0001:0006e022       ?GetHalftoneBrush@CDC@@SGPAVCBrush@@XZ 5f86f022 f
 0001:0006e095       ?DrawDragRect@CDC@@QAEXPBUtagRECT@@UtagSIZE@@01PAVCBrush@@2@Z 5f86f095 f
 0001:0006e3aa       ?FillSolidRect@CDC@@QAEXPBUtagRECT@@K@Z 5f86f3aa f
 0001:0006e3d4       ?Draw3dRect@CDC@@QAEXPBUtagRECT@@KK@Z 5f86f3d4 f
 0001:0006e3ff       ?Draw3dRect@CDC@@QAEXHHHHKK@Z 5f86f3ff f
 0001:0006e469       ?CreatePointFont@CFont@@QAEHHPBGPAVCDC@@@Z 5f86f469 f
 0001:0006e4ae       ?CreatePointFontIndirect@CFont@@QAEHPBUtagLOGFONTW@@PAVCDC@@@Z 5f86f4ae f
 0001:0006e553       ?NormalizeRect@CRect@@QAEXXZ 5f86f553 f
 0001:0006e572       ?InflateRect@CRect@@QAEXPBUtagRECT@@@Z 5f86f572 f
 0001:0006e58f       ?InflateRect@CRect@@QAEXHHHH@Z 5f86f58f f
 0001:0006e5ad       ?DeflateRect@CRect@@QAEXPBUtagRECT@@@Z 5f86f5ad f
 0001:0006e5ca       ?DeflateRect@CRect@@QAEXHHHH@Z 5f86f5ca f
 0001:0006e5e8       ?MulDiv@CRect@@QBE?AV1@HH@Z 5f86f5e8 f
 0001:0006e650       ?GetMessageMap@CEditView@@MBEPBUAFX_MSGMAP@@XZ 5f86f650 f
 0001:0006e656       ??_E_AFX_EDIT_STATE@@UAEPAXI@Z 5f86f656 f
 0001:0006e656       ??_G_AFX_EDIT_STATE@@UAEPAXI@Z 5f86f656 f
 0001:0006e671       ??0CEditView@@QAE@XZ       5f86f671 f
 0001:0006e6c4       ??_GCEditView@@UAEPAXI@Z   5f86f6c4 f
 0001:0006e6c4       ??_ECEditView@@UAEPAXI@Z   5f86f6c4 f
 0001:0006e6e0       ??1CEditView@@UAE@XZ       5f86f6e0 f
 0001:0006e73a       ?PreCreateWindow@CEditView@@MAEHAAUtagCREATESTRUCTW@@@Z 5f86f73a f
 0001:0006e74d       ?OnCreate@CEditView@@IAEHPAUtagCREATESTRUCTW@@@Z 5f86f74d f
 0001:0006e831       ?OnDestroy@CEditView@@IAEXXZ 5f86f831 f
 0001:0006e850       ?CalcWindowRect@CEditView@@MAEXPAUtagRECT@@I@Z 5f86f850 f
 0001:0006e8ac       ?DeleteContents@CEditView@@UAEXXZ 5f86f8ac f
 0001:0006e8b4       ?Serialize@CEditView@@UAEXAAVCArchive@@@Z 5f86f8b4 f
 0001:0006e90c       ?ReadFromArchive@CEditView@@QAEXAAVCArchive@@I@Z 5f86f90c f
 0001:0006e9a5       ?WriteToArchive@CEditView@@QAEXAAVCArchive@@@Z 5f86f9a5 f
 0001:0006ea08       ?SerializeRaw@CEditView@@QAEXAAVCArchive@@@Z 5f86fa08 f
 0001:0006ea59       ?_AfxEndOfLine@@YGIPBGII@Z 5f86fa59 f
 0001:0006ea80       ?_AfxNextLine@@YGIPBGII@Z  5f86fa80 f
 0001:0006eab5       ?_AfxClipLine@@YGIPAVCDC@@QAHHHPBGII@Z 5f86fab5 f
 0001:0006ebae       ?OnPreparePrinting@CEditView@@MAEHPAUCPrintInfo@@@Z 5f86fbae f
 0001:0006ebba       ?OnBeginPrinting@CEditView@@MAEXPAVCDC@@PAUCPrintInfo@@@Z 5f86fbba f
 0001:0006ec9d       ?PaginateTo@CEditView@@IAEHPAVCDC@@PAUCPrintInfo@@@Z 5f86fc9d f
 0001:0006ed70       ?OnPrepareDC@CEditView@@UAEXPAVCDC@@PAUCPrintInfo@@@Z 5f86fd70 f
 0001:0006ed92       ?PrintInsideRect@CEditView@@QAEIPAVCDC@@AAUtagRECT@@II@Z 5f86fd92 f
 0001:0006f079       ?OnPrint@CEditView@@MAEXPAVCDC@@PAUCPrintInfo@@@Z 5f870079 f
 0001:0006f10e       ?OnEndPrinting@CEditView@@MAEXPAVCDC@@PAUCPrintInfo@@@Z 5f87010e f
 0001:0006f13a       ?OnUpdateNeedSel@CEditView@@IAEXPAVCCmdUI@@@Z 5f87013a f
 0001:0006f16e       ?OnUpdateNeedClip@CEditView@@IAEXPAVCCmdUI@@@Z 5f87016e f
 0001:0006f188       ?OnUpdateNeedText@CEditView@@IAEXPAVCCmdUI@@@Z 5f870188 f
 0001:0006f1a5       ?OnUpdateNeedFind@CEditView@@IAEXPAVCCmdUI@@@Z 5f8701a5 f
 0001:0006f1e3       ?OnEditChange@CEditView@@IAEHXZ 5f8701e3 f
 0001:0006f1f0       ?OnEditCut@CEditView@@IAEXXZ 5f8701f0 f
 0001:0006f203       ?OnEditCopy@CEditView@@IAEXXZ 5f870203 f
 0001:0006f216       ?OnEditPaste@CEditView@@IAEXXZ 5f870216 f
 0001:0006f229       ?OnEditUndo@CEditView@@IAEXXZ 5f870229 f
 0001:0006f23c       ?OnEditSelectAll@CEditView@@IAEXXZ 5f87023c f
 0001:0006f265       ?OnSetFont@CEditView@@IAEJIJ@Z 5f870265 f
 0001:0006f287       ?SetPrinterFont@CEditView@@QAEXPAVCFont@@@Z 5f870287 f
 0001:0006f298       ?GetPrinterFont@CEditView@@QBEPAVCFont@@XZ 5f870298 f
 0001:0006f2a1       ?LockBuffer@CEditView@@QBEPBGXZ 5f8702a1 f
 0001:0006f2bb       ?UnlockBuffer@CEditView@@QBEXXZ 5f8702bb f
 0001:0006f2d5       ?GetBufferLength@CEditView@@QBEIXZ 5f8702d5 f
 0001:0006f2f3       ?GetSelectedText@CEditView@@QBEXAAVCString@@@Z 5f8702f3 f
 0001:0006f360       ?OnEditFind@CEditView@@IAEXXZ 5f870360 f
 0001:0006f368       ?OnEditReplace@CEditView@@IAEXXZ 5f870368 f
 0001:0006f370       ?OnEditRepeat@CEditView@@IAEXXZ 5f870370 f
 0001:0006f3aa       ?OnEditFindReplace@CEditView@@IAEXH@Z 5f8703aa f
 0001:0006f4e2       ?OnFindNext@CEditView@@MAEXPBGHH@Z 5f8704e2 f
 0001:0006f536       ?OnReplaceSel@CEditView@@MAEXPBGHH0@Z 5f870536 f
 0001:0006f5ad       ?OnReplaceAll@CEditView@@MAEXPBG0H@Z 5f8705ad f
 0001:0006f637       ?InitializeReplace@CEditView@@IAEHXZ 5f870637 f
 0001:0006f6b3       ?OnFindReplaceCmd@CEditView@@IAEJIJ@Z 5f8706b3 f
 0001:0006f7f3       ?SameAsSelected@CEditView@@IAEHPBGH@Z 5f8707f3 f
 0001:0006f88d       ?FindTextW@CEditView@@QAEHPBGHH@Z 5f87088d f
 0001:0006fa4a       ?OnTextNotFound@CEditView@@MAEXPBG@Z 5f870a4a f
 0001:0006fa55       ?SetTabStops@CEditView@@QAEXH@Z 5f870a55 f
 0001:0006fa83       ?GetMessageMap@CListView@@MBEPBUAFX_MSGMAP@@XZ 5f870a83 f
 0001:0006fa89       ?PreCreateWindow@CListView@@UAEHAAUtagCREATESTRUCTW@@@Z 5f870a89 f
 0001:0006fa95       ?OnChildNotify@CListView@@MAEHIIJPAJ@Z 5f870a95 f
 0001:0006fac3       ?RemoveImageList@CListView@@IAEXH@Z 5f870ac3 f
 0001:0006fafc       ?OnNcDestroy@CListView@@QAEXXZ 5f870afc f
 0001:0006fb21       ?GetMessageMap@CTreeView@@MBEPBUAFX_MSGMAP@@XZ 5f870b21 f
 0001:0006fb27       ?RemoveImageList@CTreeView@@IAEXH@Z 5f870b27 f
 0001:0006fb60       ?OnDestroy@CTreeView@@QAEXXZ 5f870b60 f
 0001:0006fbc9       ??0CReObject@@QAE@XZ       5f870bc9 f
 0001:0006fbe6       ??0CReObject@@QAE@PAVCRichEditCntrItem@@@Z 5f870be6 f
 0001:0006fc4b       ?GetMessageMap@CRichEditView@@MBEPBUAFX_MSGMAP@@XZ 5f870c4b f
 0001:0006fc51       ??1CRichEditView@@UAE@XZ   5f870c51 f
 0001:0006fd8f       ?PrintInsideRect@CRichEditView@@QAEJPAVCDC@@AAUtagRECT@@JJH@Z 5f870d8f f
 0001:0006fe64       ?_GetBaseInterfaceMap@CRichEditView@@KGPBUAFX_INTERFACEMAP@@XZ 5f870e64 f
 0001:0006fe6a       ?GetInterfaceMap@CRichEditView@@MBEPBUAFX_INTERFACEMAP@@XZ 5f870e6a f
 0001:0006fe70       ?QueryInterface@XRichEditOleCallback@CRichEditView@@UAGJABU_GUID@@PAPAX@Z 5f870e70 f
 0001:0006fe8a       ?GetNewStorage@XRichEditOleCallback@CRichEditView@@UAGJPAPAUIStorage@@@Z 5f870e8a f
 0001:0006fefe       ?GetInPlaceContext@XRichEditOleCallback@CRichEditView@@UAGJPAPAUIOleInPlaceFrame@@PAPAUIOleInPlaceUIWindow@@PAUtagOIFI@@@Z 5f870efe f
 0001:0006ff4e       ?ShowContainerUI@XRichEditOleCallback@CRichEditView@@UAGJH@Z 5f870f4e f
 0001:0006ff98       ?QueryInsertObject@XRichEditOleCallback@CRichEditView@@UAGJPAU_GUID@@PAUIStorage@@J@Z 5f870f98 f
 0001:0006ffcf       ?DeleteObject@XRichEditOleCallback@CRichEditView@@UAGJPAUIOleObject@@@Z 5f870fcf f
 0001:0006ffe8       ?QueryAcceptData@XRichEditOleCallback@CRichEditView@@UAGJPAUIDataObject@@PAGKHPAX@Z 5f870fe8 f
 0001:00070041       ?ContextSensitiveHelp@XRichEditOleCallback@CRichEditView@@UAGJH@Z 5f871041 f
 0001:00070049       ?GetClipboardData@XRichEditOleCallback@CRichEditView@@UAGJPAU_charrange@@KPAPAUIDataObject@@@Z 5f871049 f
 0001:000700df       ?GetDragDropEffect@XRichEditOleCallback@CRichEditView@@UAGJHKPAK@Z 5f8710df f
 0001:00070116       ?GetContextMenu@XRichEditOleCallback@CRichEditView@@UAGJGPAUIOleObject@@PAU_charrange@@PAPAUHMENU__@@@Z 5f871116 f
 0001:0007017b       ?OnCharEffect@CRichEditView@@QAEXKK@Z 5f87117b f
 0001:000701ce       ?OnParaAlign@CRichEditView@@QAEXG@Z 5f8711ce f
 0001:00070206       ?OnUpdateNeedFind@CRichEditView@@IAEXPAVCCmdUI@@@Z 5f871206 f
 0001:0007024c       ?OnEditPaste@CRichEditView@@IAEXXZ 5f87124c f
 0001:00070262       ?OnEditClear@CRichEditView@@IAEXXZ 5f871262 f
 0001:00070275       ?OnEditUndo@CRichEditView@@IAEXXZ 5f871275 f
 0001:0007029b       ?OnEditSelectAll@CRichEditView@@IAEXXZ 5f87129b f
 0001:000702a5       ?OnEditFind@CRichEditView@@IAEXXZ 5f8712a5 f
 0001:000702ad       ?OnEditReplace@CRichEditView@@IAEXXZ 5f8712ad f
 0001:000702b5       ?OnEditRepeat@CRichEditView@@IAEXXZ 5f8712b5 f
 0001:000702e3       ?OnInsertObject@CRichEditView@@IAEXXZ 5f8712e3 f
 0001:00070400       ?OnEditProperties@CRichEditView@@IAEXXZ 5f871400 f
 0001:00070490       ?OnUpdateEditProperties@CRichEditView@@IAEXPAVCCmdUI@@@Z 5f871490 f
 0001:000704ad       ?OnCharBold@CRichEditView@@IAEXXZ 5f8714ad f
 0001:000704b7       ?OnCharItalic@CRichEditView@@IAEXXZ 5f8714b7 f
 0001:000704c1       ?OnCharUnderline@CRichEditView@@IAEXXZ 5f8714c1 f
 0001:000704cb       ?OnParaCenter@CRichEditView@@IAEXXZ 5f8714cb f
 0001:000704d3       ?OnParaLeft@CRichEditView@@IAEXXZ 5f8714d3 f
 0001:000704db       ?OnParaRight@CRichEditView@@IAEXXZ 5f8714db f
 0001:000704e3       ?OnBullet@CRichEditView@@IAEXXZ 5f8714e3 f
 0001:0007055e       ?OnFormatFont@CRichEditView@@IAEXXZ 5f87155e f
 0001:000705e1       ?OnColorPick@CRichEditView@@IAEXK@Z 5f8715e1 f
 0001:00070623       ?OnColorDefault@CRichEditView@@IAEXXZ 5f871623 f
 0001:00070659       ?OnEditPasteSpecial@CRichEditView@@IAEXXZ 5f871659 f
 0001:000707c1       ?OnDropFiles@CRichEditView@@IAEXPAUHDROP__@@@Z 5f8717c1 f
 0001:0007088a       ?OnDevModeChange@CRichEditView@@IAEXPAG@Z 5f87188a f
 0001:000708e2       ?IsRichEditFormat@CRichEditView@@SAHG@Z 5f8718e2 f
 0001:00070991       ?SetCharFormat@CRichEditView@@QAEXU_charformat@@@Z 5f871991 f
 0001:000709e4       ?SetParaFormat@CRichEditView@@QAEHAAU_paraformat@@@Z 5f8719e4 f
 0001:00070a3c       ?GetSelectedItem@CRichEditView@@QBEPAVCRichEditCntrItem@@XZ 5f871a3c f
 0001:00070ab0       ?GetInPlaceActiveItem@CRichEditView@@QBEPAVCRichEditCntrItem@@XZ 5f871ab0 f
 0001:00070b2a       ?InsertItem@CRichEditView@@QAEJPAVCRichEditCntrItem@@@Z 5f871b2a f
 0001:00070baa       ?InsertFileAsObject@CRichEditView@@QAEXPBG@Z 5f871baa f
 0001:00070c7a       ?DoPaste@CRichEditView@@QAEXAAVCOleDataObject@@GPAX@Z 5f871c7a f
 0001:00070e77       ?GetContextMenu@CRichEditView@@MAEPAUHMENU__@@GPAUIOleObject@@PAU_charrange@@@Z 5f871e77 f
 0001:00070e7c       ?GetClipboardData@CRichEditView@@MAEJPAU_charrange@@KPAUIDataObject@@PAPAU3@@Z 5f871e7c f
 0001:00070e84       ?QueryAcceptData@CRichEditView@@MAEJPAUIDataObject@@PAGKHPAX@Z 5f871e84 f
 0001:00070f50       ?GetWindowContext@CRichEditView@@QAEJPAPAUIOleInPlaceFrame@@PAPAUIOleInPlaceUIWindow@@PAUtagOIFI@@@Z 5f871f50 f
 0001:00070f85       ?ShowContainerUI@CRichEditView@@QAEJH@Z 5f871f85 f
 0001:00070fc1       ?AdjustDialogPosition@CRichEditView@@QAEXPAVCDialog@@@Z 5f871fc1 f
 0001:0007108b       ?OnEditFindReplace@CRichEditView@@IAEXH@Z 5f87208b f
 0001:000711dd       ?OnFindNext@CRichEditView@@MAEXPBGHHH@Z 5f8721dd f
 0001:0007123d       ?OnReplaceSel@CRichEditView@@MAEXPBGHHH0@Z 5f87223d f
 0001:000712ee       ?OnReplaceAll@CRichEditView@@MAEXPBG0HH@Z 5f8722ee f
 0001:000713e3       ?OnFindReplaceCmd@CRichEditView@@IAEJIJ@Z 5f8723e3 f
 0001:00071543       ?SameAsSelected@CRichEditView@@IAEHPBGHH@Z 5f872543 f
 0001:000715b2       ?FindTextW@CRichEditView@@QAEHPAV_AFX_RICHEDIT_STATE@@@Z 5f8725b2 f
 0001:000715c8       ?FindTextW@CRichEditView@@QAEHPBGHH@Z 5f8725c8 f
 0001:0007161a       ?FindTextSimple@CRichEditView@@QAEHPAV_AFX_RICHEDIT_STATE@@@Z 5f87261a f
 0001:00071630       ?FindTextSimple@CRichEditView@@QAEHPBGHH@Z 5f872630 f
 0001:00071746       ?FindAndSelect@CRichEditView@@QAEJKAAU_findtextexa@@@Z 5f872746 f
 0001:00071787       ?TextNotFound@CRichEditView@@QAEXPBG@Z 5f872787 f
 0001:0007179d       ?OnTextNotFound@CRichEditView@@MAEXPBG@Z 5f87279d f
 0001:000717a8       ?IsSelected@CRichEditView@@MBEHPBVCObject@@@Z 5f8727a8 f
 0001:000717bb       ??_GCRichEditDoc@@UAEPAXI@Z 5f8727bb f
 0001:000717bb       ??_ECRichEditDoc@@UAEPAXI@Z 5f8727bb f
 0001:000717d7       ??1CRichEditDoc@@UAE@XZ    5f8727d7 f
 0001:000717ea       ?GetInPlaceActiveItem@CRichEditDoc@@UAEPAVCOleClientItem@@PAVCWnd@@@Z 5f8727ea f
 0001:00071805       ?LookupItem@CRichEditDoc@@QBEPAVCRichEditCntrItem@@PAUIOleObject@@@Z 5f872805 f
 0001:00071850       ?CreateClientItem@CRichEditDoc@@UBEPAVCRichEditCntrItem@@PAU_reobject@@@Z 5f872850 f
 0001:0007188f       ?MarkItemsClear@CRichEditDoc@@IBEXXZ 5f87288f f
 0001:000718d5       ?DeleteUnmarkedItems@CRichEditDoc@@IBEXXZ 5f8728d5 f
 0001:00071936       ?UpdateObjectCache@CRichEditDoc@@IAEXXZ 5f872936 f
 0001:000719f9       ?GetPrimarySelectedItem@CRichEditDoc@@UAEPAVCOleClientItem@@PAVCView@@@Z 5f8729f9 f
 0001:00071a54       ??0CRichEditCntrItem@@QAE@PAU_reobject@@PAVCRichEditDoc@@@Z 5f872a54 f
 0001:00071ad1       ??1CRichEditCntrItem@@UAE@XZ 5f872ad1 f
 0001:00071b11       ?OnDeactivateUI@CRichEditCntrItem@@UAEXH@Z 5f872b11 f
 0001:00071b44       ?ShowContainerUI@CRichEditCntrItem@@QAEJH@Z 5f872b44 f
 0001:00071b91       ?CanActivate@CRichEditCntrItem@@UAEHXZ 5f872b91 f
 0001:00071bbd       ?GetWindowContext@CRichEditCntrItem@@QAEJPAPAUIOleInPlaceFrame@@PAPAUIOleInPlaceUIWindow@@PAUtagOIFI@@@Z 5f872bbd f
 0001:00071bf9       ?ConvertTo@CRichEditCntrItem@@UAEHABU_GUID@@@Z 5f872bf9 f
 0001:00071c83       ?ActivateAs@CRichEditCntrItem@@UAEHPBGABU_GUID@@1@Z 5f872c83 f
 0001:00071cab       ?SetDrawAspect@CRichEditCntrItem@@UAEXW4tagDVASPECT@@@Z 5f872cab f
 0001:00071cd7       ?SyncToRichEditObject@CRichEditCntrItem@@QAEXAAU_reobject@@@Z 5f872cd7 f
 0001:00071ce6       ?GetClientSite@CRichEditCntrItem@@UAEPAUIOleClientSite@@XZ 5f872ce6 f
 0001:00071d2e       ?OutputString@CDumpContext@@IAEXPBG@Z 5f872d2e f
 0001:00071d63       ??0CDumpContext@@QAE@PAVCFile@@@Z 5f872d63 f
 0001:00071d72       ?Flush@CDumpContext@@QAEXXZ 5f872d72 f
 0001:00071d7f       ??6CDumpContext@@QAEAAV0@PBG@Z 5f872d7f f
 0001:00071e15       ??6CDumpContext@@QAEAAV0@E@Z 5f872e15 f
 0001:00071e47       ??6CDumpContext@@QAEAAV0@G@Z 5f872e47 f
 0001:00071e79       ??6CDumpContext@@QAEAAV0@I@Z 5f872e79 f
 0001:00071ea9       ??6CDumpContext@@QAEAAV0@J@Z 5f872ea9 f
 0001:00071ed9       ??6CDumpContext@@QAEAAV0@K@Z 5f872ed9 f
 0001:00071f09       ??6CDumpContext@@QAEAAV0@H@Z 5f872f09 f
 0001:00071f39       ??6CDumpContext@@QAEAAV0@PBVCObject@@@Z 5f872f39 f
 0001:00071f5e       ??6CDumpContext@@QAEAAV0@ABVCObject@@@Z 5f872f5e f
 0001:00071f6a       ??6CDumpContext@@QAEAAV0@PBX@Z 5f872f6a f
 0001:00071f9a       ?HexDump@CDumpContext@@QAEXPBGPAEHH@Z 5f872f9a f
 0001:0007202d       ??6CDumpContext@@QAEAAV0@PBD@Z 5f87302d f
 0001:00072077       ??1CIPAddressCtrl@@UAE@XZ  5f873077 f
 0001:000720af       ?Create@CIPAddressCtrl@@QAEHKABUtagRECT@@PAVCWnd@@I@Z 5f8730af f
 0001:000720e0       ?GetAddress@CIPAddressCtrl@@QAEHAAE000@Z 5f8730e0 f
 0001:00072124       ?_AfxParseURLWorker@@YGHPBGPAUURL_COMPONENTSW@@AAKAAGK@Z 5f873124 f
 0001:0007225c       ?AfxParseURLEx@@YGHPBGAAKAAVCString@@2AAG22K@Z 5f87325c f
 0001:00072329       ?AfxParseURL@@YGHPBGAAKAAVCString@@2AAG@Z 5f873329 f
 0001:000723b7       ?AfxGetInternetHandleType@@YGKPAX@Z 5f8733b7 f
 0001:000723eb       ?_AfxQueryCStringInternetOption@@YGHPAXKAAVCString@@@Z 5f8733eb f
 0001:00072453       ?AfxInternetStatusCallback@@YGXPAXKK0K@Z 5f873453 f
 0001:00072483       ?Lookup@CSessionMapPtrToPtr@@QAEHPAXAAPAVCInternetSession@@@Z 5f873483 f
 0001:000724b1       ??1CInternetSession@@UAE@XZ 5f8734b1 f
 0001:000724e4       ??0CInternetSession@@QAE@PBGKK00K@Z 5f8734e4 f
 0001:0007255e       ?SetAt@CSessionMapPtrToPtr@@QAEXPAXPAVCInternetSession@@@Z 5f87355e f
 0001:00072589       ?Close@CInternetSession@@UAEXXZ 5f873589 f
 0001:000725ba       ?RemoveKey@CSessionMapPtrToPtr@@QAEXPAX@Z 5f8735ba f
 0001:000725df       ?GetGopherConnection@CInternetSession@@QAEPAVCGopherConnection@@PBG00G@Z 5f8735df f
 0001:00072627       ?GetFtpConnection@CInternetSession@@QAEPAVCFtpConnection@@PBG00GH@Z 5f873627 f
 0001:00072672       ?GetHttpConnection@CInternetSession@@QAEPAVCHttpConnection@@PBGG00@Z 5f873672 f
 0001:000726ba       ?GetHttpConnection@CInternetSession@@QAEPAVCHttpConnection@@PBGKG00@Z 5f8736ba f
 0001:00072705       ?OpenURL@CInternetSession@@QAEPAVCStdioFile@@PBGKK0K@Z 5f873705 f
 0001:000728cb       ?SetOption@CInternetSession@@QAEHKPAXKK@Z 5f8738cb f
 0001:000728e7       ?QueryOption@CInternetSession@@QBEHKPAXPAK@Z 5f8738e7 f
 0001:000728ff       ?QueryOption@CInternetSession@@QBEHKAAK@Z 5f8738ff f
 0001:00072921       ?QueryOption@CInternetSession@@QBEHKAAVCString@@@Z 5f873921 f
 0001:00072934       ?OnStatusCallback@CInternetSession@@UAEXKKPAXK@Z 5f873934 f
 0001:00072953       ?EnableStatusCallback@CInternetSession@@QAEHH@Z 5f873953 f
 0001:000729af       ?SetCookie@CInternetSession@@SAHPBDPBG1@Z 5f8739af f
 0001:000729c2       ?GetCookie@CInternetSession@@SAHPBDPBGPAGK@Z 5f8739c2 f
 0001:000729da       ?GetCookieLength@CInternetSession@@SAKPBDPBG@Z 5f8739da f
 0001:000729fb       ?GetCookie@CInternetSession@@SAHPBDPBGAAVCString@@@Z 5f8739fb f
 0001:00072a49       ??0CInternetFile@@IAE@PAX0PBG1KH@Z 5f873a49 f
 0001:00072ac9       ??_GCInternetFile@@UAEPAXI@Z 5f873ac9 f
 0001:00072ac9       ??_ECInternetFile@@UAEPAXI@Z 5f873ac9 f
 0001:00072ae5       ??0CInternetFile@@IAE@PAXPBGPAVCInternetConnection@@H@Z 5f873ae5 f
 0001:00072b90       ?QueryOption@CInternetFile@@QBEHKPAXPAK@Z 5f873b90 f
 0001:00072ba8       ?QueryOption@CInternetFile@@QBEHKAAK@Z 5f873ba8 f
 0001:00072bca       ?QueryOption@CInternetFile@@QBEHKAAVCString@@@Z 5f873bca f
 0001:00072bdd       ?SetOption@CInternetFile@@QAEHKPAXKK@Z 5f873bdd f
 0001:00072bf9       ?SetReadBufferSize@CInternetFile@@QAEHI@Z 5f873bf9 f
 0001:00072c99       ?SetWriteBufferSize@CInternetFile@@QAEHI@Z 5f873c99 f
 0001:00072d01       ?Seek@CInternetFile@@UAEJJI@Z 5f873d01 f
 0001:00072d6d       ?Abort@CInternetFile@@UAEXXZ 5f873d6d f
 0001:00072d85       ?Flush@CInternetFile@@UAEXXZ 5f873d85 f
 0001:00072dcf       ?Read@CInternetFile@@UAEIPAXI@Z 5f873dcf f
 0001:00072ef6       ?Write@CInternetFile@@UAEXPBXI@Z 5f873ef6 f
 0001:00072fb3       ?WriteString@CInternetFile@@UAEXPBG@Z 5f873fb3 f
 0001:00072fe2       ?ReadString@CInternetFile@@UAEPAGPAGI@Z 5f873fe2 f
 0001:000730ad       ?ReadString@CInternetFile@@UAEHAAVCString@@@Z 5f8740ad f
 0001:00073157       ?GetLength@CInternetFile@@UBEKXZ 5f874157 f
 0001:00073181       ?UnlockRange@CInternetFile@@UAEXKK@Z 5f874181 f
 0001:00073189       ?SetLength@CInternetFile@@UAEXK@Z 5f874189 f
 0001:00073191       ?Duplicate@CInternetFile@@UBEPAVCFile@@XZ 5f874191 f
 0001:00073199       ??0CInternetConnection@@QAE@PAVCInternetSession@@PBGGK@Z 5f874199 f
 0001:000731f6       ??_GCInternetConnection@@UAEPAXI@Z 5f8741f6 f
 0001:000731f6       ??_ECInternetConnection@@UAEPAXI@Z 5f8741f6 f
 0001:00073212       ?SetOption@CInternetConnection@@QAEHKPAXKK@Z 5f874212 f
 0001:0007322e       ?QueryOption@CInternetConnection@@QBEHKPAXPAK@Z 5f87422e f
 0001:00073246       ?QueryOption@CInternetConnection@@QBEHKAAK@Z 5f874246 f
 0001:00073268       ?QueryOption@CInternetConnection@@QBEHKAAVCString@@@Z 5f874268 f
 0001:0007327b       ??1CFtpConnection@@UAE@XZ  5f87427b f
 0001:000732b6       ??_ECFtpConnection@@UAEPAXI@Z 5f8742b6 f
 0001:000732b6       ??_GCFtpConnection@@UAEPAXI@Z 5f8742b6 f
 0001:000732d2       ??0CFtpConnection@@QAE@PAVCInternetSession@@PAXPBGK@Z 5f8742d2 f
 0001:00073369       ??0CFtpConnection@@QAE@PAVCInternetSession@@PBG11KGH@Z 5f874369 f
 0001:00073411       ?Remove@CFtpConnection@@QAEHPBG@Z 5f874411 f
 0001:00073421       ?Rename@CFtpConnection@@QAEHPBG0@Z 5f874421 f
 0001:00073435       ?CreateDirectoryW@CFtpConnection@@QAEHPBG@Z 5f874435 f
 0001:00073445       ?RemoveDirectoryW@CFtpConnection@@QAEHPBG@Z 5f874445 f
 0001:00073455       ?SetCurrentDirectoryW@CFtpConnection@@QAEHPBG@Z 5f874455 f
 0001:00073465       ?GetCurrentDirectoryW@CFtpConnection@@QBEHPAGPAK@Z 5f874465 f
 0001:00073479       ?GetCurrentDirectoryAsURL@CFtpConnection@@QBEHAAVCString@@@Z 5f874479 f
 0001:0007351a       ?GetCurrentDirectoryAsURL@CFtpConnection@@QBEHPAGPAK@Z 5f87451a f
 0001:00073590       ?GetCurrentDirectoryW@CFtpConnection@@QBEHAAVCString@@@Z 5f874590 f
 0001:000735d2       ?OpenFile@CFtpConnection@@QAEPAVCInternetFile@@PBGKKK@Z 5f8745d2 f
 0001:0007364d       ?PutFile@CFtpConnection@@QAEHPBG0KK@Z 5f87464d f
 0001:00073672       ?GetFile@CFtpConnection@@QAEHPBG0HKKK@Z 5f874672 f
 0001:0007369d       ??1CGopherConnection@@UAE@XZ 5f87469d f
 0001:000736a3       ??1CInternetConnection@@UAE@XZ 5f8746a3 f
 0001:000736eb       ??_ECGopherConnection@@UAEPAXI@Z 5f8746eb f
 0001:000736eb       ??_GCGopherConnection@@UAEPAXI@Z 5f8746eb f
 0001:00073707       ??0CGopherConnection@@QAE@PAVCInternetSession@@PBG11KG@Z 5f874707 f
 0001:00073784       ??0CGopherConnection@@QAE@PAVCInternetSession@@PAXPBGK@Z 5f874784 f
 0001:00073801       ?CreateLocator@CGopherConnection@@SA?AVCGopherLocator@@PBG@Z 5f874801 f
 0001:00073859       ?CreateLocator@CGopherConnection@@SA?AVCGopherLocator@@PBG00KG@Z 5f874859 f
 0001:000738e3       ?CreateLocator@CGopherConnection@@QAE?AVCGopherLocator@@PBG0K@Z 5f8748e3 f
 0001:00073976       ?GetAttribute@CGopherConnection@@QAEHAAVCGopherLocator@@VCString@@AAV3@@Z 5f874976 f
 0001:000739ec       ?OpenFile@CGopherConnection@@QAEPAVCGopherFile@@AAVCGopherLocator@@KPBGK@Z 5f8749ec f
 0001:00073a5f       ?Close@CGopherConnection@@UAEXXZ 5f874a5f f
 0001:00073a5f       ?Close@CInternetConnection@@MAEXXZ 5f874a5f f
 0001:00073a83       ??1CHttpConnection@@UAE@XZ 5f874a83 f
 0001:00073abe       ??_ECHttpConnection@@UAEPAXI@Z 5f874abe f
 0001:00073abe       ??_GCHttpConnection@@UAEPAXI@Z 5f874abe f
 0001:00073ada       ??0CHttpConnection@@QAE@PAVCInternetSession@@PAXPBGK@Z 5f874ada f
 0001:00073b5c       ??0CHttpConnection@@QAE@PAVCInternetSession@@PBGG11K@Z 5f874b5c f
 0001:00073be5       ??0CHttpConnection@@QAE@PAVCInternetSession@@PBGKG11K@Z 5f874be5 f
 0001:00073c6f       ?OpenRequest@CHttpConnection@@QAEPAVCHttpFile@@PBG00KPAPBG0K@Z 5f874c6f f
 0001:00073ceb       ?OpenRequest@CHttpConnection@@QAEPAVCHttpFile@@HPBG0KPAPBG0K@Z 5f874ceb f
 0001:00073d24       ??0CHttpFile@@IAE@PAX0PBG11K@Z 5f874d24 f
 0001:00073d80       ??_ECHttpFile@@UAEPAXI@Z   5f874d80 f
 0001:00073d80       ??_GCHttpFile@@UAEPAXI@Z   5f874d80 f
 0001:00073d9c       ??0CHttpFile@@IAE@PAXPBG1PAVCHttpConnection@@@Z 5f874d9c f
 0001:00073df2       ??1CHttpFile@@UAE@XZ       5f874df2 f
 0001:00073e3c       ?Close@CInternetFile@@UAEXXZ 5f874e3c f
 0001:00073e3c       ?Close@CHttpFile@@UAEXXZ   5f874e3c f
 0001:00073e8a       ?ErrorDlg@CHttpFile@@QAEKPAVCWnd@@KKPAPAX@Z 5f874e8a f
 0001:00073ec9       ?GetVerb@CHttpFile@@QBE?AVCString@@XZ 5f874ec9 f
 0001:00073ee4       ?GetObjectW@CHttpFile@@QBE?AVCString@@XZ 5f874ee4 f
 0001:00073eff       ?GetFileURL@CHttpFile@@UBE?AVCString@@XZ 5f874eff f
 0001:00073f94       ?AddRequestHeaders@CHttpFile@@QAEHPBGKH@Z 5f874f94 f
 0001:00073fc7       ?AddRequestHeaders@CHttpFile@@QAEHAAVCString@@K@Z 5f874fc7 f
 0001:00073fdd       ?SendRequest@CHttpFile@@QAEHPBGKPAXK@Z 5f874fdd f
 0001:00074010       ?EndRequest@CHttpFile@@QAEHKPAU_INTERNET_BUFFERSW@@K@Z 5f875010 f
 0001:00074048       ?SendRequestEx@CHttpFile@@QAEHKKK@Z 5f875048 f
 0001:0007408f       ?SendRequestEx@CHttpFile@@QAEHPAU_INTERNET_BUFFERSW@@0KK@Z 5f87508f f
 0001:000740cf       ?SendRequest@CHttpFile@@QAEHAAVCString@@PAXK@Z 5f8750cf f
 0001:000740ea       ?QueryInfo@CHttpFile@@QBEHKPAXPAK1@Z 5f8750ea f
 0001:00074106       ?QueryInfo@CHttpFile@@QBEHKAAKPAK@Z 5f875106 f
 0001:0007412d       ?QueryInfo@CHttpFile@@QBEHKPAU_SYSTEMTIME@@PAK@Z 5f87512d f
 0001:00074154       ?QueryInfoStatusCode@CHttpFile@@QBEHAAK@Z 5f875154 f
 0001:0007419d       ?QueryInfo@CHttpFile@@QBEHKAAVCString@@PAK@Z 5f87519d f
 0001:00074208       ??0CGopherFile@@IAE@PAXAAVCGopherLocator@@PAVCGopherConnection@@@Z 5f875208 f
 0001:00074251       ??_GCGopherFile@@UAEPAXI@Z 5f875251 f
 0001:00074251       ??_ECGopherFile@@UAEPAXI@Z 5f875251 f
 0001:0007426d       ??0CGopherFile@@IAE@PAX0PBGKK@Z 5f87526d f
 0001:000742be       ??1CGopherFile@@UAE@XZ     5f8752be f
 0001:000742f9       ??0CFtpFileFind@@QAE@PAVCFtpConnection@@K@Z 5f8752f9 f
 0001:00074329       ??_GCFtpFileFind@@UAEPAXI@Z 5f875329 f
 0001:00074329       ??_ECFtpFileFind@@UAEPAXI@Z 5f875329 f
 0001:00074345       ??1CFtpFileFind@@UAE@XZ    5f875345 f
 0001:0007434b       ??1CFileFind@@UAE@XZ       5f87534b f
 0001:0007438d       ?FindFile@CFtpFileFind@@UAEHPBGK@Z 5f87538d f
 0001:000744ed       ?FindNextFileW@CFtpFileFind@@UAEHXZ 5f8754ed f
 0001:00074528       ?GetFileURL@CFtpFileFind@@UBE?AVCString@@XZ 5f875528 f
 0001:000745d3       ??0CGopherFileFind@@QAE@PAVCGopherConnection@@K@Z 5f8755d3 f
 0001:000745fd       ??_ECGopherFileFind@@UAEPAXI@Z 5f8755fd f
 0001:000745fd       ??_GCGopherFileFind@@UAEPAXI@Z 5f8755fd f
 0001:00074619       ??1CGopherFileFind@@UAE@XZ 5f875619 f
 0001:00074624       ?FindFile@CGopherFileFind@@UAEHPBGK@Z 5f875624 f
 0001:00074673       ?FindFile@CGopherFileFind@@UAEHAAVCGopherLocator@@PBGK@Z 5f875673 f
 0001:000746d7       ?FindNextFileW@CGopherFileFind@@UAEHXZ 5f8756d7 f
 0001:00074712       ?CloseContext@CGopherFileFind@@MAEXXZ 5f875712 f
 0001:0007472e       ?GetFileName@CGopherFileFind@@UBE?AVCString@@XZ 5f87572e f
 0001:0007474a       ?IsDots@CGopherFileFind@@UBEHXZ 5f87574a f
 0001:0007474d       ?GetLastWriteTime@CGopherFileFind@@UBEHPAU_FILETIME@@@Z 5f87574d f
 0001:00074777       ?GetLastAccessTime@CGopherFileFind@@UBEHPAU_FILETIME@@@Z 5f875777 f
 0001:00074783       ?GetLastWriteTime@CGopherFileFind@@UBEHAAVCTime@@@Z 5f875783 f
 0001:000747b0       ?GetLastAccessTime@CGopherFileFind@@UBEHAAVCTime@@@Z 5f8757b0 f
 0001:000747bc       ?GetLocator@CGopherFileFind@@QBE?AVCGopherLocator@@XZ 5f8757bc f
 0001:000747de       ?GetScreenName@CGopherFileFind@@QBE?AVCString@@XZ 5f8757de f
 0001:0007483e       ?GetLength@CGopherFileFind@@UBEKXZ 5f87583e f
 0001:0007484f       ?GetLength64@CGopherFileFind@@UBE_JXZ 5f87584f f
 0001:00074863       ??0CGopherLocator@@AAE@PBGK@Z 5f875863 f
 0001:000748ca       ?AfxThrowInternetException@@YGXKK@Z 5f8758ca f
 0001:00074920       ?GetErrorMessage@CInternetException@@UAEHPAGIPAI@Z 5f875920 f
 0001:00074a0d       ??0CInternetException@@QAE@K@Z 5f875a0d f
 0001:00074a28       ??_ECInternetException@@UAEPAXI@Z 5f875a28 f
 0001:00074a28       ??_GCInternetException@@UAEPAXI@Z 5f875a28 f
 0001:00074a44       ??1CInternetException@@UAE@XZ 5f875a44 f
 0001:00074a4b       ??_ECSessionMapPtrToPtr@@UAEPAXI@Z 5f875a4b f
 0001:00074a4b       ??_GCSessionMapPtrToPtr@@UAEPAXI@Z 5f875a4b f
 0001:00074a67       ?GetRuntimeClass@CMemoryException@@UBEPAUCRuntimeClass@@XZ 5f875a67 f
 0001:00074a6d       ?GetRuntimeClass@CNotSupportedException@@UBEPAUCRuntimeClass@@XZ 5f875a6d f
 0001:00074a73       ?GetRuntimeClass@CArchiveException@@UBEPAUCRuntimeClass@@XZ 5f875a73 f
 0001:00074a79       ?_GetBaseClass@CStdioFile@@KGPAUCRuntimeClass@@XZ 5f875a79 f
 0001:00074a7f       ?GetRuntimeClass@CStdioFile@@UBEPAUCRuntimeClass@@XZ 5f875a7f f
 0001:00074a85       ?_GetBaseClass@CSharedFile@@KGPAUCRuntimeClass@@XZ 5f875a85 f
 0001:00074a8b       ?GetRuntimeClass@CSharedFile@@UBEPAUCRuntimeClass@@XZ 5f875a8b f
 0001:00074a91       ?GetRuntimeClass@CFileException@@UBEPAUCRuntimeClass@@XZ 5f875a91 f
 0001:00074a97       ?CreateObject@CByteArray@@SGPAVCObject@@XZ 5f875a97 f
 0001:00074aae       ?GetRuntimeClass@CByteArray@@UBEPAUCRuntimeClass@@XZ 5f875aae f
 0001:00074ab4       ??5@YGAAVCArchive@@AAV0@AAPAVCByteArray@@@Z 5f875ab4 f
 0001:00074acf       ?CreateObject@CDWordArray@@SGPAVCObject@@XZ 5f875acf f
 0001:00074ae6       ?GetRuntimeClass@CDWordArray@@UBEPAUCRuntimeClass@@XZ 5f875ae6 f
 0001:00074aec       ??5@YGAAVCArchive@@AAV0@AAPAVCDWordArray@@@Z 5f875aec f
 0001:00074b07       ?GetRuntimeClass@CPtrArray@@UBEPAUCRuntimeClass@@XZ 5f875b07 f
 0001:00074b0d       ?CreateObject@CObArray@@SGPAVCObject@@XZ 5f875b0d f
 0001:00074b24       ?GetRuntimeClass@CObArray@@UBEPAUCRuntimeClass@@XZ 5f875b24 f
 0001:00074b2a       ??5@YGAAVCArchive@@AAV0@AAPAVCObArray@@@Z 5f875b2a f
 0001:00074b45       ?CreateObject@CStringArray@@SGPAVCObject@@XZ 5f875b45 f
 0001:00074b5c       ?GetRuntimeClass@CStringArray@@UBEPAUCRuntimeClass@@XZ 5f875b5c f
 0001:00074b62       ??5@YGAAVCArchive@@AAV0@AAPAVCStringArray@@@Z 5f875b62 f
 0001:00074b7d       ?GetRuntimeClass@CUIntArray@@UBEPAUCRuntimeClass@@XZ 5f875b7d f
 0001:00074b83       ?CreateObject@CWordArray@@SGPAVCObject@@XZ 5f875b83 f
 0001:00074b9a       ?GetRuntimeClass@CWordArray@@UBEPAUCRuntimeClass@@XZ 5f875b9a f
 0001:00074ba0       ??5@YGAAVCArchive@@AAV0@AAPAVCWordArray@@@Z 5f875ba0 f
 0001:00074bbb       ?CreateObject@CObList@@SGPAVCObject@@XZ 5f875bbb f
 0001:00074bd4       ?GetRuntimeClass@CObList@@UBEPAUCRuntimeClass@@XZ 5f875bd4 f
 0001:00074bda       ??5@YGAAVCArchive@@AAV0@AAPAVCObList@@@Z 5f875bda f
 0001:00074bf5       ?GetRuntimeClass@CPtrList@@UBEPAUCRuntimeClass@@XZ 5f875bf5 f
 0001:00074bfb       ?CreateObject@CStringList@@SGPAVCObject@@XZ 5f875bfb f
 0001:00074c14       ?GetRuntimeClass@CStringList@@UBEPAUCRuntimeClass@@XZ 5f875c14 f
 0001:00074c1a       ??5@YGAAVCArchive@@AAV0@AAPAVCStringList@@@Z 5f875c1a f
 0001:00074c35       ?GetRuntimeClass@CMapPtrToPtr@@UBEPAUCRuntimeClass@@XZ 5f875c35 f
 0001:00074c3b       ?GetRuntimeClass@CMapPtrToWord@@UBEPAUCRuntimeClass@@XZ 5f875c3b f
 0001:00074c41       ?CreateObject@CMapStringToOb@@SGPAVCObject@@XZ 5f875c41 f
 0001:00074c5a       ?GetRuntimeClass@CMapStringToOb@@UBEPAUCRuntimeClass@@XZ 5f875c5a f
 0001:00074c60       ??5@YGAAVCArchive@@AAV0@AAPAVCMapStringToOb@@@Z 5f875c60 f
 0001:00074c7b       ?GetRuntimeClass@CMapStringToPtr@@UBEPAUCRuntimeClass@@XZ 5f875c7b f
 0001:00074c81       ?CreateObject@CMapStringToString@@SGPAVCObject@@XZ 5f875c81 f
 0001:00074c9a       ?GetRuntimeClass@CMapStringToString@@UBEPAUCRuntimeClass@@XZ 5f875c9a f
 0001:00074ca0       ??5@YGAAVCArchive@@AAV0@AAPAVCMapStringToString@@@Z 5f875ca0 f
 0001:00074cbb       ?CreateObject@CMapWordToOb@@SGPAVCObject@@XZ 5f875cbb f
 0001:00074cd4       ?GetRuntimeClass@CMapWordToOb@@UBEPAUCRuntimeClass@@XZ 5f875cd4 f
 0001:00074cda       ??5@YGAAVCArchive@@AAV0@AAPAVCMapWordToOb@@@Z 5f875cda f
 0001:00074cf5       ?GetRuntimeClass@CMapWordToPtr@@UBEPAUCRuntimeClass@@XZ 5f875cf5 f
 0001:00074cfb       ??1AFX_MAINTAIN_STATE@@QAE@XZ 5f875cfb f
 0001:00074d37       ??1?$CThreadLocal@V_AFX_THREAD_STATE@@@@QAE@XZ 5f875d37 f
 0001:00074d3c       ??_EAFX_MODULE_STATE@@UAEPAXI@Z 5f875d3c f
 0001:00074d3c       ??_GAFX_MODULE_STATE@@UAEPAXI@Z 5f875d3c f
 0001:00074d84       ?RemoveAll@CTypeLibCacheMap@@UAEXPAX@Z 5f875d84 f
 0001:00074dc8       ??1?$CEmbeddedButActsLikePtr@VCMapPtrToPtr@@@@QAE@XZ 5f875dc8 f
 0001:00074df3       ??1?$CEmbeddedButActsLikePtr@VCPtrList@@@@QAE@XZ 5f875df3 f
 0001:00074df8       ?AfxGetAppModuleState@@YGPAVAFX_MODULE_STATE@@XZ 5f875df8 f
 0001:00074e08       ?Unlock@CTypeLibCache@@QAEXXZ 5f875e08 f
 0001:00074f01       ?AssignInstance@CThreadSlotData@@QAEXPAUHINSTANCE__@@@Z 5f875f01 f
 0001:00074f5e       ?AfxInitLocalData@@YGXPAUHINSTANCE__@@@Z 5f875f5e f
 0001:00074f74       ?_GetBaseClass@CCriticalSection@@KGPAUCRuntimeClass@@XZ 5f875f74 f
 0001:00074f7a       ?GetRuntimeClass@CCriticalSection@@UBEPAUCRuntimeClass@@XZ 5f875f7a f
 0001:00074f80       ?GetRuntimeClass@CEvent@@UBEPAUCRuntimeClass@@XZ 5f875f80 f
 0001:00074f86       ?GetRuntimeClass@CSemaphore@@UBEPAUCRuntimeClass@@XZ 5f875f86 f
 0001:00074f8c       ?GetRuntimeClass@CMutex@@UBEPAUCRuntimeClass@@XZ 5f875f8c f
 0001:00074f92       ?CreateObject@CWnd@@SGPAVCObject@@XZ 5f875f92 f
 0001:00074fc4       ??1CTempWnd@@UAE@XZ        5f875fc4 f
 0001:00074fc9       ?GetRuntimeClass@CTempWnd@@UBEPAUCRuntimeClass@@XZ 5f875fc9 f
 0001:00074fd3       ?CreateObject@CFrameWnd@@SGPAVCObject@@XZ 5f875fd3 f
 0001:00075008       ?CreateObject@CMDIFrameWnd@@SGPAVCObject@@XZ 5f876008 f
 0001:0007503d       ?GetRuntimeClass@CMDIFrameWnd@@UBEPAUCRuntimeClass@@XZ 5f87603d f
 0001:00075043       ?GetRuntimeClass@CToolTipCtrl@@UBEPAUCRuntimeClass@@XZ 5f876043 f
 0001:00075049       ?CreateObject@CMiniFrameWnd@@SGPAVCObject@@XZ 5f876049 f
 0001:0007507e       ??_ECControlBar@@UAEPAXI@Z 5f87607e f
 0001:0007507e       ??_GCControlBar@@UAEPAXI@Z 5f87607e f
 0001:0007509a       ?OnBarStyleChange@CControlBar@@UAEXKK@Z 5f87609a f
 0001:000750c0       ?SetOwner@CToolBar@@QAEXPAVCWnd@@@Z 5f8760c0 f
 0001:00075127       ?SetHeight@CToolBar@@QAEXH@Z 5f876127 f
 0001:0007518a       ?LoadToolBar@CToolBar@@QAEHPBG@Z 5f87618a f
 0001:0007525c       ?SetBitmap@CToolBar@@QAEHPAUHBITMAP__@@@Z 5f87625c f
 0001:0007530b       ?GetRuntimeClass@CToolBar@@UBEPAUCRuntimeClass@@XZ 5f87630b f
 0001:00075311       ?GetRuntimeClass@CDialogBar@@UBEPAUCRuntimeClass@@XZ 5f876311 f
 0001:00075331       ?GetRuntimeClass@CStatusBar@@UBEPAUCRuntimeClass@@XZ 5f876331 f
 0001:00075337       ?GetRuntimeClass@CDockBar@@UBEPAUCRuntimeClass@@XZ 5f876337 f
 0001:0007533d       ?CreateObject@CMiniDockFrameWnd@@SGPAVCObject@@XZ 5f87633d f
 0001:00075372       ?_GetBaseClass@CMiniDockFrameWnd@@KGPAUCRuntimeClass@@XZ 5f876372 f
 0001:00075378       ?GetRuntimeClass@CMiniDockFrameWnd@@UBEPAUCRuntimeClass@@XZ 5f876378 f
 0001:0007537e       ?CreateObject@CDockState@@SGPAVCObject@@XZ 5f87637e f
 0001:000753b0       ?GetRuntimeClass@CDockState@@UBEPAUCRuntimeClass@@XZ 5f8763b0 f
 0001:000753b6       ??5@YGAAVCArchive@@AAV0@AAPAVCDockState@@@Z 5f8763b6 f
 0001:000753d1       ?_GetBaseClass@CPreviewDC@@KGPAUCRuntimeClass@@XZ 5f8763d1 f
 0001:000753d7       ?GetRuntimeClass@CPreviewDC@@UBEPAUCRuntimeClass@@XZ 5f8763d7 f
 0001:000753dd       ?GetRuntimeClass@CMetaFileDC@@UBEPAUCRuntimeClass@@XZ 5f8763dd f
 0001:000753e3       ?GetRuntimeClass@CReBar@@UBEPAUCRuntimeClass@@XZ 5f8763e3 f
 0001:000753e9       ?GetRuntimeClass@CStatic@@UBEPAUCRuntimeClass@@XZ 5f8763e9 f
 0001:000753ef       ?GetRuntimeClass@CButton@@UBEPAUCRuntimeClass@@XZ 5f8763ef f
 0001:000753f5       ?GetRuntimeClass@CEdit@@UBEPAUCRuntimeClass@@XZ 5f8763f5 f
 0001:000753fb       ?GetRuntimeClass@CScrollBar@@UBEPAUCRuntimeClass@@XZ 5f8763fb f
 0001:00075401       ?_GetBaseClass@CDragListBox@@KGPAUCRuntimeClass@@XZ 5f876401 f
 0001:00075407       ?GetRuntimeClass@CDragListBox@@UBEPAUCRuntimeClass@@XZ 5f876407 f
 0001:0007540d       ?GetRuntimeClass@CSpinButtonCtrl@@UBEPAUCRuntimeClass@@XZ 5f87640d f
 0001:00075413       ?GetRuntimeClass@CSliderCtrl@@UBEPAUCRuntimeClass@@XZ 5f876413 f
 0001:00075419       ?GetRuntimeClass@CProgressCtrl@@UBEPAUCRuntimeClass@@XZ 5f876419 f
 0001:0007541f       ?_GetBaseClass@CComboBoxEx@@KGPAUCRuntimeClass@@XZ 5f87641f f
 0001:00075425       ?GetRuntimeClass@CComboBoxEx@@UBEPAUCRuntimeClass@@XZ 5f876425 f
 0001:0007542b       ?GetRuntimeClass@CHeaderCtrl@@UBEPAUCRuntimeClass@@XZ 5f87642b f
 0001:00075431       ?GetRuntimeClass@CHotKeyCtrl@@UBEPAUCRuntimeClass@@XZ 5f876431 f
 0001:00075437       ?GetRuntimeClass@CAnimateCtrl@@UBEPAUCRuntimeClass@@XZ 5f876437 f
 0001:0007543d       ?GetRuntimeClass@CTabCtrl@@UBEPAUCRuntimeClass@@XZ 5f87643d f
 0001:00075443       ?GetRuntimeClass@CTreeCtrl@@UBEPAUCRuntimeClass@@XZ 5f876443 f
 0001:00075449       ?GetRuntimeClass@CListCtrl@@UBEPAUCRuntimeClass@@XZ 5f876449 f
 0001:0007544f       ?GetRuntimeClass@CToolBarCtrl@@UBEPAUCRuntimeClass@@XZ 5f87644f f
 0001:00075455       ?GetRuntimeClass@CStatusBarCtrl@@UBEPAUCRuntimeClass@@XZ 5f876455 f
 0001:0007545b       ?CreateObject@CImageList@@SGPAVCObject@@XZ 5f87645b f
 0001:00075472       ?GetRuntimeClass@CImageList@@UBEPAUCRuntimeClass@@XZ 5f876472 f
 0001:00075478       ?CreateObject@CTempImageList@@SGPAVCObject@@XZ 5f876478 f
 0001:0007549e       ??_ECTempImageList@@UAEPAXI@Z 5f87649e f
 0001:0007549e       ??_GCTempImageList@@UAEPAXI@Z 5f87649e f
 0001:000754be       ??1CTempImageList@@UAE@XZ  5f8764be f
 0001:000754be       ??1CImageList@@UAE@XZ      5f8764be f
 0001:000754f1       ?GetRuntimeClass@CTempImageList@@UBEPAUCRuntimeClass@@XZ 5f8764f1 f
 0001:000754f7       ?GetRuntimeClass@CRichEditCtrl@@UBEPAUCRuntimeClass@@XZ 5f8764f7 f
 0001:000754fe       ?GetRuntimeClass@CCheckListBox@@UBEPAUCRuntimeClass@@XZ 5f8764fe f
 0001:00075504       ?CreateObject@?$CProcessLocal@V_AFX_CHECKLIST_STATE@@@@SGPAVCNoTrackObject@@XZ 5f876504 f
 0001:00075535       ?GetRuntimeClass@CBitmapButton@@UBEPAUCRuntimeClass@@XZ 5f876535 f
 0001:0007553b       ?GetRuntimeClass@CPropertyPage@@UBEPAUCRuntimeClass@@XZ 5f87653b f
 0001:00075541       ?GetRuntimeClass@CPropertySheet@@UBEPAUCRuntimeClass@@XZ 5f876541 f
 0001:00075547       ?GetRuntimeClass@CPropertyPageEx@@UBEPAUCRuntimeClass@@XZ 5f876547 f
 0001:0007554d       ?GetRuntimeClass@CPropertySheetEx@@UBEPAUCRuntimeClass@@XZ 5f87654d f
 0001:00075553       ?GetRuntimeClass@CFileDialog@@UBEPAUCRuntimeClass@@XZ 5f876553 f
 0001:00075559       ?GetRuntimeClass@CPrintDialog@@UBEPAUCRuntimeClass@@XZ 5f876559 f
 0001:0007555f       ?GetRuntimeClass@CPageSetupDialog@@UBEPAUCRuntimeClass@@XZ 5f87655f f
 0001:00075565       ?GetRuntimeClass@CColorDialog@@UBEPAUCRuntimeClass@@XZ 5f876565 f
 0001:0007556b       ?CreateObject@?$CProcessLocal@V_AFX_COLOR_STATE@@@@SGPAVCNoTrackObject@@XZ 5f87656b f
 0001:00075581       ?GetRuntimeClass@CFontDialog@@UBEPAUCRuntimeClass@@XZ 5f876581 f
 0001:00075587       ?GetRuntimeClass@CFindReplaceDialog@@UBEPAUCRuntimeClass@@XZ 5f876587 f
 0001:0007558d       ?AfxGetPropSheetFont@@YGHAAVCString@@AAGH@Z 5f87658d f
 0001:00075640       ?CreateObject@?$CProcessLocal@U_AFX_PROPPAGEFONTINFO@@@@SGPAVCNoTrackObject@@XZ 5f876640 f
 0001:0007565e       ??_G_AFX_PROPPAGEFONTINFO@@UAEPAXI@Z 5f87665e f
 0001:0007565e       ??_E_AFX_PROPPAGEFONTINFO@@UAEPAXI@Z 5f87665e f
 0001:00075679       ??1_AFX_PROPPAGEFONTINFO@@UAE@XZ 5f876679 f
 0001:00075689       ?GetRuntimeClass@CIPAddressCtrl@@UBEPAUCRuntimeClass@@XZ 5f876689 f
 0001:0007568f       ?GetRuntimeClass@CReBarCtrl@@UBEPAUCRuntimeClass@@XZ 5f87668f f
 0001:00075695       ?GetRuntimeClass@CResourceException@@UBEPAUCRuntimeClass@@XZ 5f876695 f
 0001:0007569b       ?GetRuntimeClass@CUserException@@UBEPAUCRuntimeClass@@XZ 5f87669b f
 0001:000756a1       ?CreateObject@CDC@@SGPAVCObject@@XZ 5f8766a1 f
 0001:000756b8       ?GetRuntimeClass@CClientDC@@UBEPAUCRuntimeClass@@XZ 5f8766b8 f
 0001:000756be       ?GetRuntimeClass@CWindowDC@@UBEPAUCRuntimeClass@@XZ 5f8766be f
 0001:000756c4       ?GetRuntimeClass@CPaintDC@@UBEPAUCRuntimeClass@@XZ 5f8766c4 f
 0001:000756ca       ?CreateObject@CGdiObject@@SGPAVCObject@@XZ 5f8766ca f
 0001:000756e4       ?GetRuntimeClass@CPen@@UBEPAUCRuntimeClass@@XZ 5f8766e4 f
 0001:000756ea       ?GetRuntimeClass@CBrush@@UBEPAUCRuntimeClass@@XZ 5f8766ea f
 0001:000756f0       ?GetRuntimeClass@CFont@@UBEPAUCRuntimeClass@@XZ 5f8766f0 f
 0001:000756f6       ?GetRuntimeClass@CBitmap@@UBEPAUCRuntimeClass@@XZ 5f8766f6 f
 0001:000756fc       ?GetRuntimeClass@CPalette@@UBEPAUCRuntimeClass@@XZ 5f8766fc f
 0001:00075702       ?GetRuntimeClass@CRgn@@UBEPAUCRuntimeClass@@XZ 5f876702 f
 0001:0007570c       ??1CTempDC@@UAE@XZ         5f87670c f
 0001:00075711       ?GetRuntimeClass@CTempDC@@UBEPAUCRuntimeClass@@XZ 5f876711 f
 0001:0007571a       ?_GetBaseClass@CTempGdiObject@@KGPAUCRuntimeClass@@XZ 5f87671a f
 0001:00075720       ?GetRuntimeClass@CTempGdiObject@@UBEPAUCRuntimeClass@@XZ 5f876720 f
 0001:00075728       ?CreateObject@CMenu@@SGPAVCObject@@XZ 5f876728 f
 0001:00075745       ?_GetBaseClass@CTempMenu@@KGPAUCRuntimeClass@@XZ 5f876745 f
 0001:0007574b       ?GetRuntimeClass@CTempMenu@@UBEPAUCRuntimeClass@@XZ 5f87674b f
 0001:00075752       ?AfxEnableWin31Compatibility@@YGXXZ 5f876752 f
 0001:00075794       ?_AfxLoadDotBitmap@@YGXXZ  5f876794 f
 0001:00075874       ?GetRuntimeClass@CDocTemplate@@UBEPAUCRuntimeClass@@XZ 5f876874 f
 0001:0007587a       ?GetRuntimeClass@CSingleDocTemplate@@UBEPAUCRuntimeClass@@XZ 5f87687a f
 0001:00075880       ?GetRuntimeClass@CMultiDocTemplate@@UBEPAUCRuntimeClass@@XZ 5f876880 f
 0001:00075886       ?_AfxDeleteRegKey@@YGHPBG@Z 5f876886 f
 0001:0007598b       ?GetRuntimeClass@CDocManager@@UBEPAUCRuntimeClass@@XZ 5f87698b f
 0001:00075991       ?GetRuntimeClass@CSplitterWnd@@UBEPAUCRuntimeClass@@XZ 5f876991 f
 0001:00075997       ?GetRuntimeClass@CScrollView@@UBEPAUCRuntimeClass@@XZ 5f876997 f
 0001:0007599d       ?CreateObject@CEditView@@SGPAVCObject@@XZ 5f87699d f
 0001:000759cf       ?GetRuntimeClass@CEditView@@UBEPAUCRuntimeClass@@XZ 5f8769cf f
 0001:000759d5       ?CreateObject@?$CProcessLocal@V_AFX_EDIT_STATE@@@@SGPAVCNoTrackObject@@XZ 5f8769d5 f
 0001:00075a06       ?CreateObject@CPreviewView@@SGPAVCObject@@XZ 5f876a06 f
 0001:00075a3b       ?GetRuntimeClass@CPreviewView@@UBEPAUCRuntimeClass@@XZ 5f876a3b f
 0001:00075a41       ?CreateObject@CListView@@SGPAVCObject@@XZ 5f876a41 f
 0001:00075a89       ?GetRuntimeClass@CListView@@UBEPAUCRuntimeClass@@XZ 5f876a89 f
 0001:00075a8f       ?CreateObject@CTreeView@@SGPAVCObject@@XZ 5f876a8f f
 0001:00075ad7       ?GetRuntimeClass@CTreeView@@UBEPAUCRuntimeClass@@XZ 5f876ad7 f
 0001:00075add       ?CreateObject@?$CProcessLocal@V_AFX_MAIL_STATE@@@@SGPAVCNoTrackObject@@XZ 5f876add f
 0001:00075b07       ??_GCWinApp@@UAEPAXI@Z     5f876b07 f
 0001:00075b07       ??_ECWinApp@@UAEPAXI@Z     5f876b07 f
 0001:00075b23       ?InitInstance@CWinApp@@UAEHXZ 5f876b23 f
 0001:00075b7d       ?ParseParam@CCommandLineInfo@@UAEXPBDHH@Z 5f876b7d f
 0001:00075ba6       ?ParseParamFlag@CCommandLineInfo@@IAEXPBD@Z 5f876ba6 f
 0001:00075cb5       ?ParseParamNotFlag@CCommandLineInfo@@IAEXPBD@Z 5f876cb5 f
 0001:00075d62       ?_GetBaseClass@CWinApp@@KGPAUCRuntimeClass@@XZ 5f876d62 f
 0001:00075d68       ?GetRuntimeClass@CWinApp@@UBEPAUCRuntimeClass@@XZ 5f876d68 f
 0001:00075e54       ?Unregister@CWinApp@@QAEHXZ 5f876e54 f
 0001:00075f8b       ?DelRegTree@CWinApp@@QAEJPAUHKEY__@@ABVCString@@@Z 5f876f8b f
 0001:00075f9b       ?AfxDelRegTreeHelper@@YGJPAUHKEY__@@ABVCString@@@Z 5f876f9b f
 0001:0007606d       ?RegisterShellFileTypesCompat@CWinApp@@IAEXXZ 5f87706d f
 0001:0007607b       ?UnregisterShellFileTypes@CWinApp@@IAEXXZ 5f87707b f
 0001:00076081       ?UnregisterShellFileTypes@CDocManager@@QAEXXZ 5f877081 f
 0001:00076300       ?SetRegistryKey@CWinApp@@IAEXI@Z 5f877300 f
 0001:000763db       ?SetDialogBkColor@CWinApp@@IAEXKK@Z 5f8773db f
 0001:00076571       ?AfxGetCtl3dState@@YGPAV_AFX_CTL3D_STATE@@XZ 5f877571 f
 0001:00076581       ?GetRuntimeClass@CInternetException@@UBEPAUCRuntimeClass@@XZ 5f877581 f
 0001:00076587       ?GetRuntimeClass@CHttpFile@@UBEPAUCRuntimeClass@@XZ 5f877587 f
 0001:0007658d       ?_GetBaseClass@CGopherFile@@KGPAUCRuntimeClass@@XZ 5f87758d f
 0001:00076593       ?GetRuntimeClass@CGopherFile@@UBEPAUCRuntimeClass@@XZ 5f877593 f
 0001:00076599       ?GetRuntimeClass@CInternetSession@@UBEPAUCRuntimeClass@@XZ 5f877599 f
 0001:0007659f       ?GetRuntimeClass@CFtpConnection@@UBEPAUCRuntimeClass@@XZ 5f87759f f
 0001:000765a5       ?GetRuntimeClass@CHttpConnection@@UBEPAUCRuntimeClass@@XZ 5f8775a5 f
 0001:000765ab       ?_GetBaseClass@CGopherConnection@@KGPAUCRuntimeClass@@XZ 5f8775ab f
 0001:000765b1       ?GetRuntimeClass@CGopherConnection@@UBEPAUCRuntimeClass@@XZ 5f8775b1 f
 0001:000765b7       ?GetRuntimeClass@CFtpFileFind@@UBEPAUCRuntimeClass@@XZ 5f8775b7 f
 0001:000765bd       ?GetRuntimeClass@CGopherFileFind@@UBEPAUCRuntimeClass@@XZ 5f8775bd f
 0001:000765c3       ?GetRuntimeClass@CFileFind@@UBEPAUCRuntimeClass@@XZ 5f8775c3 f
 0001:000765c9       ?_GetBaseClass@CSocket@@KGPAUCRuntimeClass@@XZ 5f8775c9 f
 0001:000765cf       ?GetRuntimeClass@CSocket@@UBEPAUCRuntimeClass@@XZ 5f8775cf f
 0001:000765d5       ?GetRuntimeClass@CSocketFile@@UBEPAUCRuntimeClass@@XZ 5f8775d5 f
 0001:000765db       ?CreateObject@?$CProcessLocal@V_AFX_SOCK_STATE@@@@SGPAVCNoTrackObject@@XZ 5f8775db f
 0001:0007664c       ?AfxBSTR2CString@@YGXPAVCString@@PAG@Z 5f87764c f
 0001:00076678       ?AfxAllocTaskWideString@@YGPAGPBG@Z 5f877678 f
 0001:000766b3       ?AfxAllocTaskWideString@@YGPAGPBD@Z 5f8776b3 f
 0001:000766f3       ?AfxAllocTaskAnsiString@@YGPADPBG@Z 5f8776f3 f
 0001:00076736       ?AfxAllocTaskAnsiString@@YGPADPBD@Z 5f877736 f
 0001:0007676f       ?GetRuntimeClass@COleDispatchException@@UBEPAUCRuntimeClass@@XZ 5f87776f f
 0001:00076775       ?GetRuntimeClass@COleInsertDialog@@UBEPAUCRuntimeClass@@XZ 5f877775 f
 0001:0007677b       ?GetRuntimeClass@COleConvertDialog@@UBEPAUCRuntimeClass@@XZ 5f87777b f
 0001:00076781       ?GetRuntimeClass@COleChangeIconDialog@@UBEPAUCRuntimeClass@@XZ 5f877781 f
 0001:00076787       ?_GetBaseClass@COleUpdateDialog@@KGPAUCRuntimeClass@@XZ 5f877787 f
 0001:0007678d       ?GetRuntimeClass@COleUpdateDialog@@UBEPAUCRuntimeClass@@XZ 5f87778d f
 0001:00076793       ?GetRuntimeClass@COlePasteSpecialDialog@@UBEPAUCRuntimeClass@@XZ 5f877793 f
 0001:00076799       ?GetRuntimeClass@COleBusyDialog@@UBEPAUCRuntimeClass@@XZ 5f877799 f
 0001:0007679f       ?GetRuntimeClass@COlePropertiesDialog@@UBEPAUCRuntimeClass@@XZ 5f87779f f
 0001:000767a5       ?_GetBaseClass@COleChangeSourceDialog@@KGPAUCRuntimeClass@@XZ 5f8777a5 f
 0001:000767ab       ?GetRuntimeClass@COleChangeSourceDialog@@UBEPAUCRuntimeClass@@XZ 5f8777ab f
 0001:000767b1       ?CreateObject@CDocItem@@SGPAVCObject@@XZ 5f8777b1 f
 0001:000767e3       ??5@YGAAVCArchive@@AAV0@AAPAVCDocItem@@@Z 5f8777e3 f
 0001:000767fe       ?_GetBaseClass@COleDocument@@KGPAUCRuntimeClass@@XZ 5f8777fe f
 0001:00076804       ?GetRuntimeClass@COleDocument@@UBEPAUCRuntimeClass@@XZ 5f877804 f
 0001:0007680a       ?_GetBaseClass@COleServerItem@@KGPAUCRuntimeClass@@XZ 5f87780a f
 0001:00076810       ?GetRuntimeClass@COleServerItem@@UBEPAUCRuntimeClass@@XZ 5f877810 f
 0001:0007681a       ??_ECOleObjectFactory@@UAEPAXI@Z 5f87781a f
 0001:0007681a       ??_GCOleObjectFactory@@UAEPAXI@Z 5f87781a f
 0001:0007683a       ?UnregisterAll@COleObjectFactory@@SGHXZ 5f87783a f
 0001:000768bb       ?CreateObject@COleIPFrameWnd@@SGPAVCObject@@XZ 5f8778bb f
 0001:000768f0       ?GetRuntimeClass@COleIPFrameWnd@@UBEPAUCRuntimeClass@@XZ 5f8778f0 f
 0001:000768f6       ?GetRuntimeClass@COleException@@UBEPAUCRuntimeClass@@XZ 5f8778f6 f
 0001:000768fc       ?GetRuntimeClass@COleStreamFile@@UBEPAUCRuntimeClass@@XZ 5f8778fc f
 0001:00076902       ?_GetBaseClass@COleServerDoc@@KGPAUCRuntimeClass@@XZ 5f877902 f
 0001:00076908       ?GetRuntimeClass@COleServerDoc@@UBEPAUCRuntimeClass@@XZ 5f877908 f
 0001:0007690e       ?CreateObject@CRichEditCntrItem@@SGPAVCObject@@XZ 5f87790e f
 0001:00076945       ?_GetBaseClass@CRichEditCntrItem@@KGPAUCRuntimeClass@@XZ 5f877945 f
 0001:0007694b       ?GetRuntimeClass@CRichEditCntrItem@@UBEPAUCRuntimeClass@@XZ 5f87794b f
 0001:00076951       ??5@YGAAVCArchive@@AAV0@AAPAVCRichEditCntrItem@@@Z 5f877951 f
 0001:0007696c       ?GetRuntimeClass@CRichEditDoc@@UBEPAUCRuntimeClass@@XZ 5f87796c f
 0001:00076972       ?CreateObject@CRichEditView@@SGPAVCObject@@XZ 5f877972 f
 0001:000769a7       ?GetRuntimeClass@CRichEditView@@UBEPAUCRuntimeClass@@XZ 5f8779a7 f
 0001:000769ad       ??I?$_CIP@UIMoniker@@$1?IID_IMoniker@@3U_GUID@@B@@QAEPAPAUIMoniker@@XZ 5f8779ad f
 0001:000769bc       ??7?$_CIP@UIBindCtx@@$1?IID_IBindCtx@@3U_GUID@@B@@QAEHXZ 5f8779bc f
 0001:000769c4       ??0?$CIP@UIBindHost@@$1?IID_IBindHost@@3U_GUID@@B@@QAE@PAUIBindHost@@H@Z 5f8779c4 f
 0001:000769da       ?Detach@?$_CIP@UIStream@@$1?IID_IStream@@3U_GUID@@B@@QAEXXZ 5f8779da f
 0001:000769de       ??0?$_CIP@UIBindCtx@@$1?IID_IBindCtx@@3U_GUID@@B@@QAE@PAUIBindCtx@@H@Z 5f8779de f
 0001:000769f9       ??0?$_CIP@UIMoniker@@$1?IID_IMoniker@@3U_GUID@@B@@QAE@XZ 5f8779f9 f
 0001:000769ff       ?GetRuntimeClass@CDateTimeCtrl@@UBEPAUCRuntimeClass@@XZ 5f8779ff f
 0001:00076a05       ?GetRuntimeClass@CMonthCalCtrl@@UBEPAUCRuntimeClass@@XZ 5f877a05 f
 0001:00076a0b       ?CreateObject@CHtmlView@@SGPAVCObject@@XZ 5f877a0b f
 0001:00076a40       ?GetRuntimeClass@CHtmlView@@UBEPAUCRuntimeClass@@XZ 5f877a40 f
 0001:00076a46       ?_GetBaseClass@CAsyncMonikerFile@@KGPAUCRuntimeClass@@XZ 5f877a46 f
 0001:00076a4c       ?GetRuntimeClass@CAsyncMonikerFile@@UBEPAUCRuntimeClass@@XZ 5f877a4c f
 0001:00076a52       ??C?$_CIP@UIBinding@@$1?IID_IBinding@@3U_GUID@@B@@QBEPAUIBinding@@XZ 5f877a52 f
 0001:00076a55       ?Release@?$_CIP@UIBinding@@$1?IID_IBinding@@3U_GUID@@B@@QAEXXZ 5f877a55 f
 0001:00076a65       ??0?$CIP@UIBindHost@@$1?IID_IBindHost@@3U_GUID@@B@@QAE@XZ 5f877a65 f
 0001:00076a71       ??4?$CIP@UIBindHost@@$1?IID_IBindHost@@3U_GUID@@B@@QAEAAV0@PAUIBindHost@@@Z 5f877a71 f
 0001:00076a83       ?QueryInterface@?$_CIP@UIBindHost@@$1?IID_IBindHost@@3U_GUID@@B@@QAEJPAUIUnknown@@@Z 5f877a83 f
 0001:00076acb       ?QueryInterface@?$_CIP@UIBindStatusCallback@@$1?IID_IBindStatusCallback@@3U_GUID@@B@@QAEJPAUIUnknown@@@Z 5f877acb f
 0001:00076b13       ?QueryInterface@?$_CIP@UIServiceProvider@@$1?IID_IServiceProvider@@3U_GUID@@B@@QAEJPAUIUnknown@@@Z 5f877b13 f
 0001:00076b5b       ?GetIID@?$_CIP@UIBindHost@@$1?IID_IBindHost@@3U_GUID@@B@@SAABU_GUID@@XZ 5f877b5b f
 0001:00076b61       ?Attach@?$_CIP@UIBindHost@@$1?IID_IBindHost@@3U_GUID@@B@@QAEXPAUIBindHost@@@Z 5f877b61 f
 0001:00076b73       ?GetIID@?$_CIP@UIBindStatusCallback@@$1?IID_IBindStatusCallback@@3U_GUID@@B@@SAABU_GUID@@XZ 5f877b73 f
 0001:00076b79       ?GetIID@?$_CIP@UIServiceProvider@@$1?IID_IServiceProvider@@3U_GUID@@B@@SAABU_GUID@@XZ 5f877b79 f
 0001:00076b7f       ?_AddRef@?$_CIP@UIBindStatusCallback@@$1?IID_IBindStatusCallback@@3U_GUID@@B@@AAEXXZ 5f877b7f f
 0001:00076b8c       ?_Release@?$_CIP@UIBindStatusCallback@@$1?IID_IBindStatusCallback@@3U_GUID@@B@@AAEXXZ 5f877b8c f
 0001:00076b8c       ??1?$CIP@UIServiceProvider@@$1?IID_IServiceProvider@@3U_GUID@@B@@QAE@XZ 5f877b8c f
 0001:00076b99       ??1?$_CIP@UIServiceProvider@@$1?IID_IServiceProvider@@3U_GUID@@B@@QAE@XZ 5f877b99 f
 0001:00076b9b       ??4?$_CIP@UIBinding@@$1?IID_IBinding@@3U_GUID@@B@@QAEAAV0@PAUIBinding@@@Z 5f877b9b f
 0001:00076bc1       ?_GetBaseClass@COleResizeBar@@KGPAUCRuntimeClass@@XZ 5f877bc1 f
 0001:00076bc7       ?GetRuntimeClass@COleResizeBar@@UBEPAUCRuntimeClass@@XZ 5f877bc7 f
 0001:00076bcd       ?GetRuntimeClass@COleControl@@UBEPAUCRuntimeClass@@XZ 5f877bcd f
 0001:00076bd3       ?CreateObject@?$CThreadLocal@V_AFXCTL_AMBIENT_CACHE@@@@SGPAVCNoTrackObject@@XZ 5f877bd3 f
 0001:00076c04       ?_GetBaseClass@CCachedDataPathProperty@@KGPAUCRuntimeClass@@XZ 5f877c04 f
 0001:00076c0a       ?GetRuntimeClass@CCachedDataPathProperty@@UBEPAUCRuntimeClass@@XZ 5f877c0a f
 0001:00076c10       ?CreateObject@CColorPropPage@@SGPAVCObject@@XZ 5f877c10 f
 0001:00076c45       ?GetRuntimeClass@CColorPropPage@@UBEPAUCRuntimeClass@@XZ 5f877c45 f
 0001:00076c4b       ?CreateObject@CFontPropPage@@SGPAVCObject@@XZ 5f877c4b f
 0001:00076c80       ?GetRuntimeClass@CFontPropPage@@UBEPAUCRuntimeClass@@XZ 5f877c80 f
 0001:00076c86       ?CreateObject@CPicturePropPage@@SGPAVCObject@@XZ 5f877c86 f
 0001:00076cbb       ?GetRuntimeClass@CPicturePropPage@@UBEPAUCRuntimeClass@@XZ 5f877cbb f
 0001:00076cc1       ?_GetBaseClass@CStockPropPage@@KGPAUCRuntimeClass@@XZ 5f877cc1 f
 0001:00076cc7       ?GetRuntimeClass@CStockPropPage@@UBEPAUCRuntimeClass@@XZ 5f877cc7 f
 0001:00076ccd       ?_GetBaseClass@CDBException@@KGPAUCRuntimeClass@@XZ 5f877ccd f
 0001:00076cd3       ?GetRuntimeClass@CDBException@@UBEPAUCRuntimeClass@@XZ 5f877cd3 f
 0001:00076cd9       ?GetRuntimeClass@CDatabase@@UBEPAUCRuntimeClass@@XZ 5f877cd9 f
 0001:00076cdf       ?GetRuntimeClass@CRecordset@@UBEPAUCRuntimeClass@@XZ 5f877cdf f
 0001:00076ce5       ?CreateObject@?$CProcessLocal@V_AFX_DB_STATE@@@@SGPAVCNoTrackObject@@XZ 5f877ce5 f
 0001:00076cfa       ?GetRuntimeClass@CRecordView@@UBEPAUCRuntimeClass@@XZ 5f877cfa f
 0001:00076d00       ?GetRuntimeClass@CLongBinary@@UBEPAUCRuntimeClass@@XZ 5f877d00 f
 0001:00076d06       ?_GetBaseClass@COleDBRecordView@@KGPAUCRuntimeClass@@XZ 5f877d06 f
 0001:00076d0c       ?GetRuntimeClass@COleDBRecordView@@UBEPAUCRuntimeClass@@XZ 5f877d0c f
 0001:00076d12       ?GetRuntimeClass@CDynLinkLibrary@@UBEPAUCRuntimeClass@@XZ 5f877d12 f
 0001:00076d18       ??0CDynLinkLibrary@@QAE@PAUHINSTANCE__@@0@Z 5f877d18 f
 0001:00076de6       ?AfxCoreInitModule@@YGXXZ  5f877de6 f
 0001:00076e4f       _DllGetClassObject@12      5f877e4f f
 0001:00076e7d       _DllCanUnloadNow@0         5f877e7d f
 0001:00076ea0       _DllRegisterServer@0       5f877ea0 f
 0001:00076ed2       _DllUnregisterServer@0     5f877ed2 f
 0001:00076f04       ?AfxWndProcDllOle@@YGJPAUHWND__@@IIJ@Z 5f877f04 f
 0001:00076f4a       ??1_AFX_MAIL_STATE@@UAE@XZ 5f877f4a f
 0001:00076f5f       ??_E_AFX_MAIL_STATE@@UAEPAXI@Z 5f877f5f f
 0001:00076f5f       ??_G_AFX_MAIL_STATE@@UAEPAXI@Z 5f877f5f f
 0001:00076f7a       ?OnFileSendMail@CDocument@@IAEXXZ 5f877f7a f
 0001:00077300       ?OnFileSendMail@COleDocument@@IAEXXZ 5f878300 f
 0001:00077367       ??0COleClientItem@@QAE@PAVCOleDocument@@@Z 5f878367 f
 0001:00077403       ??_ECOleClientItem@@UAEPAXI@Z 5f878403 f
 0001:00077403       ??_GCOleClientItem@@UAEPAXI@Z 5f878403 f
 0001:0007741f       ?Delete@COleClientItem@@QAEXH@Z 5f87841f f
 0001:0007747d       ?Release@COleClientItem@@UAEXW4tagOLECLOSE@@@Z 5f87847d f
 0001:0007752f       ?Close@COleClientItem@@QAEXW4tagOLECLOSE@@@Z 5f87852f f
 0001:000775a8       ?GetNewItemNumber@COleClientItem@@QAEKXZ 5f8785a8 f
 0001:000775f7       ?GetItemName@COleClientItem@@QBEXPAG@Z 5f8785f7 f
 0001:0007760f       ?GetIconFromRegistry@COleClientItem@@QBEPAUHICON__@@XZ 5f87860f f
 0001:00077643       ?GetIconFromRegistry@COleClientItem@@SAPAUHICON__@@AAU_GUID@@@Z 5f878643 f
 0001:00077846       ?UpdateItemType@COleClientItem@@QAEXXZ 5f878846 f
 0001:00077899       ?FinishCreate@COleClientItem@@MAEHJ@Z 5f878899 f
 0001:000779a9       ?CreateFromClipboard@COleClientItem@@QAEHW4tagOLERENDER@@GPAUtagFORMATETC@@@Z 5f8789a9 f
 0001:00077a08       ?CreateLinkFromClipboard@COleClientItem@@QAEHW4tagOLERENDER@@GPAUtagFORMATETC@@@Z 5f878a08 f
 0001:00077a67       ?CreateStaticFromClipboard@COleClientItem@@QAEHW4tagOLERENDER@@GPAUtagFORMATETC@@@Z 5f878a67 f
 0001:00077ac6       ?CreateFromData@COleClientItem@@QAEHPAVCOleDataObject@@W4tagOLERENDER@@GPAUtagFORMATETC@@@Z 5f878ac6 f
 0001:00077b34       ?CreateLinkFromData@COleClientItem@@QAEHPAVCOleDataObject@@W4tagOLERENDER@@GPAUtagFORMATETC@@@Z 5f878b34 f
 0001:00077ba2       ?CreateStaticFromData@COleClientItem@@QAEHPAVCOleDataObject@@W4tagOLERENDER@@GPAUtagFORMATETC@@@Z 5f878ba2 f
 0001:00077c10       ?CreateFromFile@COleClientItem@@QAEHPBGABU_GUID@@W4tagOLERENDER@@GPAUtagFORMATETC@@@Z 5f878c10 f
 0001:00077c75       ?CreateLinkFromFile@COleClientItem@@QAEHPBGW4tagOLERENDER@@GPAUtagFORMATETC@@@Z 5f878c75 f
 0001:00077cd7       ?CreateNewItem@COleClientItem@@QAEHABU_GUID@@W4tagOLERENDER@@GPAUtagFORMATETC@@@Z 5f878cd7 f
 0001:00077d39       ?CreateCloneFrom@COleClientItem@@QAEHPBV1@@Z 5f878d39 f
 0001:00077de6       ?IsModified@COleClientItem@@QBEHXZ 5f878de6 f
 0001:00077e57       ?GetItemStorageFlat@COleClientItem@@QAEXXZ 5f878e57 f
 0001:00077ea0       ?ReadItemFlat@COleClientItem@@QAEXAAVCArchive@@@Z 5f878ea0 f
 0001:00077fab       ?WriteItemFlat@COleClientItem@@QAEXAAVCArchive@@@Z 5f878fab f
 0001:00078064       ?ReadItemCompound@COleClientItem@@QAEXAAVCArchive@@@Z 5f879064 f
 0001:0007817e       ?WriteItemCompound@COleClientItem@@QAEXAAVCArchive@@@Z 5f87917e f
 0001:00078281       ?GetItemStorage@COleClientItem@@UAEXXZ 5f879281 f
 0001:0007828e       ?GetItemStorageCompound@COleClientItem@@QAEXXZ 5f87928e f
 0001:000782ee       ?ReadItem@COleClientItem@@UAEXAAVCArchive@@@Z 5f8792ee f
 0001:0007830a       ?WriteItem@COleClientItem@@UAEXAAVCArchive@@@Z 5f87930a f
 0001:00078326       ?CommitItem@COleClientItem@@UAEXH@Z 5f879326 f
 0001:00078384       ?Serialize@COleClientItem@@UAEXAAVCArchive@@@Z 5f879384 f
 0001:000784c4       ?OnChange@COleClientItem@@UAEXW4OLE_NOTIFICATION@@K@Z 5f8794c4 f
 0001:000784df       ?OnGetItemPosition@COleClientItem@@MAEXAAVCRect@@@Z 5f8794df f
 0001:000784e2       ?OnGetClipRect@COleClientItem@@MAEXAAVCRect@@@Z 5f8794e2 f
 0001:000784f5       ?OnShowItem@COleClientItem@@MAEXXZ 5f8794f5 f
 0001:00078580       ?GetClassID@COleClientItem@@QBEXPAU_GUID@@@Z 5f879580 f
 0001:000785a2       ?GetExtent@COleClientItem@@QAEHPAUtagSIZE@@W4tagDVASPECT@@@Z 5f8795a2 f
 0001:000785cf       ?GetCachedExtent@COleClientItem@@QAEHPAUtagSIZE@@W4tagDVASPECT@@@Z 5f8795cf f
 0001:00078609       ?SetIconicMetafile@COleClientItem@@QAEHPAX@Z 5f879609 f
 0001:00078694       ?GetIconicMetafile@COleClientItem@@QAEPAXXZ 5f879694 f
 0001:000787af       ?SetDrawAspect@COleClientItem@@UAEXW4tagDVASPECT@@@Z 5f8797af f
 0001:000787e2       ?GetPrintDeviceInfo@COleClientItem@@IAEHPAPAUIOleCache@@PAPAUtagDVTARGETDEVICE@@PAK@Z 5f8797e2 f
 0001:00078873       ?AttachDataObject@COleClientItem@@QBEXAAVCOleDataObject@@@Z 5f879873 f
 0001:0007888f       ?Draw@COleClientItem@@QAEHPAVCDC@@PBUtagRECT@@W4tagDVASPECT@@@Z 5f87988f f
 0001:000789a8       ?GetEmbeddedItemData@COleClientItem@@IAEXPAUtagSTGMEDIUM@@@Z 5f8799a8 f
 0001:00078a51       ?AddCachedData@COleClientItem@@IAEXPAVCOleDataSource@@@Z 5f879a51 f
 0001:00078b1e       ?GetLinkSourceData@COleClientItem@@IAEHPAUtagSTGMEDIUM@@@Z 5f879b1e f
 0001:00078c24       ?GetObjectDescriptorData@COleClientItem@@IAEXPAUtagPOINT@@PAUtagSIZE@@PAUtagSTGMEDIUM@@@Z 5f879c24 f
 0001:00078cce       ?SetHostNames@COleClientItem@@QAEXPBG0@Z 5f879cce f
 0001:00078cf3       ?SetExtent@COleClientItem@@QAEXABVCSize@@W4tagDVASPECT@@@Z 5f879cf3 f
 0001:00078d18       ?_GetBaseInterfaceMap@COleClientItem@@KGPBUAFX_INTERFACEMAP@@XZ 5f879d18 f
 0001:00078d1e       ?GetInterfaceMap@COleClientItem@@MBEPBUAFX_INTERFACEMAP@@XZ 5f879d1e f
 0001:00078d24       ?AddRef@XOleClientSite@COleClientItem@@UAGKXZ 5f879d24 f
 0001:00078d33       ?Release@XOleClientSite@COleClientItem@@UAGKXZ 5f879d33 f
 0001:00078d42       ?QueryInterface@XOleClientSite@COleClientItem@@UAGJABU_GUID@@PAPAX@Z 5f879d42 f
 0001:00078d59       ?SaveObject@XOleClientSite@COleClientItem@@UAGJXZ 5f879d59 f
 0001:00078ddb       ?GetMoniker@XOleClientSite@COleClientItem@@UAGJKKPAPAUIMoniker@@@Z 5f879ddb f
 0001:00078f54       ?GetContainer@XOleClientSite@COleClientItem@@UAGJPAPAUIOleContainer@@@Z 5f879f54 f
 0001:00078f7a       ?ShowObject@XOleClientSite@COleClientItem@@UAGJXZ 5f879f7a f
 0001:00078fda       ?OnShowWindow@XOleClientSite@COleClientItem@@UAGJH@Z 5f879fda f
 0001:0007905a       ?RequestNewObjectLayout@XOleClientSite@COleClientItem@@UAGJXZ 5f87a05a f
 0001:00079062       ?AddRef@XAdviseSink@COleClientItem@@UAGKXZ 5f87a062 f
 0001:00079071       ?Release@XAdviseSink@COleClientItem@@UAGKXZ 5f87a071 f
 0001:00079080       ?QueryInterface@XAdviseSink@COleClientItem@@UAGJABU_GUID@@PAPAX@Z 5f87a080 f
 0001:00079097       ?OnDataChange@XAdviseSink@COleClientItem@@UAGXPAUtagFORMATETC@@PAUtagSTGMEDIUM@@@Z 5f87a097 f
 0001:000790e1       ?OnViewChange@XAdviseSink@COleClientItem@@UAGXKJ@Z 5f87a0e1 f
 0001:00079127       ?OnSave@XAdviseSink@COleClientItem@@UAGXXZ 5f87a127 f
 0001:0007916c       ?OnClose@XAdviseSink@COleClientItem@@UAGXXZ 5f87a16c f
 0001:000791b1       ?GetClientSite@COleClientItem@@MAEPAUIOleClientSite@@XZ 5f87a1b1 f
 0001:000791bc       ?Activate@COleClientItem@@QAEXJPAVCView@@PAUtagMSG@@@Z 5f87a1bc f
 0001:0007928a       ?CheckGeneral@COleClientItem@@MAEXJ@Z 5f87a28a f
 0001:000792a4       ?CopyToClipboard@COleClientItem@@QAEXH@Z 5f87a2a4 f
 0001:000792f7       ?OnGetClipboardData@COleClientItem@@UAEPAVCOleDataSource@@HPAUtagPOINT@@PAUtagSIZE@@@Z 5f87a2f7 f
 0001:00079374       ?DoDragDrop@COleClientItem@@QAEKPBUtagRECT@@VCPoint@@HK0@Z 5f87a374 f
 0001:0007944d       ?GetClipboardData@COleClientItem@@QAEXPAVCOleDataSource@@HPAUtagPOINT@@PAUtagSIZE@@@Z 5f87a44d f
 0001:000794f7       ?CanPaste@COleClientItem@@SGHXZ 5f87a4f7 f
 0001:00079567       ?CanPasteLink@COleClientItem@@SGHXZ 5f87a567 f
 0001:000795a5       ?CanCreateFromData@COleClientItem@@SGHPBVCOleDataObject@@@Z 5f87a5a5 f
 0001:000795df       ?CanCreateLinkFromData@COleClientItem@@SGHPBVCOleDataObject@@@Z 5f87a5df f
 0001:00079619       ?ConvertTo@COleClientItem@@UAEHABU_GUID@@@Z 5f87a619 f
 0001:000796bb       ?Reload@COleClientItem@@QAEHXZ 5f87a6bb f
 0001:000796f9       ?ActivateAs@COleClientItem@@UAEHPBGABU_GUID@@1@Z 5f87a6f9 f
 0001:00079748       ?SetPrintDevice@COleClientItem@@QAEHPBUtagDVTARGETDEVICE@@@Z 5f87a748 f
 0001:00079838       ?SetPrintDevice@COleClientItem@@QAEHPBUtagPDW@@@Z 5f87a838 f
 0001:00079867       ?GetUserType@COleClientItem@@QAEXW4tagUSERCLASSTYPE@@AAVCString@@@Z 5f87a867 f
 0001:000798a3       ?Run@COleClientItem@@QAEXXZ 5f87a8a3 f
 0001:000798c9       ?UpdateLink@COleClientItem@@QAEHXZ 5f87a8c9 f
 0001:000798fd       ?FreezeLink@COleClientItem@@UAEHXZ 5f87a8fd f
 0001:00079a48       ?GetLinkUpdateOptions@COleClientItem@@QAE?AW4tagOLEUPDATE@@XZ 5f87aa48 f
 0001:00079a85       ?SetLinkUpdateOptions@COleClientItem@@QAEXW4tagOLEUPDATE@@@Z 5f87aa85 f
 0001:00079abc       ??_GCOleDocument@@UAEPAXI@Z 5f87aabc f
 0001:00079abc       ??_ECOleDocument@@UAEPAXI@Z 5f87aabc f
 0001:00079afc       ?AddItem@COleDocument@@UAEXPAVCDocItem@@@Z 5f87aafc f
 0001:00079b15       ?RemoveItem@COleDocument@@UAEXPAVCDocItem@@@Z 5f87ab15 f
 0001:00079b39       ?GetNextItem@COleDocument@@UBEPAVCDocItem@@AAPAU__POSITION@@@Z 5f87ab39 f
 0001:00079b9e       ?SetPathName@COleDocument@@UAEXPBGH@Z 5f87ab9e f
 0001:00079bfd       ?Serialize@COleDocument@@UAEXAAVCArchive@@@Z 5f87abfd f
 0001:00079cad       ?CommitItems@COleDocument@@QAEXH@Z 5f87acad f
 0001:00079ce2       ?HasBlankItems@COleDocument@@QBEHXZ 5f87ace2 f
 0001:00079e0d       ?GetFirstFrame@COleDocument@@QAEPAVCFrameWnd@@XZ 5f87ae0d f
 0001:00079e37       ?GetMoniker@COleDocument@@UAEPAUIMoniker@@W4tagOLEGETMONIKER@@@Z 5f87ae37 f
 0001:00079fbf       ?OnSaveDocument@COleDocument@@UAEHPBG@Z 5f87afbf f
 0001:0007a15b       ?SaveToStorage@COleDocument@@MAEXPAVCObject@@@Z 5f87b15b f
 0001:0007a2c6       ?LoadFromStorage@COleDocument@@MAEXXZ 5f87b2c6 f
 0001:0007a424       ??0CDocItem@@IAE@XZ        5f87b424 f
 0001:0007a43a       ??_GCDocItem@@UAEPAXI@Z    5f87b43a f
 0001:0007a43a       ??_ECDocItem@@UAEPAXI@Z    5f87b43a f
 0001:0007a456       ?Serialize@CDocItem@@UAEXAAVCArchive@@@Z 5f87b456 f
 0001:0007a47a       ?ApplyPrintDevice@COleDocument@@QAEHPBUtagDVTARGETDEVICE@@@Z 5f87b47a f
 0001:0007a4e0       ?ApplyPrintDevice@COleDocument@@QAEHPBUtagPDW@@@Z 5f87b4e0 f
 0001:0007a50f       ?AfxThrowOleException@@YGXJ@Z 5f87b50f f
 0001:0007a55d       ?GetErrorMessage@COleException@@UAEHPAGIPAI@Z 5f87b55d f
 0001:0007a5b8       ?Process@COleException@@SGJPBVCException@@@Z 5f87b5b8 f
 0001:0007a606       ?AfxMergeMenus@@YGPAUHMENU__@@PAU1@0PAJHH@Z 5f87b606 f
 0001:0007a7d9       ?AfxUnmergeMenus@@YGXPAUHMENU__@@00@Z 5f87b7d9 f
 0001:0007a881       ?_AfxFillFormatEtc@@YGPAUtagFORMATETC@@PAU1@G0@Z 5f87b881 f
 0001:0007a8b0       ?_AfxCopyGlobalMemory@@YGPAXPAX0@Z 5f87b8b0 f
 0001:0007a91c       ?_AfxCopyStgMedium@@YGHGPAUtagSTGMEDIUM@@0@Z 5f87b91c f
 0001:0007ab5b       ?_AfxOleGetObjectDescriptorData@@YGPAXU_GUID@@KUtagSIZE@@U_POINTL@@KPBG3@Z 5f87bb5b f
 0001:0007ac4a       ?_AfxOleGetObjectDescriptorData@@YGPAXPAUIOleObject@@PBGKU_POINTL@@PAUtagSIZE@@@Z 5f87bc4a f
 0001:0007ae48       ?_AfxOleDoConvert@@YGJPAUIStorage@@ABU_GUID@@@Z 5f87be48 f
 0001:0007af05       ?_AfxOleDoTreatAsClass@@YGJPBGABU_GUID@@1@Z 5f87bf05 f
 0001:0007af8b       ?_AfxOleCreateTargetDevice@@YGPAUtagDVTARGETDEVICE@@PAUtagDEVNAMES@@PAU_devicemodeW@@@Z 5f87bf8b f
 0001:0007b0ec       ?_AfxOleCreateTargetDevice@@YGPAUtagDVTARGETDEVICE@@PAUtagPDW@@@Z 5f87c0ec f
 0001:0007b13b       ?_AfxOleGetFirstMoniker@@YGPAUIMoniker@@PAU1@@Z 5f87c13b f
 0001:0007b1a3       ?_AfxOleGetLenFilePrefixOfMoniker@@YGKPAUIMoniker@@@Z 5f87c1a3 f
 0001:0007b237       ?_AfxOleCopyTargetDevice@@YGPAUtagDVTARGETDEVICE@@PAU1@@Z 5f87c237 f
 0001:0007b266       ?_AfxOleCopyFormatEtc@@YGXPAUtagFORMATETC@@0@Z 5f87c266 f
 0001:0007b298       ?_AfxOleCreateDC@@YGPAUHDC__@@PAUtagDVTARGETDEVICE@@@Z 5f87c298 f
 0001:0007b2e3       ?_AfxDeleteMetafilePict@@YGXPAX@Z 5f87c2e3 f
 0001:0007b30c       ?_AfxXformSizeInPixelsToHimetric@@YGXPAUHDC__@@PAUtagSIZE@@1@Z 5f87c30c f
 0001:0007b373       ?_AfxXformSizeInHimetricToPixels@@YGXPAUHDC__@@PAUtagSIZE@@1@Z 5f87c373 f
 0001:0007b3e0       ??0COleStreamFile@@QAE@PAUIStream@@@Z 5f87c3e0 f
 0001:0007b475       ?Detach@COleStreamFile@@QAEPAUIStream@@XZ 5f87c475 f
 0001:0007b47d       ?Attach@COleStreamFile@@QAEXPAUIStream@@@Z 5f87c47d f
 0001:0007b48b       ?_AfxReadFromStream@@YGJPAUIStream@@PAXIAAK@Z 5f87c48b f
 0001:0007b4b4       ?_AfxFillOleFileException@@YGXPAVCFileException@@J@Z 5f87c4b4 f
 0001:0007b51d       ?_AfxThrowOleFileException@@YGXJ@Z 5f87c51d f
 0001:0007b5a3       ?GetStatus@COleStreamFile@@QBEHAAUCFileStatus@@@Z 5f87c5a3 f
 0001:0007b634       ?GetStorageName@COleStreamFile@@UBE?BVCString@@XZ 5f87c634 f
 0001:0007b64f       ?GetPosition@COleStreamFile@@UBEKXZ 5f87c64f f
 0001:0007b67c       ?OpenStream@COleStreamFile@@QAEHPAUIStorage@@PBGKPAVCFileException@@@Z 5f87c67c f
 0001:0007b6b8       ?CreateStream@COleStreamFile@@QAEHPAUIStorage@@PBGKPAVCFileException@@@Z 5f87c6b8 f
 0001:0007b73a       ?CreateMemoryStream@COleStreamFile@@QAEHPAVCFileException@@@Z 5f87c73a f
 0001:0007b76b       ?Duplicate@COleStreamFile@@UBEPAVCFile@@XZ 5f87c76b f
 0001:0007b7e3       ?Seek@COleStreamFile@@UAEJJI@Z 5f87c7e3 f
 0001:0007b818       ?SetLength@COleStreamFile@@UAEXK@Z 5f87c818 f
 0001:0007b838       ?GetLength@COleStreamFile@@UBEKXZ 5f87c838 f
 0001:0007b85c       ?Read@COleStreamFile@@UAEIPAXI@Z 5f87c85c f
 0001:0007b882       ?Write@COleStreamFile@@UAEXPBXI@Z 5f87c882 f
 0001:0007b8ac       ?LockRange@COleStreamFile@@UAEXKK@Z 5f87c8ac f
 0001:0007b8da       ?UnlockRange@COleStreamFile@@UAEXKK@Z 5f87c8da f
 0001:0007b908       ?Abort@COleStreamFile@@UAEXXZ 5f87c908 f
 0001:0007b92d       ?Flush@COleStreamFile@@UAEXXZ 5f87c92d f
 0001:0007b943       ?Close@COleStreamFile@@UAEXXZ 5f87c943 f
 0001:0007b966       ?GetStream@COleStreamFile@@QBEPAUIStream@@XZ 5f87c966 f
 0001:0007b96a       ?EnableAggregation@CCmdTarget@@QAEXXZ 5f87c96a f
 0001:0007b9e3       ?AddRef@CInnerUnknown@@UAGKXZ 5f87c9e3 f
 0001:0007b9f4       ?Release@CInnerUnknown@@UAGKXZ 5f87c9f4 f
 0001:0007ba35       ?QueryInterface@CInnerUnknown@@UAGJABU_GUID@@PAPAX@Z 5f87ca35 f
 0001:0007ba7c       ?GetControllingUnknown@CCmdTarget@@QAEPAUIUnknown@@XZ 5f87ca7c f
 0001:0007ba8e       ?Flush@CMonikerFile@@UAEXXZ 5f87ca8e f
 0001:0007ba9c       ?Open@CMonikerFile@@MAEHPBGPAUIBindHost@@PAUIBindStatusCallback@@PAUIBindCtx@@PAVCFileException@@@Z 5f87ca9c f
 0001:0007bac2       ?Attach@CMonikerFile@@IAEHPBGPAUIBindHost@@PAUIBindStatusCallback@@PAUIBindCtx@@PAVCFileException@@@Z 5f87cac2 f
 0001:0007bb85       ?Open@CMonikerFile@@UAEHPBGPAVCFileException@@@Z 5f87cb85 f
 0001:0007bc0e       ?Open@CMonikerFile@@UAEHPAUIMoniker@@PAVCFileException@@@Z 5f87cc0e f
 0001:0007bc9a       ?Open@CMonikerFile@@MAEHPAUIMoniker@@PAUIBindHost@@PAUIBindStatusCallback@@PAUIBindCtx@@PAVCFileException@@@Z 5f87cc9a f
 0001:0007bcc0       ?Attach@CMonikerFile@@IAEHPAUIMoniker@@PAUIBindHost@@PAUIBindStatusCallback@@PAUIBindCtx@@PAVCFileException@@@Z 5f87ccc0 f
 0001:0007bd78       ?Close@CMonikerFile@@UAEXXZ 5f87cd78 f
 0001:0007bd9b       ?Detach@CMonikerFile@@QAEHPAVCFileException@@@Z 5f87cd9b f
 0001:0007bdfd       ?CreateBindHost@CMonikerFile@@KAPAUIBindHost@@XZ 5f87cdfd f
 0001:0007be3f       ??0_AfxBindHost@@QAE@XZ    5f87ce3f f
 0001:0007be55       ?AddRef@_AfxBindHost@@UAGKXZ 5f87ce55 f
 0001:0007be66       ?Release@_AfxBindHost@@UAGKXZ 5f87ce66 f
 0001:0007be90       ?QueryInterface@_AfxBindHost@@UAGJABU_GUID@@PAPAX@Z 5f87ce90 f
 0001:0007bee5       ?CreateMoniker@_AfxBindHost@@UAGJPAGPAUIBindCtx@@PAPAUIMoniker@@K@Z 5f87cee5 f
 0001:0007bf28       ?MonikerBindToStorage@_AfxBindHost@@UAGJPAUIMoniker@@PAUIBindCtx@@PAUIBindStatusCallback@@ABU_GUID@@PAPAX@Z 5f87cf28 f
 0001:0007c00d       ?MonikerBindToObject@_AfxBindHost@@EAGJPAUIMoniker@@PAUIBindCtx@@PAUIBindStatusCallback@@ABU_GUID@@PAPAX@Z 5f87d00d f
 0001:0007c015       ??0IBindHost@@QAE@XZ       5f87d015 f
 0001:0007c027       ??_G_AfxBindHost@@QAEPAXI@Z 5f87d027 f
 0001:0007c043       ??1_AfxBindHost@@QAE@XZ    5f87d043 f
 0001:0007c04a       ??0IUnknown@@QAE@XZ        5f87d04a f
 0001:0007c04d       ?CreateBindContext@CMonikerFile@@IAEPAUIBindCtx@@PAVCFileException@@@Z 5f87d04d f
 0001:0007c052       ?PostBindToStream@CMonikerFile@@MAEHPAVCFileException@@@Z 5f87d052 f
 0001:0007c0b1       ?_AfxTrySPForBindHost@@YGPAUIBindHost@@PAUIServiceProvider@@@Z 5f87d0b1 f
 0001:0007c0d7       ?_AfxTryQIForBindHost@@YGPAUIBindHost@@PAUIUnknown@@@Z 5f87d0d7 f
 0001:0007c126       ??0CAsyncMonikerFile@@QAE@XZ 5f87d126 f
 0001:0007c165       ?EndCallbacks@CAsyncMonikerFile@@IAEXXZ 5f87d165 f
 0001:0007c188       ?Orphan@_AfxBindStatusCallback@@QAEXXZ 5f87d188 f
 0001:0007c18d       ?GetInnerUnknown@_AfxBindStatusCallback@@QAEPAUIUnknown@@XZ 5f87d18d f
 0001:0007c191       ?Read@CAsyncMonikerFile@@UAEIPAXI@Z 5f87d191 f
 0001:0007c1c5       ?Close@CAsyncMonikerFile@@UAEXXZ 5f87d1c5 f
 0001:0007c202       ?Open@CAsyncMonikerFile@@UAEHPAUIMoniker@@PAUIBindHost@@PAVCFileException@@@Z 5f87d202 f
 0001:0007c2e8       ??1?$CIP@UIUnknown@@$1?IID_IUnknown@@3U_GUID@@B@@QAE@XZ 5f87d2e8 f
 0001:0007c2ed       ?Open@CAsyncMonikerFile@@UAEHPBGPAUIBindHost@@PAVCFileException@@@Z 5f87d2ed f
 0001:0007c3d3       ?Open@CAsyncMonikerFile@@UAEHPBGPAVCFileException@@@Z 5f87d3d3 f
 0001:0007c42f       ?Open@CAsyncMonikerFile@@UAEHPAUIMoniker@@PAVCFileException@@@Z 5f87d42f f
 0001:0007c48b       ?Open@CAsyncMonikerFile@@UAEHPBGPAUIServiceProvider@@PAVCFileException@@@Z 5f87d48b f
 0001:0007c540       ?Open@CAsyncMonikerFile@@UAEHPBGPAUIUnknown@@PAVCFileException@@@Z 5f87d540 f
 0001:0007c62f       ?Open@CAsyncMonikerFile@@UAEHPAUIMoniker@@PAUIServiceProvider@@PAVCFileException@@@Z 5f87d62f f
 0001:0007c6e4       ?Open@CAsyncMonikerFile@@UAEHPAUIMoniker@@PAUIUnknown@@PAVCFileException@@@Z 5f87d6e4 f
 0001:0007c7d9       ?PostBindToStream@CAsyncMonikerFile@@MAEHPAVCFileException@@@Z 5f87d7d9 f
 0001:0007c7ff       ?CreateBindStatusCallback@CAsyncMonikerFile@@MAEPAUIUnknown@@PAU2@@Z 5f87d7ff f
 0001:0007c859       ??0_AfxBindStatusCallback@@QAE@PAVCAsyncMonikerFile@@PAUIUnknown@@@Z 5f87d859 f
 0001:0007c8a7       ??0CInnerUnknown@_AfxBindStatusCallback@@QAE@XZ 5f87d8a7 f
 0001:0007c8b9       ?SetpThis@CInnerUnknown@_AfxBindStatusCallback@@QAEXPAV2@@Z 5f87d8b9 f
 0001:0007c8c3       ?AddRef@CInnerUnknown@_AfxBindStatusCallback@@UAGKXZ 5f87d8c3 f
 0001:0007c8d7       ?Release@CInnerUnknown@_AfxBindStatusCallback@@UAGKXZ 5f87d8d7 f
 0001:0007c905       ?QueryInterface@CInnerUnknown@_AfxBindStatusCallback@@UAGJABU_GUID@@PAPAX@Z 5f87d905 f
 0001:0007c963       ?AddRef@_AfxBindStatusCallback@@UAGKXZ 5f87d963 f
 0001:0007c973       ?Release@_AfxBindStatusCallback@@UAGKXZ 5f87d973 f
 0001:0007c983       ?QueryInterface@_AfxBindStatusCallback@@UAGJABU_GUID@@PAPAX@Z 5f87d983 f
 0001:0007c99a       ?GetBindInfo@_AfxBindStatusCallback@@EAGJPAKPAU_tagBINDINFO@@@Z 5f87d99a f
 0001:0007ca43       ?OnStartBinding@_AfxBindStatusCallback@@EAGJKPAUIBinding@@@Z 5f87da43 f
 0001:0007cada       ?GetPriority@_AfxBindStatusCallback@@EAGJPAJ@Z 5f87dada f
 0001:0007cb6a       ?OnProgress@_AfxBindStatusCallback@@EAGJKKKPBG@Z 5f87db6a f
 0001:0007cbfd       ?OnDataAvailable@_AfxBindStatusCallback@@EAGJKKPAUtagFORMATETC@@PAUtagSTGMEDIUM@@@Z 5f87dbfd f
 0001:0007cd06       ?OnLowResource@_AfxBindStatusCallback@@EAGJK@Z 5f87dd06 f
 0001:0007cd86       ?OnStopBinding@_AfxBindStatusCallback@@EAGJJPBG@Z 5f87dd86 f
 0001:0007ce29       ?OnObjectAvailable@_AfxBindStatusCallback@@EAGJABU_GUID@@PAUIUnknown@@@Z 5f87de29 f
 0001:0007ce31       ??_G_AfxBindStatusCallback@@QAEPAXI@Z 5f87de31 f
 0001:0007ce4d       ??1_AfxBindStatusCallback@@QAE@XZ 5f87de4d f
 0001:0007ce8b       ??0IBindStatusCallback@@QAE@XZ 5f87de8b f
 0001:0007ce9d       ?GetBindInfo@CAsyncMonikerFile@@MBEKXZ 5f87de9d f
 0001:0007cea1       ?GetPriority@CAsyncMonikerFile@@MBEJXZ 5f87dea1 f
 0001:0007cea4       ?OnLowResource@CAsyncMonikerFile@@MAEXXZ 5f87dea4 f
 0001:0007cea5       ?OnStopBinding@CAsyncMonikerFile@@MAEXJPBG@Z 5f87dea5 f
 0001:0007cea8       ?OnProgress@CAsyncMonikerFile@@MAEXKKKPBG@Z 5f87dea8 f
 0001:0007ceab       ??0COleFrameHook@@QAE@PAVCFrameWnd@@PAVCOleClientItem@@@Z 5f87deab f
 0001:0007cf19       ??_ECOleFrameHook@@UAEPAXI@Z 5f87df19 f
 0001:0007cf19       ??_GCOleFrameHook@@UAEPAXI@Z 5f87df19 f
 0001:0007cf35       ??1COleFrameHook@@UAE@XZ   5f87df35 f
 0001:0007cf80       ?OnRecalcLayout@COleFrameHook@@UAEXXZ 5f87df80 f
 0001:0007cfc2       ?OnDocActivate@COleFrameHook@@UAEHH@Z 5f87dfc2 f
 0001:0007d03e       ?OnContextHelp@COleFrameHook@@UAEHH@Z 5f87e03e f
 0001:0007d062       ?OnMenuSelect@COleFrameHook@@UAEHIIPAUHMENU__@@@Z 5f87e062 f
 0001:0007d0e1       ?OnInitMenu@COleFrameHook@@UAEXPAVCMenu@@@Z 5f87e0e1 f
 0001:0007d0fe       ?OnInitMenuPopup@COleFrameHook@@UAEHPAVCMenu@@HH@Z 5f87e0fe f
 0001:0007d151       ?OnPreTranslateMessage@COleFrameHook@@UAEHPAUtagMSG@@@Z 5f87e151 f
 0001:0007d1d7       ?OnActivate@COleFrameHook@@UAEXH@Z 5f87e1d7 f
 0001:0007d205       ?OnEnableModeless@COleFrameHook@@UAEXH@Z 5f87e205 f
 0001:0007d224       ?OnUpdateFrameTitle@COleFrameHook@@UAEHXZ 5f87e224 f
 0001:0007d23f       ?OnPaletteChanged@COleFrameHook@@UAEXPAVCWnd@@@Z 5f87e23f f
 0001:0007d26a       ?OnQueryNewPalette@COleFrameHook@@UAEHXZ 5f87e26a f
 0001:0007d28c       ?NotifyAllInPlace@COleFrameHook@@QAEHHP81@AEHH@Z@Z 5f87e28c f
 0001:0007d375       ?DoContextSensitiveHelp@COleFrameHook@@QAEHH@Z 5f87e375 f
 0001:0007d38e       ?DoEnableModeless@COleFrameHook@@QAEHH@Z 5f87e38e f
 0001:0007d3c8       ?CanActivate@COleClientItem@@MAEHXZ 5f87e3c8 f
 0001:0007d46f       ?OnActivate@COleClientItem@@UAEXXZ 5f87e46f f
 0001:0007d4a3       ?OnActivateUI@COleClientItem@@UAEXXZ 5f87e4a3 f
 0001:0007d524       ?OnShowControlBars@COleClientItem@@UAEHPAVCFrameWnd@@H@Z 5f87e524 f
 0001:0007d5af       ?OnGetWindowContext@COleClientItem@@MAEHPAPAVCFrameWnd@@0PAUtagOIFI@@@Z 5f87e5af f
 0001:0007d62b       ?OnScrollBy@COleClientItem@@MAEHVCSize@@@Z 5f87e62b f
 0001:0007d66e       ?OnDeactivateUI@COleClientItem@@UAEXH@Z 5f87e66e f
 0001:0007d7c8       ?OnDeactivate@COleClientItem@@UAEXXZ 5f87e7c8 f
 0001:0007d821       ?OnDiscardUndoState@COleClientItem@@MAEXXZ 5f87e821 f
 0001:0007d822       ?DeactivateUI@COleClientItem@@QAEXXZ 5f87e822 f
 0001:0007d822       ?OnDeactivateAndUndo@COleClientItem@@MAEXXZ 5f87e822 f
 0001:0007d85e       ?OnChangeItemPosition@COleClientItem@@MAEHABVCRect@@@Z 5f87e85e f
 0001:0007d8b8       ?OnInsertMenus@COleClientItem@@UAEXPAVCMenu@@PAUtagOleMenuGroupWidths@@@Z 5f87e8b8 f
 0001:0007d8f1       ?OnSetMenu@COleClientItem@@UAEXPAVCMenu@@PAXPAUHWND__@@@Z 5f87e8f1 f
 0001:0007d962       ?OnRemoveMenus@COleClientItem@@UAEXPAVCMenu@@@Z 5f87e962 f
 0001:0007d986       ?OnUpdateFrameTitle@COleClientItem@@UAEHXZ 5f87e986 f
 0001:0007d989       ?Deactivate@COleClientItem@@QAEXXZ 5f87e989 f
 0001:0007d9e0       ?SetItemRects@COleClientItem@@QAEHPBUtagRECT@@0@Z 5f87e9e0 f
 0001:0007da4b       ?ReactivateAndUndo@COleClientItem@@QAEHXZ 5f87ea4b f
 0001:0007da8a       ?GetInPlaceWindow@COleClientItem@@QAEPAVCWnd@@XZ 5f87ea8a f
 0001:0007dabb       ?_GetBaseInterfaceMap@COleFrameHook@@KGPBUAFX_INTERFACEMAP@@XZ 5f87eabb f
 0001:0007dac1       ?GetInterfaceMap@COleFrameHook@@MBEPBUAFX_INTERFACEMAP@@XZ 5f87eac1 f
 0001:0007dac7       ?GetInterfaceHook@COleFrameHook@@UAEPAUIUnknown@@PBX@Z 5f87eac7 f
 0001:0007dafb       ?AddRef@XOleCommandTarget@COleFrameHook@@UAGKXZ 5f87eafb f
 0001:0007db0a       ?Release@XOleCommandTarget@COleFrameHook@@UAGKXZ 5f87eb0a f
 0001:0007db19       ?QueryInterface@XOleCommandTarget@COleFrameHook@@UAGJABU_GUID@@PAPAX@Z 5f87eb19 f
 0001:0007db30       ?Exec@XOleCommandTarget@COleFrameHook@@UAGJPBU_GUID@@KKPAUtagVARIANT@@1@Z 5f87eb30 f
 0001:0007db6d       ?QueryStatus@XOleCommandTarget@COleFrameHook@@UAGJPBU_GUID@@KQAU_tagOLECMD@@PAU_tagOLECMDTEXT@@@Z 5f87eb6d f
 0001:0007dba7       ?AddRef@XOleInPlaceFrame@COleFrameHook@@UAGKXZ 5f87eba7 f
 0001:0007dbb6       ?Release@XOleInPlaceFrame@COleFrameHook@@UAGKXZ 5f87ebb6 f
 0001:0007dbc5       ?QueryInterface@XOleInPlaceFrame@COleFrameHook@@UAGJABU_GUID@@PAPAX@Z 5f87ebc5 f
 0001:0007dbdc       ?GetWindow@XOleInPlaceFrame@COleFrameHook@@UAGJPAPAUHWND__@@@Z 5f87ebdc f
 0001:0007dbfa       ?ContextSensitiveHelp@XOleInPlaceFrame@COleFrameHook@@UAGJH@Z 5f87ebfa f
 0001:0007dc92       ?GetBorder@XOleInPlaceFrame@COleFrameHook@@UAGJPAUtagRECT@@@Z 5f87ec92 f
 0001:0007dd32       ?RequestBorderSpace@XOleInPlaceFrame@COleFrameHook@@UAGJPBUtagRECT@@@Z 5f87ed32 f
 0001:0007dd86       ?SetBorderSpace@XOleInPlaceFrame@COleFrameHook@@UAGJPBUtagRECT@@@Z 5f87ed86 f
 0001:0007de05       ?SetActiveObject@XOleInPlaceFrame@COleFrameHook@@UAGJPAUIOleInPlaceActiveObject@@PBG@Z 5f87ee05 f
 0001:0007dea5       ?InsertMenus@XOleInPlaceFrame@COleFrameHook@@UAGJPAUHMENU__@@PAUtagOleMenuGroupWidths@@@Z 5f87eea5 f
 0001:0007df1d       ?SetMenu@XOleInPlaceFrame@COleFrameHook@@UAGJPAUHMENU__@@PAXPAUHWND__@@@Z 5f87ef1d f
 0001:0007df98       ?RemoveMenus@XOleInPlaceFrame@COleFrameHook@@UAGJPAUHMENU__@@@Z 5f87ef98 f
 0001:0007e00d       ?SetStatusText@XOleInPlaceFrame@COleFrameHook@@UAGJPBG@Z 5f87f00d f
 0001:0007e02d       ?EnableModeless@XOleInPlaceFrame@COleFrameHook@@UAGJH@Z 5f87f02d f
 0001:0007e0a4       ?TranslateAcceleratorW@XOleInPlaceFrame@COleFrameHook@@UAGJPAUtagMSG@@G@Z 5f87f0a4 f
 0001:0007e142       ?AddRef@XOleIPSite@COleClientItem@@UAGKXZ 5f87f142 f
 0001:0007e151       ?Release@XOleIPSite@COleClientItem@@UAGKXZ 5f87f151 f
 0001:0007e160       ?QueryInterface@XOleIPSite@COleClientItem@@UAGJABU_GUID@@PAPAX@Z 5f87f160 f
 0001:0007e177       ?GetWindow@XOleIPSite@COleClientItem@@UAGJPAPAUHWND__@@@Z 5f87f177 f
 0001:0007e19c       ?ContextSensitiveHelp@XOleIPSite@COleClientItem@@UAGJH@Z 5f87f19c f
 0001:0007e1bf       ?CanInPlaceActivate@XOleIPSite@COleClientItem@@UAGJXZ 5f87f1bf f
 0001:0007e208       ?OnInPlaceActivate@XOleIPSite@COleClientItem@@UAGJXZ 5f87f208 f
 0001:0007e274       ?OnUIActivate@XOleIPSite@COleClientItem@@UAGJXZ 5f87f274 f
 0001:0007e2e0       ?GetWindowContext@XOleIPSite@COleClientItem@@UAGJPAPAUIOleInPlaceFrame@@PAPAUIOleInPlaceUIWindow@@PAUtagRECT@@2PAUtagOIFI@@@Z 5f87f2e0 f
 0001:0007e45b       ?Scroll@XOleIPSite@COleClientItem@@UAGJUtagSIZE@@@Z 5f87f45b f
 0001:0007e4d0       ?OnUIDeactivate@XOleIPSite@COleClientItem@@UAGJH@Z 5f87f4d0 f
 0001:0007e53f       ?OnInPlaceDeactivate@XOleIPSite@COleClientItem@@UAGJXZ 5f87f53f f
 0001:0007e5ab       ?DiscardUndoState@XOleIPSite@COleClientItem@@UAGJXZ 5f87f5ab f
 0001:0007e617       ?DeactivateAndUndo@XOleIPSite@COleClientItem@@UAGJXZ 5f87f617 f
 0001:0007e683       ?OnPosRectChange@XOleIPSite@COleClientItem@@UAGJPBUtagRECT@@@Z 5f87f683 f
 0001:0007e700       ?_AfxOlePropertiesEnabled@@YGHXZ 5f87f700 f
 0001:0007e748       ?_AfxParseDisplayName@@YAJPAUIMoniker@@PAUIBindCtx@@PAGPAKPAPAU1@@Z 5f87f748 f
 0001:0007e7fc       ??0COleUILinkInfo@@QAE@PAVCOleDocument@@@Z 5f87f7fc f
 0001:0007e81c       ?Release@COleUILinkInfo@@UAGKXZ 5f87f81c f
 0001:0007e821       ?GetNextLink@COleUILinkInfo@@UAGKK@Z 5f87f821 f
 0001:0007e86e       ?SetLinkUpdateOptions@COleUILinkInfo@@UAGJKK@Z 5f87f86e f
 0001:0007e8c0       ?GetLinkUpdateOptions@COleUILinkInfo@@UAGJKPAK@Z 5f87f8c0 f
 0001:0007e925       ?SetLinkSource@COleUILinkInfo@@UAGJKPAGKPAKH@Z 5f87f925 f
 0001:0007eaea       ?GetLinkSource@COleUILinkInfo@@UAGJKPAPAGPAK00PAH2@Z 5f87faea f
 0001:0007ec32       ?OpenLinkSource@COleUILinkInfo@@UAGJK@Z 5f87fc32 f
 0001:0007ec85       ?UpdateLink@COleUILinkInfo@@UAGJKHH@Z 5f87fc85 f
 0001:0007ecf7       ?CancelLink@COleUILinkInfo@@UAGJK@Z 5f87fcf7 f
 0001:0007ed6d       ?GetLastUpdate@COleUILinkInfo@@UAGJKPAU_FILETIME@@@Z 5f87fd6d f
 0001:0007ed72       ??0COleInsertDialog@@QAE@KPAVCWnd@@@Z 5f87fd72 f
 0001:0007ee13       ??_GCOleInsertDialog@@UAEPAXI@Z 5f87fe13 f
 0001:0007ee13       ??_ECOleInsertDialog@@UAEPAXI@Z 5f87fe13 f
 0001:0007ee2f       ??1COleDialog@@UAE@XZ      5f87fe2f f
 0001:0007ee34       ?AddClassIDToList@COleInsertDialog@@IAEXAAPAU_GUID@@AAH1PAU2@@Z 5f87fe34 f
 0001:0007eeaa       ?DoModal@COleInsertDialog@@QAEHK@Z 5f87feaa f
 0001:0007f13d       ?DoModal@COleInsertDialog@@UAEHXZ 5f88013d f
 0001:0007f168       ?GetSelectionType@COleInsertDialog@@QBEIXZ 5f880168 f
 0001:0007f17c       ?CreateItem@COleInsertDialog@@QAEHPAVCOleClientItem@@@Z 5f88017c f
 0001:0007f208       ??0COleConvertDialog@@QAE@PAVCOleClientItem@@KPAU_GUID@@PAVCWnd@@@Z 5f880208 f
 0001:0007f37c       ??_GCOleConvertDialog@@UAEPAXI@Z 5f88037c f
 0001:0007f37c       ??_ECOleConvertDialog@@UAEPAXI@Z 5f88037c f
 0001:0007f398       ?DoModal@COleConvertDialog@@UAEHXZ 5f880398 f
 0001:0007f3c3       ?DoConvert@COleConvertDialog@@QAEHPAVCOleClientItem@@@Z 5f8803c3 f
 0001:0007f4cd       ?GetSelectionType@COleConvertDialog@@QBEIXZ 5f8804cd f
 0001:0007f504       ??0COleChangeIconDialog@@QAE@PAVCOleClientItem@@KPAVCWnd@@@Z 5f880504 f
 0001:0007f5a0       ??_GCOleChangeIconDialog@@UAEPAXI@Z 5f8805a0 f
 0001:0007f5a0       ??_ECOleChangeIconDialog@@UAEPAXI@Z 5f8805a0 f
 0001:0007f5bc       ?DoModal@COleChangeIconDialog@@UAEHXZ 5f8805bc f
 0001:0007f5e7       ?DoChangeIcon@COleChangeIconDialog@@QAEHPAVCOleClientItem@@@Z 5f8805e7 f
 0001:0007f615       ??0COleLinksDialog@@QAE@PAVCOleDocument@@PAVCView@@KPAVCWnd@@@Z 5f880615 f
 0001:0007f6c7       ??_GCOleLinksDialog@@UAEPAXI@Z 5f8806c7 f
 0001:0007f6c7       ??_ECOleLinksDialog@@UAEPAXI@Z 5f8806c7 f
 0001:0007f6e3       ?DoModal@COleLinksDialog@@UAEHXZ 5f8806e3 f
 0001:0007f718       ??0COleUpdateDialog@@QAE@PAVCOleDocument@@HHPAVCWnd@@@Z 5f880718 f
 0001:0007f783       ??_GCOleUpdateDialog@@UAEPAXI@Z 5f880783 f
 0001:0007f783       ??_ECOleUpdateDialog@@UAEPAXI@Z 5f880783 f
 0001:0007f79f       ??1COleUpdateDialog@@UAE@XZ 5f88079f f
 0001:0007f7dd       ?DoModal@COleUpdateDialog@@UAEHXZ 5f8807dd f
 0001:0007f840       ??0COlePasteSpecialDialog@@QAE@KPAVCOleDataObject@@PAVCWnd@@@Z 5f880840 f
 0001:0007f91c       ??_GCOlePasteSpecialDialog@@UAEPAXI@Z 5f88091c f
 0001:0007f91c       ??_ECOlePasteSpecialDialog@@UAEPAXI@Z 5f88091c f
 0001:0007f938       ?DoModal@COlePasteSpecialDialog@@UAEHXZ 5f880938 f
 0001:0007f973       ?GetSelectionType@COlePasteSpecialDialog@@QBEIXZ 5f880973 f
 0001:0007f9c1       ?AddLinkEntry@COlePasteSpecialDialog@@QAE?AW4tagOLEUIPASTEFLAG@@I@Z 5f8809c1 f
 0001:0007fa14       ?AddFormat@COlePasteSpecialDialog@@QAEXIKIHH@Z 5f880a14 f
 0001:0007fb00       ?AddFormat@COlePasteSpecialDialog@@QAEXABUtagFORMATETC@@PAG1K@Z 5f880b00 f
 0001:0007fb73       ?AddStandardFormats@COlePasteSpecialDialog@@QAEXH@Z 5f880b73 f
 0001:0007fbe7       ?CreateItem@COlePasteSpecialDialog@@QAEHPAVCOleClientItem@@@Z 5f880be7 f
 0001:0007fcba       ?AfxOleHookProc@@YGIPAUHWND__@@IIJ@Z 5f880cba f
 0001:0007fd05       ??0COleDialog@@QAE@PAVCWnd@@@Z 5f880d05 f
 0001:0007fd23       ?MapResult@COleDialog@@QAEHI@Z 5f880d23 f
 0001:0007fd41       ??0COleBusyDialog@@QAE@PAUHTASK__@@HKPAVCWnd@@@Z 5f880d41 f
 0001:0007fd95       ??_GCOleBusyDialog@@UAEPAXI@Z 5f880d95 f
 0001:0007fd95       ??_ECOleBusyDialog@@UAEPAXI@Z 5f880d95 f
 0001:0007fdb1       ?DoModal@COleBusyDialog@@UAEHXZ 5f880db1 f
 0001:0007fe41       ??0COlePropertiesDialog@@QAE@PAVCOleClientItem@@IIPAVCWnd@@@Z 5f880e41 f
 0001:0007ff9b       ??_ECOlePropertiesDialog@@UAEPAXI@Z 5f880f9b f
 0001:0007ff9b       ??_GCOlePropertiesDialog@@UAEPAXI@Z 5f880f9b f
 0001:0007ffb7       ?DoModal@COlePropertiesDialog@@UAEHXZ 5f880fb7 f
 0001:00080003       ?OnInitDialog@COlePropertiesDialog@@UAEHXZ 5f881003 f
 0001:0008002a       ?QueryInterface@XOleUIObjInfo@COlePropertiesDialog@@UAGJABU_GUID@@PAPAX@Z 5f88102a f
 0001:00080032       ?GetObjectInfo@XOleUIObjInfo@COlePropertiesDialog@@UAGJKPAKPAPAG111@Z 5f881032 f
 0001:00080210       ?GetConvertInfo@XOleUIObjInfo@COlePropertiesDialog@@UAGJKPAU_GUID@@PAG0PAPAU3@PAI@Z 5f881210 f
 0001:0008026b       ?ConvertObject@XOleUIObjInfo@COlePropertiesDialog@@UAGJKABU_GUID@@@Z 5f88126b f
 0001:00080296       ?GetViewInfo@XOleUIObjInfo@COlePropertiesDialog@@UAGJKPAPAXPAKPAH@Z 5f881296 f
 0001:000802cf       ?SetViewInfo@XOleUIObjInfo@COlePropertiesDialog@@UAGJKPAXKHH@Z 5f8812cf f
 0001:00080362       ??0COleChangeSourceDialog@@QAE@PAVCOleClientItem@@PAVCWnd@@@Z 5f881362 f
 0001:000803ed       ??_GCOleChangeSourceDialog@@UAEPAXI@Z 5f8813ed f
 0001:000803ed       ??_ECOleChangeSourceDialog@@UAEPAXI@Z 5f8813ed f
 0001:00080409       ?DoModal@COleChangeSourceDialog@@UAEHXZ 5f881409 f
 0001:00080434       ?PreInitDialog@COleChangeSourceDialog@@UAEXXZ 5f881434 f
 0001:0008044e       ??1COleChangeSourceDialog@@UAE@XZ 5f88144e f
 0001:00080480       ?ReportError@COleClientItem@@UBEHJ@Z 5f881480 f
 0001:000804ce       ?DoVerb@COleClientItem@@UAEHJPAVCView@@PAUtagMSG@@@Z 5f8814ce f
 0001:000805ca       ?GetPrimarySelectedItem@COleDocument@@UAEPAVCOleClientItem@@PAVCView@@@Z 5f8815ca f
 0001:00080660       ?AfxOleSetEditMenu@@YGXPAVCOleClientItem@@PAVCMenu@@IIII@Z 5f881660 f
 0001:000806f6       ?OnUpdatePasteMenu@COleDocument@@IAEXPAVCCmdUI@@@Z 5f8816f6 f
 0001:0008070d       ?OnUpdatePasteLinkMenu@COleDocument@@IAEXPAVCCmdUI@@@Z 5f88170d f
 0001:00080724       ?OnUpdateEditLinksMenu@COleDocument@@IAEXPAVCCmdUI@@@Z 5f881724 f
 0001:00080762       ?OnEditLinks@COleDocument@@IAEXXZ 5f881762 f
 0001:000807b6       ?OnEditConvert@COleDocument@@IAEXXZ 5f8817b6 f
 0001:0008082e       ?OnUpdateEditChangeIcon@COleDocument@@IAEXPAVCCmdUI@@@Z 5f88182e f
 0001:0008085c       ?OnEditChangeIcon@COleDocument@@IAEXXZ 5f88185c f
 0001:000808d3       ?OnUpdateObjectVerbMenu@COleDocument@@IAEXPAVCCmdUI@@@Z 5f8818d3 f
 0001:00080962       ?Attach@COleDataObject@@QAEXPAUIDataObject@@H@Z 5f881962 f
 0001:0008098f       ?Detach@COleDataObject@@QAEPAUIDataObject@@XZ 5f88198f f
 0001:000809a2       ?GetIDataObject@COleDataObject@@QAEPAUIDataObject@@H@Z 5f8819a2 f
 0001:000809c3       ?BeginEnumFormats@COleDataObject@@QAEXXZ 5f8819c3 f
 0001:000809e7       ?GetNextFormat@COleDataObject@@QAEHPAUtagFORMATETC@@@Z 5f8819e7 f
 0001:00080a15       ?GetFileData@COleDataObject@@QAEPAVCFile@@GPAUtagFORMATETC@@@Z 5f881a15 f
 0001:00080bde       ?GetGlobalData@COleDataObject@@QAEPAXGPAUtagFORMATETC@@@Z 5f881bde f
 0001:00080c7c       ?GetData@COleDataObject@@QAEHGPAUtagSTGMEDIUM@@PAUtagFORMATETC@@@Z 5f881c7c f
 0001:00080cde       ?EnsureClipboardObject@COleDataObject@@QAEXXZ 5f881cde f
 0001:00080d0d       ??0COleDataSource@@QAE@XZ  5f881d0d f
 0001:00080d38       ?Empty@COleDataSource@@QAEXXZ 5f881d38 f
 0001:00080d89       ?SetClipboard@COleDataSource@@QAEXXZ 5f881d89 f
 0001:00080deb       ?GetCacheEntry@COleDataSource@@IAEPAUAFX_DATACACHE_ENTRY@@PAUtagFORMATETC@@W4tagDATADIR@@@Z 5f881deb f
 0001:00080e8e       ?CacheGlobalData@COleDataSource@@QAEXGPAXPAUtagFORMATETC@@@Z 5f881e8e f
 0001:00080ec9       ?CacheData@COleDataSource@@QAEXGPAUtagSTGMEDIUM@@PAUtagFORMATETC@@@Z 5f881ec9 f
 0001:00080f00       ?DelayRenderFileData@COleDataSource@@QAEXGPAUtagFORMATETC@@@Z 5f881f00 f
 0001:00080f36       ?DelayRenderData@COleDataSource@@QAEXGPAUtagFORMATETC@@@Z 5f881f36 f
 0001:00080f85       ?DelaySetData@COleDataSource@@QAEXGPAUtagFORMATETC@@@Z 5f881f85 f
 0001:00080fb7       ?Lookup@COleDataSource@@IBEPAUAFX_DATACACHE_ENTRY@@PAUtagFORMATETC@@W4tagDATADIR@@@Z 5f881fb7 f
 0001:00081043       ?OnRenderFileData@COleDataSource@@UAEHPAUtagFORMATETC@@PAVCFile@@@Z 5f882043 f
 0001:00081048       ?OnRenderData@COleDataSource@@UAEHPAUtagFORMATETC@@PAUtagSTGMEDIUM@@@Z 5f882048 f
 0001:0008119c       ?OnSetData@COleDataSource@@UAEHPAUtagFORMATETC@@PAUtagSTGMEDIUM@@H@Z 5f88219c f
 0001:000811a1       ?GetInterfaceMap@CEnumFormatEtc@@MBEPBUAFX_INTERFACEMAP@@XZ 5f8821a1 f
 0001:000811a7       ??0CEnumFormatEtc@@QAE@XZ  5f8821a7 f
 0001:000811c5       ??_GCEnumFormatEtc@@UAEPAXI@Z 5f8821c5 f
 0001:000811c5       ??_ECEnumFormatEtc@@UAEPAXI@Z 5f8821c5 f
 0001:000811e1       ??1CEnumFormatEtc@@UAE@XZ  5f8821e1 f
 0001:0008121a       ?OnNext@CEnumFormatEtc@@MAEHPAX@Z 5f88221a f
 0001:00081249       ?AddFormat@CEnumFormatEtc@@QAEXPBUtagFORMATETC@@@Z 5f882249 f
 0001:000812bf       ?GetInterfaceMap@COleDataSource@@MBEPBUAFX_INTERFACEMAP@@XZ 5f8822bf f
 0001:000812c5       ?AddRef@XDataObject@COleDataSource@@UAGKXZ 5f8822c5 f
 0001:000812d4       ?Release@XDataObject@COleDataSource@@UAGKXZ 5f8822d4 f
 0001:000812e3       ?QueryInterface@XDataObject@COleDataSource@@UAGJABU_GUID@@PAPAX@Z 5f8822e3 f
 0001:000812fa       ?GetData@XDataObject@COleDataSource@@UAGJPAUtagFORMATETC@@PAUtagSTGMEDIUM@@@Z 5f8822fa f
 0001:000813bc       ?GetDataHere@XDataObject@COleDataSource@@UAGJPAUtagFORMATETC@@PAUtagSTGMEDIUM@@@Z 5f8823bc f
 0001:00081471       ?QueryGetData@XDataObject@COleDataSource@@UAGJPAUtagFORMATETC@@@Z 5f882471 f
 0001:00081494       ?GetCanonicalFormatEtc@XDataObject@COleDataSource@@UAGJPAUtagFORMATETC@@0@Z 5f882494 f
 0001:0008149c       ?SetData@XDataObject@COleDataSource@@UAGJPAUtagFORMATETC@@PAUtagSTGMEDIUM@@H@Z 5f88249c f
 0001:00081534       ?EnumFormatEtc@XDataObject@COleDataSource@@UAGJKPAPAUIEnumFORMATETC@@@Z 5f882534 f
 0001:000815db       ?DAdvise@XDataObject@COleDataSource@@UAGJPAUtagFORMATETC@@KPAUIAdviseSink@@PAK@Z 5f8825db f
 0001:000815ea       ?DUnadvise@XDataObject@COleDataSource@@UAGJK@Z 5f8825ea f
 0001:000815f2       ?EnumDAdvise@XDataObject@COleDataSource@@UAGJPAPAUIEnumSTATDATA@@@Z 5f8825f2 f
 0001:00081601       ??0CEnumArray@@QAE@IPBXIH@Z 5f882601 f
 0001:00081640       ??_GCEnumArray@@UAEPAXI@Z  5f882640 f
 0001:00081640       ??_ECEnumArray@@UAEPAXI@Z  5f882640 f
 0001:0008165c       ?OnNext@CEnumArray@@MAEHPAX@Z 5f88265c f
 0001:0008168c       ?OnSkip@CEnumArray@@MAEHXZ 5f88268c f
 0001:000816a4       ?OnReset@CEnumArray@@MAEXXZ 5f8826a4 f
 0001:000816a9       ?OnClone@CEnumArray@@MAEPAV1@XZ 5f8826a9 f
 0001:000816ef       ?AddRef@XEnumVOID@CEnumArray@@UAGKXZ 5f8826ef f
 0001:000816fe       ?Release@XEnumVOID@CEnumArray@@UAGKXZ 5f8826fe f
 0001:0008170d       ?QueryInterface@XEnumVOID@CEnumArray@@UAGJABU_GUID@@PAPAX@Z 5f88270d f
 0001:00081724       ?Next@XEnumVOID@CEnumArray@@UAGJKPAXPAK@Z 5f882724 f
 0001:000817c6       ?Skip@XEnumVOID@CEnumArray@@UAGJK@Z 5f8827c6 f
 0001:0008183e       ?Reset@XEnumVOID@CEnumArray@@UAGJXZ 5f88283e f
 0001:00081881       ?Clone@XEnumVOID@CEnumArray@@UAGJPAPAUIEnumVOID@@@Z 5f882881 f
 0001:0008193b       ?VerifyLicenseKey@COleObjectFactory@@MAEHPAG@Z 5f88293b f
 0001:00081998       ?LockServer@XClassFactory@COleObjectFactory@@UAGJH@Z 5f882998 f
 0001:00081a08       ?GetLicInfo@XClassFactory@COleObjectFactory@@UAGJPAUtagLICINFO@@@Z 5f882a08 f
 0001:00081a76       ?RequestLicKey@XClassFactory@COleObjectFactory@@UAGJKPAPAG@Z 5f882a76 f
 0001:00081b4e       ??0COleCntrFrameWnd@@QAE@PAVCOleIPFrameWnd@@@Z 5f882b4e f
 0001:00081b8f       ??_ECOleCntrFrameWnd@@UAEPAXI@Z 5f882b8f f
 0001:00081b8f       ??_GCOleCntrFrameWnd@@UAEPAXI@Z 5f882b8f f
 0001:00081bab       ??1COleCntrFrameWnd@@UAE@XZ 5f882bab f
 0001:00081bea       ?RecalcLayout@COleCntrFrameWnd@@UAEXH@Z 5f882bea f
 0001:00081c7a       ?OnCmdMsg@COleCntrFrameWnd@@UAEHIHPAXPAUAFX_CMDHANDLERINFO@@@Z 5f882c7a f
 0001:00081cd6       ?PostNcDestroy@COleCntrFrameWnd@@MAEXXZ 5f882cd6 f
 0001:00081cd7       ?_GetBaseMessageMap@COleIPFrameWnd@@KGPBUAFX_MSGMAP@@XZ 5f882cd7 f
 0001:00081cdd       ?GetMessageMap@COleIPFrameWnd@@MBEPBUAFX_MSGMAP@@XZ 5f882cdd f
 0001:00081ce3       ??0COleIPFrameWnd@@QAE@XZ  5f882ce3 f
 0001:00081d5b       ?OnCreate@COleIPFrameWnd@@IAEHPAUtagCREATESTRUCTW@@@Z 5f882d5b f
 0001:00081da2       ?OnDestroy@COleIPFrameWnd@@IAEXXZ 5f882da2 f
 0001:00081ded       ?OnCreateControlBars@COleIPFrameWnd@@UAEHPAVCWnd@@0@Z 5f882ded f
 0001:00081df3       ?OnCreateControlBars@COleIPFrameWnd@@UAEHPAVCFrameWnd@@0@Z 5f882df3 f
 0001:00081e06       ?OnIdleUpdateCmdUI@COleIPFrameWnd@@IAEXXZ 5f882e06 f
 0001:00081e23       ?OnIdleUpdateCmdUI@COleCntrFrameWnd@@QAEXXZ 5f882e23 f
 0001:00081e63       ?OnWindowPosChanging@COleIPFrameWnd@@IAEXPAUtagWINDOWPOS@@@Z 5f882e63 f
 0001:00081ea3       ?OnSetMessageString@COleIPFrameWnd@@UAEJIJ@Z 5f882ea3 f
 0001:00081f2c       ?LoadFrame@COleIPFrameWnd@@UAEHIKPAVCWnd@@PAUCCreateContext@@@Z 5f882f2c f
 0001:00081f7c       ?OnSize@COleIPFrameWnd@@IAEXIHH@Z 5f882f7c f
 0001:00081f7f       ?OnResizeChild@COleIPFrameWnd@@IAEJIJ@Z 5f882f7f f
 0001:0008203b       ?OnRequestPositionChange@COleIPFrameWnd@@MAEXPBUtagRECT@@@Z 5f88303b f
 0001:0008205a       ?OnRecalcParent@COleIPFrameWnd@@IAEJIJ@Z 5f88305a f
 0001:00082086       ?RecalcLayout@COleIPFrameWnd@@UAEXH@Z 5f883086 f
 0001:000821e4       ?RepositionFrame@COleIPFrameWnd@@UAEXPBUtagRECT@@0@Z 5f8831e4 f
 0001:00082233       ?PreTranslateMessage@COleIPFrameWnd@@UAEHPAUtagMSG@@@Z 5f883233 f
 0001:000822b8       ?OnUpdateControlBarMenu@COleIPFrameWnd@@IAEXPAVCCmdUI@@@Z 5f8832b8 f
 0001:00082322       ?OnBarCheck@COleIPFrameWnd@@IAEHI@Z 5f883322 f
 0001:00082381       ?OnContextHelp@COleIPFrameWnd@@IAEXXZ 5f883381 f
 0001:0008241b       ?GetInPlaceMenu@COleIPFrameWnd@@MAEPAUHMENU__@@XZ 5f88341b f
 0001:0008242a       ?BuildSharedMenu@COleIPFrameWnd@@MAEHXZ 5f88342a f
 0001:000824c4       ?DestroySharedMenu@COleIPFrameWnd@@MAEXXZ 5f8834c4 f
 0001:0008252b       ??_ECOleLinkingDoc@@UAEPAXI@Z 5f88352b f
 0001:0008252b       ??_GCOleLinkingDoc@@UAEPAXI@Z 5f88352b f
 0001:00082547       ?GetMoniker@COleLinkingDoc@@UAEPAUIMoniker@@W4tagOLEGETMONIKER@@@Z 5f883547 f
 0001:000825de       ?OnSaveDocument@COleLinkingDoc@@UAEHPBG@Z 5f8835de f
 0001:00082651       ?SaveToStorage@COleLinkingDoc@@MAEXPAVCObject@@@Z 5f883651 f
 0001:0008269e       ?GetContainer@COleLinkingDoc@@UAEPAUIOleItemContainer@@XZ 5f88369e f
 0001:000826b5       ?OnGetLinkedItem@COleLinkingDoc@@MAEPAVCOleServerItem@@PBG@Z 5f8836b5 f
 0001:000826ba       ?OnFindEmbeddedItem@COleLinkingDoc@@MAEPAVCOleClientItem@@PBG@Z 5f8836ba f
 0001:00082708       ?ReportSaveLoadException@COleLinkingDoc@@UAEXPBGPAVCException@@HI@Z 5f883708 f
 0001:00082737       ?EndDeferErrors@COleLinkingDoc@@QAEJJ@Z 5f883737 f
 0001:0008277e       ?AddRef@XPersistFile@COleLinkingDoc@@UAGKXZ 5f88377e f
 0001:00082790       ?GetClassID@XPersistFile@COleLinkingDoc@@UAGJPAU_GUID@@@Z 5f883790 f
 0001:000827c3       ?IsDirty@XPersistFile@COleLinkingDoc@@UAGJXZ 5f8837c3 f
 0001:0008280f       ?Load@XPersistFile@COleLinkingDoc@@UAGJPBGK@Z 5f88380f f
 0001:000828ed       ?Save@XPersistFile@COleLinkingDoc@@UAGJPBGH@Z 5f8838ed f
 0001:0008299c       ?SaveCompleted@XPersistFile@COleLinkingDoc@@UAGJPBG@Z 5f88399c f
 0001:00082a01       ?GetCurFile@XPersistFile@COleLinkingDoc@@UAGJPAPAG@Z 5f883a01 f
 0001:00082a39       ?AddRef@XOleItemContainer@COleLinkingDoc@@UAGKXZ 5f883a39 f
 0001:00082a4b       ?Release@XOleItemContainer@COleLinkingDoc@@UAGKXZ 5f883a4b f
 0001:00082a5d       ?QueryInterface@XOleItemContainer@COleLinkingDoc@@UAGJABU_GUID@@PAPAX@Z 5f883a5d f
 0001:00082a77       ?EnumObjects@XOleItemContainer@COleLinkingDoc@@UAGJKPAPAUIEnumUnknown@@@Z 5f883a77 f
 0001:00082a86       ?ParseDisplayName@XOleItemContainer@COleLinkingDoc@@UAGJPAUIBindCtx@@PAGPAKPAPAUIMoniker@@@Z 5f883a86 f
 0001:00082b57       ?LockContainer@XOleItemContainer@COleLinkingDoc@@UAGJH@Z 5f883b57 f
 0001:00082b71       ?GetObjectW@XOleItemContainer@COleLinkingDoc@@UAGJPAGKPAUIBindCtx@@ABU_GUID@@PAPAX@Z 5f883b71 f
 0001:00082c61       ?GetObjectStorage@XOleItemContainer@COleLinkingDoc@@UAGJPAGPAUIBindCtx@@ABU_GUID@@PAPAX@Z 5f883c61 f
 0001:00082cf2       ?IsRunning@XOleItemContainer@COleLinkingDoc@@UAGJPAG@Z 5f883cf2 f
 0001:00082d8f       ??1COleTemplateServer@@UAE@XZ 5f883d8f f
 0001:00082d94       ?OnCmdMsg@COleTemplateServer@@MAEHIHPAXPAUAFX_CMDHANDLERINFO@@@Z 5f883d94 f
 0001:00082db9       ?Unregister@COleTemplateServer@@QAEHXZ 5f883db9 f
 0001:00082eed       ?OnCreateObject@COleTemplateServer@@MAEPAVCCmdTarget@@XZ 5f883eed f
 0001:00082f21       ?AfxDllGetClassObject@@YGJABU_GUID@@0PAPAX@Z 5f883f21 f
 0001:00082fdf       ?AfxDllCanUnloadNow@@YGJXZ 5f883fdf f
 0001:0008304e       ??0COleDropSource@@QAE@XZ  5f88404e f
 0001:000830de       ??1COleDropSource@@UAE@XZ  5f8840de f
 0001:000830e3       ?QueryContinueDrag@COleDropSource@@UAEJHK@Z 5f8840e3 f
 0001:00083116       ?GiveFeedback@COleDropSource@@UAEJK@Z 5f884116 f
 0001:00083125       ?OnBeginDrag@COleDropSource@@UAEHPAVCWnd@@@Z 5f884125 f
 0001:0008325b       ?GetInterfaceMap@COleDropSource@@MBEPBUAFX_INTERFACEMAP@@XZ 5f88425b f
 0001:00083261       ?AddRef@XDropSource@COleDropSource@@UAGKXZ 5f884261 f
 0001:00083270       ?Release@XDropSource@COleDropSource@@UAGKXZ 5f884270 f
 0001:0008327f       ?QueryInterface@XDropSource@COleDropSource@@UAGJABU_GUID@@PAPAX@Z 5f88427f f
 0001:00083296       ?QueryContinueDrag@XDropSource@COleDropSource@@UAGJHK@Z 5f884296 f
 0001:000832ae       ?GiveFeedback@XDropSource@COleDropSource@@UAGJK@Z 5f8842ae f
 0001:000832f2       ?DoDragDrop@COleDataSource@@QAEKKPBUtagRECT@@PAVCOleDropSource@@@Z 5f8842f2 f
 0001:00083407       ?OnDragScroll@COleDropTarget@@UAEKPAVCWnd@@KVCPoint@@@Z 5f884407 f
 0001:00083649       ?OnDragEnter@COleDropTarget@@UAEKPAVCWnd@@PAVCOleDataObject@@KVCPoint@@@Z 5f884649 f
 0001:0008367b       ?OnDragOver@COleDropTarget@@UAEKPAVCWnd@@PAVCOleDataObject@@KVCPoint@@@Z 5f88467b f
 0001:000836ad       ?OnDrop@COleDropTarget@@UAEHPAVCWnd@@PAVCOleDataObject@@KVCPoint@@@Z 5f8846ad f
 0001:000836df       ?OnDropEx@COleDropTarget@@UAEKPAVCWnd@@PAVCOleDataObject@@KKVCPoint@@@Z 5f8846df f
 0001:00083719       ?OnDragLeave@COleDropTarget@@UAEXPAVCWnd@@@Z 5f884719 f
 0001:0008373c       ?_AfxFilterDropEffect@@YGKKK@Z 5f88473c f
 0001:00083770       ?DragEnter@XDropTarget@COleDropTarget@@UAGJPAUIDataObject@@KU_POINTL@@PAK@Z 5f884770 f
 0001:0008386e       ?DragOver@XDropTarget@COleDropTarget@@UAGJKU_POINTL@@PAK@Z 5f88486e f
 0001:00083957       ?DragLeave@XDropTarget@COleDropTarget@@UAGJXZ 5f884957 f
 0001:000839df       ?Drop@XDropTarget@COleDropTarget@@UAGJPAUIDataObject@@KU_POINTL@@PAK@Z 5f8849df f
 0001:00083b09       ?BeginBusyState@COleMessageFilter@@UAEXXZ 5f884b09 f
 0001:00083b0d       ?EndBusyState@COleMessageFilter@@UAEXXZ 5f884b0d f
 0001:00083b19       ?IsSignificantMessage@COleMessageFilter@@UAEHPAUtagMSG@@@Z 5f884b19 f
 0001:00083b6f       ?OnBusyDialog@COleMessageFilter@@UAEHPAUHTASK__@@@Z 5f884b6f f
 0001:00083bea       ?OnNotRespondingDialog@COleMessageFilter@@UAEHPAUHTASK__@@@Z 5f884bea f
 0001:00083c66       ?GetInterfaceMap@COleMessageFilter@@MBEPBUAFX_INTERFACEMAP@@XZ 5f884c66 f
 0001:00083c6c       ?QueryInterface@XMessageFilter@COleMessageFilter@@UAGJABU_GUID@@PAPAX@Z 5f884c6c f
 0001:00083cad       ?RetryRejectedCall@XMessageFilter@COleMessageFilter@@UAGKPAUHTASK__@@KK@Z 5f884cad f
 0001:00083db4       ??_ECOleServerDoc@@UAEPAXI@Z 5f884db4 f
 0001:00083db4       ??_GCOleServerDoc@@UAEPAXI@Z 5f884db4 f
 0001:00083e34       ?GetEmbeddedItem@COleServerDoc@@QAEPAVCOleServerItem@@XZ 5f884e34 f
 0001:00083e59       ?GetDocObjectServer@COleServerDoc@@MAEPAVCDocObjectServer@@PAUIOleDocumentSite@@@Z 5f884e59 f
 0001:00083e5e       ?OnExecOleCmd@COleServerDoc@@MAEJPBU_GUID@@KKPAUtagVARIANT@@1@Z 5f884e5e f
 0001:00083eab       ?NotifyRename@COleServerDoc@@QAEXPBG@Z 5f884eab f
 0001:00083f4b       ?OnUpdate@COleServerItem@@UAEXPAV1@JPAVCObject@@W4tagDVASPECT@@@Z 5f884f4b f
 0001:00083f59       ?GetZoomFactor@COleServerDoc@@QBEHPAUtagSIZE@@0PBUtagRECT@@@Z 5f884f59 f
 0001:0008403e       ?GetItemPosition@COleServerDoc@@QBEXPAUtagRECT@@@Z 5f88503e f
 0001:00084059       ?GetItemClipRect@COleServerDoc@@QBEXPAUtagRECT@@@Z 5f885059 f
 0001:00084074       ?OnGetLinkedItem@COleServerDoc@@UAEPAVCOleServerItem@@PBG@Z 5f885074 f
 0001:000840b5       ?OnClose@COleServerDoc@@MAEXW4tagOLECLOSE@@@Z 5f8850b5 f
 0001:00084176       ?SaveModifiedPrompt@COleServerDoc@@IAEHXZ 5f885176 f
 0001:00084214       ?GetFileTypeString@COleServerDoc@@MAEHAAVCString@@@Z 5f885214 f
 0001:0008423c       ?OnSetHostNames@COleServerDoc@@MAEXPBG0@Z 5f88523c f
 0001:000842e7       ?SaveEmbedding@COleServerDoc@@QAEXXZ 5f8852e7 f
 0001:00084315       ?OnUpdateDocument@COleServerDoc@@UAEHXZ 5f885315 f
 0001:0008436f       ?GetMoniker@COleServerDoc@@UAEPAUIMoniker@@W4tagOLEGETMONIKER@@@Z 5f88536f f
 0001:000843d1       ?GetMessageMap@COleServerDoc@@MBEPBUAFX_MSGMAP@@XZ 5f8853d1 f
 0001:000843d7       ?OnFileUpdate@COleServerDoc@@IAEXXZ 5f8853d7 f
 0001:000843ee       ?OnFileSaveCopyAs@COleServerDoc@@IAEXXZ 5f8853ee f
 0001:00084497       ?OnUpdateFileUpdate@COleServerDoc@@IAEXPAVCCmdUI@@@Z 5f885497 f
 0001:000844a8       ?OnSaveDocument@COleServerDoc@@UAEHPBG@Z 5f8854a8 f
 0001:00084537       ?OnShowDocument@COleServerDoc@@MAEXH@Z 5f885537 f
 0001:000847f6       ?OnNewEmbedding@COleServerDoc@@MAEXPAUIStorage@@@Z 5f8857f6 f
 0001:0008488d       ?OnOpenEmbedding@COleServerDoc@@MAEXPAUIStorage@@@Z 5f88588d f
 0001:00084928       ?OnSaveEmbedding@COleServerDoc@@MAEXPAUIStorage@@@Z 5f885928 f
 0001:000849af       ?_AfxGetWindow32@@YGPAUHWND__@@PAU1@@Z 5f8859af f
 0001:000849f0       ?ActivateInPlace@COleServerDoc@@QAEHXZ 5f8859f0 f
 0001:00084dee       ?CreateInPlaceFrame@COleServerDoc@@MAEPAVCOleIPFrameWnd@@PAVCWnd@@@Z 5f885dee f
 0001:00084ea3       ?DestroyInPlaceFrame@COleServerDoc@@MAEXPAVCOleIPFrameWnd@@@Z 5f885ea3 f
 0001:00084f8d       ?ConnectView@COleServerDoc@@IAEXPAVCWnd@@PAVCView@@@Z 5f885f8d f
 0001:00084fe4       ?OnFrameWindowActivate@COleServerDoc@@MAEXH@Z 5f885fe4 f
 0001:0008505b       ?OnDocWindowActivate@COleServerDoc@@MAEXH@Z 5f88605b f
 0001:0008519a       ?OnShowControlBars@COleServerDoc@@MAEXPAVCFrameWnd@@H@Z 5f88619a f
 0001:000851fc       ?OnResizeBorder@COleServerDoc@@UAEXPBUtagRECT@@PAUIOleInPlaceUIWindow@@H@Z 5f8861fc f
 0001:0008538a       ?OnDeactivate@COleServerDoc@@UAEXXZ 5f88638a f
 0001:00085417       ?OnDeactivateUI@COleServerDoc@@UAEXH@Z 5f886417 f
 0001:0008551a       ?OnSetItemRects@COleServerDoc@@MAEXPBUtagRECT@@0@Z 5f88651a f
 0001:00085537       ?OnReactivateAndUndo@COleServerDoc@@MAEHXZ 5f886537 f
 0001:0008553a       ?RequestPositionChange@COleServerDoc@@QAEXPBUtagRECT@@@Z 5f88653a f
 0001:00085565       ?ScrollContainerBy@COleServerDoc@@QAEHVCSize@@@Z 5f886565 f
 0001:0008559f       ?DeactivateAndUndo@COleServerDoc@@QAEHXZ 5f88659f f
 0001:000855d1       ?DiscardUndoState@COleServerDoc@@QAEHXZ 5f8865d1 f
 0001:00085603       ?GetClassID@XPersistStorage@COleServerDoc@@UAGJPAU_GUID@@@Z 5f886603 f
 0001:00085624       ?IsDirty@XPersistStorage@COleServerDoc@@UAGJXZ 5f886624 f
 0001:00085641       ?InitNew@XPersistStorage@COleServerDoc@@UAGJPAUIStorage@@@Z 5f886641 f
 0001:000856b7       ?Load@XPersistStorage@COleServerDoc@@UAGJPAUIStorage@@@Z 5f8866b7 f
 0001:00085746       ?Save@XPersistStorage@COleServerDoc@@UAGJPAUIStorage@@H@Z 5f886746 f
 0001:00085814       ?SaveCompleted@XPersistStorage@COleServerDoc@@UAGJPAUIStorage@@@Z 5f886814 f
 0001:000858a2       ?HandsOffStorage@XPersistStorage@COleServerDoc@@UAGJXZ 5f8868a2 f
 0001:0008590f       ?AddRef@XOleObject@COleServerDoc@@UAGKXZ 5f88690f f
 0001:00085921       ?Release@XOleObject@COleServerDoc@@UAGKXZ 5f886921 f
 0001:00085933       ?QueryInterface@XOleObject@COleServerDoc@@UAGJABU_GUID@@PAPAX@Z 5f886933 f
 0001:0008594d       ?SetClientSite@XOleObject@COleServerDoc@@UAGJPAUIOleClientSite@@@Z 5f88694d f
 0001:000859cc       ?GetClientSite@XOleObject@COleServerDoc@@UAGJPAPAUIOleClientSite@@@Z 5f8869cc f
 0001:000859f9       ?SetHostNames@XOleObject@COleServerDoc@@UAGJPBG0@Z 5f8869f9 f
 0001:00085a62       ?Close@XOleObject@COleServerDoc@@UAGJK@Z 5f886a62 f
 0001:00085af5       ?SetMoniker@XOleObject@COleServerDoc@@UAGJKPAUIMoniker@@@Z 5f886af5 f
 0001:00085b79       ?GetMoniker@XOleObject@COleServerDoc@@UAGJKKPAPAUIMoniker@@@Z 5f886b79 f
 0001:00085baa       ?InitFromData@XOleObject@COleServerDoc@@UAGJPAUIDataObject@@HK@Z 5f886baa f
 0001:00085c58       ?GetClipboardData@XOleObject@COleServerDoc@@UAGJKPAPAUIDataObject@@@Z 5f886c58 f
 0001:00085ce6       ?DoVerb@XOleObject@COleServerDoc@@UAGJJPAUtagMSG@@PAUIOleClientSite@@JPAUHWND__@@PBUtagRECT@@@Z 5f886ce6 f
 0001:00085d7d       ?EnumVerbs@XOleObject@COleServerDoc@@UAGJPAPAUIEnumOLEVERB@@@Z 5f886d7d f
 0001:00085db7       ?Update@XOleObject@COleServerDoc@@UAGJXZ 5f886db7 f
 0001:00085e31       ?IsUpToDate@XOleObject@COleServerDoc@@UAGJXZ 5f886e31 f
 0001:00085eae       ?GetUserClassID@XOleObject@COleServerDoc@@UAGJPAU_GUID@@@Z 5f886eae f
 0001:00085ecf       ?GetUserType@XOleObject@COleServerDoc@@UAGJKPAPAG@Z 5f886ecf f
 0001:00085f0c       ?SetExtent@XOleObject@COleServerDoc@@UAGJKPAUtagSIZE@@@Z 5f886f0c f
 0001:00085fa3       ?GetExtent@XOleObject@COleServerDoc@@UAGJKPAUtagSIZE@@@Z 5f886fa3 f
 0001:00086040       ?Advise@XOleObject@COleServerDoc@@UAGJPAUIAdviseSink@@PAK@Z 5f887040 f
 0001:000860ce       ?Unadvise@XOleObject@COleServerDoc@@UAGJK@Z 5f8870ce f
 0001:00086159       ?EnumAdvise@XOleObject@COleServerDoc@@UAGJPAPAUIEnumSTATDATA@@@Z 5f887159 f
 0001:000861e4       ?GetMiscStatus@XOleObject@COleServerDoc@@UAGJKPAK@Z 5f8871e4 f
 0001:00086221       ?SetColorScheme@XOleObject@COleServerDoc@@UAGJPAUtagLOGPALETTE@@@Z 5f887221 f
 0001:0008629b       ?AddRef@XDataObject@COleServerDoc@@UAGKXZ 5f88729b f
 0001:000862ad       ?Release@XDataObject@COleServerDoc@@UAGKXZ 5f8872ad f
 0001:000862bf       ?QueryInterface@XDataObject@COleServerDoc@@UAGJABU_GUID@@PAPAX@Z 5f8872bf f
 0001:000862d9       ?GetData@XDataObject@COleServerDoc@@UAGJPAUtagFORMATETC@@PAUtagSTGMEDIUM@@@Z 5f8872d9 f
 0001:00086367       ?GetDataHere@XDataObject@COleServerDoc@@UAGJPAUtagFORMATETC@@PAUtagSTGMEDIUM@@@Z 5f887367 f
 0001:000863f5       ?QueryGetData@XDataObject@COleServerDoc@@UAGJPAUtagFORMATETC@@@Z 5f8873f5 f
 0001:00086480       ?GetCanonicalFormatEtc@XDataObject@COleServerDoc@@UAGJPAUtagFORMATETC@@0@Z 5f887480 f
 0001:00086488       ?SetData@XDataObject@COleServerDoc@@UAGJPAUtagFORMATETC@@PAUtagSTGMEDIUM@@H@Z 5f887488 f
 0001:00086519       ?EnumFormatEtc@XDataObject@COleServerDoc@@UAGJKPAPAUIEnumFORMATETC@@@Z 5f887519 f
 0001:000865a7       ?DAdvise@XDataObject@COleServerDoc@@UAGJPAUtagFORMATETC@@KPAUIAdviseSink@@PAK@Z 5f8875a7 f
 0001:0008663b       ?DUnadvise@XDataObject@COleServerDoc@@UAGJK@Z 5f88763b f
 0001:000866c6       ?EnumDAdvise@XDataObject@COleServerDoc@@UAGJPAPAUIEnumSTATDATA@@@Z 5f8876c6 f
 0001:00086751       ?AddRef@XOleInPlaceObject@COleServerDoc@@UAGKXZ 5f887751 f
 0001:00086763       ?Release@XOleInPlaceObject@COleServerDoc@@UAGKXZ 5f887763 f
 0001:00086775       ?QueryInterface@XOleInPlaceObject@COleServerDoc@@UAGJABU_GUID@@PAPAX@Z 5f887775 f
 0001:0008678f       ?GetWindow@XOleInPlaceObject@COleServerDoc@@UAGJPAPAUHWND__@@@Z 5f88778f f
 0001:000867b0       ?ContextSensitiveHelp@XOleInPlaceObject@COleServerDoc@@UAGJH@Z 5f8877b0 f
 0001:000867d1       ?InPlaceDeactivate@XOleInPlaceObject@COleServerDoc@@UAGJXZ 5f8877d1 f
 0001:00086865       ?UIDeactivate@XOleInPlaceObject@COleServerDoc@@UAGJXZ 5f887865 f
 0001:00086905       ?SetObjectRects@XOleInPlaceObject@COleServerDoc@@UAGJPBUtagRECT@@0@Z 5f887905 f
 0001:0008697a       ?ReactivateAndUndo@XOleInPlaceObject@COleServerDoc@@UAGJXZ 5f88797a f
 0001:000869f6       ?AddRef@XOleInPlaceActiveObject@COleServerDoc@@UAGKXZ 5f8879f6 f
 0001:00086a08       ?Release@XOleInPlaceActiveObject@COleServerDoc@@UAGKXZ 5f887a08 f
 0001:00086a1a       ?QueryInterface@XOleInPlaceActiveObject@COleServerDoc@@UAGJABU_GUID@@PAPAX@Z 5f887a1a f
 0001:00086a34       ?GetWindow@XOleInPlaceActiveObject@COleServerDoc@@UAGJPAPAUHWND__@@@Z 5f887a34 f
 0001:00086a59       ?ContextSensitiveHelp@XOleInPlaceActiveObject@COleServerDoc@@UAGJH@Z 5f887a59 f
 0001:00086ada       ?TranslateAcceleratorW@XOleInPlaceActiveObject@COleServerDoc@@UAGJPAUtagMSG@@@Z 5f887ada f
 0001:00086b8c       ?OnFrameWindowActivate@XOleInPlaceActiveObject@COleServerDoc@@UAGJH@Z 5f887b8c f
 0001:00086bfe       ?OnDocWindowActivate@XOleInPlaceActiveObject@COleServerDoc@@UAGJH@Z 5f887bfe f
 0001:00086c70       ?ResizeBorder@XOleInPlaceActiveObject@COleServerDoc@@UAGJPBUtagRECT@@PAUIOleInPlaceUIWindow@@H@Z 5f887c70 f
 0001:00086ce8       ?EnableModeless@XOleInPlaceActiveObject@COleServerDoc@@UAGJH@Z 5f887ce8 f
 0001:00086d91       ??0COleServerItem@@IAE@PAVCOleServerDoc@@H@Z 5f887d91 f
 0001:00086e50       ??_GCOleServerItem@@UAEPAXI@Z 5f887e50 f
 0001:00086e50       ??_ECOleServerItem@@UAEPAXI@Z 5f887e50 f
 0001:00086e6c       ??1CItemDataSource@COleServerItem@@UAE@XZ 5f887e6c f
 0001:00086e71       ??_GCItemDataSource@COleServerItem@@UAEPAXI@Z 5f887e71 f
 0001:00086e71       ??_ECItemDataSource@COleServerItem@@UAEPAXI@Z 5f887e71 f
 0001:00086e8d       ?IsBlank@COleServerItem@@MBEHXZ 5f887e8d f
 0001:00086e91       ?IsConnected@COleServerItem@@QBEHXZ 5f887e91 f
 0001:00086eb2       ?NotifyClient@COleServerItem@@QAEXW4OLE_NOTIFICATION@@K@Z 5f887eb2 f
 0001:00086f1b       ?GetDataObject@COleServerItem@@QAEPAUIDataObject@@XZ 5f887f1b f
 0001:00086f26       ?GetOleObject@COleServerItem@@QAEPAUIOleObject@@XZ 5f887f26 f
 0001:00086f31       ?OnQueryUpdateItems@COleServerItem@@UAEHXZ 5f887f31 f
 0001:00086f6c       ?OnUpdateItems@COleServerItem@@UAEXXZ 5f887f6c f
 0001:00086faf       ?OnSetExtent@COleServerItem@@UAEHW4tagDVASPECT@@ABVCSize@@@Z 5f887faf f
 0001:00086fcf       ?OnGetExtent@COleServerItem@@UAEHW4tagDVASPECT@@AAVCSize@@@Z 5f887fcf f
 0001:00086fdf       ?OnDoVerb@COleServerItem@@UAEXJ@Z 5f887fdf f
 0001:00087049       ?OnDrawEx@COleServerItem@@UAEHPAVCDC@@W4tagDVASPECT@@AAVCSize@@@Z 5f888049 f
 0001:00087064       ?OnShow@COleServerItem@@MAEXXZ 5f888064 f
 0001:0008707f       ?OnOpen@COleServerItem@@MAEXXZ 5f88807f f
 0001:0008708d       ?OnHide@COleServerItem@@MAEXXZ 5f88808d f
 0001:0008709b       ?GetMetafileData@COleServerItem@@MAEHPAUtagFORMATETC@@PAUtagSTGMEDIUM@@@Z 5f88809b f
 0001:0008720f       ?OnInitFromData@COleServerItem@@UAEHPAVCOleDataObject@@H@Z 5f88820f f
 0001:0008721e       ?CopyToClipboard@COleServerItem@@QAEXH@Z 5f88821e f
 0001:00087235       ?OnGetClipboardData@COleServerItem@@UAEPAVCOleDataSource@@HPAUtagPOINT@@PAUtagSIZE@@@Z 5f888235 f
 0001:000872b2       ?DoDragDrop@COleServerItem@@QAEKPBUtagRECT@@VCPoint@@HK0@Z 5f8882b2 f
 0001:0008738b       ?GetClipboardData@COleServerItem@@QAEXPAVCOleDataSource@@HPAUtagPOINT@@PAUtagSIZE@@@Z 5f88838b f
 0001:00087435       ?GetEmbedSourceData@COleServerItem@@QAEXPAUtagSTGMEDIUM@@@Z 5f888435 f
 0001:00087527       ?AddOtherClipboardData@COleServerItem@@QAEXPAVCOleDataSource@@@Z 5f888527 f
 0001:000875c2       ?GetMoniker@COleServerItem@@QAEPAUIMoniker@@W4tagOLEGETMONIKER@@@Z 5f8885c2 f
 0001:000875e5       ?GetLinkSourceData@COleServerItem@@QAEHPAUtagSTGMEDIUM@@@Z 5f8885e5 f
 0001:0008769d       ?GetObjectDescriptorData@COleServerItem@@QAEXPAUtagPOINT@@PAUtagSIZE@@PAUtagSTGMEDIUM@@@Z 5f88869d f
 0001:00087741       ?OnSaveEmbedding@COleServerItem@@MAEXPAUIStorage@@@Z 5f888741 f
 0001:0008779b       ?OnRenderFileData@COleServerItem@@UAEHPAUtagFORMATETC@@PAVCFile@@@Z 5f88879b f
 0001:000877a0       ?OnRenderData@COleServerItem@@UAEHPAUtagFORMATETC@@PAUtagSTGMEDIUM@@@Z 5f8887a0 f
 0001:000877c4       ?OnSetData@COleServerItem@@UAEHPAUtagFORMATETC@@PAUtagSTGMEDIUM@@H@Z 5f8887c4 f
 0001:000877c9       ?GetInterfaceMap@COleServerItem@@MBEPBUAFX_INTERFACEMAP@@XZ 5f8887c9 f
 0001:000877cf       ?AddRef@XOleObject@COleServerItem@@UAGKXZ 5f8887cf f
 0001:000877de       ?Release@XOleObject@COleServerItem@@UAGKXZ 5f8887de f
 0001:000877ed       ?QueryInterface@XOleObject@COleServerItem@@UAGJABU_GUID@@PAPAX@Z 5f8887ed f
 0001:00087804       ?OnFinalRelease@COleServerItem@@UAEXXZ 5f888804 f
 0001:00087847       ?SetClientSite@XOleObject@COleServerItem@@UAGJPAUIOleClientSite@@@Z 5f888847 f
 0001:0008784f       ?GetClientSite@XOleObject@COleServerItem@@UAGJPAPAUIOleClientSite@@@Z 5f88884f f
 0001:0008785e       ?SetHostNames@XOleObject@COleServerItem@@UAGJPBG0@Z 5f88885e f
 0001:00087866       ?GetMoniker@XOleObject@COleServerItem@@UAGJKKPAPAUIMoniker@@@Z 5f888866 f
 0001:00087966       ?InitFromData@XOleObject@COleServerItem@@UAGJPAUIDataObject@@HK@Z 5f888966 f
 0001:0008796e       ?GetClipboardData@XOleObject@COleServerItem@@UAGJKPAPAUIDataObject@@@Z 5f88896e f
 0001:000879f2       ?DoVerb@XOleObject@COleServerItem@@UAGJJPAUtagMSG@@PAUIOleClientSite@@JPAUHWND__@@PBUtagRECT@@@Z 5f8889f2 f
 0001:00087a7f       ?EnumVerbs@XOleObject@COleServerItem@@UAGJPAPAUIEnumOLEVERB@@@Z 5f888a7f f
 0001:00087ab1       ?Update@XOleObject@COleServerItem@@UAGJXZ 5f888ab1 f
 0001:00087b21       ?IsUpToDate@XOleObject@COleServerItem@@UAGJXZ 5f888b21 f
 0001:00087b94       ?GetUserClassID@XOleObject@COleServerItem@@UAGJPAU_GUID@@@Z 5f888b94 f
 0001:00087bad       ?GetUserType@XOleObject@COleServerItem@@UAGJKPAPAG@Z 5f888bad f
 0001:00087be2       ?SetExtent@XOleObject@COleServerItem@@UAGJKPAUtagSIZE@@@Z 5f888be2 f
 0001:00087bea       ?GetExtent@XOleObject@COleServerItem@@UAGJKPAUtagSIZE@@@Z 5f888bea f
 0001:00087c7d       ?Advise@XOleObject@COleServerItem@@UAGJPAUIAdviseSink@@PAK@Z 5f888c7d f
 0001:00087cb6       ?GetMiscStatus@XOleObject@COleServerItem@@UAGJKPAK@Z 5f888cb6 f
 0001:00087ceb       ?SetColorScheme@XOleObject@COleServerItem@@UAGJPAUtagLOGPALETTE@@@Z 5f888ceb f
 0001:00087d5b       ?AddRef@XDataObject@COleServerItem@@UAGKXZ 5f888d5b f
 0001:00087d6a       ?Release@XDataObject@COleServerItem@@UAGKXZ 5f888d6a f
 0001:00087d79       ?QueryInterface@XDataObject@COleServerItem@@UAGJABU_GUID@@PAPAX@Z 5f888d79 f
 0001:00087d90       ?GetData@XDataObject@COleServerItem@@UAGJPAUtagFORMATETC@@PAUtagSTGMEDIUM@@@Z 5f888d90 f
 0001:00087da8       ?GetDataHere@XDataObject@COleServerItem@@UAGJPAUtagFORMATETC@@PAUtagSTGMEDIUM@@@Z 5f888da8 f
 0001:00087dc0       ?QueryGetData@XDataObject@COleServerItem@@UAGJPAUtagFORMATETC@@@Z 5f888dc0 f
 0001:00087dd4       ?SetData@XDataObject@COleServerItem@@UAGJPAUtagFORMATETC@@PAUtagSTGMEDIUM@@H@Z 5f888dd4 f
 0001:00087df0       ?EnumFormatEtc@XDataObject@COleServerItem@@UAGJKPAPAUIEnumFORMATETC@@@Z 5f888df0 f
 0001:00087e08       ?DAdvise@XDataObject@COleServerItem@@UAGJPAUtagFORMATETC@@KPAUIAdviseSink@@PAK@Z 5f888e08 f
 0001:00087eb3       ?DUnadvise@XDataObject@COleServerItem@@UAGJK@Z 5f888eb3 f
 0001:00087ed2       ?EnumDAdvise@XDataObject@COleServerItem@@UAGJPAPAUIEnumSTATDATA@@@Z 5f888ed2 f
 0001:00087ef5       ?OnRenderGlobalData@CItemDataSource@COleServerItem@@MAEHPAUtagFORMATETC@@PAPAX@Z 5f888ef5 f
 0001:00087f0c       ?OnRenderFileData@CItemDataSource@COleServerItem@@MAEHPAUtagFORMATETC@@PAVCFile@@@Z 5f888f0c f
 0001:00087f23       ?OnRenderData@CItemDataSource@COleServerItem@@MAEHPAUtagFORMATETC@@PAUtagSTGMEDIUM@@@Z 5f888f23 f
 0001:00087f56       ?OnSetData@CItemDataSource@COleServerItem@@MAEHPAUtagFORMATETC@@PAUtagSTGMEDIUM@@H@Z 5f888f56 f
 0001:00087f71       ?AfxOleRegisterServerClassCompat@@YGHABU_GUID@@PBG11W4OLE_APPTYPE@@PAPBG3@Z 5f888f71 f
 0001:0008804c       ?AfxOleUnregisterServerClass@@YGHABU_GUID@@PBG11W4OLE_APPTYPE@@PAPBG3@Z 5f88904c f
 0001:000880ff       ?AfxOleUnregisterHelper@@YGHPBQBG0HPAUHKEY__@@@Z 5f8890ff f
 0001:000881ca       ??0COleResizeBar@@QAE@XZ   5f8891ca f
 0001:00088211       ??1COleResizeBar@@UAE@XZ   5f889211 f
 0001:0008824c       ?Create@COleResizeBar@@QAEHPAVCWnd@@KI@Z 5f88924c f
 0001:0008828e       ?_GetBaseMessageMap@COleResizeBar@@KGPBUAFX_MSGMAP@@XZ 5f88928e f
 0001:00088294       ?GetMessageMap@COleResizeBar@@MBEPBUAFX_MSGMAP@@XZ 5f889294 f
 0001:0008829a       ?OnEraseBkgnd@COleResizeBar@@IAEHPAVCDC@@@Z 5f88929a f
 0001:000882a0       ?OnPaint@COleResizeBar@@IAEXXZ 5f8892a0 f
 0001:00088318       ?OnSize@COleResizeBar@@IAEXIHH@Z 5f889318 f
 0001:00088342       ?OnSetCursor@COleResizeBar@@IAEHPAVCWnd@@II@Z 5f889342 f
 0001:00088392       ?OnLButtonDown@COleResizeBar@@IAEXIVCPoint@@@Z 5f889392 f
 0001:0008847d       ?OnSizeParent@COleResizeBar@@IAEJIJ@Z 5f88947d f
 0001:000884b2       ?OnUpdateCmdUI@COleResizeBar@@UAEXPAVCFrameWnd@@H@Z 5f8894b2 f
 0001:000884b5       ?GetStandardProp@CCmdTarget@@IAEXPBUAFX_DISPMAP_ENTRY@@PAUtagVARIANT@@PAI@Z 5f8894b5 f
 0001:00088583       ?SetStandardProp@CCmdTarget@@IAEJPBUAFX_DISPMAP_ENTRY@@PAUtagDISPPARAMS@@PAI@Z 5f889583 f
 0001:000886f7       ?MemberIDFromName@CCmdTarget@@KGJPBUAFX_DISPMAP@@PBG@Z 5f8896f7 f
 0001:000887ef       ?GetNotSupported@CCmdTarget@@QAEXXZ 5f8897ef f
 0001:000887fe       ?SetNotSupported@CCmdTarget@@QAEXXZ 5f8897fe f
 0001:0008880d       ?GetIDispatch@CCmdTarget@@QAEPAUIDispatch@@H@Z 5f88980d f
 0001:0008882c       ?FromIDispatch@CCmdTarget@@SGPAV1@PAUIDispatch@@@Z 5f88982c f
 0001:00088842       ?IsResultExpected@CCmdTarget@@QAEHXZ 5f889842 f
 0001:0008884d       ?SetSysString@CString@@QBEPAGPAPAG@Z 5f88984d f
 0001:00088a71       ?GetTypeInfoCount@COleDispatchImpl@@UAGJPAI@Z 5f889a71 f
 0001:00088a89       ?GetTypeInfo@COleDispatchImpl@@UAGJIKPAPAUITypeInfo@@@Z 5f889a89 f
 0001:00088acf       ?GetIDsOfNames@COleDispatchImpl@@UAGJABU_GUID@@PAPAGIKPAJ@Z 5f889acf f
 0001:00088f07       ??1COleDispatchException@@UAE@XZ 5f889f07 f
 0001:00088f58       ??_GCOleDispatchException@@UAEPAXI@Z 5f889f58 f
 0001:00088f58       ??_ECOleDispatchException@@UAEPAXI@Z 5f889f58 f
 0001:00088f74       ?Process@COleDispatchException@@SGXPAUtagEXCEPINFO@@PBVCException@@@Z 5f889f74 f
 0001:00089067       ??0COleDispatchException@@QAE@PBGIG@Z 5f88a067 f
 0001:00089101       ?GetErrorMessage@COleDispatchException@@UAEHPAGIPAI@Z 5f88a101 f
 0001:00089123       ?AfxThrowOleDispatchException@@YGXGPBGI@Z 5f88a123 f
 0001:00089168       ?AfxThrowOleDispatchException@@YGXGII@Z 5f88a168 f
 0001:000891d4       ?AfxGetClassIDFromString@@YGJPBGPAU_GUID@@@Z 5f88a1d4 f
 0001:000891f4       ??0COleDispatchDriver@@QAE@PAUIDispatch@@H@Z 5f88a1f4 f
 0001:00089206       ??0COleDispatchDriver@@QAE@ABV0@@Z 5f88a206 f
 0001:00089228       ??4COleDispatchDriver@@QAEABV0@ABV0@@Z 5f88a228 f
 0001:00089295       ?CreateDispatch@COleDispatchDriver@@QAEHPBGPAVCOleException@@@Z 5f88a295 f
 0001:000892cf       ?AttachDispatch@COleDispatchDriver@@QAEXPAUIDispatch@@H@Z 5f88a2cf f
 0001:000892e8       ?DetachDispatch@COleDispatchDriver@@QAEPAUIDispatch@@XZ 5f88a2e8 f
 0001:0008951c       ?_AfxMultMultDivDiv@@YGJHHHHH@Z 5f88a51c f
 0001:0008967b       ??0CPreviewDC@@QAE@XZ      5f88a67b f
 0001:000896a7       ??_GCPreviewDC@@UAEPAXI@Z  5f88a6a7 f
 0001:000896a7       ??_ECPreviewDC@@UAEPAXI@Z  5f88a6a7 f
 0001:000896c3       ?SetOutputDC@CPreviewDC@@UAEXPAUHDC__@@@Z 5f88a6c3 f
 0001:00089712       ?ReleaseOutputDC@CPreviewDC@@UAEXXZ 5f88a712 f
 0001:0008972a       ?SetAttribDC@CPreviewDC@@UAEXPAUHDC__@@@Z 5f88a72a f
 0001:00089751       ??1CPreviewDC@@UAE@XZ      5f88a751 f
 0001:0008978d       ?SetScaleRatio@CPreviewDC@@QAEXHH@Z 5f88a78d f
 0001:000897b6       ?SaveDC@CPreviewDC@@UAEHXZ 5f88a7b6 f
 0001:00089805       ?RestoreDC@CPreviewDC@@UAEHH@Z 5f88a805 f
 0001:0008984a       ?MirrorAttributes@CPreviewDC@@IAEXXZ 5f88a84a f
 0001:00089924       ?SelectStockObject@CPreviewDC@@UAEPAVCGdiObject@@H@Z 5f88a924 f
 0001:00089994       ?MirrorFont@CPreviewDC@@IAEXXZ 5f88a994 f
 0001:00089b41       ?SelectObject@CPreviewDC@@UAEPAVCFont@@PAV2@@Z 5f88ab41 f
 0001:00089b80       ?SetBkColor@CPreviewDC@@UAEKK@Z 5f88ab80 f
 0001:00089bb1       ?SetTextColor@CPreviewDC@@UAEKK@Z 5f88abb1 f
 0001:00089be2       ?SetMapMode@CPreviewDC@@UAEHH@Z 5f88abe2 f
 0001:00089c05       ?SetViewportOrg@CPreviewDC@@UAE?AVCPoint@@HH@Z 5f88ac05 f
 0001:00089c3a       ?OffsetViewportOrg@CPreviewDC@@UAE?AVCPoint@@HH@Z 5f88ac3a f
 0001:00089c6f       ?SetViewportExt@CPreviewDC@@UAE?AVCSize@@HH@Z 5f88ac6f f
 0001:00089ca6       ?ScaleViewportExt@CPreviewDC@@UAE?AVCSize@@HHHH@Z 5f88aca6 f
 0001:00089ce3       ?SetWindowExt@CPreviewDC@@UAE?AVCSize@@HH@Z 5f88ace3 f
 0001:00089d1a       ?ScaleWindowExt@CPreviewDC@@UAE?AVCSize@@HHHH@Z 5f88ad1a f
 0001:00089d57       ?_AfxComputeNextTab@@YGHHIPAHHH@Z 5f88ad57 f
 0001:00089d8b       ?ComputeDeltas@CPreviewDC@@IAE?AVCSize@@AAHPBGAAIHIPAHHPAG30@Z 5f88ad8b f
 0001:00089fe3       ?TextOutW@CPreviewDC@@UAEHHHPBGH@Z 5f88afe3 f
 0001:0008a000       ?ExtTextOutW@CPreviewDC@@UAEHHHIPBUtagRECT@@PBGIPAH@Z 5f88b000 f
 0001:0008a111       ?TabbedTextOutW@CPreviewDC@@UAE?AVCSize@@HHPBGHHPAHH@Z 5f88b111 f
 0001:0008a231       ?DrawTextW@CPreviewDC@@UAEHPBGHPAUtagRECT@@I@Z 5f88b231 f
 0001:0008a277       ?GrayStringW@CPreviewDC@@UAEHPAVCBrush@@P6GHPAUHDC__@@JH@ZJHHHHH@Z 5f88b277 f
 0001:0008a28f       ?Escape@CPreviewDC@@UAEHHHPBDPAX@Z 5f88b28f f
 0001:0008a31d       ?MirrorMappingMode@CPreviewDC@@IAEXH@Z 5f88b31d f
 0001:0008a422       ?MirrorViewportOrg@CPreviewDC@@IAEXXZ 5f88b422 f
 0001:0008a48c       ?SetTopLeftOffset@CPreviewDC@@QAEXVCSize@@@Z 5f88b48c f
 0001:0008a4a2       ?ClipToPage@CPreviewDC@@QAEXXZ 5f88b4a2 f
 0001:0008a524       ?PrinterDPtoScreenDP@CPreviewDC@@QBEXPAUtagPOINT@@@Z 5f88b524 f
 0001:0008a57d       ??0CMetaFileDC@@QAE@XZ     5f88b57d f
 0001:0008a58f       ?SetOutputDC@CMetaFileDC@@MAEXPAUHDC__@@@Z 5f88b58f f
 0001:0008a592       ?ReleaseOutputDC@CMetaFileDC@@MAEXXZ 5f88b592 f
 0001:0008a593       ?SetAttribDC@CMetaFileDC@@UAEXPAUHDC__@@@Z 5f88b593 f
 0001:0008a5b8       ?GetClipBox@CMetaFileDC@@UBEHPAUtagRECT@@@Z 5f88b5b8 f
 0001:0008a5c8       ?PtVisible@CMetaFileDC@@UBEHHH@Z 5f88b5c8 f
 0001:0008a5dc       ?RectVisible@CMetaFileDC@@UBEHPBUtagRECT@@@Z 5f88b5dc f
 0001:0008a5e2       ?TextOutW@CMetaFileDC@@UAEHHHPBGH@Z 5f88b5e2 f
 0001:0008a64f       ?ExtTextOutW@CMetaFileDC@@UAEHHHIPBUtagRECT@@PBGIPAH@Z 5f88b64f f
 0001:0008a6b0       ?TabbedTextOutW@CMetaFileDC@@UAE?AVCSize@@HHPBGHHPAHH@Z 5f88b6b0 f
 0001:0008a80a       ?AdjustCP@CMetaFileDC@@IAEXH@Z 5f88b80a f
 0001:0008a86d       ?DrawTextW@CMetaFileDC@@UAEHPBGHPAUtagRECT@@I@Z 5f88b86d f
 0001:0008a8f3       ?Escape@CMetaFileDC@@UAEHHHPBDPAX@Z 5f88b8f3 f
 0001:0008a9a4       ?SetViewportOrg@CMetaFileDC@@UAE?AVCPoint@@HH@Z 5f88b9a4 f
 0001:0008a9e2       ?OffsetViewportOrg@CMetaFileDC@@UAE?AVCPoint@@HH@Z 5f88b9e2 f
 0001:0008aa20       ?SetViewportExt@CMetaFileDC@@UAE?AVCSize@@HH@Z 5f88ba20 f
 0001:0008aa5e       ?ScaleViewportExt@CMetaFileDC@@UAE?AVCSize@@HHHH@Z 5f88ba5e f
 0001:0008aac1       ?OnCancel@CPrintingDialog@@UAEXXZ 5f88bac1 f
 0001:0008ae06       ??_GCPrintingDialog@@UAEPAXI@Z 5f88be06 f
 0001:0008ae06       ??_ECPrintingDialog@@UAEPAXI@Z 5f88be06 f
 0001:0008ae29       ??0CPrintPreviewState@@QAE@XZ 5f88be29 f
 0001:0008ae4b       ?OnFilePrintPreview@CView@@IAEXXZ 5f88be4b f
 0001:0008ae96       ?DoPrintPreview@CView@@QAEHIPAV1@PAUCRuntimeClass@@PAUCPrintPreviewState@@@Z 5f88be96 f
 0001:0008b04d       ?_AfxPreviewCloseProc@@YGHPAVCFrameWnd@@@Z 5f88c04d f
 0001:0008b067       ?_GetBaseMessageMap@CPreviewView@@KGPBUAFX_MSGMAP@@XZ 5f88c067 f
 0001:0008b06d       ?GetMessageMap@CPreviewView@@MBEPBUAFX_MSGMAP@@XZ 5f88c06d f
 0001:0008b073       ??0CPreviewView@@QAE@XZ    5f88c073 f
 0001:0008b116       ??_ECPreviewView@@UAEPAXI@Z 5f88c116 f
 0001:0008b116       ??_GCPreviewView@@UAEPAXI@Z 5f88c116 f
 0001:0008b132       ??0PAGE_INFO@CPreviewView@@QAE@XZ 5f88c132 f
 0001:0008b135       ??1CPreviewView@@UAE@XZ    5f88c135 f
 0001:0008b1de       ?OnCreate@CPreviewView@@IAEHPAUtagCREATESTRUCTW@@@Z 5f88c1de f
 0001:0008b202       ?SetPrintView@CPreviewView@@QAEHPAVCView@@@Z 5f88c202 f
 0001:0008b466       ?OnSize@CPreviewView@@IAEXIHH@Z 5f88c466 f
 0001:0008b4cc       ?OnActivateView@CPreviewView@@MAEXHPAVCView@@0@Z 5f88c4cc f
 0001:0008b51b       ?OnPreviewClose@CPreviewView@@IAEXXZ 5f88c51b f
 0001:0008b55f       ?CalcScaleRatio@CPreviewView@@MAE?AVCSize@@V2@0@Z 5f88c55f f
 0001:0008b58e       ?PositionPage@CPreviewView@@MAEXI@Z 5f88c58e f
 0001:0008b644       ?CalcPageDisplaySize@CPreviewView@@IAE?AVCSize@@XZ 5f88c644 f
 0001:0008b6c8       ?SetScaledSize@CPreviewView@@IAEXI@Z 5f88c6c8 f
 0001:0008b823       ?OnPrepareDC@CPreviewView@@UAEXPAVCDC@@PAUCPrintInfo@@@Z 5f88c823 f
 0001:0008b857       ?OnEraseBkgnd@CPreviewView@@IAEHPAVCDC@@@Z 5f88c857 f
 0001:0008b8e7       ?OnDraw@CPreviewView@@MAEXPAVCDC@@@Z 5f88c8e7 f
 0001:0008bcef       ?OnHScroll@CPreviewView@@IAEXIIPAVCScrollBar@@@Z 5f88ccef f
 0001:0008bd0c       ?OnVScroll@CPreviewView@@IAEXIIPAVCScrollBar@@@Z 5f88cd0c f
 0001:0008bdf3       ?OnNumPageChange@CPreviewView@@IAEXXZ 5f88cdf3 f
 0001:0008be32       ?OnNextPage@CPreviewView@@IAEXXZ 5f88ce32 f
 0001:0008be42       ?OnPrevPage@CPreviewView@@IAEXXZ 5f88ce42 f
 0001:0008be52       ?OnPreviewPrint@CPreviewView@@IAEXXZ 5f88ce52 f
 0001:0008be75       ?FindPageRect@CPreviewView@@IAEHAAVCPoint@@AAI@Z 5f88ce75 f
 0001:0008bf3f       ?OnLButtonDown@CPreviewView@@IAEXIVCPoint@@@Z 5f88cf3f f
 0001:0008bf7d       ?SetZoomState@CPreviewView@@IAEXIIVCPoint@@@Z 5f88cf7d f
 0001:0008bfa1       ?OnZoomIn@CPreviewView@@IAEXXZ 5f88cfa1 f
 0001:0008bfbd       ?OnZoomOut@CPreviewView@@IAEXXZ 5f88cfbd f
 0001:0008bfd8       ?DoZoom@CPreviewView@@IAEXIVCPoint@@@Z 5f88cfd8 f
 0001:0008c147       ?SetCurrentPage@CPreviewView@@IAEXIH@Z 5f88d147 f
 0001:0008c1d9       ?OnDisplayPageNumber@CPreviewView@@MAEXII@Z 5f88d1d9 f
 0001:0008c29e       ?OnUpdateNumPageChange@CPreviewView@@IAEXPAVCCmdUI@@@Z 5f88d29e f
 0001:0008c342       ?OnUpdateNextPage@CPreviewView@@IAEXPAVCCmdUI@@@Z 5f88d342 f
 0001:0008c379       ?OnUpdatePrevPage@CPreviewView@@IAEXPAVCCmdUI@@@Z 5f88d379 f
 0001:0008c3a2       ?OnUpdateZoomIn@CPreviewView@@IAEXPAVCCmdUI@@@Z 5f88d3a2 f
 0001:0008c3be       ?OnUpdateZoomOut@CPreviewView@@IAEXPAVCCmdUI@@@Z 5f88d3be f
 0001:0008c3d9       ?OnSetCursor@CPreviewView@@IAEHPAVCWnd@@II@Z 5f88d3d9 f
 0001:0008c46a       ?GetPrinterDeviceDefaults@CWinApp@@QAEHPAUtagPDW@@@Z 5f88d46a f
 0001:0008c59e       ?OnFilePrintSetup@CWinApp@@IAEXXZ 5f88d59e f
 0001:0008c5f3       ?SelectPrinter@CWinApp@@QAEXPAX0H@Z 5f88d5f3 f
 0001:0008c64d       ??1_AFX_SOCK_STATE@@UAE@XZ 5f88d64d f
 0001:0008c67a       ??_G_AFX_SOCK_STATE@@UAEPAXI@Z 5f88d67a f
 0001:0008c67a       ??_E_AFX_SOCK_STATE@@UAEPAXI@Z 5f88d67a f
 0001:0008c695       ?AfxSocketTerm@@YGXXZ      5f88d695 f
 0001:0008c6c7       ?AfxSocketInit@@YGHPAUWSAData@@@Z 5f88d6c7 f
 0001:0008c72a       ??0CAsyncSocket@@QAE@XZ    5f88d72a f
 0001:0008c737       ?Create@CAsyncSocket@@QAEHIHJPBG@Z 5f88d737 f
 0001:0008c783       ?Attach@CAsyncSocket@@QAEHIJ@Z 5f88d783 f
 0001:0008c7a5       ?Detach@CAsyncSocket@@QAEIXZ 5f88d7a5 f
 0001:0008c7cc       ?GetPeerName@CAsyncSocket@@QAEHAAVCString@@AAI@Z 5f88d7cc f
 0001:0008c832       ?GetSockName@CAsyncSocket@@QAEHAAVCString@@AAI@Z 5f88d832 f
 0001:0008c898       ?Accept@CAsyncSocket@@UAEHAAV1@PAUsockaddr@@PAH@Z 5f88d898 f
 0001:0008c911       ?Bind@CAsyncSocket@@QAEHIPBG@Z 5f88d911 f
 0001:0008c9c2       ?Close@CAsyncSocket@@UAEXXZ 5f88d9c2 f
 0001:0008c9e2       ?Connect@CAsyncSocket@@QAEHPBGI@Z 5f88d9e2 f
 0001:0008ca90       ?Receive@CAsyncSocket@@UAEHPAXHH@Z 5f88da90 f
 0001:0008caa7       ?ReceiveFrom@CAsyncSocket@@QAEHPAXHAAVCString@@AAIH@Z 5f88daa7 f
 0001:0008cb0e       ?Send@CAsyncSocket@@UAEHPBXHH@Z 5f88db0e f
 0001:0008cb25       ?SendTo@CAsyncSocket@@QAEHPBXHIPBGH@Z 5f88db25 f
 0001:0008cbed       ?AsyncSelect@CAsyncSocket@@QAEHJ@Z 5f88dbed f
 0001:0008cc17       ?OnClose@CAsyncSocket@@MAEXH@Z 5f88dc17 f
 0001:0008cc1a       ?LookupHandle@CAsyncSocket@@SGPAV1@IH@Z 5f88dc1a f
 0001:0008cc3c       ?AttachHandle@CAsyncSocket@@SGXIPAV1@H@Z 5f88dc3c f
 0001:0008cd03       ?DetachHandle@CAsyncSocket@@SGXIH@Z 5f88dd03 f
 0001:0008cda9       ?KillSocket@CAsyncSocket@@SGXIPAV1@@Z 5f88dda9 f
 0001:0008cde8       ?DoCallBack@CAsyncSocket@@SGXIJ@Z 5f88dde8 f
 0001:0008cebe       ?Socket@CAsyncSocket@@QAEHHJHH@Z 5f88debe f
 0001:0008cef6       ?ReceiveFromHelper@CAsyncSocket@@MAEHPAXHPAUsockaddr@@PAHH@Z 5f88def6 f
 0001:0008cf14       ?SendToHelper@CAsyncSocket@@MAEHPBXHPBUsockaddr@@HH@Z 5f88df14 f
 0001:0008cf32       ?ConnectHelper@CAsyncSocket@@MAEHPBUsockaddr@@H@Z 5f88df32 f
 0001:0008cf4f       ??0CSocket@@QAE@XZ         5f88df4f f
 0001:0008cf70       ?CancelBlockingCall@CSocket@@QAEXXZ 5f88df70 f
 0001:0008cf7f       ?OnMessagePending@CSocket@@MAEHXZ 5f88df7f f
 0001:0008cfa9       ??1CSocket@@UAE@XZ         5f88dfa9 f
 0001:0008cfe7       ?Accept@CSocket@@UAEHAAVCAsyncSocket@@PAUsockaddr@@PAH@Z 5f88dfe7 f
 0001:0008d038       ?Close@CSocket@@UAEXXZ     5f88e038 f
 0001:0008d05c       ?Receive@CSocket@@UAEHPAXHH@Z 5f88e05c f
 0001:0008d0ac       ?Send@CSocket@@UAEHPBXHH@Z 5f88e0ac f
 0001:0008d0fa       ?SendChunk@CSocket@@QAEHPBXHH@Z 5f88e0fa f
 0001:0008d136       ?ConnectHelper@CSocket@@MAEHPBUsockaddr@@H@Z 5f88e136 f
 0001:0008d19c       ?ReceiveFromHelper@CSocket@@MAEHPAXHPAUsockaddr@@PAHH@Z 5f88e19c f
 0001:0008d1f2       ?SendToHelper@CSocket@@MAEHPBXHPBUsockaddr@@HH@Z 5f88e1f2 f
 0001:0008d246       ?ProcessAuxQueue@CSocket@@SGHXZ 5f88e246 f
 0001:0008d29d       ?AuxQueueAdd@CSocket@@KGXIIJ@Z 5f88e29d f
 0001:0008d2cf       ?PumpMessages@CSocket@@MAEHI@Z 5f88e2cf f
 0001:0008d468       ??0CSocketFile@@QAE@PAVCSocket@@H@Z 5f88e468 f
 0001:0008d48a       ??_GCSocketFile@@UAEPAXI@Z 5f88e48a f
 0001:0008d48a       ??_ECSocketFile@@UAEPAXI@Z 5f88e48a f
 0001:0008d4a6       ??1CSocketFile@@UAE@XZ     5f88e4a6 f
 0001:0008d4b1       ?Read@CSocketFile@@UAEIPAXI@Z 5f88e4b1 f
 0001:0008d534       ?Write@CSocketFile@@UAEXPBXI@Z 5f88e534 f
 0001:0008d55d       ?Close@CSocketFile@@UAEXXZ 5f88e55d f
 0001:0008d562       ?Open@CSocketFile@@UAEHPBGIPAVCFileException@@@Z 5f88e562 f
 0001:0008d56c       ?Duplicate@CSocketFile@@UBEPAVCFile@@XZ 5f88e56c f
 0001:0008d574       ?Seek@CSocketFile@@UAEJJI@Z 5f88e574 f
 0001:0008d579       ?SetLength@CSocketFile@@UAEXK@Z 5f88e579 f
 0001:0008d581       ?LockRange@CSocketFile@@UAEXKK@Z 5f88e581 f
 0001:0008d589       ?Flush@CSocketFile@@UAEXXZ 5f88e589 f
 0001:0008d58a       ?Abort@CSocketFile@@UAEXXZ 5f88e58a f
 0001:0008d58f       ??0CSocketWnd@@QAE@XZ      5f88e58f f
 0001:0008d5a1       ??_ECSocketWnd@@UAEPAXI@Z  5f88e5a1 f
 0001:0008d5a1       ??_GCSocketWnd@@UAEPAXI@Z  5f88e5a1 f
 0001:0008d5bd       ??1CSocketWnd@@UAE@XZ      5f88e5bd f
 0001:0008d5c2       ?OnSocketNotify@CSocketWnd@@IAEJIJ@Z 5f88e5c2 f
 0001:0008d5de       ?OnSocketDead@CSocketWnd@@IAEJIJ@Z 5f88e5de f
 0001:0008d5fa       ?_GetBaseMessageMap@CSocketWnd@@KGPBUAFX_MSGMAP@@XZ 5f88e5fa f
 0001:0008d600       ?GetMessageMap@CSocketWnd@@MBEPBUAFX_MSGMAP@@XZ 5f88e600 f
 0001:0008d6a6       ?AfxLoadLibrary@@YGPAUHINSTANCE__@@PBG@Z 5f88e6a6 f
 0001:0008d6c7       ?AfxFreeLibrary@@YGHPAUHINSTANCE__@@@Z 5f88e6c7 f
 0001:0008d6e8       ??_ECBitmap@@UAEPAXI@Z     5f88e6e8 f
 0001:0008d733       ??_ECBitmapButton@@UAEPAXI@Z 5f88e733 f
 0001:0008d77e       ??_ECBrush@@UAEPAXI@Z      5f88e77e f
 0001:0008d7c9       ??_ECButton@@UAEPAXI@Z     5f88e7c9 f
 0001:0008d814       ??_ECByteArray@@UAEPAXI@Z  5f88e814 f
 0001:0008d85f       ??_ECCmdTarget@@UAEPAXI@Z  5f88e85f f
 0001:0008d8aa       ??_ECComboBox@@UAEPAXI@Z   5f88e8aa f
 0001:0008d8f5       ??_ECDC@@UAEPAXI@Z         5f88e8f5 f
 0001:0008d940       ??_ECDWordArray@@UAEPAXI@Z 5f88e940 f
 0001:0008d98b       ??_ECDialog@@UAEPAXI@Z     5f88e98b f
 0001:0008d9d6       ??_ECDialogBar@@UAEPAXI@Z  5f88e9d6 f
 0001:0008da24       ??_ECEdit@@UAEPAXI@Z       5f88ea24 f
 0001:0008da6f       ??_ECFile@@UAEPAXI@Z       5f88ea6f f
 0001:0008daba       ??_ECFont@@UAEPAXI@Z       5f88eaba f
 0001:0008db05       ??_ECFrameWnd@@UAEPAXI@Z   5f88eb05 f
 0001:0008db53       ??_ECGdiObject@@UAEPAXI@Z  5f88eb53 f
 0001:0008db9e       ??_ECListBox@@UAEPAXI@Z    5f88eb9e f
 0001:0008dbe9       ??_ECCheckListBox@@UAEPAXI@Z 5f88ebe9 f
 0001:0008dc34       ??_ECMapPtrToPtr@@UAEPAXI@Z 5f88ec34 f
 0001:0008dc7f       ??_ECMapPtrToWord@@UAEPAXI@Z 5f88ec7f f
 0001:0008dcca       ??_ECMapStringToOb@@UAEPAXI@Z 5f88ecca f
 0001:0008dd15       ??_ECMapStringToPtr@@UAEPAXI@Z 5f88ed15 f
 0001:0008dd60       ??_ECMapStringToString@@UAEPAXI@Z 5f88ed60 f
 0001:0008ddab       ??_ECMapWordToOb@@UAEPAXI@Z 5f88edab f
 0001:0008ddf6       ??_ECMapWordToPtr@@UAEPAXI@Z 5f88edf6 f
 0001:0008de41       ??_ECMemFile@@UAEPAXI@Z    5f88ee41 f
 0001:0008de8c       ??_ECMenu@@UAEPAXI@Z       5f88ee8c f
 0001:0008ded7       ??_ECMetaFileDC@@UAEPAXI@Z 5f88eed7 f
 0001:0008df22       ??_ECObArray@@UAEPAXI@Z    5f88ef22 f
 0001:0008df6d       ??_ECObList@@UAEPAXI@Z     5f88ef6d f
 0001:0008dfb8       ??_ECPalette@@UAEPAXI@Z    5f88efb8 f
 0001:0008e003       ??_ECPen@@UAEPAXI@Z        5f88f003 f
 0001:0008e04e       ??_ECPtrArray@@UAEPAXI@Z   5f88f04e f
 0001:0008e0c0       ??_ECRectTracker@@UAEPAXI@Z 5f88f0c0 f
 0001:0008e10b       ??_ECRgn@@UAEPAXI@Z        5f88f10b f
 0001:0008e156       ??_ECScrollBar@@UAEPAXI@Z  5f88f156 f
 0001:0008e1a1       ??_ECSharedFile@@UAEPAXI@Z 5f88f1a1 f
 0001:0008e1ec       ??_ECSplitterWnd@@UAEPAXI@Z 5f88f1ec f
 0001:0008e23a       ??_ECStatic@@UAEPAXI@Z     5f88f23a f
 0001:0008e285       ??_ECStatusBar@@UAEPAXI@Z  5f88f285 f
 0001:0008e2d3       ??_ECStdioFile@@UAEPAXI@Z  5f88f2d3 f
 0001:0008e31e       ??_ECStringArray@@UAEPAXI@Z 5f88f31e f
 0001:0008e369       ??_ECStringList@@UAEPAXI@Z 5f88f369 f
 0001:0008e3b4       ??_ECToolBar@@UAEPAXI@Z    5f88f3b4 f
 0001:0008e402       ??_ECUIntArray@@UAEPAXI@Z  5f88f402 f
 0001:0008e44d       ??_ECWnd@@UAEPAXI@Z        5f88f44d f
 0001:0008e498       ??_ECWordArray@@UAEPAXI@Z  5f88f498 f
 0001:0008e4e3       ??_ECFileFind@@UAEPAXI@Z   5f88f4e3 f
 0001:0008e52e       ??_ECInternetSession@@UAEPAXI@Z 5f88f52e f
 0001:0008e579       ??_ECDragListBox@@UAEPAXI@Z 5f88f579 f
 0001:0008e5c4       ??_ECStatusBarCtrl@@UAEPAXI@Z 5f88f5c4 f
 0001:0008e60f       ??_ECListCtrl@@UAEPAXI@Z   5f88f60f f
 0001:0008e65a       ??_ECTreeCtrl@@UAEPAXI@Z   5f88f65a f
 0001:0008e6a5       ??_ECSpinButtonCtrl@@UAEPAXI@Z 5f88f6a5 f
 0001:0008e6f0       ??_ECSliderCtrl@@UAEPAXI@Z 5f88f6f0 f
 0001:0008e73b       ??_ECProgressCtrl@@UAEPAXI@Z 5f88f73b f
 0001:0008e786       ??_ECHeaderCtrl@@UAEPAXI@Z 5f88f786 f
 0001:0008e7d1       ??_ECHotKeyCtrl@@UAEPAXI@Z 5f88f7d1 f
 0001:0008e81c       ??_ECToolTipCtrl@@UAEPAXI@Z 5f88f81c f
 0001:0008e867       ??_ECTabCtrl@@UAEPAXI@Z    5f88f867 f
 0001:0008e8b2       ??_ECAnimateCtrl@@UAEPAXI@Z 5f88f8b2 f
 0001:0008e8fd       ??_ECImageList@@UAEPAXI@Z  5f88f8fd f
 0001:0008e948       ??_ECToolBarCtrl@@UAEPAXI@Z 5f88f948 f
 0001:0008e993       ??_ECRichEditCtrl@@UAEPAXI@Z 5f88f993 f
 0001:0008e9de       ??_ECMirrorFile@@UAEPAXI@Z 5f88f9de f
 0001:0008ea29       ??0CMirrorFile@@QAE@XZ     5f88fa29 f
 0001:0008ea60       ??_ECDockState@@UAEPAXI@Z  5f88fa60 f
 0001:0008eaab       ??_ECListView@@UAEPAXI@Z   5f88faab f
 0001:0008eaf6       ??_ECTreeView@@UAEPAXI@Z   5f88faf6 f
 0001:0008eb41       ??_ECCommandLineInfo@@UAEPAXI@Z 5f88fb41 f
 0001:0008ebb3       ??_ECPageSetupDialog@@UAEPAXI@Z 5f88fbb3 f
 0001:0008ec01       ??_ECSemaphore@@UAEPAXI@Z  5f88fc01 f
 0001:0008ec4c       ??_ECMutex@@UAEPAXI@Z      5f88fc4c f
 0001:0008ec97       ??_ECEvent@@UAEPAXI@Z      5f88fc97 f
 0001:0008ece2       ??_ECCriticalSection@@UAEPAXI@Z 5f88fce2 f
 0001:0008ed2d       ??_ECOleDataSource@@UAEPAXI@Z 5f88fd2d f
 0001:0008ed78       ??_ECOleDropSource@@UAEPAXI@Z 5f88fd78 f
 0001:0008edc3       ??_ECMonikerFile@@UAEPAXI@Z 5f88fdc3 f
 0001:0008ee0e       ??_ECOleResizeBar@@UAEPAXI@Z 5f88fe0e f
 0001:0008ee5c       ??_ECAsyncMonikerFile@@UAEPAXI@Z 5f88fe5c f
 0001:0008eea7       ??_ECCachedDataPathProperty@@UAEPAXI@Z 5f88fea7 f
 0001:0008eef2       ??_ECDataPathProperty@@UAEPAXI@Z 5f88fef2 f
 0001:0008ef3d       ??_ECOleStreamFile@@UAEPAXI@Z 5f88ff3d f
 0001:0008ef88       ??_ECOleTemplateServer@@UAEPAXI@Z 5f88ff88 f
 0001:0008efd3       ??_ECOleDropTarget@@UAEPAXI@Z 5f88ffd3 f
 0001:0008f01e       ??_ECOleIPFrameWnd@@UAEPAXI@Z 5f89001e f
 0001:0008f06c       ??_ECOleDocIPFrameWnd@@UAEPAXI@Z 5f89006c f
 0001:0008f0ba       ??_ECRichEditView@@UAEPAXI@Z 5f8900ba f
 0001:0008f108       ??_ECRichEditCntrItem@@UAEPAXI@Z 5f890108 f
 0001:0008f156       ??_ECDatabase@@UAEPAXI@Z   5f890156 f
 0001:0008f1a1       ??_ECLongBinary@@UAEPAXI@Z 5f8901a1 f
 0001:0008f1ec       ??_ECDaoWorkspace@@UAEPAXI@Z 5f8901ec f
 0001:0008f237       ??_ECDaoException@@UAEPAXI@Z 5f890237 f
 0001:0008f282       ??_ECDaoDatabase@@UAEPAXI@Z 5f890282 f
 0001:0008f2cd       ??_ECDaoRecordset@@UAEPAXI@Z 5f8902cd f
 0001:0008f31b       ??_ECAsyncSocket@@UAEPAXI@Z 5f89031b f
 0001:0008f366       ??_ECSocket@@UAEPAXI@Z     5f890366 f
 0001:0008f3b1       ?_AfxBinaryCompatibleStubFunction@@YAXXZ 5f8903b1 f
 0001:0008f3b7       ___CxxFrameHandler         5f8903b7 f
 0001:0008f447       ??1CObject@@UAE@XZ         5f890447 f
 0001:0008f4ce       ??1CFileException@@UAE@XZ  5f8904ce f
 0001:0008fad1       ??1CNoTrackObject@@UAE@XZ  5f890ad1 f
 0001:0008fb51       ??1AFX_MAINTAIN_STATE2@@QAE@XZ 5f890b51 f
 0001:0008fc37       ??1CWaitCursor@@QAE@XZ     5f890c37 f
 0001:0008fd43       ??1CPushRoutingFrame@@QAE@XZ 5f890d43 f
 0001:0008fee9       ??1CBrush@@UAE@XZ          5f890ee9 f
 0001:0009011b       ??1CMiniFrameWnd@@UAE@XZ   5f89111b f
 0001:00090334       ??1CRgn@@UAE@XZ            5f891334 f
 0001:00090529       ??1CBitmap@@UAE@XZ         5f891529 f
 0001:00090645       ??1CDialogTemplate@@QAE@XZ 5f891645 f
 0001:00090810       ??1CPropertyPage@@UAE@XZ   5f891810 f
 0001:0009090d       ??1CPropertySheet@@UAE@XZ  5f89190d f
 0001:00090c05       ??1CGdiObject@@UAE@XZ      5f891c05 f
 0001:000910bd       ??1CFileDialog@@UAE@XZ     5f8920bd f
 0001:000911b7       ??1CNewTypeDlg@@UAE@XZ     5f8921b7 f
 0001:00091210       ??1CPushRoutingView@@QAE@XZ 5f892210 f
 0001:000912e6       ??1CPrintingDialog@@UAE@XZ 5f8922e6 f
 0001:000913fe       ??1CCtrlView@@UAE@XZ       5f8923fe f
 0001:00091448       ??1CUIntArray@@UAE@XZ      5f892448 f
 0001:000915c1       ??1CPen@@UAE@XZ            5f8925c1 f
 0001:000919f9       ??1CStdioFile@@UAE@XZ      5f8929f9 f
 0001:00091b6e       ??1CGopherLocator@@UAE@XZ  5f892b6e f
 0001:00091ca3       ??1CInternetFile@@UAE@XZ   5f892ca3 f
 0001:00091fc2       ??1CAsyncSocket@@UAE@XZ    5f892fc2 f
 0001:00092025       ??1CDocItem@@UAE@XZ        5f893025 f
 0001:00092345       ??1CSharedFile@@UAE@XZ     5f893345 f
 0001:00092386       ??1COleStreamFile@@UAE@XZ  5f893386 f
 0001:000925d5       ??1COleLinksDialog@@UAE@XZ 5f8935d5 f
 0001:000926a0       ??1COleSafeArray@@QAE@XZ   5f8936a0 f
 0001:00092a10       ??1COleBusyDialog@@UAE@XZ  5f893a10 f
 0001:000930a6       ??1CMetaFileDC@@UAE@XZ     5f8940a6 f
 0001:000932c8       ??1COleConvertDialog@@UAE@XZ 5f8942c8 f
 0001:00093316       ??1COleChangeIconDialog@@UAE@XZ 5f894316 f
 0001:00093414       ??1COleClientItem@@UAE@XZ  5f894414 f
 0001:000934d4       ??1COleInsertDialog@@UAE@XZ 5f8944d4 f
 0001:00093527       ??1CReObject@@QAE@XZ       5f894527 f
 0001:00093583       ??1COlePasteSpecialDialog@@UAE@XZ 5f894583 f
 0001:00093ac3       ??1CByteArray@@UAE@XZ      5f894ac3 f
 0001:00093c00       ??1CFont@@UAE@XZ           5f894c00 f
 0001:00093c74       ??1CEnumArray@@UAE@XZ      5f894c74 f
 0001:00093e8d       ??1?$CComPtr@UIRowsetChange@@@ATL@@QAE@XZ 5f894e8d f
 0001:00093ff3       ??1CManualAccessor@ATL@@QAE@XZ 5f894ff3 f
 0001:000945c7       ??1COleCmdUI@@QAE@XZ       5f8955c7 f
 0001:000946b0       ??1CMonikerFile@@UAE@XZ    5f8956b0 f
 0001:00095135       ??1CStringArray@@UAE@XZ    5f896135 f
 0001:000951c7       ??1CPropertySet@@QAE@XZ    5f8961c7 f
 0001:000954cb       ??1CPropbagPropExchange@@QAE@XZ 5f8964cb f
 0001:0009555e       ??1CStockPropPage@@UAE@XZ  5f89655e f
 0001:000955d7       ??1COlePropertyPage@@UAE@XZ 5f8965d7 f
 0001:000957c3       ??1CFontComboBox@@UAE@XZ   5f8967c3 f
 0001:00095e37       ??1CDBException@@UAE@XZ    5f896e37 f
 0001:00096444       ??1CDaoRelationInfo@@UAE@XZ 5f897444 f
 0001:000964b6       ??1CDaoRelationFieldInfo@@QAE@XZ 5f8974b6 f
 0001:0009676f       ??1CDaoFieldInfo@@QAE@XZ   5f89776f f
 0001:000968ec       ??1CDaoIndexInfo@@UAE@XZ   5f8978ec f
 0001:000972cf       ??1CAsyncMonikerFile@@UAE@XZ 5f8982cf f
 0001:00097337       ??1CDataPathProperty@@UAE@XZ 5f898337 f
 0002:00000000       __imp___initterm           5f899000  
 0002:00000004       __imp_?terminate@@YAXXZ    5f899004  
 0002:00000008       __imp___except_handler3    5f899008  
 0002:0000000c       __imp___adjust_fdiv        5f89900c  
 0002:00000010       __imp___onexit             5f899010  
 0002:00000014       __imp____dllonexit         5f899014  
 0002:00000018       __imp_??1type_info@@UAE@XZ 5f899018  
 0002:0000001c       __imp___wcsnicmp           5f89901c  
 0002:00000020       __imp__wcsncpy             5f899020  
 0002:00000024       __imp__wcscpy              5f899024  
 0002:00000028       __imp___ltow               5f899028  
 0002:0000002c       __imp___ultow              5f89902c  
 0002:00000030       __imp___itow               5f899030  
 0002:00000034       __imp__modf                5f899034  
 0002:00000038       __imp__ceil                5f899038  
 0002:0000003c       __imp__fabs                5f89903c  
 0002:00000040       __imp__floor               5f899040  
 0002:00000044       __imp__labs                5f899044  
 0002:00000048       __imp___ftol               5f899048  
 0002:0000004c       __imp___wsplitpath         5f89904c  
 0002:00000050       __imp___EH_prolog          5f899050  
 0002:00000054       __imp___wfullpath          5f899054  
 0002:00000058       __imp___wtol               5f899058  
 0002:0000005c       __imp____p___argc          5f89905c  
 0002:00000060       __imp____p___wargv         5f899060  
 0002:00000064       __imp___beginthreadex      5f899064  
 0002:00000068       __imp___endthreadex        5f899068  
 0002:0000006c       __imp___wcsdup             5f89906c  
 0002:00000070       __imp___expand             5f899070  
 0002:00000074       __imp__swprintf            5f899074  
 0002:00000078       __imp__wcstod              5f899078  
 0002:0000007c       __imp__wcstol              5f89907c  
 0002:00000080       __imp__wcstoul             5f899080  
 0002:00000084       __imp__abs                 5f899084  
 0002:00000088       __imp__calloc              5f899088  
 0002:0000008c       __imp___msize              5f89908c  
 0002:00000090       __imp___purecall           5f899090  
 0002:00000094       __imp__wcsftime            5f899094  
 0002:00000098       __imp__localtime           5f899098  
 0002:0000009c       __imp__gmtime              5f89909c  
 0002:000000a0       __imp__mktime              5f8990a0  
 0002:000000a4       __imp__iswspace            5f8990a4  
 0002:000000a8       __imp___wtoi               5f8990a8  
 0002:000000ac       __imp__iswdigit            5f8990ac  
 0002:000000b0       __imp__wcsncmp             5f8990b0  
 0002:000000b4       __imp__wcslen              5f8990b4  
 0002:000000b8       __imp__vswprintf           5f8990b8  
 0002:000000bc       __imp__wcsrchr             5f8990bc  
 0002:000000c0       __imp__wcscspn             5f8990c0  
 0002:000000c4       __imp__wcsspn              5f8990c4  
 0002:000000c8       __imp__wcsstr              5f8990c8  
 0002:000000cc       __imp___wcsrev             5f8990cc  
 0002:000000d0       __imp___wcslwr             5f8990d0  
 0002:000000d4       __imp___wcsupr             5f8990d4  
 0002:000000d8       __imp__wcspbrk             5f8990d8  
 0002:000000dc       __imp__wcschr              5f8990dc  
 0002:000000e0       __imp__wcscmp              5f8990e0  
 0002:000000e4       __imp__realloc             5f8990e4  
 0002:000000e8       __imp__fclose              5f8990e8  
 0002:000000ec       __imp__fflush              5f8990ec  
 0002:000000f0       __imp__fseek               5f8990f0  
 0002:000000f4       __imp__ftell               5f8990f4  
 0002:000000f8       __imp__fgetws              5f8990f8  
 0002:000000fc       __imp__fputws              5f8990fc  
 0002:00000100       __imp__fwrite              5f899100  
 0002:00000104       __imp__fread               5f899104  
 0002:00000108       __imp__clearerr            5f899108  
 0002:0000010c       __imp___open_osfhandle     5f89910c  
 0002:00000110       __imp___fdopen             5f899110  
 0002:00000114       __imp____doserrno          5f899114  
 0002:00000118       __imp___get_osfhandle      5f899118  
 0002:0000011c       __imp__memset              5f89911c  
 0002:00000120       __imp__abort               5f899120  
 0002:00000124       __imp__free                5f899124  
 0002:00000128       __imp__malloc              5f899128  
 0002:0000012c       __imp__memcmp              5f89912c  
 0002:00000130       __imp__memmove             5f899130  
 0002:00000134       __imp__memcpy              5f899134  
 0002:00000138       __imp___CxxThrowException@8 5f899138  
 0002:0000013c       __imp__time                5f89913c  
 0002:00000140       __imp____CxxFrameHandler   5f899140  
 0002:00000148       __imp__lstrcmpiW@8         5f899148  
 0002:0000014c       __imp__GetShortPathNameW@12 5f89914c  
 0002:00000150       __imp__GetThreadLocale@0   5f899150  
 0002:00000154       __imp__GetStringTypeExW@20 5f899154  
 0002:00000158       __imp__GetModuleFileNameW@12 5f899158  
 0002:0000015c       __imp__GlobalLock@4        5f89915c  
 0002:00000160       __imp__GlobalAlloc@8       5f899160  
 0002:00000164       __imp__GlobalReAlloc@12    5f899164  
 0002:00000168       __imp__GlobalUnlock@4      5f899168  
 0002:0000016c       __imp__GlobalFree@4        5f89916c  
 0002:00000170       __imp__GetFileAttributesW@4 5f899170  
 0002:00000174       __imp__GetFileSize@8       5f899174  
 0002:00000178       __imp__GetFileTime@16      5f899178  
 0002:0000017c       __imp__LocalFileTimeToFileTime@8 5f89917c  
 0002:00000180       __imp__SystemTimeToFileTime@8 5f899180  
 0002:00000184       __imp__SetFileTime@16      5f899184  
 0002:00000188       __imp__SetFileAttributesW@8 5f899188  
 0002:0000018c       __imp__InterlockedIncrement@4 5f89918c  
 0002:00000190       __imp__InterlockedDecrement@4 5f899190  
 0002:00000194       __imp__WideCharToMultiByte@32 5f899194  
 0002:00000198       __imp__MultiByteToWideChar@24 5f899198  
 0002:0000019c       __imp__LocalFree@4         5f89919c  
 0002:000001a0       __imp__FormatMessageW@28   5f8991a0  
 0002:000001a4       __imp__FileTimeToSystemTime@8 5f8991a4  
 0002:000001a8       __imp__FileTimeToLocalFileTime@8 5f8991a8  
 0002:000001ac       __imp__LocalAlloc@8        5f8991ac  
 0002:000001b0       __imp__InitializeCriticalSection@4 5f8991b0  
 0002:000001b4       __imp__TlsAlloc@0          5f8991b4  
 0002:000001b8       __imp__DeleteCriticalSection@4 5f8991b8  
 0002:000001bc       __imp__GlobalHandle@4      5f8991bc  
 0002:000001c0       __imp__TlsFree@4           5f8991c0  
 0002:000001c4       __imp__LeaveCriticalSection@4 5f8991c4  
 0002:000001c8       __imp__EnterCriticalSection@4 5f8991c8  
 0002:000001cc       __imp__TlsSetValue@8       5f8991cc  
 0002:000001d0       __imp__LocalReAlloc@12     5f8991d0  
 0002:000001d4       __imp__TlsGetValue@4       5f8991d4  
 0002:000001d8       __imp__WaitForSingleObject@8 5f8991d8  
 0002:000001dc       __imp__CreateSemaphoreW@16 5f8991dc  
 0002:000001e0       __imp__ReleaseSemaphore@12 5f8991e0  
 0002:000001e4       __imp__CreateMutexW@12     5f8991e4  
 0002:000001e8       __imp__ReleaseMutex@4      5f8991e8  
 0002:000001ec       __imp__CreateEventW@16     5f8991ec  
 0002:000001f0       __imp__WaitForMultipleObjects@16 5f8991f0  
 0002:000001f4       __imp__FindFirstFileW@8    5f8991f4  
 0002:000001f8       __imp__GetFullPathNameW@16 5f8991f8  
 0002:000001fc       __imp__GlobalFindAtomW@4   5f8991fc  
 0002:00000200       __imp__InterlockedExchange@8 5f899200  
 0002:00000204       __imp__GetCurrentThreadId@0 5f899204  
 0002:00000208       __imp__lstrcatW@8          5f899208  
 0002:0000020c       __imp__GetVersion@0        5f89920c  
 0002:00000210       __imp__LockResource@4      5f899210  
 0002:00000214       __imp__LoadResource@8      5f899214  
 0002:00000218       __imp__FindResourceW@12    5f899218  
 0002:0000021c       __imp__FreeLibrary@4       5f89921c  
 0002:00000220       __imp__LoadLibraryA@4      5f899220  
 0002:00000224       __imp__GlobalGetAtomNameW@12 5f899224  
 0002:00000228       __imp__GetModuleHandleA@4  5f899228  
 0002:0000022c       __imp__MulDiv@12           5f89922c  
 0002:00000230       __imp__GetProfileIntW@12   5f899230  
 0002:00000234       __imp__VirtualProtect@16   5f899234  
 0002:00000238       __imp__lstrcpyA@8          5f899238  
 0002:0000023c       __imp__SizeofResource@8    5f89923c  
 0002:00000240       __imp__GetProcessVersion@4 5f899240  
 0002:00000244       __imp__lstrcmpW@8          5f899244  
 0002:00000248       __imp__GlobalFlags@4       5f899248  
 0002:0000024c       __imp__GetTempFileNameW@16 5f89924c  
 0002:00000250       __imp__GetDiskFreeSpaceW@20 5f899250  
 0002:00000254       __imp__LocalUnlock@4       5f899254  
 0002:00000258       __imp__LocalLock@4         5f899258  
 0002:0000025c       __imp__GetTempPathW@8      5f89925c  
 0002:00000260       __imp__SearchPathW@24      5f899260  
 0002:00000264       __imp__SetEvent@4          5f899264  
 0002:00000268       __imp__ResumeThread@4      5f899268  
 0002:0000026c       __imp__SetThreadPriority@8 5f89926c  
 0002:00000270       __imp__SuspendThread@4     5f899270  
 0002:00000274       __imp__GetCurrentThread@0  5f899274  
 0002:00000278       __imp__lstrcmpiA@8         5f899278  
 0002:0000027c       __imp__SetErrorMode@4      5f89927c  
 0002:00000280       __imp__GetPrivateProfileIntW@16 5f899280  
 0002:00000284       __imp__GetPrivateProfileStringW@24 5f899284  
 0002:00000288       __imp__WritePrivateProfileStringW@16 5f899288  
 0002:0000028c       __imp__GetCurrentDirectoryW@8 5f89928c  
 0002:00000290       __imp__FindNextFileW@8     5f899290  
 0002:00000294       __imp__GetTickCount@0      5f899294  
 0002:00000298       __imp__CopyFileW@12        5f899298  
 0002:0000029c       __imp__GetUserDefaultLCID@0 5f89929c  
 0002:000002a0       __imp__IsDBCSLeadByte@4    5f8992a0  
 0002:000002a4       __imp__lstrcatA@8          5f8992a4  
 0002:000002a8       __imp__GetSystemDirectoryA@8 5f8992a8  
 0002:000002ac       __imp__GetVolumeInformationW@32 5f8992ac  
 0002:000002b0       __imp__LoadLibraryW@4      5f8992b0  
 0002:000002b4       __imp__FindClose@4         5f8992b4  
 0002:000002b8       __imp__lstrcpyW@8          5f8992b8  
 0002:000002bc       __imp__MoveFileW@8         5f8992bc  
 0002:000002c0       __imp__GetProcAddress@8    5f8992c0  
 0002:000002c4       __imp__DeleteFileW@4       5f8992c4  
 0002:000002c8       __imp__LockFile@20         5f8992c8  
 0002:000002cc       __imp__SetEndOfFile@4      5f8992cc  
 0002:000002d0       __imp__UnlockFile@20       5f8992d0  
 0002:000002d4       __imp__SetFilePointer@16   5f8992d4  
 0002:000002d8       __imp__CloseHandle@4       5f8992d8  
 0002:000002dc       __imp__FlushFileBuffers@4  5f8992dc  
 0002:000002e0       __imp__CreateFileW@28      5f8992e0  
 0002:000002e4       __imp__WriteFile@20        5f8992e4  
 0002:000002e8       __imp__ReadFile@20         5f8992e8  
 0002:000002ec       __imp__lstrlenA@4          5f8992ec  
 0002:000002f0       __imp__GetCurrentProcess@0 5f8992f0  
 0002:000002f4       __imp__DuplicateHandle@28  5f8992f4  
 0002:000002f8       __imp__lstrlenW@4          5f8992f8  
 0002:000002fc       __imp__lstrcmpA@8          5f8992fc  
 0002:00000300       __imp__OutputDebugStringW@4 5f899300  
 0002:00000304       __imp__IsBadStringPtrA@8   5f899304  
 0002:00000308       __imp__IsBadReadPtr@8      5f899308  
 0002:0000030c       __imp__IsBadWritePtr@8     5f89930c  
 0002:00000310       __imp__GetLastError@0      5f899310  
 0002:00000314       __imp__IsBadStringPtrW@8   5f899314  
 0002:00000318       __imp__lstrcpynW@12        5f899318  
 0002:0000031c       __imp__GetModuleHandleW@4  5f89931c  
 0002:00000320       __imp__SetLastError@4      5f899320  
 0002:00000324       __imp__GlobalDeleteAtom@4  5f899324  
 0002:00000328       __imp__GlobalSize@4        5f899328  
 0002:0000032c       __imp__GlobalAddAtomW@4    5f89932c  
 0002:00000330       __imp__RaiseException@16   5f899330  
 0002:00000338       __imp__CreatePen@12        5f899338  
 0002:0000033c       __imp__GetTextFaceW@12     5f89933c  
 0002:00000340       __imp__EnumFontFamiliesW@16 5f899340  
 0002:00000344       __imp__GetPixel@12         5f899344  
 0002:00000348       __imp__CreatePalette@4     5f899348  
 0002:0000034c       __imp__GetPaletteEntries@16 5f89934c  
 0002:00000350       __imp__RealizePalette@4    5f899350  
 0002:00000354       __imp__OffsetRgn@12        5f899354  
 0002:00000358       __imp__SetBrushOrgEx@16    5f899358  
 0002:0000035c       __imp__CreateMetaFileW@4   5f89935c  
 0002:00000360       __imp__CopyMetaFileW@8     5f899360  
 0002:00000364       __imp__LPtoDP@12           5f899364  
 0002:00000368       __imp__SetAbortProc@8      5f899368  
 0002:0000036c       __imp__StartPage@4         5f89936c  
 0002:00000370       __imp__EndPage@4           5f899370  
 0002:00000374       __imp__EndDoc@4            5f899374  
 0002:00000378       __imp__AbortDoc@4          5f899378  
 0002:0000037c       __imp__DPtoLP@12           5f89937c  
 0002:00000380       __imp__CombineRgn@16       5f899380  
 0002:00000384       __imp__SetRectRgn@20       5f899384  
 0002:00000388       __imp__GetMapMode@4        5f899388  
 0002:0000038c       __imp__CreateDIBPatternBrushPt@8 5f89938c  
 0002:00000390       __imp__CreateHatchBrush@8  5f899390  
 0002:00000394       __imp__ExtCreatePen@20     5f899394  
 0002:00000398       __imp__PlayMetaFile@8      5f899398  
 0002:0000039c       __imp__EnumMetaFile@16     5f89939c  
 0002:000003a0       __imp__GetObjectType@4     5f8993a0  
 0002:000003a4       __imp__PlayMetaFileRecord@16 5f8993a4  
 0002:000003a8       __imp__ExtSelectClipRgn@12 5f8993a8  
 0002:000003ac       __imp__SelectClipPath@8    5f8993ac  
 0002:000003b0       __imp__CreateRectRgn@16    5f8993b0  
 0002:000003b4       __imp__GetClipRgn@8        5f8993b4  
 0002:000003b8       __imp__PolyBezierTo@12     5f8993b8  
 0002:000003bc       __imp__SetColorAdjustment@8 5f8993bc  
 0002:000003c0       __imp__PolylineTo@12       5f8993c0  
 0002:000003c4       __imp__PolyDraw@16         5f8993c4  
 0002:000003c8       __imp__SetArcDirection@8   5f8993c8  
 0002:000003cc       __imp__ArcTo@36            5f8993cc  
 0002:000003d0       __imp__SetMapperFlags@8    5f8993d0  
 0002:000003d4       __imp__SetTextCharacterExtra@8 5f8993d4  
 0002:000003d8       __imp__SetTextJustification@12 5f8993d8  
 0002:000003dc       __imp__SetTextAlign@8      5f8993dc  
 0002:000003e0       __imp__LineTo@12           5f8993e0  
 0002:000003e4       __imp__OffsetClipRgn@12    5f8993e4  
 0002:000003e8       __imp__ExcludeClipRect@20  5f8993e8  
 0002:000003ec       __imp__SelectClipRgn@8     5f8993ec  
 0002:000003f0       __imp__OffsetWindowOrgEx@16 5f8993f0  
 0002:000003f4       __imp__SetStretchBltMode@8 5f8993f4  
 0002:000003f8       __imp__SetROP2@8           5f8993f8  
 0002:000003fc       __imp__SetPolyFillMode@8   5f8993fc  
 0002:00000400       __imp__SetBkMode@8         5f899400  
 0002:00000404       __imp__SelectPalette@12    5f899404  
 0002:00000408       __imp__StartDocW@8         5f899408  
 0002:0000040c       __imp__CreateDCW@16        5f89940c  
 0002:00000410       __imp__CreateRectRgnIndirect@4 5f899410  
 0002:00000414       __imp__Rectangle@20        5f899414  
 0002:00000418       __imp__UnrealizeObject@4   5f899418  
 0002:0000041c       __imp__PatBlt@24           5f89941c  
 0002:00000420       __imp__CreateBitmap@20     5f899420  
 0002:00000424       __imp__CreatePatternBrush@4 5f899424  
 0002:00000428       __imp__TextOutW@20         5f899428  
 0002:0000042c       __imp__CloseMetaFile@4     5f89942c  
 0002:00000430       __imp__DeleteMetaFile@4    5f899430  
 0002:00000434       __imp__RectVisible@8       5f899434  
 0002:00000438       __imp__PtVisible@12        5f899438  
 0002:0000043c       __imp__IntersectClipRect@20 5f89943c  
 0002:00000440       __imp__GetViewportOrgEx@8  5f899440  
 0002:00000444       __imp__GetWindowOrgEx@8    5f899444  
 0002:00000448       __imp__SetWindowOrgEx@16   5f899448  
 0002:0000044c       __imp__GetDeviceCaps@8     5f89944c  
 0002:00000450       __imp__Escape@20           5f899450  
 0002:00000454       __imp__GetTextExtentPoint32A@16 5f899454  
 0002:00000458       __imp__GetCurrentPositionEx@8 5f899458  
 0002:0000045c       __imp__MoveToEx@16         5f89945c  
 0002:00000460       __imp__ScaleWindowExtEx@24 5f899460  
 0002:00000464       __imp__SetWindowExtEx@16   5f899464  
 0002:00000468       __imp__ScaleViewportExtEx@24 5f899468  
 0002:0000046c       __imp__SetViewportExtEx@16 5f89946c  
 0002:00000470       __imp__OffsetViewportOrgEx@16 5f899470  
 0002:00000474       __imp__SetViewportOrgEx@16 5f899474  
 0002:00000478       __imp__SetMapMode@8        5f899478  
 0002:0000047c       __imp__GetROP2@4           5f89947c  
 0002:00000480       __imp__GetBkMode@4         5f899480  
 0002:00000484       __imp__GetViewportExtEx@8  5f899484  
 0002:00000488       __imp__GetPolyFillMode@4   5f899488  
 0002:0000048c       __imp__GetStretchBltMode@4 5f89948c  
 0002:00000490       __imp__GetTextAlign@4      5f899490  
 0002:00000494       __imp__GetNearestColor@8   5f899494  
 0002:00000498       __imp__GetBkColor@4        5f899498  
 0002:0000049c       __imp__GetTextColor@4      5f89949c  
 0002:000004a0       __imp__SaveDC@4            5f8994a0  
 0002:000004a4       __imp__GetStockObject@4    5f8994a4  
 0002:000004a8       __imp__RestoreDC@8         5f8994a8  
 0002:000004ac       __imp__GetCharWidthW@16    5f8994ac  
 0002:000004b0       __imp__DeleteObject@4      5f8994b0  
 0002:000004b4       __imp__CreateFontW@56      5f8994b4  
 0002:000004b8       __imp__StretchDIBits@52    5f8994b8  
 0002:000004bc       __imp__DeleteDC@4          5f8994bc  
 0002:000004c0       __imp__CreateCompatibleBitmap@12 5f8994c0  
 0002:000004c4       __imp__GetTextExtentPoint32W@16 5f8994c4  
 0002:000004c8       __imp__ExtTextOutW@32      5f8994c8  
 0002:000004cc       __imp__CreateSolidBrush@4  5f8994cc  
 0002:000004d0       __imp__BitBlt@36           5f8994d0  
 0002:000004d4       __imp__CreateFontIndirectW@4 5f8994d4  
 0002:000004d8       __imp__CreateCompatibleDC@4 5f8994d8  
 0002:000004dc       __imp__GetTextMetricsW@8   5f8994dc  
 0002:000004e0       __imp__GetObjectW@12       5f8994e0  
 0002:000004e4       __imp__SelectObject@8      5f8994e4  
 0002:000004e8       __imp__SetTextColor@8      5f8994e8  
 0002:000004ec       __imp__GetClipBox@8        5f8994ec  
 0002:000004f0       __imp__SetBkColor@8        5f8994f0  
 0002:000004f4       __imp__GetWindowExtEx@8    5f8994f4  
 0002:000004fc       __imp__GetCursorPos@4      5f8994fc  
 0002:00000500       __imp__UnhookWindowsHookEx@4 5f899500  
 0002:00000504       __imp__MsgWaitForMultipleObjects@20 5f899504  
 0002:00000508       __imp__GetWindowRect@8     5f899508  
 0002:0000050c       __imp__GetWindowPlacement@8 5f89950c  
 0002:00000510       __imp__IsIconic@4          5f899510  
 0002:00000514       __imp__SystemParametersInfoW@16 5f899514  
 0002:00000518       __imp__IntersectRect@12    5f899518  
 0002:0000051c       __imp__OffsetRect@12       5f89951c  
 0002:00000520       __imp__RegisterWindowMessageW@4 5f899520  
 0002:00000524       __imp__SetWindowPos@28     5f899524  
 0002:00000528       __imp__SetWindowLongW@12   5f899528  
 0002:0000052c       __imp__GetWindowLongW@8    5f89952c  
 0002:00000530       __imp__GetWindow@8         5f899530  
 0002:00000534       __imp__SendMessageW@16     5f899534  
 0002:00000538       __imp__SetForegroundWindow@4 5f899538  
 0002:0000053c       __imp__GetForegroundWindow@0 5f89953c  
 0002:00000540       __imp__GetLastActivePopup@4 5f899540  
 0002:00000544       __imp__GetMessagePos@0     5f899544  
 0002:00000548       __imp__GetMessageTime@0    5f899548  
 0002:0000054c       __imp__RemovePropW@8       5f89954c  
 0002:00000550       __imp__CallWindowProcW@20  5f899550  
 0002:00000554       __imp__GetPropW@8          5f899554  
 0002:00000558       __imp__SetPropW@12         5f899558  
 0002:0000055c       __imp__CallNextHookEx@16   5f89955c  
 0002:00000560       __imp__SetWindowsHookExW@16 5f899560  
 0002:00000564       __imp__CreateWindowExW@48  5f899564  
 0002:00000568       __imp__DestroyWindow@4     5f899568  
 0002:0000056c       __imp__DefWindowProcW@16   5f89956c  
 0002:00000570       __imp__GetKeyState@4       5f899570  
 0002:00000574       __imp__GetDlgCtrlID@4      5f899574  
 0002:00000578       __imp__GetWindowTextW@12   5f899578  
 0002:0000057c       __imp__GetWindowTextLengthW@4 5f89957c  
 0002:00000580       __imp__GetDlgItem@8        5f899580  
 0002:00000584       __imp__SetWindowPlacement@8 5f899584  
 0002:00000588       __imp__TrackPopupMenu@28   5f899588  
 0002:0000058c       __imp__GetMenuItemID@8     5f89958c  
 0002:00000590       __imp__GetSubMenu@8        5f899590  
 0002:00000594       __imp__GetMenuItemCount@4  5f899594  
 0002:00000598       __imp__GetMenu@4           5f899598  
 0002:0000059c       __imp__RegisterClassW@4    5f89959c  
 0002:000005a0       __imp__GetClassInfoW@12    5f8995a0  
 0002:000005a4       __imp__WinHelpW@16         5f8995a4  
 0002:000005a8       __imp__GetCapture@0        5f8995a8  
 0002:000005ac       __imp__GetParent@4         5f8995ac  
 0002:000005b0       __imp__IsChild@8           5f8995b0  
 0002:000005b4       __imp__MessageBoxW@16      5f8995b4  
 0002:000005b8       __imp__GetTopWindow@4      5f8995b8  
 0002:000005bc       __imp__SetScrollPos@16     5f8995bc  
 0002:000005c0       __imp__GetScrollPos@8      5f8995c0  
 0002:000005c4       __imp__SetScrollRange@20   5f8995c4  
 0002:000005c8       __imp__GetScrollRange@16   5f8995c8  
 0002:000005cc       __imp__ShowScrollBar@12    5f8995cc  
 0002:000005d0       __imp__SetScrollInfo@16    5f8995d0  
 0002:000005d4       __imp__GetScrollInfo@12    5f8995d4  
 0002:000005d8       __imp__ScrollWindow@20     5f8995d8  
 0002:000005dc       __imp__IsWindowVisible@4   5f8995dc  
 0002:000005e0       __imp__EnableWindow@8      5f8995e0  
 0002:000005e4       __imp__EndDeferWindowPos@4 5f8995e4  
 0002:000005e8       __imp__CopyRect@8          5f8995e8  
 0002:000005ec       __imp__BeginDeferWindowPos@4 5f8995ec  
 0002:000005f0       __imp__GetClientRect@8     5f8995f0  
 0002:000005f4       __imp__DeferWindowPos@32   5f8995f4  
 0002:000005f8       __imp__EqualRect@8         5f8995f8  
 0002:000005fc       __imp__ScreenToClient@8    5f8995fc  
 0002:00000600       __imp__AdjustWindowRectEx@16 5f899600  
 0002:00000604       __imp__SetFocus@4          5f899604  
 0002:00000608       __imp__IsWindow@4          5f899608  
 0002:0000060c       __imp__SetActiveWindow@4   5f89960c  
 0002:00000610       __imp__GetFocus@0          5f899610  
 0002:00000614       __imp__DispatchMessageW@4  5f899614  
 0002:00000618       __imp__PeekMessageW@20     5f899618  
 0002:0000061c       __imp__GetSysColor@4       5f89961c  
 0002:00000620       __imp__MapWindowPoints@16  5f899620  
 0002:00000624       __imp__SendDlgItemMessageA@20 5f899624  
 0002:00000628       __imp__SendDlgItemMessageW@20 5f899628  
 0002:0000062c       __imp__UpdateWindow@4      5f89962c  
 0002:00000630       __imp__PostMessageW@16     5f899630  
 0002:00000634       __imp__LoadIconW@8         5f899634  
 0002:00000638       __imp__SetRectEmpty@4      5f899638  
 0002:0000063c       __imp__LoadAcceleratorsW@8 5f89963c  
 0002:00000640       __imp__TranslateAcceleratorW@12 5f899640  
 0002:00000644       __imp__ReleaseCapture@0    5f899644  
 0002:00000648       __imp__SetCursor@4         5f899648  
 0002:0000064c       __imp__IsWindowEnabled@4   5f89964c  
 0002:00000650       __imp__GetDesktopWindow@0  5f899650  
 0002:00000654       __imp__ShowWindow@8        5f899654  
 0002:00000658       __imp__GetActiveWindow@0   5f899658  
 0002:0000065c       __imp__DestroyMenu@4       5f89965c  
 0002:00000660       __imp__LoadMenuW@8         5f899660  
 0002:00000664       __imp__SetMenu@8           5f899664  
 0002:00000668       __imp__ReuseDDElParam@20   5f899668  
 0002:0000066c       __imp__UnpackDDElParam@16  5f89966c  
 0002:00000670       __imp__InvalidateRect@12   5f899670  
 0002:00000674       __imp__BringWindowToTop@4  5f899674  
 0002:00000678       __imp__LoadCursorW@8       5f899678  
 0002:0000067c       __imp__SetCapture@4        5f89967c  
 0002:00000680       __imp__WaitMessage@0       5f899680  
 0002:00000684       __imp__GetSystemMetrics@4  5f899684  
 0002:00000688       __imp__GetWindowThreadProcessId@8 5f899688  
 0002:0000068c       __imp__WindowFromPoint@8   5f89968c  
 0002:00000690       __imp__ClientToScreen@8    5f899690  
 0002:00000694       __imp__TranslateMessage@4  5f899694  
 0002:00000698       __imp__GetMessageW@16      5f899698  
 0002:0000069c       __imp__DefFrameProcW@20    5f89969c  
 0002:000006a0       __imp__TranslateMDISysAccel@8 5f8996a0  
 0002:000006a4       __imp__DrawMenuBar@4       5f8996a4  
 0002:000006a8       __imp__DefMDIChildProcW@16 5f8996a8  
 0002:000006ac       __imp__RedrawWindow@16     5f8996ac  
 0002:000006b0       __imp__LoadBitmapW@8       5f8996b0  
 0002:000006b4       __imp__InflateRect@12      5f8996b4  
 0002:000006b8       __imp__PtInRect@12         5f8996b8  
 0002:000006bc       __imp__ReleaseDC@8         5f8996bc  
 0002:000006c0       __imp__InvertRect@8        5f8996c0  
 0002:000006c4       __imp__GetWindowDC@4       5f8996c4  
 0002:000006c8       __imp__FillRect@12         5f8996c8  
 0002:000006cc       __imp__SetTimer@16         5f8996cc  
 0002:000006d0       __imp__KillTimer@8         5f8996d0  
 0002:000006d4       __imp__SetRect@20          5f8996d4  
 0002:000006d8       __imp__GetDC@4             5f8996d8  
 0002:000006dc       __imp__IsZoomed@4          5f8996dc  
 0002:000006e0       __imp__SetParent@8         5f8996e0  
 0002:000006e4       __imp__IsRectEmpty@4       5f8996e4  
 0002:000006e8       __imp__AppendMenuW@16      5f8996e8  
 0002:000006ec       __imp__DeleteMenu@12       5f8996ec  
 0002:000006f0       __imp__GetSystemMenu@8     5f8996f0  
 0002:000006f4       __imp__GetDCEx@12          5f8996f4  
 0002:000006f8       __imp__LockWindowUpdate@4  5f8996f8  
 0002:000006fc       __imp__GetTabbedTextExtentA@20 5f8996fc  
 0002:00000700       __imp__DrawTextW@20        5f899700  
 0002:00000704       __imp__GrayStringW@36      5f899704  
 0002:00000708       __imp__UnionRect@12        5f899708  
 0002:0000070c       __imp__DrawFocusRect@8     5f89970c  
 0002:00000710       __imp__CreateDialogIndirectParamW@20 5f899710  
 0002:00000714       __imp__EndDialog@8         5f899714  
 0002:00000718       __imp__GetNextDlgTabItem@12 5f899718  
 0002:0000071c       __imp__wvsprintfW@12       5f89971c  
 0002:00000720       __imp__GetAsyncKeyState@4  5f899720  
 0002:00000724       __imp__MapDialogRect@8     5f899724  
 0002:00000728       __imp__GetDialogBaseUnits@0 5f899728  
 0002:0000072c       __imp__BeginPaint@8        5f89972c  
 0002:00000730       __imp__EndPaint@8          5f899730  
 0002:00000734       __imp__TabbedTextOutW@32   5f899734  
 0002:00000738       __imp__GetSysColorBrush@4  5f899738  
 0002:0000073c       __imp__GetClassNameW@12    5f89973c  
 0002:00000740       __imp__SetWindowTextW@8    5f899740  
 0002:00000744       __imp__CheckDlgButton@12   5f899744  
 0002:00000748       __imp__CheckRadioButton@16 5f899748  
 0002:0000074c       __imp__GetDlgItemInt@16    5f89974c  
 0002:00000750       __imp__GetDlgItemTextW@16  5f899750  
 0002:00000754       __imp__SetDlgItemInt@16    5f899754  
 0002:00000758       __imp__SetDlgItemTextW@12  5f899758  
 0002:0000075c       __imp__IsDlgButtonChecked@8 5f89975c  
 0002:00000760       __imp__ScrollWindowEx@32   5f899760  
 0002:00000764       __imp__IsDialogMessageW@8  5f899764  
 0002:00000768       __imp__MoveWindow@24       5f899768  
 0002:0000076c       __imp__EnableMenuItem@12   5f89976c  
 0002:00000770       __imp__CheckMenuItem@12    5f899770  
 0002:00000774       __imp__SetMenuItemBitmaps@20 5f899774  
 0002:00000778       __imp__ModifyMenuW@20      5f899778  
 0002:0000077c       __imp__GetMenuState@12     5f89977c  
 0002:00000780       __imp__GetMenuCheckMarkDimensions@0 5f899780  
 0002:00000784       __imp__DestroyIcon@4       5f899784  
 0002:00000788       __imp__SetCursorPos@8      5f899788  
 0002:0000078c       __imp__DestroyCursor@4     5f89978c  
 0002:00000790       __imp__FindWindowW@8       5f899790  
 0002:00000794       __imp__GetTabbedTextExtentW@20 5f899794  
 0002:00000798       __imp__IsClipboardFormatAvailable@4 5f899798  
 0002:0000079c       __imp__MessageBeep@4       5f89979c  
 0002:000007a0       __imp__RemoveMenu@12       5f8997a0  
 0002:000007a4       __imp__ValidateRect@8      5f8997a4  
 0002:000007a8       __imp__PostQuitMessage@4   5f8997a8  
 0002:000007ac       __imp__UnregisterClassW@8  5f8997ac  
 0002:000007b0       __imp__ShowOwnedPopups@8   5f8997b0  
 0002:000007b4       __imp__InsertMenuW@20      5f8997b4  
 0002:000007b8       __imp__GetMenuStringW@20   5f8997b8  
 0002:000007bc       __imp__RegisterClipboardFormatW@4 5f8997bc  
 0002:000007c0       __imp__CopyAcceleratorTableW@12 5f8997c0  
 0002:000007c4       __imp__InSendMessage@0     5f8997c4  
 0002:000007c8       __imp__PostThreadMessageW@16 5f8997c8  
 0002:000007cc       __imp__CreateMenu@0        5f8997cc  
 0002:000007d0       __imp__WindowFromDC@4      5f8997d0  
 0002:000007d4       __imp__CountClipboardFormats@0 5f8997d4  
 0002:000007d8       __imp__SetWindowContextHelpId@8 5f8997d8  
 0002:000007dc       __imp__CharNextW@4         5f8997dc  
 0002:000007e0       __imp__GetNextDlgGroupItem@12 5f8997e0  
 0002:000007e4       __imp__ClipCursor@4        5f8997e4  
 0002:000007e8       __imp__DrawEdge@16         5f8997e8  
 0002:000007ec       __imp__EnumChildWindows@12 5f8997ec  
 0002:000007f0       __imp__InvalidateRgn@12    5f8997f0  
 0002:000007f4       __imp__FrameRect@12        5f8997f4  
 0002:000007f8       __imp__LoadStringW@16      5f8997f8  
 0002:000007fc       __imp__MessageBoxA@16      5f8997fc  
 0002:00000800       __imp__CharUpperW@4        5f899800  
 0002:00000804       __imp__wsprintfW           5f899804  
 0002:00000810       ?classCTempWnd@CTempWnd@@2UCRuntimeClass@@B 5f899810  
 0002:00000828       ??_C@_08EHJM@CTempWnd?$AA@ 5f899828  
 0002:00000838       ??_7type_info@@6B@         5f899838  
 0002:00000840       ??_R1A@?0A@A@type_info@@8  5f899840  
 0002:00000858       ??_R2type_info@@8          5f899858  
 0002:00000860       ??_R3type_info@@8          5f899860  
 0002:00000870       ??_R4type_info@@6B@        5f899870  
 0002:00000888       ??_R1A@?0A@A@CObject@@8    5f899888  
 0002:000008a4       ??_7CObject@@6B@           5f8998a4  
 0002:000008b8       ??_R2CObject@@8            5f8998b8  
 0002:000008c0       ??_R3CObject@@8            5f8998c0  
 0002:000008d0       ??_R4CObject@@6B@          5f8998d0  
 0002:000008e8       ??_7CWnd@@6B@              5f8998e8  
 0002:000009a8       ??_R1A@?0A@A@CCmdTarget@@8 5f8999a8  
 0002:000009c0       ??_R1A@?0A@A@CWnd@@8       5f8999c0  
 0002:000009d8       ??_R2CWnd@@8               5f8999d8  
 0002:000009e8       ??_R3CWnd@@8               5f8999e8  
 0002:000009f8       ??_R4CWnd@@6B@             5f8999f8  
 0002:00000a10       ??_7CCmdTarget@@6B@        5f899a10  
 0002:00000a68       ??_R2CCmdTarget@@8         5f899a68  
 0002:00000a78       ??_R3CCmdTarget@@8         5f899a78  
 0002:00000a88       ??_R4CCmdTarget@@6B@       5f899a88  
 0002:00000aa0       ?messageMap@CWnd@@1UAFX_MSGMAP@@B 5f899aa0  
 0002:00000aa8       ?_messageEntries@CWnd@@0QBUAFX_MSGMAP_ENTRY@@B 5f899aa8  
 0002:00000d48       ?messageMap@CCmdTarget@@1UAFX_MSGMAP@@B 5f899d48  
 0002:00000d50       ?_messageEntries@CCmdTarget@@0QBUAFX_MSGMAP_ENTRY@@B 5f899d50  
 0002:00000d68       ??_R1A@?0A@A@CCmdUI@@8     5f899d68  
 0002:00000d84       ??_7CCmdUI@@6B@            5f899d84  
 0002:00000d94       ??_R2CCmdUI@@8             5f899d94  
 0002:00000da0       ??_R3CCmdUI@@8             5f899da0  
 0002:00000db0       ??_R4CCmdUI@@6B@           5f899db0  
 0002:00000dc8       ?messageMap@CStatusBar@@1UAFX_MSGMAP@@B 5f899dc8  
 0002:00000dd0       ?_messageEntries@CStatusBar@@0QBUAFX_MSGMAP_ENTRY@@B 5f899dd0  
 0002:00000ed8       ?messageMap@CView@@1UAFX_MSGMAP@@B 5f899ed8  
 0002:00000ee0       ?_messageEntries@CView@@0QBUAFX_MSGMAP_ENTRY@@B 5f899ee0  
 0002:00001000       ?classCCmdTarget@CCmdTarget@@2UCRuntimeClass@@B 5f89a000  
 0002:00001018       ??_C@_0L@MION@CCmdTarget?$AA@ 5f89a018  
 0002:00001028       ?messageMap@CDocument@@1UAFX_MSGMAP@@B 5f89a028  
 0002:00001030       ?_messageEntries@CDocument@@0QBUAFX_MSGMAP_ENTRY@@B 5f89a030  
 0002:00001090       ?classCOleObjectFactory@COleObjectFactory@@2UCRuntimeClass@@B 5f89a090  
 0002:000010a8       ??_C@_0BC@HKPN@COleObjectFactory?$AA@ 5f89a0a8  
 0002:000010c0       ?messageMap@CToolBar@@1UAFX_MSGMAP@@B 5f89a0c0  
 0002:000010c8       ?_messageEntries@CToolBar@@0QBUAFX_MSGMAP_ENTRY@@B 5f89a0c8  
 0002:00001200       ?messageMap@CControlBar@@1UAFX_MSGMAP@@B 5f89a200  
 0002:00001208       ?_messageEntries@CControlBar@@0QBUAFX_MSGMAP_ENTRY@@B 5f89a208  
 0002:000013b8       ?messageMap@CDockBar@@1UAFX_MSGMAP@@B 5f89a3b8  
 0002:000013c0       ?_messageEntries@CDockBar@@0QBUAFX_MSGMAP_ENTRY@@B 5f89a3c0  
 0002:00001454       ??_7CStatusCmdUI@@6B@      5f89a454  
 0002:00001468       ??_R1A@?0A@A@CStatusCmdUI@@8 5f89a468  
 0002:00001480       ??_R2CStatusCmdUI@@8       5f89a480  
 0002:00001490       ??_R3CStatusCmdUI@@8       5f89a490  
 0002:000014a0       ??_R4CStatusCmdUI@@6B@     5f89a4a0  
 0002:000014b8       ??_7CToolCmdUI@@6B@        5f89a4b8  
 0002:000014c8       ??_R1A@?0A@A@CToolCmdUI@@8 5f89a4c8  
 0002:000014e0       ??_R2CToolCmdUI@@8         5f89a4e0  
 0002:000014f0       ??_R3CToolCmdUI@@8         5f89a4f0  
 0002:00001500       ??_R4CToolCmdUI@@6B@       5f89a500  
 0002:00001518       ?classCSplitterWnd@CSplitterWnd@@2UCRuntimeClass@@B 5f89a518  
 0002:00001530       ??_C@_0N@JGP@CSplitterWnd?$AA@ 5f89a530  
 0002:00001540       ?classCWnd@CWnd@@2UCRuntimeClass@@B 5f89a540  
 0002:00001558       ??_C@_04MBPC@CWnd?$AA@     5f89a558  
 0002:00001560       ?classCObject@CObject@@2UCRuntimeClass@@B 5f89a560  
 0002:00001578       ??_C@_07EFMO@CObject?$AA@  5f89a578  
 0002:00001580       ?messageMap@CCtrlView@@1UAFX_MSGMAP@@B 5f89a580  
 0002:00001588       ?_messageEntries@CCtrlView@@0QBUAFX_MSGMAP_ENTRY@@B 5f89a588  
 0002:000015b8       ?_pfnUninitialized@@3Q6AHI@ZA 5f89a5b8  
 0002:000015bc       ?_afxOldWndProc@@3QBGB     5f89a5bc  
 0002:000015e4       ??_7CTempWnd@@6B@          5f89a5e4  
 0002:000016a8       ??_R1A@?0A@A@CTempWnd@@8   5f89a6a8  
 0002:000016c0       ??_R2CTempWnd@@8           5f89a6c0  
 0002:000016d8       ??_R3CTempWnd@@8           5f89a6d8  
 0002:000016e8       ??_R4CTempWnd@@6B@         5f89a6e8  
 0002:00001700       ??_R1A@?0A@A@CMenu@@8      5f89a700  
 0002:0000171c       ??_7CMenu@@6B@             5f89a71c  
 0002:00001738       ??_R2CMenu@@8              5f89a738  
 0002:00001748       ??_R3CMenu@@8              5f89a748  
 0002:00001758       ??_R4CMenu@@6B@            5f89a758  
 0002:00001770       ?classCTempMenu@CTempMenu@@2UCRuntimeClass@@B 5f89a770  
 0002:00001788       ??_C@_09NDEG@CTempMenu?$AA@ 5f89a788  
 0002:00001798       ??_7CTempMenu@@6B@         5f89a798  
 0002:000017b8       ??_R1A@?0A@A@CTempMenu@@8  5f89a7b8  
 0002:000017d0       ??_R2CTempMenu@@8          5f89a7d0  
 0002:000017e0       ??_R3CTempMenu@@8          5f89a7e0  
 0002:000017f0       ??_R4CTempMenu@@6B@        5f89a7f0  
 0002:00001804       ??_C@_19ENHM@?$AA?$CG?$AA?$CF?$AAd?$AA?5?$AA?$AA@ 5f89a804  
 0002:00001814       ??_7CTestCmdUI@@6B@        5f89a814  
 0002:00001828       ??_R1A@?0A@A@CTestCmdUI@@8 5f89a828  
 0002:00001840       ??_R2CTestCmdUI@@8         5f89a840  
 0002:00001850       ??_R3CTestCmdUI@@8         5f89a850  
 0002:00001860       ??_R4CTestCmdUI@@6B@       5f89a860  
 0002:00001874       ??_C@_1BG@PFLE@?$AAM?$AAA?$AAP?$AAI?$AA3?$AA2?$AA?4?$AAD?$AAL?$AAL?$AA?$AA@ 5f89a874  
 0002:0000188c       ??_C@_19DFMB@?$AAM?$AAA?$AAI?$AAL?$AA?$AA@ 5f89a88c  
 0002:00001898       ??_C@_19IMNH@?$AAM?$AAA?$AAP?$AAI?$AA?$AA@ 5f89a898  
 0002:000018a8       ?classCOleServerItem@COleServerItem@@2UCRuntimeClass@@B 5f89a8a8  
 0002:000018c0       ??_C@_0P@ODMG@COleServerItem?$AA@ 5f89a8c0  
 0002:000018d4       ??_7CDC@@6B@               5f89a8d4  
 0002:00001950       ??_R1A@?0A@A@CDC@@8        5f89a950  
 0002:00001968       ??_R2CDC@@8                5f89a968  
 0002:00001978       ??_R3CDC@@8                5f89a978  
 0002:00001988       ??_R4CDC@@6B@              5f89a988  
 0002:000019a0       ?classCTempGdiObject@CTempGdiObject@@2UCRuntimeClass@@B 5f89a9a0  
 0002:000019b8       ??_C@_0P@LOPC@CTempGdiObject?$AA@ 5f89a9b8  
 0002:000019c8       ?classCTempDC@CTempDC@@2UCRuntimeClass@@B 5f89a9c8  
 0002:000019e0       ??_C@_07LHDN@CTempDC?$AA@  5f89a9e0  
 0002:000019e8       ??_R1A@?0A@A@CGdiObject@@8 5f89a9e8  
 0002:00001a04       ??_7_AFX_THREAD_STATE@@6B@ 5f89aa04  
 0002:00001a08       ??_R1A@?0A@A@CNoTrackObject@@8 5f89aa08  
 0002:00001a20       ??_R1A@?0A@A@_AFX_THREAD_STATE@@8 5f89aa20  
 0002:00001a38       ??_R2_AFX_THREAD_STATE@@8  5f89aa38  
 0002:00001a48       ??_R3_AFX_THREAD_STATE@@8  5f89aa48  
 0002:00001a58       ??_R4_AFX_THREAD_STATE@@6B@ 5f89aa58  
 0002:00001a70       ??_R1A@?0A@A@CMapPtrToPtr@@8 5f89aa70  
 0002:00001a8c       ??_7CMapPtrToPtr@@6B@      5f89aa8c  
 0002:00001aa0       ??_R2CMapPtrToPtr@@8       5f89aaa0  
 0002:00001ab0       ??_R3CMapPtrToPtr@@8       5f89aab0  
 0002:00001ac0       ??_R4CMapPtrToPtr@@6B@     5f89aac0  
 0002:00001ad8       ??_7AFX_MODULE_THREAD_STATE@@6B@ 5f89aad8  
 0002:00001ae0       ??_R1A@?0A@A@AFX_MODULE_THREAD_STATE@@8 5f89aae0  
 0002:00001af8       ??_R2AFX_MODULE_THREAD_STATE@@8 5f89aaf8  
 0002:00001b08       ??_R3AFX_MODULE_THREAD_STATE@@8 5f89ab08  
 0002:00001b18       ??_R4AFX_MODULE_THREAD_STATE@@6B@ 5f89ab18  
 0002:00001b30       ??_7CPtrList@@6B@          5f89ab30  
 0002:00001b48       ??_R1A@?0A@A@CPtrList@@8   5f89ab48  
 0002:00001b60       ??_R2CPtrList@@8           5f89ab60  
 0002:00001b70       ??_R3CPtrList@@8           5f89ab70  
 0002:00001b80       ??_R4CPtrList@@6B@         5f89ab80  
 0002:00001b94       ??_C@_0L@DPAJ@MSVCRT?4DLL?$AA@ 5f89ab94  
 0002:00001ba4       ??_7AFX_MODULE_STATE@@6B@  5f89aba4  
 0002:00001ba8       ??_R1A@?0A@A@AFX_MODULE_STATE@@8 5f89aba8  
 0002:00001bc0       ??_R2AFX_MODULE_STATE@@8   5f89abc0  
 0002:00001bd0       ??_R3AFX_MODULE_STATE@@8   5f89abd0  
 0002:00001be0       ??_R4AFX_MODULE_STATE@@6B@ 5f89abe0  
 0002:00001bf8       ??_7CThreadData@@6B@       5f89abf8  
 0002:00001c00       ??_R1A@?0A@A@CThreadData@@8 5f89ac00  
 0002:00001c18       ??_R2CThreadData@@8        5f89ac18  
 0002:00001c28       ??_R3CThreadData@@8        5f89ac28  
 0002:00001c38       ??_R4CThreadData@@6B@      5f89ac38  
 0002:00001c50       ??_R1A@?0A@A@CException@@8 5f89ac50  
 0002:00001c68       ??_R1A@?0A@A@CWinThread@@8 5f89ac68  
 0002:00001c84       ??_7CWinThread@@6B@        5f89ac84  
 0002:00001d08       ??_R2CWinThread@@8         5f89ad08  
 0002:00001d18       ??_R3CWinThread@@8         5f89ad18  
 0002:00001d28       ??_R4CWinThread@@6B@       5f89ad28  
 0002:00001d54       ??_7_AFX_CTL3D_THREAD@@6B@ 5f89ad54  
 0002:00001d58       ??_R1A@?0A@A@_AFX_CTL3D_THREAD@@8 5f89ad58  
 0002:00001d70       ??_R2_AFX_CTL3D_THREAD@@8  5f89ad70  
 0002:00001d80       ??_R3_AFX_CTL3D_THREAD@@8  5f89ad80  
 0002:00001d90       ??_R4_AFX_CTL3D_THREAD@@6B@ 5f89ad90  
 0002:00001da8       __sz_ole32                 5f89ada8  
 0002:00001dc0       __DELAY_IMPORT_DESCRIPTOR_OLEPRO32 5f89adc0  
 0002:00001de0       __DELAY_IMPORT_DESCRIPTOR_ADVAPI32 5f89ade0  
 0002:00001e00       __DELAY_IMPORT_DESCRIPTOR_ole32 5f89ae00  
 0002:00001e20       __DELAY_IMPORT_DESCRIPTOR_OLEAUT32 5f89ae20  
 0002:00001e40       __DELAY_IMPORT_DESCRIPTOR_COMCTL32 5f89ae40  
 0002:00001e60       __DELAY_IMPORT_DESCRIPTOR_SHELL32 5f89ae60  
 0002:00001e80       __DELAY_IMPORT_DESCRIPTOR_comdlg32 5f89ae80  
 0002:00001ea0       __DELAY_IMPORT_DESCRIPTOR_WINSPOOL 5f89aea0  
 0002:00001ec0       __DELAY_IMPORT_DESCRIPTOR_WININET 5f89aec0  
 0002:00001ee0       __DELAY_IMPORT_DESCRIPTOR_WSOCK32 5f89aee0  
 0002:00001f00       __DELAY_IMPORT_DESCRIPTOR_oledlg 5f89af00  
 0002:00001f20       __DELAY_IMPORT_DESCRIPTOR_urlmon 5f89af20  
 0002:00001f40       __DELAY_IMPORT_DESCRIPTOR_ODBC32 5f89af40  
 0002:00002418       _IID_IUnknown              5f89b418  
 0002:00002428       _IID_IDispatch             5f89b428  
 0002:00002438       ?interfaceMap@CCmdTarget@@1UAFX_INTERFACEMAP@@B 5f89b438  
 0002:00002440       ?_interfaceEntries@CCmdTarget@@0QBUAFX_INTERFACEMAP_ENTRY@@B 5f89b440  
 0002:00002450       ??_C@_11A@?$AA?$AA@        5f89b450  
 0002:00002458       ?classCOleClientItem@COleClientItem@@2UCRuntimeClass@@B 5f89b458  
 0002:00002470       ??_C@_0P@JNNP@COleClientItem?$AA@ 5f89b470  
 0002:00002480       ??_C@_17LFFB@?$AA?5?$AA?9?$AA?5?$AA?$AA@ 5f89b480  
 0002:00002488       ?interfaceMap@COleServerDoc@@1UAFX_INTERFACEMAP@@B 5f89b488  
 0002:00002490       ?_interfaceEntries@COleServerDoc@@0QBUAFX_INTERFACEMAP_ENTRY@@B 5f89b490  
 0002:000024c8       _IID_IOleWindow            5f89b4c8  
 0002:000024d8       _IID_IOleObject            5f89b4d8  
 0002:000024e8       _IID_IPersistStorage       5f89b4e8  
 0002:000024f8       _IID_IDataObject           5f89b4f8  
 0002:00002508       _IID_IOleInPlaceObject     5f89b508  
 0002:00002518       _IID_IOleInPlaceActiveObject 5f89b518  
 0002:00002528       ?interfaceMap@COleLinkingDoc@@1UAFX_INTERFACEMAP@@B 5f89b528  
 0002:00002530       ?_interfaceEntries@COleLinkingDoc@@0QBUAFX_INTERFACEMAP_ENTRY@@B 5f89b530  
 0002:00002560       _IID_IPersistFile          5f89b560  
 0002:00002570       _IID_IOleItemContainer     5f89b570  
 0002:00002580       _IID_IOleContainer         5f89b580  
 0002:00002590       _IID_IParseDisplayName     5f89b590  
 0002:000025a0       _IID_IPersist              5f89b5a0  
 0002:000025b0       ??_R1A@?0A@A@CFile@@8      5f89b5b0  
 0002:000025cc       ??_7CFile@@6B@             5f89b5cc  
 0002:00002628       ??_R2CFile@@8              5f89b628  
 0002:00002638       ??_R3CFile@@8              5f89b638  
 0002:00002648       ??_R4CFile@@6B@            5f89b648  
 0002:00002660       ?classCRichEditView@CRichEditView@@2UCRuntimeClass@@B 5f89b660  
 0002:00002678       ??_C@_0O@OMMG@CRichEditView?$AA@ 5f89b678  
 0002:0000268c       ??_7CSessionMapPtrToPtr@@6B@ 5f89b68c  
 0002:000026a4       ??_7CCriticalSection@@6B@  5f89b6a4  
 0002:000026c8       ??_R1A@?0A@A@CSyncObject@@8 5f89b6c8  
 0002:000026e0       ??_R1A@?0A@A@CSessionMapPtrToPtr@@8 5f89b6e0  
 0002:000026f8       ??_R2CSessionMapPtrToPtr@@8 5f89b6f8  
 0002:00002708       ??_R3CSessionMapPtrToPtr@@8 5f89b708  
 0002:00002718       ??_R4CSessionMapPtrToPtr@@6B@ 5f89b718  
 0002:00002730       ??_R1A@?0A@A@CCriticalSection@@8 5f89b730  
 0002:00002748       ??_R2CCriticalSection@@8   5f89b748  
 0002:00002758       ??_R3CCriticalSection@@8   5f89b758  
 0002:00002768       ??_R4CCriticalSection@@6B@ 5f89b768  
 0002:00002780       ??_7CSyncObject@@6B@       5f89b780  
 0002:000027a0       ??_R2CSyncObject@@8        5f89b7a0  
 0002:000027b0       ??_R3CSyncObject@@8        5f89b7b0  
 0002:000027c0       ??_R4CSyncObject@@6B@      5f89b7c0  
 0002:000027d8       ??_7CMemoryException@@6B@  5f89b7d8  
 0002:000027f8       ??_R1A@?0A@A@CSimpleException@@8 5f89b7f8  
 0002:00002810       ??_R1A@?0A@A@CMemoryException@@8 5f89b810  
 0002:00002828       ??_R2CMemoryException@@8   5f89b828  
 0002:00002840       ??_R3CMemoryException@@8   5f89b840  
 0002:00002850       ??_R4CMemoryException@@6B@ 5f89b850  
 0002:00002868       ??_7CNotSupportedException@@6B@ 5f89b868  
 0002:00002888       ??_R1A@?0A@A@CNotSupportedException@@8 5f89b888  
 0002:000028a0       ??_R2CNotSupportedException@@8 5f89b8a0  
 0002:000028b8       ??_R3CNotSupportedException@@8 5f89b8b8  
 0002:000028c8       ??_R4CNotSupportedException@@6B@ 5f89b8c8  
 0002:000028e0       ??_7CResourceException@@6B@ 5f89b8e0  
 0002:00002900       ??_R1A@?0A@A@CResourceException@@8 5f89b900  
 0002:00002918       ??_R2CResourceException@@8 5f89b918  
 0002:00002930       ??_R3CResourceException@@8 5f89b930  
 0002:00002940       ??_R4CResourceException@@6B@ 5f89b940  
 0002:00002958       ??_7CUserException@@6B@    5f89b958  
 0002:00002978       ??_R1A@?0A@A@CUserException@@8 5f89b978  
 0002:00002990       ??_R2CUserException@@8     5f89b990  
 0002:000029a8       ??_R3CUserException@@8     5f89b9a8  
 0002:000029b8       ??_R4CUserException@@6B@   5f89b9b8  
 0002:000029d0       ??_R1A@?0A@A@COleObjectFactory@@8 5f89b9d0  
 0002:000029ec       ??_7COleObjectFactory@@6B@ 5f89b9ec  
 0002:00002a60       ??_R2COleObjectFactory@@8  5f89ba60  
 0002:00002a70       ??_R3COleObjectFactory@@8  5f89ba70  
 0002:00002a80       ??_R4COleObjectFactory@@6B@ 5f89ba80  
 0002:00002a98       ??_7CWinApp@@6B@           5f89ba98  
 0002:00002b40       ??_R1A@?0A@A@CWinApp@@8    5f89bb40  
 0002:00002b58       ??_R2CWinApp@@8            5f89bb58  
 0002:00002b70       ??_R3CWinApp@@8            5f89bb70  
 0002:00002b80       ??_R4CWinApp@@6B@          5f89bb80  
 0002:00002b98       ??_7CDynLinkLibrary@@6B@   5f89bb98  
 0002:00002bf0       ??_R1A@?0A@A@CDynLinkLibrary@@8 5f89bbf0  
 0002:00002c08       ??_R2CDynLinkLibrary@@8    5f89bc08  
 0002:00002c18       ??_R3CDynLinkLibrary@@8    5f89bc18  
 0002:00002c28       ??_R4CDynLinkLibrary@@6B@  5f89bc28  
 0002:00002c40       ??_7_AFX_CTL3D_STATE@@6B@  5f89bc40  
 0002:00002c48       ??_R1A@?0A@A@_AFX_CTL3D_STATE@@8 5f89bc48  
 0002:00002c60       ??_R2_AFX_CTL3D_STATE@@8   5f89bc60  
 0002:00002c70       ??_R3_AFX_CTL3D_STATE@@8   5f89bc70  
 0002:00002c80       ??_R4_AFX_CTL3D_STATE@@6B@ 5f89bc80  
 0002:00002c98       ??_7COleMessageFilter@@6B@ 5f89bc98  
 0002:00002d08       ??_R1A@?0A@A@COleMessageFilter@@8 5f89bd08  
 0002:00002d20       ??_R2COleMessageFilter@@8  5f89bd20  
 0002:00002d30       ??_R3COleMessageFilter@@8  5f89bd30  
 0002:00002d40       ??_R4COleMessageFilter@@6B@ 5f89bd40  
 0002:00002d58       ??_7_AFX_WIN_STATE@@6B@    5f89bd58  
 0002:00002d60       ??_R1A@?0A@A@_AFX_WIN_STATE@@8 5f89bd60  
 0002:00002d78       ??_R2_AFX_WIN_STATE@@8     5f89bd78  
 0002:00002d88       ??_R3_AFX_WIN_STATE@@8     5f89bd88  
 0002:00002d98       ??_R4_AFX_WIN_STATE@@6B@   5f89bd98  
 0002:00002db0       __sz_ADVAPI32              5f89bdb0  
 0002:00002dd8       ??_7CCommandLineInfo@@6B@  5f89bdd8  
 0002:00002df8       ??_R1A@?0A@A@CCommandLineInfo@@8 5f89bdf8  
 0002:00002e10       ??_R2CCommandLineInfo@@8   5f89be10  
 0002:00002e20       ??_R3CCommandLineInfo@@8   5f89be20  
 0002:00002e30       ??_R4CCommandLineInfo@@6B@ 5f89be30  
 0002:00002e48       ??_7CPtrArray@@6B@         5f89be48  
 0002:00002e60       ??_R1A@?0A@A@CPtrArray@@8  5f89be60  
 0002:00002e78       ??_R2CPtrArray@@8          5f89be78  
 0002:00002e88       ??_R3CPtrArray@@8          5f89be88  
 0002:00002e98       ??_R4CPtrArray@@6B@        5f89be98  
 0002:00002eb0       ??_R1A@?0A@A@CDocTemplate@@8 5f89beb0  
 0002:00002ecc       ??_7CDocTemplate@@6B@      5f89becc  
 0002:00002f64       ??_7CRecentFileList@@6B@   5f89bf64  
 0002:00002f80       ??_R2CDocTemplate@@8       5f89bf80  
 0002:00002f90       ??_R3CDocTemplate@@8       5f89bf90  
 0002:00002fa0       ??_R4CDocTemplate@@6B@     5f89bfa0  
 0002:00002fb8       ??_R1A@?0A@A@CRecentFileList@@8 5f89bfb8  
 0002:00002fd0       ??_R2CRecentFileList@@8    5f89bfd0  
 0002:00002fd8       ??_R3CRecentFileList@@8    5f89bfd8  
 0002:00002fe8       ??_R4CRecentFileList@@6B@  5f89bfe8  
 0002:00003000       ??_7CDocManager@@6B@       5f89c000  
 0002:00003048       ??_R1A@?0A@A@CDocManager@@8 5f89c048  
 0002:00003060       ??_R2CDocManager@@8        5f89c060  
 0002:00003070       ??_R3CDocManager@@8        5f89c070  
 0002:00003080       ??_R4CDocManager@@6B@      5f89c080  
 0002:00003098       ??_R1A@?0A@A@CFrameWnd@@8  5f89c098  
 0002:000030b4       ??_7CFrameWnd@@6B@         5f89c0b4  
 0002:000031b0       ??_R2CFrameWnd@@8          5f89c1b0  
 0002:000031c8       ??_R3CFrameWnd@@8          5f89c1c8  
 0002:000031d8       ??_R4CFrameWnd@@6B@        5f89c1d8  
 0002:000031f0       ??_7CStatusBar@@6B@        5f89c1f0  
 0002:000032e0       ??_R1A@?0A@A@CControlBar@@8 5f89c2e0  
 0002:000032f8       ??_R1A@?0A@A@CStatusBar@@8 5f89c2f8  
 0002:00003310       ??_R2CStatusBar@@8         5f89c310  
 0002:00003328       ??_R3CStatusBar@@8         5f89c328  
 0002:00003338       ??_R4CStatusBar@@6B@       5f89c338  
 0002:00003350       ??_7CControlBar@@6B@       5f89c350  
 0002:00003438       ??_R2CControlBar@@8        5f89c438  
 0002:00003450       ??_R3CControlBar@@8        5f89c450  
 0002:00003460       ??_R4CControlBar@@6B@      5f89c460  
 0002:00003478       ??_7CToolBar@@6B@          5f89c478  
 0002:00003568       ??_R1A@?0A@A@CToolBar@@8   5f89c568  
 0002:00003580       ??_R2CToolBar@@8           5f89c580  
 0002:00003598       ??_R3CToolBar@@8           5f89c598  
 0002:000035a8       ??_R4CToolBar@@6B@         5f89c5a8  
 0002:000035c0       ??_7CDockBar@@6B@          5f89c5c0  
 0002:000036b0       ??_R1A@?0A@A@CDockBar@@8   5f89c6b0  
 0002:000036c8       ??_R2CDockBar@@8           5f89c6c8  
 0002:000036e0       ??_R3CDockBar@@8           5f89c6e0  
 0002:000036f0       ??_R4CDockBar@@6B@         5f89c6f0  
 0002:00003708       ??_7CDockContext@@6B@      5f89c708  
 0002:00003718       ??_R1A@?0A@A@CDockContext@@8 5f89c718  
 0002:00003730       ??_R2CDockContext@@8       5f89c730  
 0002:00003738       ??_R3CDockContext@@8       5f89c738  
 0002:00003748       ??_R4CDockContext@@6B@     5f89c748  
 0002:00003760       ??_R1A@?0A@A@CDocument@@8  5f89c760  
 0002:00003778       ??_R1A@?0A@A@COleDocument@@8 5f89c778  
 0002:00003790       ??_R1A@?0A@A@COleLinkingDoc@@8 5f89c790  
 0002:000037a8       ??_R1A@?0A@A@COleServerDoc@@8 5f89c7a8  
 0002:000037c4       ??_7COleServerDoc@@6B@     5f89c7c4  
 0002:00003910       ??_R2COleServerDoc@@8      5f89c910  
 0002:00003930       ??_R3COleServerDoc@@8      5f89c930  
 0002:00003940       ??_R4COleServerDoc@@6B@    5f89c940  
 0002:00003958       ??_7COleLinkingDoc@@6B@    5f89c958  
 0002:00003a50       ??_R2COleLinkingDoc@@8     5f89ca50  
 0002:00003a68       ??_R3COleLinkingDoc@@8     5f89ca68  
 0002:00003a78       ??_R4COleLinkingDoc@@6B@   5f89ca78  
 0002:00003a90       ??_7COleDocument@@6B@      5f89ca90  
 0002:00003b78       ??_R2COleDocument@@8       5f89cb78  
 0002:00003b90       ??_R3COleDocument@@8       5f89cb90  
 0002:00003ba0       ??_R4COleDocument@@6B@     5f89cba0  
 0002:00003bb8       ??_7CDocument@@6B@         5f89cbb8  
 0002:00003c70       ??_R2CDocument@@8          5f89cc70  
 0002:00003c80       ??_R3CDocument@@8          5f89cc80  
 0002:00003c90       ??_R4CDocument@@6B@        5f89cc90  
 0002:00003ca8       ??_7CObList@@6B@           5f89cca8  
 0002:00003cc0       ??_R1A@?0A@A@CObList@@8    5f89ccc0  
 0002:00003cd8       ??_R2CObList@@8            5f89ccd8  
 0002:00003ce8       ??_R3CObList@@8            5f89cce8  
 0002:00003cf8       ??_R4CObList@@6B@          5f89ccf8  
 0002:00003d10       ??_R1A@?0A@A@CView@@8      5f89cd10  
 0002:00003d2c       ??_7CView@@6B@             5f89cd2c  
 0002:00003e40       ??_R2CView@@8              5f89ce40  
 0002:00003e58       ??_R3CView@@8              5f89ce58  
 0002:00003e68       ??_R4CView@@6B@            5f89ce68  
 0002:00003e80       ??_7CDockState@@6B@        5f89ce80  
 0002:00003e98       ??_R1A@?0A@A@CDockState@@8 5f89ce98  
 0002:00003eb0       ??_R2CDockState@@8         5f89ceb0  
 0002:00003ec0       ??_R3CDockState@@8         5f89cec0  
 0002:00003ed0       ??_R4CDockState@@6B@       5f89ced0  
 0002:00003ee8       ??_7CSingleDocTemplate@@6B@ 5f89cee8  
 0002:00003f80       ??_R1A@?0A@A@CSingleDocTemplate@@8 5f89cf80  
 0002:00003f98       ??_R2CSingleDocTemplate@@8 5f89cf98  
 0002:00003fb0       ??_R3CSingleDocTemplate@@8 5f89cfb0  
 0002:00003fc0       ??_R4CSingleDocTemplate@@6B@ 5f89cfc0  
 0002:00003fd4       ??_C@_1BC@GMME@?$AAs?$AAo?$AAf?$AAt?$AAw?$AAa?$AAr?$AAe?$AA?$AA@ 5f89cfd4  
 0002:00003fec       ??_7CMemFile@@6B@          5f89cfec  
 0002:00004060       ??_R1A@?0A@A@CMemFile@@8   5f89d060  
 0002:00004078       ??_R2CMemFile@@8           5f89d078  
 0002:00004088       ??_R3CMemFile@@8           5f89d088  
 0002:00004098       ??_R4CMemFile@@6B@         5f89d098  
 0002:000040b0       ??_7CDWordArray@@6B@       5f89d0b0  
 0002:000040c8       ??_R1A@?0A@A@CDWordArray@@8 5f89d0c8  
 0002:000040e0       ??_R2CDWordArray@@8        5f89d0e0  
 0002:000040f0       ??_R3CDWordArray@@8        5f89d0f0  
 0002:00004100       ??_R4CDWordArray@@6B@      5f89d100  
 0002:00004118       ??_7_AFX_RICHEDIT_STATE@@6B@ 5f89d118  
 0002:00004120       ??_R1A@?0A@A@_AFX_EDIT_STATE@@8 5f89d120  
 0002:00004138       ??_R1A@?0A@A@_AFX_RICHEDIT_STATE@@8 5f89d138  
 0002:00004150       ??_R2_AFX_RICHEDIT_STATE@@8 5f89d150  
 0002:00004160       ??_R3_AFX_RICHEDIT_STATE@@8 5f89d160  
 0002:00004170       ??_R4_AFX_RICHEDIT_STATE@@6B@ 5f89d170  
 0002:00004188       ??_7_AFX_EDIT_STATE@@6B@   5f89d188  
 0002:00004190       ??_R2_AFX_EDIT_STATE@@8    5f89d190  
 0002:000041a0       ??_R3_AFX_EDIT_STATE@@8    5f89d1a0  
 0002:000041b0       ??_R4_AFX_EDIT_STATE@@6B@  5f89d1b0  
 0002:000041c8       ??_7_AFX_OLE_STATE@@6B@    5f89d1c8  
 0002:000041d0       ??_R1A@?0A@A@_AFX_OLE_STATE@@8 5f89d1d0  
 0002:000041e8       ??_R2_AFX_OLE_STATE@@8     5f89d1e8  
 0002:000041f8       ??_R3_AFX_OLE_STATE@@8     5f89d1f8  
 0002:00004208       ??_R4_AFX_OLE_STATE@@6B@   5f89d208  
 0002:00004230       ??_7CComboBox@@6B@         5f89d230  
 0002:00004300       ??_R1A@?0A@A@CComboBox@@8  5f89d300  
 0002:00004318       ??_R2CComboBox@@8          5f89d318  
 0002:00004330       ??_R3CComboBox@@8          5f89d330  
 0002:00004340       ??_R4CComboBox@@6B@        5f89d340  
 0002:00004358       ?interfaceMap@COleObjectFactory@@1UAFX_INTERFACEMAP@@B 5f89d358  
 0002:00004360       ?_interfaceEntries@COleObjectFactory@@0QBUAFX_INTERFACEMAP_ENTRY@@B 5f89d360  
 0002:00004378       _IID_IClassFactory         5f89d378  
 0002:00004388       _IID_IClassFactory2        5f89d388  
 0002:0000439c       ??_7CDialog@@6B@           5f89d39c  
 0002:00004478       ??_R1A@?0A@A@CDialog@@8    5f89d478  
 0002:00004490       ??_R2CDialog@@8            5f89d490  
 0002:000044a8       ??_R3CDialog@@8            5f89d4a8  
 0002:000044b8       ??_R4CDialog@@6B@          5f89d4b8  
 0002:000044d0       ??_7CGdiObject@@6B@        5f89d4d0  
 0002:000044e8       ??_R2CGdiObject@@8         5f89d4e8  
 0002:000044f8       ??_R3CGdiObject@@8         5f89d4f8  
 0002:00004508       ??_R4CGdiObject@@6B@       5f89d508  
 0002:00004520       ?messageMap@CDialog@@1UAFX_MSGMAP@@B 5f89d520  
 0002:00004528       ?_messageEntries@CDialog@@0QBUAFX_MSGMAP_ENTRY@@B 5f89d528  
 0002:00004604       ??_7CMapStringToPtr@@6B@   5f89d604  
 0002:00004618       ??_R1A@?0A@A@CMapStringToPtr@@8 5f89d618  
 0002:00004630       ??_R2CMapStringToPtr@@8    5f89d630  
 0002:00004640       ??_R3CMapStringToPtr@@8    5f89d640  
 0002:00004650       ??_R4CMapStringToPtr@@6B@  5f89d650  
 0002:00004668       ?messageMap@CPrintDialog@@1UAFX_MSGMAP@@B 5f89d668  
 0002:00004670       ?_messageEntries@CPrintDialog@@0QBUAFX_MSGMAP_ENTRY@@B 5f89d670  
 0002:000046a0       ?messageMap@CCommonDialog@@1UAFX_MSGMAP@@B 5f89d6a0  
 0002:000046a8       ?_messageEntries@CCommonDialog@@0QBUAFX_MSGMAP_ENTRY@@B 5f89d6a8  
 0002:000046dc       ??_7CTempGdiObject@@6B@    5f89d6dc  
 0002:000046f0       ??_R1A@?0A@A@CTempGdiObject@@8 5f89d6f0  
 0002:00004708       ??_R2CTempGdiObject@@8     5f89d708  
 0002:00004718       ??_R3CTempGdiObject@@8     5f89d718  
 0002:00004728       ??_R4CTempGdiObject@@6B@   5f89d728  
 0002:0000473c       ??_C@_0BC@COEH@MonitorFromWindow?$AA@ 5f89d73c  
 0002:00004750       ??_C@_0BB@NDAA@GetSystemMetrics?$AA@ 5f89d750  
 0002:00004764       ??_C@_1O@EJK@?$AAU?$AAS?$AAE?$AAR?$AA3?$AA2?$AA?$AA@ 5f89d764  
 0002:00004774       ?_afxWndControlBar@@3QBGB  5f89d774  
 0002:00004798       ?_afxWndMDIFrame@@3QBGB    5f89d798  
 0002:000047b8       ?_afxWndFrameOrView@@3QBGB 5f89d7b8  
 0002:000047dc       ??_C@_0BF@CELH@InitCommonControlsEx?$AA@ 5f89d7dc  
 0002:000047f4       ??_C@_0N@BMKC@COMCTL32?4DLL?$AA@ 5f89d7f4  
 0002:00004808       ?classCDialog@CDialog@@2UCRuntimeClass@@B 5f89d808  
 0002:00004820       ??_C@_07IJJI@CDialog?$AA@  5f89d820  
 0002:0000482c       ??_7CTempDC@@6B@           5f89d82c  
 0002:000048a8       ??_R1A@?0A@A@CTempDC@@8    5f89d8a8  
 0002:000048c0       ??_R2CTempDC@@8            5f89d8c0  
 0002:000048d0       ??_R3CTempDC@@8            5f89d8d0  
 0002:000048e0       ??_R4CTempDC@@6B@          5f89d8e0  
 0002:000048f8       ??_7CPrintDialog@@6B@      5f89d8f8  
 0002:000049d8       ??_R1A@?0A@A@CCommonDialog@@8 5f89d9d8  
 0002:000049f0       ??_R1A@?0A@A@CPrintDialog@@8 5f89d9f0  
 0002:00004a08       ??_R2CPrintDialog@@8       5f89da08  
 0002:00004a28       ??_R3CPrintDialog@@8       5f89da28  
 0002:00004a38       ??_R4CPrintDialog@@6B@     5f89da38  
 0002:00004a50       ??_7CPrintingDialog@@6B@   5f89da50  
 0002:00004b28       ??_R1A@?0A@A@CPrintingDialog@@8 5f89db28  
 0002:00004b40       ??_R2CPrintingDialog@@8    5f89db40  
 0002:00004b58       ??_R3CPrintingDialog@@8    5f89db58  
 0002:00004b68       ??_R4CPrintingDialog@@6B@  5f89db68  
 0002:00004b80       ??_7CException@@6B@        5f89db80  
 0002:00004ba0       ??_R2CException@@8         5f89dba0  
 0002:00004bb0       ??_R3CException@@8         5f89dbb0  
 0002:00004bc0       ??_R4CException@@6B@       5f89dbc0  
 0002:00004bd8       _GUID_NULL                 5f89dbd8  
 0002:00004be8       ?classCView@CView@@2UCRuntimeClass@@B 5f89dbe8  
 0002:00004c00       ??_C@_05KON@CView?$AA@     5f89dc00  
 0002:00004c0c       ??_7CPaintDC@@6B@          5f89dc0c  
 0002:00004c88       ??_R1A@?0A@A@CPaintDC@@8   5f89dc88  
 0002:00004ca0       ??_R2CPaintDC@@8           5f89dca0  
 0002:00004cb0       ??_R3CPaintDC@@8           5f89dcb0  
 0002:00004cc0       ??_R4CPaintDC@@6B@         5f89dcc0  
 0002:00004cd8       __sz_comdlg32              5f89dcd8  
 0002:00004d08       ??_7CFileException@@6B@    5f89dd08  
 0002:00004d28       ??_R1A@?0A@A@CFileException@@8 5f89dd28  
 0002:00004d40       ??_R2CFileException@@8     5f89dd40  
 0002:00004d50       ??_R3CFileException@@8     5f89dd50  
 0002:00004d60       ??_R4CFileException@@6B@   5f89dd60  
 0002:00004d78       ??_7CButton@@6B@           5f89dd78  
 0002:00004e40       ??_R1A@?0A@A@CButton@@8    5f89de40  
 0002:00004e58       ??_R2CButton@@8            5f89de58  
 0002:00004e70       ??_R3CButton@@8            5f89de70  
 0002:00004e80       ??_R4CButton@@6B@          5f89de80  
 0002:00004e94       ??_C@_0L@LFP@CByteArray?$AA@ 5f89de94  
 0002:00004ea0       ??_C@_0M@JHEJ@CDWordArray?$AA@ 5f89dea0  
 0002:00004eac       ??_C@_08PPJP@CObArray?$AA@ 5f89deac  
 0002:00004eb8       ??_C@_0N@FMIP@CStringArray?$AA@ 5f89deb8  
 0002:00004ec8       ??_C@_0L@KEGG@CWordArray?$AA@ 5f89dec8  
 0002:00004ed4       ??_C@_07ICCG@CObList?$AA@  5f89ded4  
 0002:00004edc       ??_C@_0M@JCPP@CStringList?$AA@ 5f89dedc  
 0002:00004ee8       ??_C@_0P@FLNF@CMapStringToOb?$AA@ 5f89dee8  
 0002:00004ef8       ??_C@_0BD@HCIA@CMapStringToString?$AA@ 5f89def8  
 0002:00004f0c       ??_C@_0N@DJOC@CMapWordToOb?$AA@ 5f89df0c  
 0002:00004f1c       ??_C@_1CK@HBPJ@?$AAc?$AAo?$AAm?$AAm?$AAc?$AAt?$AAr?$AAl?$AA_?$AAD?$AAr?$AAa?$AAg?$AAL?$AAi?$AAs?$AAt?$AAM?$AAs?$AAg@ 5f89df1c  
 0002:00004f48       ??_C@_0L@HPAN@CDockState?$AA@ 5f89df48  
 0002:00004f54       ??_C@_1CI@PGNH@?$AAc?$AAo?$AAm?$AAm?$AAd?$AAl?$AAg?$AA_?$AAF?$AAi?$AAn?$AAd?$AAR?$AAe?$AAp?$AAl?$AAa?$AAc?$AAe?$AA?$AA@ 5f89df54  
 0002:00004f7c       ??_C@_1DE@GHMD@?$AAR?$AAi?$AAc?$AAh?$AAE?$AAd?$AAi?$AAt?$AA?5?$AAT?$AAe?$AAx?$AAt?$AA?5?$AAa?$AAn?$AAd?$AA?5?$AAO?$AAb@ 5f89df7c  
 0002:00004fb0       ??_C@_1CC@FCIJ@?$AAR?$AAi?$AAc?$AAh?$AA?5?$AAT?$AAe?$AAx?$AAt?$AA?5?$AAF?$AAo?$AAr?$AAm?$AAa?$AAt?$AA?$AA@ 5f89dfb0  
 0002:00004fd4       ??_C@_1BE@OIFD@?$AAF?$AAi?$AAl?$AAe?$AAN?$AAa?$AAm?$AAe?$AAW?$AA?$AA@ 5f89dfd4  
 0002:00004fe8       ??_C@_1BC@LEEL@?$AAF?$AAi?$AAl?$AAe?$AAN?$AAa?$AAm?$AAe?$AA?$AA@ 5f89dfe8  
 0002:00004ffc       ??_C@_1CO@MJBN@?$AAL?$AAi?$AAn?$AAk?$AA?5?$AAS?$AAo?$AAu?$AAr?$AAc?$AAe?$AA?5?$AAD?$AAe?$AAs?$AAc?$AAr?$AAi?$AAp?$AAt@ 5f89dffc  
 0002:0000502c       ??_C@_1CE@PGMB@?$AAO?$AAb?$AAj?$AAe?$AAc?$AAt?$AA?5?$AAD?$AAe?$AAs?$AAc?$AAr?$AAi?$AAp?$AAt?$AAo?$AAr?$AA?$AA@ 5f89e02c  
 0002:00005050       ??_C@_1BI@PBNI@?$AAL?$AAi?$AAn?$AAk?$AA?5?$AAS?$AAo?$AAu?$AAr?$AAc?$AAe?$AA?$AA@ 5f89e050  
 0002:00005068       ??_C@_1BK@EEJA@?$AAE?$AAm?$AAb?$AAe?$AAd?$AA?5?$AAS?$AAo?$AAu?$AAr?$AAc?$AAe?$AA?$AA@ 5f89e068  
 0002:00005084       ??_C@_1CA@NPFJ@?$AAE?$AAm?$AAb?$AAe?$AAd?$AAd?$AAe?$AAd?$AA?5?$AAO?$AAb?$AAj?$AAe?$AAc?$AAt?$AA?$AA@ 5f89e084  
 0002:000050a4       ??_C@_1BG@JFDH@?$AAO?$AAb?$AAj?$AAe?$AAc?$AAt?$AAL?$AAi?$AAn?$AAk?$AA?$AA@ 5f89e0a4  
 0002:000050bc       ??_C@_1BE@MPFF@?$AAO?$AAw?$AAn?$AAe?$AAr?$AAL?$AAi?$AAn?$AAk?$AA?$AA@ 5f89e0bc  
 0002:000050d0       ??_C@_1O@OGPB@?$AAN?$AAa?$AAt?$AAi?$AAv?$AAe?$AA?$AA@ 5f89e0d0  
 0002:000050e0       ??_C@_08NNLJ@CDocItem?$AA@ 5f89e0e0  
 0002:000050ec       ??_C@_0BC@CJOP@CRichEditCntrItem?$AA@ 5f89e0ec  
 0002:00005100       ?classCColorPropPage@CColorPropPage@@2UCRuntimeClass@@B 5f89e100  
 0002:00005118       ??_C@_0P@PKCG@CColorPropPage?$AA@ 5f89e118  
 0002:00005150       ?guid@CColorPropPage@@2U_GUID@@B 5f89e150  
 0002:00005164       ??_7CColorPropPageFactory@CColorPropPage@@6B@ 5f89e164  
 0002:000051d8       ??_R1A@?0A@A@CColorPropPageFactory@CColorPropPage@@8 5f89e1d8  
 0002:000051f0       ??_R2CColorPropPageFactory@CColorPropPage@@8 5f89e1f0  
 0002:00005208       ??_R3CColorPropPageFactory@CColorPropPage@@8 5f89e208  
 0002:00005218       ??_R4CColorPropPageFactory@CColorPropPage@@6B@ 5f89e218  
 0002:00005230       ??_7XClassFactory@COleObjectFactory@@6B@ 5f89e230  
 0002:00005250       ??_R1A@?0A@A@IUnknown@@8   5f89e250  
 0002:00005268       ??_R1A@?0A@A@IClassFactory@@8 5f89e268  
 0002:00005280       ??_R1A@?0A@A@IClassFactory2@@8 5f89e280  
 0002:00005298       ??_R1A@?0A@A@XClassFactory@COleObjectFactory@@8 5f89e298  
 0002:000052b0       ??_R2XClassFactory@COleObjectFactory@@8 5f89e2b0  
 0002:000052c8       ??_R3XClassFactory@COleObjectFactory@@8 5f89e2c8  
 0002:000052d8       ??_R4XClassFactory@COleObjectFactory@@6B@ 5f89e2d8  
 0002:000052f0       ?classCFontPropPage@CFontPropPage@@2UCRuntimeClass@@B 5f89e2f0  
 0002:00005308       ??_C@_0O@IMID@CFontPropPage?$AA@ 5f89e308  
 0002:00005340       ?guid@CFontPropPage@@2U_GUID@@B 5f89e340  
 0002:00005354       ??_7CFontPropPageFactory@CFontPropPage@@6B@ 5f89e354  
 0002:000053c8       ??_R1A@?0A@A@CFontPropPageFactory@CFontPropPage@@8 5f89e3c8  
 0002:000053e0       ??_R2CFontPropPageFactory@CFontPropPage@@8 5f89e3e0  
 0002:000053f8       ??_R3CFontPropPageFactory@CFontPropPage@@8 5f89e3f8  
 0002:00005408       ??_R4CFontPropPageFactory@CFontPropPage@@6B@ 5f89e408  
 0002:00005420       ?classCPicturePropPage@CPicturePropPage@@2UCRuntimeClass@@B 5f89e420  
 0002:00005438       ??_C@_0BB@EHCI@CPicturePropPage?$AA@ 5f89e438  
 0002:00005480       ?guid@CPicturePropPage@@2U_GUID@@B 5f89e480  
 0002:00005494       ??_7CPicturePropPageFactory@CPicturePropPage@@6B@ 5f89e494  
 0002:00005508       ??_R1A@?0A@A@CPicturePropPageFactory@CPicturePropPage@@8 5f89e508  
 0002:00005520       ??_R2CPicturePropPageFactory@CPicturePropPage@@8 5f89e520  
 0002:00005538       ??_R3CPicturePropPageFactory@CPicturePropPage@@8 5f89e538  
 0002:00005548       ??_R4CPicturePropPageFactory@CPicturePropPage@@6B@ 5f89e548  
 0002:0000555c       ??_C@_19KGAM@?$AA?4?$AAI?$AAN?$AAI?$AA?$AA@ 5f89e55c  
 0002:00005568       ??_C@_19CLBK@?$AA?4?$AAH?$AAL?$AAP?$AA?$AA@ 5f89e568  
 0002:00005578       ??_7_AFX_BASE_MODULE_STATE@@6B@ 5f89e578  
 0002:00005580       ??_R1A@?0A@A@_AFX_BASE_MODULE_STATE@@8 5f89e580  
 0002:00005598       ??_R2_AFX_BASE_MODULE_STATE@@8 5f89e598  
 0002:000055a8       ??_R3_AFX_BASE_MODULE_STATE@@8 5f89e5a8  
 0002:000055b8       ??_R4_AFX_BASE_MODULE_STATE@@6B@ 5f89e5b8  
 0002:000055d0       ??_7XMessageFilter@COleMessageFilter@@6B@ 5f89e5d0  
 0002:000055e8       ??_R1A@?0A@A@IMessageFilter@@8 5f89e5e8  
 0002:00005600       ??_R1A@?0A@A@XMessageFilter@COleMessageFilter@@8 5f89e600  
 0002:00005618       ??_R2XMessageFilter@COleMessageFilter@@8 5f89e618  
 0002:00005628       ??_R3XMessageFilter@COleMessageFilter@@8 5f89e628  
 0002:00005638       ??_R4XMessageFilter@COleMessageFilter@@6B@ 5f89e638  
 0002:00005650       __sz_COMCTL32              5f89e650  
 0002:00005678       ??_C@_17BCJF@?$AAI?$AA6?$AA4?$AA?$AA@ 5f89e678  
 0002:00005684       ??_7COleTemplateServer@@6B@ 5f89e684  
 0002:000056f8       ??_R1A@?0A@A@COleTemplateServer@@8 5f89e6f8  
 0002:00005710       ??_R2COleTemplateServer@@8 5f89e710  
 0002:00005728       ??_R3COleTemplateServer@@8 5f89e728  
 0002:00005738       ??_R4COleTemplateServer@@6B@ 5f89e738  
 0002:0000574c       ?_afxPreviewEntry@@3QBGB   5f89e74c  
 0002:00005768       ?_afxPreviewSection@@3QBGB 5f89e768  
 0002:0000577c       ?_afxFileEntry@@3QBGB      5f89e77c  
 0002:0000578c       ?_afxFileSection@@3QBGB    5f89e78c  
 0002:000057bc       ??_C@_1CG@HFFM@?$AAA?$AAf?$AAx?$AA?3?$AA?$CF?$AAx?$AA?3?$AA?$CF?$AAx?$AA?3?$AA?$CF?$AAx?$AA?3?$AA?$CF?$AAx?$AA?3?$AA?$CF?$AAx?$AA?$AA@ 5f89e7bc  
 0002:000057e4       ??_C@_1CA@IKCD@?$AAT?$AAo?$AAo?$AAl?$AAb?$AAa?$AAr?$AAW?$AAi?$AAn?$AAd?$AAo?$AAw?$AA3?$AA2?$AA?$AA@ 5f89e7e4  
 0002:00005804       ??_C@_0O@CDEE@DllGetVersion?$AA@ 5f89e804  
 0002:00005814       ??_C@_1BA@NPHH@?$AAM?$AAa?$AAr?$AAl?$AAe?$AAt?$AAt?$AA?$AA@ 5f89e814  
 0002:00005828       ?_afxSysColorMap@@3QBUAFX_COLORMAP@@B 5f89e828  
 0002:00005848       ??_C@_1CG@LDD@?$AAm?$AAs?$AAc?$AAt?$AAl?$AAs?$AA_?$AAs?$AAt?$AAa?$AAt?$AAu?$AAs?$AAb?$AAa?$AAr?$AA3?$AA2?$AA?$AA@ 5f89e848  
 0002:00005874       ??_7CClientDC@@6B@         5f89e874  
 0002:000058f0       ??_R1A@?0A@A@CClientDC@@8  5f89e8f0  
 0002:00005908       ??_R2CClientDC@@8          5f89e908  
 0002:00005918       ??_R3CClientDC@@8          5f89e918  
 0002:00005928       ??_R4CClientDC@@6B@        5f89e928  
 0002:0000593c       ?dwDockBarMap@CFrameWnd@@1QAY01$$CBKA 5f89e93c  
 0002:00005960       ?classCMiniDockFrameWnd@CMiniDockFrameWnd@@2UCRuntimeClass@@B 5f89e960  
 0002:00005978       ??_C@_0BC@NGKE@CMiniDockFrameWnd?$AA@ 5f89e978  
 0002:00005990       __sz_SHELL32               5f89e990  
 0002:000059b4       ??_7XOleInPlaceActiveObject@COleServerDoc@@6B@ 5f89e9b4  
 0002:000059e0       ??_7XOleInPlaceObject@COleServerDoc@@6B@ 5f89e9e0  
 0002:00005a08       ??_7XDataObject@COleServerDoc@@6B@ 5f89ea08  
 0002:00005a3c       ??_7XOleObject@COleServerDoc@@6B@ 5f89ea3c  
 0002:00005aa0       ??_7XPersistStorage@COleServerDoc@@6B@ 5f89eaa0  
 0002:00005ac8       ??_R1A@?0A@A@IOleWindow@@8 5f89eac8  
 0002:00005ae0       ??_R1A@?0A@A@IDataObject@@8 5f89eae0  
 0002:00005af8       ??_R1A@?0A@A@IPersist@@8   5f89eaf8  
 0002:00005b10       ??_R1A@?0A@A@IOleObject@@8 5f89eb10  
 0002:00005b28       ??_R1A@?0A@A@XOleObject@COleServerDoc@@8 5f89eb28  
 0002:00005b40       ??_R2XOleObject@COleServerDoc@@8 5f89eb40  
 0002:00005b50       ??_R3XOleObject@COleServerDoc@@8 5f89eb50  
 0002:00005b60       ??_R4XOleObject@COleServerDoc@@6B@ 5f89eb60  
 0002:00005b78       ??_R1A@?0A@A@IPersistStorage@@8 5f89eb78  
 0002:00005b90       ??_R1A@?0A@A@XPersistStorage@COleServerDoc@@8 5f89eb90  
 0002:00005ba8       ??_R2XPersistStorage@COleServerDoc@@8 5f89eba8  
 0002:00005bc0       ??_R3XPersistStorage@COleServerDoc@@8 5f89ebc0  
 0002:00005bd0       ??_R4XPersistStorage@COleServerDoc@@6B@ 5f89ebd0  
 0002:00005be8       ??_R1A@?0A@A@IOleInPlaceActiveObject@@8 5f89ebe8  
 0002:00005c00       ??_R1A@?0A@A@XOleInPlaceActiveObject@COleServerDoc@@8 5f89ec00  
 0002:00005c18       ??_R2XOleInPlaceActiveObject@COleServerDoc@@8 5f89ec18  
 0002:00005c30       ??_R3XOleInPlaceActiveObject@COleServerDoc@@8 5f89ec30  
 0002:00005c40       ??_R4XOleInPlaceActiveObject@COleServerDoc@@6B@ 5f89ec40  
 0002:00005c58       ??_R1A@?0A@A@IOleInPlaceObject@@8 5f89ec58  
 0002:00005c70       ??_R1A@?0A@A@XOleInPlaceObject@COleServerDoc@@8 5f89ec70  
 0002:00005c88       ??_R2XOleInPlaceObject@COleServerDoc@@8 5f89ec88  
 0002:00005ca0       ??_R3XOleInPlaceObject@COleServerDoc@@8 5f89eca0  
 0002:00005cb0       ??_R4XOleInPlaceObject@COleServerDoc@@6B@ 5f89ecb0  
 0002:00005cc8       ??_R1A@?0A@A@XDataObject@COleServerDoc@@8 5f89ecc8  
 0002:00005ce0       ??_R2XDataObject@COleServerDoc@@8 5f89ece0  
 0002:00005cf0       ??_R3XDataObject@COleServerDoc@@8 5f89ecf0  
 0002:00005d00       ??_R4XDataObject@COleServerDoc@@6B@ 5f89ed00  
 0002:00005d18       ??_7XOleItemContainer@COleLinkingDoc@@6B@ 5f89ed18  
 0002:00005d40       ??_7XPersistFile@COleLinkingDoc@@6B@ 5f89ed40  
 0002:00005d68       ??_R1A@?0A@A@IPersistFile@@8 5f89ed68  
 0002:00005d80       ??_R1A@?0A@A@XPersistFile@COleLinkingDoc@@8 5f89ed80  
 0002:00005d98       ??_R2XPersistFile@COleLinkingDoc@@8 5f89ed98  
 0002:00005db0       ??_R3XPersistFile@COleLinkingDoc@@8 5f89edb0  
 0002:00005dc0       ??_R4XPersistFile@COleLinkingDoc@@6B@ 5f89edc0  
 0002:00005dd8       ??_R1A@?0A@A@IParseDisplayName@@8 5f89edd8  
 0002:00005df0       ??_R1A@?0A@A@IOleContainer@@8 5f89edf0  
 0002:00005e08       ??_R1A@?0A@A@IOleItemContainer@@8 5f89ee08  
 0002:00005e20       ??_R1A@?0A@A@XOleItemContainer@COleLinkingDoc@@8 5f89ee20  
 0002:00005e38       ??_R2XOleItemContainer@COleLinkingDoc@@8 5f89ee38  
 0002:00005e50       ??_R3XOleItemContainer@COleLinkingDoc@@8 5f89ee50  
 0002:00005e60       ??_R4XOleItemContainer@COleLinkingDoc@@6B@ 5f89ee60  
 0002:00005e78       ??_7CWindowDC@@6B@         5f89ee78  
 0002:00005ef8       ??_R1A@?0A@A@CWindowDC@@8  5f89eef8  
 0002:00005f10       ??_R2CWindowDC@@8          5f89ef10  
 0002:00005f20       ??_R3CWindowDC@@8          5f89ef20  
 0002:00005f30       ??_R4CWindowDC@@6B@        5f89ef30  
 0002:00005f48       ??_7CRichEditDoc@@6B@      5f89ef48  
 0002:00006098       ??_R1A@?0A@A@CRichEditDoc@@8 5f89f098  
 0002:000060b0       ??_R2CRichEditDoc@@8       5f89f0b0  
 0002:000060d0       ??_R3CRichEditDoc@@8       5f89f0d0  
 0002:000060e0       ??_R4CRichEditDoc@@6B@     5f89f0e0  
 0002:000060f4       ??_C@_1BC@IAEH@?$AAR?$AAI?$AAC?$AAH?$AAE?$AAD?$AAI?$AAT?$AA?$AA@ 5f89f0f4  
 0002:0000610c       ??_7CRichEditView@@6B@     5f89f10c  
 0002:0000624c       ??_7XRichEditOleCallback@CRichEditView@@6B@ 5f89f24c  
 0002:00006280       ??_R1A@?0A@A@CCtrlView@@8  5f89f280  
 0002:00006298       ??_R1A@?0A@A@CRichEditView@@8 5f89f298  
 0002:000062b0       ??_R2CRichEditView@@8      5f89f2b0  
 0002:000062d0       ??_R3CRichEditView@@8      5f89f2d0  
 0002:000062e0       ??_R4CRichEditView@@6B@    5f89f2e0  
 0002:000062f8       ??_R1A@?0A@A@IRichEditOleCallback@@8 5f89f2f8  
 0002:00006310       ??_R1A@?0A@A@XRichEditOleCallback@CRichEditView@@8 5f89f310  
 0002:00006328       ??_R2XRichEditOleCallback@CRichEditView@@8 5f89f328  
 0002:00006338       ??_R3XRichEditOleCallback@CRichEditView@@8 5f89f338  
 0002:00006348       ??_R4XRichEditOleCallback@CRichEditView@@6B@ 5f89f348  
 0002:00006360       ??_7CCtrlView@@6B@         5f89f360  
 0002:00006470       ??_R2CCtrlView@@8          5f89f470  
 0002:00006488       ??_R3CCtrlView@@8          5f89f488  
 0002:00006498       ??_R4CCtrlView@@6B@        5f89f498  
 0002:000064ac       ??_C@_0N@GEKM@RICHED32?4DLL?$AA@ 5f89f4ac  
 0002:000064bc       ??_C@_1BC@DNEF@?$AAC?$AAO?$AAM?$AAB?$AAO?$AAB?$AAO?$AAX?$AA?$AA@ 5f89f4bc  
 0002:000064d0       ?classCCtrlView@CCtrlView@@2UCRuntimeClass@@B 5f89f4d0  
 0002:000064e8       ??_C@_09OBAN@CCtrlView?$AA@ 5f89f4e8  
 0002:000064f8       ?messageMap@CFrameWnd@@1UAFX_MSGMAP@@B 5f89f4f8  
 0002:00006500       ?_messageEntries@CFrameWnd@@0QBUAFX_MSGMAP_ENTRY@@B 5f89f500  
 0002:00006968       ?messageMap@CMDIChildWnd@@1UAFX_MSGMAP@@B 5f89f968  
 0002:00006970       ?_messageEntries@CMDIChildWnd@@0QBUAFX_MSGMAP_ENTRY@@B 5f89f970  
 0002:00006a7c       ??_7CMultiDocTemplate@@6B@ 5f89fa7c  
 0002:00006b10       ??_R1A@?0A@A@CMultiDocTemplate@@8 5f89fb10  
 0002:00006b28       ??_R2CMultiDocTemplate@@8  5f89fb28  
 0002:00006b40       ??_R3CMultiDocTemplate@@8  5f89fb40  
 0002:00006b50       ??_R4CMultiDocTemplate@@6B@ 5f89fb50  
 0002:00006b68       ??_7CScrollView@@6B@       5f89fb68  
 0002:00006c78       ??_R1A@?0A@A@CScrollView@@8 5f89fc78  
 0002:00006c90       ??_R2CScrollView@@8        5f89fc90  
 0002:00006ca8       ??_R3CScrollView@@8        5f89fca8  
 0002:00006cb8       ??_R4CScrollView@@6B@      5f89fcb8  
 0002:00006cd0       ??_7COleDropTarget@@6B@    5f89fcd0  
 0002:00006d48       ??_R1A@?0A@A@COleDropTarget@@8 5f89fd48  
 0002:00006d60       ??_R2COleDropTarget@@8     5f89fd60  
 0002:00006d70       ??_R3COleDropTarget@@8     5f89fd70  
 0002:00006d80       ??_R4COleDropTarget@@6B@   5f89fd80  
 0002:00006d98       _IID_IDropTarget           5f89fd98  
 0002:00006da8       ?interfaceMap@COleDropTarget@@1UAFX_INTERFACEMAP@@B 5f89fda8  
 0002:00006db0       ?_interfaceEntries@COleDropTarget@@0QBUAFX_INTERFACEMAP_ENTRY@@B 5f89fdb0  
 0002:000072b0       ??_C@_15KLDP@?$AA?$CF?$AAd?$AA?$AA@ 5f8a02b0  
 0002:000072b8       ??_C@_1M@EPCN@?$AAC?$AAL?$AAS?$AAI?$AAD?$AA?$AA@ 5f8a02b8  
 0002:000072c8       ??_7CMDIFrameWnd@@6B@      5f8a02c8  
 0002:000073d0       ??_R1A@?0A@A@CMDIFrameWnd@@8 5f8a03d0  
 0002:000073e8       ??_R2CMDIFrameWnd@@8       5f8a03e8  
 0002:00007400       ??_R3CMDIFrameWnd@@8       5f8a0400  
 0002:00007410       ??_R4CMDIFrameWnd@@6B@     5f8a0410  
 0002:00007424       ??_C@_1BE@MFDJ@?$AAm?$AAd?$AAi?$AAc?$AAl?$AAi?$AAe?$AAn?$AAt?$AA?$AA@ 5f8a0424  
 0002:00007438       ??_C@_1O@IKOG@?$AAs?$AAy?$AAs?$AAt?$AAe?$AAm?$AA?$AA@ 5f8a0438  
 0002:00007446       ?_afxShellNewValue@@3QBGB  5f8a0446  
 0002:00007448       ?_afxShellNewValueName@@3QBGB 5f8a0448  
 0002:0000745c       ?_afxDDEPrintTo@@3QBGB     5f8a045c  
 0002:0000749c       ?_afxDDEPrint@@3QBGB       5f8a049c  
 0002:000074b8       ?_afxDDEOpen@@3QBGB        5f8a04b8  
 0002:000074d4       ?_afxDDEExec@@3QBGB        5f8a04d4  
 0002:000074e4       ?_afxDDEArg@@3QBGB         5f8a04e4  
 0002:000074f0       ?_afxCommand@@3QBGB        5f8a04f0  
 0002:00007500       ?_afxIconIndexFmt@@3QBGB   5f8a0500  
 0002:00007508       ?_afxShellNewFmt@@3QBGB    5f8a0508  
 0002:00007520       ?_afxDefaultIconFmt@@3QBGB 5f8a0520  
 0002:00007540       ?_afxShellPrintToFmt@@3QBGB 5f8a0540  
 0002:00007568       ?_afxShellPrintFmt@@3QBGB  5f8a0568  
 0002:0000758c       ?_afxShellOpenFmt@@3QBGB   5f8a058c  
 0002:000075b4       ??_7CMDIChildWnd@@6B@      5f8a05b4  
 0002:000076b8       ??_R1A@?0A@A@CMDIChildWnd@@8 5f8a06b8  
 0002:000076d0       ??_R2CMDIChildWnd@@8       5f8a06d0  
 0002:000076e8       ??_R3CMDIChildWnd@@8       5f8a06e8  
 0002:000076f8       ??_R4CMDIChildWnd@@6B@     5f8a06f8  
 0002:00007788       ??_7XDropTarget@COleDropTarget@@6B@ 5f8a0788  
 0002:000077a8       ??_R1A@?0A@A@IDropTarget@@8 5f8a07a8  
 0002:000077c0       ??_R1A@?0A@A@XDropTarget@COleDropTarget@@8 5f8a07c0  
 0002:000077d8       ??_R2XDropTarget@COleDropTarget@@8 5f8a07d8  
 0002:000077e8       ??_R3XDropTarget@COleDropTarget@@8 5f8a07e8  
 0002:000077f8       ??_R4XDropTarget@COleDropTarget@@6B@ 5f8a07f8  
 0002:00007810       ?classCMDIChildWnd@CMDIChildWnd@@2UCRuntimeClass@@B 5f8a0810  
 0002:00007828       ??_C@_0N@NPHP@CMDIChildWnd?$AA@ 5f8a0828  
 0002:00007838       ?classCFrameWnd@CFrameWnd@@2UCRuntimeClass@@B 5f8a0838  
 0002:00007850       ??_C@_09HNKJ@CFrameWnd?$AA@ 5f8a0850  
 0002:0000785c       ?_afxRetVal@@3QBIB         5f8a085c  
 0002:00007898       ?_afxByRef@@3QBIB          5f8a0898  
 0002:000078d4       ?_afxByValue@@3QBIB        5f8a08d4  
 0002:0000790c       ??_C@_1BE@IDHE@?$AAE?$AAm?$AAb?$AAe?$AAd?$AAd?$AAi?$AAn?$AAg?$AA?$AA@ 5f8a090c  
 0002:00007924       ??_7COleDispatchImpl@@6B@  5f8a0924  
 0002:00007948       ??_R1A@?0A@A@IDispatch@@8  5f8a0948  
 0002:00007960       ??_R1A@?0A@A@COleDispatchImpl@@8 5f8a0960  
 0002:00007978       ??_R2COleDispatchImpl@@8   5f8a0978  
 0002:00007988       ??_R3COleDispatchImpl@@8   5f8a0988  
 0002:00007998       ??_R4COleDispatchImpl@@6B@ 5f8a0998  
 0002:000079b0       __sz_OLEAUT32              5f8a09b0  
 0002:000079c4       ??_C@_1BG@GHOC@?$AAA?$AAu?$AAt?$AAo?$AAm?$AAa?$AAt?$AAi?$AAo?$AAn?$AA?$AA@ 5f8a09c4  
 0002:000079e0       ??_7CEdit@@6B@             5f8a09e0  
 0002:00007aa0       ??_R1A@?0A@A@CEdit@@8      5f8a0aa0  
 0002:00007ab8       ??_R2CEdit@@8              5f8a0ab8  
 0002:00007ad0       ??_R3CEdit@@8              5f8a0ad0  
 0002:00007ae0       ??_R4CEdit@@6B@            5f8a0ae0  
 0002:00007af8       ??_7CStatic@@6B@           5f8a0af8  
 0002:00007bb8       ??_R1A@?0A@A@CStatic@@8    5f8a0bb8  
 0002:00007bd0       ??_R2CStatic@@8            5f8a0bd0  
 0002:00007be8       ??_R3CStatic@@8            5f8a0be8  
 0002:00007bf8       ??_R4CStatic@@6B@          5f8a0bf8  
 0002:00007c10       ?classCNotSupportedException@CNotSupportedException@@2UCRuntimeClass@@B 5f8a0c10  
 0002:00007c28       ??_C@_0BH@JODH@CNotSupportedException?$AA@ 5f8a0c28  
 0002:00007c40       ?classCMemoryException@CMemoryException@@2UCRuntimeClass@@B 5f8a0c40  
 0002:00007c58       ??_C@_0BB@NODM@CMemoryException?$AA@ 5f8a0c58  
 0002:00007c70       ?classCException@CException@@2UCRuntimeClass@@B 5f8a0c70  
 0002:00007c88       ??_C@_0L@CMNH@CException?$AA@ 5f8a0c88  
 0002:00007c94       ??_C@_1O@DAJD@?$AA?$CI?$AAN?$AAU?$AAL?$AAL?$AA?$CJ?$AA?$AA@ 5f8a0c94  
 0002:00007ca4       ??_C@_15NIED@?$AA?$CF?$AAu?$AA?$AA@ 5f8a0ca4  
 0002:00007cac       ??_C@_19JHMD@?$AA0?$AAx?$AA?$CF?$AAX?$AA?$AA@ 5f8a0cac  
 0002:00007cb8       ??_C@_17EFBD@?$AA?$CF?$AAl?$AAd?$AA?$AA@ 5f8a0cb8  
 0002:00007cc0       ??_C@_17DGGP@?$AA?$CF?$AAl?$AAu?$AA?$AA@ 5f8a0cc0  
 0002:00007cc8       ??_C@_19KF@?$AAN?$AAU?$AAL?$AAL?$AA?$AA@ 5f8a0cc8  
 0002:00007cd4       ??_C@_19LOGG@?$AA$?$AA?$CF?$AAl?$AAX?$AA?$AA@ 5f8a0cd4  
 0002:00007ce0       ??_C@_13DEJI@?$AA?6?$AA?$AA@ 5f8a0ce0  
 0002:00007ce4       ??_C@_1M@JKLL@?$AA?5?$AA?$CF?$AA0?$AA2?$AAX?$AA?$AA@ 5f8a0ce4  
 0002:00007cf0       ?classCArchiveException@CArchiveException@@2UCRuntimeClass@@B 5f8a0cf0  
 0002:00007d08       ??_C@_0BC@BIF@CArchiveException?$AA@ 5f8a0d08  
 0002:00007d20       ??_7CArchiveException@@6B@ 5f8a0d20  
 0002:00007d40       ??_7CArchiveStream@@6B@    5f8a0d40  
 0002:00007d78       ?classCFile@CFile@@2UCRuntimeClass@@B 5f8a0d78  
 0002:00007d90       ??_C@_05GM@CFile?$AA@      5f8a0d90  
 0002:00007d98       _afxIID_IShellLinkW        5f8a0d98  
 0002:00007da8       _afxCLSID_ShellLink        5f8a0da8  
 0002:00007db8       ??_C@_0BC@KFKC@DllGetClassObject?$AA@ 5f8a0db8  
 0002:00007dcc       ??_C@_1GG@OAL@?$AA?$HL?$AA?$CF?$AA0?$AA8?$AAX?$AA?9?$AA?$CF?$AA0?$AA4?$AAX?$AA?9?$AA?$CF?$AA0?$AA4?$AAX?$AA?9?$AA?$CF?$AA0?$AA2?$AAX@ 5f8a0dcc  
 0002:00007e34       ??_C@_1BO@DEPG@?$AAI?$AAn?$AAP?$AAr?$AAo?$AAc?$AAS?$AAe?$AAr?$AAv?$AAe?$AAr?$AA3?$AA2?$AA?$AA@ 5f8a0e34  
 0002:00007e58       ?classCStdioFile@CStdioFile@@2UCRuntimeClass@@B 5f8a0e58  
 0002:00007e70       ??_C@_0L@JAPO@CStdioFile?$AA@ 5f8a0e70  
 0002:00007e80       ??_7CStdioFile@@6B@        5f8a0e80  
 0002:00007ee8       ?classCMemFile@CMemFile@@2UCRuntimeClass@@B 5f8a0ee8  
 0002:00007f00       ??_C@_08EMMO@CMemFile?$AA@ 5f8a0f00  
 0002:00007f10       ?classCSharedFile@CSharedFile@@2UCRuntimeClass@@B 5f8a0f10  
 0002:00007f28       ??_C@_0M@DHDK@CSharedFile?$AA@ 5f8a0f28  
 0002:00007f38       ??_7CSharedFile@@6B@       5f8a0f38  
 0002:00007fa8       ?classCFileException@CFileException@@2UCRuntimeClass@@B 5f8a0fa8  
 0002:00007fc0       ??_C@_0P@HFKI@CFileException?$AA@ 5f8a0fc0  
 0002:00007fd4       ??_7CByteArray@@6B@        5f8a0fd4  
 0002:00007fe8       ?classCPtrArray@CPtrArray@@2UCRuntimeClass@@B 5f8a0fe8  
 0002:00008000       ??_C@_09BHCJ@CPtrArray?$AA@ 5f8a1000  
 0002:00008010       ??_7CObArray@@6B@          5f8a1010  
 0002:00008028       ??_7CStringArray@@6B@      5f8a1028  
 0002:00008040       ?classCUIntArray@CUIntArray@@2UCRuntimeClass@@B 5f8a1040  
 0002:00008058       ??_C@_0L@OIGA@CUIntArray?$AA@ 5f8a1058  
 0002:00008068       ??_7CUIntArray@@6B@        5f8a1068  
 0002:00008080       ??_7CWordArray@@6B@        5f8a1080  
 0002:00008098       ?classCPtrList@CPtrList@@2UCRuntimeClass@@B 5f8a1098  
 0002:000080b0       ??_C@_08DEKG@CPtrList?$AA@ 5f8a10b0  
 0002:000080c0       ??_7CStringList@@6B@       5f8a10c0  
 0002:000080d8       ?classCMapPtrToPtr@CMapPtrToPtr@@2UCRuntimeClass@@B 5f8a10d8  
 0002:000080f0       ??_C@_0N@EGND@CMapPtrToPtr?$AA@ 5f8a10f0  
 0002:00008100       ?classCMapPtrToWord@CMapPtrToWord@@2UCRuntimeClass@@B 5f8a1100  
 0002:00008118       ??_C@_0O@CNGA@CMapPtrToWord?$AA@ 5f8a1118  
 0002:0000812c       ??_7CMapPtrToWord@@6B@     5f8a112c  
 0002:00008144       ??_7CMapStringToOb@@6B@    5f8a1144  
 0002:00008158       ?classCMapStringToPtr@CMapStringToPtr@@2UCRuntimeClass@@B 5f8a1158  
 0002:00008170       ??_C@_0BA@PAMN@CMapStringToPtr?$AA@ 5f8a1170  
 0002:00008184       ??_7CMapStringToString@@6B@ 5f8a1184  
 0002:0000819c       ??_7CMapWordToOb@@6B@      5f8a119c  
 0002:000081b0       ?classCMapWordToPtr@CMapWordToPtr@@2UCRuntimeClass@@B 5f8a11b0  
 0002:000081c8       ??_C@_0O@MJKP@CMapWordToPtr?$AA@ 5f8a11c8  
 0002:000081dc       ??_7CMapWordToPtr@@6B@     5f8a11dc  
 0002:000081f0       ??_C@_19HABD@?$AA?$CF?$AA0?$AA2?$AAd?$AA?$AA@ 5f8a11f0  
 0002:00008200       ?classCSyncObject@CSyncObject@@2UCRuntimeClass@@B 5f8a1200  
 0002:00008218       ??_C@_0M@EHIL@CSyncObject?$AA@ 5f8a1218  
 0002:00008228       ?classCCriticalSection@CCriticalSection@@2UCRuntimeClass@@B 5f8a1228  
 0002:00008240       ??_C@_0BB@HCJ@CCriticalSection?$AA@ 5f8a1240  
 0002:00008258       ?classCMutex@CMutex@@2UCRuntimeClass@@B 5f8a1258  
 0002:00008270       ??_C@_06HCIL@CMutex?$AA@   5f8a1270  
 0002:00008278       ?classCSemaphore@CSemaphore@@2UCRuntimeClass@@B 5f8a1278  
 0002:00008290       ??_C@_0L@NFMO@CSemaphore?$AA@ 5f8a1290  
 0002:000082a0       ?classCEvent@CEvent@@2UCRuntimeClass@@B 5f8a12a0  
 0002:000082b8       ??_C@_06BPGE@CEvent?$AA@   5f8a12b8  
 0002:000082c4       ??_7CSemaphore@@6B@        5f8a12c4  
 0002:000082e8       ??_7CMutex@@6B@            5f8a12e8  
 0002:0000830c       ??_7CEvent@@6B@            5f8a130c  
 0002:0000832c       ?_afxWnd@@3QBGB            5f8a132c  
 0002:00008340       ?_afxWndOleControl@@3QBGB  5f8a1340  
 0002:00008364       ??_C@_0BA@OPCN@GetMonitorInfoW?$AA@ 5f8a1364  
 0002:00008374       ??_C@_0BE@KPOG@EnumDisplayMonitors?$AA@ 5f8a1374  
 0002:00008388       ??_C@_0BB@GJCM@MonitorFromPoint?$AA@ 5f8a1388  
 0002:0000839c       ??_C@_0BA@GOHF@MonitorFromRect?$AA@ 5f8a139c  
 0002:000083ac       ??_C@_1BA@FHJ@?$AAD?$AAI?$AAS?$AAP?$AAL?$AAA?$AAY?$AA?$AA@ 5f8a13ac  
 0002:000083bc       ??_C@_1BE@KCHN@?$AAA?$AAf?$AAx?$AA?3?$AA?$CF?$AAx?$AA?3?$AA?$CF?$AAx?$AA?$AA@ 5f8a13bc  
 0002:000083d0       ?classCControlBar@CControlBar@@2UCRuntimeClass@@B 5f8a13d0  
 0002:000083e8       ??_C@_0M@GCON@CControlBar?$AA@ 5f8a13e8  
 0002:000083f4       ??_C@_1CA@JHCA@?$AAM?$AAS?$AAW?$AAH?$AAE?$AAE?$AAL?$AA_?$AAR?$AAO?$AAL?$AAL?$AAM?$AAS?$AAG?$AA?$AA@ 5f8a13f4  
 0002:00008414       ??_C@_17LJFH@?$AA?3?$AA?$CF?$AAd?$AA?$AA@ 5f8a1414  
 0002:00008420       ?classCMDIFrameWnd@CMDIFrameWnd@@2UCRuntimeClass@@B 5f8a1420  
 0002:00008438       ??_C@_0N@FPEB@CMDIFrameWnd?$AA@ 5f8a1438  
 0002:00008448       ?messageMap@CMDIFrameWnd@@1UAFX_MSGMAP@@B 5f8a1448  
 0002:00008450       ?_messageEntries@CMDIFrameWnd@@0QBUAFX_MSGMAP_ENTRY@@B 5f8a1450  
 0002:000085d0       ?classCToolTipCtrl@CToolTipCtrl@@2UCRuntimeClass@@B 5f8a15d0  
 0002:000085e8       ??_C@_0N@OELH@CToolTipCtrl?$AA@ 5f8a15e8  
 0002:000085f8       ?messageMap@CToolTipCtrl@@1UAFX_MSGMAP@@B 5f8a15f8  
 0002:00008600       ?_messageEntries@CToolTipCtrl@@0QBUAFX_MSGMAP_ENTRY@@B 5f8a1600  
 0002:0000867c       ??_7CToolTipCtrl@@6B@      5f8a167c  
 0002:0000873c       ??_C@_1CC@BIKB@?$AAt?$AAo?$AAo?$AAl?$AAt?$AAi?$AAp?$AAs?$AA_?$AAc?$AAl?$AAa?$AAs?$AAs?$AA3?$AA2?$AA?$AA@ 5f8a173c  
 0002:00008760       ?classCMiniFrameWnd@CMiniFrameWnd@@2UCRuntimeClass@@B 5f8a1760  
 0002:00008778       ??_C@_0O@NPLL@CMiniFrameWnd?$AA@ 5f8a1778  
 0002:00008788       ?messageMap@CMiniFrameWnd@@1UAFX_MSGMAP@@B 5f8a1788  
 0002:00008790       ?_messageEntries@CMiniFrameWnd@@0QBUAFX_MSGMAP_ENTRY@@B 5f8a1790  
 0002:00008914       ??_7CMiniFrameWnd@@6B@     5f8a1914  
 0002:00008a10       ??_C@_1BI@PPN@?$AAS?$AAm?$AAa?$AAl?$AAl?$AA?5?$AAF?$AAo?$AAn?$AAt?$AAs?$AA?$AA@ 5f8a1a10  
 0002:00008a28       ??_C@_1BC@NHJA@?$AAT?$AAe?$AAr?$AAm?$AAi?$AAn?$AAa?$AAl?$AA?$AA@ 5f8a1a28  
 0002:00008a40       ??_7CBrush@@6B@            5f8a1a40  
 0002:00008a58       ?classCToolBar@CToolBar@@2UCRuntimeClass@@B 5f8a1a58  
 0002:00008a70       ??_C@_08NCEL@CToolBar?$AA@ 5f8a1a70  
 0002:00008a80       ?classCDialogBar@CDialogBar@@2UCRuntimeClass@@B 5f8a1a80  
 0002:00008a98       ??_C@_0L@KJOE@CDialogBar?$AA@ 5f8a1a98  
 0002:00008aa8       ?messageMap@CDialogBar@@1UAFX_MSGMAP@@B 5f8a1aa8  
 0002:00008ab0       ?_messageEntries@CDialogBar@@0QBUAFX_MSGMAP_ENTRY@@B 5f8a1ab0  
 0002:00008ae4       ??_7CDialogBar@@6B@        5f8a1ae4  
 0002:00008bd0       ?classCStatusBar@CStatusBar@@2UCRuntimeClass@@B 5f8a1bd0  
 0002:00008be8       ??_C@_0L@BNMI@CStatusBar?$AA@ 5f8a1be8  
 0002:00008bf8       ?classCDockBar@CDockBar@@2UCRuntimeClass@@B 5f8a1bf8  
 0002:00008c10       ??_C@_08EABA@CDockBar?$AA@ 5f8a1c10  
 0002:00008c20       ?messageMap@CMiniDockFrameWnd@@1UAFX_MSGMAP@@B 5f8a1c20  
 0002:00008c28       ?_messageEntries@CMiniDockFrameWnd@@0QBUAFX_MSGMAP_ENTRY@@B 5f8a1c28  
 0002:00008ca4       ??_7CMiniDockFrameWnd@@6B@ 5f8a1ca4  
 0002:00008da4       ?_afxBar@@3QBGB            5f8a1da4  
 0002:00008db4       ?_afxScreenCY@@3QBGB       5f8a1db4  
 0002:00008dc8       ?_afxScreenCX@@3QBGB       5f8a1dc8  
 0002:00008ddc       ?_afxBars@@3QBGB           5f8a1ddc  
 0002:00008de8       ?_afxFloating@@3QBGB       5f8a1de8  
 0002:00008dfc       ?_afxHorz@@3QBGB           5f8a1dfc  
 0002:00008e08       ?_afxBarID@@3QBGB          5f8a1e08  
 0002:00008e14       ?_afxMRUFloatYPos@@3QBGB   5f8a1e14  
 0002:00008e30       ?_afxMRUFloatXPos@@3QBGB   5f8a1e30  
 0002:00008e4c       ?_afxMRUFloatStyle@@3QBGB  5f8a1e4c  
 0002:00008e68       ?_afxMRUDockBottomPos@@3QBGB 5f8a1e68  
 0002:00008e8c       ?_afxMRUDockTopPos@@3QBGB  5f8a1e8c  
 0002:00008ea8       ?_afxMRUDockRightPos@@3QBGB 5f8a1ea8  
 0002:00008ec8       ?_afxMRUDockLeftPos@@3QBGB 5f8a1ec8  
 0002:00008ee8       ?_afxMRUDockID@@3QBGB      5f8a1ee8  
 0002:00008efc       ?_afxDocking@@3QBGB        5f8a1efc  
 0002:00008f0c       ?_afxMRUWidth@@3QBGB       5f8a1f0c  
 0002:00008f20       ?_afxYPos@@3QBGB           5f8a1f20  
 0002:00008f2c       ?_afxXPos@@3QBGB           5f8a1f2c  
 0002:00008f38       ?_afxSummarySection@@3QBGB 5f8a1f38  
 0002:00008f50       ?_afxBarSection@@3QBGB     5f8a1f50  
 0002:00008f64       ?_afxVisible@@3QBGB        5f8a1f64  
 0002:00008f78       ?classCPreviewDC@CPreviewDC@@2UCRuntimeClass@@B 5f8a1f78  
 0002:00008f90       ??_C@_0L@MCGA@CPreviewDC?$AA@ 5f8a1f90  
 0002:00008fa0       ??_7CPreviewDC@@6B@        5f8a1fa0  
 0002:0000901c       ??_C@_01POCP@?7?$AA@       5f8a201c  
 0002:0000901e       ??_C@_01PFH@A?$AA@         5f8a201e  
 0002:00009020       ?classCMetaFileDC@CMetaFileDC@@2UCRuntimeClass@@B 5f8a2020  
 0002:00009038       ??_C@_0M@MIEC@CMetaFileDC?$AA@ 5f8a2038  
 0002:00009048       ??_7CMetaFileDC@@6B@       5f8a2048  
 0002:00009100       ?_afxRectInfo@@3QBUAFX_RECTINFO@@B 5f8a2100  
 0002:00009120       ?_afxHandleInfo@@3QBUAFX_HANDLEINFO@@B 5f8a2120  
 0002:00009224       ??_7CRectTracker@@6B@      5f8a2224  
 0002:00009240       ?classCReBar@CReBar@@2UCRuntimeClass@@B 5f8a2240  
 0002:00009258       ??_C@_06JANL@CReBar?$AA@   5f8a2258  
 0002:00009260       ?messageMap@CReBar@@1UAFX_MSGMAP@@B 5f8a2260  
 0002:00009268       ?_messageEntries@CReBar@@0QBUAFX_MSGMAP_ENTRY@@B 5f8a2268  
 0002:0000935c       ??_7CReBar@@6B@            5f8a235c  
 0002:00009444       ??_C@_1BM@CPLN@?$AAR?$AAe?$AAB?$AAa?$AAr?$AAW?$AAi?$AAn?$AAd?$AAo?$AAw?$AA3?$AA2?$AA?$AA@ 5f8a2444  
 0002:00009460       ?classCScrollBar@CScrollBar@@2UCRuntimeClass@@B 5f8a2460  
 0002:00009478       ??_C@_0L@JCLK@CScrollBar?$AA@ 5f8a2478  
 0002:00009488       ?classCEdit@CEdit@@2UCRuntimeClass@@B 5f8a2488  
 0002:000094a0       ??_C@_05KKIE@CEdit?$AA@    5f8a24a0  
 0002:000094a8       ?classCComboBox@CComboBox@@2UCRuntimeClass@@B 5f8a24a8  
 0002:000094c0       ??_C@_09JMHE@CComboBox?$AA@ 5f8a24c0  
 0002:000094d0       ?classCListBox@CListBox@@2UCRuntimeClass@@B 5f8a24d0  
 0002:000094e8       ??_C@_08NBK@CListBox?$AA@  5f8a24e8  
 0002:000094f8       ?classCButton@CButton@@2UCRuntimeClass@@B 5f8a24f8  
 0002:00009510       ??_C@_07NNHJ@CButton?$AA@  5f8a2510  
 0002:00009518       ?classCStatic@CStatic@@2UCRuntimeClass@@B 5f8a2518  
 0002:00009530       ??_C@_07HEEJ@CStatic?$AA@  5f8a2530  
 0002:00009538       ??_C@_1O@GCMM@?$AAS?$AAT?$AAA?$AAT?$AAI?$AAC?$AA?$AA@ 5f8a2538  
 0002:00009548       ??_C@_1O@GKDM@?$AAB?$AAU?$AAT?$AAT?$AAO?$AAN?$AA?$AA@ 5f8a2548  
 0002:00009558       ??_C@_1BA@BJGI@?$AAL?$AAI?$AAS?$AAT?$AAB?$AAO?$AAX?$AA?$AA@ 5f8a2558  
 0002:0000956c       ??_7CListBox@@6B@          5f8a256c  
 0002:00009644       ??_C@_19CJM@?$AAE?$AAD?$AAI?$AAT?$AA?$AA@ 5f8a2644  
 0002:00009650       ??_C@_1BE@JGEP@?$AAS?$AAC?$AAR?$AAO?$AAL?$AAL?$AAB?$AAA?$AAR?$AA?$AA@ 5f8a2650  
 0002:00009668       ??_7CScrollBar@@6B@        5f8a2668  
 0002:00009728       ?classCRichEditCtrl@CRichEditCtrl@@2UCRuntimeClass@@B 5f8a2728  
 0002:00009740       ??_C@_0O@KLOD@CRichEditCtrl?$AA@ 5f8a2740  
 0002:00009750       ?classCTempImageList@CTempImageList@@2UCRuntimeClass@@B 5f8a2750  
 0002:00009768       ??_C@_0P@OCOD@CTempImageList?$AA@ 5f8a2768  
 0002:00009778       ?classCImageList@CImageList@@2UCRuntimeClass@@B 5f8a2778  
 0002:00009790       ??_C@_0L@HBAH@CImageList?$AA@ 5f8a2790  
 0002:000097a0       ?classCStatusBarCtrl@CStatusBarCtrl@@2UCRuntimeClass@@B 5f8a27a0  
 0002:000097b8       ??_C@_0P@NMO@CStatusBarCtrl?$AA@ 5f8a27b8  
 0002:000097c8       ?classCToolBarCtrl@CToolBarCtrl@@2UCRuntimeClass@@B 5f8a27c8  
 0002:000097e0       ??_C@_0N@HNL@CToolBarCtrl?$AA@ 5f8a27e0  
 0002:000097f0       ?classCListCtrl@CListCtrl@@2UCRuntimeClass@@B 5f8a27f0  
 0002:00009808       ??_C@_09IAHO@CListCtrl?$AA@ 5f8a2808  
 0002:00009818       ?classCTreeCtrl@CTreeCtrl@@2UCRuntimeClass@@B 5f8a2818  
 0002:00009830       ??_C@_09CIBI@CTreeCtrl?$AA@ 5f8a2830  
 0002:00009840       ?classCTabCtrl@CTabCtrl@@2UCRuntimeClass@@B 5f8a2840  
 0002:00009858       ??_C@_08IFFI@CTabCtrl?$AA@ 5f8a2858  
 0002:00009868       ?classCAnimateCtrl@CAnimateCtrl@@2UCRuntimeClass@@B 5f8a2868  
 0002:00009880       ??_C@_0N@PPEM@CAnimateCtrl?$AA@ 5f8a2880  
 0002:00009890       ?classCHotKeyCtrl@CHotKeyCtrl@@2UCRuntimeClass@@B 5f8a2890  
 0002:000098a8       ??_C@_0M@IPHC@CHotKeyCtrl?$AA@ 5f8a28a8  
 0002:000098b8       ?classCHeaderCtrl@CHeaderCtrl@@2UCRuntimeClass@@B 5f8a28b8  
 0002:000098d0       ??_C@_0M@HNGK@CHeaderCtrl?$AA@ 5f8a28d0  
 0002:000098e0       ?classCComboBoxEx@CComboBoxEx@@2UCRuntimeClass@@B 5f8a28e0  
 0002:000098f8       ??_C@_0M@BDBF@CComboBoxEx?$AA@ 5f8a28f8  
 0002:00009908       ?classCProgressCtrl@CProgressCtrl@@2UCRuntimeClass@@B 5f8a2908  
 0002:00009920       ??_C@_0O@ECFI@CProgressCtrl?$AA@ 5f8a2920  
 0002:00009930       ?classCSliderCtrl@CSliderCtrl@@2UCRuntimeClass@@B 5f8a2930  
 0002:00009948       ??_C@_0M@POGH@CSliderCtrl?$AA@ 5f8a2948  
 0002:00009958       ?classCSpinButtonCtrl@CSpinButtonCtrl@@2UCRuntimeClass@@B 5f8a2958  
 0002:00009970       ??_C@_0BA@MANL@CSpinButtonCtrl?$AA@ 5f8a2970  
 0002:00009980       ?classCDragListBox@CDragListBox@@2UCRuntimeClass@@B 5f8a2980  
 0002:00009998       ??_C@_0N@BPBM@CDragListBox?$AA@ 5f8a2998  
 0002:000099a8       ?messageMap@CTabCtrl@@1UAFX_MSGMAP@@B 5f8a29a8  
 0002:000099b0       ?_messageEntries@CTabCtrl@@0QBUAFX_MSGMAP_ENTRY@@B 5f8a29b0  
 0002:000099e0       ?messageMap@CTreeCtrl@@1UAFX_MSGMAP@@B 5f8a29e0  
 0002:000099e8       ?_messageEntries@CTreeCtrl@@0QBUAFX_MSGMAP_ENTRY@@B 5f8a29e8  
 0002:00009a18       ?messageMap@CListCtrl@@1UAFX_MSGMAP@@B 5f8a2a18  
 0002:00009a20       ?_messageEntries@CListCtrl@@0QBUAFX_MSGMAP_ENTRY@@B 5f8a2a20  
 0002:00009a50       ?messageMap@CToolBarCtrl@@1UAFX_MSGMAP@@B 5f8a2a50  
 0002:00009a58       ?_messageEntries@CToolBarCtrl@@0QBUAFX_MSGMAP_ENTRY@@B 5f8a2a58  
 0002:00009a8c       ??_7CDragListBox@@6B@      5f8a2a8c  
 0002:00009b7c       ??_7CRgn@@6B@              5f8a2b7c  
 0002:00009b94       ??_7CToolBarCtrl@@6B@      5f8a2b94  
 0002:00009c58       ??_7CStatusBarCtrl@@6B@    5f8a2c58  
 0002:00009d1c       ??_C@_1BM@DGLL@?$AAS?$AAy?$AAs?$AAL?$AAi?$AAs?$AAt?$AAV?$AAi?$AAe?$AAw?$AA3?$AA2?$AA?$AA@ 5f8a2d1c  
 0002:00009d3c       ??_7CListCtrl@@6B@         5f8a2d3c  
 0002:00009e00       ??_C@_1BM@DBCI@?$AAS?$AAy?$AAs?$AAT?$AAr?$AAe?$AAe?$AAV?$AAi?$AAe?$AAw?$AA3?$AA2?$AA?$AA@ 5f8a2e00  
 0002:00009e20       ??_7CTreeCtrl@@6B@         5f8a2e20  
 0002:00009ee0       ??_C@_1CA@JDKO@?$AAm?$AAs?$AAc?$AAt?$AAl?$AAs?$AA_?$AAu?$AAp?$AAd?$AAo?$AAw?$AAn?$AA3?$AA2?$AA?$AA@ 5f8a2ee0  
 0002:00009f04       ??_7CSpinButtonCtrl@@6B@   5f8a2f04  
 0002:00009fc4       ??_C@_1CE@EHFJ@?$AAm?$AAs?$AAc?$AAt?$AAl?$AAs?$AA_?$AAt?$AAr?$AAa?$AAc?$AAk?$AAb?$AAa?$AAr?$AA3?$AA2?$AA?$AA@ 5f8a2fc4  
 0002:00009fec       ??_7CSliderCtrl@@6B@       5f8a2fec  
 0002:0000a0ac       ??_C@_1CE@ECOJ@?$AAm?$AAs?$AAc?$AAt?$AAl?$AAs?$AA_?$AAp?$AAr?$AAo?$AAg?$AAr?$AAe?$AAs?$AAs?$AA3?$AA2?$AA?$AA@ 5f8a30ac  
 0002:0000a0d4       ??_7CProgressCtrl@@6B@     5f8a30d4  
 0002:0000a194       ??_C@_1BI@FFDG@?$AAS?$AAy?$AAs?$AAH?$AAe?$AAa?$AAd?$AAe?$AAr?$AA3?$AA2?$AA?$AA@ 5f8a3194  
 0002:0000a1b0       ??_7CHeaderCtrl@@6B@       5f8a31b0  
 0002:0000a274       ??_C@_1CA@BKDN@?$AAm?$AAs?$AAc?$AAt?$AAl?$AAs?$AA_?$AAh?$AAo?$AAt?$AAk?$AAe?$AAy?$AA3?$AA2?$AA?$AA@ 5f8a3274  
 0002:0000a298       ??_7CHotKeyCtrl@@6B@       5f8a3298  
 0002:0000a358       ??_C@_1CA@OIHL@?$AAS?$AAy?$AAs?$AAT?$AAa?$AAb?$AAC?$AAo?$AAn?$AAt?$AAr?$AAo?$AAl?$AA3?$AA2?$AA?$AA@ 5f8a3358  
 0002:0000a37c       ??_7CTabCtrl@@6B@          5f8a337c  
 0002:0000a440       ??_C@_1BK@MPBJ@?$AAS?$AAy?$AAs?$AAA?$AAn?$AAi?$AAm?$AAa?$AAt?$AAe?$AA3?$AA2?$AA?$AA@ 5f8a3440  
 0002:0000a460       ??_7CAnimateCtrl@@6B@      5f8a3460  
 0002:0000a524       ??_7CRichEditCtrl@@6B@     5f8a3524  
 0002:0000a5e8       ??_7CImageList@@6B@        5f8a35e8  
 0002:0000a600       ??_7CTempImageList@@6B@    5f8a3600  
 0002:0000a618       ?classCCheckListBox@CCheckListBox@@2UCRuntimeClass@@B 5f8a3618  
 0002:0000a630       ??_C@_0O@KOFM@CCheckListBox?$AA@ 5f8a3630  
 0002:0000a640       ?messageMap@CCheckListBox@@1UAFX_MSGMAP@@B 5f8a3640  
 0002:0000a648       ?_messageEntries@CCheckListBox@@0QBUAFX_MSGMAP_ENTRY@@B 5f8a3648  
 0002:0000a7b4       ??_7CBitmap@@6B@           5f8a37b4  
 0002:0000a7cc       ??_7_AFX_CHECKLIST_STATE@@6B@ 5f8a37cc  
 0002:0000a7d0       ?classCBitmapButton@CBitmapButton@@2UCRuntimeClass@@B 5f8a37d0  
 0002:0000a7e8       ??_C@_0O@FPOC@CBitmapButton?$AA@ 5f8a37e8  
 0002:0000a7f8       ??_C@_13LOIM@?$AAU?$AA?$AA@ 5f8a37f8  
 0002:0000a7fc       ??_C@_13MNPA@?$AAD?$AA?$AA@ 5f8a37fc  
 0002:0000a800       ??_C@_13GJNN@?$AAF?$AA?$AA@ 5f8a3800  
 0002:0000a804       ??_C@_13DEHF@?$AAX?$AA?$AA@ 5f8a3804  
 0002:0000a808       ??_C@_19JGFH@?$AAE?$AAd?$AAi?$AAt?$AA?$AA@ 5f8a3808  
 0002:0000a814       ??_C@_19OFHG@?$AAH?$AAe?$AAl?$AAv?$AA?$AA@ 5f8a3814  
 0002:0000a820       ??_C@_1BM@LDDO@?$AAM?$AAS?$AA?5?$AAS?$AAa?$AAn?$AAs?$AA?5?$AAS?$AAe?$AAr?$AAi?$AAf?$AA?$AA@ 5f8a3820  
 0002:0000a83c       ??_C@_1BK@PLLM@?$AAM?$AAS?$AA?5?$AAS?$AAh?$AAe?$AAl?$AAl?$AA?5?$AAD?$AAl?$AAg?$AA?$AA@ 5f8a383c  
 0002:0000a858       ??_C@_17MFIG@?$AA?$CF?$AAh?$AAd?$AA?$AA@ 5f8a3858  
 0002:0000a860       ??_C@_17CGJG@?$AA?$CF?$AAs?$AAd?$AA?$AA@ 5f8a3860  
 0002:0000a868       __real@8@00000000000000000000 5f8a3868  
 0002:0000a870       ??_C@_19PPNN@?$AA?$CF?$AA?4?$AA?$CK?$AAg?$AA?$AA@ 5f8a3870  
 0002:0000a880       ?classCPropertySheetEx@CPropertySheetEx@@2UCRuntimeClass@@B 5f8a3880  
 0002:0000a898       ??_C@_0BB@NMHF@CPropertySheetEx?$AA@ 5f8a3898  
 0002:0000a8b0       ?classCPropertyPageEx@CPropertyPageEx@@2UCRuntimeClass@@B 5f8a38b0  
 0002:0000a8c8       ??_C@_0BA@MOPN@CPropertyPageEx?$AA@ 5f8a38c8  
 0002:0000a8d8       ?classCPropertySheet@CPropertySheet@@2UCRuntimeClass@@B 5f8a38d8  
 0002:0000a8f0       ??_C@_0P@PIP@CPropertySheet?$AA@ 5f8a38f0  
 0002:0000a900       ?classCPropertyPage@CPropertyPage@@2UCRuntimeClass@@B 5f8a3900  
 0002:0000a918       ??_C@_0O@DMH@CPropertyPage?$AA@ 5f8a3918  
 0002:0000a928       ?_afxPropSheetIDs@@3QBHB   5f8a3928  
 0002:0000a938       ?messageMap@CPropertySheet@@1UAFX_MSGMAP@@B 5f8a3938  
 0002:0000a940       ?_messageEntries@CPropertySheet@@0QBUAFX_MSGMAP_ENTRY@@B 5f8a3940  
 0002:0000aa00       ?messageMap@CPropertyPage@@1UAFX_MSGMAP@@B 5f8a3a00  
 0002:0000aa08       ?_messageEntries@CPropertyPage@@0QBUAFX_MSGMAP_ENTRY@@B 5f8a3a08  
 0002:0000aa54       ??_7CPropertyPage@@6B@     5f8a3a54  
 0002:0000ab50       ??_7CPropertySheet@@6B@    5f8a3b50  
 0002:0000ac20       ??_7CPropertyPageEx@@6B@   5f8a3c20  
 0002:0000ad1c       ??_7CPropertySheetEx@@6B@  5f8a3d1c  
 0002:0000ade8       ??_C@_1CI@HAOL@?$AAc?$AAo?$AAm?$AAm?$AAd?$AAl?$AAg?$AA_?$AAS?$AAe?$AAt?$AAR?$AAG?$AAB?$AAC?$AAo?$AAl?$AAo?$AAr?$AA?$AA@ 5f8a3de8  
 0002:0000ae10       ??_C@_1BK@KCME@?$AAc?$AAo?$AAm?$AAm?$AAd?$AAl?$AAg?$AA_?$AAh?$AAe?$AAl?$AAp?$AA?$AA@ 5f8a3e10  
 0002:0000ae2c       ??_C@_1CA@HL@?$AAc?$AAo?$AAm?$AAm?$AAd?$AAl?$AAg?$AA_?$AAC?$AAo?$AAl?$AAo?$AAr?$AAO?$AAK?$AA?$AA@ 5f8a3e2c  
 0002:0000ae4c       ??_C@_1CG@GOBL@?$AAc?$AAo?$AAm?$AAm?$AAd?$AAl?$AAg?$AA_?$AAF?$AAi?$AAl?$AAe?$AAN?$AAa?$AAm?$AAe?$AAO?$AAK?$AA?$AA@ 5f8a3e4c  
 0002:0000ae74       ??_C@_1CO@EDLA@?$AAc?$AAo?$AAm?$AAm?$AAd?$AAl?$AAg?$AA_?$AAS?$AAh?$AAa?$AAr?$AAe?$AAV?$AAi?$AAo?$AAl?$AAa?$AAt?$AAi@ 5f8a3e74  
 0002:0000aea4       ??_C@_1DG@FJGG@?$AAc?$AAo?$AAm?$AAm?$AAd?$AAl?$AAg?$AA_?$AAL?$AAB?$AAS?$AAe?$AAl?$AAC?$AAh?$AAa?$AAn?$AAg?$AAe?$AAd@ 5f8a3ea4  
 0002:0000aee0       ?classCFileDialog@CFileDialog@@2UCRuntimeClass@@B 5f8a3ee0  
 0002:0000aef8       ??_C@_0M@JEJA@CFileDialog?$AA@ 5f8a3ef8  
 0002:0000af08       ??_7CFileDialog@@6B@       5f8a3f08  
 0002:0000b000       ??_7CCommonDialog@@6B@     5f8a4000  
 0002:0000b0d8       ?classCPageSetupDialog@CPageSetupDialog@@2UCRuntimeClass@@B 5f8a40d8  
 0002:0000b0f0       ??_C@_0BB@KMEP@CPageSetupDialog?$AA@ 5f8a40f0  
 0002:0000b108       ?classCPrintDialog@CPrintDialog@@2UCRuntimeClass@@B 5f8a4108  
 0002:0000b120       ??_C@_0N@KDJG@CPrintDialog?$AA@ 5f8a4120  
 0002:0000b134       ??_7CPageSetupDialog@@6B@  5f8a4134  
 0002:0000b218       ?classCColorDialog@CColorDialog@@2UCRuntimeClass@@B 5f8a4218  
 0002:0000b230       ??_C@_0N@GCDM@CColorDialog?$AA@ 5f8a4230  
 0002:0000b240       ?messageMap@CColorDialog@@1UAFX_MSGMAP@@B 5f8a4240  
 0002:0000b248       ?_messageEntries@CColorDialog@@0QBUAFX_MSGMAP_ENTRY@@B 5f8a4248  
 0002:0000b27c       ??_7_AFX_COLOR_STATE@@6B@  5f8a427c  
 0002:0000b284       ??_7CColorDialog@@6B@      5f8a4284  
 0002:0000b360       ?classCFontDialog@CFontDialog@@2UCRuntimeClass@@B 5f8a4360  
 0002:0000b378       ??_C@_0M@EOLC@CFontDialog?$AA@ 5f8a4378  
 0002:0000b388       ??_7CFontDialog@@6B@       5f8a4388  
 0002:0000b460       ?classCFindReplaceDialog@CFindReplaceDialog@@2UCRuntimeClass@@B 5f8a4460  
 0002:0000b478       ??_C@_0BD@HPIP@CFindReplaceDialog?$AA@ 5f8a4478  
 0002:0000b490       ??_7CFindReplaceDialog@@6B@ 5f8a4490  
 0002:0000b56c       ??_7_AFX_PROPPAGEFONTINFO@@6B@ 5f8a456c  
 0002:0000b570       ??_C@_1GK@FNIL@?$AAA?$AAB?$AAC?$AAD?$AAE?$AAF?$AAG?$AAH?$AAI?$AAJ?$AAK?$AAL?$AAM?$AAN?$AAO?$AAP?$AAQ?$AAR?$AAS?$AAT@ 5f8a4570  
 0002:0000b5dc       ??_C@_1O@KHFL@?$AAS?$AAy?$AAs?$AAt?$AAe?$AAm?$AA?$AA@ 5f8a45dc  
 0002:0000b5f0       ?classCReBarCtrl@CReBarCtrl@@2UCRuntimeClass@@B 5f8a45f0  
 0002:0000b608       ??_C@_0L@GONC@CReBarCtrl?$AA@ 5f8a4608  
 0002:0000b618       ?classCIPAddressCtrl@CIPAddressCtrl@@2UCRuntimeClass@@B 5f8a4618  
 0002:0000b630       ??_C@_0P@PBFM@CIPAddressCtrl?$AA@ 5f8a4630  
 0002:0000b644       ??_7CIPAddressCtrl@@6B@    5f8a4644  
 0002:0000b704       ??_C@_1BO@OJBJ@?$AAS?$AAy?$AAs?$AAI?$AAP?$AAA?$AAd?$AAd?$AAr?$AAe?$AAs?$AAs?$AA3?$AA2?$AA?$AA@ 5f8a4704  
 0002:0000b724       ??_C@_1BK@JEIN@?$AAC?$AAo?$AAm?$AAb?$AAo?$AAB?$AAo?$AAx?$AAE?$AAx?$AA3?$AA2?$AA?$AA@ 5f8a4724  
 0002:0000b744       ??_7CComboBoxEx@@6B@       5f8a4744  
 0002:0000b818       ?classCRgn@CRgn@@2UCRuntimeClass@@B 5f8a4818  
 0002:0000b830       ??_C@_04HJNG@CRgn?$AA@     5f8a4830  
 0002:0000b838       ?classCPalette@CPalette@@2UCRuntimeClass@@B 5f8a4838  
 0002:0000b850       ??_C@_08CIF@CPalette?$AA@  5f8a4850  
 0002:0000b860       ?classCBitmap@CBitmap@@2UCRuntimeClass@@B 5f8a4860  
 0002:0000b878       ??_C@_07HNEL@CBitmap?$AA@  5f8a4878  
 0002:0000b880       ?classCFont@CFont@@2UCRuntimeClass@@B 5f8a4880  
 0002:0000b898       ??_C@_05MCKJ@CFont?$AA@    5f8a4898  
 0002:0000b8a0       ?classCBrush@CBrush@@2UCRuntimeClass@@B 5f8a48a0  
 0002:0000b8b8       ??_C@_06PNF@CBrush?$AA@    5f8a48b8  
 0002:0000b8c0       ?classCPen@CPen@@2UCRuntimeClass@@B 5f8a48c0  
 0002:0000b8d8       ??_C@_04PAKO@CPen?$AA@     5f8a48d8  
 0002:0000b8e0       ?classCGdiObject@CGdiObject@@2UCRuntimeClass@@B 5f8a48e0  
 0002:0000b8f8       ??_C@_0L@CNBG@CGdiObject?$AA@ 5f8a48f8  
 0002:0000b908       ?classCPaintDC@CPaintDC@@2UCRuntimeClass@@B 5f8a4908  
 0002:0000b920       ??_C@_08HFDK@CPaintDC?$AA@ 5f8a4920  
 0002:0000b930       ?classCWindowDC@CWindowDC@@2UCRuntimeClass@@B 5f8a4930  
 0002:0000b948       ??_C@_09NFPO@CWindowDC?$AA@ 5f8a4948  
 0002:0000b958       ?classCClientDC@CClientDC@@2UCRuntimeClass@@B 5f8a4958  
 0002:0000b970       ??_C@_09HIEC@CClientDC?$AA@ 5f8a4970  
 0002:0000b980       ?classCDC@CDC@@2UCRuntimeClass@@B 5f8a4980  
 0002:0000b998       ??_C@_03NJOH@CDC?$AA@      5f8a4998  
 0002:0000b9a0       ?classCUserException@CUserException@@2UCRuntimeClass@@B 5f8a49a0  
 0002:0000b9b8       ??_C@_0P@BHHD@CUserException?$AA@ 5f8a49b8  
 0002:0000b9c8       ?classCResourceException@CResourceException@@2UCRuntimeClass@@B 5f8a49c8  
 0002:0000b9e0       ??_C@_0BD@GMHI@CResourceException?$AA@ 5f8a49e0  
 0002:0000b9f4       ??_C@_09EBEO@GetLayout?$AA@ 5f8a49f4  
 0002:0000ba00       ??_C@_09JDFO@GDI32?4DLL?$AA@ 5f8a4a00  
 0002:0000ba0c       ??_C@_09GMOM@SetLayout?$AA@ 5f8a4a0c  
 0002:0000ba1c       ??_7CPen@@6B@              5f8a4a1c  
 0002:0000ba30       ?classCMenu@CMenu@@2UCRuntimeClass@@B 5f8a4a30  
 0002:0000ba48       ??_C@_05BJMA@CMenu?$AA@    5f8a4a48  
 0002:0000ba50       ??_C@_1BC@EMPM@?$AAc?$AAo?$AAm?$AAb?$AAo?$AAb?$AAo?$AAx?$AA?$AA@ 5f8a4a50  
 0002:0000ba64       ?_afxDot@@3QBEB            5f8a4a64  
 0002:0000ba70       ?dispatchMap@CCmdTarget@@1UAFX_DISPMAP@@B 5f8a4a70  
 0002:0000ba80       ?_dispatchEntries@CCmdTarget@@0QBUAFX_DISPMAP_ENTRY@@B 5f8a4a80  
 0002:0000baa0       ?eventsinkMap@CCmdTarget@@1UAFX_EVENTSINKMAP@@B 5f8a4aa0  
 0002:0000bab0       ?_eventsinkEntries@CCmdTarget@@0QBUAFX_EVENTSINKMAP_ENTRY@@B 5f8a4ab0  
 0002:0000bad8       ?connectionMap@CCmdTarget@@1UAFX_CONNECTIONMAP@@B 5f8a4ad8  
 0002:0000bae0       ?_connectionEntries@CCmdTarget@@0QBUAFX_CONNECTIONMAP_ENTRY@@B 5f8a4ae0  
 0002:0000bae8       ?commandMap@CCmdTarget@@1UAFX_OLECMDMAP@@B 5f8a4ae8  
 0002:0000baf0       ?_commandEntries@CCmdTarget@@0QBUAFX_OLECMDMAP_ENTRY@@B 5f8a4af0  
 0002:0000bb00       ?classCDocument@CDocument@@2UCRuntimeClass@@B 5f8a4b00  
 0002:0000bb18       ??_C@_09IIIN@CDocument?$AA@ 5f8a4b18  
 0002:0000bb24       ??_C@_1O@OEBA@?$AA?5?$AA?$CD?$AA?$CF?$AA?$DL?$AA?1?$AA?2?$AA?$AA@ 5f8a4b24  
 0002:0000bb34       ??_C@_17PPBM@?$AAM?$AAF?$AAC?$AA?$AA@ 5f8a4b34  
 0002:0000bb3c       ??_C@_0M@JIL@ReplaceFile?$AA@ 5f8a4b3c  
 0002:0000bb48       ??_C@_08OBID@KERNEL32?$AA@ 5f8a4b48  
 0002:0000bb58       ??_7CMirrorFile@@6B@       5f8a4b58  
 0002:0000bbb8       ?classCDocTemplate@CDocTemplate@@2UCRuntimeClass@@B 5f8a4bb8  
 0002:0000bbd0       ??_C@_0N@BKAE@CDocTemplate?$AA@ 5f8a4bd0  
 0002:0000bbe0       ?classCSingleDocTemplate@CSingleDocTemplate@@2UCRuntimeClass@@B 5f8a4be0  
 0002:0000bbf8       ??_C@_0BD@BIBJ@CSingleDocTemplate?$AA@ 5f8a4bf8  
 0002:0000bc10       ?classCMultiDocTemplate@CMultiDocTemplate@@2UCRuntimeClass@@B 5f8a4c10  
 0002:0000bc28       ??_C@_0BC@HJJP@CMultiDocTemplate?$AA@ 5f8a4c28  
 0002:0000bc40       ?classCDocManager@CDocManager@@2UCRuntimeClass@@B 5f8a4c40  
 0002:0000bc58       ??_C@_0M@FJOK@CDocManager?$AA@ 5f8a4c58  
 0002:0000bc68       ?messageMap@CNewTypeDlg@@1UAFX_MSGMAP@@B 5f8a4c68  
 0002:0000bc70       ?_messageEntries@CNewTypeDlg@@0QBUAFX_MSGMAP_ENTRY@@B 5f8a4c70  
 0002:0000bca0       ?_afxPrintToArg@@3QBGB     5f8a4ca0  
 0002:0000bcd4       ?_afxPrintArg@@3QBGB       5f8a4cd4  
 0002:0000bce8       ?_afxOpenArg@@3QBGB        5f8a4ce8  
 0002:0000bcf4       ??_C@_17EICA@?$AA?$CK?$AA?4?$AA?$CK?$AA?$AA@ 5f8a4cf4  
 0002:0000bcfc       ??_C@_17OMHC@?$AA?$CC?$AA?0?$AA?$CC?$AA?$AA@ 5f8a4cfc  
 0002:0000bd04       ??_C@_1BG@LIGO@?$AA?$FL?$AAp?$AAr?$AAi?$AAn?$AAt?$AAt?$AAo?$AA?$CI?$AA?$CC?$AA?$AA@ 5f8a4d04  
 0002:0000bd1c       ??_C@_1BC@CMHH@?$AA?$FL?$AAp?$AAr?$AAi?$AAn?$AAt?$AA?$CI?$AA?$CC?$AA?$AA@ 5f8a4d1c  
 0002:0000bd30       ??_C@_1BA@NGLM@?$AA?$FL?$AAo?$AAp?$AAe?$AAn?$AA?$CI?$AA?$CC?$AA?$AA@ 5f8a4d30  
 0002:0000bd44       ??_7CNewTypeDlg@@6B@       5f8a4d44  
 0002:0000be20       ?messageMap@CSplitterWnd@@1UAFX_MSGMAP@@B 5f8a4e20  
 0002:0000be28       ?_messageEntries@CSplitterWnd@@0QBUAFX_MSGMAP_ENTRY@@B 5f8a4e28  
 0002:0000bfdc       ??_7CSplitterWnd@@6B@      5f8a4fdc  
 0002:0000c108       ?classCScrollView@CScrollView@@2UCRuntimeClass@@B 5f8a5108  
 0002:0000c120       ??_C@_0M@DAH@CScrollView?$AA@ 5f8a5120  
 0002:0000c130       ?sizeDefault@CScrollView@@2UtagSIZE@@B 5f8a5130  
 0002:0000c138       ?messageMap@CScrollView@@1UAFX_MSGMAP@@B 5f8a5138  
 0002:0000c140       ?_messageEntries@CScrollView@@0QBUAFX_MSGMAP_ENTRY@@B 5f8a5140  
 0002:0000c1b8       ??_C@_1O@JDNM@?$AAM?$AAo?$AAu?$AAs?$AAe?$AAZ?$AA?$AA@ 5f8a51b8  
 0002:0000c1c8       ??_C@_1CC@LAMD@?$AAM?$AAa?$AAg?$AAe?$AAl?$AAl?$AAa?$AAn?$AA?5?$AAM?$AAS?$AAW?$AAH?$AAE?$AAE?$AAL?$AA?$AA@ 5f8a51c8  
 0002:0000c1ec       ??_C@_1CC@BFDC@?$AAW?$AAh?$AAe?$AAe?$AAl?$AAS?$AAc?$AAr?$AAo?$AAl?$AAl?$AAL?$AAi?$AAn?$AAe?$AAs?$AA?$AA@ 5f8a51ec  
 0002:0000c210       ??_C@_1CM@EIGA@?$AAC?$AAo?$AAn?$AAt?$AAr?$AAo?$AAl?$AA?5?$AAP?$AAa?$AAn?$AAe?$AAl?$AA?2?$AAD?$AAe?$AAs?$AAk?$AAt?$AAo@ 5f8a5210  
 0002:0000c23c       ??_C@_1CK@GMOB@?$AAM?$AAS?$AAH?$AA_?$AAS?$AAC?$AAR?$AAO?$AAL?$AAL?$AA_?$AAL?$AAI?$AAN?$AAE?$AAS?$AA_?$AAM?$AAS?$AAG@ 5f8a523c  
 0002:0000c268       ?classCFormView@CFormView@@2UCRuntimeClass@@B 5f8a5268  
 0002:0000c280       ??_C@_09MHPF@CFormView?$AA@ 5f8a5280  
 0002:0000c290       ?messageMap@CFormView@@1UAFX_MSGMAP@@B 5f8a5290  
 0002:0000c298       ?_messageEntries@CFormView@@0QBUAFX_MSGMAP_ENTRY@@B 5f8a5298  
 0002:0000c314       ??_7CFormView@@6B@         5f8a5314  
 0002:0000c428       ?classCEditView@CEditView@@2UCRuntimeClass@@B 5f8a5428  
 0002:0000c440       ??_C@_09PCCM@CEditView?$AA@ 5f8a5440  
 0002:0000c44c       ?dwStyleDefault@CEditView@@2KB 5f8a544c  
 0002:0000c450       ?nMaxSize@CEditView@@2IB   5f8a5450  
 0002:0000c458       ?messageMap@CEditView@@1UAFX_MSGMAP@@B 5f8a5458  
 0002:0000c460       ?_messageEntries@CEditView@@0QBUAFX_MSGMAP_ENTRY@@B 5f8a5460  
 0002:0000c6d4       ??_7CEditView@@6B@         5f8a56d4  
 0002:0000c7f8       ??_C@_1CI@IJEE@?$AAL?$AAu?$AAc?$AAi?$AAd?$AAa?$AA?5?$AAS?$AAa?$AAn?$AAs?$AA?5?$AAU?$AAn?$AAi?$AAc?$AAo?$AAd?$AAe?$AA?$AA@ 5f8a57f8  
 0002:0000c820       ??_C@_13MCKD@?$AA?7?$AA?$AA@ 5f8a5820  
 0002:0000c828       ?classCPreviewView@CPreviewView@@2UCRuntimeClass@@B 5f8a5828  
 0002:0000c840       ??_C@_0N@LOLK@CPreviewView?$AA@ 5f8a5840  
 0002:0000c850       ?messageMap@CPreviewView@@1UAFX_MSGMAP@@B 5f8a5850  
 0002:0000c858       ?_messageEntries@CPreviewView@@0QBUAFX_MSGMAP_ENTRY@@B 5f8a5858  
 0002:0000ca3c       ??_7CPreviewView@@6B@      5f8a5a3c  
 0002:0000cb58       ?classCTreeView@CTreeView@@2UCRuntimeClass@@B 5f8a5b58  
 0002:0000cb70       ??_C@_09GPDN@CTreeView?$AA@ 5f8a5b70  
 0002:0000cb80       ?classCListView@CListView@@2UCRuntimeClass@@B 5f8a5b80  
 0002:0000cb98       ??_C@_09MHFL@CListView?$AA@ 5f8a5b98  
 0002:0000cba8       ?messageMap@CTreeView@@1UAFX_MSGMAP@@B 5f8a5ba8  
 0002:0000cbb0       ?_messageEntries@CTreeView@@0QBUAFX_MSGMAP_ENTRY@@B 5f8a5bb0  
 0002:0000cbe0       ?messageMap@CListView@@1UAFX_MSGMAP@@B 5f8a5be0  
 0002:0000cbe8       ?_messageEntries@CListView@@0QBUAFX_MSGMAP_ENTRY@@B 5f8a5be8  
 0002:0000cc1c       ??_7CListView@@6B@         5f8a5c1c  
 0002:0000cd34       ??_7CTreeView@@6B@         5f8a5d34  
 0002:0000ce48       ??_7_AFX_MAIL_STATE@@6B@   5f8a5e48  
 0002:0000ce4c       ??_C@_17OCMI@?$AAa?$AAf?$AAx?$AA?$AA@ 5f8a5e4c  
 0002:0000ce54       ??_C@_0N@HFFA@MAPISendMail?$AA@ 5f8a5e54  
 0002:0000ce64       ??_C@_0L@ICPG@MAPI32?4DLL?$AA@ 5f8a5e64  
 0002:0000ce70       ?classCWinThread@CWinThread@@2UCRuntimeClass@@B 5f8a5e70  
 0002:0000ce88       ??_C@_0L@BKIL@CWinThread?$AA@ 5f8a5e88  
 0002:0000ce98       ?classCWinApp@CWinApp@@2UCRuntimeClass@@B 5f8a5e98  
 0002:0000ceb0       ??_C@_07DHEF@CWinApp?$AA@  5f8a5eb0  
 0002:0000ceb8       ?messageMap@CWinApp@@1UAFX_MSGMAP@@B 5f8a5eb8  
 0002:0000cec0       ?_messageEntries@CWinApp@@0QBUAFX_MSGMAP_ENTRY@@B 5f8a5ec0  
 0002:0000cf20       ??_C@_0L@POJA@Automation?$AA@ 5f8a5f20  
 0002:0000cf2c       ??_C@_09LHIP@Embedding?$AA@ 5f8a5f2c  
 0002:0000cf38       ??_C@_03FNJD@dde?$AA@      5f8a5f38  
 0002:0000cf3c       ??_C@_0M@HIDL@Unregserver?$AA@ 5f8a5f3c  
 0002:0000cf48       ??_C@_0L@MNBE@Unregister?$AA@ 5f8a5f48  
 0002:0000cf54       ??_C@_01FOFA@p?$AA@        5f8a5f54  
 0002:0000cf56       ??_C@_02OBFC@pt?$AA@       5f8a5f56  
 0002:0000cf5c       ??_C@_13HMCP@?$AA?2?$AA?$AA@ 5f8a5f5c  
 0002:0000cf60       ??_C@_1BE@JFBP@?$AAS?$AAo?$AAf?$AAt?$AAw?$AAa?$AAr?$AAe?$AA?2?$AA?$AA@ 5f8a5f60  
 0002:0000cf74       ??_C@_0M@PMCB@CTL3D32?4DLL?$AA@ 5f8a5f74  
 0002:0000cf80       ??_C@_19BHME@?$AA?2?$AA?4?$AA?4?$AA?4?$AA?$AA@ 5f8a5f80  
 0002:0000cf90       ?classCGopherFileFind@CGopherFileFind@@2UCRuntimeClass@@B 5f8a5f90  
 0002:0000cfa8       ??_C@_0BA@FPGB@CGopherFileFind?$AA@ 5f8a5fa8  
 0002:0000cfb8       ?classCFtpFileFind@CFtpFileFind@@2UCRuntimeClass@@B 5f8a5fb8  
 0002:0000cfd0       ??_C@_0N@NGMH@CFtpFileFind?$AA@ 5f8a5fd0  
 0002:0000cfe0       ?classCGopherConnection@CGopherConnection@@2UCRuntimeClass@@B 5f8a5fe0  
 0002:0000cff8       ??_C@_0BC@JCEC@CGopherConnection?$AA@ 5f8a5ff8  
 0002:0000d010       ?classCHttpConnection@CHttpConnection@@2UCRuntimeClass@@B 5f8a6010  
 0002:0000d028       ??_C@_0BA@OLNH@CHttpConnection?$AA@ 5f8a6028  
 0002:0000d038       ?classCFtpConnection@CFtpConnection@@2UCRuntimeClass@@B 5f8a6038  
 0002:0000d050       ??_C@_0P@HPOD@CFtpConnection?$AA@ 5f8a6050  
 0002:0000d060       ?classCInternetConnection@CInternetConnection@@2UCRuntimeClass@@B 5f8a6060  
 0002:0000d078       ??_C@_0BE@NNFJ@CInternetConnection?$AA@ 5f8a6078  
 0002:0000d090       ?classCInternetSession@CInternetSession@@2UCRuntimeClass@@B 5f8a6090  
 0002:0000d0a8       ??_C@_0BB@BEAH@CInternetSession?$AA@ 5f8a60a8  
 0002:0000d0c0       ?classCGopherFile@CGopherFile@@2UCRuntimeClass@@B 5f8a60c0  
 0002:0000d0d8       ??_C@_0M@HDHO@CGopherFile?$AA@ 5f8a60d8  
 0002:0000d0e8       ?classCHttpFile@CHttpFile@@2UCRuntimeClass@@B 5f8a60e8  
 0002:0000d100       ??_C@_09IMKB@CHttpFile?$AA@ 5f8a6100  
 0002:0000d110       ?classCInternetFile@CInternetFile@@2UCRuntimeClass@@B 5f8a6110  
 0002:0000d128       ??_C@_0O@FDJM@CInternetFile?$AA@ 5f8a6128  
 0002:0000d138       ?classCInternetException@CInternetException@@2UCRuntimeClass@@B 5f8a6138  
 0002:0000d150       ??_C@_0BD@EMID@CInternetException?$AA@ 5f8a6150  
 0002:0000d164       ?szHtmlVerbs@CHttpConnection@@1QBQBGB 5f8a6164  
 0002:0000d180       ??_C@_1O@IMGP@?$AAU?$AAN?$AAL?$AAI?$AAN?$AAK?$AA?$AA@ 5f8a6180  
 0002:0000d190       ??_C@_1O@FBDO@?$AAD?$AAE?$AAL?$AAE?$AAT?$AAE?$AA?$AA@ 5f8a6190  
 0002:0000d1a0       ??_C@_19FNLP@?$AAL?$AAI?$AAN?$AAK?$AA?$AA@ 5f8a61a0  
 0002:0000d1ac       ??_C@_17ILBJ@?$AAP?$AAU?$AAT?$AA?$AA@ 5f8a61ac  
 0002:0000d1b4       ??_C@_19NFGA@?$AAH?$AAE?$AAA?$AAD?$AA?$AA@ 5f8a61b4  
 0002:0000d1c0       ??_C@_17KJPO@?$AAG?$AAE?$AAT?$AA?$AA@ 5f8a61c0  
 0002:0000d1c8       ??_C@_19KJFA@?$AAP?$AAO?$AAS?$AAT?$AA?$AA@ 5f8a61c8  
 0002:0000d1d4       ?_afxURLhttp@@3QBGB        5f8a61d4  
 0002:0000d1e4       ?_afxURLftp@@3QBGB         5f8a61e4  
 0002:0000d1f8       ??_7CInternetSession@@6B@  5f8a61f8  
 0002:0000d218       ??_7CInternetFile@@6B@     5f8a6218  
 0002:0000d284       ??_7CInternetConnection@@6B@ 5f8a6284  
 0002:0000d2a0       ??_7CFtpConnection@@6B@    5f8a62a0  
 0002:0000d2bc       ??_7CGopherConnection@@6B@ 5f8a62bc  
 0002:0000d2d8       ??_7CHttpConnection@@6B@   5f8a62d8  
 0002:0000d2f0       ??_C@_1BC@IFNG@?$AAH?$AAT?$AAT?$AAP?$AA?1?$AA1?$AA?4?$AA0?$AA?$AA@ 5f8a62f0  
 0002:0000d308       ??_7CHttpFile@@6B@         5f8a6308  
 0002:0000d378       ??_7CGopherFile@@6B@       5f8a6378  
 0002:0000d3e4       ??_7CFtpFileFind@@6B@      5f8a63e4  
 0002:0000d438       ??_C@_15OGLP@?$AA?2?$AA?1?$AA?$AA@ 5f8a6438  
 0002:0000d440       ??_C@_13HGEN@?$AA?$CK?$AA?$AA@ 5f8a6440  
 0002:0000d448       ??_7CGopherFileFind@@6B@   5f8a6448  
 0002:0000d4ac       ??_7CGopherLocator@@6B@    5f8a64ac  
 0002:0000d4c0       ??_C@_0M@KFA@WININET?4DLL?$AA@ 5f8a64c0  
 0002:0000d4d0       ??_7CInternetException@@6B@ 5f8a64d0  
 0002:0000d4f0       ?classCFileFind@CFileFind@@2UCRuntimeClass@@B 5f8a64f0  
 0002:0000d508       ??_C@_09CGCC@CFileFind?$AA@ 5f8a6508  
 0002:0000d518       ??_7CFileFind@@6B@         5f8a6518  
 0002:0000d56c       ??_C@_07LDFI@file?3?1?1?$AA@ 5f8a656c  
 0002:0000d578       ?classCSocketFile@CSocketFile@@2UCRuntimeClass@@B 5f8a6578  
 0002:0000d590       ??_C@_0M@FJKI@CSocketFile?$AA@ 5f8a6590  
 0002:0000d5a0       ?classCSocket@CSocket@@2UCRuntimeClass@@B 5f8a65a0  
 0002:0000d5b8       ??_C@_07MBCI@CSocket?$AA@  5f8a65b8  
 0002:0000d5c0       ?classCAsyncSocket@CAsyncSocket@@2UCRuntimeClass@@B 5f8a65c0  
 0002:0000d5d8       ??_C@_0N@CCKH@CAsyncSocket?$AA@ 5f8a65d8  
 0002:0000d5e8       ?messageMap@CSocketWnd@@1UAFX_MSGMAP@@B 5f8a65e8  
 0002:0000d5f0       ?_messageEntries@CSocketWnd@@0QBUAFX_MSGMAP_ENTRY@@B 5f8a65f0  
 0002:0000d63c       ??_7_AFX_SOCK_STATE@@6B@   5f8a663c  
 0002:0000d644       ??_7CAsyncSocket@@6B@      5f8a6644  
 0002:0000d68c       ??_C@_1DC@CDHD@?$AAS?$AAo?$AAc?$AAk?$AAe?$AAt?$AA?5?$AAN?$AAo?$AAt?$AAi?$AAf?$AAi?$AAc?$AAa?$AAt?$AAi?$AAo?$AAn?$AA?5@ 5f8a668c  
 0002:0000d6c4       ??_7CSocket@@6B@           5f8a66c4  
 0002:0000d718       ??_7CSocketFile@@6B@       5f8a6718  
 0002:0000d778       ??_7CSocketWnd@@6B@        5f8a6778  
 0002:0000d838       ?classCOleLinkingDoc@COleLinkingDoc@@2UCRuntimeClass@@B 5f8a6838  
 0002:0000d850       ??_C@_0P@EIOM@COleLinkingDoc?$AA@ 5f8a6850  
 0002:0000d860       ?interfaceMap@COleClientItem@@1UAFX_INTERFACEMAP@@B 5f8a6860  
 0002:0000d868       ?_interfaceEntries@COleClientItem@@0QBUAFX_INTERFACEMAP_ENTRY@@B 5f8a6868  
 0002:0000d894       ??_7COleClientItem@@6B@    5f8a6894  
 0002:0000d980       ??_7XOleIPSite@COleClientItem@@6B@ 5f8a6980  
 0002:0000d9c0       ??_7XAdviseSink@COleClientItem@@6B@ 5f8a69c0  
 0002:0000d9e4       ??_7XOleClientSite@COleClientItem@@6B@ 5f8a69e4  
 0002:0000da08       ??_C@_1BM@EINE@?$AAE?$AAm?$AAb?$AAe?$AAd?$AAd?$AAi?$AAn?$AAg?$AA?5?$AA?$CF?$AAl?$AAu?$AA?$AA@ 5f8a6a08  
 0002:0000da24       ??_C@_1BI@FPKN@?$AAD?$AAo?$AAc?$AAS?$AAh?$AAo?$AAr?$AAt?$AAc?$AAu?$AAt?$AA?$AA@ 5f8a6a24  
 0002:0000da3c       ??_C@_1BI@EMMJ@?$AAD?$AAe?$AAf?$AAa?$AAu?$AAl?$AAt?$AAI?$AAc?$AAo?$AAn?$AA?$AA@ 5f8a6a3c  
 0002:0000da54       ??_C@_1M@MDBL@?$AAc?$AAl?$AAs?$AAi?$AAd?$AA?$AA@ 5f8a6a54  
 0002:0000da60       ?interfaceMap@COleFrameHook@@1UAFX_INTERFACEMAP@@B 5f8a6a60  
 0002:0000da68       ?_interfaceEntries@COleFrameHook@@0QBUAFX_INTERFACEMAP_ENTRY@@B 5f8a6a68  
 0002:0000da8c       ??_7COleFrameHook@@6B@     5f8a6a8c  
 0002:0000db18       ??_7XOleCommandTarget@COleFrameHook@@6B@ 5f8a6b18  
 0002:0000db30       ??_7XOleInPlaceFrame@COleFrameHook@@6B@ 5f8a6b30  
 0002:0000db70       ?interfaceMap@COleDataSource@@1UAFX_INTERFACEMAP@@B 5f8a6b70  
 0002:0000db78       ?_interfaceEntries@COleDataSource@@0QBUAFX_INTERFACEMAP_ENTRY@@B 5f8a6b78  
 0002:0000db88       ?interfaceMap@CEnumFormatEtc@@1UAFX_INTERFACEMAP@@B 5f8a6b88  
 0002:0000db90       ?_interfaceEntries@CEnumFormatEtc@@0QBUAFX_INTERFACEMAP_ENTRY@@B 5f8a6b90  
 0002:0000dba4       ??_7COleDataSource@@6B@    5f8a6ba4  
 0002:0000dc10       ??_7XDataObject@COleDataSource@@6B@ 5f8a6c10  
 0002:0000dc44       ??_7CEnumFormatEtc@@6B@    5f8a6c44  
 0002:0000dcb0       ?classCOleDispatchException@COleDispatchException@@2UCRuntimeClass@@B 5f8a6cb0  
 0002:0000dcc8       ??_C@_0BG@OGI@COleDispatchException?$AA@ 5f8a6cc8  
 0002:0000dce4       ??_7COleDispatchException@@6B@ 5f8a6ce4  
 0002:0000dd00       ?classCOlePasteSpecialDialog@COlePasteSpecialDialog@@2UCRuntimeClass@@B 5f8a6d00  
 0002:0000dd18       ??_C@_0BH@NAFF@COlePasteSpecialDialog?$AA@ 5f8a6d18  
 0002:0000dd30       ?classCOleUpdateDialog@COleUpdateDialog@@2UCRuntimeClass@@B 5f8a6d30  
 0002:0000dd48       ??_C@_0BB@HGD@COleUpdateDialog?$AA@ 5f8a6d48  
 0002:0000dd60       ?classCOleLinksDialog@COleLinksDialog@@2UCRuntimeClass@@B 5f8a6d60  
 0002:0000dd78       ??_C@_0BA@PIHM@COleLinksDialog?$AA@ 5f8a6d78  
 0002:0000dd88       ?classCOleChangeIconDialog@COleChangeIconDialog@@2UCRuntimeClass@@B 5f8a6d88  
 0002:0000dda0       ??_C@_0BF@JMPM@COleChangeIconDialog?$AA@ 5f8a6da0  
 0002:0000ddb8       ?classCOleConvertDialog@COleConvertDialog@@2UCRuntimeClass@@B 5f8a6db8  
 0002:0000ddd0       ??_C@_0BC@CIPN@COleConvertDialog?$AA@ 5f8a6dd0  
 0002:0000dde8       ?classCOleInsertDialog@COleInsertDialog@@2UCRuntimeClass@@B 5f8a6de8  
 0002:0000de00       ??_C@_0BB@KPPE@COleInsertDialog?$AA@ 5f8a6e00  
 0002:0000de18       ??_7COleUILinkInfo@@6B@    5f8a6e18  
 0002:0000de4c       ??_7COleInsertDialog@@6B@  5f8a6e4c  
 0002:0000df24       ??_C@_1CG@POCI@?$AAC?$AAL?$AAS?$AAI?$AAD?$AA?2?$AA?$CF?$AAs?$AA?2?$AAD?$AAo?$AAc?$AAO?$AAb?$AAj?$AAe?$AAc?$AAt?$AA?$AA@ 5f8a6f24  
 0002:0000df4c       ??_C@_1BE@ILGK@?$AAD?$AAo?$AAc?$AAO?$AAb?$AAj?$AAe?$AAc?$AAt?$AA?$AA@ 5f8a6f4c  
 0002:0000df60       ??_C@_1BE@NGOH@?$AAO?$AAl?$AAe?$AA1?$AAC?$AAl?$AAa?$AAs?$AAs?$AA?$AA@ 5f8a6f60  
 0002:0000df74       ??_C@_1BG@HHA@?$AAI?$AAn?$AAs?$AAe?$AAr?$AAt?$AAa?$AAb?$AAl?$AAe?$AA?$AA@ 5f8a6f74  
 0002:0000df90       ??_7COleConvertDialog@@6B@ 5f8a6f90  
 0002:0000e06c       ??_7COleChangeIconDialog@@6B@ 5f8a706c  
 0002:0000e148       ??_7COleLinksDialog@@6B@   5f8a7148  
 0002:0000e224       ??_7COleUpdateDialog@@6B@  5f8a7224  
 0002:0000e300       ??_7COlePasteSpecialDialog@@6B@ 5f8a7300  
 0002:0000e3d8       ?classCOleBusyDialog@COleBusyDialog@@2UCRuntimeClass@@B 5f8a73d8  
 0002:0000e3f0       ??_C@_0P@CLOH@COleBusyDialog?$AA@ 5f8a73f0  
 0002:0000e400       ?classCOleDialog@COleDialog@@2UCRuntimeClass@@B 5f8a7400  
 0002:0000e418       ??_C@_0L@HMIO@COleDialog?$AA@ 5f8a7418  
 0002:0000e428       ??_7COleDialog@@6B@        5f8a7428  
 0002:0000e504       ??_7COleBusyDialog@@6B@    5f8a7504  
 0002:0000e5e0       ?classCOleChangeSourceDialog@COleChangeSourceDialog@@2UCRuntimeClass@@B 5f8a75e0  
 0002:0000e5f8       ??_C@_0BH@HBLJ@COleChangeSourceDialog?$AA@ 5f8a75f8  
 0002:0000e610       ?classCOlePropertiesDialog@COlePropertiesDialog@@2UCRuntimeClass@@B 5f8a7610  
 0002:0000e628       ??_C@_0BF@IDJJ@COlePropertiesDialog?$AA@ 5f8a7628  
 0002:0000e644       ??_7COlePropertiesDialog@@6B@ 5f8a7644  
 0002:0000e724       ??_7XOleUIObjInfo@COlePropertiesDialog@@6B@ 5f8a7724  
 0002:0000e744       ??_C@_15DEDE@?$AA?$CF?$AAs?$AA?$AA@ 5f8a7744  
 0002:0000e750       ??_7COleChangeSourceDialog@@6B@ 5f8a7750  
 0002:0000e828       __real@8@3ffb8000000000000000 5f8a7828  
 0002:0000e830       __real@4@3ffb8000000000000000 5f8a7830  
 0002:0000e838       __real@8@3feec22e450672894800 5f8a7838  
 0002:0000e840       __real@8@400fa8c0000000000000 5f8a7840  
 0002:0000e848       __real@8@bfedc22e450672894800 5f8a7848  
 0002:0000e850       __real@8@3fedc22e450672894800 5f8a7850  
 0002:0000e858       __real@8@c012a081a00000000000 5f8a7858  
 0002:0000e860       __real@8@4014b492040000000000 5f8a7860  
 0002:0000e868       __real@8@bfff8000000000000000 5f8a7868  
 0002:0000e870       __real@8@4003c000000000000000 5f8a7870  
 0002:0000e878       __real@8@4004f000000000000000 5f8a7878  
 0002:0000e880       __real@8@4009b400000000000000 5f8a7880  
 0002:0000e888       __real@8@3ffaaaaaaaaaaaaaa800 5f8a7888  
 0002:0000e890       __real@8@3ff4b60b60b60b60b800 5f8a7890  
 0002:0000e898       __real@8@4014dcb2640000000000 5f8a7898  
 0002:0000e8a0       __real@8@c014dcb2640000000000 5f8a78a0  
 0002:0000e8a8       ?classCOleDocument@COleDocument@@2UCRuntimeClass@@B 5f8a78a8  
 0002:0000e8c0       ??_C@_0N@KLEF@COleDocument?$AA@ 5f8a78c0  
 0002:0000e8d0       ??_C@_1BC@DBBK@?$AAC?$AAo?$AAn?$AAt?$AAe?$AAn?$AAt?$AAs?$AA?$AA@ 5f8a78d0  
 0002:0000e8e8       ??_7CDocItem@@6B@          5f8a78e8  
 0002:0000e948       ?interfaceMap@COleDropSource@@1UAFX_INTERFACEMAP@@B 5f8a7948  
 0002:0000e950       ?_interfaceEntries@COleDropSource@@0QBUAFX_INTERFACEMAP_ENTRY@@B 5f8a7950  
 0002:0000e9a0       ??_7COleDropSource@@6B@    5f8a79a0  
 0002:0000ea08       ??_7XDropSource@COleDropSource@@6B@ 5f8a7a08  
 0002:0000ea20       ?interfaceMap@COleMessageFilter@@1UAFX_INTERFACEMAP@@B 5f8a7a20  
 0002:0000ea28       ?_interfaceEntries@COleMessageFilter@@0QBUAFX_INTERFACEMAP_ENTRY@@B 5f8a7a28  
 0002:0000ea38       ?_afxSignificantMsgs@@3QBIB 5f8a7a38  
 0002:0000ea78       ??_7CEnumArray@@6B@        5f8a7a78  
 0002:0000eae4       ??_7XEnumVOID@CEnumArray@@6B@ 5f8a7ae4  
 0002:0000eb00       ?classCOleIPFrameWnd@COleIPFrameWnd@@2UCRuntimeClass@@B 5f8a7b00  
 0002:0000eb18       ??_C@_0P@CBLJ@COleIPFrameWnd?$AA@ 5f8a7b18  
 0002:0000eb28       ?messageMap@COleIPFrameWnd@@1UAFX_MSGMAP@@B 5f8a7b28  
 0002:0000eb30       ?_messageEntries@COleIPFrameWnd@@0QBUAFX_MSGMAP_ENTRY@@B 5f8a7b30  
 0002:0000ec6c       ??_7COleCntrFrameWnd@@6B@  5f8a7c6c  
 0002:0000ed6c       ??_7COleIPFrameWnd@@6B@    5f8a7d6c  
 0002:0000ee88       ?classCOleException@COleException@@2UCRuntimeClass@@B 5f8a7e88  
 0002:0000eea0       ??_C@_0O@EEPE@COleException?$AA@ 5f8a7ea0  
 0002:0000eeb4       ??_7COleException@@6B@     5f8a7eb4  
 0002:0000eed0       ?classCOleStreamFile@COleStreamFile@@2UCRuntimeClass@@B 5f8a7ed0  
 0002:0000eee8       ??_C@_0P@CGBG@COleStreamFile?$AA@ 5f8a7ee8  
 0002:0000eefc       ??_7COleStreamFile@@6B@    5f8a7efc  
 0002:0000ef60       ?classCOleServerDoc@COleServerDoc@@2UCRuntimeClass@@B 5f8a7f60  
 0002:0000ef78       ??_C@_0O@ELE@COleServerDoc?$AA@ 5f8a7f78  
 0002:0000ef88       ?messageMap@COleServerDoc@@1UAFX_MSGMAP@@B 5f8a7f88  
 0002:0000ef90       ?_messageEntries@COleServerDoc@@0QBUAFX_MSGMAP_ENTRY@@B 5f8a7f90  
 0002:0000f008       ?interfaceMap@COleServerItem@@1UAFX_INTERFACEMAP@@B 5f8a8008  
 0002:0000f010       ?_interfaceEntries@COleServerItem@@0QBUAFX_INTERFACEMAP_ENTRY@@B 5f8a8010  
 0002:0000f02c       ??_7COleServerItem@@6B@    5f8a802c  
 0002:0000f0dc       ??_7XDataObject@COleServerItem@@6B@ 5f8a80dc  
 0002:0000f110       ??_7XOleObject@COleServerItem@@6B@ 5f8a8110  
 0002:0000f174       ??_7CItemDataSource@COleServerItem@@6B@ 5f8a8174  
 0002:0000f26c       ??_7CInnerUnknown@@6B@     5f8a826c  
 0002:0000f278       ?interfaceMap@CEnumOleVerb@@1UAFX_INTERFACEMAP@@B 5f8a8278  
 0002:0000f280       ?_interfaceEntries@CEnumOleVerb@@0QBUAFX_INTERFACEMAP_ENTRY@@B 5f8a8280  
 0002:0000f294       ??_7CEnumOleVerb@@6B@      5f8a8294  
 0002:0000f2fc       ??_C@_1BO@JDJE@?$AA?$DM?$AAu?$AAn?$AAk?$AAn?$AAo?$AAw?$AAn?$AA?5?$AAv?$AAe?$AAr?$AAb?$AA?$DO?$AA?$AA@ 5f8a82fc  
 0002:0000f320       ?classCRichEditDoc@CRichEditDoc@@2UCRuntimeClass@@B 5f8a8320  
 0002:0000f338       ??_C@_0N@HOLH@CRichEditDoc?$AA@ 5f8a8338  
 0002:0000f348       ?interfaceMap@CRichEditView@@1UAFX_INTERFACEMAP@@B 5f8a8348  
 0002:0000f350       ?_interfaceEntries@CRichEditView@@0QBUAFX_INTERFACEMAP_ENTRY@@B 5f8a8350  
 0002:0000f360       ?messageMap@CRichEditView@@1UAFX_MSGMAP@@B 5f8a8360  
 0002:0000f368       ?_messageEntries@CRichEditView@@0QBUAFX_MSGMAP_ENTRY@@B 5f8a8368  
 0002:0000f638       ??_C@_15MLJJ@?$AA?6?$AA?$AN?$AA?$AA@ 5f8a8638  
 0002:0000f644       ??_7CRichEditCntrItem@@6B@ 5f8a8644  
 0002:0000f730       ??_7CTypeLibCacheMap@@6B@  5f8a8730  
 0002:0000f748       ?classCMonikerFile@CMonikerFile@@2UCRuntimeClass@@B 5f8a8748  
 0002:0000f760       ??_C@_0N@CIKC@CMonikerFile?$AA@ 5f8a8760  
 0002:0000f774       ??_7CMonikerFile@@6B@      5f8a8774  
 0002:0000f7ec       ??_7_AfxBindHost@@6B@      5f8a87ec  
 0002:0000f808       ??_7IBindHost@@6B@         5f8a8808  
 0002:0000f820       ?classCMonthCalCtrl@CMonthCalCtrl@@2UCRuntimeClass@@B 5f8a8820  
 0002:0000f838       ??_C@_0O@MIA@CMonthCalCtrl?$AA@ 5f8a8838  
 0002:0000f848       ?classCDateTimeCtrl@CDateTimeCtrl@@2UCRuntimeClass@@B 5f8a8848  
 0002:0000f860       ??_C@_0O@BJFB@CDateTimeCtrl?$AA@ 5f8a8860  
 0002:0000f870       ??_C@_1CE@IFHN@?$AAS?$AAy?$AAs?$AAD?$AAa?$AAt?$AAe?$AAT?$AAi?$AAm?$AAe?$AAP?$AAi?$AAc?$AAk?$AA3?$AA2?$AA?$AA@ 5f8a8870  
 0002:0000f898       ??_7CDateTimeCtrl@@6B@     5f8a8898  
 0002:0000f958       ??_C@_1BM@FKA@?$AAS?$AAy?$AAs?$AAM?$AAo?$AAn?$AAt?$AAh?$AAC?$AAa?$AAl?$AA3?$AA2?$AA?$AA@ 5f8a8958  
 0002:0000f978       ??_7CMonthCalCtrl@@6B@     5f8a8978  
 0002:0000fa38       ?classCHtmlView@CHtmlView@@2UCRuntimeClass@@B 5f8a8a38  
 0002:0000fa50       ??_C@_09GHGJ@CHtmlView?$AA@ 5f8a8a50  
 0002:0000fa60       ?eventsinkMap@CHtmlView@@1UAFX_EVENTSINKMAP@@B 5f8a8a60  
 0002:0000fa70       ?_eventsinkEntries@CHtmlView@@0QBUAFX_EVENTSINKMAP_ENTRY@@B 5f8a8a70  
 0002:0000fd68       ??_C@_01KLAB@?$AL?$AA@     5f8a8d68  
 0002:0000fd6a       ??_C@_02HJK@IK?$AA@        5f8a8d6a  
 0002:0000fd70       ??_C@_07LMNJ@?7LLLLLK?$AA@ 5f8a8d70  
 0002:0000fd78       ??_C@_02PINK@?7L?$AA@      5f8a8d78  
 0002:0000fd7c       ??_C@_02JAPO@?$AD?$AL?$AA@ 5f8a8d7c  
 0002:0000fd80       ??_C@_02MEEG@?$AD?$AD?$AA@ 5f8a8d80  
 0002:0000fd84       ??_C@_01FELI@?$AI?$AA@     5f8a8d84  
 0002:0000fd88       ?messageMap@CHtmlView@@1UAFX_MSGMAP@@B 5f8a8d88  
 0002:0000fd90       ?_messageEntries@CHtmlView@@0QBUAFX_MSGMAP_ENTRY@@B 5f8a8d90  
 0002:0000fe0c       ??_7CHtmlView@@6B@         5f8a8e0c  
 0002:0000ff70       ??_C@_1BI@HKIO@?$AAr?$AAe?$AAs?$AA?3?$AA?1?$AA?1?$AA?$CF?$AAs?$AA?1?$AA?$CF?$AAs?$AA?$AA@ 5f8a8f70  
 0002:0000ff88       ??_C@_1BI@OFIF@?$AAr?$AAe?$AAs?$AA?3?$AA?1?$AA?1?$AA?$CF?$AAs?$AA?1?$AA?$CF?$AAd?$AA?$AA@ 5f8a8f88  
 0002:0000ffa4       ??_7COccManager@@6B@       5f8a8fa4  
 0002:0000ffd0       ?interfaceMap@CEnumUnknown@@1UAFX_INTERFACEMAP@@B 5f8a8fd0  
 0002:0000ffd8       ?_interfaceEntries@CEnumUnknown@@0QBUAFX_INTERFACEMAP_ENTRY@@B 5f8a8fd8  
 0002:0000ffe8       ?dispatchMap@COleControlContainer@@1UAFX_DISPMAP@@B 5f8a8fe8  
 0002:0000fff8       ?_dispatchEntries@COleControlContainer@@0QBUAFX_DISPMAP_ENTRY@@B 5f8a8ff8  
 0002:00010018       ?interfaceMap@COleControlContainer@@1UAFX_INTERFACEMAP@@B 5f8a9018  
 0002:00010020       ?_interfaceEntries@COleControlContainer@@0QBUAFX_INTERFACEMAP_ENTRY@@B 5f8a9020  
 0002:0001003c       ??_7COleControlContainer@@6B@ 5f8a903c  
 0002:000100d4       ??_7XOleContainer@COleControlContainer@@6B@ 5f8a90d4  
 0002:000100f0       ??_7XOleIPFrame@COleControlContainer@@6B@ 5f8a90f0  
 0002:00010130       ??_7CFont@@6B@             5f8a9130  
 0002:00010148       ??_7CEnumUnknown@@6B@      5f8a9148  
 0002:000101b0       _IID_IDataSource           5f8a91b0  
 0002:000101d0       ?_afxAmbients@@3QBU__unnamed@@B 5f8a91d0  
 0002:00010210       ?interfaceMap@COleControlSite@@1UAFX_INTERFACEMAP@@B 5f8a9210  
 0002:00010218       ?_interfaceEntries@COleControlSite@@0QBUAFX_INTERFACEMAP_ENTRY@@B 5f8a9218  
 0002:0001025c       ??_7COleControlSite@@6B@   5f8a925c  
 0002:00010328       ??_7XRowsetNotify@COleControlSite@@6B@ 5f8a9328  
 0002:00010344       ??_7XNotifyDBEvents@COleControlSite@@6B@ 5f8a9344  
 0002:00010370       ??_7XBoundObjectSite@COleControlSite@@6B@ 5f8a9370  
 0002:00010384       ??_7XEventSink@COleControlSite@@6B@ 5f8a9384  
 0002:000103a4       ??_7XPropertyNotifySink@COleControlSite@@6B@ 5f8a93a4  
 0002:000103bc       ??_7XAmbientProps@COleControlSite@@6B@ 5f8a93bc  
 0002:000103dc       ??_7XOleControlSite@COleControlSite@@6B@ 5f8a93dc  
 0002:00010408       ??_7XOleIPSite@COleControlSite@@6B@ 5f8a9408  
 0002:00010448       ??_7XOleClientSite@COleControlSite@@6B@ 5f8a9448  
 0002:00010470       ??_7CDataSourceControl@@6B@ 5f8a9470  
 0002:00010488       __real@8@3ffbccccccccccccd000 5f8a9488  
 0002:00010494       ??_7COleControlLock@@6B@   5f8a9494  
 0002:00010498       ?classCDocObjectServerItem@CDocObjectServerItem@@2UCRuntimeClass@@B 5f8a9498  
 0002:000104b0       ??_C@_0BF@FCEC@CDocObjectServerItem?$AA@ 5f8a94b0  
 0002:000104c8       ?interfaceMap@CDocObjectServer@@1UAFX_INTERFACEMAP@@B 5f8a94c8  
 0002:000104d0       ?_interfaceEntries@CDocObjectServer@@0QBUAFX_INTERFACEMAP_ENTRY@@B 5f8a94d0  
 0002:00010500       ?messageMap@CDocObjectServer@@1UAFX_MSGMAP@@B 5f8a9500  
 0002:00010508       ?_messageEntries@CDocObjectServer@@0QBUAFX_MSGMAP_ENTRY@@B 5f8a9508  
 0002:00010520       ?classCDocObjectServer@CDocObjectServer@@2UCRuntimeClass@@B 5f8a9520  
 0002:00010538       ??_C@_0BB@ICMG@CDocObjectServer?$AA@ 5f8a9538  
 0002:00010550       ??_7CDocObjectServer@@6B@  5f8a9550  
 0002:000105bc       ??_7XPrint@CDocObjectServer@@6B@ 5f8a95bc  
 0002:000105d8       ??_7XOleCommandTarget@CDocObjectServer@@6B@ 5f8a95d8  
 0002:000105f0       ??_7XOleDocumentView@CDocObjectServer@@6B@ 5f8a95f0  
 0002:00010634       ??_7XOleDocument@CDocObjectServer@@6B@ 5f8a9634  
 0002:00010650       ??_7XOleObject@CDocObjectServer@@6B@ 5f8a9650  
 0002:000106b4       ??_7CDocObjectServerItem@@6B@ 5f8a96b4  
 0002:00010764       ??_7COleCmdUI@@6B@         5f8a9764  
 0002:00010778       ?messageMap@COleDocIPFrameWnd@@1UAFX_MSGMAP@@B 5f8a9778  
 0002:00010780       ?_messageEntries@COleDocIPFrameWnd@@0QBUAFX_MSGMAP_ENTRY@@B 5f8a9780  
 0002:00010798       ?classCOleDocIPFrameWnd@COleDocIPFrameWnd@@2UCRuntimeClass@@B 5f8a9798  
 0002:000107b0       ??_C@_0BC@DHMK@COleDocIPFrameWnd?$AA@ 5f8a97b0  
 0002:000107c8       ??_7COleDocIPFrameWnd@@6B@ 5f8a97c8  
 0002:000108e8       ?interfaceMap@COleDocObjectItem@@1UAFX_INTERFACEMAP@@B 5f8a98e8  
 0002:000108f0       ?_interfaceEntries@COleDocObjectItem@@0QBUAFX_INTERFACEMAP_ENTRY@@B 5f8a98f0  
 0002:00010900       ?classCOleDocObjectItem@COleDocObjectItem@@2UCRuntimeClass@@B 5f8a9900  
 0002:00010918       ??_C@_0BC@ODBE@COleDocObjectItem?$AA@ 5f8a9918  
 0002:00010930       ??_7COleDocObjectItem@@6B@ 5f8a9930  
 0002:00010a20       ??_7XOleDocumentSite@COleDocObjectItem@@6B@ 5f8a9a20  
 0002:00010a30       ??_C@_1M@EOJM@?$AA?$CF?$AAs?$AA?5?$AA?$CF?$AAs?$AA?$AA@ 5f8a9a30  
 0002:00010a40       ?classCAsyncMonikerFile@CAsyncMonikerFile@@2UCRuntimeClass@@B 5f8a9a40  
 0002:00010a58       ??_C@_0BC@OCAO@CAsyncMonikerFile?$AA@ 5f8a9a58  
 0002:00010a70       ??_7CAsyncMonikerFile@@6B@ 5f8a9a70  
 0002:00010b20       ??_7_AfxBindStatusCallback@@6B@ 5f8a9b20  
 0002:00010b50       ??_7CInnerUnknown@_AfxBindStatusCallback@@6B@ 5f8a9b50  
 0002:00010b60       ??_7IBindStatusCallback@@6B@ 5f8a9b60  
 0002:00010b90       ?classCOleResizeBar@COleResizeBar@@2UCRuntimeClass@@B 5f8a9b90  
 0002:00010ba8       ??_C@_0O@BGCL@COleResizeBar?$AA@ 5f8a9ba8  
 0002:00010bb8       ?messageMap@COleResizeBar@@1UAFX_MSGMAP@@B 5f8a9bb8  
 0002:00010bc0       ?_messageEntries@COleResizeBar@@0QBUAFX_MSGMAP_ENTRY@@B 5f8a9bc0  
 0002:00010c6c       ??_7COleResizeBar@@6B@     5f8a9c6c  
 0002:00010d54       ??_C@_1CC@MLNF@?$AAA?$AAf?$AAx?$AAC?$AAo?$AAn?$AAt?$AAr?$AAo?$AAl?$AAB?$AAa?$AAr?$AA4?$AA2?$AAu?$AA?$AA@ 5f8a9d54  
 0002:00010d78       ?classCOleControl@COleControl@@2UCRuntimeClass@@B 5f8a9d78  
 0002:00010d90       ??_C@_0M@EGDG@COleControl?$AA@ 5f8a9d90  
 0002:00010da0       ?messageMap@COleControl@@1UAFX_MSGMAP@@B 5f8a9da0  
 0002:00010da8       ?_messageEntries@COleControl@@0QBUAFX_MSGMAP_ENTRY@@B 5f8a9da8  
 0002:000111f8       ?eventMap@COleControl@@1UAFX_EVENTMAP@@B 5f8aa1f8  
 0002:00011208       ?interfaceMap@COleControl@@1UAFX_INTERFACEMAP@@B 5f8aa208  
 0002:00011210       ?_interfaceEntries@COleControl@@0QBUAFX_INTERFACEMAP_ENTRY@@B 5f8aa210  
 0002:000112cc       ??_7COleControl@@6B@       5f8aa2cc  
 0002:000114c8       ??_7XPropConnPt@COleControl@@6B@ 5f8aa4c8  
 0002:00011538       ??_7XEventConnPt@COleControl@@6B@ 5f8aa538  
 0002:000115a8       ??_7XPointerInactive@COleControl@@6B@ 5f8aa5a8  
 0002:000115c4       ??_7XQuickActivate@COleControl@@6B@ 5f8aa5c4  
 0002:000115e0       ??_7XFontNotification@COleControl@@6B@ 5f8aa5e0  
 0002:000115f8       ??_7XPerPropertyBrowsing@COleControl@@6B@ 5f8aa5f8  
 0002:00011618       ??_7XSpecifyPropertyPages@COleControl@@6B@ 5f8aa618  
 0002:0001162c       ??_7XProvideClassInfo@COleControl@@6B@ 5f8aa62c  
 0002:00011644       ??_7XOleControl@COleControl@@6B@ 5f8aa644  
 0002:00011664       ??_7XOleCache@COleControl@@6B@ 5f8aa664  
 0002:00011688       ??_7XOleInPlaceActiveObject@COleControl@@6B@ 5f8aa688  
 0002:000116b4       ??_7XOleInPlaceObject@COleControl@@6B@ 5f8aa6b4  
 0002:000116e4       ??_7XDataObject@COleControl@@6B@ 5f8aa6e4  
 0002:00011718       ??_7XViewObject@COleControl@@6B@ 5f8aa718  
 0002:00011758       ??_7XOleObject@COleControl@@6B@ 5f8aa758  
 0002:000117bc       ??_7XPersistPropertyBag@COleControl@@6B@ 5f8aa7bc  
 0002:000117dc       ??_7XPersistMemory@COleControl@@6B@ 5f8aa7dc  
 0002:00011804       ??_7XPersistStreamInit@COleControl@@6B@ 5f8aa804  
 0002:0001182c       ??_7XPersistStorage@COleControl@@6B@ 5f8aa82c  
 0002:00011858       ??_7CReflectorWnd@@6B@     5f8aa858  
 0002:00011918       ??_C@_1CC@IHJH@?$AAA?$AAf?$AAx?$AAO?$AAl?$AAe?$AAC?$AAo?$AAn?$AAt?$AAr?$AAo?$AAl?$AA4?$AA2?$AAu?$AA?$AA@ 5f8aa918  
 0002:00011940       ??_7CParkingWnd@@6B@       5f8aa940  
 0002:00011a00       ?connectionMap@COleControl@@1UAFX_CONNECTIONMAP@@B 5f8aaa00  
 0002:00011a08       ?_connectionEntries@COleControl@@0QBUAFX_CONNECTIONMAP_ENTRY@@B 5f8aaa08  
 0002:00011a18       ??_C@_1GI@CCPJ@?$AA?$HL?$AA?$CF?$AA0?$AA8?$AAl?$AAX?$AA?9?$AA?$CF?$AA0?$AA4?$AAX?$AA?9?$AA?$CF?$AA0?$AA4?$AAX?$AA?9?$AA?$CF?$AA0?$AA2@ 5f8aaa18  
 0002:00011a84       ??_7CControlDataSource@COleControl@@6B@ 5f8aaa84  
 0002:00011aec       ?_afxStockEvents@@3QBKB    5f8aaaec  
 0002:00011b14       ??_C@_02NCNO@B?$AC?$AA@    5f8aab14  
 0002:00011b18       ??_C@_1BC@BKHA@?$AAC?$AAo?$AAm?$AAb?$AAo?$AAB?$AAo?$AAx?$AA?$AA@ 5f8aab18  
 0002:00011b2c       ??_C@_1BA@GKFH@?$AAL?$AAi?$AAs?$AAt?$AAB?$AAo?$AAx?$AA?$AA@ 5f8aab2c  
 0002:00011b3c       ??_C@_01PAOO@B?$AA@        5f8aab3c  
 0002:00011b40       ??_C@_04CKMP@?$AC?$AC?$AD?$AD?$AA@ 5f8aab40  
 0002:00011b48       ??_C@_07FGFI@?$ACH?6?$AI?$AI?$ADK?$AA@ 5f8aab48  
 0002:00011b50       ?classCOleControlModule@COleControlModule@@2UCRuntimeClass@@B 5f8aab50  
 0002:00011b68       ??_C@_0BC@KPIB@COleControlModule?$AA@ 5f8aab68  
 0002:00011b80       ?messageMap@CControlFrameWnd@@1UAFX_MSGMAP@@B 5f8aab80  
 0002:00011b88       ?_messageEntries@CControlFrameWnd@@0QBUAFX_MSGMAP_ENTRY@@B 5f8aab88  
 0002:00011bd4       ??_7CControlFrameWnd@@6B@  5f8aabd4  
 0002:00011c98       ??_C@_1BE@MHHE@?$AAA?$AAf?$AAx?$AAW?$AAn?$AAd?$AA4?$AA2?$AAu?$AA?$AA@ 5f8aac98  
 0002:00011cb0       ?_afxFontDescDefault@@3UtagFONTDESC@@B 5f8aacb0  
 0002:00011cd0       ?interfaceMap@CEnumConnPoints@@1UAFX_INTERFACEMAP@@B 5f8aacd0  
 0002:00011cd8       ?_interfaceEntries@CEnumConnPoints@@0QBUAFX_INTERFACEMAP_ENTRY@@B 5f8aacd8  
 0002:00011ce8       ?interfaceMap@CEnumConnections@@1UAFX_INTERFACEMAP@@B 5f8aace8  
 0002:00011cf0       ?_interfaceEntries@CEnumConnections@@0QBUAFX_INTERFACEMAP_ENTRY@@B 5f8aacf0  
 0002:00011d04       ??_7CConnectionPoint@@6B@  5f8aad04  
 0002:00011d74       ??_7XConnPt@CConnectionPoint@@6B@ 5f8aad74  
 0002:00011d98       ??_7CEnumConnections@@6B@  5f8aad98  
 0002:00011e04       ??_7CEnumConnPoints@@6B@   5f8aae04  
 0002:00011e70       ??_7COleConnPtContainer@@6B@ 5f8aae70  
 0002:00011e88       ?_afx_CLSID_StdPicture2_V1@@3U_GUID@@B 5f8aae88  
 0002:00011e98       ??_C@_1BC@EBDI@?$AA_?$AAE?$AAx?$AAt?$AAe?$AAn?$AAt?$AAY?$AA?$AA@ 5f8aae98  
 0002:00011eac       ??_C@_1BC@BDCO@?$AA_?$AAE?$AAx?$AAt?$AAe?$AAn?$AAt?$AAX?$AA?$AA@ 5f8aaeac  
 0002:00011ec0       ??_C@_1BC@IEIC@?$AA_?$AAV?$AAe?$AAr?$AAs?$AAi?$AAo?$AAn?$AA?$AA@ 5f8aaec0  
 0002:00011ed8       ??_7CArchivePropExchange@@6B@ 5f8aaed8  
 0002:00011ef0       ??_7CResetPropExchange@@6B@ 5f8aaef0  
 0002:00011f08       ??_7CAsyncPropExchange@@6B@ 5f8aaf08  
 0002:00011f1c       ??_C@_1BO@FKJD@?$AAF?$AAo?$AAn?$AAt?$AAS?$AAt?$AAr?$AAi?$AAk?$AAe?$AAt?$AAh?$AAr?$AAu?$AA?$AA@ 5f8aaf1c  
 0002:00011f3c       ??_C@_1BM@KNCC@?$AAF?$AAo?$AAn?$AAt?$AAU?$AAn?$AAd?$AAe?$AAr?$AAl?$AAi?$AAn?$AAe?$AA?$AA@ 5f8aaf3c  
 0002:00011f58       ??_C@_1BG@LJAN@?$AAF?$AAo?$AAn?$AAt?$AAI?$AAt?$AAa?$AAl?$AAi?$AAc?$AA?$AA@ 5f8aaf58  
 0002:00011f70       ??_C@_1BC@KBKA@?$AAF?$AAo?$AAn?$AAt?$AAB?$AAo?$AAl?$AAd?$AA?$AA@ 5f8aaf70  
 0002:00011f84       ??_C@_1BC@DAIL@?$AAF?$AAo?$AAn?$AAt?$AAS?$AAi?$AAz?$AAe?$AA?$AA@ 5f8aaf84  
 0002:00011f98       ??_C@_1BC@NLCC@?$AAF?$AAo?$AAn?$AAt?$AAN?$AAa?$AAm?$AAe?$AA?$AA@ 5f8aaf98  
 0002:00011fb0       ?classCOlePropertyPage@COlePropertyPage@@2UCRuntimeClass@@B 5f8aafb0  
 0002:00011fc8       ??_C@_0BB@LGDG@COlePropertyPage?$AA@ 5f8aafc8  
 0002:00011fe0       ?_afxUpdateList@@3QBUNotifyInfo@@B 5f8aafe0  
 0002:00012010       ?_afxNotifyList@@3QBUNotifyInfo@@B 5f8ab010  
 0002:00012040       ??_C@_1BA@OMOJ@?$AAl?$AAi?$AAs?$AAt?$AAb?$AAo?$AAx?$AA?$AA@ 5f8ab040  
 0002:00012050       ??_C@_1O@MLLH@?$AAb?$AAu?$AAt?$AAt?$AAo?$AAn?$AA?$AA@ 5f8ab050  
 0002:00012060       ??_C@_19NPFC@?$AAe?$AAd?$AAi?$AAt?$AA?$AA@ 5f8ab060  
 0002:00012070       ?messageMap@COlePropertyPage@@1UAFX_MSGMAP@@B 5f8ab070  
 0002:00012078       ?_messageEntries@COlePropertyPage@@0QBUAFX_MSGMAP_ENTRY@@B 5f8ab078  
 0002:000120c0       ?interfaceMap@COlePropertyPage@@1UAFX_INTERFACEMAP@@B 5f8ab0c0  
 0002:000120c8       ?_interfaceEntries@COlePropertyPage@@0QBUAFX_INTERFACEMAP_ENTRY@@B 5f8ab0c8  
 0002:000120e4       ??_7AFX_DDPDATA@@6B@       5f8ab0e4  
 0002:000120fc       ??_7COlePropertyPage@@6B@  5f8ab0fc  
 0002:000121e8       ??_7XPropNotifySink@COlePropertyPage@@6B@ 5f8ab1e8  
 0002:00012200       ??_7XPropertyPage@COlePropertyPage@@6B@ 5f8ab200  
 0002:00012240       ?classCCachedDataPathProperty@CCachedDataPathProperty@@2UCRuntimeClass@@B 5f8ab240  
 0002:00012258       ??_C@_0BI@EKAI@CCachedDataPathProperty?$AA@ 5f8ab258  
 0002:00012270       ?classCDataPathProperty@CDataPathProperty@@2UCRuntimeClass@@B 5f8ab270  
 0002:00012288       ??_C@_0BC@OBPM@CDataPathProperty?$AA@ 5f8ab288  
 0002:0001229c       ?_afxAmbientFlags@@3QBKB   5f8ab29c  
 0002:000122c4       ?_afxStockProps@@3QBKB     5f8ab2c4  
 0002:00012314       ??_C@_1BG@LJOC@?$AAA?$AAp?$AAp?$AAe?$AAa?$AAr?$AAa?$AAn?$AAc?$AAe?$AA?$AA@ 5f8ab314  
 0002:0001232c       ??_C@_1BA@CGKE@?$AAE?$AAn?$AAa?$AAb?$AAl?$AAe?$AAd?$AA?$AA@ 5f8ab32c  
 0002:0001233c       ??_C@_1BI@PNDM@?$AAB?$AAo?$AAr?$AAd?$AAe?$AAr?$AAS?$AAt?$AAy?$AAl?$AAe?$AA?$AA@ 5f8ab33c  
 0002:00012354       ??_C@_19LHGG@?$AAF?$AAo?$AAn?$AAt?$AA?$AA@ 5f8ab354  
 0002:00012360       ??_C@_1BE@DJDJ@?$AAB?$AAa?$AAc?$AAk?$AAC?$AAo?$AAl?$AAo?$AAr?$AA?$AA@ 5f8ab360  
 0002:00012374       ??_C@_1BE@NMAC@?$AAF?$AAo?$AAr?$AAe?$AAC?$AAo?$AAl?$AAo?$AAr?$AA?$AA@ 5f8ab374  
 0002:00012388       ??_C@_19PMHI@?$AAT?$AAe?$AAx?$AAt?$AA?$AA@ 5f8ab388  
 0002:00012394       ??_C@_1BA@JOHB@?$AAC?$AAa?$AAp?$AAt?$AAi?$AAo?$AAn?$AA?$AA@ 5f8ab394  
 0002:000123a4       ??_C@_1BI@HFFM@?$AA_?$AAS?$AAt?$AAo?$AAc?$AAk?$AAP?$AAr?$AAo?$AAp?$AAs?$AA?$AA@ 5f8ab3a4  
 0002:000123c0       ?_afxFontDescHelv@@3UtagFONTDESC@@B 5f8ab3c0  
 0002:000123e0       ?_afx_CLSID_StdPicture_V1@@3U_GUID@@B 5f8ab3e0  
 0002:000123f0       ?_afx_CLSID_StdFont_V1@@3U_GUID@@B 5f8ab3f0  
 0002:00012404       ??_7CPropsetPropExchange@@6B@ 5f8ab404  
 0002:00012418       ?_afxPropPageClass@@3QBQBGB 5f8ab418  
 0002:00012424       ??_C@_1CE@CBLG@?$AAI?$AAn?$AAp?$AAr?$AAo?$AAc?$AAS?$AAe?$AAr?$AAv?$AAe?$AAr?$AA3?$AA2?$AA?$AA?$AA?$CF?$AA2?$AA?$AA@ 5f8ab424  
 0002:00012448       ?_afxCtrlClassID@@3QBQBGB  5f8ab448  
 0002:00012470       ??_C@_1BG@KBAC@?$AAV?$AAe?$AAr?$AAs?$AAi?$AAo?$AAn?$AA?$AA?$AA?$CF?$AA7?$AA?$AA@ 5f8ab470  
 0002:00012488       ??_C@_1BG@CKJF@?$AAT?$AAy?$AAp?$AAe?$AAL?$AAi?$AAb?$AA?$AA?$AA?$CF?$AA6?$AA?$AA@ 5f8ab488  
 0002:000124a0       ??_C@_1BC@GHKE@?$AAC?$AAo?$AAn?$AAt?$AAr?$AAo?$AAl?$AA?$AA?$AA?$AA@ 5f8ab4a0  
 0002:000124b4       ??_C@_1CA@JADL@?$AAM?$AAi?$AAs?$AAc?$AAS?$AAt?$AAa?$AAt?$AAu?$AAs?$AA?2?$AA1?$AA?$AA?$AA?$CF?$AA5?$AA?$AA@ 5f8ab4b4  
 0002:000124d4       ??_C@_1BK@KBO@?$AAM?$AAi?$AAs?$AAc?$AAS?$AAt?$AAa?$AAt?$AAu?$AAs?$AA?$AA?$AA0?$AA?$AA@ 5f8ab4d4  
 0002:000124f0       ??_C@_1CO@FFFM@?$AAT?$AAo?$AAo?$AAl?$AAb?$AAo?$AAx?$AAB?$AAi?$AAt?$AAm?$AAa?$AAp?$AA3?$AA2?$AA?$AA?$AA?$CF?$AA3?$AA?0?$AA?5@ 5f8ab4f0  
 0002:00012520       ??_C@_1CE@HDKA@?$AAI?$AAn?$AAp?$AAr?$AAo?$AAc?$AAS?$AAe?$AAr?$AAv?$AAe?$AAr?$AA3?$AA2?$AA?$AA?$AA?$CF?$AA3?$AA?$AA@ 5f8ab520  
 0002:00012544       ??_C@_1BE@EDCM@?$AAP?$AAr?$AAo?$AAg?$AAI?$AAD?$AA?$AA?$AA?$CF?$AA2?$AA?$AA@ 5f8ab544  
 0002:00012558       ?_afxCtrlProgID@@3QBQBGB   5f8ab558  
 0002:00012564       ??_C@_1BC@HIDF@?$AAC?$AAL?$AAS?$AAI?$AAD?$AA?$AA?$AA?$CF?$AA2?$AA?$AA@ 5f8ab564  
 0002:00012578       ??_C@_17BFLD@?$AA?$AA?$AA?$CF?$AA1?$AA?$AA@ 5f8ab578  
 0002:00012580       ??_C@_1BG@JIPA@?$AAI?$AAn?$AAt?$AAe?$AAr?$AAf?$AAa?$AAc?$AAe?$AA?2?$AA?$AA@ 5f8ab580  
 0002:00012598       ??_C@_1M@BFC@?$AAw?$AAi?$AAn?$AA3?$AA2?$AA?$AA@ 5f8ab598  
 0002:000125a4       ??_C@_1M@JEC@?$AAw?$AAi?$AAn?$AA1?$AA6?$AA?$AA@ 5f8ab5a4  
 0002:000125b0       ??_C@_1M@OFBC@?$AAF?$AAL?$AAA?$AAG?$AAS?$AA?$AA@ 5f8ab5b0  
 0002:000125bc       ??_C@_1BA@KOAG@?$AAH?$AAE?$AAL?$AAP?$AAD?$AAI?$AAR?$AA?$AA@ 5f8ab5bc  
 0002:000125cc       ??_C@_1BG@DNML@?$AAT?$AAY?$AAP?$AAE?$AAL?$AAI?$AAB?$AA?2?$AA?$CF?$AAs?$AA?$AA@ 5f8ab5cc  
 0002:000125e4       ??_C@_1BO@PFNJ@?$AAT?$AAh?$AAr?$AAe?$AAa?$AAd?$AAi?$AAn?$AAg?$AAM?$AAo?$AAd?$AAe?$AAl?$AA?$AA@ 5f8ab5e4  
 0002:00012604       ??_C@_1BO@OGKK@?$AAI?$AAn?$AAp?$AAr?$AAo?$AAc?$AAS?$AAe?$AAr?$AAv?$AAe?$AAr?$AA3?$AA2?$AA?$AA@ 5f8ab604  
 0002:00012624       ??_C@_1BC@CNEA@?$AAC?$AAL?$AAS?$AAI?$AAD?$AA?2?$AA?$CF?$AAs?$AA?$AA@ 5f8ab624  
 0002:00012638       ??_C@_1M@CJDN@?$AA?$CF?$AAd?$AA?4?$AA?$CF?$AAd?$AA?$AA@ 5f8ab638  
 0002:00012644       ??_C@_1CA@NEAI@?$AAT?$AAo?$AAo?$AAl?$AAb?$AAo?$AAx?$AAB?$AAi?$AAt?$AAm?$AAa?$AAp?$AA3?$AA2?$AA?$AA@ 5f8ab644  
 0002:00012664       ??_C@_1BI@FGP@?$AAC?$AAL?$AAS?$AAI?$AAD?$AA?2?$AA?$CF?$AAs?$AA?2?$AA?$CF?$AAs?$AA?$AA@ 5f8ab664  
 0002:0001267c       ??_C@_1BK@KICO@?$AAI?$AAn?$AAp?$AAr?$AAo?$AAc?$AAS?$AAe?$AAr?$AAv?$AAe?$AAr?$AA?$AA@ 5f8ab67c  
 0002:0001269c       ??_7CControlRectTracker@@6B@ 5f8ab69c  
 0002:000126b8       ?_afx_CLSID_BlobProperty@@3U_GUID@@B 5f8ab6b8  
 0002:000126cc       ??_7CBlobProperty@@6B@     5f8ab6cc  
 0002:000126f0       ??_7CPropbagPropExchange@@6B@ 5f8ab6f0  
 0002:00012708       ??_7_AFXCTL_AMBIENT_CACHE@@6B@ 5f8ab708  
 0002:00012710       ?classCWindowlessDC@CWindowlessDC@@2UCRuntimeClass@@B 5f8ab710  
 0002:00012728       ??_C@_0O@FBOP@CWindowlessDC?$AA@ 5f8ab728  
 0002:0001273c       ??_7CWindowlessDC@@6B@     5f8ab73c  
 0002:000127b8       ?messageMap@CColorPropPage@@1UAFX_MSGMAP@@B 5f8ab7b8  
 0002:000127c0       ?_messageEntries@CColorPropPage@@0QBUAFX_MSGMAP_ENTRY@@B 5f8ab7c0  
 0002:00012988       ?_afxSysColorsList@@3QBUSysColorsInfo@@B 5f8ab988  
 0002:00012a3c       ??_7CColorButton@@6B@      5f8aba3c  
 0002:00012b04       ??_7CColorPropPage@@6B@    5f8abb04  
 0002:00012bf0       ?messageMap@CFontPropPage@@1UAFX_MSGMAP@@B 5f8abbf0  
 0002:00012bf8       ?_messageEntries@CFontPropPage@@0QBUAFX_MSGMAP_ENTRY@@B 5f8abbf8  
 0002:00012d04       ??_7CFontPropPage@@6B@     5f8abd04  
 0002:00012df8       ??_7CSizeComboBox@@6B@     5f8abdf8  
 0002:00012ecc       ??_7CFontComboBox@@6B@     5f8abecc  
 0002:00012fa0       ?messageMap@CPicturePropPage@@1UAFX_MSGMAP@@B 5f8abfa0  
 0002:00012fa8       ?_messageEntries@CPicturePropPage@@0QBUAFX_MSGMAP_ENTRY@@B 5f8abfa8  
 0002:00013024       ??_7CPicturePropPage@@6B@  5f8ac024  
 0002:00013110       ?classCStockPropPage@CStockPropPage@@2UCRuntimeClass@@B 5f8ac110  
 0002:00013128       ??_C@_0P@GBDL@CStockPropPage?$AA@ 5f8ac128  
 0002:00013138       ?messageMap@CStockPropPage@@1UAFX_MSGMAP@@B 5f8ac138  
 0002:00013140       ?_messageEntries@CStockPropPage@@0QBUAFX_MSGMAP_ENTRY@@B 5f8ac140  
 0002:0001315c       ??_7CStockPropPage@@6B@    5f8ac15c  
 0002:00013248       ?classCRecordset@CRecordset@@2UCRuntimeClass@@B 5f8ac248  
 0002:00013260       ??_C@_0L@FKJL@CRecordset?$AA@ 5f8ac260  
 0002:00013270       ?classCDatabase@CDatabase@@2UCRuntimeClass@@B 5f8ac270  
 0002:00013288       ??_C@_09CDJB@CDatabase?$AA@ 5f8ac288  
 0002:00013298       ?classCDBException@CDBException@@2UCRuntimeClass@@B 5f8ac298  
 0002:000132b0       ??_C@_0N@GGEG@CDBException?$AA@ 5f8ac2b0  
 0002:000132c0       ?_afxDriverNotCapable@@3QBGB 5f8ac2c0  
 0002:000132d8       ?_afxOutOfSequence@@3QBGB  5f8ac2d8  
 0002:000132f0       ?_afxDataTruncated@@3QBGB  5f8ac2f0  
 0002:00013308       ?_afxRowFetch@@3QBGB       5f8ac308  
 0002:00013320       ?_afxForUpdate@@3QBGB      5f8ac320  
 0002:0001333c       ?_afxOrderBy@@3QBGB        5f8ac33c  
 0002:00013354       ?_afxWhere@@3QBGB          5f8ac354  
 0002:00013364       ?_afxFrom@@3QBGB           5f8ac364  
 0002:00013374       ?_afxSelect@@3QBGB         5f8ac374  
 0002:00013384       ?_afxParamCall@@3QBGB      5f8ac384  
 0002:0001338c       ?_afxCall@@3QBGB           5f8ac38c  
 0002:0001339c       ?_afxComma@@3QBGB          5f8ac39c  
 0002:000133a0       ?_afxODBCTrail@@3QBGB      5f8ac3a0  
 0002:000133b0       ??_7CDBException@@6B@      5f8ac3b0  
 0002:000133d0       ??_C@_1O@JCG@?$AAS?$AAt?$AAa?$AAt?$AAe?$AA?3?$AA?$AA@ 5f8ac3d0  
 0002:000133e0       ??_C@_1CI@LDEF@?$AA?0?$AAN?$AAa?$AAt?$AAi?$AAv?$AAe?$AA?3?$AA?$CF?$AAl?$AAd?$AA?0?$AAO?$AAr?$AAi?$AAg?$AAi?$AAn?$AA?3?$AA?$AA@ 5f8ac3e0  
 0002:00013408       ??_C@_1M@MKCN@?$AA0?$AA0?$AA0?$AA0?$AA0?$AA?$AA@ 5f8ac408  
 0002:00013418       ??_7CDatabase@@6B@         5f8ac418  
 0002:00013448       ??_C@_1M@BHKK@?$AA?$DL?$AAD?$AAS?$AAN?$AA?$DN?$AA?$AA@ 5f8ac448  
 0002:00013454       ??_C@_01PCJP@Y?$AA@        5f8ac454  
 0002:0001345c       ??_7CRecordset@@6B@        5f8ac45c  
 0002:000134c4       ??_C@_1BA@FFIB@?$AA?5?$AAU?$AAN?$AAI?$AAO?$AAN?$AA?5?$AA?$AA@ 5f8ac4c4  
 0002:000134d4       ??_C@_1BG@CONM@?$AA?5?$AAG?$AAR?$AAO?$AAU?$AAP?$AA?5?$AAB?$AAY?$AA?5?$AA?$AA@ 5f8ac4d4  
 0002:000134ec       ??_C@_1O@LFLK@?$AA?5?$AAJ?$AAO?$AAI?$AAN?$AA?5?$AA?$AA@ 5f8ac4ec  
 0002:000134fc       ??_C@_13JKDK@?$AA?0?$AA?$AA@ 5f8ac4fc  
 0002:00013500       ??_C@_1CG@BIKJ@?$AA?5?$AAW?$AAH?$AAE?$AAR?$AAE?$AA?5?$AAC?$AAU?$AAR?$AAR?$AAE?$AAN?$AAT?$AA?5?$AAO?$AAF?$AA?5?$AA?$AA@ 5f8ac500  
 0002:00013528       ??_C@_1BK@FPKL@?$AAD?$AAE?$AAL?$AAE?$AAT?$AAE?$AA?5?$AAF?$AAR?$AAO?$AAM?$AA?5?$AA?$AA@ 5f8ac528  
 0002:00013544       ??_C@_1M@FJED@?$AA?5?$AAS?$AAE?$AAT?$AA?5?$AA?$AA@ 5f8ac544  
 0002:00013550       ??_C@_1BA@MDEN@?$AAU?$AAP?$AAD?$AAA?$AAT?$AAE?$AA?5?$AA?$AA@ 5f8ac550  
 0002:00013560       ??_C@_1BE@LEJJ@?$AA?5?$AAV?$AAA?$AAL?$AAU?$AAE?$AAS?$AA?5?$AA?$CI?$AA?$AA@ 5f8ac560  
 0002:00013574       ??_C@_15NGMK@?$AA?5?$AA?$CI?$AA?$AA@ 5f8ac574  
 0002:0001357c       ??_C@_1BK@ECOF@?$AAI?$AAN?$AAS?$AAE?$AAR?$AAT?$AA?5?$AAI?$AAN?$AAT?$AAO?$AA?5?$AA?$AA@ 5f8ac57c  
 0002:0001359c       ??_7_AFX_DB_STATE@@6B@     5f8ac59c  
 0002:000135a0       ??_C@_1BI@HDAA@?$AAS?$AAt?$AAa?$AAt?$AAe?$AA?3?$AA0?$AA1?$AA0?$AA0?$AA4?$AA?$AA@ 5f8ac5a0  
 0002:000135b8       ?classCRecordView@CRecordView@@2UCRuntimeClass@@B 5f8ac5b8  
 0002:000135d0       ??_C@_0M@EAFL@CRecordView?$AA@ 5f8ac5d0  
 0002:000135e0       ?messageMap@CRecordView@@1UAFX_MSGMAP@@B 5f8ac5e0  
 0002:000135e8       ?_messageEntries@CRecordView@@0QBUAFX_MSGMAP_ENTRY@@B 5f8ac5e8  
 0002:000136c4       ??_7CRecordView@@6B@       5f8ac6c4  
 0002:000137f0       ?classCLongBinary@CLongBinary@@2UCRuntimeClass@@B 5f8ac7f0  
 0002:00013808       ??_C@_0M@DJA@CLongBinary?$AA@ 5f8ac808  
 0002:00013818       ??_7CLongBinary@@6B@       5f8ac818  
 0002:00013830       ??_7CDBVariant@@6B@        5f8ac830  
 0002:00013838       ?classCDaoRecordset@CDaoRecordset@@2UCRuntimeClass@@B 5f8ac838  
 0002:00013850       ??_C@_0O@JOIL@CDaoRecordset?$AA@ 5f8ac850  
 0002:00013860       ?classCDaoQueryDef@CDaoQueryDef@@2UCRuntimeClass@@B 5f8ac860  
 0002:00013878       ??_C@_0N@NGH@CDaoQueryDef?$AA@ 5f8ac878  
 0002:00013888       ?classCDaoTableDef@CDaoTableDef@@2UCRuntimeClass@@B 5f8ac888  
 0002:000138a0       ??_C@_0N@PHMG@CDaoTableDef?$AA@ 5f8ac8a0  
 0002:000138b0       ?classCDaoDatabase@CDaoDatabase@@2UCRuntimeClass@@B 5f8ac8b0  
 0002:000138c8       ??_C@_0N@DDLP@CDaoDatabase?$AA@ 5f8ac8c8  
 0002:000138d8       ?classCDaoWorkspace@CDaoWorkspace@@2UCRuntimeClass@@B 5f8ac8d8  
 0002:000138f0       ??_C@_0O@IEJG@CDaoWorkspace?$AA@ 5f8ac8f0  
 0002:00013900       ?classCDaoException@CDaoException@@2UCRuntimeClass@@B 5f8ac900  
 0002:00013918       ??_C@_0O@OIMH@CDaoException?$AA@ 5f8ac918  
 0002:00013928       ?_afxTable2@@3QBGB         5f8ac928  
 0002:00013938       ?_afxTransform2@@3QBGB     5f8ac938  
 0002:00013950       ?_afxOrderBy2@@3QBGB       5f8ac950  
 0002:00013968       ?_afxWhere2@@3QBGB         5f8ac968  
 0002:00013978       ?_afxFrom2@@3QBGB          5f8ac978  
 0002:00013988       ?_afxSelect2@@3QBGB        5f8ac988  
 0002:00013998       ?_afxParameters2@@3QBGB    5f8ac998  
 0002:000139b4       ??_7_AFX_DAO_STATE@@6B@    5f8ac9b4  
 0002:000139bc       ??_7CDaoIndexInfo@@6B@     5f8ac9bc  
 0002:000139c4       ??_7CDaoRelationInfo@@6B@  5f8ac9c4  
 0002:000139cc       ??_7CDaoException@@6B@     5f8ac9cc  
 0002:000139ec       ??_7CDaoWorkspace@@6B@     5f8ac9ec  
 0002:00013a18       ??_7CDaoDatabase@@6B@      5f8aca18  
 0002:00013a40       ??_7CDaoTableDef@@6B@      5f8aca40  
 0002:00013a6c       ??_7CDaoQueryDef@@6B@      5f8aca6c  
 0002:00013aac       ??_7CDaoRecordset@@6B@     5f8acaac  
 0002:00013b2c       ??_C@_13FDB@?$AA?$DL?$AA?$AA@ 5f8acb2c  
 0002:00013b30       ??_C@_1CO@HEDE@?$AAI?$AAC?$AAD?$AAA?$AAO?$AAR?$AAe?$AAc?$AAo?$AAr?$AAd?$AAs?$AAe?$AAt?$AA?4?$AAG?$AAe?$AAt?$AAR?$AAo@ 5f8acb30  
 0002:00013b60       ??_C@_1EK@JJKF@?$AAm?$AAj?$AAg?$AAc?$AAq?$AAc?$AAe?$AAj?$AAf?$AAc?$AAh?$AAc?$AAi?$AAj?$AAe?$AAc?$AAp?$AAd?$AAh?$AAc@ 5f8acb60  
 0002:00013bac       ??_C@_1EK@JBEF@?$AAm?$AAb?$AAm?$AAa?$AAb?$AAp?$AAt?$AAe?$AAb?$AAk?$AAj?$AAc?$AAd?$AAl?$AAg?$AAt?$AAj?$AAm?$AAs?$AAk@ 5f8acbac  
 0002:00013bf8       ?_afxDoublePseudoNull@@3NB 5f8acbf8  
 0002:00013c00       ?_afxFloatPseudoNull@@3MB  5f8acc00  
 0002:00013c04       ??_C@_09CGOK@?5DateTime?$AA@ 5f8acc04  
 0002:00013c10       ??_C@_0M@BGKI@?5IEEEDouble?$AA@ 5f8acc10  
 0002:00013c1c       ??_C@_0M@GOBO@?5IEEESingle?$AA@ 5f8acc1c  
 0002:00013c28       ??_C@_09GDCP@?5Currency?$AA@ 5f8acc28  
 0002:00013c34       ??_C@_05BJMF@?5Long?$AA@   5f8acc34  
 0002:00013c3c       ??_C@_06KOJB@?5Short?$AA@  5f8acc3c  
 0002:00013c44       ??_C@_05IGCC@?5Byte?$AA@   5f8acc44  
 0002:00013c4c       ??_C@_04KDMA@?5Bit?$AA@    5f8acc4c  
 0002:00013c54       ??_C@_0M@MOAI@?5LongBinary?$AA@ 5f8acc54  
 0002:00013c60       ??_C@_05BJHD@?5Text?$AA@   5f8acc60  
 0002:00013c66       ??_C@_01KMAE@?0?$AA@       5f8acc66  
 0002:00013c68       ?messageMap@CDaoRecordView@@1UAFX_MSGMAP@@B 5f8acc68  
 0002:00013c70       ?_messageEntries@CDaoRecordView@@0QBUAFX_MSGMAP_ENTRY@@B 5f8acc70  
 0002:00013d48       ?classCDaoRecordView@CDaoRecordView@@2UCRuntimeClass@@B 5f8acd48  
 0002:00013d60       ??_C@_0P@KPJP@CDaoRecordView?$AA@ 5f8acd60  
 0002:00013d74       ??_7CDaoRecordView@@6B@    5f8acd74  
 0002:00013e90       ?classCOleDBRecordView@COleDBRecordView@@2UCRuntimeClass@@B 5f8ace90  
 0002:00013ea8       ??_C@_0BB@HKOA@COleDBRecordView?$AA@ 5f8acea8  
 0002:00013ec0       ?messageMap@COleDBRecordView@@1UAFX_MSGMAP@@B 5f8acec0  
 0002:00013ec8       ?_messageEntries@COleDBRecordView@@0QBUAFX_MSGMAP_ENTRY@@B 5f8acec8  
 0002:00013fa0       ?classCDynLinkLibrary@CDynLinkLibrary@@2UCRuntimeClass@@B 5f8acfa0  
 0002:00013fb8       ??_C@_0BA@FNMJ@CDynLinkLibrary?$AA@ 5f8acfb8  
 0002:00013fc8       ??_C@_0JB@KLFG@This?5application?5or?5DLL?5can?5not?5@ 5f8acfc8  
 0002:0001405c       ??_C@_0BD@CCKL@MFC?5Runtime?5Module?$AA@ 5f8ad05c  
 0002:00014074       ??_7CPalette@@6B@          5f8ad074  
 0002:0001408c       ??_7CCheckListBox@@6B@     5f8ad08c  
 0002:0001416c       ??_7CBitmapButton@@6B@     5f8ad16c  
 0002:00014234       ??_7CDataPathProperty@@6B@ 5f8ad234  
 0002:000142f4       ??_7CCachedDataPathProperty@@6B@ 5f8ad2f4  
 0002:000143c0       _IID_IStream               5f8ad3c0  
 0002:000143d0       _IID_IOleInPlaceSite       5f8ad3d0  
 0002:000143e0       _IID_IAdviseSink           5f8ad3e0  
 0002:000143f0       _IID_IOleClientSite        5f8ad3f0  
 0002:00014400       _IID_IOleLink              5f8ad400  
 0002:00014410       _IID_IViewObject2          5f8ad410  
 0002:00014420       _IID_IPersistStream        5f8ad420  
 0002:00014430       _IID_IPersistStreamInit    5f8ad430  
 0002:00014440       _IID_IOleCache             5f8ad440  
 0002:00014450       _IID_IOleInPlaceFrame      5f8ad450  
 0002:00014460       _IID_IOleInPlaceUIWindow   5f8ad460  
 0002:00014470       _IID_IOleCommandTarget     5f8ad470  
 0002:00014480       _IID_IEnumFORMATETC        5f8ad480  
 0002:00014490       _IID_IDropSource           5f8ad490  
 0002:000144a0       _IID_IMessageFilter        5f8ad4a0  
 0002:000144b0       _IID_IStorage              5f8ad4b0  
 0002:000144c0       _IID_IOleDocumentSite      5f8ad4c0  
 0002:000144d0       _IID_IEnumOLEVERB          5f8ad4d0  
 0002:000144e0       _IID_IBindHost             5f8ad4e0  
 0002:000144f0       _IID_IWebBrowser2          5f8ad4f0  
 0002:00014500       _CLSID_WebBrowser          5f8ad500  
 0002:00014510       _IID_IEnumUnknown          5f8ad510  
 0002:00014520       _IID_IFontDisp             5f8ad520  
 0002:00014530       _IID_IRowsetNotify         5f8ad530  
 0002:00014540       _IID_IRowPosition          5f8ad540  
 0002:00014550       _IID_IRowset               5f8ad550  
 0002:00014560       _IID_IAccessor             5f8ad560  
 0002:00014570       _IID_INotifyDBEvents       5f8ad570  
 0002:00014580       _IID_IBoundObjectSite      5f8ad580  
 0002:00014590       _IID_IOleControlSite       5f8ad590  
 0002:000145a0       _IID_IPropertyNotifySink   5f8ad5a0  
 0002:000145b0       _IID_IFont                 5f8ad5b0  
 0002:000145c0       _IID_IQuickActivate        5f8ad5c0  
 0002:000145d0       _IID_IPersistMemory        5f8ad5d0  
 0002:000145e0       _IID_IOleControl           5f8ad5e0  
 0002:000145f0       _IID_IConnectionPointContainer 5f8ad5f0  
 0002:00014600       _IID_IProvideClassInfo     5f8ad600  
 0002:00014610       _IID_IProvideClassInfo2    5f8ad610  
 0002:00014620       _IID_ICursorUpdateARow     5f8ad620  
 0002:00014630       _IID_ICursorMove           5f8ad630  
 0002:00014640       _IID_ICursor               5f8ad640  
 0002:00014650       _COLUMN_COLUMNID           5f8ad650  
 0002:00014668       _COLUMN_NAME               5f8ad668  
 0002:00014680       _DBBMK_CURRENT             5f8ad680  
 0002:00014688       _IID_ISequentialStream     5f8ad688  
 0002:00014698       _IID_IBoundObject          5f8ad698  
 0002:000146a8       _IID_IPrint                5f8ad6a8  
 0002:000146b8       _IID_IOleDocumentView      5f8ad6b8  
 0002:000146c8       _IID_IOleDocument          5f8ad6c8  
 0002:000146d8       _IID_IBindStatusCallback   5f8ad6d8  
 0002:000146e8       _IID_IServiceProvider      5f8ad6e8  
 0002:000146f8       _IID_IPerPropertyBrowsing  5f8ad6f8  
 0002:00014708       _IID_ISpecifyPropertyPages 5f8ad708  
 0002:00014718       _IID_IPersistPropertyBag   5f8ad718  
 0002:00014728       _IID_IViewObject           5f8ad728  
 0002:00014738       _IID_IOleInPlaceObjectWindowless 5f8ad738  
 0002:00014748       _IID_IViewObjectEx         5f8ad748  
 0002:00014758       _IID_IPointerInactive      5f8ad758  
 0002:00014768       _CLSID_ConvertVBX          5f8ad768  
 0002:00014778       _CLSID_PersistPropset      5f8ad778  
 0002:00014788       _IID_IOleInPlaceSiteEx     5f8ad788  
 0002:00014798       _IID_IOleInPlaceSiteWindowless 5f8ad798  
 0002:000147a8       _IID_IEnumConnectionPoints 5f8ad7a8  
 0002:000147b8       _IID_IEnumConnections      5f8ad7b8  
 0002:000147c8       _IID_IConnectionPoint      5f8ad7c8  
 0002:000147d8       _IID_ISimpleFrameSite      5f8ad7d8  
 0002:000147e8       _IID_IPicture              5f8ad7e8  
 0002:000147f8       _IID_IPictureDisp          5f8ad7f8  
 0002:00014808       _CLSID_StdPicture          5f8ad808  
 0002:00014818       _IID_IPropertyPage         5f8ad818  
 0002:00014828       _IID_IPropertyPage2        5f8ad828  
 0002:00014838       _CLSID_CColorPropPage      5f8ad838  
 0002:00014848       _CLSID_CFontPropPage       5f8ad848  
 0002:00014858       _CLSID_StdFont             5f8ad858  
 0002:00014868       _GUID_COLOR                5f8ad868  
 0002:00014878       _CLSID_CDAODBEngine        5f8ad878  
 0002:00014888       _CLSID35_CDAODBEngine      5f8ad888  
 0002:00014898       _IID_IDAODBEngineW         5f8ad898  
 0002:000148a8       _IID_ICDAORecordset        5f8ad8a8  
 0002:000148b8       _IID_IDAOFieldW            5f8ad8b8  
 0002:000148c8       _IID_IDAOIndexFieldsW      5f8ad8c8  
 0002:000148d8       _CLSID30_CDAODBEngine      5f8ad8d8  
 0002:000148e8       _IID30_IDAODBEngineW       5f8ad8e8  
 0002:000148f8       _IID30_IDAOFieldW          5f8ad8f8  
 0002:00014908       _IID30_IDAOIndexFieldsW    5f8ad908  
 0002:00014918       __sz_OLEPRO32              5f8ad918  
 0002:00014928       __sz_WINSPOOL              5f8ad928  
 0002:00014938       __sz_WININET               5f8ad938  
 0002:00014948       __sz_WSOCK32               5f8ad948  
 0002:00014958       __sz_oledlg                5f8ad958  
 0002:00014968       __sz_urlmon                5f8ad968  
 0002:00014978       __sz_ODBC32                5f8ad978  
 0002:00014988       ??_R1A@?0A@A@CArchiveException@@8 5f8ad988  
 0002:000149a0       ??_R2CArchiveException@@8  5f8ad9a0  
 0002:000149b0       ??_R3CArchiveException@@8  5f8ad9b0  
 0002:000149c0       ??_R4CArchiveException@@6B@ 5f8ad9c0  
 0002:000149d8       ??_R1A@?0A@A@ISequentialStream@@8 5f8ad9d8  
 0002:000149f0       ??_R1A@?0A@A@IStream@@8    5f8ad9f0  
 0002:00014a08       ??_R1A@?0A@A@CArchiveStream@@8 5f8ada08  
 0002:00014a20       ??_R2CArchiveStream@@8     5f8ada20  
 0002:00014a38       ??_R3CArchiveStream@@8     5f8ada38  
 0002:00014a48       ??_R4CArchiveStream@@6B@   5f8ada48  
 0002:00014a60       ??_R1A@?0A@A@CStdioFile@@8 5f8ada60  
 0002:00014a78       ??_R2CStdioFile@@8         5f8ada78  
 0002:00014a88       ??_R3CStdioFile@@8         5f8ada88  
 0002:00014a98       ??_R4CStdioFile@@6B@       5f8ada98  
 0002:00014ab0       ??_R1A@?0A@A@CSharedFile@@8 5f8adab0  
 0002:00014ac8       ??_R2CSharedFile@@8        5f8adac8  
 0002:00014ae0       ??_R3CSharedFile@@8        5f8adae0  
 0002:00014af0       ??_R4CSharedFile@@6B@      5f8adaf0  
 0002:00014b08       ??_R1A@?0A@A@CByteArray@@8 5f8adb08  
 0002:00014b20       ??_R2CByteArray@@8         5f8adb20  
 0002:00014b30       ??_R3CByteArray@@8         5f8adb30  
 0002:00014b40       ??_R4CByteArray@@6B@       5f8adb40  
 0002:00014b58       ??_R1A@?0A@A@CObArray@@8   5f8adb58  
 0002:00014b70       ??_R2CObArray@@8           5f8adb70  
 0002:00014b80       ??_R3CObArray@@8           5f8adb80  
 0002:00014b90       ??_R4CObArray@@6B@         5f8adb90  
 0002:00014ba8       ??_R1A@?0A@A@CStringArray@@8 5f8adba8  
 0002:00014bc0       ??_R2CStringArray@@8       5f8adbc0  
 0002:00014bd0       ??_R3CStringArray@@8       5f8adbd0  
 0002:00014be0       ??_R4CStringArray@@6B@     5f8adbe0  
 0002:00014bf8       ??_R1A@?0A@A@CUIntArray@@8 5f8adbf8  
 0002:00014c10       ??_R2CUIntArray@@8         5f8adc10  
 0002:00014c20       ??_R3CUIntArray@@8         5f8adc20  
 0002:00014c30       ??_R4CUIntArray@@6B@       5f8adc30  
 0002:00014c48       ??_R1A@?0A@A@CWordArray@@8 5f8adc48  
 0002:00014c60       ??_R2CWordArray@@8         5f8adc60  
 0002:00014c70       ??_R3CWordArray@@8         5f8adc70  
 0002:00014c80       ??_R4CWordArray@@6B@       5f8adc80  
 0002:00014c98       ??_R1A@?0A@A@CStringList@@8 5f8adc98  
 0002:00014cb0       ??_R2CStringList@@8        5f8adcb0  
 0002:00014cc0       ??_R3CStringList@@8        5f8adcc0  
 0002:00014cd0       ??_R4CStringList@@6B@      5f8adcd0  
 0002:00014ce8       ??_R1A@?0A@A@CMapPtrToWord@@8 5f8adce8  
 0002:00014d00       ??_R2CMapPtrToWord@@8      5f8add00  
 0002:00014d10       ??_R3CMapPtrToWord@@8      5f8add10  
 0002:00014d20       ??_R4CMapPtrToWord@@6B@    5f8add20  
 0002:00014d38       ??_R1A@?0A@A@CMapStringToOb@@8 5f8add38  
 0002:00014d50       ??_R2CMapStringToOb@@8     5f8add50  
 0002:00014d60       ??_R3CMapStringToOb@@8     5f8add60  
 0002:00014d70       ??_R4CMapStringToOb@@6B@   5f8add70  
 0002:00014d88       ??_R1A@?0A@A@CMapStringToString@@8 5f8add88  
 0002:00014da0       ??_R2CMapStringToString@@8 5f8adda0  
 0002:00014db0       ??_R3CMapStringToString@@8 5f8addb0  
 0002:00014dc0       ??_R4CMapStringToString@@6B@ 5f8addc0  
 0002:00014dd8       ??_R1A@?0A@A@CMapWordToOb@@8 5f8addd8  
 0002:00014df0       ??_R2CMapWordToOb@@8       5f8addf0  
 0002:00014e00       ??_R3CMapWordToOb@@8       5f8ade00  
 0002:00014e10       ??_R4CMapWordToOb@@6B@     5f8ade10  
 0002:00014e28       ??_R1A@?0A@A@CMapWordToPtr@@8 5f8ade28  
 0002:00014e40       ??_R2CMapWordToPtr@@8      5f8ade40  
 0002:00014e50       ??_R3CMapWordToPtr@@8      5f8ade50  
 0002:00014e60       ??_R4CMapWordToPtr@@6B@    5f8ade60  
 0002:00014e78       ??_R1A@?0A@A@CSemaphore@@8 5f8ade78  
 0002:00014e90       ??_R2CSemaphore@@8         5f8ade90  
 0002:00014ea0       ??_R3CSemaphore@@8         5f8adea0  
 0002:00014eb0       ??_R4CSemaphore@@6B@       5f8adeb0  
 0002:00014ec8       ??_R1A@?0A@A@CMutex@@8     5f8adec8  
 0002:00014ee0       ??_R2CMutex@@8             5f8adee0  
 0002:00014ef0       ??_R3CMutex@@8             5f8adef0  
 0002:00014f00       ??_R4CMutex@@6B@           5f8adf00  
 0002:00014f18       ??_R1A@?0A@A@CEvent@@8     5f8adf18  
 0002:00014f30       ??_R2CEvent@@8             5f8adf30  
 0002:00014f40       ??_R3CEvent@@8             5f8adf40  
 0002:00014f50       ??_R4CEvent@@6B@           5f8adf50  
 0002:00014f68       ??_R1A@?0A@A@CToolTipCtrl@@8 5f8adf68  
 0002:00014f80       ??_R2CToolTipCtrl@@8       5f8adf80  
 0002:00014f98       ??_R3CToolTipCtrl@@8       5f8adf98  
 0002:00014fa8       ??_R4CToolTipCtrl@@6B@     5f8adfa8  
 0002:00014fc0       ??_R1A@?0A@A@CMiniFrameWnd@@8 5f8adfc0  
 0002:00014fd8       ??_R2CMiniFrameWnd@@8      5f8adfd8  
 0002:00014ff0       ??_R3CMiniFrameWnd@@8      5f8adff0  
 0002:00015000       ??_R4CMiniFrameWnd@@6B@    5f8ae000  
 0002:00015018       ??_R1A@?0A@A@CBrush@@8     5f8ae018  
 0002:00015030       ??_R2CBrush@@8             5f8ae030  
 0002:00015040       ??_R3CBrush@@8             5f8ae040  
 0002:00015050       ??_R4CBrush@@6B@           5f8ae050  
 0002:00015068       ??_R1A@?0A@A@CDialogBar@@8 5f8ae068  
 0002:00015080       ??_R2CDialogBar@@8         5f8ae080  
 0002:00015098       ??_R3CDialogBar@@8         5f8ae098  
 0002:000150a8       ??_R4CDialogBar@@6B@       5f8ae0a8  
 0002:000150c0       ??_R1A@?0A@A@CMiniDockFrameWnd@@8 5f8ae0c0  
 0002:000150d8       ??_R2CMiniDockFrameWnd@@8  5f8ae0d8  
 0002:000150f8       ??_R3CMiniDockFrameWnd@@8  5f8ae0f8  
 0002:00015108       ??_R4CMiniDockFrameWnd@@6B@ 5f8ae108  
 0002:00015120       ??_R1A@?0A@A@CPreviewDC@@8 5f8ae120  
 0002:00015138       ??_R2CPreviewDC@@8         5f8ae138  
 0002:00015148       ??_R3CPreviewDC@@8         5f8ae148  
 0002:00015158       ??_R4CPreviewDC@@6B@       5f8ae158  
 0002:00015170       ??_R1A@?0A@A@CMetaFileDC@@8 5f8ae170  
 0002:00015188       ??_R2CMetaFileDC@@8        5f8ae188  
 0002:00015198       ??_R3CMetaFileDC@@8        5f8ae198  
 0002:000151a8       ??_R4CMetaFileDC@@6B@      5f8ae1a8  
 0002:000151c0       ??_R1A@?0A@A@CRectTracker@@8 5f8ae1c0  
 0002:000151d8       ??_R2CRectTracker@@8       5f8ae1d8  
 0002:000151e0       ??_R3CRectTracker@@8       5f8ae1e0  
 0002:000151f0       ??_R4CRectTracker@@6B@     5f8ae1f0  
 0002:00015208       ??_R1A@?0A@A@CReBar@@8     5f8ae208  
 0002:00015220       ??_R2CReBar@@8             5f8ae220  
 0002:00015238       ??_R3CReBar@@8             5f8ae238  
 0002:00015248       ??_R4CReBar@@6B@           5f8ae248  
 0002:00015260       ??_R1A@?0A@A@CListBox@@8   5f8ae260  
 0002:00015278       ??_R2CListBox@@8           5f8ae278  
 0002:00015290       ??_R3CListBox@@8           5f8ae290  
 0002:000152a0       ??_R4CListBox@@6B@         5f8ae2a0  
 0002:000152b8       ??_R1A@?0A@A@CScrollBar@@8 5f8ae2b8  
 0002:000152d0       ??_R2CScrollBar@@8         5f8ae2d0  
 0002:000152e8       ??_R3CScrollBar@@8         5f8ae2e8  
 0002:000152f8       ??_R4CScrollBar@@6B@       5f8ae2f8  
 0002:00015310       ??_R1A@?0A@A@CDragListBox@@8 5f8ae310  
 0002:00015328       ??_R2CDragListBox@@8       5f8ae328  
 0002:00015340       ??_R3CDragListBox@@8       5f8ae340  
 0002:00015350       ??_R4CDragListBox@@6B@     5f8ae350  
 0002:00015368       ??_R1A@?0A@A@CRgn@@8       5f8ae368  
 0002:00015380       ??_R2CRgn@@8               5f8ae380  
 0002:00015390       ??_R3CRgn@@8               5f8ae390  
 0002:000153a0       ??_R4CRgn@@6B@             5f8ae3a0  
 0002:000153b8       ??_R1A@?0A@A@CToolBarCtrl@@8 5f8ae3b8  
 0002:000153d0       ??_R2CToolBarCtrl@@8       5f8ae3d0  
 0002:000153e8       ??_R3CToolBarCtrl@@8       5f8ae3e8  
 0002:000153f8       ??_R4CToolBarCtrl@@6B@     5f8ae3f8  
 0002:00015410       ??_R1A@?0A@A@CStatusBarCtrl@@8 5f8ae410  
 0002:00015428       ??_R2CStatusBarCtrl@@8     5f8ae428  
 0002:00015440       ??_R3CStatusBarCtrl@@8     5f8ae440  
 0002:00015450       ??_R4CStatusBarCtrl@@6B@   5f8ae450  
 0002:00015468       ??_R1A@?0A@A@CListCtrl@@8  5f8ae468  
 0002:00015480       ??_R2CListCtrl@@8          5f8ae480  
 0002:00015498       ??_R3CListCtrl@@8          5f8ae498  
 0002:000154a8       ??_R4CListCtrl@@6B@        5f8ae4a8  
 0002:000154c0       ??_R1A@?0A@A@CTreeCtrl@@8  5f8ae4c0  
 0002:000154d8       ??_R2CTreeCtrl@@8          5f8ae4d8  
 0002:000154f0       ??_R3CTreeCtrl@@8          5f8ae4f0  
 0002:00015500       ??_R4CTreeCtrl@@6B@        5f8ae500  
 0002:00015518       ??_R1A@?0A@A@CSpinButtonCtrl@@8 5f8ae518  
 0002:00015530       ??_R2CSpinButtonCtrl@@8    5f8ae530  
 0002:00015548       ??_R3CSpinButtonCtrl@@8    5f8ae548  
 0002:00015558       ??_R4CSpinButtonCtrl@@6B@  5f8ae558  
 0002:00015570       ??_R1A@?0A@A@CSliderCtrl@@8 5f8ae570  
 0002:00015588       ??_R2CSliderCtrl@@8        5f8ae588  
 0002:000155a0       ??_R3CSliderCtrl@@8        5f8ae5a0  
 0002:000155b0       ??_R4CSliderCtrl@@6B@      5f8ae5b0  
 0002:000155c8       ??_R1A@?0A@A@CProgressCtrl@@8 5f8ae5c8  
 0002:000155e0       ??_R2CProgressCtrl@@8      5f8ae5e0  
 0002:000155f8       ??_R3CProgressCtrl@@8      5f8ae5f8  
 0002:00015608       ??_R4CProgressCtrl@@6B@    5f8ae608  
 0002:00015620       ??_R1A@?0A@A@CHeaderCtrl@@8 5f8ae620  
 0002:00015638       ??_R2CHeaderCtrl@@8        5f8ae638  
 0002:00015650       ??_R3CHeaderCtrl@@8        5f8ae650  
 0002:00015660       ??_R4CHeaderCtrl@@6B@      5f8ae660  
 0002:00015678       ??_R1A@?0A@A@CHotKeyCtrl@@8 5f8ae678  
 0002:00015690       ??_R2CHotKeyCtrl@@8        5f8ae690  
 0002:000156a8       ??_R3CHotKeyCtrl@@8        5f8ae6a8  
 0002:000156b8       ??_R4CHotKeyCtrl@@6B@      5f8ae6b8  
 0002:000156d0       ??_R1A@?0A@A@CTabCtrl@@8   5f8ae6d0  
 0002:000156e8       ??_R2CTabCtrl@@8           5f8ae6e8  
 0002:00015700       ??_R3CTabCtrl@@8           5f8ae700  
 0002:00015710       ??_R4CTabCtrl@@6B@         5f8ae710  
 0002:00015728       ??_R1A@?0A@A@CAnimateCtrl@@8 5f8ae728  
 0002:00015740       ??_R2CAnimateCtrl@@8       5f8ae740  
 0002:00015758       ??_R3CAnimateCtrl@@8       5f8ae758  
 0002:00015768       ??_R4CAnimateCtrl@@6B@     5f8ae768  
 0002:00015780       ??_R1A@?0A@A@CRichEditCtrl@@8 5f8ae780  
 0002:00015798       ??_R2CRichEditCtrl@@8      5f8ae798  
 0002:000157b0       ??_R3CRichEditCtrl@@8      5f8ae7b0  
 0002:000157c0       ??_R4CRichEditCtrl@@6B@    5f8ae7c0  
 0002:000157d8       ??_R1A@?0A@A@CImageList@@8 5f8ae7d8  
 0002:000157f0       ??_R2CImageList@@8         5f8ae7f0  
 0002:00015800       ??_R3CImageList@@8         5f8ae800  
 0002:00015810       ??_R4CImageList@@6B@       5f8ae810  
 0002:00015828       ??_R1A@?0A@A@CTempImageList@@8 5f8ae828  
 0002:00015840       ??_R2CTempImageList@@8     5f8ae840  
 0002:00015850       ??_R3CTempImageList@@8     5f8ae850  
 0002:00015860       ??_R4CTempImageList@@6B@   5f8ae860  
 0002:00015878       ??_R1A@?0A@A@CBitmap@@8    5f8ae878  
 0002:00015890       ??_R2CBitmap@@8            5f8ae890  
 0002:000158a0       ??_R3CBitmap@@8            5f8ae8a0  
 0002:000158b0       ??_R4CBitmap@@6B@          5f8ae8b0  
 0002:000158c8       ??_R1A@?0A@A@_AFX_CHECKLIST_STATE@@8 5f8ae8c8  
 0002:000158e0       ??_R2_AFX_CHECKLIST_STATE@@8 5f8ae8e0  
 0002:000158f0       ??_R3_AFX_CHECKLIST_STATE@@8 5f8ae8f0  
 0002:00015900       ??_R4_AFX_CHECKLIST_STATE@@6B@ 5f8ae900  
 0002:00015918       ??_R1A@?0A@A@CPropertyPage@@8 5f8ae918  
 0002:00015930       ??_R2CPropertyPage@@8      5f8ae930  
 0002:00015948       ??_R3CPropertyPage@@8      5f8ae948  
 0002:00015958       ??_R4CPropertyPage@@6B@    5f8ae958  
 0002:00015970       ??_R1A@?0A@A@CPropertySheet@@8 5f8ae970  
 0002:00015988       ??_R2CPropertySheet@@8     5f8ae988  
 0002:000159a0       ??_R3CPropertySheet@@8     5f8ae9a0  
 0002:000159b0       ??_R4CPropertySheet@@6B@   5f8ae9b0  
 0002:000159c8       ??_R1A@?0A@A@CPropertyPageEx@@8 5f8ae9c8  
 0002:000159e0       ??_R2CPropertyPageEx@@8    5f8ae9e0  
 0002:00015a00       ??_R3CPropertyPageEx@@8    5f8aea00  
 0002:00015a10       ??_R4CPropertyPageEx@@6B@  5f8aea10  
 0002:00015a28       ??_R1A@?0A@A@CPropertySheetEx@@8 5f8aea28  
 0002:00015a40       ??_R2CPropertySheetEx@@8   5f8aea40  
 0002:00015a58       ??_R3CPropertySheetEx@@8   5f8aea58  
 0002:00015a68       ??_R4CPropertySheetEx@@6B@ 5f8aea68  
 0002:00015a80       ??_R1A@?0A@A@CFileDialog@@8 5f8aea80  
 0002:00015a98       ??_R2CFileDialog@@8        5f8aea98  
 0002:00015ab8       ??_R3CFileDialog@@8        5f8aeab8  
 0002:00015ac8       ??_R4CFileDialog@@6B@      5f8aeac8  
 0002:00015ae0       ??_R2CCommonDialog@@8      5f8aeae0  
 0002:00015af8       ??_R3CCommonDialog@@8      5f8aeaf8  
 0002:00015b08       ??_R4CCommonDialog@@6B@    5f8aeb08  
 0002:00015b20       ??_R1A@?0A@A@CPageSetupDialog@@8 5f8aeb20  
 0002:00015b38       ??_R2CPageSetupDialog@@8   5f8aeb38  
 0002:00015b58       ??_R3CPageSetupDialog@@8   5f8aeb58  
 0002:00015b68       ??_R4CPageSetupDialog@@6B@ 5f8aeb68  
 0002:00015b80       ??_R1A@?0A@A@_AFX_COLOR_STATE@@8 5f8aeb80  
 0002:00015b98       ??_R2_AFX_COLOR_STATE@@8   5f8aeb98  
 0002:00015ba8       ??_R3_AFX_COLOR_STATE@@8   5f8aeba8  
 0002:00015bb8       ??_R4_AFX_COLOR_STATE@@6B@ 5f8aebb8  
 0002:00015bd0       ??_R1A@?0A@A@CColorDialog@@8 5f8aebd0  
 0002:00015be8       ??_R2CColorDialog@@8       5f8aebe8  
 0002:00015c08       ??_R3CColorDialog@@8       5f8aec08  
 0002:00015c18       ??_R4CColorDialog@@6B@     5f8aec18  
 0002:00015c30       ??_R1A@?0A@A@CFontDialog@@8 5f8aec30  
 0002:00015c48       ??_R2CFontDialog@@8        5f8aec48  
 0002:00015c68       ??_R3CFontDialog@@8        5f8aec68  
 0002:00015c78       ??_R4CFontDialog@@6B@      5f8aec78  
 0002:00015c90       ??_R1A@?0A@A@CFindReplaceDialog@@8 5f8aec90  
 0002:00015ca8       ??_R2CFindReplaceDialog@@8 5f8aeca8  
 0002:00015cc8       ??_R3CFindReplaceDialog@@8 5f8aecc8  
 0002:00015cd8       ??_R4CFindReplaceDialog@@6B@ 5f8aecd8  
 0002:00015cf0       ??_R1A@?0A@A@_AFX_PROPPAGEFONTINFO@@8 5f8aecf0  
 0002:00015d08       ??_R2_AFX_PROPPAGEFONTINFO@@8 5f8aed08  
 0002:00015d18       ??_R3_AFX_PROPPAGEFONTINFO@@8 5f8aed18  
 0002:00015d28       ??_R4_AFX_PROPPAGEFONTINFO@@6B@ 5f8aed28  
 0002:00015d40       ??_R1A@?0A@A@CIPAddressCtrl@@8 5f8aed40  
 0002:00015d58       ??_R2CIPAddressCtrl@@8     5f8aed58  
 0002:00015d70       ??_R3CIPAddressCtrl@@8     5f8aed70  
 0002:00015d80       ??_R4CIPAddressCtrl@@6B@   5f8aed80  
 0002:00015d98       ??_R1A@?0A@A@CComboBoxEx@@8 5f8aed98  
 0002:00015db0       ??_R2CComboBoxEx@@8        5f8aedb0  
 0002:00015dc8       ??_R3CComboBoxEx@@8        5f8aedc8  
 0002:00015dd8       ??_R4CComboBoxEx@@6B@      5f8aedd8  
 0002:00015df0       ??_R1A@?0A@A@CPen@@8       5f8aedf0  
 0002:00015e08       ??_R2CPen@@8               5f8aee08  
 0002:00015e18       ??_R3CPen@@8               5f8aee18  
 0002:00015e28       ??_R4CPen@@6B@             5f8aee28  
 0002:00015e40       ??_R1A@?0A@A@CMirrorFile@@8 5f8aee40  
 0002:00015e58       ??_R2CMirrorFile@@8        5f8aee58  
 0002:00015e68       ??_R3CMirrorFile@@8        5f8aee68  
 0002:00015e78       ??_R4CMirrorFile@@6B@      5f8aee78  
 0002:00015e90       ??_R1A@?0A@A@CNewTypeDlg@@8 5f8aee90  
 0002:00015ea8       ??_R2CNewTypeDlg@@8        5f8aeea8  
 0002:00015ec0       ??_R3CNewTypeDlg@@8        5f8aeec0  
 0002:00015ed0       ??_R4CNewTypeDlg@@6B@      5f8aeed0  
 0002:00015ee8       ??_R1A@?0A@A@CSplitterWnd@@8 5f8aeee8  
 0002:00015f00       ??_R2CSplitterWnd@@8       5f8aef00  
 0002:00015f18       ??_R3CSplitterWnd@@8       5f8aef18  
 0002:00015f28       ??_R4CSplitterWnd@@6B@     5f8aef28  
 0002:00015f40       ??_R1A@?0A@A@CFormView@@8  5f8aef40  
 0002:00015f58       ??_R2CFormView@@8          5f8aef58  
 0002:00015f78       ??_R3CFormView@@8          5f8aef78  
 0002:00015f88       ??_R4CFormView@@6B@        5f8aef88  
 0002:00015fa0       ??_R1A@?0A@A@CEditView@@8  5f8aefa0  
 0002:00015fb8       ??_R2CEditView@@8          5f8aefb8  
 0002:00015fd8       ??_R3CEditView@@8          5f8aefd8  
 0002:00015fe8       ??_R4CEditView@@6B@        5f8aefe8  
 0002:00016000       ??_R1A@?0A@A@CPreviewView@@8 5f8af000  
 0002:00016018       ??_R2CPreviewView@@8       5f8af018  
 0002:00016038       ??_R3CPreviewView@@8       5f8af038  
 0002:00016048       ??_R4CPreviewView@@6B@     5f8af048  
 0002:00016060       ??_R1A@?0A@A@CListView@@8  5f8af060  
 0002:00016078       ??_R2CListView@@8          5f8af078  
 0002:00016098       ??_R3CListView@@8          5f8af098  
 0002:000160a8       ??_R4CListView@@6B@        5f8af0a8  
 0002:000160c0       ??_R1A@?0A@A@CTreeView@@8  5f8af0c0  
 0002:000160d8       ??_R2CTreeView@@8          5f8af0d8  
 0002:000160f8       ??_R3CTreeView@@8          5f8af0f8  
 0002:00016108       ??_R4CTreeView@@6B@        5f8af108  
 0002:00016120       ??_R1A@?0A@A@_AFX_MAIL_STATE@@8 5f8af120  
 0002:00016138       ??_R2_AFX_MAIL_STATE@@8    5f8af138  
 0002:00016148       ??_R3_AFX_MAIL_STATE@@8    5f8af148  
 0002:00016158       ??_R4_AFX_MAIL_STATE@@6B@  5f8af158  
 0002:00016170       ??_R1A@?0A@A@CInternetSession@@8 5f8af170  
 0002:00016188       ??_R2CInternetSession@@8   5f8af188  
 0002:00016198       ??_R3CInternetSession@@8   5f8af198  
 0002:000161a8       ??_R4CInternetSession@@6B@ 5f8af1a8  
 0002:000161c0       ??_R1A@?0A@A@CInternetFile@@8 5f8af1c0  
 0002:000161d8       ??_R2CInternetFile@@8      5f8af1d8  
 0002:000161f0       ??_R3CInternetFile@@8      5f8af1f0  
 0002:00016200       ??_R4CInternetFile@@6B@    5f8af200  
 0002:00016218       ??_R1A@?0A@A@CInternetConnection@@8 5f8af218  
 0002:00016230       ??_R2CInternetConnection@@8 5f8af230  
 0002:00016240       ??_R3CInternetConnection@@8 5f8af240  
 0002:00016250       ??_R4CInternetConnection@@6B@ 5f8af250  
 0002:00016268       ??_R1A@?0A@A@CFtpConnection@@8 5f8af268  
 0002:00016280       ??_R2CFtpConnection@@8     5f8af280  
 0002:00016290       ??_R3CFtpConnection@@8     5f8af290  
 0002:000162a0       ??_R4CFtpConnection@@6B@   5f8af2a0  
 0002:000162b8       ??_R1A@?0A@A@CGopherConnection@@8 5f8af2b8  
 0002:000162d0       ??_R2CGopherConnection@@8  5f8af2d0  
 0002:000162e0       ??_R3CGopherConnection@@8  5f8af2e0  
 0002:000162f0       ??_R4CGopherConnection@@6B@ 5f8af2f0  
 0002:00016308       ??_R1A@?0A@A@CHttpConnection@@8 5f8af308  
 0002:00016320       ??_R2CHttpConnection@@8    5f8af320  
 0002:00016330       ??_R3CHttpConnection@@8    5f8af330  
 0002:00016340       ??_R4CHttpConnection@@6B@  5f8af340  
 0002:00016358       ??_R1A@?0A@A@CHttpFile@@8  5f8af358  
 0002:00016370       ??_R2CHttpFile@@8          5f8af370  
 0002:00016388       ??_R3CHttpFile@@8          5f8af388  
 0002:00016398       ??_R4CHttpFile@@6B@        5f8af398  
 0002:000163b0       ??_R1A@?0A@A@CGopherFile@@8 5f8af3b0  
 0002:000163c8       ??_R2CGopherFile@@8        5f8af3c8  
 0002:000163e0       ??_R3CGopherFile@@8        5f8af3e0  
 0002:000163f0       ??_R4CGopherFile@@6B@      5f8af3f0  
 0002:00016408       ??_R1A@?0A@A@CFileFind@@8  5f8af408  
 0002:00016420       ??_R1A@?0A@A@CFtpFileFind@@8 5f8af420  
 0002:00016438       ??_R2CFtpFileFind@@8       5f8af438  
 0002:00016448       ??_R3CFtpFileFind@@8       5f8af448  
 0002:00016458       ??_R4CFtpFileFind@@6B@     5f8af458  
 0002:00016470       ??_R1A@?0A@A@CGopherFileFind@@8 5f8af470  
 0002:00016488       ??_R2CGopherFileFind@@8    5f8af488  
 0002:00016498       ??_R3CGopherFileFind@@8    5f8af498  
 0002:000164a8       ??_R4CGopherFileFind@@6B@  5f8af4a8  
 0002:000164c0       ??_R1A@?0A@A@CGopherLocator@@8 5f8af4c0  
 0002:000164d8       ??_R2CGopherLocator@@8     5f8af4d8  
 0002:000164e8       ??_R3CGopherLocator@@8     5f8af4e8  
 0002:000164f8       ??_R4CGopherLocator@@6B@   5f8af4f8  
 0002:00016510       ??_R1A@?0A@A@CInternetException@@8 5f8af510  
 0002:00016528       ??_R2CInternetException@@8 5f8af528  
 0002:00016538       ??_R3CInternetException@@8 5f8af538  
 0002:00016548       ??_R4CInternetException@@6B@ 5f8af548  
 0002:00016560       ??_R2CFileFind@@8          5f8af560  
 0002:00016570       ??_R3CFileFind@@8          5f8af570  
 0002:00016580       ??_R4CFileFind@@6B@        5f8af580  
 0002:00016598       ??_R1A@?0A@A@_AFX_SOCK_STATE@@8 5f8af598  
 0002:000165b0       ??_R2_AFX_SOCK_STATE@@8    5f8af5b0  
 0002:000165c0       ??_R3_AFX_SOCK_STATE@@8    5f8af5c0  
 0002:000165d0       ??_R4_AFX_SOCK_STATE@@6B@  5f8af5d0  
 0002:000165e8       ??_R1A@?0A@A@CAsyncSocket@@8 5f8af5e8  
 0002:00016600       ??_R2CAsyncSocket@@8       5f8af600  
 0002:00016610       ??_R3CAsyncSocket@@8       5f8af610  
 0002:00016620       ??_R4CAsyncSocket@@6B@     5f8af620  
 0002:00016638       ??_R1A@?0A@A@CSocket@@8    5f8af638  
 0002:00016650       ??_R2CSocket@@8            5f8af650  
 0002:00016660       ??_R3CSocket@@8            5f8af660  
 0002:00016670       ??_R4CSocket@@6B@          5f8af670  
 0002:00016688       ??_R1A@?0A@A@CSocketFile@@8 5f8af688  
 0002:000166a0       ??_R2CSocketFile@@8        5f8af6a0  
 0002:000166b0       ??_R3CSocketFile@@8        5f8af6b0  
 0002:000166c0       ??_R4CSocketFile@@6B@      5f8af6c0  
 0002:000166d8       ??_R1A@?0A@A@CSocketWnd@@8 5f8af6d8  
 0002:000166f0       ??_R2CSocketWnd@@8         5f8af6f0  
 0002:00016708       ??_R3CSocketWnd@@8         5f8af708  
 0002:00016718       ??_R4CSocketWnd@@6B@       5f8af718  
 0002:00016730       ??_R1A@?0A@A@IOleInPlaceSite@@8 5f8af730  
 0002:00016748       ??_R1A@?0A@A@XOleIPSite@COleClientItem@@8 5f8af748  
 0002:00016760       ??_R2XOleIPSite@COleClientItem@@8 5f8af760  
 0002:00016778       ??_R3XOleIPSite@COleClientItem@@8 5f8af778  
 0002:00016788       ??_R4XOleIPSite@COleClientItem@@6B@ 5f8af788  
 0002:000167a0       ??_R1A@?0A@A@IAdviseSink@@8 5f8af7a0  
 0002:000167b8       ??_R1A@?0A@A@XAdviseSink@COleClientItem@@8 5f8af7b8  
 0002:000167d0       ??_R2XAdviseSink@COleClientItem@@8 5f8af7d0  
 0002:000167e0       ??_R3XAdviseSink@COleClientItem@@8 5f8af7e0  
 0002:000167f0       ??_R4XAdviseSink@COleClientItem@@6B@ 5f8af7f0  
 0002:00016808       ??_R1A@?0A@A@IOleClientSite@@8 5f8af808  
 0002:00016820       ??_R1A@?0A@A@XOleClientSite@COleClientItem@@8 5f8af820  
 0002:00016838       ??_R2XOleClientSite@COleClientItem@@8 5f8af838  
 0002:00016848       ??_R3XOleClientSite@COleClientItem@@8 5f8af848  
 0002:00016858       ??_R4XOleClientSite@COleClientItem@@6B@ 5f8af858  
 0002:00016870       ??_R1A@?0A@A@CDocItem@@8   5f8af870  
 0002:00016888       ??_R1A@?0A@A@COleClientItem@@8 5f8af888  
 0002:000168a0       ??_R2COleClientItem@@8     5f8af8a0  
 0002:000168b8       ??_R3COleClientItem@@8     5f8af8b8  
 0002:000168c8       ??_R4COleClientItem@@6B@   5f8af8c8  
 0002:000168e0       ??_R1A@?0A@A@COleFrameHook@@8 5f8af8e0  
 0002:000168f8       ??_R2COleFrameHook@@8      5f8af8f8  
 0002:00016908       ??_R3COleFrameHook@@8      5f8af908  
 0002:00016918       ??_R4COleFrameHook@@6B@    5f8af918  
 0002:00016930       ??_R1A@?0A@A@IOleCommandTarget@@8 5f8af930  
 0002:00016948       ??_R1A@?0A@A@XOleCommandTarget@COleFrameHook@@8 5f8af948  
 0002:00016960       ??_R2XOleCommandTarget@COleFrameHook@@8 5f8af960  
 0002:00016970       ??_R3XOleCommandTarget@COleFrameHook@@8 5f8af970  
 0002:00016980       ??_R4XOleCommandTarget@COleFrameHook@@6B@ 5f8af980  
 0002:00016998       ??_R1A@?0A@A@IOleInPlaceUIWindow@@8 5f8af998  
 0002:000169b0       ??_R1A@?0A@A@IOleInPlaceFrame@@8 5f8af9b0  
 0002:000169c8       ??_R1A@?0A@A@XOleInPlaceFrame@COleFrameHook@@8 5f8af9c8  
 0002:000169e0       ??_R2XOleInPlaceFrame@COleFrameHook@@8 5f8af9e0  
 0002:000169f8       ??_R3XOleInPlaceFrame@COleFrameHook@@8 5f8af9f8  
 0002:00016a08       ??_R4XOleInPlaceFrame@COleFrameHook@@6B@ 5f8afa08  
 0002:00016a20       ??_R1A@?0A@A@XDataObject@COleDataSource@@8 5f8afa20  
 0002:00016a38       ??_R2XDataObject@COleDataSource@@8 5f8afa38  
 0002:00016a48       ??_R3XDataObject@COleDataSource@@8 5f8afa48  
 0002:00016a58       ??_R4XDataObject@COleDataSource@@6B@ 5f8afa58  
 0002:00016a70       ??_R1A@?0A@A@COleDataSource@@8 5f8afa70  
 0002:00016a88       ??_R2COleDataSource@@8     5f8afa88  
 0002:00016a98       ??_R3COleDataSource@@8     5f8afa98  
 0002:00016aa8       ??_R4COleDataSource@@6B@   5f8afaa8  
 0002:00016ac0       ??_R1A@?0A@A@CEnumArray@@8 5f8afac0  
 0002:00016ad8       ??_R1A@?0A@A@CEnumFormatEtc@@8 5f8afad8  
 0002:00016af0       ??_R2CEnumFormatEtc@@8     5f8afaf0  
 0002:00016b08       ??_R3CEnumFormatEtc@@8     5f8afb08  
 0002:00016b18       ??_R4CEnumFormatEtc@@6B@   5f8afb18  
 0002:00016b30       ??_R1A@?0A@A@COleDispatchException@@8 5f8afb30  
 0002:00016b48       ??_R2COleDispatchException@@8 5f8afb48  
 0002:00016b58       ??_R3COleDispatchException@@8 5f8afb58  
 0002:00016b68       ??_R4COleDispatchException@@6B@ 5f8afb68  
 0002:00016b80       ??_R1A@?0A@A@IOleUILinkContainerW@@8 5f8afb80  
 0002:00016b98       ??_R1A@?0A@A@IOleUILinkInfoW@@8 5f8afb98  
 0002:00016bb0       ??_R1A@?0A@A@COleUILinkInfo@@8 5f8afbb0  
 0002:00016bc8       ??_R2COleUILinkInfo@@8     5f8afbc8  
 0002:00016be0       ??_R3COleUILinkInfo@@8     5f8afbe0  
 0002:00016bf0       ??_R4COleUILinkInfo@@6B@   5f8afbf0  
 0002:00016c08       ??_R1A@?0A@A@COleDialog@@8 5f8afc08  
 0002:00016c20       ??_R1A@?0A@A@COleInsertDialog@@8 5f8afc20  
 0002:00016c38       ??_R2COleInsertDialog@@8   5f8afc38  
 0002:00016c58       ??_R3COleInsertDialog@@8   5f8afc58  
 0002:00016c68       ??_R4COleInsertDialog@@6B@ 5f8afc68  
 0002:00016c80       ??_R1A@?0A@A@COleConvertDialog@@8 5f8afc80  
 0002:00016c98       ??_R2COleConvertDialog@@8  5f8afc98  
 0002:00016cb8       ??_R3COleConvertDialog@@8  5f8afcb8  
 0002:00016cc8       ??_R4COleConvertDialog@@6B@ 5f8afcc8  
 0002:00016ce0       ??_R1A@?0A@A@COleChangeIconDialog@@8 5f8afce0  
 0002:00016cf8       ??_R2COleChangeIconDialog@@8 5f8afcf8  
 0002:00016d18       ??_R3COleChangeIconDialog@@8 5f8afd18  
 0002:00016d28       ??_R4COleChangeIconDialog@@6B@ 5f8afd28  
 0002:00016d40       ??_R1A@?0A@A@COleLinksDialog@@8 5f8afd40  
 0002:00016d58       ??_R2COleLinksDialog@@8    5f8afd58  
 0002:00016d78       ??_R3COleLinksDialog@@8    5f8afd78  
 0002:00016d88       ??_R4COleLinksDialog@@6B@  5f8afd88  
 0002:00016da0       ??_R1A@?0A@A@COleUpdateDialog@@8 5f8afda0  
 0002:00016db8       ??_R2COleUpdateDialog@@8   5f8afdb8  
 0002:00016de0       ??_R3COleUpdateDialog@@8   5f8afde0  
 0002:00016df0       ??_R4COleUpdateDialog@@6B@ 5f8afdf0  
 0002:00016e08       ??_R1A@?0A@A@COlePasteSpecialDialog@@8 5f8afe08  
 0002:00016e20       ??_R2COlePasteSpecialDialog@@8 5f8afe20  
 0002:00016e40       ??_R3COlePasteSpecialDialog@@8 5f8afe40  
 0002:00016e50       ??_R4COlePasteSpecialDialog@@6B@ 5f8afe50  
 0002:00016e68       ??_R2COleDialog@@8         5f8afe68  
 0002:00016e88       ??_R3COleDialog@@8         5f8afe88  
 0002:00016e98       ??_R4COleDialog@@6B@       5f8afe98  
 0002:00016eb0       ??_R1A@?0A@A@COleBusyDialog@@8 5f8afeb0  
 0002:00016ec8       ??_R2COleBusyDialog@@8     5f8afec8  
 0002:00016ee8       ??_R3COleBusyDialog@@8     5f8afee8  
 0002:00016ef8       ??_R4COleBusyDialog@@6B@   5f8afef8  
 0002:00016f10       ??_R1A@?0A@A@COlePropertiesDialog@@8 5f8aff10  
 0002:00016f28       ??_R2COlePropertiesDialog@@8 5f8aff28  
 0002:00016f48       ??_R3COlePropertiesDialog@@8 5f8aff48  
 0002:00016f58       ??_R4COlePropertiesDialog@@6B@ 5f8aff58  
 0002:00016f70       ??_R1A@?0A@A@IOleUIObjInfoW@@8 5f8aff70  
 0002:00016f88       ??_R1A@?0A@A@XOleUIObjInfo@COlePropertiesDialog@@8 5f8aff88  
 0002:00016fa0       ??_R2XOleUIObjInfo@COlePropertiesDialog@@8 5f8affa0  
 0002:00016fb0       ??_R3XOleUIObjInfo@COlePropertiesDialog@@8 5f8affb0  
 0002:00016fc0       ??_R4XOleUIObjInfo@COlePropertiesDialog@@6B@ 5f8affc0  
 0002:00016fd8       ??_R1A@?0A@A@COleChangeSourceDialog@@8 5f8affd8  
 0002:00016ff0       ??_R2COleChangeSourceDialog@@8 5f8afff0  
 0002:00017010       ??_R3COleChangeSourceDialog@@8 5f8b0010  
 0002:00017020       ??_R4COleChangeSourceDialog@@6B@ 5f8b0020  
 0002:00017038       ??_R2CDocItem@@8           5f8b0038  
 0002:00017048       ??_R3CDocItem@@8           5f8b0048  
 0002:00017058       ??_R4CDocItem@@6B@         5f8b0058  
 0002:00017070       ??_R1A@?0A@A@COleDropSource@@8 5f8b0070  
 0002:00017088       ??_R2COleDropSource@@8     5f8b0088  
 0002:00017098       ??_R3COleDropSource@@8     5f8b0098  
 0002:000170a8       ??_R4COleDropSource@@6B@   5f8b00a8  
 0002:000170c0       ??_R1A@?0A@A@IDropSource@@8 5f8b00c0  
 0002:000170d8       ??_R1A@?0A@A@XDropSource@COleDropSource@@8 5f8b00d8  
 0002:000170f0       ??_R2XDropSource@COleDropSource@@8 5f8b00f0  
 0002:00017100       ??_R3XDropSource@COleDropSource@@8 5f8b0100  
 0002:00017110       ??_R4XDropSource@COleDropSource@@6B@ 5f8b0110  
 0002:00017128       ??_R1A@?0A@A@IEnumVOID@@8  5f8b0128  
 0002:00017140       ??_R1A@?0A@A@XEnumVOID@CEnumArray@@8 5f8b0140  
 0002:00017158       ??_R2XEnumVOID@CEnumArray@@8 5f8b0158  
 0002:00017168       ??_R3XEnumVOID@CEnumArray@@8 5f8b0168  
 0002:00017178       ??_R4XEnumVOID@CEnumArray@@6B@ 5f8b0178  
 0002:00017190       ??_R2CEnumArray@@8         5f8b0190  
 0002:000171a0       ??_R3CEnumArray@@8         5f8b01a0  
 0002:000171b0       ??_R4CEnumArray@@6B@       5f8b01b0  
 0002:000171c8       ??_R1A@?0A@A@COleCntrFrameWnd@@8 5f8b01c8  
 0002:000171e0       ??_R2COleCntrFrameWnd@@8   5f8b01e0  
 0002:000171f8       ??_R3COleCntrFrameWnd@@8   5f8b01f8  
 0002:00017208       ??_R4COleCntrFrameWnd@@6B@ 5f8b0208  
 0002:00017220       ??_R1A@?0A@A@COleIPFrameWnd@@8 5f8b0220  
 0002:00017238       ??_R2COleIPFrameWnd@@8     5f8b0238  
 0002:00017250       ??_R3COleIPFrameWnd@@8     5f8b0250  
 0002:00017260       ??_R4COleIPFrameWnd@@6B@   5f8b0260  
 0002:00017278       ??_R1A@?0A@A@COleException@@8 5f8b0278  
 0002:00017290       ??_R2COleException@@8      5f8b0290  
 0002:000172a0       ??_R3COleException@@8      5f8b02a0  
 0002:000172b0       ??_R4COleException@@6B@    5f8b02b0  
 0002:000172c8       ??_R1A@?0A@A@COleStreamFile@@8 5f8b02c8  
 0002:000172e0       ??_R2COleStreamFile@@8     5f8b02e0  
 0002:000172f0       ??_R3COleStreamFile@@8     5f8b02f0  
 0002:00017300       ??_R4COleStreamFile@@6B@   5f8b0300  
 0002:00017318       ??_R1A@?0A@A@XDataObject@COleServerItem@@8 5f8b0318  
 0002:00017330       ??_R2XDataObject@COleServerItem@@8 5f8b0330  
 0002:00017340       ??_R3XDataObject@COleServerItem@@8 5f8b0340  
 0002:00017350       ??_R4XDataObject@COleServerItem@@6B@ 5f8b0350  
 0002:00017368       ??_R1A@?0A@A@XOleObject@COleServerItem@@8 5f8b0368  
 0002:00017380       ??_R2XOleObject@COleServerItem@@8 5f8b0380  
 0002:00017390       ??_R3XOleObject@COleServerItem@@8 5f8b0390  
 0002:000173a0       ??_R4XOleObject@COleServerItem@@6B@ 5f8b03a0  
 0002:000173b8       ??_R1A@?0A@A@CItemDataSource@COleServerItem@@8 5f8b03b8  
 0002:000173d0       ??_R2CItemDataSource@COleServerItem@@8 5f8b03d0  
 0002:000173e8       ??_R3CItemDataSource@COleServerItem@@8 5f8b03e8  
 0002:000173f8       ??_R4CItemDataSource@COleServerItem@@6B@ 5f8b03f8  
 0002:00017410       ??_R1A@?0A@A@COleServerItem@@8 5f8b0410  
 0002:00017428       ??_R2COleServerItem@@8     5f8b0428  
 0002:00017440       ??_R3COleServerItem@@8     5f8b0440  
 0002:00017450       ??_R4COleServerItem@@6B@   5f8b0450  
 0002:00017468       ??_R1A@?0A@A@CInnerUnknown@@8 5f8b0468  
 0002:00017480       ??_R2CInnerUnknown@@8      5f8b0480  
 0002:00017490       ??_R3CInnerUnknown@@8      5f8b0490  
 0002:000174a0       ??_R4CInnerUnknown@@6B@    5f8b04a0  
 0002:000174b8       ??_R1A@?0A@A@CEnumOleVerb@@8 5f8b04b8  
 0002:000174d0       ??_R2CEnumOleVerb@@8       5f8b04d0  
 0002:000174e8       ??_R3CEnumOleVerb@@8       5f8b04e8  
 0002:000174f8       ??_R4CEnumOleVerb@@6B@     5f8b04f8  
 0002:00017510       ??_R1A@?0A@A@CRichEditCntrItem@@8 5f8b0510  
 0002:00017528       ??_R2CRichEditCntrItem@@8  5f8b0528  
 0002:00017540       ??_R3CRichEditCntrItem@@8  5f8b0540  
 0002:00017550       ??_R4CRichEditCntrItem@@6B@ 5f8b0550  
 0002:00017568       ??_R1A@?0A@A@CTypeLibCacheMap@@8 5f8b0568  
 0002:00017580       ??_R2CTypeLibCacheMap@@8   5f8b0580  
 0002:00017590       ??_R3CTypeLibCacheMap@@8   5f8b0590  
 0002:000175a0       ??_R4CTypeLibCacheMap@@6B@ 5f8b05a0  
 0002:000175b8       ??_R1A@?0A@A@CMonikerFile@@8 5f8b05b8  
 0002:000175d0       ??_R2CMonikerFile@@8       5f8b05d0  
 0002:000175e8       ??_R3CMonikerFile@@8       5f8b05e8  
 0002:000175f8       ??_R4CMonikerFile@@6B@     5f8b05f8  
 0002:00017610       ??_R1A@?0A@A@IBindHost@@8  5f8b0610  
 0002:00017628       ??_R1A@?0A@A@_AfxBindHost@@8 5f8b0628  
 0002:00017640       ??_R2_AfxBindHost@@8       5f8b0640  
 0002:00017650       ??_R3_AfxBindHost@@8       5f8b0650  
 0002:00017660       ??_R4_AfxBindHost@@6B@     5f8b0660  
 0002:00017678       ??_R2IBindHost@@8          5f8b0678  
 0002:00017688       ??_R3IBindHost@@8          5f8b0688  
 0002:00017698       ??_R4IBindHost@@6B@        5f8b0698  
 0002:000176b0       ??_R1A@?0A@A@CDateTimeCtrl@@8 5f8b06b0  
 0002:000176c8       ??_R2CDateTimeCtrl@@8      5f8b06c8  
 0002:000176e0       ??_R3CDateTimeCtrl@@8      5f8b06e0  
 0002:000176f0       ??_R4CDateTimeCtrl@@6B@    5f8b06f0  
 0002:00017708       ??_R1A@?0A@A@CMonthCalCtrl@@8 5f8b0708  
 0002:00017720       ??_R2CMonthCalCtrl@@8      5f8b0720  
 0002:00017738       ??_R3CMonthCalCtrl@@8      5f8b0738  
 0002:00017748       ??_R4CMonthCalCtrl@@6B@    5f8b0748  
 0002:00017760       ??_R1A@?0A@A@CHtmlView@@8  5f8b0760  
 0002:00017778       ??_R2CHtmlView@@8          5f8b0778  
 0002:00017798       ??_R3CHtmlView@@8          5f8b0798  
 0002:000177a8       ??_R4CHtmlView@@6B@        5f8b07a8  
 0002:000177c0       ??_R1A@?0A@A@COccManager@@8 5f8b07c0  
 0002:000177d8       ??_R2COccManager@@8        5f8b07d8  
 0002:000177e8       ??_R3COccManager@@8        5f8b07e8  
 0002:000177f8       ??_R4COccManager@@6B@      5f8b07f8  
 0002:00017810       ??_R1A@?0A@A@XOleIPFrame@COleControlContainer@@8 5f8b0810  
 0002:00017828       ??_R2XOleIPFrame@COleControlContainer@@8 5f8b0828  
 0002:00017840       ??_R3XOleIPFrame@COleControlContainer@@8 5f8b0840  
 0002:00017850       ??_R4XOleIPFrame@COleControlContainer@@6B@ 5f8b0850  
 0002:00017868       ??_R1A@?0A@A@XOleContainer@COleControlContainer@@8 5f8b0868  
 0002:00017880       ??_R2XOleContainer@COleControlContainer@@8 5f8b0880  
 0002:00017898       ??_R3XOleContainer@COleControlContainer@@8 5f8b0898  
 0002:000178a8       ??_R4XOleContainer@COleControlContainer@@6B@ 5f8b08a8  
 0002:000178c0       ??_R1A@?0A@A@COleControlContainer@@8 5f8b08c0  
 0002:000178d8       ??_R2COleControlContainer@@8 5f8b08d8  
 0002:000178e8       ??_R3COleControlContainer@@8 5f8b08e8  
 0002:000178f8       ??_R4COleControlContainer@@6B@ 5f8b08f8  
 0002:00017910       ??_R1A@?0A@A@CFont@@8      5f8b0910  
 0002:00017928       ??_R2CFont@@8              5f8b0928  
 0002:00017938       ??_R3CFont@@8              5f8b0938  
 0002:00017948       ??_R4CFont@@6B@            5f8b0948  
 0002:00017960       ??_R1A@?0A@A@CEnumUnknown@@8 5f8b0960  
 0002:00017978       ??_R2CEnumUnknown@@8       5f8b0978  
 0002:00017990       ??_R3CEnumUnknown@@8       5f8b0990  
 0002:000179a0       ??_R4CEnumUnknown@@6B@     5f8b09a0  
 0002:000179b8       ??_R1A@?0A@A@XEventSink@COleControlSite@@8 5f8b09b8  
 0002:000179d0       ??_R2XEventSink@COleControlSite@@8 5f8b09d0  
 0002:000179e0       ??_R3XEventSink@COleControlSite@@8 5f8b09e0  
 0002:000179f0       ??_R4XEventSink@COleControlSite@@6B@ 5f8b09f0  
 0002:00017a08       ??_R1A@?0A@A@IPropertyNotifySink@@8 5f8b0a08  
 0002:00017a20       ??_R1A@?0A@A@XPropertyNotifySink@COleControlSite@@8 5f8b0a20  
 0002:00017a38       ??_R2XPropertyNotifySink@COleControlSite@@8 5f8b0a38  
 0002:00017a48       ??_R3XPropertyNotifySink@COleControlSite@@8 5f8b0a48  
 0002:00017a58       ??_R4XPropertyNotifySink@COleControlSite@@6B@ 5f8b0a58  
 0002:00017a70       ??_R1A@?0A@A@XAmbientProps@COleControlSite@@8 5f8b0a70  
 0002:00017a88       ??_R2XAmbientProps@COleControlSite@@8 5f8b0a88  
 0002:00017a98       ??_R3XAmbientProps@COleControlSite@@8 5f8b0a98  
 0002:00017aa8       ??_R4XAmbientProps@COleControlSite@@6B@ 5f8b0aa8  
 0002:00017ac0       ??_R1A@?0A@A@IOleControlSite@@8 5f8b0ac0  
 0002:00017ad8       ??_R1A@?0A@A@XOleControlSite@COleControlSite@@8 5f8b0ad8  
 0002:00017af0       ??_R2XOleControlSite@COleControlSite@@8 5f8b0af0  
 0002:00017b00       ??_R3XOleControlSite@COleControlSite@@8 5f8b0b00  
 0002:00017b10       ??_R4XOleControlSite@COleControlSite@@6B@ 5f8b0b10  
 0002:00017b28       ??_R1A@?0A@A@XOleIPSite@COleControlSite@@8 5f8b0b28  
 0002:00017b40       ??_R2XOleIPSite@COleControlSite@@8 5f8b0b40  
 0002:00017b58       ??_R3XOleIPSite@COleControlSite@@8 5f8b0b58  
 0002:00017b68       ??_R4XOleIPSite@COleControlSite@@6B@ 5f8b0b68  
 0002:00017b80       ??_R1A@?0A@A@XOleClientSite@COleControlSite@@8 5f8b0b80  
 0002:00017b98       ??_R2XOleClientSite@COleControlSite@@8 5f8b0b98  
 0002:00017ba8       ??_R3XOleClientSite@COleControlSite@@8 5f8b0ba8  
 0002:00017bb8       ??_R4XOleClientSite@COleControlSite@@6B@ 5f8b0bb8  
 0002:00017bd0       ??_R1A@?0A@A@COleControlSite@@8 5f8b0bd0  
 0002:00017be8       ??_R2COleControlSite@@8    5f8b0be8  
 0002:00017bf8       ??_R3COleControlSite@@8    5f8b0bf8  
 0002:00017c08       ??_R4COleControlSite@@6B@  5f8b0c08  
 0002:00017c20       ??_R1A@?0A@A@IRowsetNotify@@8 5f8b0c20  
 0002:00017c38       ??_R1A@?0A@A@XRowsetNotify@COleControlSite@@8 5f8b0c38  
 0002:00017c50       ??_R2XRowsetNotify@COleControlSite@@8 5f8b0c50  
 0002:00017c60       ??_R3XRowsetNotify@COleControlSite@@8 5f8b0c60  
 0002:00017c70       ??_R4XRowsetNotify@COleControlSite@@6B@ 5f8b0c70  
 0002:00017c88       ??_R1A@?0A@A@INotifyDBEvents@@8 5f8b0c88  
 0002:00017ca0       ??_R1A@?0A@A@XNotifyDBEvents@COleControlSite@@8 5f8b0ca0  
 0002:00017cb8       ??_R2XNotifyDBEvents@COleControlSite@@8 5f8b0cb8  
 0002:00017cc8       ??_R3XNotifyDBEvents@COleControlSite@@8 5f8b0cc8  
 0002:00017cd8       ??_R4XNotifyDBEvents@COleControlSite@@6B@ 5f8b0cd8  
 0002:00017cf0       ??_R1A@?0A@A@IBoundObjectSite@@8 5f8b0cf0  
 0002:00017d08       ??_R1A@?0A@A@XBoundObjectSite@COleControlSite@@8 5f8b0d08  
 0002:00017d20       ??_R2XBoundObjectSite@COleControlSite@@8 5f8b0d20  
 0002:00017d30       ??_R3XBoundObjectSite@COleControlSite@@8 5f8b0d30  
 0002:00017d40       ??_R4XBoundObjectSite@COleControlSite@@6B@ 5f8b0d40  
 0002:00017d58       ??_R1A@?0A@A@CDataSourceControl@@8 5f8b0d58  
 0002:00017d70       ??_R2CDataSourceControl@@8 5f8b0d70  
 0002:00017d78       ??_R3CDataSourceControl@@8 5f8b0d78  
 0002:00017d88       ??_R4CDataSourceControl@@6B@ 5f8b0d88  
 0002:00017da0       ??_R1A@?0A@A@COleControlLock@@8 5f8b0da0  
 0002:00017db8       ??_R2COleControlLock@@8    5f8b0db8  
 0002:00017dc0       ??_R3COleControlLock@@8    5f8b0dc0  
 0002:00017dd0       ??_R4COleControlLock@@6B@  5f8b0dd0  
 0002:00017de8       ??_R1A@?0A@A@XOleObject@CDocObjectServer@@8 5f8b0de8  
 0002:00017e00       ??_R2XOleObject@CDocObjectServer@@8 5f8b0e00  
 0002:00017e10       ??_R3XOleObject@CDocObjectServer@@8 5f8b0e10  
 0002:00017e20       ??_R4XOleObject@CDocObjectServer@@6B@ 5f8b0e20  
 0002:00017e38       ??_R1A@?0A@A@IPrint@@8     5f8b0e38  
 0002:00017e50       ??_R1A@?0A@A@XPrint@CDocObjectServer@@8 5f8b0e50  
 0002:00017e68       ??_R2XPrint@CDocObjectServer@@8 5f8b0e68  
 0002:00017e78       ??_R3XPrint@CDocObjectServer@@8 5f8b0e78  
 0002:00017e88       ??_R4XPrint@CDocObjectServer@@6B@ 5f8b0e88  
 0002:00017ea0       ??_R1A@?0A@A@XOleCommandTarget@CDocObjectServer@@8 5f8b0ea0  
 0002:00017eb8       ??_R2XOleCommandTarget@CDocObjectServer@@8 5f8b0eb8  
 0002:00017ec8       ??_R3XOleCommandTarget@CDocObjectServer@@8 5f8b0ec8  
 0002:00017ed8       ??_R4XOleCommandTarget@CDocObjectServer@@6B@ 5f8b0ed8  
 0002:00017ef0       ??_R1A@?0A@A@IOleDocumentView@@8 5f8b0ef0  
 0002:00017f08       ??_R1A@?0A@A@XOleDocumentView@CDocObjectServer@@8 5f8b0f08  
 0002:00017f20       ??_R2XOleDocumentView@CDocObjectServer@@8 5f8b0f20  
 0002:00017f30       ??_R3XOleDocumentView@CDocObjectServer@@8 5f8b0f30  
 0002:00017f40       ??_R4XOleDocumentView@CDocObjectServer@@6B@ 5f8b0f40  
 0002:00017f58       ??_R1A@?0A@A@IOleDocument@@8 5f8b0f58  
 0002:00017f70       ??_R1A@?0A@A@XOleDocument@CDocObjectServer@@8 5f8b0f70  
 0002:00017f88       ??_R2XOleDocument@CDocObjectServer@@8 5f8b0f88  
 0002:00017f98       ??_R3XOleDocument@CDocObjectServer@@8 5f8b0f98  
 0002:00017fa8       ??_R4XOleDocument@CDocObjectServer@@6B@ 5f8b0fa8  
 0002:00017fc0       ??_R1A@?0A@A@CDocObjectServer@@8 5f8b0fc0  
 0002:00017fd8       ??_R2CDocObjectServer@@8   5f8b0fd8  
 0002:00017fe8       ??_R3CDocObjectServer@@8   5f8b0fe8  
 0002:00017ff8       ??_R4CDocObjectServer@@6B@ 5f8b0ff8  
 0002:00018010       ??_R1A@?0A@A@CDocObjectServerItem@@8 5f8b1010  
 0002:00018028       ??_R2CDocObjectServerItem@@8 5f8b1028  
 0002:00018040       ??_R3CDocObjectServerItem@@8 5f8b1040  
 0002:00018050       ??_R4CDocObjectServerItem@@6B@ 5f8b1050  
 0002:00018068       ??_R1A@?0A@A@COleCmdUI@@8  5f8b1068  
 0002:00018080       ??_R2COleCmdUI@@8          5f8b1080  
 0002:00018090       ??_R3COleCmdUI@@8          5f8b1090  
 0002:000180a0       ??_R4COleCmdUI@@6B@        5f8b10a0  
 0002:000180b8       ??_R1A@?0A@A@COleDocIPFrameWnd@@8 5f8b10b8  
 0002:000180d0       ??_R2COleDocIPFrameWnd@@8  5f8b10d0  
 0002:000180f0       ??_R3COleDocIPFrameWnd@@8  5f8b10f0  
 0002:00018100       ??_R4COleDocIPFrameWnd@@6B@ 5f8b1100  
 0002:00018118       ??_R1A@?0A@A@IOleDocumentSite@@8 5f8b1118  
 0002:00018130       ??_R1A@?0A@A@XOleDocumentSite@COleDocObjectItem@@8 5f8b1130  
 0002:00018148       ??_R2XOleDocumentSite@COleDocObjectItem@@8 5f8b1148  
 0002:00018158       ??_R3XOleDocumentSite@COleDocObjectItem@@8 5f8b1158  
 0002:00018168       ??_R4XOleDocumentSite@COleDocObjectItem@@6B@ 5f8b1168  
 0002:00018180       ??_R1A@?0A@A@COleDocObjectItem@@8 5f8b1180  
 0002:00018198       ??_R2COleDocObjectItem@@8  5f8b1198  
 0002:000181b0       ??_R3COleDocObjectItem@@8  5f8b11b0  
 0002:000181c0       ??_R4COleDocObjectItem@@6B@ 5f8b11c0  
 0002:000181d8       ??_R1A@?0A@A@CAsyncMonikerFile@@8 5f8b11d8  
 0002:000181f0       ??_R2CAsyncMonikerFile@@8  5f8b11f0  
 0002:00018208       ??_R3CAsyncMonikerFile@@8  5f8b1208  
 0002:00018218       ??_R4CAsyncMonikerFile@@6B@ 5f8b1218  
 0002:00018230       ??_R1A@?0A@A@IBindStatusCallback@@8 5f8b1230  
 0002:00018248       ??_R1A@?0A@A@_AfxBindStatusCallback@@8 5f8b1248  
 0002:00018260       ??_R2_AfxBindStatusCallback@@8 5f8b1260  
 0002:00018270       ??_R3_AfxBindStatusCallback@@8 5f8b1270  
 0002:00018280       ??_R4_AfxBindStatusCallback@@6B@ 5f8b1280  
 0002:00018298       ??_R1A@?0A@A@CInnerUnknown@_AfxBindStatusCallback@@8 5f8b1298  
 0002:000182b0       ??_R2CInnerUnknown@_AfxBindStatusCallback@@8 5f8b12b0  
 0002:000182c0       ??_R3CInnerUnknown@_AfxBindStatusCallback@@8 5f8b12c0  
 0002:000182d0       ??_R4CInnerUnknown@_AfxBindStatusCallback@@6B@ 5f8b12d0  
 0002:000182e8       ??_R2IBindStatusCallback@@8 5f8b12e8  
 0002:000182f8       ??_R3IBindStatusCallback@@8 5f8b12f8  
 0002:00018308       ??_R4IBindStatusCallback@@6B@ 5f8b1308  
 0002:00018320       ??_R1A@?0A@A@COleResizeBar@@8 5f8b1320  
 0002:00018338       ??_R2COleResizeBar@@8      5f8b1338  
 0002:00018350       ??_R3COleResizeBar@@8      5f8b1350  
 0002:00018360       ??_R4COleResizeBar@@6B@    5f8b1360  
 0002:00018378       ??_R1A@?0A@A@XOleInPlaceActiveObject@COleControl@@8 5f8b1378  
 0002:00018390       ??_R2XOleInPlaceActiveObject@COleControl@@8 5f8b1390  
 0002:000183a8       ??_R3XOleInPlaceActiveObject@COleControl@@8 5f8b13a8  
 0002:000183b8       ??_R4XOleInPlaceActiveObject@COleControl@@6B@ 5f8b13b8  
 0002:000183d0       ??_R1A@?0A@A@IOleInPlaceObjectWindowless@@8 5f8b13d0  
 0002:000183e8       ??_R1A@?0A@A@XOleInPlaceObject@COleControl@@8 5f8b13e8  
 0002:00018400       ??_R2XOleInPlaceObject@COleControl@@8 5f8b1400  
 0002:00018418       ??_R3XOleInPlaceObject@COleControl@@8 5f8b1418  
 0002:00018428       ??_R4XOleInPlaceObject@COleControl@@6B@ 5f8b1428  
 0002:00018440       ??_R1A@?0A@A@XDataObject@COleControl@@8 5f8b1440  
 0002:00018458       ??_R2XDataObject@COleControl@@8 5f8b1458  
 0002:00018468       ??_R3XDataObject@COleControl@@8 5f8b1468  
 0002:00018478       ??_R4XDataObject@COleControl@@6B@ 5f8b1478  
 0002:00018490       ??_R1A@?0A@A@COleControl@@8 5f8b1490  
 0002:000184a8       ??_R2COleControl@@8        5f8b14a8  
 0002:000184c0       ??_R3COleControl@@8        5f8b14c0  
 0002:000184d0       ??_R4COleControl@@6B@      5f8b14d0  
 0002:000184e8       ??_R1A@?0A@A@IViewObject@@8 5f8b14e8  
 0002:00018500       ??_R1A@?0A@A@IViewObject2@@8 5f8b1500  
 0002:00018518       ??_R1A@?0A@A@IViewObjectEx@@8 5f8b1518  
 0002:00018530       ??_R1A@?0A@A@XViewObject@COleControl@@8 5f8b1530  
 0002:00018548       ??_R2XViewObject@COleControl@@8 5f8b1548  
 0002:00018560       ??_R3XViewObject@COleControl@@8 5f8b1560  
 0002:00018570       ??_R4XViewObject@COleControl@@6B@ 5f8b1570  
 0002:00018588       ??_R1A@?0A@A@IQuickActivate@@8 5f8b1588  
 0002:000185a0       ??_R1A@?0A@A@XQuickActivate@COleControl@@8 5f8b15a0  
 0002:000185b8       ??_R2XQuickActivate@COleControl@@8 5f8b15b8  
 0002:000185c8       ??_R3XQuickActivate@COleControl@@8 5f8b15c8  
 0002:000185d8       ??_R4XQuickActivate@COleControl@@6B@ 5f8b15d8  
 0002:000185f0       ??_R1A@?0A@A@XOleObject@COleControl@@8 5f8b15f0  
 0002:00018608       ??_R2XOleObject@COleControl@@8 5f8b1608  
 0002:00018618       ??_R3XOleObject@COleControl@@8 5f8b1618  
 0002:00018628       ??_R4XOleObject@COleControl@@6B@ 5f8b1628  
 0002:00018640       ??_R1A@?0A@A@XFontNotification@COleControl@@8 5f8b1640  
 0002:00018658       ??_R2XFontNotification@COleControl@@8 5f8b1658  
 0002:00018668       ??_R3XFontNotification@COleControl@@8 5f8b1668  
 0002:00018678       ??_R4XFontNotification@COleControl@@6B@ 5f8b1678  
 0002:00018690       ??_R1A@?0A@A@IPersistPropertyBag@@8 5f8b1690  
 0002:000186a8       ??_R1A@?0A@A@XPersistPropertyBag@COleControl@@8 5f8b16a8  
 0002:000186c0       ??_R2XPersistPropertyBag@COleControl@@8 5f8b16c0  
 0002:000186d8       ??_R3XPersistPropertyBag@COleControl@@8 5f8b16d8  
 0002:000186e8       ??_R4XPersistPropertyBag@COleControl@@6B@ 5f8b16e8  
 0002:00018700       ??_R1A@?0A@A@IPerPropertyBrowsing@@8 5f8b1700  
 0002:00018718       ??_R1A@?0A@A@XPerPropertyBrowsing@COleControl@@8 5f8b1718  
 0002:00018730       ??_R2XPerPropertyBrowsing@COleControl@@8 5f8b1730  
 0002:00018740       ??_R3XPerPropertyBrowsing@COleControl@@8 5f8b1740  
 0002:00018750       ??_R4XPerPropertyBrowsing@COleControl@@6B@ 5f8b1750  
 0002:00018768       ??_R1A@?0A@A@IPersistMemory@@8 5f8b1768  
 0002:00018780       ??_R1A@?0A@A@XPersistMemory@COleControl@@8 5f8b1780  
 0002:00018798       ??_R2XPersistMemory@COleControl@@8 5f8b1798  
 0002:000187b0       ??_R3XPersistMemory@COleControl@@8 5f8b17b0  
 0002:000187c0       ??_R4XPersistMemory@COleControl@@6B@ 5f8b17c0  
 0002:000187d8       ??_R1A@?0A@A@ISpecifyPropertyPages@@8 5f8b17d8  
 0002:000187f0       ??_R1A@?0A@A@XSpecifyPropertyPages@COleControl@@8 5f8b17f0  
 0002:00018808       ??_R2XSpecifyPropertyPages@COleControl@@8 5f8b1808  
 0002:00018818       ??_R3XSpecifyPropertyPages@COleControl@@8 5f8b1818  
 0002:00018828       ??_R4XSpecifyPropertyPages@COleControl@@6B@ 5f8b1828  
 0002:00018840       ??_R1A@?0A@A@XPropConnPt@COleControl@@8 5f8b1840  
 0002:00018858       ??_R2XPropConnPt@COleControl@@8 5f8b1858  
 0002:00018870       ??_R3XPropConnPt@COleControl@@8 5f8b1870  
 0002:00018880       ??_R4XPropConnPt@COleControl@@6B@ 5f8b1880  
 0002:00018898       ??_R1A@?0A@A@IProvideClassInfo@@8 5f8b1898  
 0002:000188b0       ??_R1A@?0A@A@IProvideClassInfo2@@8 5f8b18b0  
 0002:000188c8       ??_R1A@?0A@A@XProvideClassInfo@COleControl@@8 5f8b18c8  
 0002:000188e0       ??_R2XProvideClassInfo@COleControl@@8 5f8b18e0  
 0002:000188f8       ??_R3XProvideClassInfo@COleControl@@8 5f8b18f8  
 0002:00018908       ??_R4XProvideClassInfo@COleControl@@6B@ 5f8b1908  
 0002:00018920       ??_R1A@?0A@A@IPersistStreamInit@@8 5f8b1920  
 0002:00018938       ??_R1A@?0A@A@XPersistStreamInit@COleControl@@8 5f8b1938  
 0002:00018950       ??_R2XPersistStreamInit@COleControl@@8 5f8b1950  
 0002:00018968       ??_R3XPersistStreamInit@COleControl@@8 5f8b1968  
 0002:00018978       ??_R4XPersistStreamInit@COleControl@@6B@ 5f8b1978  
 0002:00018990       ??_R1A@?0A@A@CConnectionPoint@@8 5f8b1990  
 0002:000189a8       ??_R1A@?0A@A@XEventConnPt@COleControl@@8 5f8b19a8  
 0002:000189c0       ??_R2XEventConnPt@COleControl@@8 5f8b19c0  
 0002:000189d8       ??_R3XEventConnPt@COleControl@@8 5f8b19d8  
 0002:000189e8       ??_R4XEventConnPt@COleControl@@6B@ 5f8b19e8  
 0002:00018a00       ??_R1A@?0A@A@IOleControl@@8 5f8b1a00  
 0002:00018a18       ??_R1A@?0A@A@XOleControl@COleControl@@8 5f8b1a18  
 0002:00018a30       ??_R2XOleControl@COleControl@@8 5f8b1a30  
 0002:00018a40       ??_R3XOleControl@COleControl@@8 5f8b1a40  
 0002:00018a50       ??_R4XOleControl@COleControl@@6B@ 5f8b1a50  
 0002:00018a68       ??_R1A@?0A@A@XPersistStorage@COleControl@@8 5f8b1a68  
 0002:00018a80       ??_R2XPersistStorage@COleControl@@8 5f8b1a80  
 0002:00018a98       ??_R3XPersistStorage@COleControl@@8 5f8b1a98  
 0002:00018aa8       ??_R4XPersistStorage@COleControl@@6B@ 5f8b1aa8  
 0002:00018ac0       ??_R1A@?0A@A@IPointerInactive@@8 5f8b1ac0  
 0002:00018ad8       ??_R1A@?0A@A@XPointerInactive@COleControl@@8 5f8b1ad8  
 0002:00018af0       ??_R2XPointerInactive@COleControl@@8 5f8b1af0  
 0002:00018b00       ??_R3XPointerInactive@COleControl@@8 5f8b1b00  
 0002:00018b10       ??_R4XPointerInactive@COleControl@@6B@ 5f8b1b10  
 0002:00018b28       ??_R1A@?0A@A@IOleCache@@8  5f8b1b28  
 0002:00018b40       ??_R1A@?0A@A@XOleCache@COleControl@@8 5f8b1b40  
 0002:00018b58       ??_R2XOleCache@COleControl@@8 5f8b1b58  
 0002:00018b68       ??_R3XOleCache@COleControl@@8 5f8b1b68  
 0002:00018b78       ??_R4XOleCache@COleControl@@6B@ 5f8b1b78  
 0002:00018b90       ??_R1A@?0A@A@CReflectorWnd@@8 5f8b1b90  
 0002:00018ba8       ??_R2CReflectorWnd@@8      5f8b1ba8  
 0002:00018bc0       ??_R3CReflectorWnd@@8      5f8b1bc0  
 0002:00018bd0       ??_R4CReflectorWnd@@6B@    5f8b1bd0  
 0002:00018be8       ??_R1A@?0A@A@CParkingWnd@@8 5f8b1be8  
 0002:00018c00       ??_R2CParkingWnd@@8        5f8b1c00  
 0002:00018c18       ??_R3CParkingWnd@@8        5f8b1c18  
 0002:00018c28       ??_R4CParkingWnd@@6B@      5f8b1c28  
 0002:00018c40       ??_R1A@?0A@A@CControlDataSource@COleControl@@8 5f8b1c40  
 0002:00018c58       ??_R2CControlDataSource@COleControl@@8 5f8b1c58  
 0002:00018c70       ??_R3CControlDataSource@COleControl@@8 5f8b1c70  
 0002:00018c80       ??_R4CControlDataSource@COleControl@@6B@ 5f8b1c80  
 0002:00018c98       ??_R1A@?0A@A@CControlFrameWnd@@8 5f8b1c98  
 0002:00018cb0       ??_R2CControlFrameWnd@@8   5f8b1cb0  
 0002:00018cc8       ??_R3CControlFrameWnd@@8   5f8b1cc8  
 0002:00018cd8       ??_R4CControlFrameWnd@@6B@ 5f8b1cd8  
 0002:00018cf0       ??_R1A@?0A@A@IConnectionPoint@@8 5f8b1cf0  
 0002:00018d08       ??_R1A@?0A@A@XConnPt@CConnectionPoint@@8 5f8b1d08  
 0002:00018d20       ??_R2XConnPt@CConnectionPoint@@8 5f8b1d20  
 0002:00018d30       ??_R3XConnPt@CConnectionPoint@@8 5f8b1d30  
 0002:00018d40       ??_R4XConnPt@CConnectionPoint@@6B@ 5f8b1d40  
 0002:00018d58       ??_R2CConnectionPoint@@8   5f8b1d58  
 0002:00018d68       ??_R3CConnectionPoint@@8   5f8b1d68  
 0002:00018d78       ??_R4CConnectionPoint@@6B@ 5f8b1d78  
 0002:00018d90       ??_R1A@?0A@A@CEnumConnections@@8 5f8b1d90  
 0002:00018da8       ??_R2CEnumConnections@@8   5f8b1da8  
 0002:00018dc0       ??_R3CEnumConnections@@8   5f8b1dc0  
 0002:00018dd0       ??_R4CEnumConnections@@6B@ 5f8b1dd0  
 0002:00018de8       ??_R1A@?0A@A@CEnumConnPoints@@8 5f8b1de8  
 0002:00018e00       ??_R2CEnumConnPoints@@8    5f8b1e00  
 0002:00018e18       ??_R3CEnumConnPoints@@8    5f8b1e18  
 0002:00018e28       ??_R4CEnumConnPoints@@6B@  5f8b1e28  
 0002:00018e40       ??_R1A@?0A@A@IConnectionPointContainer@@8 5f8b1e40  
 0002:00018e58       ??_R1A@?0A@A@COleConnPtContainer@@8 5f8b1e58  
 0002:00018e70       ??_R2COleConnPtContainer@@8 5f8b1e70  
 0002:00018e80       ??_R3COleConnPtContainer@@8 5f8b1e80  
 0002:00018e90       ??_R4COleConnPtContainer@@6B@ 5f8b1e90  
 0002:00018ea8       ??_R1A@?0A@A@CPropExchange@@8 5f8b1ea8  
 0002:00018ec0       ??_R1A@?0A@A@CArchivePropExchange@@8 5f8b1ec0  
 0002:00018ed8       ??_R2CArchivePropExchange@@8 5f8b1ed8  
 0002:00018ee8       ??_R3CArchivePropExchange@@8 5f8b1ee8  
 0002:00018ef8       ??_R4CArchivePropExchange@@6B@ 5f8b1ef8  
 0002:00018f10       ??_R1A@?0A@A@CResetPropExchange@@8 5f8b1f10  
 0002:00018f28       ??_R2CResetPropExchange@@8 5f8b1f28  
 0002:00018f38       ??_R3CResetPropExchange@@8 5f8b1f38  
 0002:00018f48       ??_R4CResetPropExchange@@6B@ 5f8b1f48  
 0002:00018f60       ??_R1A@?0A@A@CAsyncPropExchange@@8 5f8b1f60  
 0002:00018f78       ??_R2CAsyncPropExchange@@8 5f8b1f78  
 0002:00018f88       ??_R3CAsyncPropExchange@@8 5f8b1f88  
 0002:00018f98       ??_R4CAsyncPropExchange@@6B@ 5f8b1f98  
 0002:00018fb0       ??_R1A@?0A@A@AFX_DDPDATA@@8 5f8b1fb0  
 0002:00018fc8       ??_R2AFX_DDPDATA@@8        5f8b1fc8  
 0002:00018fd8       ??_R3AFX_DDPDATA@@8        5f8b1fd8  
 0002:00018fe8       ??_R4AFX_DDPDATA@@6B@      5f8b1fe8  
 0002:00019000       ??_R1A@?0A@A@COlePropertyPage@@8 5f8b2000  
 0002:00019018       ??_R2COlePropertyPage@@8   5f8b2018  
 0002:00019030       ??_R3COlePropertyPage@@8   5f8b2030  
 0002:00019040       ??_R4COlePropertyPage@@6B@ 5f8b2040  
 0002:00019058       ??_R1A@?0A@A@XPropNotifySink@COlePropertyPage@@8 5f8b2058  
 0002:00019070       ??_R2XPropNotifySink@COlePropertyPage@@8 5f8b2070  
 0002:00019080       ??_R3XPropNotifySink@COlePropertyPage@@8 5f8b2080  
 0002:00019090       ??_R4XPropNotifySink@COlePropertyPage@@6B@ 5f8b2090  
 0002:000190a8       ??_R1A@?0A@A@IPropertyPage@@8 5f8b20a8  
 0002:000190c0       ??_R1A@?0A@A@IPropertyPage2@@8 5f8b20c0  
 0002:000190d8       ??_R1A@?0A@A@XPropertyPage@COlePropertyPage@@8 5f8b20d8  
 0002:000190f0       ??_R2XPropertyPage@COlePropertyPage@@8 5f8b20f0  
 0002:00019108       ??_R3XPropertyPage@COlePropertyPage@@8 5f8b2108  
 0002:00019118       ??_R4XPropertyPage@COlePropertyPage@@6B@ 5f8b2118  
 0002:00019130       ??_R1A@?0A@A@CPropsetPropExchange@@8 5f8b2130  
 0002:00019148       ??_R2CPropsetPropExchange@@8 5f8b2148  
 0002:00019158       ??_R3CPropsetPropExchange@@8 5f8b2158  
 0002:00019168       ??_R4CPropsetPropExchange@@6B@ 5f8b2168  
 0002:00019180       ??_R1A@?0A@A@CControlRectTracker@@8 5f8b2180  
 0002:00019198       ??_R2CControlRectTracker@@8 5f8b2198  
 0002:000191a8       ??_R3CControlRectTracker@@8 5f8b21a8  
 0002:000191b8       ??_R4CControlRectTracker@@6B@ 5f8b21b8  
 0002:000191d0       ??_R1A@?0A@A@IPersistStream@@8 5f8b21d0  
 0002:000191e8       ??_R1A@?0A@A@CBlobProperty@@8 5f8b21e8  
 0002:00019200       ??_R2CBlobProperty@@8      5f8b2200  
 0002:00019218       ??_R3CBlobProperty@@8      5f8b2218  
 0002:00019228       ??_R4CBlobProperty@@6B@    5f8b2228  
 0002:00019240       ??_R1A@?0A@A@CPropbagPropExchange@@8 5f8b2240  
 0002:00019258       ??_R2CPropbagPropExchange@@8 5f8b2258  
 0002:00019268       ??_R3CPropbagPropExchange@@8 5f8b2268  
 0002:00019278       ??_R4CPropbagPropExchange@@6B@ 5f8b2278  
 0002:00019290       ??_R1A@?0A@A@_AFXCTL_AMBIENT_CACHE@@8 5f8b2290  
 0002:000192a8       ??_R2_AFXCTL_AMBIENT_CACHE@@8 5f8b22a8  
 0002:000192b8       ??_R3_AFXCTL_AMBIENT_CACHE@@8 5f8b22b8  
 0002:000192c8       ??_R4_AFXCTL_AMBIENT_CACHE@@6B@ 5f8b22c8  
 0002:000192e0       ??_R1A@?0A@A@CWindowlessDC@@8 5f8b22e0  
 0002:000192f8       ??_R2CWindowlessDC@@8      5f8b22f8  
 0002:00019308       ??_R3CWindowlessDC@@8      5f8b2308  
 0002:00019318       ??_R4CWindowlessDC@@6B@    5f8b2318  
 0002:00019330       ??_R1A@?0A@A@CColorButton@@8 5f8b2330  
 0002:00019348       ??_R2CColorButton@@8       5f8b2348  
 0002:00019360       ??_R3CColorButton@@8       5f8b2360  
 0002:00019370       ??_R4CColorButton@@6B@     5f8b2370  
 0002:00019388       ??_R1A@?0A@A@CStockPropPage@@8 5f8b2388  
 0002:000193a0       ??_R1A@?0A@A@CColorPropPage@@8 5f8b23a0  
 0002:000193b8       ??_R2CColorPropPage@@8     5f8b23b8  
 0002:000193d8       ??_R3CColorPropPage@@8     5f8b23d8  
 0002:000193e8       ??_R4CColorPropPage@@6B@   5f8b23e8  
 0002:00019400       ??_R1A@?0A@A@CFontPropPage@@8 5f8b2400  
 0002:00019418       ??_R2CFontPropPage@@8      5f8b2418  
 0002:00019438       ??_R3CFontPropPage@@8      5f8b2438  
 0002:00019448       ??_R4CFontPropPage@@6B@    5f8b2448  
 0002:00019460       ??_R1A@?0A@A@CSizeComboBox@@8 5f8b2460  
 0002:00019478       ??_R2CSizeComboBox@@8      5f8b2478  
 0002:00019490       ??_R3CSizeComboBox@@8      5f8b2490  
 0002:000194a0       ??_R4CSizeComboBox@@6B@    5f8b24a0  
 0002:000194b8       ??_R1A@?0A@A@CFontComboBox@@8 5f8b24b8  
 0002:000194d0       ??_R2CFontComboBox@@8      5f8b24d0  
 0002:000194e8       ??_R3CFontComboBox@@8      5f8b24e8  
 0002:000194f8       ??_R4CFontComboBox@@6B@    5f8b24f8  
 0002:00019510       ??_R1A@?0A@A@CPicturePropPage@@8 5f8b2510  
 0002:00019528       ??_R2CPicturePropPage@@8   5f8b2528  
 0002:00019548       ??_R3CPicturePropPage@@8   5f8b2548  
 0002:00019558       ??_R4CPicturePropPage@@6B@ 5f8b2558  
 0002:00019570       ??_R2CStockPropPage@@8     5f8b2570  
 0002:00019590       ??_R3CStockPropPage@@8     5f8b2590  
 0002:000195a0       ??_R4CStockPropPage@@6B@   5f8b25a0  
 0002:000195b8       ??_R1A@?0A@A@CDBException@@8 5f8b25b8  
 0002:000195d0       ??_R2CDBException@@8       5f8b25d0  
 0002:000195e0       ??_R3CDBException@@8       5f8b25e0  
 0002:000195f0       ??_R4CDBException@@6B@     5f8b25f0  
 0002:00019608       ??_R1A@?0A@A@CDatabase@@8  5f8b2608  
 0002:00019620       ??_R2CDatabase@@8          5f8b2620  
 0002:00019630       ??_R3CDatabase@@8          5f8b2630  
 0002:00019640       ??_R4CDatabase@@6B@        5f8b2640  
 0002:00019658       ??_R1A@?0A@A@CRecordset@@8 5f8b2658  
 0002:00019670       ??_R2CRecordset@@8         5f8b2670  
 0002:00019680       ??_R3CRecordset@@8         5f8b2680  
 0002:00019690       ??_R4CRecordset@@6B@       5f8b2690  
 0002:000196a8       ??_R1A@?0A@A@_AFX_DB_STATE@@8 5f8b26a8  
 0002:000196c0       ??_R2_AFX_DB_STATE@@8      5f8b26c0  
 0002:000196d0       ??_R3_AFX_DB_STATE@@8      5f8b26d0  
 0002:000196e0       ??_R4_AFX_DB_STATE@@6B@    5f8b26e0  
 0002:000196f8       ??_R1A@?0A@A@CRecordView@@8 5f8b26f8  
 0002:00019710       ??_R2CRecordView@@8        5f8b2710  
 0002:00019730       ??_R3CRecordView@@8        5f8b2730  
 0002:00019740       ??_R4CRecordView@@6B@      5f8b2740  
 0002:00019758       ??_R1A@?0A@A@CLongBinary@@8 5f8b2758  
 0002:00019770       ??_R2CLongBinary@@8        5f8b2770  
 0002:00019780       ??_R3CLongBinary@@8        5f8b2780  
 0002:00019790       ??_R4CLongBinary@@6B@      5f8b2790  
 0002:000197a8       ??_R1A@?0A@A@CDBVariant@@8 5f8b27a8  
 0002:000197c0       ??_R2CDBVariant@@8         5f8b27c0  
 0002:000197c8       ??_R3CDBVariant@@8         5f8b27c8  
 0002:000197d8       ??_R4CDBVariant@@6B@       5f8b27d8  
 0002:000197f0       ??_R1A@?0A@A@_AFX_DAO_STATE@@8 5f8b27f0  
 0002:00019808       ??_R2_AFX_DAO_STATE@@8     5f8b2808  
 0002:00019818       ??_R3_AFX_DAO_STATE@@8     5f8b2818  
 0002:00019828       ??_R4_AFX_DAO_STATE@@6B@   5f8b2828  
 0002:00019840       ??_R1A@?0A@A@CDaoIndexInfo@@8 5f8b2840  
 0002:00019858       ??_R2CDaoIndexInfo@@8      5f8b2858  
 0002:00019860       ??_R3CDaoIndexInfo@@8      5f8b2860  
 0002:00019870       ??_R4CDaoIndexInfo@@6B@    5f8b2870  
 0002:00019888       ??_R1A@?0A@A@CDaoRelationInfo@@8 5f8b2888  
 0002:000198a0       ??_R2CDaoRelationInfo@@8   5f8b28a0  
 0002:000198a8       ??_R3CDaoRelationInfo@@8   5f8b28a8  
 0002:000198b8       ??_R4CDaoRelationInfo@@6B@ 5f8b28b8  
 0002:000198d0       ??_R1A@?0A@A@CDaoException@@8 5f8b28d0  
 0002:000198e8       ??_R2CDaoException@@8      5f8b28e8  
 0002:000198f8       ??_R3CDaoException@@8      5f8b28f8  
 0002:00019908       ??_R4CDaoException@@6B@    5f8b2908  
 0002:00019920       ??_R1A@?0A@A@CDaoWorkspace@@8 5f8b2920  
 0002:00019938       ??_R2CDaoWorkspace@@8      5f8b2938  
 0002:00019948       ??_R3CDaoWorkspace@@8      5f8b2948  
 0002:00019958       ??_R4CDaoWorkspace@@6B@    5f8b2958  
 0002:00019970       ??_R1A@?0A@A@CDaoDatabase@@8 5f8b2970  
 0002:00019988       ??_R2CDaoDatabase@@8       5f8b2988  
 0002:00019998       ??_R3CDaoDatabase@@8       5f8b2998  
 0002:000199a8       ??_R4CDaoDatabase@@6B@     5f8b29a8  
 0002:000199c0       ??_R1A@?0A@A@CDaoTableDef@@8 5f8b29c0  
 0002:000199d8       ??_R2CDaoTableDef@@8       5f8b29d8  
 0002:000199e8       ??_R3CDaoTableDef@@8       5f8b29e8  
 0002:000199f8       ??_R4CDaoTableDef@@6B@     5f8b29f8  
 0002:00019a10       ??_R1A@?0A@A@CDaoQueryDef@@8 5f8b2a10  
 0002:00019a28       ??_R2CDaoQueryDef@@8       5f8b2a28  
 0002:00019a38       ??_R3CDaoQueryDef@@8       5f8b2a38  
 0002:00019a48       ??_R4CDaoQueryDef@@6B@     5f8b2a48  
 0002:00019a60       ??_R1A@?0A@A@CDaoRecordset@@8 5f8b2a60  
 0002:00019a78       ??_R2CDaoRecordset@@8      5f8b2a78  
 0002:00019a88       ??_R3CDaoRecordset@@8      5f8b2a88  
 0002:00019a98       ??_R4CDaoRecordset@@6B@    5f8b2a98  
 0002:00019ab0       ??_R1A@?0A@A@CDaoRecordView@@8 5f8b2ab0  
 0002:00019ac8       ??_R2CDaoRecordView@@8     5f8b2ac8  
 0002:00019ae8       ??_R3CDaoRecordView@@8     5f8b2ae8  
 0002:00019af8       ??_R4CDaoRecordView@@6B@   5f8b2af8  
 0002:00019b10       ??_R1A@?0A@A@CPalette@@8   5f8b2b10  
 0002:00019b28       ??_R2CPalette@@8           5f8b2b28  
 0002:00019b38       ??_R3CPalette@@8           5f8b2b38  
 0002:00019b48       ??_R4CPalette@@6B@         5f8b2b48  
 0002:00019b60       ??_R1A@?0A@A@CCheckListBox@@8 5f8b2b60  
 0002:00019b78       ??_R2CCheckListBox@@8      5f8b2b78  
 0002:00019b90       ??_R3CCheckListBox@@8      5f8b2b90  
 0002:00019ba0       ??_R4CCheckListBox@@6B@    5f8b2ba0  
 0002:00019bb8       ??_R1A@?0A@A@CBitmapButton@@8 5f8b2bb8  
 0002:00019bd0       ??_R2CBitmapButton@@8      5f8b2bd0  
 0002:00019be8       ??_R3CBitmapButton@@8      5f8b2be8  
 0002:00019bf8       ??_R4CBitmapButton@@6B@    5f8b2bf8  
 0002:00019c10       ??_R1A@?0A@A@CDataPathProperty@@8 5f8b2c10  
 0002:00019c28       ??_R2CDataPathProperty@@8  5f8b2c28  
 0002:00019c48       ??_R3CDataPathProperty@@8  5f8b2c48  
 0002:00019c58       ??_R4CDataPathProperty@@6B@ 5f8b2c58  
 0002:00019c70       ??_R1A@?0A@A@CCachedDataPathProperty@@8 5f8b2c70  
 0002:00019c88       ??_R2CCachedDataPathProperty@@8 5f8b2c88  
 0002:00019ca8       ??_R3CCachedDataPathProperty@@8 5f8b2ca8  
 0002:00019cb8       ??_R4CCachedDataPathProperty@@6B@ 5f8b2cb8  
 0002:00019d28       __CT??_R0PAX@84            5f8b2d28  
 0002:00019d48       __CT??_R0PAVCObject@@@84   5f8b2d48  
 0002:00019d68       __CT??_R0PAVCException@@@84 5f8b2d68  
 0002:00019d88       __CT??_R0PAVCSimpleException@@@84 5f8b2d88  
 0002:00019da8       __CT??_R0PAVCMemoryException@@@84 5f8b2da8  
 0002:00019dc8       __CTA5PAVCMemoryException@@ 5f8b2dc8  
 0002:00019de0       __TI5PAVCMemoryException@@ 5f8b2de0  
 0002:00019df0       __CT??_R0PAVCNotSupportedException@@@84 5f8b2df0  
 0002:00019e10       __CTA5PAVCNotSupportedException@@ 5f8b2e10  
 0002:00019e28       __TI5PAVCNotSupportedException@@ 5f8b2e28  
 0002:00019f90       __CT??_R0PAVCArchiveException@@@84 5f8b2f90  
 0002:00019fb0       __CTA4PAVCArchiveException@@ 5f8b2fb0  
 0002:00019fc8       __TI4PAVCArchiveException@@ 5f8b2fc8  
 0002:0001a3a8       __CT??_R0PAVCFileException@@@84 5f8b33a8  
 0002:0001a3c8       __CTA4PAVCFileException@@  5f8b33c8  
 0002:0001a3e0       __TI4PAVCFileException@@   5f8b33e0  
 0002:0001ce28       __CT??_R0PAVCResourceException@@@84 5f8b5e28  
 0002:0001ce48       __CTA5PAVCResourceException@@ 5f8b5e48  
 0002:0001ce60       __TI5PAVCResourceException@@ 5f8b5e60  
 0002:0001ce70       __CT??_R0PAVCUserException@@@84 5f8b5e70  
 0002:0001ce90       __CTA5PAVCUserException@@  5f8b5e90  
 0002:0001cea8       __TI5PAVCUserException@@   5f8b5ea8  
 0002:0001ecc8       __CT??_R0PAVCInternetException@@@84 5f8b7cc8  
 0002:0001ece8       __CTA4PAVCInternetException@@ 5f8b7ce8  
 0002:0001ed00       __TI4PAVCInternetException@@ 5f8b7d00  
 0002:0001fec0       __CT??_R0PAVCOleDispatchException@@@84 5f8b8ec0  
 0002:0001fee0       __CTA4PAVCOleDispatchException@@ 5f8b8ee0  
 0002:0001fef8       __TI4PAVCOleDispatchException@@ 5f8b8ef8  
 0002:00021508       __CT??_R0PAVCOleException@@@84 5f8ba508  
 0002:00021528       __CTA4PAVCOleException@@   5f8ba528  
 0002:00021540       __TI4PAVCOleException@@    5f8ba540  
 0002:00022df0       __CTA3PAVCException@@      5f8bbdf0  
 0002:00022e00       __TI3PAVCException@@       5f8bbe00  
 0002:000281f0       __CT??_R0PAVCDBException@@@84 5f8c11f0  
 0002:00028210       __CTA4PAVCDBException@@    5f8c1210  
 0002:00028228       __TI4PAVCDBException@@     5f8c1228  
 0002:00028ea0       __CT??_R0PAVCDaoException@@@84 5f8c1ea0  
 0002:00028ec0       __CTA4PAVCDaoException@@   5f8c1ec0  
 0002:00028ed8       __TI4PAVCDaoException@@    5f8c1ed8  
 0003:00000000       ?_afxThreadState@@3V?$CThreadLocal@V_AFX_THREAD_STATE@@@@A 5f8cf000  
 0003:00000004       ?_afxThreadData@@3PAVCThreadSlotData@@A 5f8cf004  
 0003:00000008       ?_afxBaseModuleState@@3V?$CProcessLocal@V_AFX_BASE_MODULE_STATE@@@@A 5f8cf008  
 0003:0000000c       ?__afxThreadData@@3PAEA    5f8cf00c  
 0003:00000040       ?_afxLockInitLock@@3U_RTL_CRITICAL_SECTION@@A 5f8cf040  
 0003:00000058       ?_afxCriticalWin32s@@3HA   5f8cf058  
 0003:0000005c       ?_afxCriticalInit@@3HA     5f8cf05c  
 0003:00000060       ?_afxLockInit@@3PAHA       5f8cf060  
 0003:000000a8       ?_afxResourceLock@@3PAU_RTL_CRITICAL_SECTION@@A 5f8cf0a8  
 0003:00000240       ??_R0?AVtype_info@@@8      5f8cf240  
 0003:00000258       ?_afxAlloc64@@3VCFixedAlloc@@A 5f8cf258  
 0003:00000280       ?_afxAlloc128@@3VCFixedAlloc@@A 5f8cf280  
 0003:000002a8       ?_afxAlloc256@@3VCFixedAlloc@@A 5f8cf2a8  
 0003:000002d0       ?_afxAlloc512@@3VCFixedAlloc@@A 5f8cf2d0  
 0003:000002f8       ??_R0?AVCObject@@@8        5f8cf2f8  
 0003:00000310       ?m_nMsgDragList@CWnd@@1IB  5f8cf310  
 0003:00000318       ??_R0?AVCCmdTarget@@@8     5f8cf318  
 0003:00000338       ??_R0?AVCWnd@@@8           5f8cf338  
 0003:0000034c       ?_afxPchNil@@3PBGB         5f8cf34c  
 0003:00000350       ?_afxInitData@@3PAHA       5f8cf350  
 0003:00000360       ?_afxDataNil@@3PAUCStringData@@A 5f8cf360  
 0003:00000368       ??_R0?AVCCmdUI@@@8         5f8cf368  
 0003:00000380       ?_afxMsgCache@@3PAUAFX_MSG_CACHE@@A 5f8cf380  
 0003:00001b80       ?wndTop@CWnd@@2V1@B        5f8d0b80  
 0003:00001bc0       ?wndBottom@CWnd@@2V1@B     5f8d0bc0  
 0003:00001c00       ?wndTopMost@CWnd@@2V1@B    5f8d0c00  
 0003:00001c40       ?wndNoTopMost@CWnd@@2V1@B  5f8d0c40  
 0003:00001c80       ?_afxTickCount@@3KA        5f8d0c80  
 0003:00001c84       ?_afxTickInit@@3HA         5f8d0c84  
 0003:00001c88       ??_R0?AVCStatusCmdUI@@@8   5f8d0c88  
 0003:00001ca8       ??_R0?AVCToolCmdUI@@@8     5f8d0ca8  
 0003:00001cc8       ?s_alloc@CTempWnd@@1VCFixedAlloc@@A 5f8d0cc8  
 0003:00001cf0       ?s_alloc@CTempMenu@@1VCFixedAlloc@@A 5f8d0cf0  
 0003:00001d18       ?afxData@@3UAUX_DATA@@A    5f8d0d18  
 0003:00001d88       ??_R0?AVCTempWnd@@@8       5f8d0d88  
 0003:00001da0       ??_R0?AVCMenu@@@8          5f8d0da0  
 0003:00001db8       ??_R0?AVCTempMenu@@@8      5f8d0db8  
 0003:00001dd0       ?s_alloc@CTempGdiObject@@1VCFixedAlloc@@A 5f8d0dd0  
 0003:00001df8       ?_afxWinState@@3V?$CProcessLocal@V_AFX_WIN_STATE@@@@A 5f8d0df8  
 0003:00001e00       ??_R0?AVCDC@@@8            5f8d0e00  
 0003:00001e18       ?s_alloc@CTempDC@@1VCFixedAlloc@@A 5f8d0e18  
 0003:00001e40       ?_afxTlsRef@@3JA           5f8d0e40  
 0003:00001e48       ?s_alloc@CTempImageList@@1VCFixedAlloc@@A 5f8d0e48  
 0003:00001e70       ?_afxMsgMouseWheel@@3IA    5f8d0e70  
 0003:00001e78       __imp__OleCreatePropertyFrame@44 5f8d0e78  
 0003:00001e7c       __imp__OleTranslateColor@12 5f8d0e7c  
 0003:00001e80       __imp__OleLoadPicture@20   5f8d0e80  
 0003:00001e84       __imp__OleCreatePictureIndirect@16 5f8d0e84  
 0003:00001e88       __imp__OleCreateFontIndirect@12 5f8d0e88  
 0003:00001e90       __imp__RegDeleteValueW@8   5f8d0e90  
 0003:00001e94       __imp__RegCreateKeyExW@36  5f8d0e94  
 0003:00001e98       __imp__RegOpenKeyExW@20    5f8d0e98  
 0003:00001e9c       __imp__RegQueryValueW@16   5f8d0e9c  
 0003:00001ea0       __imp__RegSetValueW@20     5f8d0ea0  
 0003:00001ea4       __imp__RegQueryValueExW@24 5f8d0ea4  
 0003:00001ea8       __imp__RegCreateKeyW@12    5f8d0ea8  
 0003:00001eac       __imp__RegCloseKey@4       5f8d0eac  
 0003:00001eb0       __imp__RegOpenKeyW@12      5f8d0eb0  
 0003:00001eb4       __imp__SetFileSecurityW@12 5f8d0eb4  
 0003:00001eb8       __imp__GetFileSecurityW@20 5f8d0eb8  
 0003:00001ebc       __imp__RegDeleteKeyW@8     5f8d0ebc  
 0003:00001ec0       __imp__RegEnumKeyW@16      5f8d0ec0  
 0003:00001ec4       __imp__RegSetValueExW@24   5f8d0ec4  
 0003:00001ecc       __imp__StgOpenStorage@24   5f8d0ecc  
 0003:00001ed0       __imp__StgIsStorageFile@4  5f8d0ed0  
 0003:00001ed4       __imp__CoInitialize@4      5f8d0ed4  
 0003:00001ed8       __imp__StgCreateDocfile@16 5f8d0ed8  
 0003:00001edc       __imp__SetConvertStg@8     5f8d0edc  
 0003:00001ee0       __imp__RegisterDragDrop@8  5f8d0ee0  
 0003:00001ee4       __imp__CoLockObjectExternal@12 5f8d0ee4  
 0003:00001ee8       __imp__RevokeDragDrop@4    5f8d0ee8  
 0003:00001eec       __imp__CoRegisterMessageFilter@8 5f8d0eec  
 0003:00001ef0       __imp__OleRegGetMiscStatus@12 5f8d0ef0  
 0003:00001ef4       __imp__CoRegisterClassObject@20 5f8d0ef4  
 0003:00001ef8       __imp__CoRevokeClassObject@4 5f8d0ef8  
 0003:00001efc       __imp__OleTranslateAccelerator@12 5f8d0efc  
 0003:00001f00       __imp__IsAccelerator@16    5f8d0f00  
 0003:00001f04       __imp__OleCreateMenuDescriptor@8 5f8d0f04  
 0003:00001f08       __imp__OleDestroyMenuDescriptor@4 5f8d0f08  
 0003:00001f0c       __imp__GetRunningObjectTable@8 5f8d0f0c  
 0003:00001f10       __imp__WriteClassStg@8     5f8d0f10  
 0003:00001f14       __imp__OleDuplicateData@12 5f8d0f14  
 0003:00001f18       __imp__ReadClassStg@8      5f8d0f18  
 0003:00001f1c       __imp__WriteFmtUserTypeStg@12 5f8d0f1c  
 0003:00001f20       __imp__CoTreatAsClass@8    5f8d0f20  
 0003:00001f24       __imp__ReadFmtUserTypeStg@12 5f8d0f24  
 0003:00001f28       __imp__OleRegGetUserType@12 5f8d0f28  
 0003:00001f2c       __imp__GetClassFile@8      5f8d0f2c  
 0003:00001f30       __imp__CreateDataAdviseHolder@4 5f8d0f30  
 0003:00001f34       __imp__CreateFileMoniker@8 5f8d0f34  
 0003:00001f38       __imp__CreateBindCtx@8     5f8d0f38  
 0003:00001f3c       __imp__CoCreateInstance@20 5f8d0f3c  
 0003:00001f40       __imp__CLSIDFromString@8   5f8d0f40  
 0003:00001f44       __imp__CLSIDFromProgID@8   5f8d0f44  
 0003:00001f48       __imp__OleIsCurrentClipboard@4 5f8d0f48  
 0003:00001f4c       __imp__OleFlushClipboard@0 5f8d0f4c  
 0003:00001f50       __imp__CoGetClassObject@20 5f8d0f50  
 0003:00001f54       __imp__OleSetClipboard@4   5f8d0f54  
 0003:00001f58       __imp__OleGetClipboard@4   5f8d0f58  
 0003:00001f5c       __imp__CoGetMalloc@8       5f8d0f5c  
 0003:00001f60       __imp__CreateDataCache@16  5f8d0f60  
 0003:00001f64       __imp__ReadClassStm@8      5f8d0f64  
 0003:00001f68       __imp__OleLoadFromStream@12 5f8d0f68  
 0003:00001f6c       __imp__DoDragDrop@16       5f8d0f6c  
 0003:00001f70       __imp__StringFromGUID2@12  5f8d0f70  
 0003:00001f74       __imp__CoUninitialize@0    5f8d0f74  
 0003:00001f78       __imp__CoDisconnectObject@8 5f8d0f78  
 0003:00001f7c       __imp__OleRegEnumVerbs@8   5f8d0f7c  
 0003:00001f80       __imp__CreateOleAdviseHolder@4 5f8d0f80  
 0003:00001f84       __imp__CreateStreamOnHGlobal@12 5f8d0f84  
 0003:00001f88       __imp__OleSaveToStream@8   5f8d0f88  
 0003:00001f8c       __imp__CreateGenericComposite@12 5f8d0f8c  
 0003:00001f90       __imp__CreateItemMoniker@12 5f8d0f90  
 0003:00001f94       __imp__CoTaskMemFree@4     5f8d0f94  
 0003:00001f98       __imp__StringFromCLSID@8   5f8d0f98  
 0003:00001f9c       __imp__OleSetContainedObject@8 5f8d0f9c  
 0003:00001fa0       __imp__OleCreateFromData@28 5f8d0fa0  
 0003:00001fa4       __imp__OleCreateLinkFromData@28 5f8d0fa4  
 0003:00001fa8       __imp__OleCreateStaticFromData@28 5f8d0fa8  
 0003:00001fac       __imp__OleCreateFromFile@32 5f8d0fac  
 0003:00001fb0       __imp__OleInitialize@4     5f8d0fb0  
 0003:00001fb4       __imp__OleUninitialize@0   5f8d0fb4  
 0003:00001fb8       __imp__CoFreeUnusedLibraries@0 5f8d0fb8  
 0003:00001fbc       __imp__OleLockRunning@12   5f8d0fbc  
 0003:00001fc0       __imp__CoTaskMemAlloc@4    5f8d0fc0  
 0003:00001fc4       __imp__OleIsRunning@4      5f8d0fc4  
 0003:00001fc8       __imp__OleRun@4            5f8d0fc8  
 0003:00001fcc       __imp__OleQueryLinkFromData@4 5f8d0fcc  
 0003:00001fd0       __imp__OleQueryCreateFromData@4 5f8d0fd0  
 0003:00001fd4       __imp__OleSetMenuDescriptor@20 5f8d0fd4  
 0003:00001fd8       __imp__OleCreate@28        5f8d0fd8  
 0003:00001fdc       __imp__OleCreateLinkToFile@28 5f8d0fdc  
 0003:00001fe0       __imp__GetHGlobalFromILockBytes@8 5f8d0fe0  
 0003:00001fe4       __imp__StgOpenStorageOnILockBytes@24 5f8d0fe4  
 0003:00001fe8       __imp__WriteClassStm@8     5f8d0fe8  
 0003:00001fec       __imp__OleGetIconOfClass@12 5f8d0fec  
 0003:00001ff0       __imp__ReleaseStgMedium@4  5f8d0ff0  
 0003:00001ff4       __imp__OleSave@12          5f8d0ff4  
 0003:00001ff8       __imp__CreateILockBytesOnHGlobal@12 5f8d0ff8  
 0003:00001ffc       __imp__StgCreateDocfileOnILockBytes@16 5f8d0ffc  
 0003:00002000       __imp__OleLoad@16          5f8d1000  
 0003:00002008       __imp__VariantChangeType@16 5f8d1008  
 0003:0000200c       __imp__SysAllocStringLen@8 5f8d100c  
 0003:00002010       __imp__SysReAllocStringLen@12 5f8d1010  
 0003:00002014       __imp__VarDateFromStr@16   5f8d1014  
 0003:00002018       __imp__LoadRegTypeLib@20   5f8d1018  
 0003:0000201c       __imp__RegisterTypeLib@12  5f8d101c  
 0003:00002020       __imp__VariantTimeToSystemTime@12 5f8d1020  
 0003:00002024       __imp__LoadTypeLib@8       5f8d1024  
 0003:00002028       __imp__SafeArrayCreateVector@12 5f8d1028  
 0003:0000202c       __imp__SafeArrayDestroyDescriptor@4 5f8d102c  
 0003:00002030       __imp__SafeArrayDestroyData@4 5f8d1030  
 0003:00002034       __imp__SafeArrayDestroy@4  5f8d1034  
 0003:00002038       __imp__SafeArrayUnlock@4   5f8d1038  
 0003:0000203c       __imp__SafeArrayLock@4     5f8d103c  
 0003:00002040       __imp__SafeArrayPutElement@12 5f8d1040  
 0003:00002044       __imp__SafeArrayPtrOfIndex@12 5f8d1044  
 0003:00002048       __imp__SafeArrayGetElement@12 5f8d1048  
 0003:0000204c       __imp__SafeArrayAllocDescriptor@8 5f8d104c  
 0003:00002050       __imp__SafeArrayAllocData@4 5f8d1050  
 0003:00002054       __imp__SafeArrayCopy@8     5f8d1054  
 0003:00002058       __imp__VarBstrFromDate@20  5f8d1058  
 0003:0000205c       __imp__SafeArrayGetLBound@12 5f8d105c  
 0003:00002060       __imp__VarBstrFromCy@20    5f8d1060  
 0003:00002064       __imp__VarCyFromStr@16     5f8d1064  
 0003:00002068       __imp__SysAllocStringByteLen@8 5f8d1068  
 0003:0000206c       __imp__SysStringByteLen@4  5f8d106c  
 0003:00002070       __imp__SafeArrayRedim@8    5f8d1070  
 0003:00002074       __imp__SafeArrayCreate@12  5f8d1074  
 0003:00002078       __imp__SafeArrayGetDim@4   5f8d1078  
 0003:0000207c       __imp__SafeArrayGetElemsize@4 5f8d107c  
 0003:00002080       __imp__SysFreeString@4     5f8d1080  
 0003:00002084       __imp__SafeArrayGetUBound@12 5f8d1084  
 0003:00002088       __imp__SafeArrayAccessData@8 5f8d1088  
 0003:0000208c       __imp__SafeArrayUnaccessData@4 5f8d108c  
 0003:00002090       __imp__SysAllocString@4    5f8d1090  
 0003:00002094       __imp__SysStringLen@4      5f8d1094  
 0003:00002098       __imp__VariantCopy@8       5f8d1098  
 0003:0000209c       __imp__VariantClear@4      5f8d109c  
 0003:000020a4       __imp__ImageList_Destroy@4 5f8d10a4  
 0003:000020a8       __imp__CreatePropertySheetPageW@4 5f8d10a8  
 0003:000020ac       __imp__ImageList_LoadImageW@28 5f8d10ac  
 0003:000020b0       __imp__ImageList_Create@20 5f8d10b0  
 0003:000020b4       __imp__MakeDragList@4      5f8d10b4  
 0003:000020b8       __imp__InitCommonControlsEx@4 5f8d10b8  
 0003:000020bc       __imp__LBItemFromPt@16     5f8d10bc  
 0003:000020c0       __imp__InitCommonControls@0 5f8d10c0  
 0003:000020c4       __imp__ImageList_Merge@24  5f8d10c4  
 0003:000020c8       __imp__ImageList_Read@4    5f8d10c8  
 0003:000020cc       __imp__ImageList_Write@8   5f8d10cc  
 0003:000020d0       __imp__PropertySheetW@4    5f8d10d0  
 0003:000020d4       __imp__DestroyPropertySheetPage@4 5f8d10d4  
 0003:000020d8       __imp__ImageList_Duplicate@4 5f8d10d8  
 0003:000020dc       __imp__ImageList_DrawIndirect@4 5f8d10dc  
 0003:000020e4       __imp__DragFinish@4        5f8d10e4  
 0003:000020e8       __imp__DragAcceptFiles@8   5f8d10e8  
 0003:000020ec       __imp__SHGetFileInfoW@20   5f8d10ec  
 0003:000020f0       __imp__DragQueryFileW@16   5f8d10f0  
 0003:000020f4       __imp__ExtractIconW@12     5f8d10f4  
 0003:000020fc       __imp__CommDlgExtendedError@0 5f8d10fc  
 0003:00002100       __imp__FindTextW@4         5f8d1100  
 0003:00002104       __imp__ReplaceTextW@4      5f8d1104  
 0003:00002108       __imp__ChooseFontW@4       5f8d1108  
 0003:0000210c       __imp__ChooseColorW@4      5f8d110c  
 0003:00002110       __imp__PrintDlgW@4         5f8d1110  
 0003:00002114       __imp__PageSetupDlgW@4     5f8d1114  
 0003:00002118       __imp__GetOpenFileNameW@4  5f8d1118  
 0003:0000211c       __imp__GetSaveFileNameW@4  5f8d111c  
 0003:00002120       __imp__GetFileTitleW@12    5f8d1120  
 0003:00002128       __imp__OpenPrinterW@12     5f8d1128  
 0003:0000212c       __imp__DocumentPropertiesW@24 5f8d112c  
 0003:00002130       __imp__ClosePrinter@4      5f8d1130  
 0003:00002138       __imp__FtpGetCurrentDirectoryW@12 5f8d1138  
 0003:0000213c       __imp__GopherGetAttributeW@32 5f8d113c  
 0003:00002140       __imp__InternetCanonicalizeUrlW@16 5f8d1140  
 0003:00002144       __imp__FtpCreateDirectoryW@8 5f8d1144  
 0003:00002148       __imp__InternetGetLastResponseInfoW@12 5f8d1148  
 0003:0000214c       __imp__GopherFindFirstFileW@24 5f8d114c  
 0003:00002150       __imp__InternetFindNextFileW@8 5f8d1150  
 0003:00002154       __imp__FtpFindFirstFileW@20 5f8d1154  
 0003:00002158       __imp__HttpQueryInfoW@20   5f8d1158  
 0003:0000215c       __imp__HttpSendRequestExW@20 5f8d115c  
 0003:00002160       __imp__HttpEndRequestW@16  5f8d1160  
 0003:00002164       __imp__HttpSendRequestW@20 5f8d1164  
 0003:00002168       __imp__HttpAddRequestHeadersW@16 5f8d1168  
 0003:0000216c       __imp__InternetErrorDlg@20 5f8d116c  
 0003:00002170       __imp__HttpOpenRequestW@32 5f8d1170  
 0003:00002174       __imp__GopherOpenFileW@20  5f8d1174  
 0003:00002178       __imp__GopherCreateLocatorW@28 5f8d1178  
 0003:0000217c       __imp__FtpGetFileW@28      5f8d117c  
 0003:00002180       __imp__FtpPutFileW@20      5f8d1180  
 0003:00002184       __imp__FtpOpenFileW@20     5f8d1184  
 0003:00002188       __imp__FtpSetCurrentDirectoryW@8 5f8d1188  
 0003:0000218c       __imp__FtpRemoveDirectoryW@8 5f8d118c  
 0003:00002190       __imp__InternetSetStatusCallback@8 5f8d1190  
 0003:00002194       __imp__FtpRenameFileW@12   5f8d1194  
 0003:00002198       __imp__FtpDeleteFileW@8    5f8d1198  
 0003:0000219c       __imp__InternetConnectW@32 5f8d119c  
 0003:000021a0       __imp__InternetQueryDataAvailable@16 5f8d11a0  
 0003:000021a4       __imp__InternetReadFile@16 5f8d11a4  
 0003:000021a8       __imp__InternetWriteFile@16 5f8d11a8  
 0003:000021ac       __imp__InternetSetFilePointer@20 5f8d11ac  
 0003:000021b0       __imp__InternetGetCookieW@16 5f8d11b0  
 0003:000021b4       __imp__InternetSetCookieW@12 5f8d11b4  
 0003:000021b8       __imp__InternetQueryOptionW@16 5f8d11b8  
 0003:000021bc       __imp__InternetSetOptionExW@20 5f8d11bc  
 0003:000021c0       __imp__InternetOpenUrlW@24 5f8d11c0  
 0003:000021c4       __imp__InternetCloseHandle@4 5f8d11c4  
 0003:000021c8       __imp__InternetOpenW@20    5f8d11c8  
 0003:000021cc       __imp__InternetCrackUrlW@16 5f8d11cc  
 0003:000021d4       __imp__connect@12          5f8d11d4  
 0003:000021d8       __imp__ioctlsocket@12      5f8d11d8  
 0003:000021dc       __imp__WSAAsyncSelect@16   5f8d11dc  
 0003:000021e0       __imp__socket@12           5f8d11e0  
 0003:000021e4       __imp__htonl@4             5f8d11e4  
 0003:000021e8       __imp__recvfrom@24         5f8d11e8  
 0003:000021ec       __imp__WSACleanup@0        5f8d11ec  
 0003:000021f0       __imp__WSAStartup@8        5f8d11f0  
 0003:000021f4       __imp__WSASetLastError@4   5f8d11f4  
 0003:000021f8       __imp__WSAGetLastError@0   5f8d11f8  
 0003:000021fc       __imp__inet_ntoa@4         5f8d11fc  
 0003:00002200       __imp__ntohs@4             5f8d1200  
 0003:00002204       __imp__getpeername@12      5f8d1204  
 0003:00002208       __imp__send@16             5f8d1208  
 0003:0000220c       __imp__recv@16             5f8d120c  
 0003:00002210       __imp__gethostbyname@4     5f8d1210  
 0003:00002214       __imp__closesocket@4       5f8d1214  
 0003:00002218       __imp__getsockname@12      5f8d1218  
 0003:0000221c       __imp__sendto@24           5f8d121c  
 0003:00002220       __imp__htons@4             5f8d1220  
 0003:00002224       __imp__bind@12             5f8d1224  
 0003:00002228       __imp__inet_addr@4         5f8d1228  
 0003:0000222c       __imp__accept@12           5f8d122c  
 0003:00002234       __imp__OleUIConvertW@4     5f8d1234  
 0003:00002238       __imp__OleUIInsertObjectW@4 5f8d1238  
 0003:0000223c       __imp__OleUIAddVerbMenuW@36 5f8d123c  
 0003:00002240       __imp__OleUIChangeSourceW@4 5f8d1240  
 0003:00002244       __imp__OleUIObjectPropertiesW@4 5f8d1244  
 0003:00002248       __imp__OleUIBusyW@4        5f8d1248  
 0003:0000224c       __imp__OleUIPasteSpecialW@4 5f8d124c  
 0003:00002250       __imp__OleUIUpdateLinksW@16 5f8d1250  
 0003:00002254       __imp__OleUIEditLinksW@4   5f8d1254  
 0003:00002258       __imp__OleUIChangeIconW@4  5f8d1258  
 0003:00002260       __imp__RegisterBindStatusCallback@16 5f8d1260  
 0003:00002264       __imp__CreateAsyncBindCtx@16 5f8d1264  
 0003:00002268       __imp__CreateURLMoniker@12 5f8d1268  
 0003:0000226c       __imp__IsAsyncMoniker@4    5f8d126c  
 0003:00002274       __imp__SQLPrepare@12       5f8d1274  
 0003:00002278       __imp__SQLExecute@4        5f8d1278  
 0003:0000227c       __imp__SQLSetPos@16        5f8d127c  
 0003:00002280       __imp__SQLGetFunctions@12  5f8d1280  
 0003:00002284       __imp__SQLGetStmtOption@12 5f8d1284  
 0003:00002288       __imp__SQLAllocEnv@4       5f8d1288  
 0003:0000228c       __imp__SQLAllocConnect@8   5f8d128c  
 0003:00002290       __imp__SQLTransact@12      5f8d1290  
 0003:00002294       __imp__SQLSetConnectOption@12 5f8d1294  
 0003:00002298       __imp__SQLGetData@24       5f8d1298  
 0003:0000229c       __imp__SQLDriverConnect@32 5f8d129c  
 0003:000022a0       __imp__SQLDescribeCol@36   5f8d12a0  
 0003:000022a4       __imp__SQLDisconnect@4     5f8d12a4  
 0003:000022a8       __imp__SQLFreeConnect@4    5f8d12a8  
 0003:000022ac       __imp__SQLAllocStmt@8      5f8d12ac  
 0003:000022b0       __imp__SQLExecDirect@12    5f8d12b0  
 0003:000022b4       __imp__SQLNumResultCols@8  5f8d12b4  
 0003:000022b8       __imp__SQLFetch@4          5f8d12b8  
 0003:000022bc       __imp__SQLMoreResults@4    5f8d12bc  
 0003:000022c0       __imp__SQLFreeStmt@8       5f8d12c0  
 0003:000022c4       __imp__SQLCancel@4         5f8d12c4  
 0003:000022c8       __imp__SQLError@32         5f8d12c8  
 0003:000022cc       __imp__SQLExtendedFetch@20 5f8d12cc  
 0003:000022d0       __imp__SQLGetCursorName@16 5f8d12d0  
 0003:000022d4       __imp__SQLRowCount@8       5f8d12d4  
 0003:000022d8       __imp__SQLPutData@12       5f8d12d8  
 0003:000022dc       __imp__SQLParamData@8      5f8d12dc  
 0003:000022e0       __imp__SQLBindCol@24       5f8d12e0  
 0003:000022e4       __imp__SQLBindParameter@40 5f8d12e4  
 0003:000022e8       __imp__SQLGetInfo@20       5f8d12e8  
 0003:000022ec       __imp__SQLSetStmtOption@12 5f8d12ec  
 0003:000022f0       __imp__SQLFreeEnv@4        5f8d12f0  
 0003:000022f8       ??_R0?AVCTestCmdUI@@@8     5f8d12f8  
 0003:00002314       ?_afxIsMailAvail@@3HA      5f8d1314  
 0003:00002318       ??_R0?AVCGdiObject@@@8     5f8d1318  
 0003:00002338       ??_R0?AVCDialog@@@8        5f8d1338  
 0003:00002350       ??_R0?AVCMapStringToPtr@@@8 5f8d1350  
 0003:00002370       ??_R0?AVCTempGdiObject@@@8 5f8d1370  
 0003:00002390       _g_pfnGetSystemMetrics     5f8d1390  
 0003:00002394       _g_pfnMonitorFromWindow    5f8d1394  
 0003:00002398       _g_pfnMonitorFromRect      5f8d1398  
 0003:0000239c       _g_pfnMonitorFromPoint     5f8d139c  
 0003:000023a0       _g_pfnGetMonitorInfo       5f8d13a0  
 0003:000023a4       _g_pfnEnumDisplayMonitors  5f8d13a4  
 0003:000023a8       _g_fMultiMonInitDone       5f8d13a8  
 0003:000023b0       ??_R0?AVCTempDC@@@8        5f8d13b0  
 0003:000023c8       ??_R0?AVCCommonDialog@@@8  5f8d13c8  
 0003:000023e8       ??_R0?AVCPrintDialog@@@8   5f8d13e8  
 0003:00002408       ??_R0?AVCPrintingDialog@@@8 5f8d1408  
 0003:00002428       ?_afxComCtlVersion@@3HA    5f8d1428  
 0003:00002430       ??_R0?AVCPaintDC@@@8       5f8d1430  
 0003:00002448       __hmod__COMDLG32           5f8d1448  
 0003:00002450       ??_R0?AVCFileException@@@8 5f8d1450  
 0003:00002470       ??_R0?AVCButton@@@8        5f8d1470  
 0003:00002488       ??_R0?AVCNoTrackObject@@@8 5f8d1488  
 0003:000024a8       ??_R0?AV_AFX_THREAD_STATE@@@8 5f8d14a8  
 0003:000024c8       ??_R0?AVCMapPtrToPtr@@@8   5f8d14c8  
 0003:000024e8       ??_R0?AVAFX_MODULE_THREAD_STATE@@@8 5f8d14e8  
 0003:00002510       ??_R0?AVCPtrList@@@8       5f8d1510  
 0003:00002528       ??_R0?AVAFX_MODULE_STATE@@@8 5f8d1528  
 0003:00002548       __pRawDllMain              5f8d1548  
 0003:00002550       ??_R0?AUCThreadData@@@8    5f8d1550  
 0003:0000256c       ___xc_a                    5f8d156c  
 0003:0000266c       ___xc_z                    5f8d166c  
 0003:00002670       __adjust_fdiv              5f8d1670  
 0003:00002674       ___onexitend               5f8d1674  
 0003:00002678       ___onexitbegin             5f8d1678  
 0003:00002680       ??_R0?AVCException@@@8     5f8d1680  
 0003:000026a0       ??_R0?AVCWinThread@@@8     5f8d16a0  
 0003:000026ba       ?afxChNil@@3GA             5f8d16ba  
 0003:000026d4       ?_afxCtl3dThread@@3V?$CThreadLocal@V_AFX_CTL3D_THREAD@@@@A 5f8d16d4  
 0003:000026d8       ?_afxCtl3dState@@3V?$CProcessLocal@V_AFX_CTL3D_STATE@@@@A 5f8d16d8  
 0003:000026e0       ??_R0?AV_AFX_CTL3D_THREAD@@@8 5f8d16e0  
 0003:00002700       __hmod__OLE32              5f8d1700  
 0003:00002704       ___pfnDliNotifyHook        5f8d1704  
 0003:00002708       ??_R0?AVCFile@@@8          5f8d1708  
 0003:0000271c       ?_afxOleState@@3V?$CProcessLocal@V_AFX_OLE_STATE@@@@A 5f8d171c  
 0003:00002720       ??_R0?AV_AFX_OLE_STATE@@@8 5f8d1720  
 0003:00002758       ?_afxAmbientCache@@3V?$CThreadLocal@V_AFXCTL_AMBIENT_CACHE@@@@A 5f8d1758  
 0003:0000275c       ?_afxOccManager@@3V?$CProcessLocal@VCOccManager@@@@A 5f8d175c  
 0003:00002760       ?_afxUnicodeFont@@3PAUHFONT__@@A 5f8d1760  
 0003:00002764       ?_afxHalftoneBrush@@3PAUHBRUSH__@@A 5f8d1764  
 0003:00002768       ?_afxPropPageFontInfo@@3V?$CProcessLocal@U_AFX_PROPPAGEFONTINFO@@@@A 5f8d1768  
 0003:0000276c       ?_afxBlackDottedPen@@3PAUHPEN__@@A 5f8d176c  
 0003:00002770       ?_afxHatchBrush@@3PAUHBRUSH__@@A 5f8d1770  
 0003:00002774       ?_afx_hfontMiniSys@@3PAUHFONT__@@A 5f8d1774  
 0003:00002778       ?_afx_hbmMiniSys@@3PAUHBITMAP__@@A 5f8d1778  
 0003:00002788       ?_afxDbState@@3V?$CProcessLocal@V_AFX_DB_STATE@@@@A 5f8d1788  
 0003:0000278c       ?_afxSockState@@3V?$CProcessLocal@V_AFX_SOCK_STATE@@@@A 5f8d178c  
 0003:00002790       ?_afxMailState@@3V?$CProcessLocal@V_AFX_MAIL_STATE@@@@A 5f8d1790  
 0003:00002794       ?_afxEditState@@3V?$CProcessLocal@V_AFX_EDIT_STATE@@@@A 5f8d1794  
 0003:00002798       ?_afxClrState@@3V?$CProcessLocal@V_AFX_COLOR_STATE@@@@A 5f8d1798  
 0003:0000279c       ?_afxChecklistState@@3V?$CProcessLocal@V_AFX_CHECKLIST_STATE@@@@A 5f8d179c  
 0003:000027a0       ??_R0?AVCComboBox@@@8      5f8d17a0  
 0003:00004868       ?_afxSessionMap@@3VCSessionMapPtrToPtr@@A 5f8d3868  
 0003:000048a8       ??_R0?AVCSyncObject@@@8    5f8d38a8  
 0003:000048c8       ??_R0?AVCSessionMapPtrToPtr@@@8 5f8d38c8  
 0003:000048f0       ??_R0?AVCCriticalSection@@@8 5f8d38f0  
 0003:00004910       ?_simpleMemoryException@@3VCMemoryException@@A 5f8d3910  
 0003:00004a28       ??_R0?AVCSimpleException@@@8 5f8d3a28  
 0003:00004a48       ??_R0?AVCMemoryException@@@8 5f8d3a48  
 0003:00004a68       ?_simpleNotSupportedException@@3VCNotSupportedException@@A 5f8d3a68  
 0003:00004b80       ??_R0?AVCNotSupportedException@@@8 5f8d3b80  
 0003:00004ba8       ?_simpleResourceException@@3VCResourceException@@A 5f8d3ba8  
 0003:00004cc0       ??_R0?AVCResourceException@@@8 5f8d3cc0  
 0003:00004ce8       ?_simpleUserException@@3VCUserException@@A 5f8d3ce8  
 0003:00004e00       ??_R0?AVCUserException@@@8 5f8d3e00  
 0003:00004e20       ?factory@CColorPropPage@@1VCColorPropPageFactory@1@A 5f8d3e20  
 0003:00004e70       ??_R0?AVCOleObjectFactory@@@8 5f8d3e70  
 0003:00004e90       ?factory@CFontPropPage@@1VCFontPropPageFactory@1@A 5f8d3e90  
 0003:00004ee0       ?factory@CPicturePropPage@@1VCPicturePropPageFactory@1@A 5f8d3ee0  
 0003:00004f30       ?_afxOleWinApp@@3VCWinApp@@A 5f8d3f30  
 0003:00004ff8       ??_R0?AVCWinApp@@@8        5f8d3ff8  
 0003:00005010       ??_R0?AVCDynLinkLibrary@@@8 5f8d4010  
 0003:00005030       ??_R0?AV_AFX_CTL3D_STATE@@@8 5f8d4030  
 0003:00005050       ?pStaticDocManager@CDocManager@@2PAV1@A 5f8d4050  
 0003:00005058       ??_R0?AVCOleMessageFilter@@@8 5f8d4058  
 0003:00005078       ?pStaticList@CDocManager@@2PAVCPtrList@@A 5f8d4078  
 0003:0000507c       ?_afxRichEditState@@3V?$CProcessLocal@V_AFX_RICHEDIT_STATE@@@@A 5f8d407c  
 0003:00005080       ??_R0?AV_AFX_WIN_STATE@@@8 5f8d4080  
 0003:000050a0       __hmod__ADVAPI32           5f8d40a0  
 0003:000050a8       ??_R0?AVCCommandLineInfo@@@8 5f8d40a8  
 0003:000050c8       ??_R0?AVCPtrArray@@@8      5f8d40c8  
 0003:000050e0       ??_R0?AVCDocTemplate@@@8   5f8d40e0  
 0003:00005100       ??_R0?AVCRecentFileList@@@8 5f8d4100  
 0003:00005120       ??_R0?AVCDocManager@@@8    5f8d4120  
 0003:00005140       ??_R0?AVCFrameWnd@@@8      5f8d4140  
 0003:00005158       ??_R0?AVCControlBar@@@8    5f8d4158  
 0003:00005178       ??_R0?AVCStatusBar@@@8     5f8d4178  
 0003:00005198       ??_R0?AVCToolBar@@@8       5f8d4198  
 0003:000051b0       ??_R0?AVCDockBar@@@8       5f8d41b0  
 0003:000051c8       ??_R0?AVCDockContext@@@8   5f8d41c8  
 0003:000051e8       ??_R0?AVCDocument@@@8      5f8d41e8  
 0003:00005200       ??_R0?AVCOleDocument@@@8   5f8d4200  
 0003:00005220       ??_R0?AVCOleLinkingDoc@@@8 5f8d4220  
 0003:00005240       ??_R0?AVCOleServerDoc@@@8  5f8d4240  
 0003:00005260       ??_R0?AVCObList@@@8        5f8d4260  
 0003:00005278       ??_R0?AVCView@@@8          5f8d4278  
 0003:00005290       ??_R0?AVCDockState@@@8     5f8d4290  
 0003:000052b0       ??_R0?AVCSingleDocTemplate@@@8 5f8d42b0  
 0003:000052d8       ??_R0?AVCMemFile@@@8       5f8d42d8  
 0003:000052f0       ??_R0?AVCDWordArray@@@8    5f8d42f0  
 0003:00005310       ??_R0?AV_AFX_EDIT_STATE@@@8 5f8d4310  
 0003:00005330       ??_R0?AV_AFX_RICHEDIT_STATE@@@8 5f8d4330  
 0003:00005358       ?classCByteArray@CByteArray@@2UCRuntimeClass@@A 5f8d4358  
 0003:00005370       ?classCDWordArray@CDWordArray@@2UCRuntimeClass@@A 5f8d4370  
 0003:00005388       ?classCObArray@CObArray@@2UCRuntimeClass@@A 5f8d4388  
 0003:000053a0       ?classCStringArray@CStringArray@@2UCRuntimeClass@@A 5f8d43a0  
 0003:000053b8       ?classCWordArray@CWordArray@@2UCRuntimeClass@@A 5f8d43b8  
 0003:000053d0       ?classCObList@CObList@@2UCRuntimeClass@@A 5f8d43d0  
 0003:000053e8       ?classCStringList@CStringList@@2UCRuntimeClass@@A 5f8d43e8  
 0003:00005400       ?classCMapStringToOb@CMapStringToOb@@2UCRuntimeClass@@A 5f8d4400  
 0003:00005418       ?classCMapStringToString@CMapStringToString@@2UCRuntimeClass@@A 5f8d4418  
 0003:00005430       ?classCMapWordToOb@CMapWordToOb@@2UCRuntimeClass@@A 5f8d4430  
 0003:00005448       ?rectDefault@CFrameWnd@@2VCRect@@B 5f8d4448  
 0003:00005458       ?_afxWinminiTerm@@3HA      5f8d4458  
 0003:00005460       ?classCDockState@CDockState@@2UCRuntimeClass@@A 5f8d4460  
 0003:00005478       ?_afxTrackerTerm@@3DA      5f8d4478  
 0003:00005479       ?_afxWingdixTerm@@3DA      5f8d4479  
 0003:0000547c       ?_afxMsgFindReplace@@3IB   5f8d447c  
 0003:00005480       ?_afxEditviewTerm@@3DA     5f8d4480  
 0003:00005488       ?_oleData@@3UOLE_DATA@@A   5f8d4488  
 0003:000054b8       ?classCDocItem@CDocItem@@2UCRuntimeClass@@A 5f8d44b8  
 0003:000054d0       ?_afxMsgFindReplace2@@3IB  5f8d44d0  
 0003:000054d8       ?classCRichEditCntrItem@CRichEditCntrItem@@2UCRuntimeClass@@A 5f8d44d8  
 0003:000054f0       ??_R0?AVCColorPropPageFactory@CColorPropPage@@@8 5f8d44f0  
 0003:00005528       ??_R0?AUIUnknown@@@8       5f8d4528  
 0003:00005540       ??_R0?AUIClassFactory@@@8  5f8d4540  
 0003:00005560       ??_R0?AUIClassFactory2@@@8 5f8d4560  
 0003:00005580       ??_R0?AVXClassFactory@COleObjectFactory@@@8 5f8d4580  
 0003:000055b0       ??_R0?AVCFontPropPageFactory@CFontPropPage@@@8 5f8d45b0  
 0003:000055e8       ??_R0?AVCPicturePropPageFactory@CPicturePropPage@@@8 5f8d45e8  
 0003:00005620       ??_R0?AV_AFX_BASE_MODULE_STATE@@@8 5f8d4620  
 0003:00005648       ?bStaticInit@CDocManager@@2HA 5f8d4648  
 0003:00005650       ??_R0?AUIMessageFilter@@@8 5f8d4650  
 0003:00005670       ??_R0?AVXMessageFilter@COleMessageFilter@@@8 5f8d4670  
 0003:000056a0       __hmod__COMCTL32           5f8d46a0  
 0003:000056a8       ??_R0?AVCOleTemplateServer@@@8 5f8d46a8  
 0003:000056cc       ?_afxDropDownWidth@@3HA    5f8d46cc  
 0003:000056d0       ??_R0?AVCClientDC@@@8      5f8d46d0  
 0003:000056e8       __hmod__SHELL32            5f8d46e8  
 0003:000056f0       ??_R0?AUIOleWindow@@@8     5f8d46f0  
 0003:00005710       ??_R0?AUIDataObject@@@8    5f8d4710  
 0003:00005730       ??_R0?AUIPersist@@@8       5f8d4730  
 0003:00005748       ??_R0?AUIOleObject@@@8     5f8d4748  
 0003:00005768       ??_R0?AVXOleObject@COleServerDoc@@@8 5f8d4768  
 0003:00005790       ??_R0?AUIPersistStorage@@@8 5f8d4790  
 0003:000057b0       ??_R0?AVXPersistStorage@COleServerDoc@@@8 5f8d47b0  
 0003:000057e0       ??_R0?AUIOleInPlaceActiveObject@@@8 5f8d47e0  
 0003:00005808       ??_R0?AVXOleInPlaceActiveObject@COleServerDoc@@@8 5f8d4808  
 0003:00005840       ??_R0?AUIOleInPlaceObject@@@8 5f8d4840  
 0003:00005860       ??_R0?AVXOleInPlaceObject@COleServerDoc@@@8 5f8d4860  
 0003:00005890       ??_R0?AVXDataObject@COleServerDoc@@@8 5f8d4890  
 0003:000058b8       ??_R0?AUIPersistFile@@@8   5f8d48b8  
 0003:000058d8       ??_R0?AVXPersistFile@COleLinkingDoc@@@8 5f8d48d8  
 0003:00005908       ??_R0?AUIParseDisplayName@@@8 5f8d4908  
 0003:00005928       ??_R0?AUIOleContainer@@@8  5f8d4928  
 0003:00005948       ??_R0?AUIOleItemContainer@@@8 5f8d4948  
 0003:00005968       ??_R0?AVXOleItemContainer@COleLinkingDoc@@@8 5f8d4968  
 0003:00005998       ??_R0?AVCWindowDC@@@8      5f8d4998  
 0003:000059b0       ??_R0?AVCRichEditDoc@@@8   5f8d49b0  
 0003:000059d0       ??_R0?AVCCtrlView@@@8      5f8d49d0  
 0003:000059e8       ??_R0?AVCRichEditView@@@8  5f8d49e8  
 0003:00005a08       ??_R0?AUIRichEditOleCallback@@@8 5f8d4a08  
 0003:00005a30       ??_R0?AVXRichEditOleCallback@CRichEditView@@@8 5f8d4a30  
 0003:00005a64       ?lMaxSize@CRichEditView@@2KA 5f8d4a64  
 0003:00005a68       ??_R0?AVCMultiDocTemplate@@@8 5f8d4a68  
 0003:00005a88       ??_R0?AVCScrollView@@@8    5f8d4a88  
 0003:00005aa8       ??_R0?AVCOleDropTarget@@@8 5f8d4aa8  
 0003:00005ac8       ??_R0?AVCMDIFrameWnd@@@8   5f8d4ac8  
 0003:00005ae8       ??_R0?AVCMDIChildWnd@@@8   5f8d4ae8  
 0003:00005b08       ??_R0?AUIDropTarget@@@8    5f8d4b08  
 0003:00005b28       ??_R0?AVXDropTarget@COleDropTarget@@@8 5f8d4b28  
 0003:00005b58       ?nScrollInterval@COleDropTarget@@1IA 5f8d4b58  
 0003:00005b5c       ?nScrollDelay@COleDropTarget@@1IA 5f8d4b5c  
 0003:00005b60       ?nScrollInset@COleDropTarget@@1HA 5f8d4b60  
 0003:00005b68       ??_R0?AUIDispatch@@@8      5f8d4b68  
 0003:00005b80       ??_R0?AVCOleDispatchImpl@@@8 5f8d4b80  
 0003:00005ba0       __hmod__OLEAUT32           5f8d4ba0  
 0003:00005ba8       ??_R0?AVCEdit@@@8          5f8d4ba8  
 0003:00005bc0       ??_R0?AVCStatic@@@8        5f8d4bc0  
 0003:00005bd8       ??_R0PAVCException@@@8     5f8d4bd8  
 0003:00005bf8       ??_R0PAX@8                 5f8d4bf8  
 0003:00005c08       ??_R0PAVCObject@@@8        5f8d4c08  
 0003:00005c20       ??_R0PAVCSimpleException@@@8 5f8d4c20  
 0003:00005c40       ??_R0PAVCMemoryException@@@8 5f8d4c40  
 0003:00005c60       ??_R0PAVCNotSupportedException@@@8 5f8d4c60  
 0003:00005c88       ??_R0PAVCArchiveException@@@8 5f8d4c88  
 0003:00005ca8       ??_R0?AVCArchiveException@@@8 5f8d4ca8  
 0003:00005cc8       ??_R0?AUISequentialStream@@@8 5f8d4cc8  
 0003:00005ce8       ??_R0?AUIStream@@@8        5f8d4ce8  
 0003:00005d00       ??_R0?AVCArchiveStream@@@8 5f8d4d00  
 0003:00005d20       ??_R0?AVCStdioFile@@@8     5f8d4d20  
 0003:00005d40       ??_R0?AVCSharedFile@@@8    5f8d4d40  
 0003:00005d60       ??_R0PAVCFileException@@@8 5f8d4d60  
 0003:00005d80       ??_R0?AVCByteArray@@@8     5f8d4d80  
 0003:00005da0       ??_R0?AVCObArray@@@8       5f8d4da0  
 0003:00005db8       ??_R0?AVCStringArray@@@8   5f8d4db8  
 0003:00005dd8       ??_R0?AVCUIntArray@@@8     5f8d4dd8  
 0003:00005df8       ??_R0?AVCWordArray@@@8     5f8d4df8  
 0003:00005e18       ??_R0?AVCStringList@@@8    5f8d4e18  
 0003:00005e38       ??_R0?AVCMapPtrToWord@@@8  5f8d4e38  
 0003:00005e58       ??_R0?AVCMapStringToOb@@@8 5f8d4e58  
 0003:00005e78       ??_R0?AVCMapStringToString@@@8 5f8d4e78  
 0003:00005ea0       ??_R0?AVCMapWordToOb@@@8   5f8d4ea0  
 0003:00005ec0       ??_R0?AVCMapWordToPtr@@@8  5f8d4ec0  
 0003:00005ee0       ??_R0?AVCSemaphore@@@8     5f8d4ee0  
 0003:00005f00       ??_R0?AVCMutex@@@8         5f8d4f00  
 0003:00005f18       ??_R0?AVCEvent@@@8         5f8d4f18  
 0003:00005f30       ??_R0PAVCUserException@@@8 5f8d4f30  
 0003:00005f50       ??_R0?AVCToolTipCtrl@@@8   5f8d4f50  
 0003:00005f70       ??_R0?AVCMiniFrameWnd@@@8  5f8d4f70  
 0003:00005f90       ??_R0?AVCBrush@@@8         5f8d4f90  
 0003:00005fa8       ??_R0?AVCDialogBar@@@8     5f8d4fa8  
 0003:00005fc8       ??_R0?AVCMiniDockFrameWnd@@@8 5f8d4fc8  
 0003:00005fe8       ??_R0?AVCPreviewDC@@@8     5f8d4fe8  
 0003:00006008       ??_R0?AVCMetaFileDC@@@8    5f8d5008  
 0003:00006028       ??_R0?AVCRectTracker@@@8   5f8d5028  
 0003:00006048       ??_R0?AVCReBar@@@8         5f8d5048  
 0003:00006060       ??_R0?AVCListBox@@@8       5f8d5060  
 0003:00006078       ??_R0?AVCScrollBar@@@8     5f8d5078  
 0003:00006098       ??_R0?AVCDragListBox@@@8   5f8d5098  
 0003:000060b8       ??_R0?AVCRgn@@@8           5f8d50b8  
 0003:000060d0       ??_R0?AVCToolBarCtrl@@@8   5f8d50d0  
 0003:000060f0       ??_R0?AVCStatusBarCtrl@@@8 5f8d50f0  
 0003:00006110       ??_R0?AVCListCtrl@@@8      5f8d5110  
 0003:00006128       ??_R0?AVCTreeCtrl@@@8      5f8d5128  
 0003:00006140       ??_R0?AVCSpinButtonCtrl@@@8 5f8d5140  
 0003:00006160       ??_R0?AVCSliderCtrl@@@8    5f8d5160  
 0003:00006180       ??_R0?AVCProgressCtrl@@@8  5f8d5180  
 0003:000061a0       ??_R0?AVCHeaderCtrl@@@8    5f8d51a0  
 0003:000061c0       ??_R0?AVCHotKeyCtrl@@@8    5f8d51c0  
 0003:000061e0       ??_R0?AVCTabCtrl@@@8       5f8d51e0  
 0003:000061f8       ??_R0?AVCAnimateCtrl@@@8   5f8d51f8  
 0003:00006218       ??_R0?AVCRichEditCtrl@@@8  5f8d5218  
 0003:00006238       ??_R0?AVCImageList@@@8     5f8d5238  
 0003:00006258       ??_R0?AVCTempImageList@@@8 5f8d5258  
 0003:00006278       ??_R0?AVCBitmap@@@8        5f8d5278  
 0003:00006290       ??_R0?AV_AFX_CHECKLIST_STATE@@@8 5f8d5290  
 0003:000062b4       ?_afxPropSheetButtons@@3PAHA 5f8d52b4  
 0003:000062c8       ??_R0?AVCPropertyPage@@@8  5f8d52c8  
 0003:000062e8       ??_R0?AVCPropertySheet@@@8 5f8d52e8  
 0003:00006308       ??_R0?AVCPropertyPageEx@@@8 5f8d5308  
 0003:00006328       ??_R0?AVCPropertySheetEx@@@8 5f8d5328  
 0003:00006348       ??_R0?AVCFileDialog@@@8    5f8d5348  
 0003:00006368       ??_R0?AVCPageSetupDialog@@@8 5f8d5368  
 0003:00006388       ??_R0?AV_AFX_COLOR_STATE@@@8 5f8d5388  
 0003:000063a8       ??_R0?AVCColorDialog@@@8   5f8d53a8  
 0003:000063c8       ??_R0?AVCFontDialog@@@8    5f8d53c8  
 0003:000063e8       ??_R0?AVCFindReplaceDialog@@@8 5f8d53e8  
 0003:00006410       ??_R0?AU_AFX_PROPPAGEFONTINFO@@@8 5f8d5410  
 0003:00006438       ??_R0?AVCIPAddressCtrl@@@8 5f8d5438  
 0003:00006458       ??_R0?AVCComboBoxEx@@@8    5f8d5458  
 0003:00006478       ??_R0?AVCPen@@@8           5f8d5478  
 0003:00006490       ??_R0PAVCResourceException@@@8 5f8d5490  
 0003:000064b4       ?_dispatchEntryCount@CCmdTarget@@0IA 5f8d54b4  
 0003:000064b8       ?_dwStockPropMask@CCmdTarget@@0KA 5f8d54b8  
 0003:000064bc       ?_eventsinkEntryCount@CCmdTarget@@0IA 5f8d54bc  
 0003:000064c0       ??_R0?AVCMirrorFile@@@8    5f8d54c0  
 0003:000064e0       ??_R0?AVCNewTypeDlg@@@8    5f8d54e0  
 0003:00006500       ??_R0?AVCSplitterWnd@@@8   5f8d5500  
 0003:00006520       ??_R0?AVCFormView@@@8      5f8d5520  
 0003:00006538       ??_R0?AVCEditView@@@8      5f8d5538  
 0003:00006550       ??_R0?AVCPreviewView@@@8   5f8d5550  
 0003:00006570       ??_R0?AVCListView@@@8      5f8d5570  
 0003:00006588       ??_R0?AVCTreeView@@@8      5f8d5588  
 0003:000065a0       ??_R0?AV_AFX_MAIL_STATE@@@8 5f8d55a0  
 0003:000065c0       ??_R0?AVCInternetSession@@@8 5f8d55c0  
 0003:000065e0       ??_R0?AVCInternetFile@@@8  5f8d55e0  
 0003:00006600       ??_R0?AVCInternetConnection@@@8 5f8d5600  
 0003:00006628       ??_R0?AVCFtpConnection@@@8 5f8d5628  
 0003:00006648       ??_R0?AVCGopherConnection@@@8 5f8d5648  
 0003:00006668       ??_R0?AVCHttpConnection@@@8 5f8d5668  
 0003:00006688       ??_R0?AVCHttpFile@@@8      5f8d5688  
 0003:000066a0       ??_R0?AVCGopherFile@@@8    5f8d56a0  
 0003:000066c0       ??_R0?AVCFileFind@@@8      5f8d56c0  
 0003:000066d8       ??_R0?AVCFtpFileFind@@@8   5f8d56d8  
 0003:000066f8       ??_R0?AVCGopherFileFind@@@8 5f8d56f8  
 0003:00006718       ??_R0?AVCGopherLocator@@@8 5f8d5718  
 0003:00006738       ??_R0PAVCInternetException@@@8 5f8d5738  
 0003:00006760       ??_R0?AVCInternetException@@@8 5f8d5760  
 0003:00006788       ??_R0?AV_AFX_SOCK_STATE@@@8 5f8d5788  
 0003:000067a8       ??_R0?AVCAsyncSocket@@@8   5f8d57a8  
 0003:000067c8       ??_R0?AVCSocket@@@8        5f8d57c8  
 0003:000067e0       ??_R0?AVCSocketFile@@@8    5f8d57e0  
 0003:00006800       ??_R0?AVCSocketWnd@@@8     5f8d5800  
 0003:00006820       ??_R0?AUIOleInPlaceSite@@@8 5f8d5820  
 0003:00006840       ??_R0?AVXOleIPSite@COleClientItem@@@8 5f8d5840  
 0003:00006868       ??_R0?AUIAdviseSink@@@8    5f8d5868  
 0003:00006888       ??_R0?AVXAdviseSink@COleClientItem@@@8 5f8d5888  
 0003:000068b8       ??_R0?AUIOleClientSite@@@8 5f8d58b8  
 0003:000068d8       ??_R0?AVXOleClientSite@COleClientItem@@@8 5f8d58d8  
 0003:00006908       ??_R0?AVCDocItem@@@8       5f8d5908  
 0003:00006920       ??_R0?AVCOleClientItem@@@8 5f8d5920  
 0003:00006940       ??_R0?AVCOleFrameHook@@@8  5f8d5940  
 0003:00006960       ??_R0?AUIOleCommandTarget@@@8 5f8d5960  
 0003:00006980       ??_R0?AVXOleCommandTarget@COleFrameHook@@@8 5f8d5980  
 0003:000069b0       ??_R0?AUIOleInPlaceUIWindow@@@8 5f8d59b0  
 0003:000069d8       ??_R0?AUIOleInPlaceFrame@@@8 5f8d59d8  
 0003:000069f8       ??_R0?AVXOleInPlaceFrame@COleFrameHook@@@8 5f8d59f8  
 0003:00006a28       ??_R0?AVXDataObject@COleDataSource@@@8 5f8d5a28  
 0003:00006a58       ??_R0?AVCOleDataSource@@@8 5f8d5a58  
 0003:00006a78       ??_R0?AVCEnumArray@@@8     5f8d5a78  
 0003:00006a98       ??_R0?AVCEnumFormatEtc@@@8 5f8d5a98  
 0003:00006ab8       ??_R0PAVCOleException@@@8  5f8d5ab8  
 0003:00006ad8       ??_R0?AVCOleDispatchException@@@8 5f8d5ad8  
 0003:00006b00       ??_R0PAVCOleDispatchException@@@8 5f8d5b00  
 0003:00006b28       ??_R0?AUIOleUILinkContainerW@@@8 5f8d5b28  
 0003:00006b50       ??_R0?AUIOleUILinkInfoW@@@8 5f8d5b50  
 0003:00006b70       ??_R0?AVCOleUILinkInfo@@@8 5f8d5b70  
 0003:00006b90       ??_R0?AVCOleDialog@@@8     5f8d5b90  
 0003:00006bb0       ??_R0?AVCOleInsertDialog@@@8 5f8d5bb0  
 0003:00006bd0       ??_R0?AVCOleConvertDialog@@@8 5f8d5bd0  
 0003:00006bf0       ??_R0?AVCOleChangeIconDialog@@@8 5f8d5bf0  
 0003:00006c18       ??_R0?AVCOleLinksDialog@@@8 5f8d5c18  
 0003:00006c38       ??_R0?AVCOleUpdateDialog@@@8 5f8d5c38  
 0003:00006c58       ??_R0?AVCOlePasteSpecialDialog@@@8 5f8d5c58  
 0003:00006c80       ??_R0?AVCOleBusyDialog@@@8 5f8d5c80  
 0003:00006ca0       ??_R0?AVCOlePropertiesDialog@@@8 5f8d5ca0  
 0003:00006cc8       ??_R0?AUIOleUIObjInfoW@@@8 5f8d5cc8  
 0003:00006ce8       ??_R0?AVXOleUIObjInfo@COlePropertiesDialog@@@8 5f8d5ce8  
 0003:00006d20       ??_R0?AVCOleChangeSourceDialog@@@8 5f8d5d20  
 0003:00006d48       ?_afxMonthDays@@3PAHA      5f8d5d48  
 0003:00006d80       ??_R0?AVCOleDropSource@@@8 5f8d5d80  
 0003:00006da0       ??_R0?AUIDropSource@@@8    5f8d5da0  
 0003:00006dc0       ??_R0?AVXDropSource@COleDropSource@@@8 5f8d5dc0  
 0003:00006df0       ??_R0?AUIEnumVOID@@@8      5f8d5df0  
 0003:00006e08       ??_R0?AVXEnumVOID@CEnumArray@@@8 5f8d5e08  
 0003:00006e30       ??_R0?AVCOleCntrFrameWnd@@@8 5f8d5e30  
 0003:00006e50       ??_R0?AVCOleIPFrameWnd@@@8 5f8d5e50  
 0003:00006e70       ??_R0?AVCOleException@@@8  5f8d5e70  
 0003:00006e90       ??_R0?AVCOleStreamFile@@@8 5f8d5e90  
 0003:00006eb0       ??_R0?AVXDataObject@COleServerItem@@@8 5f8d5eb0  
 0003:00006ee0       ??_R0?AVXOleObject@COleServerItem@@@8 5f8d5ee0  
 0003:00006f08       ??_R0?AVCItemDataSource@COleServerItem@@@8 5f8d5f08  
 0003:00006f38       ??_R0?AVCOleServerItem@@@8 5f8d5f38  
 0003:00006f58       ??_R0?AVCInnerUnknown@@@8  5f8d5f58  
 0003:00006f78       ??_R0?AVCEnumOleVerb@@@8   5f8d5f78  
 0003:00006f98       ??_R0?AVCRichEditCntrItem@@@8 5f8d5f98  
 0003:00006fb8       ??_R0?AVCTypeLibCacheMap@@@8 5f8d5fb8  
 0003:00006fd8       ??_R0?AVCMonikerFile@@@8   5f8d5fd8  
 0003:00006ff8       ??_R0?AUIBindHost@@@8      5f8d5ff8  
 0003:00007010       ??_R0?AV_AfxBindHost@@@8   5f8d6010  
 0003:00007030       ??_R0?AVCDateTimeCtrl@@@8  5f8d6030  
 0003:00007050       ??_R0?AVCMonthCalCtrl@@@8  5f8d6050  
 0003:0000706c       ?_eventsinkEntryCount@CHtmlView@@0IA 5f8d606c  
 0003:00007078       ??_R0?AVCHtmlView@@@8      5f8d6078  
 0003:00007090       ??_R0?AVCOccManager@@@8    5f8d6090  
 0003:000070ac       ?_dwStockPropMask@COleControlContainer@@0KA 5f8d60ac  
 0003:000070b0       ?_dispatchEntryCount@COleControlContainer@@0IA 5f8d60b0  
 0003:000070b8       ??_R0?AVXOleIPFrame@COleControlContainer@@@8 5f8d60b8  
 0003:000070e8       ??_R0?AVXOleContainer@COleControlContainer@@@8 5f8d60e8  
 0003:00007120       ??_R0?AVCOleControlContainer@@@8 5f8d6120  
 0003:00007148       ??_R0?AVCFont@@@8          5f8d6148  
 0003:00007160       ??_R0?AVCEnumUnknown@@@8   5f8d6160  
 0003:00007180       ??_R0?AVXEventSink@COleControlSite@@@8 5f8d6180  
 0003:000071b0       ??_R0?AUIPropertyNotifySink@@@8 5f8d61b0  
 0003:000071d8       ??_R0?AVXPropertyNotifySink@COleControlSite@@@8 5f8d61d8  
 0003:00007210       ??_R0?AVXAmbientProps@COleControlSite@@@8 5f8d6210  
 0003:00007240       ??_R0?AUIOleControlSite@@@8 5f8d6240  
 0003:00007260       ??_R0?AVXOleControlSite@COleControlSite@@@8 5f8d6260  
 0003:00007290       ??_R0?AVXOleIPSite@COleControlSite@@@8 5f8d6290  
 0003:000072c0       ??_R0?AVXOleClientSite@COleControlSite@@@8 5f8d62c0  
 0003:000072f0       ??_R0?AVCOleControlSite@@@8 5f8d62f0  
 0003:00007310       ??_R0?AUIRowsetNotify@@@8  5f8d6310  
 0003:00007330       ??_R0?AVXRowsetNotify@COleControlSite@@@8 5f8d6330  
 0003:00007360       ??_R0?AUINotifyDBEvents@@@8 5f8d6360  
 0003:00007380       ??_R0?AVXNotifyDBEvents@COleControlSite@@@8 5f8d6380  
 0003:000073b0       ??_R0?AUIBoundObjectSite@@@8 5f8d63b0  
 0003:000073d0       ??_R0?AVXBoundObjectSite@COleControlSite@@@8 5f8d63d0  
 0003:00007400       ??_R0?AVCDataSourceControl@@@8 5f8d6400  
 0003:00007428       __GUID_0c733a05_2a1c_11ce_ade5_00aa0044773d 5f8d6428  
 0003:00007438       __GUID_0c733a11_2a1c_11ce_ade5_00aa0044773d 5f8d6438  
 0003:00007448       __GUID_0c733a8c_2a1c_11ce_ade5_00aa0044773d 5f8d6448  
 0003:00007458       ??_R0?AVCOleControlLock@@@8 5f8d6458  
 0003:00007478       ??_R0?AVXOleObject@CDocObjectServer@@@8 5f8d6478  
 0003:000074a8       ??_R0?AUIPrint@@@8         5f8d64a8  
 0003:000074c0       ??_R0?AVXPrint@CDocObjectServer@@@8 5f8d64c0  
 0003:000074e8       ??_R0?AVXOleCommandTarget@CDocObjectServer@@@8 5f8d64e8  
 0003:00007520       ??_R0?AUIOleDocumentView@@@8 5f8d6520  
 0003:00007540       ??_R0?AVXOleDocumentView@CDocObjectServer@@@8 5f8d6540  
 0003:00007570       ??_R0?AUIOleDocument@@@8   5f8d6570  
 0003:00007590       ??_R0?AVXOleDocument@CDocObjectServer@@@8 5f8d6590  
 0003:000075c0       ??_R0?AVCDocObjectServer@@@8 5f8d65c0  
 0003:000075e0       ??_R0?AVCDocObjectServerItem@@@8 5f8d65e0  
 0003:00007608       ??_R0?AVCOleCmdUI@@@8      5f8d6608  
 0003:00007620       ??_R0?AVCOleDocIPFrameWnd@@@8 5f8d6620  
 0003:00007640       ??_R0?AUIOleDocumentSite@@@8 5f8d6640  
 0003:00007660       ??_R0?AVXOleDocumentSite@COleDocObjectItem@@@8 5f8d6660  
 0003:00007698       ??_R0?AVCOleDocObjectItem@@@8 5f8d6698  
 0003:000076b8       ??_R0?AVCAsyncMonikerFile@@@8 5f8d66b8  
 0003:000076d8       ??_R0?AUIBindStatusCallback@@@8 5f8d66d8  
 0003:00007700       ??_R0?AV_AfxBindStatusCallback@@@8 5f8d6700  
 0003:00007728       ??_R0?AVCInnerUnknown@_AfxBindStatusCallback@@@8 5f8d6728  
 0003:00007760       ??_R0?AVCOleResizeBar@@@8  5f8d6760  
 0003:00007780       ??_R0?AVXOleInPlaceActiveObject@COleControl@@@8 5f8d6780  
 0003:000077b8       ??_R0?AUIOleInPlaceObjectWindowless@@@8 5f8d67b8  
 0003:000077e8       ??_R0?AVXOleInPlaceObject@COleControl@@@8 5f8d67e8  
 0003:00007818       ??_R0?AVXDataObject@COleControl@@@8 5f8d6818  
 0003:00007840       ??_R0?AVCOleControl@@@8    5f8d6840  
 0003:00007860       ??_R0?AUIViewObject@@@8    5f8d6860  
 0003:00007880       ??_R0?AUIViewObject2@@@8   5f8d6880  
 0003:000078a0       ??_R0?AUIViewObjectEx@@@8  5f8d68a0  
 0003:000078c0       ??_R0?AVXViewObject@COleControl@@@8 5f8d68c0  
 0003:000078e8       ??_R0?AUIQuickActivate@@@8 5f8d68e8  
 0003:00007908       ??_R0?AVXQuickActivate@COleControl@@@8 5f8d6908  
 0003:00007938       ??_R0?AVXOleObject@COleControl@@@8 5f8d6938  
 0003:00007960       ??_R0?AVXFontNotification@COleControl@@@8 5f8d6960  
 0003:00007990       ??_R0?AUIPersistPropertyBag@@@8 5f8d6990  
 0003:000079b8       ??_R0?AVXPersistPropertyBag@COleControl@@@8 5f8d69b8  
 0003:000079e8       ??_R0?AUIPerPropertyBrowsing@@@8 5f8d69e8  
 0003:00007a10       ??_R0?AVXPerPropertyBrowsing@COleControl@@@8 5f8d6a10  
 0003:00007a40       ??_R0?AUIPersistMemory@@@8 5f8d6a40  
 0003:00007a60       ??_R0?AVXPersistMemory@COleControl@@@8 5f8d6a60  
 0003:00007a90       ??_R0?AUISpecifyPropertyPages@@@8 5f8d6a90  
 0003:00007ab8       ??_R0?AVXSpecifyPropertyPages@COleControl@@@8 5f8d6ab8  
 0003:00007ae8       ??_R0?AVXPropConnPt@COleControl@@@8 5f8d6ae8  
 0003:00007b10       ??_R0?AUIProvideClassInfo@@@8 5f8d6b10  
 0003:00007b30       ??_R0?AUIProvideClassInfo2@@@8 5f8d6b30  
 0003:00007b58       ??_R0?AVXProvideClassInfo@COleControl@@@8 5f8d6b58  
 0003:00007b88       ??_R0?AUIPersistStreamInit@@@8 5f8d6b88  
 0003:00007bb0       ??_R0?AVXPersistStreamInit@COleControl@@@8 5f8d6bb0  
 0003:00007be0       ??_R0?AVCConnectionPoint@@@8 5f8d6be0  
 0003:00007c00       ??_R0?AVXEventConnPt@COleControl@@@8 5f8d6c00  
 0003:00007c28       ??_R0?AUIOleControl@@@8    5f8d6c28  
 0003:00007c48       ??_R0?AVXOleControl@COleControl@@@8 5f8d6c48  
 0003:00007c70       ??_R0?AVXPersistStorage@COleControl@@@8 5f8d6c70  
 0003:00007ca0       ??_R0?AUIPointerInactive@@@8 5f8d6ca0  
 0003:00007cc0       ??_R0?AVXPointerInactive@COleControl@@@8 5f8d6cc0  
 0003:00007cf0       ??_R0?AUIOleCache@@@8      5f8d6cf0  
 0003:00007d08       ??_R0?AVXOleCache@COleControl@@@8 5f8d6d08  
 0003:00007d30       ??_R0?AVCReflectorWnd@@@8  5f8d6d30  
 0003:00007d50       ??_R0?AVCParkingWnd@@@8    5f8d6d50  
 0003:00007d70       ??_R0?AVCControlDataSource@COleControl@@@8 5f8d6d70  
 0003:00007da0       ??_R0?AVCControlFrameWnd@@@8 5f8d6da0  
 0003:00007dc0       ??_R0?AUIConnectionPoint@@@8 5f8d6dc0  
 0003:00007de0       ??_R0?AVXConnPt@CConnectionPoint@@@8 5f8d6de0  
 0003:00007e08       ??_R0?AVCEnumConnections@@@8 5f8d6e08  
 0003:00007e28       ??_R0?AVCEnumConnPoints@@@8 5f8d6e28  
 0003:00007e48       ??_R0?AUIConnectionPointContainer@@@8 5f8d6e48  
 0003:00007e70       ??_R0?AVCOleConnPtContainer@@@8 5f8d6e70  
 0003:00007e98       ??_R0?AVCPropExchange@@@8  5f8d6e98  
 0003:00007eb8       ??_R0?AVCArchivePropExchange@@@8 5f8d6eb8  
 0003:00007ee0       ??_R0?AVCResetPropExchange@@@8 5f8d6ee0  
 0003:00007f08       ??_R0?AVCAsyncPropExchange@@@8 5f8d6f08  
 0003:00007f30       ??_R0?AUAFX_DDPDATA@@@8    5f8d6f30  
 0003:00007f50       ??_R0?AVCOlePropertyPage@@@8 5f8d6f50  
 0003:00007f70       ??_R0?AVXPropNotifySink@COlePropertyPage@@@8 5f8d6f70  
 0003:00007fa0       ??_R0?AUIPropertyPage@@@8  5f8d6fa0  
 0003:00007fc0       ??_R0?AUIPropertyPage2@@@8 5f8d6fc0  
 0003:00007fe0       ??_R0?AVXPropertyPage@COlePropertyPage@@@8 5f8d6fe0  
 0003:00008010       ??_R0?AVCPropsetPropExchange@@@8 5f8d7010  
 0003:00008060       ??_R0?AVCControlRectTracker@@@8 5f8d7060  
 0003:00008088       ??_R0?AUIPersistStream@@@8 5f8d7088  
 0003:000080a8       ??_R0?AVCBlobProperty@@@8  5f8d70a8  
 0003:000080c8       ??_R0?AVCPropbagPropExchange@@@8 5f8d70c8  
 0003:000080f0       ??_R0?AV_AFXCTL_AMBIENT_CACHE@@@8 5f8d70f0  
 0003:00008118       ??_R0?AVCWindowlessDC@@@8  5f8d7118  
 0003:00008138       ??_R0?AVCColorButton@@@8   5f8d7138  
 0003:00008158       ??_R0?AVCStockPropPage@@@8 5f8d7158  
 0003:00008178       ??_R0?AVCColorPropPage@@@8 5f8d7178  
 0003:00008198       ?_afxTTDefaults@@3PAHA     5f8d7198  
 0003:000081d8       ??_R0?AVCFontPropPage@@@8  5f8d71d8  
 0003:000081f8       ??_R0?AVCSizeComboBox@@@8  5f8d71f8  
 0003:00008218       ??_R0?AVCFontComboBox@@@8  5f8d7218  
 0003:00008238       ?_afxPictDescEmpty@@3UtagPICTDESC@@A 5f8d7238  
 0003:00008250       ??_R0?AVCPicturePropPage@@@8 5f8d7250  
 0003:00008270       ??_R0PAVCDBException@@@8   5f8d7270  
 0003:00008290       ??_R0?AVCDBException@@@8   5f8d7290  
 0003:000082b0       ??_R0?AVCDatabase@@@8      5f8d72b0  
 0003:000082c8       ??_R0?AVCRecordset@@@8     5f8d72c8  
 0003:000082e8       ??_R0?AV_AFX_DB_STATE@@@8  5f8d72e8  
 0003:00008308       ??_R0?AVCRecordView@@@8    5f8d7308  
 0003:00008328       ??_R0?AVCLongBinary@@@8    5f8d7328  
 0003:00008348       ??_R0?AVCDBVariant@@@8     5f8d7348  
 0003:00008368       ?_afxNullVariant@@3UtagVARIANT@@A 5f8d7368  
 0003:00008378       ?_afxOptionalVariant@@3UtagVARIANT@@A 5f8d7378  
 0003:00008388       ??_R0?AV_AFX_DAO_STATE@@@8 5f8d7388  
 0003:000083a8       ??_R0?AUCDaoIndexInfo@@@8  5f8d73a8  
 0003:000083c8       ??_R0?AUCDaoRelationInfo@@@8 5f8d73c8  
 0003:000083e8       ??_R0?AVCDaoException@@@8  5f8d73e8  
 0003:00008408       ??_R0PAVCDaoException@@@8  5f8d7408  
 0003:00008428       ??_R0?AVCDaoWorkspace@@@8  5f8d7428  
 0003:00008448       ??_R0?AVCDaoDatabase@@@8   5f8d7448  
 0003:00008468       ??_R0?AVCDaoTableDef@@@8   5f8d7468  
 0003:00008488       ??_R0?AVCDaoQueryDef@@@8   5f8d7488  
 0003:000084a8       ??_R0?AVCDaoRecordset@@@8  5f8d74a8  
 0003:000084c8       ??_R0?AVCDaoRecordView@@@8 5f8d74c8  
 0003:000084e8       ??_R0?AVCPalette@@@8       5f8d74e8  
 0003:00008500       ??_R0?AVCCheckListBox@@@8  5f8d7500  
 0003:00008520       ??_R0?AVCBitmapButton@@@8  5f8d7520  
 0003:00008540       ??_R0?AVCDataPathProperty@@@8 5f8d7540  
 0003:00008560       ??_R0?AVCCachedDataPathProperty@@@8 5f8d7560  
 0003:00008588       ?_afxGotScrollLines@@3HA   5f8d7588  
 0003:00008590       ?_afx_sizeMiniSys@@3UtagSIZE@@A 5f8d7590  
 0003:00008598       ?_afxHandleSize@@3HA       5f8d7598  
 0003:0000859c       ?_afxCursors@@3PAPAUHICON__@@A 5f8d759c  
 0003:000085c8       ?_afxMsgSETRGB@@3IA        5f8d75c8  
 0003:000085cc       ?_afxMsgHELP@@3IA          5f8d75cc  
 0003:000085d0       ?_afxMsgCOLOROK@@3IA       5f8d75d0  
 0003:000085d4       ?_afxMsgFILEOK@@3IA        5f8d75d4  
 0003:000085d8       ?_afxMsgSHAREVI@@3IA       5f8d75d8  
 0003:000085dc       ?_afxMsgLBSELCHANGE@@3IA   5f8d75dc  
 0003:000085e0       ?_afx_idcPrimaryLast@@3IA  5f8d75e0  
 0003:000085e4       ?_afx_hcurDestroy@@3PAUHICON__@@A 5f8d75e4  
 0003:000085e8       ?_afx_hcurLast@@3PAUHICON__@@A 5f8d75e8  
 0003:0000860c       ?nDragDelay@COleDropSource@@1IA 5f8d760c  
 0003:00008610       ?nDragMinDist@COleDropSource@@1IA 5f8d7610  
 0003:00008640       ?_afxLargeZero@@3T_LARGE_INTEGER@@A 5f8d7640  
 0003:00008648       ?hPal@@3PAUHPALETTE__@@A   5f8d7648  
 0003:0000864c       ?idClicked@CColorButton@@2IA 5f8d764c  
 0003:00008650       __hmod__OLEPRO32           5f8d7650  
 0003:00008654       __hmod__WINSPOOL           5f8d7654  
 0003:00008658       __hmod__WININET            5f8d7658  
 0003:0000865c       __hmod__WSOCK32            5f8d765c  
 0003:00008660       __hmod__OLEDLG             5f8d7660  
 0003:00008664       __hmod__URLMON             5f8d7664  
 0003:00008668       __hmod__ODBC32             5f8d7668  
 0003:0000866c       ___puiHead                 5f8d766c  
 0003:00008670       ___pfnDliFailureHook       5f8d7670  

 entry point at        0001:000047e6

 Static symbols

